 variants

 Timestamp is 5dee3649 (Mon Dec 09 18:55:53 2019)

 Preferred load address is 10000000

 Start         Length     Name                   Class
 0001:00000000 00001efbH .text$di                CODE
 0001:00001f00 00017cdeH .text$mn                CODE
 0001:00019be0 000046e4H .text$x                 CODE
 0001:0001e2d0 0000077bH .text$yd                CODE
 0002:00000000 000008ccH .idata$5                DATA
 0002:000008cc 00000004H .CRT$XCA                DATA
 0002:000008d0 000001b8H .CRT$XCU                DATA
 0002:00000a88 00000004H .CRT$XCZ                DATA
 0002:00000a8c 00000004H .CRT$XIA                DATA
 0002:00000a90 00000004H .CRT$XIAA               DATA
 0002:00000a94 00000004H .CRT$XIC                DATA
 0002:00000a98 00000004H .CRT$XIZ                DATA
 0002:00000aa0 00003280H .rdata                  DATA
 0002:00003d20 00000070H .rdata$debug            DATA
 0002:00003d90 00001148H .rdata$r                DATA
 0002:00004ee0 0000027cH .rdata$sxdata           DATA
 0002:0000515c 00000004H .rtc$IAA                DATA
 0002:00005160 00000004H .rtc$IZZ                DATA
 0002:00005164 00000004H .rtc$TAA                DATA
 0002:00005168 00000004H .rtc$TZZ                DATA
 0002:00005170 00004d14H .xdata$x                DATA
 0002:00009e90 00000051H .edata                  DATA
 0002:00009ee4 000000c8H .idata$2                DATA
 0002:00009fac 00000014H .idata$3                DATA
 0002:00009fc0 000008ccH .idata$4                DATA
 0002:0000a88c 000072ccH .idata$6                DATA
 0003:00000000 000000b4H .data                   DATA
 0003:000000b8 00000950H .data$r                 DATA
 0003:00000a08 000005dcH .bss                    DATA
 0004:00000000 00000058H .rsrc$01                DATA
 0004:00000060 00000180H .rsrc$02                DATA

  Address         Publics by Value              Rva+Base       Lib:Object

 0000:00000000       __except_list              00000000     <absolute>
 0000:00000000       ___guard_fids_count        00000000     <absolute>
 0000:00000000       ___guard_flags             00000000     <absolute>
 0000:00000000       ___guard_fids_table        00000000     <absolute>
 0000:0000009f       ___safe_se_handler_count   0000009f     <absolute>
 0000:00009876       __ldused                   00009876     <absolute>
 0000:00009876       __fltused                  00009876     <absolute>
 0000:00000000       ___ImageBase               10000000     <linker-defined>
 0001:00001f00       ??$_Allocate@D@std@@YAPADIPAD@Z 10002f00 f i AssemblySamtoolsMpileup.obj
 0001:00001f30       ??$_Move@AAPAUData@QListData@@@std@@YA$$QAPAUData@QListData@@AAPAU12@@Z 10002f30 f i AssemblySamtoolsMpileup.obj
 0001:00001f40       ??$acquireMemoryFence@H@?$QGenericAtomicOps@U?$QAtomicOpsBySize@$03@@@@SAXABH@Z 10002f40 f i AssemblySamtoolsMpileup.obj
 0001:00001f50       ??$addressof@D@std@@YAPADAAD@Z 10002f50 f i AssemblySamtoolsMpileup.obj
 0001:00001f60       ??$atomic@H@?$QAtomicOpsBySize@$03@@CAPAJPAH@Z 10002f60 f i AssemblySamtoolsMpileup.obj
 0001:00001f70       ??$construct@PADAAPAD@?$_Wrap_alloc@V?$allocator@D@std@@@std@@QAEXPAPADAAPAD@Z 10002f70 f i AssemblySamtoolsMpileup.obj
 0001:00001f90       ??$construct@PADAAPAD@?$allocator@D@std@@QAEXPAPADAAPAD@Z 10002f90 f i AssemblySamtoolsMpileup.obj
 0001:00001fb0       ??$construct@PADAAPAD@?$allocator_traits@V?$allocator@D@std@@@std@@SAXAAV?$allocator@D@1@PAPADAAPAD@Z 10002fb0 f i AssemblySamtoolsMpileup.obj
 0001:00001fd0       ??$deref@H@?$QAtomicOpsBySize@$03@@SA_NAAH@Z 10002fd0 f i AssemblySamtoolsMpileup.obj
 0001:00001ff0       ??$destroy@PAD@?$_Wrap_alloc@V?$allocator@D@std@@@std@@QAEXPAPAD@Z 10002ff0 f i AssemblySamtoolsMpileup.obj
 0001:00002000       ??$destroy@PAD@?$allocator@D@std@@QAEXPAPAD@Z 10003000 f i AssemblySamtoolsMpileup.obj
 0001:00002010       ??$destroy@PAD@?$allocator_traits@V?$allocator@D@std@@@std@@SAXAAV?$allocator@D@1@PAPAD@Z 10003010 f i AssemblySamtoolsMpileup.obj
 0001:00002020       ??$forward@AAPAD@std@@YAAAPADAAPAD@Z 10003020 f i AssemblySamtoolsMpileup.obj
 0001:00002030       ??$load@H@?$QGenericAtomicOps@U?$QAtomicOpsBySize@$03@@@@SAHABH@Z 10003030 f i AssemblySamtoolsMpileup.obj
 0001:00002040       ??$loadAcquire@H@?$QGenericAtomicOps@U?$QAtomicOpsBySize@$03@@@@SAHABH@Z 10003040 f i AssemblySamtoolsMpileup.obj
 0001:00002050       ??$orderedMemoryFence@H@?$QGenericAtomicOps@U?$QAtomicOpsBySize@$03@@@@SAXABH@Z 10003050 f i AssemblySamtoolsMpileup.obj
 0001:00002060       ??$qMapLessThanKey@VQString@@@@YA_NABVQString@@0@Z 10003060 f i AssemblySamtoolsMpileup.obj
 0001:00002070       ??$qMetaTypeId@V?$QSharedDataPointer@VDbiDataHandler@Workflow@U2@@@@@@YAHXZ 10003070 f i AssemblySamtoolsMpileup.obj
 0001:00002080       ??$qMetaTypeId@VU2DbiRef@U2@@@@YAHXZ 10003080 f i AssemblySamtoolsMpileup.obj
 0001:00002090       ??$qRegisterMetaType@V?$QSharedDataPointer@VDbiDataHandler@Workflow@U2@@@@@@YAHPBDPAV?$QSharedDataPointer@VDbiDataHandler@Workflow@U2@@@@W4DefinedType@?$MetaTypeDefinedHelper@V?$QSharedDataPointer@VDbiDataHandler@Workflow@U2@@@@$00@QtPrivate@@@Z 10003090 f i AssemblySamtoolsMpileup.obj
 0001:00002150       ??$qRegisterMetaType@VU2DbiRef@U2@@@@YAHPBDPAVU2DbiRef@U2@@W4DefinedType@?$MetaTypeDefinedHelper@VU2DbiRef@U2@@$00@QtPrivate@@@Z 10003150 f i AssemblySamtoolsMpileup.obj
 0001:00002210       ??$qRegisterNormalizedMetaType@V?$QSharedDataPointer@VDbiDataHandler@Workflow@U2@@@@@@YAHABVQByteArray@@PAV?$QSharedDataPointer@VDbiDataHandler@Workflow@U2@@@@W4DefinedType@?$MetaTypeDefinedHelper@V?$QSharedDataPointer@VDbiDataHandler@Workflow@U2@@@@$00@QtPrivate@@@Z 10003210 f i AssemblySamtoolsMpileup.obj
 0001:00002270       ??$qRegisterNormalizedMetaType@VU2DbiRef@U2@@@@YAHABVQByteArray@@PAVU2DbiRef@U2@@W4DefinedType@?$MetaTypeDefinedHelper@VU2DbiRef@U2@@$00@QtPrivate@@@Z 10003270 f i AssemblySamtoolsMpileup.obj
 0001:000022d0       ??$qSwap@PAUData@QListData@@@@YAXAAPAUData@QListData@@0@Z 100032d0 f i AssemblySamtoolsMpileup.obj
 0001:000022f0       ??$qVariantFromValue@V?$QSharedDataPointer@VDbiDataHandler@Workflow@U2@@@@@@YA?AVQVariant@@ABV?$QSharedDataPointer@VDbiDataHandler@Workflow@U2@@@@@Z 100032f0 f i AssemblySamtoolsMpileup.obj
 0001:00002320       ??$qVariantFromValue@VU2DbiRef@U2@@@@YA?AVQVariant@@ABVU2DbiRef@U2@@@Z 10003320 f i AssemblySamtoolsMpileup.obj
 0001:00002350       ??$ref@H@?$QAtomicOpsBySize@$03@@SA_NAAH@Z 10003350 f i AssemblySamtoolsMpileup.obj
 0001:00002370       ??$releaseMemoryFence@H@?$QGenericAtomicOps@U?$QAtomicOpsBySize@$03@@@@SAXABH@Z 10003370 f i AssemblySamtoolsMpileup.obj
 0001:00002380       ??$storeRelease@HH@?$QGenericAtomicOps@U?$QAtomicOpsBySize@$03@@@@SAXAAHH@Z 10003380 f i AssemblySamtoolsMpileup.obj
 0001:00002390       ??$swap@PAUData@QListData@@@std@@YAXAAPAUData@QListData@@0@Z 10003390 f i AssemblySamtoolsMpileup.obj
 0001:000023b0       ??0?$QFlags@W4OpenModeFlag@QIODevice@@@@QAE@W4OpenModeFlag@QIODevice@@@Z 100033b0 f i AssemblySamtoolsMpileup.obj
 0001:000023c0       ??0?$QFlags@W4TaskFlag@U2@@@@QAE@W4TaskFlag@U2@@@Z 100033c0 f i AssemblySamtoolsMpileup.obj
 0001:000023d0       ??0?$QFlags@W4TypeFlag@QMetaType@@@@QAE@VQFlag@@@Z 100033d0 f i AssemblySamtoolsMpileup.obj
 0001:000023e0       ??0?$QForeachContainer@V?$QList@PAVGObject@U2@@@@@@QAE@ABV?$QList@PAVGObject@U2@@@@@Z 100033e0 f i AssemblySamtoolsMpileup.obj
 0001:00002420       ??0?$QForeachContainer@V?$QList@VQString@@@@@@QAE@ABV?$QList@VQString@@@@@Z 10003420 f i AssemblySamtoolsMpileup.obj
 0001:00002460       ??0?$QList@PAVGObject@U2@@@@QAE@ABV0@@Z 10003460 f i AssemblySamtoolsMpileup.obj
 0001:00002520       ??0?$QList@PAVTask@U2@@@@QAE@$$QAV0@@Z 10003520 f i AssemblySamtoolsMpileup.obj
 0001:00002540       ??0?$QList@PAVTask@U2@@@@QAE@XZ 10003540 f i AssemblySamtoolsMpileup.obj
 0001:00002550       ??0?$QList@V?$QMap@VQString@@VQVariant@@@@@@QAE@XZ 10003550 f i AssemblySamtoolsMpileup.obj
 0001:00002560       ??0?$QList@VQString@@@@QAE@ABV0@@Z 10003560 f i AssemblySamtoolsMpileup.obj
 0001:00002620       ??0?$QList@VQString@@@@QAE@XZ 10003620 f i AssemblySamtoolsMpileup.obj
 0001:00002630       ??0?$QMap@VQString@@VQVariant@@@@QAE@ABV0@@Z 10003630 f i AssemblySamtoolsMpileup.obj
 0001:000026a0       ??0?$QMap@VQString@@VQVariant@@@@QAE@XZ 100036a0 f i AssemblySamtoolsMpileup.obj
 0001:000026b0       ??0?$QScopedPointer@VDocument@U2@@U?$QScopedPointerDeleter@VDocument@U2@@@@@@QAE@PAVDocument@U2@@@Z 100036b0 f i AssemblySamtoolsMpileup.obj
 0001:000026c0       ??0?$QScopedPointer@VQProcess@@U?$QScopedPointerDeleter@VQProcess@@@@@@QAE@PAVQProcess@@@Z 100036c0 f i AssemblySamtoolsMpileup.obj
 0001:000026d0       ??0?$QSharedDataPointer@VDbiDataHandler@Workflow@U2@@@@QAE@ABV0@@Z 100036d0 f i AssemblySamtoolsMpileup.obj
 0001:000026f0       ??0?$QSharedDataPointer@VDbiDataHandler@Workflow@U2@@@@QAE@XZ 100036f0 f i AssemblySamtoolsMpileup.obj
 0001:00002700       ??0?$_String_alloc@$0A@U?$_String_base_types@DV?$allocator@D@std@@@std@@@std@@QAE@ABV?$allocator@D@1@@Z 10003700 f i AssemblySamtoolsMpileup.obj
 0001:00002720       ??0?$_String_val@U?$_Simple_types@D@std@@@std@@QAE@XZ 10003720 f i AssemblySamtoolsMpileup.obj
 0001:00002740       ??0?$_Wrap_alloc@V?$allocator@D@std@@@std@@QAE@XZ 10003740 f i AssemblySamtoolsMpileup.obj
 0001:00002750       ??0?$allocator@D@std@@QAE@XZ 10003750 f i AssemblySamtoolsMpileup.obj
 0001:00002760       ??0?$basic_string@DU?$char_traits@D@std@@V?$allocator@D@2@@std@@QAE@PBD@Z 10003760 f i AssemblySamtoolsMpileup.obj
 0001:000027c0       ??0CallVariantsTask@LocalWorkflow@U2@@QAE@ABVCallVariantsTaskSettings@12@PAVDbiDataStorage@Workflow@2@@Z 100037c0 f   AssemblySamtoolsMpileup.obj
 0001:00002970       ??0CallVariantsTaskSettings@LocalWorkflow@U2@@QAE@ABV012@@Z 10003970 f i AssemblySamtoolsMpileup.obj
 0001:00002b90       ??0QFlag@@QAE@H@Z          10003b90 f i AssemblySamtoolsMpileup.obj
 0001:00002ba0       ??0QLatin1Char@@QAE@D@Z    10003ba0 f i AssemblySamtoolsMpileup.obj
 0001:00002bb0       ??0QStringList@@QAE@ABV0@@Z 10003bb0 f i AssemblySamtoolsMpileup.obj
 0001:00002bd0       ??0QStringList@@QAE@XZ     10003bd0 f i AssemblySamtoolsMpileup.obj
 0001:00002be0       ??0SamtoolsMpileupTask@LocalWorkflow@U2@@QAE@ABVCallVariantsTaskSettings@12@@Z 10003be0 f   AssemblySamtoolsMpileup.obj
 0001:00002ca0       ??0_Generic_error_category@std@@QAE@XZ 10003ca0 f i AssemblySamtoolsMpileup.obj
 0001:00002cb0       ??0_Ignore@std@@QAE@XZ     10003cb0 f i AssemblySamtoolsMpileup.obj
 0001:00002cc0       ??0_Iostream_error_category@std@@QAE@XZ 10003cc0 f i AssemblySamtoolsMpileup.obj
 0001:00002cd0       ??0_System_error_category@std@@QAE@XZ 10003cd0 f i AssemblySamtoolsMpileup.obj
 0001:00002ce0       ??0const_iterator@?$QList@PAVGObject@U2@@@@QAE@PAUNode@1@@Z 10003ce0 f i AssemblySamtoolsMpileup.obj
 0001:00002cf0       ??0const_iterator@?$QList@VQString@@@@QAE@PAUNode@1@@Z 10003cf0 f i AssemblySamtoolsMpileup.obj
 0001:00002d00       ??0error_category@std@@QAE@XZ 10003d00 f i AssemblySamtoolsMpileup.obj
 0001:00002d10       ??0error_condition@std@@QAE@HABVerror_category@1@@Z 10003d10 f i AssemblySamtoolsMpileup.obj
 0001:00002d30       ??0iterator@?$QList@VFormatDetectionResult@U2@@@@QAE@PAUNode@1@@Z 10003d30 f i AssemblySamtoolsMpileup.obj
 0001:00002d40       ??0iterator@?$QMap@VQString@@VQVariant@@@@QAE@PAU?$QMapNode@VQString@@VQVariant@@@@@Z 10003d40 f i AssemblySamtoolsMpileup.obj
 0001:00002d50       ??1?$QForeachContainer@V?$QList@PAVGObject@U2@@@@@@QAE@XZ 10003d50 f i AssemblySamtoolsMpileup.obj
 0001:00002d80       ??1?$QForeachContainer@V?$QList@VQString@@@@@@QAE@XZ 10003d80 f i AssemblySamtoolsMpileup.obj
 0001:00002d90       ??1?$QList@PAVGObject@U2@@@@QAE@XZ 10003d90 f i AssemblySamtoolsMpileup.obj
 0001:00002dc0       ??1?$QList@PAVTask@U2@@@@QAE@XZ 10003dc0 f i AssemblySamtoolsMpileup.obj
 0001:00002df0       ??1?$QList@V?$QMap@VQString@@VQVariant@@@@@@QAE@XZ 10003df0 f i AssemblySamtoolsMpileup.obj
 0001:00002e40       ??1?$QList@VFormatDetectionResult@U2@@@@QAE@XZ 10003e40 f i AssemblySamtoolsMpileup.obj
 0001:00002e70       ??1?$QList@VQString@@@@QAE@XZ 10003e70 f i AssemblySamtoolsMpileup.obj
 0001:00002ed0       ??1?$QMap@VQString@@VQVariant@@@@QAE@XZ 10003ed0 f i AssemblySamtoolsMpileup.obj
 0001:00002f20       ??1?$QScopedPointer@VDocument@U2@@U?$QScopedPointerDeleter@VDocument@U2@@@@@@QAE@XZ 10003f20 f i AssemblySamtoolsMpileup.obj
 0001:00002f30       ??1?$QScopedPointer@VQProcess@@U?$QScopedPointerDeleter@VQProcess@@@@@@QAE@XZ 10003f30 f i AssemblySamtoolsMpileup.obj
 0001:00002f40       ??1?$QSharedDataPointer@VDbiDataHandler@Workflow@U2@@@@QAE@XZ 10003f40 f i AssemblySamtoolsMpileup.obj
 0001:00002f60       ??1?$basic_string@DU?$char_traits@D@std@@V?$allocator@D@2@@std@@QAE@XZ 10003f60 f i AssemblySamtoolsMpileup.obj
 0001:00002f90       ??1CallVariantsTask@LocalWorkflow@U2@@UAE@XZ 10003f90 f i AssemblySamtoolsMpileup.obj
 0001:00003040       ??1CallVariantsTaskSettings@LocalWorkflow@U2@@QAE@XZ 10004040 f i AssemblySamtoolsMpileup.obj
 0001:00003100       ??1QStringList@@QAE@XZ     10004100 f i AssemblySamtoolsMpileup.obj
 0001:00003110       ??1SamtoolsMpileupTask@LocalWorkflow@U2@@UAE@XZ 10004110 f i AssemblySamtoolsMpileup.obj
 0001:00003170       ??1_Generic_error_category@std@@UAE@XZ 10004170 f i AssemblySamtoolsMpileup.obj
 0001:00003180       ??1_Iostream_error_category@std@@UAE@XZ 10004180 f i AssemblySamtoolsMpileup.obj
 0001:00003190       ??1_System_error_category@std@@UAE@XZ 10004190 f i AssemblySamtoolsMpileup.obj
 0001:000031a0       ??1error_category@std@@UAE@XZ 100041a0 f i AssemblySamtoolsMpileup.obj
 0001:000031b0       ??2@YAPAXIPAX@Z            100041b0 f i AssemblySamtoolsMpileup.obj
 0001:000031c0       ??3@YAXPAX0@Z              100041c0 f i AssemblySamtoolsMpileup.obj
 0001:000031d0       ??4?$QList@VQString@@@@QAEAAV0@ABV0@@Z 100041d0 f i AssemblySamtoolsMpileup.obj
 0001:00003210       ??6QStringList@@QAEAAV0@ABV?$QList@VQString@@@@@Z 10004210 f i AssemblySamtoolsMpileup.obj
 0001:00003230       ??6QStringList@@QAEAAV0@ABVQString@@@Z 10004230 f i AssemblySamtoolsMpileup.obj
 0001:00003250       ??8error_category@std@@QBE_NABV01@@Z 10004250 f i AssemblySamtoolsMpileup.obj
 0001:00003260       ??8error_condition@std@@QBE_NABV01@@Z 10004260 f i AssemblySamtoolsMpileup.obj
 0001:00003280       ??9const_iterator@?$QList@PAVGObject@U2@@@@QBE_NABV01@@Z 10004280 f i AssemblySamtoolsMpileup.obj
 0001:000032a0       ??9const_iterator@?$QList@VQString@@@@QBE_NABV01@@Z 100042a0 f i AssemblySamtoolsMpileup.obj
 0001:000032c0       ??A?$QMap@VQString@@VQVariant@@@@QAEAAVQVariant@@ABVQString@@@Z 100042c0 f i AssemblySamtoolsMpileup.obj
 0001:00003390       ??B?$QScopedPointer@VDocument@U2@@U?$QScopedPointerDeleter@VDocument@U2@@@@@@QBEPQ0@PAVDocument@U2@@XZ 10004390 f i AssemblySamtoolsMpileup.obj
 0001:000033a0       ??BQFlag@@QBEHXZ           100043a0 f i AssemblySamtoolsMpileup.obj
 0001:000033b0       ??C?$QScopedPointer@VDocument@U2@@U?$QScopedPointerDeleter@VDocument@U2@@@@@@QBEPAVDocument@U2@@XZ 100043b0 f i AssemblySamtoolsMpileup.obj
 0001:000033c0       ??Dconst_iterator@?$QList@PAVGObject@U2@@@@QBEABQAVGObject@U2@@XZ 100043c0 f i AssemblySamtoolsMpileup.obj
 0001:000033d0       ??Dconst_iterator@?$QList@VQString@@@@QBEABVQString@@XZ 100043d0 f i AssemblySamtoolsMpileup.obj
 0001:000033e0       ??Diterator@?$QList@VFormatDetectionResult@U2@@@@QBEAAVFormatDetectionResult@U2@@XZ 100043e0 f i AssemblySamtoolsMpileup.obj
 0001:000033f0       ??Diterator@?$QMap@VQString@@VQVariant@@@@QBEAAVQVariant@@XZ 100043f0 f i AssemblySamtoolsMpileup.obj
 0001:00003400       ??Econst_iterator@?$QList@PAVGObject@U2@@@@QAEAAV01@XZ 10004400 f i AssemblySamtoolsMpileup.obj
 0001:00003410       ??Econst_iterator@?$QList@VQString@@@@QAEAAV01@XZ 10004410 f i AssemblySamtoolsMpileup.obj
 0001:00003420       ??H@YA?BVQString@@ABV0@0@Z 10004420 f i AssemblySamtoolsMpileup.obj
 0001:00003490       ??Y?$QList@VQString@@@@QAEAAV0@ABV0@@Z 10004490 f i AssemblySamtoolsMpileup.obj
 0001:00003590       ??_5?$QFlags@W4TypeFlag@QMetaType@@@@QAEAAV0@W4TypeFlag@QMetaType@@@Z 10004590 f i AssemblySamtoolsMpileup.obj
 0001:000035a0       ??_G?$QMap@VQString@@VQVariant@@@@QAEPAXI@Z 100045a0 f i AssemblySamtoolsMpileup.obj
 0001:00003600       ??_G?$QSharedDataPointer@VDbiDataHandler@Workflow@U2@@@@QAEPAXI@Z 10004600 f i AssemblySamtoolsMpileup.obj
 0001:00003640       ??_ECallVariantsTask@LocalWorkflow@U2@@UAEPAXI@Z 10004640 f i AssemblySamtoolsMpileup.obj
 0001:00003640       ??_GCallVariantsTask@LocalWorkflow@U2@@UAEPAXI@Z 10004640 f i AssemblySamtoolsMpileup.obj
 0001:00003670       ??_GFormatDetectionResult@U2@@QAEPAXI@Z 10004670 f i AssemblySamtoolsMpileup.obj
 0001:000036a0       ??_ELoadDocumentTask@U2@@UAEPAXI@Z 100046a0 f i AssemblySamtoolsMpileup.obj
 0001:000036a0       ??_GLoadDocumentTask@U2@@UAEPAXI@Z 100046a0 f i AssemblySamtoolsMpileup.obj
 0001:000036d0       ??_GQString@@QAEPAXI@Z     100046d0 f i AssemblySamtoolsMpileup.obj
 0001:00003700       ??_GQVariant@@QAEPAXI@Z    10004700 f i AssemblySamtoolsMpileup.obj
 0001:00003730       ??_GSamtoolsMpileupTask@LocalWorkflow@U2@@UAEPAXI@Z 10004730 f i AssemblySamtoolsMpileup.obj
 0001:00003730       ??_ESamtoolsMpileupTask@LocalWorkflow@U2@@UAEPAXI@Z 10004730 f i AssemblySamtoolsMpileup.obj
 0001:000037a0       ??_GU2DbiRef@U2@@QAEPAXI@Z 100047a0 f i AssemblySamtoolsMpileup.obj
 0001:000037d0       ??_G_Generic_error_category@std@@UAEPAXI@Z 100047d0 f i AssemblySamtoolsMpileup.obj
 0001:000037d0       ??_E_Generic_error_category@std@@UAEPAXI@Z 100047d0 f i AssemblySamtoolsMpileup.obj
 0001:00003800       ??_G_Iostream_error_category@std@@UAEPAXI@Z 10004800 f i AssemblySamtoolsMpileup.obj
 0001:00003800       ??_E_Iostream_error_category@std@@UAEPAXI@Z 10004800 f i AssemblySamtoolsMpileup.obj
 0001:00003830       ??_E_System_error_category@std@@UAEPAXI@Z 10004830 f i AssemblySamtoolsMpileup.obj
 0001:00003830       ??_G_System_error_category@std@@UAEPAXI@Z 10004830 f i AssemblySamtoolsMpileup.obj
 0001:00003860       ??_Gerror_category@std@@UAEPAXI@Z 10004860 f i AssemblySamtoolsMpileup.obj
 0001:00003860       ??_Eerror_category@std@@UAEPAXI@Z 10004860 f i AssemblySamtoolsMpileup.obj
 0001:00003890       ?Construct@?$QMetaTypeFunctionHelper@V?$QSharedDataPointer@VDbiDataHandler@Workflow@U2@@@@$00@QtMetaTypePrivate@@SAPAXPAXPBX@Z 10004890 f i AssemblySamtoolsMpileup.obj
 0001:000038e0       ?Construct@?$QMetaTypeFunctionHelper@VU2DbiRef@U2@@$00@QtMetaTypePrivate@@SAPAXPAXPBX@Z 100048e0 f i AssemblySamtoolsMpileup.obj
 0001:000039f0       ?Create@?$QMetaTypeFunctionHelper@V?$QSharedDataPointer@VDbiDataHandler@Workflow@U2@@@@$00@QtMetaTypePrivate@@SAPAXPBX@Z 100049f0 f i AssemblySamtoolsMpileup.obj
 0001:00003a40       ?Create@?$QMetaTypeFunctionHelper@VU2DbiRef@U2@@$00@QtMetaTypePrivate@@SAPAXPBX@Z 10004a40 f i AssemblySamtoolsMpileup.obj
 0001:00003b50       ?Delete@?$QMetaTypeFunctionHelper@V?$QSharedDataPointer@VDbiDataHandler@Workflow@U2@@@@$00@QtMetaTypePrivate@@SAXPAX@Z 10004b50 f i AssemblySamtoolsMpileup.obj
 0001:00003b90       ?Delete@?$QMetaTypeFunctionHelper@VU2DbiRef@U2@@$00@QtMetaTypePrivate@@SAXPAX@Z 10004b90 f i AssemblySamtoolsMpileup.obj
 0001:00003bb0       ?Destruct@?$QMetaTypeFunctionHelper@V?$QSharedDataPointer@VDbiDataHandler@Workflow@U2@@@@$00@QtMetaTypePrivate@@SAXPAX@Z 10004bb0 f i AssemblySamtoolsMpileup.obj
 0001:00003be0       ?Destruct@?$QMetaTypeFunctionHelper@VU2DbiRef@U2@@$00@QtMetaTypePrivate@@SAXPAX@Z 10004be0 f i AssemblySamtoolsMpileup.obj
 0001:00003bf0       ?_Copy@?$basic_string@DU?$char_traits@D@std@@V?$allocator@D@2@@std@@QAEXII@Z 10004bf0 f i AssemblySamtoolsMpileup.obj
 0001:00003d40       ?_Eos@?$basic_string@DU?$char_traits@D@std@@V?$allocator@D@2@@std@@QAEXI@Z 10004d40 f i AssemblySamtoolsMpileup.obj
 0001:00003d70       ?_Getal@?$_String_alloc@$0A@U?$_String_base_types@DV?$allocator@D@std@@@std@@@std@@QBE?AU?$_Wrap_alloc@V?$allocator@D@std@@@2@XZ 10004d70 f i AssemblySamtoolsMpileup.obj
 0001:00003d80       ?_Grow@?$basic_string@DU?$char_traits@D@std@@V?$allocator@D@2@@std@@QAE_NI_N@Z 10004d80 f i AssemblySamtoolsMpileup.obj
 0001:00003e30       ?_Inside@?$basic_string@DU?$char_traits@D@std@@V?$allocator@D@2@@std@@QAE_NPBD@Z 10004e30 f i AssemblySamtoolsMpileup.obj
 0001:00003e70       ?_Myptr@?$_String_val@U?$_Simple_types@D@std@@@std@@QAEPADXZ 10004e70 f i AssemblySamtoolsMpileup.obj
 0001:00003e80       ?_Myptr@?$_String_val@U?$_Simple_types@D@std@@@std@@QBEPBDXZ 10004e80 f i AssemblySamtoolsMpileup.obj
 0001:00003e90       ?_Tidy@?$basic_string@DU?$char_traits@D@std@@V?$allocator@D@2@@std@@QAEX_NI@Z 10004e90 f i AssemblySamtoolsMpileup.obj
 0001:00003ee0       ?_Xlen@?$basic_string@DU?$char_traits@D@std@@V?$allocator@D@2@@std@@QBEXXZ 10004ee0 f i AssemblySamtoolsMpileup.obj
 0001:00003ef0       ?_Xran@?$basic_string@DU?$char_traits@D@std@@V?$allocator@D@2@@std@@QBEXXZ 10004ef0 f i AssemblySamtoolsMpileup.obj
 0001:00003f00       ?allocate@?$_Wrap_alloc@V?$allocator@D@std@@@std@@QAEPADI@Z 10004f00 f i AssemblySamtoolsMpileup.obj
 0001:00003f30       ?allocate@?$allocator@D@std@@QAEPADI@Z 10004f30 f i AssemblySamtoolsMpileup.obj
 0001:00003f60       ?append@?$QList@PAVTask@U2@@@@QAEXABQAVTask@U2@@@Z 10004f60 f i AssemblySamtoolsMpileup.obj
 0001:00003ff0       ?append@?$QList@V?$QMap@VQString@@VQVariant@@@@@@QAEXABV?$QMap@VQString@@VQVariant@@@@@Z 10004ff0 f i AssemblySamtoolsMpileup.obj
 0001:000040d0       ?append@?$QList@VQString@@@@QAEXABVQString@@@Z 100050d0 f i AssemblySamtoolsMpileup.obj
 0001:000041c0       ?assign@?$basic_string@DU?$char_traits@D@std@@V?$allocator@D@2@@std@@QAEAAV12@ABV12@II@Z 100051c0 f i AssemblySamtoolsMpileup.obj
 0001:000042e0       ?assign@?$basic_string@DU?$char_traits@D@std@@V?$allocator@D@2@@std@@QAEAAV12@PBD@Z 100052e0 f i AssemblySamtoolsMpileup.obj
 0001:00004320       ?assign@?$basic_string@DU?$char_traits@D@std@@V?$allocator@D@2@@std@@QAEAAV12@PBDI@Z 10005320 f i AssemblySamtoolsMpileup.obj
 0001:00004420       ?assign@?$char_traits@D@std@@SAXAADABD@Z 10005420 f i AssemblySamtoolsMpileup.obj
 0001:00004430       ?begin@?$QList@PAVGObject@U2@@@@QBE?AVconst_iterator@1@XZ 10005430 f i AssemblySamtoolsMpileup.obj
 0001:00004450       ?begin@?$QList@VFormatDetectionResult@U2@@@@QAE?AViterator@1@XZ 10005450 f i AssemblySamtoolsMpileup.obj
 0001:00004490       ?begin@?$QList@VQString@@@@QBE?AVconst_iterator@1@XZ 10005490 f i AssemblySamtoolsMpileup.obj
 0001:000044b0       ?category@error_code@std@@QBEABVerror_category@2@XZ 100054b0 f i AssemblySamtoolsMpileup.obj
 0001:000044c0       ?category@error_condition@std@@QBEABVerror_category@2@XZ 100054c0 f i AssemblySamtoolsMpileup.obj
 0001:000044d0       ?checkExitCode@SamtoolsMpileupTask@LocalWorkflow@U2@@AAEXPAVQProcess@@ABVQString@@@Z 100054d0 f   AssemblySamtoolsMpileup.obj
 0001:00004630       ?cleanup@?$QScopedPointerDeleter@VDocument@U2@@@@SAXPAVDocument@U2@@@Z 10005630 f i AssemblySamtoolsMpileup.obj
 0001:00004650       ?cleanup@?$QScopedPointerDeleter@VQProcess@@@@SAXPAVQProcess@@@Z 10005650 f i AssemblySamtoolsMpileup.obj
 0001:00004670       ?copy@?$QMapNode@VQString@@VQVariant@@@@QBEPAU1@PAU?$QMapData@VQString@@VQVariant@@@@@Z 10005670 f i AssemblySamtoolsMpileup.obj
 0001:00004700       ?copy@?$char_traits@D@std@@SAPADPADPBDI@Z 10005700 f i AssemblySamtoolsMpileup.obj
 0001:00004720       ?create@?$QMapData@VQString@@VQVariant@@@@SAPAU1@XZ 10005720 f i AssemblySamtoolsMpileup.obj
 0001:00004730       ?createNode@?$QMapData@VQString@@VQVariant@@@@QAEPAU?$QMapNode@VQString@@VQVariant@@@@ABVQString@@ABVQVariant@@PAU2@_N@Z 10005730 f i AssemblySamtoolsMpileup.obj
 0001:000047f0       ?dealloc@?$QList@PAVGObject@U2@@@@AAEXPAUData@QListData@@@Z 100057f0 f i AssemblySamtoolsMpileup.obj
 0001:00004810       ?dealloc@?$QList@PAVTask@U2@@@@AAEXPAUData@QListData@@@Z 10005810 f i AssemblySamtoolsMpileup.obj
 0001:00004830       ?dealloc@?$QList@V?$QMap@VQString@@VQVariant@@@@@@AAEXPAUData@QListData@@@Z 10005830 f i AssemblySamtoolsMpileup.obj
 0001:00004860       ?dealloc@?$QList@VFormatDetectionResult@U2@@@@AAEXPAUData@QListData@@@Z 10005860 f i AssemblySamtoolsMpileup.obj
 0001:000048c0       ?dealloc@?$QList@VQString@@@@AAEXPAUData@QListData@@@Z 100058c0 f i AssemblySamtoolsMpileup.obj
 0001:00004900       ?deallocate@?$_Wrap_alloc@V?$allocator@D@std@@@std@@QAEXPADI@Z 10005900 f i AssemblySamtoolsMpileup.obj
 0001:00004920       ?deallocate@?$allocator@D@std@@QAEXPADI@Z 10005920 f i AssemblySamtoolsMpileup.obj
 0001:00004940       ?default_error_condition@_System_error_category@std@@UBE?AVerror_condition@2@H@Z 10005940 f i AssemblySamtoolsMpileup.obj
 0001:00004980       ?default_error_condition@error_category@std@@UBE?AVerror_condition@2@H@Z 10005980 f i AssemblySamtoolsMpileup.obj
 0001:000049a0       ?deref@?$QBasicAtomicInteger@H@@QAE_NXZ 100059a0 f i AssemblySamtoolsMpileup.obj
 0001:000049b0       ?deref@RefCount@QtPrivate@@QAE_NXZ 100059b0 f i AssemblySamtoolsMpileup.obj
 0001:000049d0       ?destroy@?$QMapData@VQString@@VQVariant@@@@QAEXXZ 100059d0 f i AssemblySamtoolsMpileup.obj
 0001:00004a00       ?destroySubTree@?$QMapNode@VQString@@VQVariant@@@@QAEXXZ 10005a00 f i AssemblySamtoolsMpileup.obj
 0001:00004a40       ?detach@?$QList@VFormatDetectionResult@U2@@@@QAEXXZ 10005a40 f i AssemblySamtoolsMpileup.obj
 0001:00004a60       ?detach@?$QMap@VQString@@VQVariant@@@@QAEXXZ 10005a60 f i AssemblySamtoolsMpileup.obj
 0001:00004a80       ?detach_helper@?$QList@VFormatDetectionResult@U2@@@@AAEXH@Z 10005a80 f i AssemblySamtoolsMpileup.obj
 0001:00004b50       ?detach_helper@?$QList@VFormatDetectionResult@U2@@@@AAEXXZ 10005b50 f i AssemblySamtoolsMpileup.obj
 0001:00004b60       ?detach_helper@?$QMap@VQString@@VQVariant@@@@AAEXXZ 10005b60 f i AssemblySamtoolsMpileup.obj
 0001:00004be0       ?detach_helper_grow@?$QList@PAVTask@U2@@@@AAEPAUNode@1@HH@Z 10005be0 f i AssemblySamtoolsMpileup.obj
 0001:00004cf0       ?detach_helper_grow@?$QList@V?$QMap@VQString@@VQVariant@@@@@@AAEPAUNode@1@HH@Z 10005cf0 f i AssemblySamtoolsMpileup.obj
 0001:00004e60       ?detach_helper_grow@?$QList@VQString@@@@AAEPAUNode@1@HH@Z 10005e60 f i AssemblySamtoolsMpileup.obj
 0001:00004fe0       ?end@?$QList@PAVGObject@U2@@@@QBE?AVconst_iterator@1@XZ 10005fe0 f i AssemblySamtoolsMpileup.obj
 0001:00005000       ?end@?$QList@VQString@@@@QBE?AVconst_iterator@1@XZ 10006000 f i AssemblySamtoolsMpileup.obj
 0001:00005020       ?end@?$QMapData@VQString@@VQVariant@@@@QAEPAU?$QMapNode@VQString@@VQVariant@@@@XZ 10006020 f i AssemblySamtoolsMpileup.obj
 0001:00005030       ?ensureFileExists@CallVariantsTask@LocalWorkflow@U2@@AAE_NABVQString@@W4FileType@123@@Z 10006030 f   AssemblySamtoolsMpileup.obj
 0001:00005150       ?equivalent@error_category@std@@UBE_NABVerror_code@2@H@Z 10006150 f i AssemblySamtoolsMpileup.obj
 0001:00005170       ?equivalent@error_category@std@@UBE_NHABVerror_condition@2@@Z 10006170 f i AssemblySamtoolsMpileup.obj
 0001:000051b0       ?erase@?$basic_string@DU?$char_traits@D@std@@V?$allocator@D@2@@std@@QAEAAV12@I@Z 100061b0 f i AssemblySamtoolsMpileup.obj
 0001:000051f0       ?erase@?$basic_string@DU?$char_traits@D@std@@V?$allocator@D@2@@std@@QAEAAV12@II@Z 100061f0 f i AssemblySamtoolsMpileup.obj
 0001:00005290       ?findNode@?$QMapData@VQString@@VQVariant@@@@QBEPAU?$QMapNode@VQString@@VQVariant@@@@ABVQString@@@Z 10006290 f i AssemblySamtoolsMpileup.obj
 0001:000052d0       ?first@?$QList@VFormatDetectionResult@U2@@@@QAEAAVFormatDetectionResult@U2@@XZ 100062d0 f i AssemblySamtoolsMpileup.obj
 0001:00005300       ?generic_category@std@@YAABVerror_category@1@XZ 10006300 f i AssemblySamtoolsMpileup.obj
 0001:00005310       ?getBcfViewArgs@CallVariantsTaskSettings@LocalWorkflow@U2@@QBE?AVQStringList@@XZ 10006310 f   AssemblySamtoolsMpileup.obj
 0001:00005970       ?getMpiliupArgs@CallVariantsTaskSettings@LocalWorkflow@U2@@QBE?AVQStringList@@XZ 10006970 f   AssemblySamtoolsMpileup.obj
 0001:00005f20       ?getVarFilterArgs@CallVariantsTaskSettings@LocalWorkflow@U2@@QBE?AVQStringList@@XZ 10006f20 f   AssemblySamtoolsMpileup.obj
 0001:00006410       ?insert@?$QMap@VQString@@VQVariant@@@@QAE?AViterator@1@ABVQString@@ABVQVariant@@@Z 10007410 f i AssemblySamtoolsMpileup.obj
 0001:000064d0       ?isEmpty@?$QList@VFormatDetectionResult@U2@@@@QBE_NXZ 100074d0 f i AssemblySamtoolsMpileup.obj
 0001:000064e0       ?isEmpty@?$QList@VQString@@@@QBE_NXZ 100074e0 f i AssemblySamtoolsMpileup.obj
 0001:000064f0       ?isNull@?$QScopedPointer@VDocument@U2@@U?$QScopedPointerDeleter@VDocument@U2@@@@@@QBE_NXZ 100074f0 f i AssemblySamtoolsMpileup.obj
 0001:00006500       ?isShared@RefCount@QtPrivate@@QBE_NXZ 10007500 f i AssemblySamtoolsMpileup.obj
 0001:00006520       ?leftNode@?$QMapNode@VQString@@VQVariant@@@@QBEPAU1@XZ 10007520 f i AssemblySamtoolsMpileup.obj
 0001:00006530       ?length@?$char_traits@D@std@@SAIPBD@Z 10007530 f i AssemblySamtoolsMpileup.obj
 0001:00006550       ?load@?$QBasicAtomicInteger@H@@QBEHXZ 10007550 f i AssemblySamtoolsMpileup.obj
 0001:00006560       ?loadAcquire@?$QBasicAtomicInteger@H@@QBEHXZ 10007560 f i AssemblySamtoolsMpileup.obj
 0001:00006570       ?lowerBound@?$QMapNode@VQString@@VQVariant@@@@QAEPAU1@ABVQString@@@Z 10007570 f i AssemblySamtoolsMpileup.obj
 0001:000065b0       ?max_size@?$_Wrap_alloc@V?$allocator@D@std@@@std@@QBEIXZ 100075b0 f i AssemblySamtoolsMpileup.obj
 0001:000065c0       ?max_size@?$allocator@D@std@@QBEIXZ 100075c0 f i AssemblySamtoolsMpileup.obj
 0001:000065d0       ?max_size@?$allocator_traits@V?$allocator@D@std@@@std@@SAIABV?$allocator@D@2@@Z 100075d0 f i AssemblySamtoolsMpileup.obj
 0001:000065e0       ?max_size@?$basic_string@DU?$char_traits@D@std@@V?$allocator@D@2@@std@@QBEIXZ 100075e0 f i AssemblySamtoolsMpileup.obj
 0001:000065f0       ?message@_Generic_error_category@std@@UBE?AV?$basic_string@DU?$char_traits@D@std@@V?$allocator@D@2@@2@H@Z 100075f0 f i AssemblySamtoolsMpileup.obj
 0001:00006670       ?message@_Iostream_error_category@std@@UBE?AV?$basic_string@DU?$char_traits@D@std@@V?$allocator@D@2@@2@H@Z 10007670 f i AssemblySamtoolsMpileup.obj
 0001:000066c0       ?message@_System_error_category@std@@UBE?AV?$basic_string@DU?$char_traits@D@std@@V?$allocator@D@2@@2@H@Z 100076c0 f i AssemblySamtoolsMpileup.obj
 0001:00006740       ?move@?$char_traits@D@std@@SAPADPADPBDI@Z 10007740 f i AssemblySamtoolsMpileup.obj
 0001:00006760       ?name@_Generic_error_category@std@@UBEPBDXZ 10007760 f i AssemblySamtoolsMpileup.obj
 0001:00006770       ?name@_Iostream_error_category@std@@UBEPBDXZ 10007770 f i AssemblySamtoolsMpileup.obj
 0001:00006780       ?name@_System_error_category@std@@UBEPBDXZ 10007780 f i AssemblySamtoolsMpileup.obj
 0001:00006790       ?node_construct@?$QList@PAVTask@U2@@@@AAEXPAUNode@1@ABQAVTask@U2@@@Z 10007790 f i AssemblySamtoolsMpileup.obj
 0001:000067b0       ?node_construct@?$QList@V?$QMap@VQString@@VQVariant@@@@@@AAEXPAUNode@1@ABV?$QMap@VQString@@VQVariant@@@@@Z 100077b0 f i AssemblySamtoolsMpileup.obj
 0001:00006830       ?node_construct@?$QList@VQString@@@@AAEXPAUNode@1@ABVQString@@@Z 10007830 f i AssemblySamtoolsMpileup.obj
 0001:00006880       ?node_copy@?$QList@PAVGObject@U2@@@@AAEXPAUNode@1@00@Z 10007880 f i AssemblySamtoolsMpileup.obj
 0001:000068b0       ?node_copy@?$QList@PAVTask@U2@@@@AAEXPAUNode@1@00@Z 100078b0 f i AssemblySamtoolsMpileup.obj
 0001:000068e0       ?node_copy@?$QList@V?$QMap@VQString@@VQVariant@@@@@@AAEXPAUNode@1@00@Z 100078e0 f i AssemblySamtoolsMpileup.obj
 0001:00006a10       ?node_copy@?$QList@VFormatDetectionResult@U2@@@@AAEXPAUNode@1@00@Z 10007a10 f i AssemblySamtoolsMpileup.obj
 0001:00006ae0       ?node_copy@?$QList@VQString@@@@AAEXPAUNode@1@00@Z 10007ae0 f i AssemblySamtoolsMpileup.obj
 0001:00006b80       ?node_destruct@?$QList@PAVGObject@U2@@@@AAEXPAUNode@1@0@Z 10007b80 f i AssemblySamtoolsMpileup.obj
 0001:00006b90       ?node_destruct@?$QList@PAVTask@U2@@@@AAEXPAUNode@1@0@Z 10007b90 f i AssemblySamtoolsMpileup.obj
 0001:00006ba0       ?node_destruct@?$QList@PAVTask@U2@@@@AAEXPAUNode@1@@Z 10007ba0 f i AssemblySamtoolsMpileup.obj
 0001:00006bb0       ?node_destruct@?$QList@V?$QMap@VQString@@VQVariant@@@@@@AAEXPAUNode@1@0@Z 10007bb0 f i AssemblySamtoolsMpileup.obj
 0001:00006c30       ?node_destruct@?$QList@V?$QMap@VQString@@VQVariant@@@@@@AAEXPAUNode@1@@Z 10007c30 f i AssemblySamtoolsMpileup.obj
 0001:00006c90       ?node_destruct@?$QList@VFormatDetectionResult@U2@@@@AAEXPAUNode@1@0@Z 10007c90 f i AssemblySamtoolsMpileup.obj
 0001:00006cd0       ?node_destruct@?$QList@VQString@@@@AAEXPAUNode@1@0@Z 10007cd0 f i AssemblySamtoolsMpileup.obj
 0001:00006d00       ?node_destruct@?$QList@VQString@@@@AAEXPAUNode@1@@Z 10007d00 f i AssemblySamtoolsMpileup.obj
 0001:00006d10       ?onSubTaskFinished@CallVariantsTask@LocalWorkflow@U2@@UAE?AV?$QList@PAVTask@U2@@@@PAVTask@3@@Z 10007d10 f   AssemblySamtoolsMpileup.obj
 0001:00007520       ?prepare@CallVariantsTask@LocalWorkflow@U2@@UAEXXZ 10008520 f   AssemblySamtoolsMpileup.obj
 0001:000077d0       ?prepare@SamtoolsMpileupTask@LocalWorkflow@U2@@UAEXXZ 100087d0 f   AssemblySamtoolsMpileup.obj
 0001:00007a30       ?qt_metatype_id@?$QMetaTypeId2@V?$QSharedDataPointer@VDbiDataHandler@Workflow@U2@@@@@@SAHXZ 10008a30 f i AssemblySamtoolsMpileup.obj
 0001:00007a40       ?qt_metatype_id@?$QMetaTypeId2@VU2DbiRef@U2@@@@SAHXZ 10008a40 f i AssemblySamtoolsMpileup.obj
 0001:00007a50       ?qt_metatype_id@?$QMetaTypeId@V?$QSharedDataPointer@VDbiDataHandler@Workflow@U2@@@@@@SAHXZ 10008a50 f i AssemblySamtoolsMpileup.obj
 0001:00007af0       ?qt_metatype_id@?$QMetaTypeId@VU2DbiRef@U2@@@@SAHXZ 10008af0 f i AssemblySamtoolsMpileup.obj
 0001:00007b90       ?qt_metatype_id@?$QMetaTypeIdHelper@V?$QSharedDataPointer@VDbiDataHandler@Workflow@U2@@@@$00@QtPrivate@@SAHXZ 10008b90 f i AssemblySamtoolsMpileup.obj
 0001:00007ba0       ?qt_metatype_id@?$QMetaTypeIdHelper@VU2DbiRef@U2@@$00@QtPrivate@@SAHXZ 10008ba0 f i AssemblySamtoolsMpileup.obj
 0001:00007bb0       ?qt_noop@@YAXXZ            10008bb0 f i AssemblySamtoolsMpileup.obj
 0001:00007bc0       ?ref@?$QBasicAtomicInteger@H@@QAE_NXZ 10008bc0 f i AssemblySamtoolsMpileup.obj
 0001:00007be0       ?ref@RefCount@QtPrivate@@QAE_NXZ 10008be0 f i AssemblySamtoolsMpileup.obj
 0001:00007c00       ?registerConverter@?$AssociativeContainerConverterHelper@V?$QSharedDataPointer@VDbiDataHandler@Workflow@U2@@@@$0A@@QtPrivate@@SA_NH@Z 10008c00 f i AssemblySamtoolsMpileup.obj
 0001:00007c10       ?registerConverter@?$AssociativeContainerConverterHelper@VU2DbiRef@U2@@$0A@@QtPrivate@@SA_NH@Z 10008c10 f i AssemblySamtoolsMpileup.obj
 0001:00007c20       ?registerConverter@?$IsPair@V?$QSharedDataPointer@VDbiDataHandler@Workflow@U2@@@@@QtPrivate@@SA_NH@Z 10008c20 f i AssemblySamtoolsMpileup.obj
 0001:00007c30       ?registerConverter@?$IsPair@VU2DbiRef@U2@@@QtPrivate@@SA_NH@Z 10008c30 f i AssemblySamtoolsMpileup.obj
 0001:00007c40       ?registerConverter@?$MetaTypeSmartPointerHelper@V?$QSharedDataPointer@VDbiDataHandler@Workflow@U2@@@@X@QtPrivate@@SA_NH@Z 10008c40 f i AssemblySamtoolsMpileup.obj
 0001:00007c50       ?registerConverter@?$MetaTypeSmartPointerHelper@VU2DbiRef@U2@@X@QtPrivate@@SA_NH@Z 10008c50 f i AssemblySamtoolsMpileup.obj
 0001:00007c60       ?registerConverter@?$SequentialContainerConverterHelper@V?$QSharedDataPointer@VDbiDataHandler@Workflow@U2@@@@$0A@@QtPrivate@@SA_NH@Z 10008c60 f i AssemblySamtoolsMpileup.obj
 0001:00007c70       ?registerConverter@?$SequentialContainerConverterHelper@VU2DbiRef@U2@@$0A@@QtPrivate@@SA_NH@Z 10008c70 f i AssemblySamtoolsMpileup.obj
 0001:00007c80       ?rightNode@?$QMapNode@VQString@@VQVariant@@@@QBEPAU1@XZ 10008c80 f i AssemblySamtoolsMpileup.obj
 0001:00007c90       ?root@?$QMapData@VQString@@VQVariant@@@@QBEPAU?$QMapNode@VQString@@VQVariant@@@@XZ 10008c90 f i AssemblySamtoolsMpileup.obj
 0001:00007cb0       ?run@SamtoolsMpileupTask@LocalWorkflow@U2@@UAEXXZ 10008cb0 f   AssemblySamtoolsMpileup.obj
 0001:00008250       ?size@?$QList@VQString@@@@QBEHXZ 10009250 f i AssemblySamtoolsMpileup.obj
 0001:00008260       ?size@?$basic_string@DU?$char_traits@D@std@@V?$allocator@D@2@@std@@QBEIXZ 10009260 f i AssemblySamtoolsMpileup.obj
 0001:00008270       ?start@SamtoolsMpileupTask@LocalWorkflow@U2@@AAEXABVProcessRun@3@ABVQString@@@Z 10009270 f   AssemblySamtoolsMpileup.obj
 0001:00008350       ?storeRelease@?$QBasicAtomicInteger@H@@QAEXH@Z 10009350 f i AssemblySamtoolsMpileup.obj
 0001:00008360       ?swap@?$QList@VQString@@@@QAEXAAV1@@Z 10009360 f i AssemblySamtoolsMpileup.obj
 0001:00008380       ?system_category@std@@YAABVerror_category@1@XZ 10009380 f i AssemblySamtoolsMpileup.obj
 0001:00008390       ?t@Node@?$QList@PAVGObject@U2@@@@QAEAAPAVGObject@U2@@XZ 10009390 f i AssemblySamtoolsMpileup.obj
 0001:000083a0       ?t@Node@?$QList@VFormatDetectionResult@U2@@@@QAEAAVFormatDetectionResult@U2@@XZ 100093a0 f i AssemblySamtoolsMpileup.obj
 0001:000083b0       ?t@Node@?$QList@VQString@@@@QAEAAVQString@@XZ 100093b0 f i AssemblySamtoolsMpileup.obj
 0001:000083c0       ?tmpFilePath@CallVariantsTask@LocalWorkflow@U2@@SA?AVQString@@ABV4@0AAVU2OpStatus@3@@Z 100093c0 f   AssemblySamtoolsMpileup.obj
 0001:00008470       ?toString@CallVariantsTask@LocalWorkflow@U2@@CA?AVQString@@W4FileType@123@@Z 10009470 f   AssemblySamtoolsMpileup.obj
 0001:00008620       ?tr@CallVariantsTask@LocalWorkflow@U2@@SA?AVQString@@PBD0H@Z 10009620 f i AssemblySamtoolsMpileup.obj
 0001:00008650       ?tr@SamtoolsMpileupTask@LocalWorkflow@U2@@SA?AVQString@@PBD0H@Z 10009650 f i AssemblySamtoolsMpileup.obj
 0001:00008680       ?value@?$MetaObjectForType@V?$QSharedDataPointer@VDbiDataHandler@Workflow@U2@@@@$0A@@QtPrivate@@SAPBUQMetaObject@@XZ 10009680 f i AssemblySamtoolsMpileup.obj
 0001:00008690       ?value@?$MetaObjectForType@VU2DbiRef@U2@@$0A@@QtPrivate@@SAPBUQMetaObject@@XZ 10009690 f i AssemblySamtoolsMpileup.obj
 0001:000086a0       ?value@error_code@std@@QBEHXZ 100096a0 f i AssemblySamtoolsMpileup.obj
 0001:000086b0       ?value@error_condition@std@@QBEHXZ 100096b0 f i AssemblySamtoolsMpileup.obj
 0001:000086c0       _hypot                     100096c0 f i AssemblySamtoolsMpileup.obj
 0001:000086f0       ??$_Move@AAPAVDataType@U2@@@std@@YA$$QAPAVDataType@U2@@AAPAV12@@Z 100096f0 f i SamtoolMpileupWorker.obj
 0001:00008700       ??$getAttributeValue@H@Attribute@U2@@QBEHPAVWorkflowContext@Workflow@1@@Z 10009700 f i SamtoolMpileupWorker.obj
 0001:00008ad0       ??$getAttributeValue@M@Attribute@U2@@QBEMPAVWorkflowContext@Workflow@1@@Z 10009ad0 f i SamtoolMpileupWorker.obj
 0001:00008b40       ??$getAttributeValue@VQString@@@Attribute@U2@@QBE?AVQString@@PAVWorkflowContext@Workflow@1@@Z 10009b40 f i SamtoolMpileupWorker.obj
 0001:00008ed0       ??$getAttributeValue@_N@Attribute@U2@@QBE_NPAVWorkflowContext@Workflow@1@@Z 10009ed0 f i SamtoolMpileupWorker.obj
 0001:00008f10       ??$getAttributeValueWithoutScript@H@Attribute@U2@@QBEHXZ 10009f10 f i SamtoolMpileupWorker.obj
 0001:00008f50       ??$getAttributeValueWithoutScript@M@Attribute@U2@@QBEMXZ 10009f50 f i SamtoolMpileupWorker.obj
 0001:00008fb0       ??$getAttributeValueWithoutScript@V?$QMap@VQString@@V1@@@@Attribute@U2@@QBE?AV?$QMap@VQString@@V1@@@XZ 10009fb0 f i SamtoolMpileupWorker.obj
 0001:00008fd0       ??$getAttributeValueWithoutScript@VQString@@@Attribute@U2@@QBE?AVQString@@XZ 10009fd0 f i SamtoolMpileupWorker.obj
 0001:00008ff0       ??$getAttributeValueWithoutScript@_N@Attribute@U2@@QBE_NXZ 10009ff0 f i SamtoolMpileupWorker.obj
 0001:00009030       ??$getValue@H@BaseWorker@LocalWorkflow@U2@@IBEHABVQString@@@Z 1000a030 f i SamtoolMpileupWorker.obj
 0001:00009060       ??$getValue@M@BaseWorker@LocalWorkflow@U2@@IBEMABVQString@@@Z 1000a060 f i SamtoolMpileupWorker.obj
 0001:000090e0       ??$getValue@VQString@@@BaseWorker@LocalWorkflow@U2@@IBE?AVQString@@ABV3@@Z 1000a0e0 f i SamtoolMpileupWorker.obj
 0001:000091f0       ??$getValue@_N@BaseWorker@LocalWorkflow@U2@@IBE_NABVQString@@@Z 1000a1f0 f i SamtoolMpileupWorker.obj
 0001:00009250       ??$qMapLessThanKey@VDescriptor@U2@@@@YA_NABVDescriptor@U2@@0@Z 1000a250 f i SamtoolMpileupWorker.obj
 0001:00009270       ??$qMetaTypeId@H@@YAHXZ    1000a270 f i SamtoolMpileupWorker.obj
 0001:00009280       ??$qMetaTypeId@M@@YAHXZ    1000a280 f i SamtoolMpileupWorker.obj
 0001:00009290       ??$qMetaTypeId@VQString@@@@YAHXZ 1000a290 f i SamtoolMpileupWorker.obj
 0001:000092a0       ??$qMetaTypeId@_N@@YAHXZ   1000a2a0 f i SamtoolMpileupWorker.obj
 0001:000092b0       ??$qSwap@PAVDataType@U2@@@@YAXAAPAVDataType@U2@@0@Z 1000a2b0 f i SamtoolMpileupWorker.obj
 0001:000092d0       ??$qobject_cast@PAVCallVariantsTask@LocalWorkflow@U2@@@@YAPAVCallVariantsTask@LocalWorkflow@U2@@PAVQObject@@@Z 1000a2d0 f i SamtoolMpileupWorker.obj
 0001:000092f0       ??$qobject_cast@PAVIntegralBusPort@Workflow@U2@@@@YAPAVIntegralBusPort@Workflow@U2@@PAVQObject@@@Z 1000a2f0 f i SamtoolMpileupWorker.obj
 0001:00009310       ??$qvariant_cast@H@@YAHABVQVariant@@@Z 1000a310 f i SamtoolMpileupWorker.obj
 0001:00009350       ??$qvariant_cast@M@@YAMABVQVariant@@@Z 1000a350 f i SamtoolMpileupWorker.obj
 0001:000093b0       ??$qvariant_cast@V?$QMap@VQString@@V1@@@@@YA?AV?$QMap@VQString@@V1@@@ABVQVariant@@@Z 1000a3b0 f i SamtoolMpileupWorker.obj
 0001:00009430       ??$qvariant_cast@VQString@@@@YA?AVQString@@ABVQVariant@@@Z 1000a430 f i SamtoolMpileupWorker.obj
 0001:00009450       ??$qvariant_cast@_N@@YA_NABVQVariant@@@Z 1000a450 f i SamtoolMpileupWorker.obj
 0001:00009490       ??$swap@PAVDataType@U2@@@std@@YAXAAPAVDataType@U2@@0@Z 1000a490 f i SamtoolMpileupWorker.obj
 0001:000094b0       ??$value@H@QVariant@@QBEHXZ 1000a4b0 f i SamtoolMpileupWorker.obj
 0001:000094f0       ??$value@M@QVariant@@QBEMXZ 1000a4f0 f i SamtoolMpileupWorker.obj
 0001:00009550       ??$value@V?$QMap@VQString@@V1@@@@QVariant@@QBE?AV?$QMap@VQString@@V1@@@XZ 1000a550 f i SamtoolMpileupWorker.obj
 0001:00009570       ??$value@VQString@@@QVariant@@QBE?AVQString@@XZ 1000a570 f i SamtoolMpileupWorker.obj
 0001:00009590       ??$value@_N@QVariant@@QBE_NXZ 1000a590 f i SamtoolMpileupWorker.obj
 0001:000095d0       ??0?$PrompterBase@VCallVariantsPrompter@LocalWorkflow@U2@@@U2@@QAE@PAVActor@Workflow@1@_N@Z 1000a5d0 f i SamtoolMpileupWorker.obj
 0001:00009600       ??0?$QExplicitlySharedDataPointer@VDataType@U2@@@@QAE@ABV0@@Z 1000a600 f i SamtoolMpileupWorker.obj
 0001:00009620       ??0?$QExplicitlySharedDataPointer@VDataType@U2@@@@QAE@PAVDataType@U2@@@Z 1000a620 f i SamtoolMpileupWorker.obj
 0001:00009640       ??0?$QExplicitlySharedDataPointer@VDataType@U2@@@@QAE@XZ 1000a640 f i SamtoolMpileupWorker.obj
 0001:00009650       ??0?$QForeachContainer@$$CBV?$QList@V?$QMap@VQString@@VQVariant@@@@@@@@QAE@ABV?$QList@V?$QMap@VQString@@VQVariant@@@@@@@Z 1000a650 f i SamtoolMpileupWorker.obj
 0001:00009690       ??0?$QForeachContainer@V?$QList@PAVPort@Workflow@U2@@@@@@QAE@ABV?$QList@PAVPort@Workflow@U2@@@@@Z 1000a690 f i SamtoolMpileupWorker.obj
 0001:000096d0       ??0?$QForeachContainer@V?$QList@VDescriptor@U2@@@@@@QAE@ABV?$QList@VDescriptor@U2@@@@@Z 1000a6d0 f i SamtoolMpileupWorker.obj
 0001:00009710       ??0?$QHash@VQString@@UQHashDummyValue@@@@QAE@XZ 1000a710 f i SamtoolMpileupWorker.obj
 0001:00009720       ??0?$QList@PAVAttribute@U2@@@@QAE@XZ 1000a720 f i SamtoolMpileupWorker.obj
 0001:00009730       ??0?$QList@PAVPort@Workflow@U2@@@@QAE@ABV0@@Z 1000a730 f i SamtoolMpileupWorker.obj
 0001:000097f0       ??0?$QList@PAVPortDescriptor@Workflow@U2@@@@QAE@XZ 1000a7f0 f i SamtoolMpileupWorker.obj
 0001:00009800       ??0?$QList@V?$QMap@VQString@@VQVariant@@@@@@QAE@ABV0@@Z 1000a800 f i SamtoolMpileupWorker.obj
 0001:000098c0       ??0?$QList@VDescriptor@U2@@@@QAE@$$QAV0@@Z 1000a8c0 f i SamtoolMpileupWorker.obj
 0001:000098e0       ??0?$QList@VDescriptor@U2@@@@QAE@ABV0@@Z 1000a8e0 f i SamtoolMpileupWorker.obj
 0001:000099a0       ??0?$QList@VDescriptor@U2@@@@QAE@XZ 1000a9a0 f i SamtoolMpileupWorker.obj
 0001:000099b0       ??0?$QList@VMessage@Workflow@U2@@@@QAE@XZ 1000a9b0 f i SamtoolMpileupWorker.obj
 0001:000099c0       ??0?$QList@VQVariant@@@@QAE@XZ 1000a9c0 f i SamtoolMpileupWorker.obj
 0001:000099d0       ??0?$QMap@VDescriptor@U2@@V?$QExplicitlySharedDataPointer@VDataType@U2@@@@@@QAE@XZ 1000a9d0 f i SamtoolMpileupWorker.obj
 0001:000099e0       ??0?$QMap@VQString@@PAVPropertyDelegate@U2@@@@QAE@XZ 1000a9e0 f i SamtoolMpileupWorker.obj
 0001:000099f0       ??0?$QMap@VQString@@V1@@@QAE@ABV0@@Z 1000a9f0 f i SamtoolMpileupWorker.obj
 0001:00009a60       ??0?$QMap@VQString@@VQScriptValue@@@@QAE@XZ 1000aa60 f i SamtoolMpileupWorker.obj
 0001:00009a70       ??0?$QMapIterator@VQString@@V1@@@QAE@ABV?$QMap@VQString@@V1@@@@Z 1000aa70 f i SamtoolMpileupWorker.obj
 0001:00009ab0       ??0?$QSet@VQString@@@@QAE@XZ 1000aab0 f i SamtoolMpileupWorker.obj
 0001:00009ac0       ??0CallVariantsPrompter@LocalWorkflow@U2@@QAE@PAVActor@Workflow@2@@Z 1000aac0 f i SamtoolMpileupWorker.obj
 0001:00009af0       ??0CallVariantsTaskSettings@LocalWorkflow@U2@@QAE@XZ 1000aaf0 f i SamtoolMpileupWorker.obj
 0001:00009bb0       ??0CallVariantsWorker@LocalWorkflow@U2@@QAE@PAVActor@Workflow@2@@Z 1000abb0 f   SamtoolMpileupWorker.obj
 0001:00009c70       ??0CallVariantsWorkerFactory@LocalWorkflow@U2@@QAE@XZ 1000ac70 f i SamtoolMpileupWorker.obj
 0001:00009c90       ??0EmptySlotValidator@LocalWorkflow@U2@@QAE@ABVQString@@@Z 1000ac90 f i SamtoolMpileupWorker.obj
 0001:00009cf0       ??0ScientificDoubleDelegate@LocalWorkflow@U2@@QAE@PAVQObject@@@Z 1000acf0 f   SamtoolMpileupWorker.obj
 0001:00009d10       ??0ScientificDoubleWidget@LocalWorkflow@U2@@QAE@PAVQWidget@@@Z 1000ad10 f   SamtoolMpileupWorker.obj
 0001:00009e20       ??0const_iterator@?$QList@PAVPort@Workflow@U2@@@@QAE@PAUNode@1@@Z 1000ae20 f i SamtoolMpileupWorker.obj
 0001:00009e30       ??0const_iterator@?$QList@V?$QMap@VQString@@VQVariant@@@@@@QAE@PAUNode@1@@Z 1000ae30 f i SamtoolMpileupWorker.obj
 0001:00009e40       ??0const_iterator@?$QList@VDescriptor@U2@@@@QAE@PAUNode@1@@Z 1000ae40 f i SamtoolMpileupWorker.obj
 0001:00009e50       ??0const_iterator@?$QMap@VDescriptor@U2@@VQVariant@@@@QAE@PBU?$QMapNode@VDescriptor@U2@@VQVariant@@@@@Z 1000ae50 f i SamtoolMpileupWorker.obj
 0001:00009e60       ??0const_iterator@?$QMap@VQString@@V1@@@QAE@PBU?$QMapNode@VQString@@V1@@@@Z 1000ae60 f i SamtoolMpileupWorker.obj
 0001:00009e70       ??0iterator@?$QList@VMessage@Workflow@U2@@@@QAE@PAUNode@1@@Z 1000ae70 f i SamtoolMpileupWorker.obj
 0001:00009e80       ??0iterator@?$QMap@VDescriptor@U2@@V?$QExplicitlySharedDataPointer@VDataType@U2@@@@@@QAE@PAU?$QMapNode@VDescriptor@U2@@V?$QExplicitlySharedDataPointer@VDataType@U2@@@@@@@Z 1000ae80 f i SamtoolMpileupWorker.obj
 0001:00009e90       ??0iterator@?$QMap@VQString@@PAVPropertyDelegate@U2@@@@QAE@PAU?$QMapNode@VQString@@PAVPropertyDelegate@U2@@@@@Z 1000ae90 f i SamtoolMpileupWorker.obj
 0001:00009ea0       ??0iterator@?$QMap@VQString@@VQScriptValue@@@@QAE@PAU?$QMapNode@VQString@@VQScriptValue@@@@@Z 1000aea0 f i SamtoolMpileupWorker.obj
 0001:00009eb0       ??1?$PrompterBase@VCallVariantsPrompter@LocalWorkflow@U2@@@U2@@UAE@XZ 1000aeb0 f i SamtoolMpileupWorker.obj
 0001:00009ec0       ??1?$QExplicitlySharedDataPointer@VDataType@U2@@@@QAE@XZ 1000aec0 f i SamtoolMpileupWorker.obj
 0001:00009ee0       ??1?$QForeachContainer@$$CBV?$QList@V?$QMap@VQString@@VQVariant@@@@@@@@QAE@XZ 1000aee0 f i SamtoolMpileupWorker.obj
 0001:00009f30       ??1?$QForeachContainer@V?$QList@PAVPort@Workflow@U2@@@@@@QAE@XZ 1000af30 f i SamtoolMpileupWorker.obj
 0001:00009f60       ??1?$QForeachContainer@V?$QList@VDescriptor@U2@@@@@@QAE@XZ 1000af60 f i SamtoolMpileupWorker.obj
 0001:00009f90       ??1?$QHash@VQString@@UQHashDummyValue@@@@QAE@XZ 1000af90 f i SamtoolMpileupWorker.obj
 0001:00009fc0       ??1?$QHashNode@VQString@@UQHashDummyValue@@@@QAE@XZ 1000afc0 f i SamtoolMpileupWorker.obj
 0001:00009fd0       ??1?$QList@PAVActor@Workflow@U2@@@@QAE@XZ 1000afd0 f i SamtoolMpileupWorker.obj
 0001:0000a000       ??1?$QList@PAVAttribute@U2@@@@QAE@XZ 1000b000 f i SamtoolMpileupWorker.obj
 0001:0000a030       ??1?$QList@PAVExternalToolListener@U2@@@@QAE@XZ 1000b030 f i SamtoolMpileupWorker.obj
 0001:0000a060       ??1?$QList@PAVPort@Workflow@U2@@@@QAE@XZ 1000b060 f i SamtoolMpileupWorker.obj
 0001:0000a090       ??1?$QList@PAVPortDescriptor@Workflow@U2@@@@QAE@XZ 1000b090 f i SamtoolMpileupWorker.obj
 0001:0000a0c0       ??1?$QList@VDescriptor@U2@@@@QAE@XZ 1000b0c0 f i SamtoolMpileupWorker.obj
 0001:0000a0f0       ??1?$QList@VMessage@Workflow@U2@@@@QAE@XZ 1000b0f0 f i SamtoolMpileupWorker.obj
 0001:0000a120       ??1?$QList@VQVariant@@@@QAE@XZ 1000b120 f i SamtoolMpileupWorker.obj
 0001:0000a150       ??1?$QMap@VDescriptor@U2@@V?$QExplicitlySharedDataPointer@VDataType@U2@@@@@@QAE@XZ 1000b150 f i SamtoolMpileupWorker.obj
 0001:0000a1a0       ??1?$QMap@VQString@@PAVPropertyDelegate@U2@@@@QAE@XZ 1000b1a0 f i SamtoolMpileupWorker.obj
 0001:0000a210       ??1?$QMap@VQString@@V1@@@QAE@XZ 1000b210 f i SamtoolMpileupWorker.obj
 0001:0000a260       ??1?$QMap@VQString@@VQScriptValue@@@@QAE@XZ 1000b260 f i SamtoolMpileupWorker.obj
 0001:0000a2b0       ??1?$QMapIterator@VQString@@V1@@@QAE@XZ 1000b2b0 f i SamtoolMpileupWorker.obj
 0001:0000a300       ??1?$QSet@VQString@@@@QAE@XZ 1000b300 f i SamtoolMpileupWorker.obj
 0001:0000a330       ??1CallVariantsPrompter@LocalWorkflow@U2@@UAE@XZ 1000b330 f i SamtoolMpileupWorker.obj
 0001:0000a340       ??1CallVariantsWorker@LocalWorkflow@U2@@UAE@XZ 1000b340 f i SamtoolMpileupWorker.obj
 0001:0000a3f0       ??1CallVariantsWorkerFactory@LocalWorkflow@U2@@UAE@XZ 1000b3f0 f i SamtoolMpileupWorker.obj
 0001:0000a400       ??1EmptySlotValidator@LocalWorkflow@U2@@UAE@XZ 1000b400 f i SamtoolMpileupWorker.obj
 0001:0000a450       ??1ScientificDoubleDelegate@LocalWorkflow@U2@@UAE@XZ 1000b450 f i SamtoolMpileupWorker.obj
 0001:0000a460       ??1ScientificDoubleWidget@LocalWorkflow@U2@@UAE@XZ 1000b460 f i SamtoolMpileupWorker.obj
 0001:0000a470       ??4?$QExplicitlySharedDataPointer@VDataType@U2@@@@QAEAAV0@$$QAV0@@Z 1000b470 f i SamtoolMpileupWorker.obj
 0001:0000a490       ??4?$QExplicitlySharedDataPointer@VDataType@U2@@@@QAEAAV0@ABV0@@Z 1000b490 f i SamtoolMpileupWorker.obj
 0001:0000a4e0       ??4?$QList@V?$QMap@VQString@@VQVariant@@@@@@QAEAAV0@$$QAV0@@Z 1000b4e0 f i SamtoolMpileupWorker.obj
 0001:0000a500       ??4?$QList@VQString@@@@QAEAAV0@$$QAV0@@Z 1000b500 f i SamtoolMpileupWorker.obj
 0001:0000a520       ??4CallVariantsTaskSettings@LocalWorkflow@U2@@QAEAAV012@ABV012@@Z 1000b520 f i SamtoolMpileupWorker.obj
 0001:0000a6f0       ??6?$QList@PAVAttribute@U2@@@@QAEAAV0@ABQAVAttribute@U2@@@Z 1000b6f0 f i SamtoolMpileupWorker.obj
 0001:0000a710       ??6?$QList@PAVPortDescriptor@Workflow@U2@@@@QAEAAV0@ABQAVPortDescriptor@Workflow@U2@@@Z 1000b710 f i SamtoolMpileupWorker.obj
 0001:0000a730       ??6?$QList@VQString@@@@QAEAAV0@ABVQString@@@Z 1000b730 f i SamtoolMpileupWorker.obj
 0001:0000a750       ??6?$QList@VQVariant@@@@QAEAAV0@ABVQVariant@@@Z 1000b750 f i SamtoolMpileupWorker.obj
 0001:0000a770       ??8const_iterator@?$QMap@VDescriptor@U2@@VQVariant@@@@QBE_NABV01@@Z 1000b770 f i SamtoolMpileupWorker.obj
 0001:0000a790       ??9@YA_NABVQString@@0@Z    1000b790 f i SamtoolMpileupWorker.obj
 0001:0000a7b0       ??9const_iterator@?$QList@PAVPort@Workflow@U2@@@@QBE_NABV01@@Z 1000b7b0 f i SamtoolMpileupWorker.obj
 0001:0000a7d0       ??9const_iterator@?$QList@V?$QMap@VQString@@VQVariant@@@@@@QBE_NABV01@@Z 1000b7d0 f i SamtoolMpileupWorker.obj
 0001:0000a7f0       ??9const_iterator@?$QList@VDescriptor@U2@@@@QBE_NABV01@@Z 1000b7f0 f i SamtoolMpileupWorker.obj
 0001:0000a810       ??9const_iterator@?$QMap@VDescriptor@U2@@VQVariant@@@@QBE_NABV01@@Z 1000b810 f i SamtoolMpileupWorker.obj
 0001:0000a830       ??9const_iterator@?$QMap@VQString@@V1@@@QBE_NABV01@@Z 1000b830 f i SamtoolMpileupWorker.obj
 0001:0000a850       ??A?$QMap@VDescriptor@U2@@V?$QExplicitlySharedDataPointer@VDataType@U2@@@@@@QAEAAV?$QExplicitlySharedDataPointer@VDataType@U2@@@@ABVDescriptor@U2@@@Z 1000b850 f i SamtoolMpileupWorker.obj
 0001:0000a910       ??A?$QMap@VQString@@PAVPropertyDelegate@U2@@@@QAEAAPAVPropertyDelegate@U2@@ABVQString@@@Z 1000b910 f i SamtoolMpileupWorker.obj
 0001:0000a990       ??A?$QMap@VQString@@VQScriptValue@@@@QAEAAVQScriptValue@@ABVQString@@@Z 1000b990 f i SamtoolMpileupWorker.obj
 0001:0000aa60       ??C?$QExplicitlySharedDataPointer@VDataType@U2@@@@QAEPAVDataType@U2@@XZ 1000ba60 f i SamtoolMpileupWorker.obj
 0001:0000aa70       ??Dconst_iterator@?$QList@PAVPort@Workflow@U2@@@@QBEABQAVPort@Workflow@U2@@XZ 1000ba70 f i SamtoolMpileupWorker.obj
 0001:0000aa80       ??Dconst_iterator@?$QList@V?$QMap@VQString@@VQVariant@@@@@@QBEABV?$QMap@VQString@@VQVariant@@@@XZ 1000ba80 f i SamtoolMpileupWorker.obj
 0001:0000aa90       ??Dconst_iterator@?$QList@VDescriptor@U2@@@@QBEABVDescriptor@U2@@XZ 1000ba90 f i SamtoolMpileupWorker.obj
 0001:0000aaa0       ??Dconst_iterator@?$QMap@VQString@@V1@@@QBEABVQString@@XZ 1000baa0 f i SamtoolMpileupWorker.obj
 0001:0000aab0       ??Diterator@?$QList@VMessage@Workflow@U2@@@@QBEAAVMessage@Workflow@U2@@XZ 1000bab0 f i SamtoolMpileupWorker.obj
 0001:0000aac0       ??Diterator@?$QMap@VDescriptor@U2@@V?$QExplicitlySharedDataPointer@VDataType@U2@@@@@@QBEAAV?$QExplicitlySharedDataPointer@VDataType@U2@@@@XZ 1000bac0 f i SamtoolMpileupWorker.obj
 0001:0000aad0       ??Diterator@?$QMap@VQString@@PAVPropertyDelegate@U2@@@@QBEAAPAVPropertyDelegate@U2@@XZ 1000bad0 f i SamtoolMpileupWorker.obj
 0001:0000aae0       ??Diterator@?$QMap@VQString@@VQScriptValue@@@@QBEAAVQScriptValue@@XZ 1000bae0 f i SamtoolMpileupWorker.obj
 0001:0000aaf0       ??Econst_iterator@?$QList@PAVPort@Workflow@U2@@@@QAEAAV01@XZ 1000baf0 f i SamtoolMpileupWorker.obj
 0001:0000ab00       ??Econst_iterator@?$QList@V?$QMap@VQString@@VQVariant@@@@@@QAEAAV01@XZ 1000bb00 f i SamtoolMpileupWorker.obj
 0001:0000ab10       ??Econst_iterator@?$QList@VDescriptor@U2@@@@QAEAAV01@XZ 1000bb10 f i SamtoolMpileupWorker.obj
 0001:0000ab20       ??Econst_iterator@?$QMap@VDescriptor@U2@@VQVariant@@@@QAEAAV01@XZ 1000bb20 f i SamtoolMpileupWorker.obj
 0001:0000ab40       ??Econst_iterator@?$QMap@VQString@@V1@@@QAE?AV01@H@Z 1000bb40 f i SamtoolMpileupWorker.obj
 0001:0000ab60       ??H@YA?BVQString@@ABV0@PBD@Z 1000bb60 f i SamtoolMpileupWorker.obj
 0001:0000ac00       ??H@YA?BVQString@@PBDABV0@@Z 1000bc00 f i SamtoolMpileupWorker.obj
 0001:0000ac70       ??Yiterator@?$QList@VMessage@Workflow@U2@@@@QAEAAV01@H@Z 1000bc70 f i SamtoolMpileupWorker.obj
 0001:0000ac81       ??_E?$PrompterBase@VCallVariantsPrompter@LocalWorkflow@U2@@@U2@@WM@AEPAXI@Z 1000bc81 f i SamtoolMpileupWorker.obj
 0001:0000ac89       ??_ECallVariantsPrompter@LocalWorkflow@U2@@WM@AEPAXI@Z 1000bc89 f i SamtoolMpileupWorker.obj
 0001:0000ac91       ??_ECallVariantsWorker@LocalWorkflow@U2@@W7AEPAXI@Z 1000bc91 f i SamtoolMpileupWorker.obj
 0001:0000ac99       ??_ECallVariantsWorker@LocalWorkflow@U2@@WBA@AEPAXI@Z 1000bc99 f i SamtoolMpileupWorker.obj
 0001:0000aca1       ??_ECallVariantsWorkerFactory@LocalWorkflow@U2@@W7AEPAXI@Z 1000bca1 f i SamtoolMpileupWorker.obj
 0001:0000aca9       ??_EIntegralBusActorPrototype@Workflow@U2@@W7AEPAXI@Z 1000bca9 f i SamtoolMpileupWorker.obj
 0001:0000acb1       ??_EQLineEdit@@W7AEPAXI@Z  1000bcb1 f i SamtoolMpileupWorker.obj
 0001:0000acb9       ??_EScientificDoubleWidget@LocalWorkflow@U2@@W7AEPAXI@Z 1000bcb9 f i SamtoolMpileupWorker.obj
 0001:0000acd0       ??_G?$PrompterBase@VCallVariantsPrompter@LocalWorkflow@U2@@@U2@@UAEPAXI@Z 1000bcd0 f i SamtoolMpileupWorker.obj
 0001:0000acd0       ??_E?$PrompterBase@VCallVariantsPrompter@LocalWorkflow@U2@@@U2@@UAEPAXI@Z 1000bcd0 f i SamtoolMpileupWorker.obj
 0001:0000ad00       ??_G?$QExplicitlySharedDataPointer@VDataType@U2@@@@QAEPAXI@Z 1000bd00 f i SamtoolMpileupWorker.obj
 0001:0000ad40       ??_G?$QHashNode@VQString@@UQHashDummyValue@@@@QAEPAXI@Z 1000bd40 f i SamtoolMpileupWorker.obj
 0001:0000ad70       ??_GAttribute@U2@@UAEPAXI@Z 1000bd70 f i SamtoolMpileupWorker.obj
 0001:0000ad70       ??_EAttribute@U2@@UAEPAXI@Z 1000bd70 f i SamtoolMpileupWorker.obj
 0001:0000ada0       ??_ECallVariantsPrompter@LocalWorkflow@U2@@UAEPAXI@Z 1000bda0 f i SamtoolMpileupWorker.obj
 0001:0000ada0       ??_GCallVariantsPrompter@LocalWorkflow@U2@@UAEPAXI@Z 1000bda0 f i SamtoolMpileupWorker.obj
 0001:0000add0       ??_ECallVariantsWorker@LocalWorkflow@U2@@UAEPAXI@Z 1000bdd0 f i SamtoolMpileupWorker.obj
 0001:0000add0       ??_GCallVariantsWorker@LocalWorkflow@U2@@UAEPAXI@Z 1000bdd0 f i SamtoolMpileupWorker.obj
 0001:0000ae00       ??_ECallVariantsWorkerFactory@LocalWorkflow@U2@@UAEPAXI@Z 1000be00 f i SamtoolMpileupWorker.obj
 0001:0000ae00       ??_GCallVariantsWorkerFactory@LocalWorkflow@U2@@UAEPAXI@Z 1000be00 f i SamtoolMpileupWorker.obj
 0001:0000ae30       ??_GComboBoxDelegate@U2@@UAEPAXI@Z 1000be30 f i SamtoolMpileupWorker.obj
 0001:0000ae30       ??_EComboBoxDelegate@U2@@UAEPAXI@Z 1000be30 f i SamtoolMpileupWorker.obj
 0001:0000ae60       ??_GDelegateEditor@U2@@UAEPAXI@Z 1000be60 f i SamtoolMpileupWorker.obj
 0001:0000ae60       ??_EDelegateEditor@U2@@UAEPAXI@Z 1000be60 f i SamtoolMpileupWorker.obj
 0001:0000ae90       ??_GDescriptor@U2@@UAEPAXI@Z 1000be90 f i SamtoolMpileupWorker.obj
 0001:0000ae90       ??_EDescriptor@U2@@UAEPAXI@Z 1000be90 f i SamtoolMpileupWorker.obj
 0001:0000aec0       ??_EDoubleSpinBoxDelegate@U2@@UAEPAXI@Z 1000bec0 f i SamtoolMpileupWorker.obj
 0001:0000aec0       ??_GDoubleSpinBoxDelegate@U2@@UAEPAXI@Z 1000bec0 f i SamtoolMpileupWorker.obj
 0001:0000aef0       ??_EEmptySlotValidator@LocalWorkflow@U2@@UAEPAXI@Z 1000bef0 f i SamtoolMpileupWorker.obj
 0001:0000aef0       ??_GEmptySlotValidator@LocalWorkflow@U2@@UAEPAXI@Z 1000bef0 f i SamtoolMpileupWorker.obj
 0001:0000af60       ??_EIntegralBusActorPrototype@Workflow@U2@@UAEPAXI@Z 1000bf60 f i SamtoolMpileupWorker.obj
 0001:0000af60       ??_GIntegralBusActorPrototype@Workflow@U2@@UAEPAXI@Z 1000bf60 f i SamtoolMpileupWorker.obj
 0001:0000af90       ??_GMapDataType@U2@@UAEPAXI@Z 1000bf90 f i SamtoolMpileupWorker.obj
 0001:0000af90       ??_EMapDataType@U2@@UAEPAXI@Z 1000bf90 f i SamtoolMpileupWorker.obj
 0001:0000afc0       ??_GMessage@Workflow@U2@@QAEPAXI@Z 1000bfc0 f i SamtoolMpileupWorker.obj
 0001:0000aff0       ??_GPortDescriptor@Workflow@U2@@UAEPAXI@Z 1000bff0 f i SamtoolMpileupWorker.obj
 0001:0000aff0       ??_EPortDescriptor@Workflow@U2@@UAEPAXI@Z 1000bff0 f i SamtoolMpileupWorker.obj
 0001:0000b020       ??_EPortRelationDescriptor@U2@@UAEPAXI@Z 1000c020 f i SamtoolMpileupWorker.obj
 0001:0000b020       ??_GPortRelationDescriptor@U2@@UAEPAXI@Z 1000c020 f i SamtoolMpileupWorker.obj
 0001:0000b050       ??_EQDoubleValidator@@UAEPAXI@Z 1000c050 f i SamtoolMpileupWorker.obj
 0001:0000b050       ??_GQDoubleValidator@@UAEPAXI@Z 1000c050 f i SamtoolMpileupWorker.obj
 0001:0000b080       ??_EQLineEdit@@UAEPAXI@Z   1000c080 f i SamtoolMpileupWorker.obj
 0001:0000b080       ??_GQLineEdit@@UAEPAXI@Z   1000c080 f i SamtoolMpileupWorker.obj
 0001:0000b0b0       ??_GQScriptValue@@QAEPAXI@Z 1000c0b0 f i SamtoolMpileupWorker.obj
 0001:0000b0e0       ??_EScientificDoubleDelegate@LocalWorkflow@U2@@UAEPAXI@Z 1000c0e0 f i SamtoolMpileupWorker.obj
 0001:0000b0e0       ??_GScientificDoubleDelegate@LocalWorkflow@U2@@UAEPAXI@Z 1000c0e0 f i SamtoolMpileupWorker.obj
 0001:0000b110       ??_GScientificDoubleWidget@LocalWorkflow@U2@@UAEPAXI@Z 1000c110 f i SamtoolMpileupWorker.obj
 0001:0000b110       ??_EScientificDoubleWidget@LocalWorkflow@U2@@UAEPAXI@Z 1000c110 f i SamtoolMpileupWorker.obj
 0001:0000b140       ??_ESpinBoxDelegate@U2@@UAEPAXI@Z 1000c140 f i SamtoolMpileupWorker.obj
 0001:0000b140       ??_GSpinBoxDelegate@U2@@UAEPAXI@Z 1000c140 f i SamtoolMpileupWorker.obj
 0001:0000b170       ??_EURLDelegate@U2@@UAEPAXI@Z 1000c170 f i SamtoolMpileupWorker.obj
 0001:0000b170       ??_GURLDelegate@U2@@UAEPAXI@Z 1000c170 f i SamtoolMpileupWorker.obj
 0001:0000b1a0       ??_GVisibilityRelation@U2@@UAEPAXI@Z 1000c1a0 f i SamtoolMpileupWorker.obj
 0001:0000b1a0       ??_EVisibilityRelation@U2@@UAEPAXI@Z 1000c1a0 f i SamtoolMpileupWorker.obj
 0001:0000b1d0       ??_GWorkflowNotification@U2@@QAEPAXI@Z 1000c1d0 f i SamtoolMpileupWorker.obj
 0001:0000b200       ?append@?$QList@PAVAttribute@U2@@@@QAEXABQAVAttribute@U2@@@Z 1000c200 f i SamtoolMpileupWorker.obj
 0001:0000b290       ?append@?$QList@PAVPortDescriptor@Workflow@U2@@@@QAEXABQAVPortDescriptor@Workflow@U2@@@Z 1000c290 f i SamtoolMpileupWorker.obj
 0001:0000b320       ?append@?$QList@VDescriptor@U2@@@@QAEXABVDescriptor@U2@@@Z 1000c320 f i SamtoolMpileupWorker.obj
 0001:0000b410       ?append@?$QList@VMessage@Workflow@U2@@@@QAEXABVMessage@Workflow@U2@@@Z 1000c410 f i SamtoolMpileupWorker.obj
 0001:0000b4f0       ?append@?$QList@VQVariant@@@@QAEXABVQVariant@@@Z 1000c4f0 f i SamtoolMpileupWorker.obj
 0001:0000b5d0       ?append@?$QList@VWorkflowNotification@U2@@@@QAEXABVWorkflowNotification@U2@@@Z 1000c5d0 f i SamtoolMpileupWorker.obj
 0001:0000b6b0       ?begin@?$QList@PAVPort@Workflow@U2@@@@QBE?AVconst_iterator@1@XZ 1000c6b0 f i SamtoolMpileupWorker.obj
 0001:0000b6d0       ?begin@?$QList@V?$QMap@VQString@@VQVariant@@@@@@QBE?AVconst_iterator@1@XZ 1000c6d0 f i SamtoolMpileupWorker.obj
 0001:0000b6f0       ?begin@?$QList@VDescriptor@U2@@@@QBE?AVconst_iterator@1@XZ 1000c6f0 f i SamtoolMpileupWorker.obj
 0001:0000b710       ?begin@?$QList@VMessage@Workflow@U2@@@@QAE?AViterator@1@XZ 1000c710 f i SamtoolMpileupWorker.obj
 0001:0000b750       ?begin@?$QMap@VDescriptor@U2@@VQVariant@@@@QBE?AVconst_iterator@1@XZ 1000c750 f i SamtoolMpileupWorker.obj
 0001:0000b770       ?begin@?$QMapData@VDescriptor@U2@@VQVariant@@@@QAEPAU?$QMapNode@VDescriptor@U2@@VQVariant@@@@XZ 1000c770 f i SamtoolMpileupWorker.obj
 0001:0000b780       ?begin@?$QMapData@VQString@@V1@@@QAEPAU?$QMapNode@VQString@@V1@@@XZ 1000c780 f i SamtoolMpileupWorker.obj
 0001:0000b790       ?checkState@CallVariantsWorker@LocalWorkflow@U2@@AAEXAAVU2OpStatus@3@@Z 1000c790 f   SamtoolMpileupWorker.obj
 0001:0000b9e0       ?cleanup@CallVariantsWorker@LocalWorkflow@U2@@UAEXXZ 1000c9e0 f   SamtoolMpileupWorker.obj
 0001:0000b9f0       ?clear@?$QList@V?$QMap@VQString@@VQVariant@@@@@@QAEXXZ 1000c9f0 f i SamtoolMpileupWorker.obj
 0001:0000ba50       ?clear@?$QList@VQString@@@@QAEXXZ 1000ca50 f i SamtoolMpileupWorker.obj
 0001:0000ba70       ?clearResults@CallVariantsTask@LocalWorkflow@U2@@QAEXXZ 1000ca70 f i SamtoolMpileupWorker.obj
 0001:0000bad0       ?clone@ScientificDoubleDelegate@LocalWorkflow@U2@@UAEPAVPropertyDelegate@3@XZ 1000cad0 f   SamtoolMpileupWorker.obj
 0001:0000bb50       ?composeRichDoc@CallVariantsPrompter@LocalWorkflow@U2@@MAE?AVQString@@XZ 1000cb50 f   SamtoolMpileupWorker.obj
 0001:0000bfe0       ?concrete@?$QHash@VQString@@UQHashDummyValue@@@@CAPAU?$QHashNode@VQString@@UQHashDummyValue@@@@PAUNode@QHashData@@@Z 1000cfe0 f i SamtoolMpileupWorker.obj
 0001:0000bff0       ?constBegin@?$QMap@VQString@@V1@@@QBE?AVconst_iterator@1@XZ 1000cff0 f i SamtoolMpileupWorker.obj
 0001:0000c010       ?constEnd@?$QMap@VQString@@V1@@@QBE?AVconst_iterator@1@XZ 1000d010 f i SamtoolMpileupWorker.obj
 0001:0000c030       ?contains@?$QMap@VQString@@VQVariant@@@@QBE_NABVQString@@@Z 1000d030 f i SamtoolMpileupWorker.obj
 0001:0000c070       ?copy@?$QMapNode@VDescriptor@U2@@V?$QExplicitlySharedDataPointer@VDataType@U2@@@@@@QBEPAU1@PAU?$QMapData@VDescriptor@U2@@V?$QExplicitlySharedDataPointer@VDataType@U2@@@@@@@Z 1000d070 f i SamtoolMpileupWorker.obj
 0001:0000c100       ?copy@?$QMapNode@VQString@@PAVPropertyDelegate@U2@@@@QBEPAU1@PAU?$QMapData@VQString@@PAVPropertyDelegate@U2@@@@@Z 1000d100 f i SamtoolMpileupWorker.obj
 0001:0000c190       ?copy@?$QMapNode@VQString@@V1@@@QBEPAU1@PAU?$QMapData@VQString@@V1@@@@Z 1000d190 f i SamtoolMpileupWorker.obj
 0001:0000c220       ?copy@?$QMapNode@VQString@@VQScriptValue@@@@QBEPAU1@PAU?$QMapData@VQString@@VQScriptValue@@@@@Z 1000d220 f i SamtoolMpileupWorker.obj
 0001:0000c2b0       ?create@?$QMapData@VDescriptor@U2@@V?$QExplicitlySharedDataPointer@VDataType@U2@@@@@@SAPAU1@XZ 1000d2b0 f i SamtoolMpileupWorker.obj
 0001:0000c2c0       ?create@?$QMapData@VQString@@PAVPropertyDelegate@U2@@@@SAPAU1@XZ 1000d2c0 f i SamtoolMpileupWorker.obj
 0001:0000c2d0       ?create@?$QMapData@VQString@@V1@@@SAPAU1@XZ 1000d2d0 f i SamtoolMpileupWorker.obj
 0001:0000c2e0       ?create@?$QMapData@VQString@@VQScriptValue@@@@SAPAU1@XZ 1000d2e0 f i SamtoolMpileupWorker.obj
 0001:0000c2f0       ?createDescription@?$PrompterBase@VCallVariantsPrompter@LocalWorkflow@U2@@@U2@@UAEPAVActorDocument@Workflow@2@PAVActor@42@@Z 1000d2f0 f i SamtoolMpileupWorker.obj
 0001:0000c590       ?createEditor@ScientificDoubleDelegate@LocalWorkflow@U2@@UBEPAVQWidget@@PAV4@ABVQStyleOptionViewItem@@ABVQModelIndex@@@Z 1000d590 f   SamtoolMpileupWorker.obj
 0001:0000c600       ?createNode@?$QMapData@VDescriptor@U2@@V?$QExplicitlySharedDataPointer@VDataType@U2@@@@@@QAEPAU?$QMapNode@VDescriptor@U2@@V?$QExplicitlySharedDataPointer@VDataType@U2@@@@@@ABVDescriptor@U2@@ABV?$QExplicitlySharedDataPointer@VDataType@U2@@@@PAU2@_N@Z 1000d600 f i SamtoolMpileupWorker.obj
 0001:0000c6c0       ?createNode@?$QMapData@VQString@@PAVPropertyDelegate@U2@@@@QAEPAU?$QMapNode@VQString@@PAVPropertyDelegate@U2@@@@ABVQString@@ABQAVPropertyDelegate@U2@@PAU2@_N@Z 1000d6c0 f i SamtoolMpileupWorker.obj
 0001:0000c760       ?createNode@?$QMapData@VQString@@V1@@@QAEPAU?$QMapNode@VQString@@V1@@@ABVQString@@0PAU2@_N@Z 1000d760 f i SamtoolMpileupWorker.obj
 0001:0000c820       ?createNode@?$QMapData@VQString@@VQScriptValue@@@@QAEPAU?$QMapNode@VQString@@VQScriptValue@@@@ABVQString@@ABVQScriptValue@@PAU2@_N@Z 1000d820 f i SamtoolMpileupWorker.obj
 0001:0000c8e0       ?createWizardWidget@ScientificDoubleDelegate@LocalWorkflow@U2@@UBEPAVPropertyWidget@3@AAVU2OpStatus@3@PAVQWidget@@@Z 1000d8e0 f   SamtoolMpileupWorker.obj
 0001:0000c950       ?createWorker@CallVariantsWorkerFactory@LocalWorkflow@U2@@UAEPAVWorker@Workflow@3@PAVActor@53@@Z 1000d950 f i SamtoolMpileupWorker.obj
 0001:0000c9d0       ?dealloc@?$QList@PAVActor@Workflow@U2@@@@AAEXPAUData@QListData@@@Z 1000d9d0 f i SamtoolMpileupWorker.obj
 0001:0000c9f0       ?dealloc@?$QList@PAVAttribute@U2@@@@AAEXPAUData@QListData@@@Z 1000d9f0 f i SamtoolMpileupWorker.obj
 0001:0000ca10       ?dealloc@?$QList@PAVExternalToolListener@U2@@@@AAEXPAUData@QListData@@@Z 1000da10 f i SamtoolMpileupWorker.obj
 0001:0000ca30       ?dealloc@?$QList@PAVPort@Workflow@U2@@@@AAEXPAUData@QListData@@@Z 1000da30 f i SamtoolMpileupWorker.obj
 0001:0000ca50       ?dealloc@?$QList@PAVPortDescriptor@Workflow@U2@@@@AAEXPAUData@QListData@@@Z 1000da50 f i SamtoolMpileupWorker.obj
 0001:0000ca70       ?dealloc@?$QList@VDescriptor@U2@@@@AAEXPAUData@QListData@@@Z 1000da70 f i SamtoolMpileupWorker.obj
 0001:0000cac0       ?dealloc@?$QList@VMessage@Workflow@U2@@@@AAEXPAUData@QListData@@@Z 1000dac0 f i SamtoolMpileupWorker.obj
 0001:0000cb20       ?dealloc@?$QList@VQVariant@@@@AAEXPAUData@QListData@@@Z 1000db20 f i SamtoolMpileupWorker.obj
 0001:0000cb80       ?dealloc@?$QList@VWorkflowNotification@U2@@@@AAEXPAUData@QListData@@@Z 1000db80 f i SamtoolMpileupWorker.obj
 0001:0000cbe0       ?deleteNode2@?$QHash@VQString@@UQHashDummyValue@@@@CAXPAUNode@QHashData@@@Z 1000dbe0 f i SamtoolMpileupWorker.obj
 0001:0000cbf0       ?destroy@?$QMapData@VDescriptor@U2@@V?$QExplicitlySharedDataPointer@VDataType@U2@@@@@@QAEXXZ 1000dbf0 f i SamtoolMpileupWorker.obj
 0001:0000cc20       ?destroy@?$QMapData@VQString@@PAVPropertyDelegate@U2@@@@QAEXXZ 1000dc20 f i SamtoolMpileupWorker.obj
 0001:0000cc70       ?destroy@?$QMapData@VQString@@V1@@@QAEXXZ 1000dc70 f i SamtoolMpileupWorker.obj
 0001:0000cca0       ?destroy@?$QMapData@VQString@@VQScriptValue@@@@QAEXXZ 1000dca0 f i SamtoolMpileupWorker.obj
 0001:0000ccd0       ?destroySubTree@?$QMapNode@VDescriptor@U2@@V?$QExplicitlySharedDataPointer@VDataType@U2@@@@@@QAEXXZ 1000dcd0 f i SamtoolMpileupWorker.obj
 0001:0000cd20       ?destroySubTree@?$QMapNode@VQString@@PAVPropertyDelegate@U2@@@@QAEXXZ 1000dd20 f i SamtoolMpileupWorker.obj
 0001:0000cd50       ?destroySubTree@?$QMapNode@VQString@@V1@@@QAEXXZ 1000dd50 f i SamtoolMpileupWorker.obj
 0001:0000cd80       ?destroySubTree@?$QMapNode@VQString@@VQScriptValue@@@@QAEXXZ 1000dd80 f i SamtoolMpileupWorker.obj
 0001:0000cdc0       ?detach@?$QList@VMessage@Workflow@U2@@@@QAEXXZ 1000ddc0 f i SamtoolMpileupWorker.obj
 0001:0000cde0       ?detach@?$QMap@VDescriptor@U2@@V?$QExplicitlySharedDataPointer@VDataType@U2@@@@@@QAEXXZ 1000dde0 f i SamtoolMpileupWorker.obj
 0001:0000ce00       ?detach@?$QMap@VQString@@PAVPropertyDelegate@U2@@@@QAEXXZ 1000de00 f i SamtoolMpileupWorker.obj
 0001:0000ce20       ?detach@?$QMap@VQString@@VQScriptValue@@@@QAEXXZ 1000de20 f i SamtoolMpileupWorker.obj
 0001:0000ce40       ?detach_helper@?$QList@VDescriptor@U2@@@@AAEXH@Z 1000de40 f i SamtoolMpileupWorker.obj
 0001:0000cf10       ?detach_helper@?$QList@VMessage@Workflow@U2@@@@AAEXH@Z 1000df10 f i SamtoolMpileupWorker.obj
 0001:0000cfe0       ?detach_helper@?$QList@VMessage@Workflow@U2@@@@AAEXXZ 1000dfe0 f i SamtoolMpileupWorker.obj
 0001:0000cff0       ?detach_helper@?$QMap@VDescriptor@U2@@V?$QExplicitlySharedDataPointer@VDataType@U2@@@@@@AAEXXZ 1000dff0 f i SamtoolMpileupWorker.obj
 0001:0000d070       ?detach_helper@?$QMap@VQString@@PAVPropertyDelegate@U2@@@@AAEXXZ 1000e070 f i SamtoolMpileupWorker.obj
 0001:0000d120       ?detach_helper@?$QMap@VQString@@VQScriptValue@@@@AAEXXZ 1000e120 f i SamtoolMpileupWorker.obj
 0001:0000d1a0       ?detach_helper_grow@?$QList@PAVAttribute@U2@@@@AAEPAUNode@1@HH@Z 1000e1a0 f i SamtoolMpileupWorker.obj
 0001:0000d2b0       ?detach_helper_grow@?$QList@PAVPortDescriptor@Workflow@U2@@@@AAEPAUNode@1@HH@Z 1000e2b0 f i SamtoolMpileupWorker.obj
 0001:0000d3c0       ?detach_helper_grow@?$QList@VDescriptor@U2@@@@AAEPAUNode@1@HH@Z 1000e3c0 f i SamtoolMpileupWorker.obj
 0001:0000d510       ?detach_helper_grow@?$QList@VMessage@Workflow@U2@@@@AAEPAUNode@1@HH@Z 1000e510 f i SamtoolMpileupWorker.obj
 0001:0000d660       ?detach_helper_grow@?$QList@VQVariant@@@@AAEPAUNode@1@HH@Z 1000e660 f i SamtoolMpileupWorker.obj
 0001:0000d7b0       ?detach_helper_grow@?$QList@VWorkflowNotification@U2@@@@AAEPAUNode@1@HH@Z 1000e7b0 f i SamtoolMpileupWorker.obj
 0001:0000d900       ?end@?$QList@PAVPort@Workflow@U2@@@@QBE?AVconst_iterator@1@XZ 1000e900 f i SamtoolMpileupWorker.obj
 0001:0000d920       ?end@?$QList@V?$QMap@VQString@@VQVariant@@@@@@QBE?AVconst_iterator@1@XZ 1000e920 f i SamtoolMpileupWorker.obj
 0001:0000d940       ?end@?$QList@VDescriptor@U2@@@@QBE?AVconst_iterator@1@XZ 1000e940 f i SamtoolMpileupWorker.obj
 0001:0000d960       ?end@?$QMap@VDescriptor@U2@@VQVariant@@@@QBE?AVconst_iterator@1@XZ 1000e960 f i SamtoolMpileupWorker.obj
 0001:0000d980       ?end@?$QMapData@VDescriptor@U2@@V?$QExplicitlySharedDataPointer@VDataType@U2@@@@@@QAEPAU?$QMapNode@VDescriptor@U2@@V?$QExplicitlySharedDataPointer@VDataType@U2@@@@@@XZ 1000e980 f i SamtoolMpileupWorker.obj
 0001:0000d990       ?end@?$QMapData@VDescriptor@U2@@VQVariant@@@@QAEPAU?$QMapNode@VDescriptor@U2@@VQVariant@@@@XZ 1000e990 f i SamtoolMpileupWorker.obj
 0001:0000d9a0       ?end@?$QMapData@VQString@@PAVPropertyDelegate@U2@@@@QAEPAU?$QMapNode@VQString@@PAVPropertyDelegate@U2@@@@XZ 1000e9a0 f i SamtoolMpileupWorker.obj
 0001:0000d9b0       ?end@?$QMapData@VQString@@V1@@@QAEPAU?$QMapNode@VQString@@V1@@@XZ 1000e9b0 f i SamtoolMpileupWorker.obj
 0001:0000d9c0       ?end@?$QMapData@VQString@@VQScriptValue@@@@QAEPAU?$QMapNode@VQString@@VQScriptValue@@@@XZ 1000e9c0 f i SamtoolMpileupWorker.obj
 0001:0000d9d0       ?erase@?$QList@VMessage@Workflow@U2@@@@QAE?AViterator@1@V21@@Z 1000e9d0 f i SamtoolMpileupWorker.obj
 0001:0000da50       ?findNode@?$QMapData@VDescriptor@U2@@V?$QExplicitlySharedDataPointer@VDataType@U2@@@@@@QBEPAU?$QMapNode@VDescriptor@U2@@V?$QExplicitlySharedDataPointer@VDataType@U2@@@@@@ABVDescriptor@U2@@@Z 1000ea50 f i SamtoolMpileupWorker.obj
 0001:0000da90       ?findNode@?$QMapData@VDescriptor@U2@@VQVariant@@@@QBEPAU?$QMapNode@VDescriptor@U2@@VQVariant@@@@ABVDescriptor@U2@@@Z 1000ea90 f i SamtoolMpileupWorker.obj
 0001:0000dad0       ?findNode@?$QMapData@VQString@@PAVIntegralBus@Workflow@U2@@@@QBEPAU?$QMapNode@VQString@@PAVIntegralBus@Workflow@U2@@@@ABVQString@@@Z 1000ead0 f i SamtoolMpileupWorker.obj
 0001:0000db10       ?findNode@?$QMapData@VQString@@PAVPropertyDelegate@U2@@@@QBEPAU?$QMapNode@VQString@@PAVPropertyDelegate@U2@@@@ABVQString@@@Z 1000eb10 f i SamtoolMpileupWorker.obj
 0001:0000db50       ?findNode@?$QMapData@VQString@@VQScriptValue@@@@QBEPAU?$QMapNode@VQString@@VQScriptValue@@@@ABVQString@@@Z 1000eb50 f i SamtoolMpileupWorker.obj
 0001:0000db90       ?first@?$QList@VMessage@Workflow@U2@@@@QAEAAVMessage@Workflow@U2@@XZ 1000eb90 f i SamtoolMpileupWorker.obj
 0001:0000dbc0       ?freeData@?$QHash@VQString@@UQHashDummyValue@@@@AAEXPAUQHashData@@@Z 1000ebc0 f i SamtoolMpileupWorker.obj
 0001:0000dbe0       ?getDisplayValue@ScientificDoubleDelegate@LocalWorkflow@U2@@UBE?AVQVariant@@ABV4@@Z 1000ebe0 f   SamtoolMpileupWorker.obj
 0001:0000dc00       ?getResultUrl@CallVariantsTask@LocalWorkflow@U2@@QAE?AVQString@@XZ 1000ec00 f i SamtoolMpileupWorker.obj
 0001:0000dc30       ?getResults@CallVariantsTask@LocalWorkflow@U2@@QAEABV?$QList@V?$QMap@VQString@@VQVariant@@@@@@XZ 1000ec30 f i SamtoolMpileupWorker.obj
 0001:0000dc40       ?getSettings@CallVariantsWorker@LocalWorkflow@U2@@AAE?AVCallVariantsTaskSettings@23@XZ 1000ec40 f   SamtoolMpileupWorker.obj
 0001:0000e570       ?hasAssembly@CallVariantsWorker@LocalWorkflow@U2@@ABE_NXZ 1000f570 f   SamtoolMpileupWorker.obj
 0001:0000e5c0       ?hasNext@?$QMapIterator@VQString@@V1@@@QBE_NXZ 1000f5c0 f i SamtoolMpileupWorker.obj
 0001:0000e5d0       ?hasReferenceInPort@CallVariantsWorker@LocalWorkflow@U2@@ABE_NXZ 1000f5d0 f   SamtoolMpileupWorker.obj
 0001:0000e610       ?init@CallVariantsWorker@LocalWorkflow@U2@@UAEXXZ 1000f610 f   SamtoolMpileupWorker.obj
 0001:0000e7f0       ?init@CallVariantsWorkerFactory@LocalWorkflow@U2@@SAXXZ 1000f7f0 f   SamtoolMpileupWorker.obj
 0001:00015460       ?initDatasetMode@CallVariantsWorker@LocalWorkflow@U2@@AAEXXZ 10016460 f   SamtoolMpileupWorker.obj
 0001:000157c0       ?insert@?$QMap@VDescriptor@U2@@V?$QExplicitlySharedDataPointer@VDataType@U2@@@@@@QAE?AViterator@1@ABVDescriptor@U2@@ABV?$QExplicitlySharedDataPointer@VDataType@U2@@@@@Z 100167c0 f i SamtoolMpileupWorker.obj
 0001:000158c0       ?insert@?$QMap@VQString@@PAVPropertyDelegate@U2@@@@QAE?AViterator@1@ABVQString@@ABQAVPropertyDelegate@U2@@@Z 100168c0 f i SamtoolMpileupWorker.obj
 0001:00015980       ?insert@?$QMap@VQString@@VQScriptValue@@@@QAE?AViterator@1@ABVQString@@ABVQScriptValue@@@Z 10016980 f i SamtoolMpileupWorker.obj
 0001:00015a40       ?invoke@?$MetaTypeInvoker@U?$QVariantValueHelper@H@QtPrivate@@ABVQVariant@@H@QtPrivate@@SAHABVQVariant@@@Z 10016a40 f i SamtoolMpileupWorker.obj
 0001:00015a80       ?invoke@?$MetaTypeInvoker@U?$QVariantValueHelper@M@QtPrivate@@ABVQVariant@@M@QtPrivate@@SAMABVQVariant@@@Z 10016a80 f i SamtoolMpileupWorker.obj
 0001:00015ae0       ?invoke@?$MetaTypeInvoker@U?$QVariantValueHelper@VQString@@@QtPrivate@@ABVQVariant@@VQString@@@QtPrivate@@SA?AVQString@@ABVQVariant@@@Z 10016ae0 f i SamtoolMpileupWorker.obj
 0001:00015b00       ?invoke@?$MetaTypeInvoker@U?$QVariantValueHelper@_N@QtPrivate@@ABVQVariant@@_N@QtPrivate@@SA_NABVQVariant@@@Z 10016b00 f i SamtoolMpileupWorker.obj
 0001:00015b40       ?isEmpty@?$QList@PAVActor@Workflow@U2@@@@QBE_NXZ 10016b40 f i SamtoolMpileupWorker.obj
 0001:00015b50       ?isEmpty@?$QList@VMessage@Workflow@U2@@@@QBE_NXZ 10016b50 f i SamtoolMpileupWorker.obj
 0001:00015b60       ?isReady@CallVariantsWorker@LocalWorkflow@U2@@UBE_NXZ 10016b60 f   SamtoolMpileupWorker.obj
 0001:00015c10       ?key@?$QMapIterator@VQString@@V1@@@QBEABVQString@@XZ 10016c10 f i SamtoolMpileupWorker.obj
 0001:00015c20       ?key@const_iterator@?$QMap@VDescriptor@U2@@VQVariant@@@@QBEABVDescriptor@U2@@XZ 10016c20 f i SamtoolMpileupWorker.obj
 0001:00015c30       ?key@const_iterator@?$QMap@VQString@@V1@@@QBEABVQString@@XZ 10016c30 f i SamtoolMpileupWorker.obj
 0001:00015c40       ?leftNode@?$QMapNode@VDescriptor@U2@@V?$QExplicitlySharedDataPointer@VDataType@U2@@@@@@QBEPAU1@XZ 10016c40 f i SamtoolMpileupWorker.obj
 0001:00015c50       ?leftNode@?$QMapNode@VDescriptor@U2@@VQVariant@@@@QBEPAU1@XZ 10016c50 f i SamtoolMpileupWorker.obj
 0001:00015c60       ?leftNode@?$QMapNode@VQString@@PAVIntegralBus@Workflow@U2@@@@QBEPAU1@XZ 10016c60 f i SamtoolMpileupWorker.obj
 0001:00015c70       ?leftNode@?$QMapNode@VQString@@PAVPropertyDelegate@U2@@@@QBEPAU1@XZ 10016c70 f i SamtoolMpileupWorker.obj
 0001:00015c80       ?leftNode@?$QMapNode@VQString@@V1@@@QBEPAU1@XZ 10016c80 f i SamtoolMpileupWorker.obj
 0001:00015c90       ?leftNode@?$QMapNode@VQString@@VQScriptValue@@@@QBEPAU1@XZ 10016c90 f i SamtoolMpileupWorker.obj
 0001:00015ca0       ?lowerBound@?$QMapNode@VDescriptor@U2@@V?$QExplicitlySharedDataPointer@VDataType@U2@@@@@@QAEPAU1@ABVDescriptor@U2@@@Z 10016ca0 f i SamtoolMpileupWorker.obj
 0001:00015ce0       ?lowerBound@?$QMapNode@VDescriptor@U2@@VQVariant@@@@QAEPAU1@ABVDescriptor@U2@@@Z 10016ce0 f i SamtoolMpileupWorker.obj
 0001:00015d20       ?lowerBound@?$QMapNode@VQString@@PAVIntegralBus@Workflow@U2@@@@QAEPAU1@ABVQString@@@Z 10016d20 f i SamtoolMpileupWorker.obj
 0001:00015d60       ?lowerBound@?$QMapNode@VQString@@PAVPropertyDelegate@U2@@@@QAEPAU1@ABVQString@@@Z 10016d60 f i SamtoolMpileupWorker.obj
 0001:00015da0       ?lowerBound@?$QMapNode@VQString@@VQScriptValue@@@@QAEPAU1@ABVQString@@@Z 10016da0 f i SamtoolMpileupWorker.obj
 0001:00015de0       ?metaType@?$QVariantValueHelper@H@QtPrivate@@SAHABVQVariant@@@Z 10016de0 f i SamtoolMpileupWorker.obj
 0001:00015e20       ?metaType@?$QVariantValueHelper@M@QtPrivate@@SAMABVQVariant@@@Z 10016e20 f i SamtoolMpileupWorker.obj
 0001:00015e70       ?metaType@?$QVariantValueHelper@VQString@@@QtPrivate@@SA?AVQString@@ABVQVariant@@@Z 10016e70 f i SamtoolMpileupWorker.obj
 0001:00015f30       ?metaType@?$QVariantValueHelper@_N@QtPrivate@@SA_NABVQVariant@@@Z 10016f30 f i SamtoolMpileupWorker.obj
 0001:00015f70       ?next@?$QMapIterator@VQString@@V1@@@QAE?AVconst_iterator@?$QMap@VQString@@V1@@@XZ 10016f70 f i SamtoolMpileupWorker.obj
 0001:00015fa0       ?nextNode@?$QMapNode@VDescriptor@U2@@VQVariant@@@@QBEPBU1@XZ 10016fa0 f i SamtoolMpileupWorker.obj
 0001:00015fb0       ?nextNode@?$QMapNode@VQString@@V1@@@QBEPBU1@XZ 10016fb0 f i SamtoolMpileupWorker.obj
 0001:00015fc0       ?node_construct@?$QList@PAVAttribute@U2@@@@AAEXPAUNode@1@ABQAVAttribute@U2@@@Z 10016fc0 f i SamtoolMpileupWorker.obj
 0001:00015fe0       ?node_construct@?$QList@PAVPortDescriptor@Workflow@U2@@@@AAEXPAUNode@1@ABQAVPortDescriptor@Workflow@U2@@@Z 10016fe0 f i SamtoolMpileupWorker.obj
 0001:00016000       ?node_construct@?$QList@VDescriptor@U2@@@@AAEXPAUNode@1@ABVDescriptor@U2@@@Z 10017000 f i SamtoolMpileupWorker.obj
 0001:00016090       ?node_construct@?$QList@VMessage@Workflow@U2@@@@AAEXPAUNode@1@ABVMessage@Workflow@U2@@@Z 10017090 f i SamtoolMpileupWorker.obj
 0001:00016110       ?node_construct@?$QList@VQVariant@@@@AAEXPAUNode@1@ABVQVariant@@@Z 10017110 f i SamtoolMpileupWorker.obj
 0001:00016190       ?node_construct@?$QList@VWorkflowNotification@U2@@@@AAEXPAUNode@1@ABVWorkflowNotification@U2@@@Z 10017190 f i SamtoolMpileupWorker.obj
 0001:00016210       ?node_copy@?$QList@PAVAttribute@U2@@@@AAEXPAUNode@1@00@Z 10017210 f i SamtoolMpileupWorker.obj
 0001:00016240       ?node_copy@?$QList@PAVPort@Workflow@U2@@@@AAEXPAUNode@1@00@Z 10017240 f i SamtoolMpileupWorker.obj
 0001:00016270       ?node_copy@?$QList@PAVPortDescriptor@Workflow@U2@@@@AAEXPAUNode@1@00@Z 10017270 f i SamtoolMpileupWorker.obj
 0001:000162a0       ?node_copy@?$QList@VDescriptor@U2@@@@AAEXPAUNode@1@00@Z 100172a0 f i SamtoolMpileupWorker.obj
 0001:00016370       ?node_copy@?$QList@VMessage@Workflow@U2@@@@AAEXPAUNode@1@00@Z 10017370 f i SamtoolMpileupWorker.obj
 0001:00016440       ?node_copy@?$QList@VQVariant@@@@AAEXPAUNode@1@00@Z 10017440 f i SamtoolMpileupWorker.obj
 0001:00016510       ?node_copy@?$QList@VWorkflowNotification@U2@@@@AAEXPAUNode@1@00@Z 10017510 f i SamtoolMpileupWorker.obj
 0001:000165e0       ?node_destruct@?$QList@PAVActor@Workflow@U2@@@@AAEXPAUNode@1@0@Z 100175e0 f i SamtoolMpileupWorker.obj
 0001:000165f0       ?node_destruct@?$QList@PAVAttribute@U2@@@@AAEXPAUNode@1@0@Z 100175f0 f i SamtoolMpileupWorker.obj
 0001:00016600       ?node_destruct@?$QList@PAVAttribute@U2@@@@AAEXPAUNode@1@@Z 10017600 f i SamtoolMpileupWorker.obj
 0001:00016610       ?node_destruct@?$QList@PAVExternalToolListener@U2@@@@AAEXPAUNode@1@0@Z 10017610 f i SamtoolMpileupWorker.obj
 0001:00016620       ?node_destruct@?$QList@PAVPort@Workflow@U2@@@@AAEXPAUNode@1@0@Z 10017620 f i SamtoolMpileupWorker.obj
 0001:00016630       ?node_destruct@?$QList@PAVPortDescriptor@Workflow@U2@@@@AAEXPAUNode@1@0@Z 10017630 f i SamtoolMpileupWorker.obj
 0001:00016640       ?node_destruct@?$QList@PAVPortDescriptor@Workflow@U2@@@@AAEXPAUNode@1@@Z 10017640 f i SamtoolMpileupWorker.obj
 0001:00016650       ?node_destruct@?$QList@VDescriptor@U2@@@@AAEXPAUNode@1@0@Z 10017650 f i SamtoolMpileupWorker.obj
 0001:00016680       ?node_destruct@?$QList@VDescriptor@U2@@@@AAEXPAUNode@1@@Z 10017680 f i SamtoolMpileupWorker.obj
 0001:000166a0       ?node_destruct@?$QList@VMessage@Workflow@U2@@@@AAEXPAUNode@1@0@Z 100176a0 f i SamtoolMpileupWorker.obj
 0001:000166e0       ?node_destruct@?$QList@VMessage@Workflow@U2@@@@AAEXPAUNode@1@@Z 100176e0 f i SamtoolMpileupWorker.obj
 0001:00016710       ?node_destruct@?$QList@VQVariant@@@@AAEXPAUNode@1@0@Z 10017710 f i SamtoolMpileupWorker.obj
 0001:00016750       ?node_destruct@?$QList@VQVariant@@@@AAEXPAUNode@1@@Z 10017750 f i SamtoolMpileupWorker.obj
 0001:00016780       ?node_destruct@?$QList@VWorkflowNotification@U2@@@@AAEXPAUNode@1@0@Z 10017780 f i SamtoolMpileupWorker.obj
 0001:000167c0       ?node_destruct@?$QList@VWorkflowNotification@U2@@@@AAEXPAUNode@1@@Z 100177c0 f i SamtoolMpileupWorker.obj
 0001:000167f0       ?processError@CallVariantsWorker@LocalWorkflow@U2@@AAEXABVU2OpStatus@3@@Z 100177f0 f   SamtoolMpileupWorker.obj
 0001:000168b0       ?qt_metatype_id@?$QMetaTypeId2@H@@SAHXZ 100178b0 f i SamtoolMpileupWorker.obj
 0001:000168c0       ?qt_metatype_id@?$QMetaTypeId2@M@@SAHXZ 100178c0 f i SamtoolMpileupWorker.obj
 0001:000168d0       ?qt_metatype_id@?$QMetaTypeId2@VQString@@@@SAHXZ 100178d0 f i SamtoolMpileupWorker.obj
 0001:000168e0       ?qt_metatype_id@?$QMetaTypeId2@_N@@SAHXZ 100178e0 f i SamtoolMpileupWorker.obj
 0001:000168f0       ?removeFirst@?$QList@VMessage@Workflow@U2@@@@QAEXXZ 100178f0 f i SamtoolMpileupWorker.obj
 0001:00016930       ?reserve@?$QList@VDescriptor@U2@@@@QAEXH@Z 10017930 f i SamtoolMpileupWorker.obj
 0001:00016960       ?rightNode@?$QMapNode@VDescriptor@U2@@V?$QExplicitlySharedDataPointer@VDataType@U2@@@@@@QBEPAU1@XZ 10017960 f i SamtoolMpileupWorker.obj
 0001:00016970       ?rightNode@?$QMapNode@VDescriptor@U2@@VQVariant@@@@QBEPAU1@XZ 10017970 f i SamtoolMpileupWorker.obj
 0001:00016980       ?rightNode@?$QMapNode@VQString@@PAVIntegralBus@Workflow@U2@@@@QBEPAU1@XZ 10017980 f i SamtoolMpileupWorker.obj
 0001:00016990       ?rightNode@?$QMapNode@VQString@@PAVPropertyDelegate@U2@@@@QBEPAU1@XZ 10017990 f i SamtoolMpileupWorker.obj
 0001:000169a0       ?rightNode@?$QMapNode@VQString@@V1@@@QBEPAU1@XZ 100179a0 f i SamtoolMpileupWorker.obj
 0001:000169b0       ?rightNode@?$QMapNode@VQString@@VQScriptValue@@@@QBEPAU1@XZ 100179b0 f i SamtoolMpileupWorker.obj
 0001:000169c0       ?root@?$QMapData@VDescriptor@U2@@V?$QExplicitlySharedDataPointer@VDataType@U2@@@@@@QBEPAU?$QMapNode@VDescriptor@U2@@V?$QExplicitlySharedDataPointer@VDataType@U2@@@@@@XZ 100179c0 f i SamtoolMpileupWorker.obj
 0001:000169d0       ?root@?$QMapData@VDescriptor@U2@@VQVariant@@@@QBEPAU?$QMapNode@VDescriptor@U2@@VQVariant@@@@XZ 100179d0 f i SamtoolMpileupWorker.obj
 0001:000169e0       ?root@?$QMapData@VQString@@PAVIntegralBus@Workflow@U2@@@@QBEPAU?$QMapNode@VQString@@PAVIntegralBus@Workflow@U2@@@@XZ 100179e0 f i SamtoolMpileupWorker.obj
 0001:000169f0       ?root@?$QMapData@VQString@@PAVPropertyDelegate@U2@@@@QBEPAU?$QMapNode@VQString@@PAVPropertyDelegate@U2@@@@XZ 100179f0 f i SamtoolMpileupWorker.obj
 0001:00016a00       ?root@?$QMapData@VQString@@V1@@@QBEPAU?$QMapNode@VQString@@V1@@@XZ 10017a00 f i SamtoolMpileupWorker.obj
 0001:00016a10       ?root@?$QMapData@VQString@@VQScriptValue@@@@QBEPAU?$QMapNode@VQString@@VQScriptValue@@@@XZ 10017a10 f i SamtoolMpileupWorker.obj
 0001:00016a20       ?setEditorData@ScientificDoubleDelegate@LocalWorkflow@U2@@UBEXPAVQWidget@@ABVQModelIndex@@@Z 10017a20 f   SamtoolMpileupWorker.obj
 0001:00016aa0       ?setModelData@ScientificDoubleDelegate@LocalWorkflow@U2@@UBEXPAVQWidget@@PAVQAbstractItemModel@@ABVQModelIndex@@@Z 10017aa0 f   SamtoolMpileupWorker.obj
 0001:00016b10       ?setValue@ScientificDoubleWidget@LocalWorkflow@U2@@UAEXABVQVariant@@@Z 10017b10 f   SamtoolMpileupWorker.obj
 0001:00016b80       ?size@?$QMap@VDescriptor@U2@@VQVariant@@@@QBEHXZ 10017b80 f i SamtoolMpileupWorker.obj
 0001:00016b90       ?sl_taskFinished@CallVariantsWorker@LocalWorkflow@U2@@AAEXXZ 10017b90 f   SamtoolMpileupWorker.obj
 0001:00016df0       ?t@Node@?$QList@PAVPort@Workflow@U2@@@@QAEAAPAVPort@Workflow@U2@@XZ 10017df0 f i SamtoolMpileupWorker.obj
 0001:00016e00       ?t@Node@?$QList@V?$QMap@VQString@@VQVariant@@@@@@QAEAAV?$QMap@VQString@@VQVariant@@@@XZ 10017e00 f i SamtoolMpileupWorker.obj
 0001:00016e10       ?t@Node@?$QList@VDescriptor@U2@@@@QAEAAVDescriptor@U2@@XZ 10017e10 f i SamtoolMpileupWorker.obj
 0001:00016e20       ?t@Node@?$QList@VMessage@Workflow@U2@@@@QAEAAVMessage@Workflow@U2@@XZ 10017e20 f i SamtoolMpileupWorker.obj
 0001:00016e40       ?takeAssembly@CallVariantsWorker@LocalWorkflow@U2@@AAEXAAVU2OpStatus@3@@Z 10017e40 f   SamtoolMpileupWorker.obj
 0001:00017160       ?takeFirst@?$QList@VMessage@Workflow@U2@@@@QAE?AVMessage@Workflow@U2@@XZ 10018160 f i SamtoolMpileupWorker.obj
 0001:00017220       ?takeReference@CallVariantsWorker@LocalWorkflow@U2@@AAEXAAVU2OpStatus@3@@Z 10018220 f   SamtoolMpileupWorker.obj
 0001:00017460       ?tick@CallVariantsWorker@LocalWorkflow@U2@@UAEPAVTask@3@XZ 10018460 f   SamtoolMpileupWorker.obj
 0001:000177c0       ?tr@CallVariantsPrompter@LocalWorkflow@U2@@SA?AVQString@@PBD0H@Z 100187c0 f i SamtoolMpileupWorker.obj
 0001:000177f0       ?tr@CallVariantsWorker@LocalWorkflow@U2@@SA?AVQString@@PBD0H@Z 100187f0 f i SamtoolMpileupWorker.obj
 0001:00017820       ?uniqueKeys@?$QMap@VDescriptor@U2@@VQVariant@@@@QBE?AV?$QList@VDescriptor@U2@@@@XZ 10018820 f i SamtoolMpileupWorker.obj
 0001:00017920       ?validate@EmptySlotValidator@LocalWorkflow@U2@@UBE_NPBVConfiguration@3@AAV?$QList@VWorkflowNotification@U2@@@@@Z 10018920 f i SamtoolMpileupWorker.obj
 0001:00017bd0       ?value@?$QMap@VDescriptor@U2@@VQVariant@@@@QBE?BVQVariant@@ABVDescriptor@U2@@ABV2@@Z 10018bd0 f i SamtoolMpileupWorker.obj
 0001:00017c30       ?value@?$QMap@VQString@@PAVIntegralBus@Workflow@U2@@@@QBEQAVIntegralBus@Workflow@U2@@ABVQString@@ABQAV234@@Z 10018c30 f i SamtoolMpileupWorker.obj
 0001:00017c80       ?value@?$QMap@VQString@@VQVariant@@@@QBE?BVQVariant@@ABVQString@@ABV2@@Z 10018c80 f i SamtoolMpileupWorker.obj
 0001:00017cf0       ?value@?$QMapIterator@VQString@@V1@@@QBEABVQString@@XZ 10018cf0 f i SamtoolMpileupWorker.obj
 0001:00017d00       ?value@ScientificDoubleWidget@LocalWorkflow@U2@@UAE?AVQVariant@@XZ 10018d00 f   SamtoolMpileupWorker.obj
 0001:00017d80       ??0SamtoolsPlugin@U2@@QAE@XZ 10018d80 f   SamtoolsPlugin.obj
 0001:00017e30       ??1SamtoolsPlugin@U2@@UAE@XZ 10018e30 f i SamtoolsPlugin.obj
 0001:00017e40       ??_ESamtoolsPlugin@U2@@UAEPAXI@Z 10018e40 f i SamtoolsPlugin.obj
 0001:00017e40       ??_GSamtoolsPlugin@U2@@UAEPAXI@Z 10018e40 f i SamtoolsPlugin.obj
 0001:00017e70       ?tr@SamtoolsPlugin@U2@@SA?AVQString@@PBD0H@Z 10018e70 f i SamtoolsPlugin.obj
 0001:00017ea0       _ugene_plugin_init         10018ea0 f   SamtoolsPlugin.obj
 0001:00017ec0       ??C?$QScopedPointer@VQObjectData@@U?$QScopedPointerDeleter@VQObjectData@@@@@@QBEPAVQObjectData@@XZ 10018ec0 f i moc_AssemblySamtoolsMpileup.obj
 0001:00017ed0       ?metaObject@CallVariantsTask@LocalWorkflow@U2@@UBEPBUQMetaObject@@XZ 10018ed0 f   moc_AssemblySamtoolsMpileup.obj
 0001:00017ef0       ?metaObject@SamtoolsMpileupTask@LocalWorkflow@U2@@UBEPBUQMetaObject@@XZ 10018ef0 f   moc_AssemblySamtoolsMpileup.obj
 0001:00017f10       ?qt_metacall@CallVariantsTask@LocalWorkflow@U2@@UAEHW4Call@QMetaObject@@HPAPAX@Z 10018f10 f   moc_AssemblySamtoolsMpileup.obj
 0001:00017f20       ?qt_metacall@SamtoolsMpileupTask@LocalWorkflow@U2@@UAEHW4Call@QMetaObject@@HPAPAX@Z 10018f20 f   moc_AssemblySamtoolsMpileup.obj
 0001:00017f30       ?qt_metacast@CallVariantsTask@LocalWorkflow@U2@@UAEPAXPBD@Z 10018f30 f   moc_AssemblySamtoolsMpileup.obj
 0001:00017f90       ?qt_metacast@SamtoolsMpileupTask@LocalWorkflow@U2@@UAEPAXPBD@Z 10018f90 f   moc_AssemblySamtoolsMpileup.obj
 0001:00017ff0       ?qt_static_metacall@CallVariantsTask@LocalWorkflow@U2@@CAXPAVQObject@@W4Call@QMetaObject@@HPAPAX@Z 10018ff0 f   moc_AssemblySamtoolsMpileup.obj
 0001:00018000       ?qt_static_metacall@SamtoolsMpileupTask@LocalWorkflow@U2@@CAXPAVQObject@@W4Call@QMetaObject@@HPAPAX@Z 10019000 f   moc_AssemblySamtoolsMpileup.obj
 0001:00018010       ?metaObject@CallVariantsPrompter@LocalWorkflow@U2@@UBEPBUQMetaObject@@XZ 10019010 f   moc_SamtoolMpileupWorker.obj
 0001:00018030       ?metaObject@CallVariantsWorker@LocalWorkflow@U2@@UBEPBUQMetaObject@@XZ 10019030 f   moc_SamtoolMpileupWorker.obj
 0001:00018050       ?metaObject@ScientificDoubleWidget@LocalWorkflow@U2@@UBEPBUQMetaObject@@XZ 10019050 f   moc_SamtoolMpileupWorker.obj
 0001:00018070       ?qt_metacall@CallVariantsPrompter@LocalWorkflow@U2@@UAEHW4Call@QMetaObject@@HPAPAX@Z 10019070 f   moc_SamtoolMpileupWorker.obj
 0001:00018080       ?qt_metacall@CallVariantsWorker@LocalWorkflow@U2@@UAEHW4Call@QMetaObject@@HPAPAX@Z 10019080 f   moc_SamtoolMpileupWorker.obj
 0001:000180e0       ?qt_metacall@ScientificDoubleWidget@LocalWorkflow@U2@@UAEHW4Call@QMetaObject@@HPAPAX@Z 100190e0 f   moc_SamtoolMpileupWorker.obj
 0001:00018150       ?qt_metacast@CallVariantsPrompter@LocalWorkflow@U2@@UAEPAXPBD@Z 10019150 f   moc_SamtoolMpileupWorker.obj
 0001:000181b0       ?qt_metacast@CallVariantsWorker@LocalWorkflow@U2@@UAEPAXPBD@Z 100191b0 f   moc_SamtoolMpileupWorker.obj
 0001:00018210       ?qt_metacast@ScientificDoubleWidget@LocalWorkflow@U2@@UAEPAXPBD@Z 10019210 f   moc_SamtoolMpileupWorker.obj
 0001:00018270       ?qt_static_metacall@CallVariantsPrompter@LocalWorkflow@U2@@CAXPAVQObject@@W4Call@QMetaObject@@HPAPAX@Z 10019270 f   moc_SamtoolMpileupWorker.obj
 0001:00018280       ?qt_static_metacall@CallVariantsWorker@LocalWorkflow@U2@@CAXPAVQObject@@W4Call@QMetaObject@@HPAPAX@Z 10019280 f   moc_SamtoolMpileupWorker.obj
 0001:000182a0       ?qt_static_metacall@ScientificDoubleWidget@LocalWorkflow@U2@@CAXPAVQObject@@W4Call@QMetaObject@@HPAPAX@Z 100192a0 f   moc_SamtoolMpileupWorker.obj
 0001:000182d0       ?metaObject@SamtoolsPlugin@U2@@UBEPBUQMetaObject@@XZ 100192d0 f   moc_SamtoolsPlugin.obj
 0001:000182f0       ?qt_metacall@SamtoolsPlugin@U2@@UAEHW4Call@QMetaObject@@HPAPAX@Z 100192f0 f   moc_SamtoolsPlugin.obj
 0001:00018300       ?qt_metacast@SamtoolsPlugin@U2@@UAEPAXPBD@Z 10019300 f   moc_SamtoolsPlugin.obj
 0001:00018360       ?qt_static_metacall@SamtoolsPlugin@U2@@CAXPAVQObject@@W4Call@QMetaObject@@HPAPAX@Z 10019360 f   moc_SamtoolsPlugin.obj
 0001:00018362       ?getAppSettings@AppContext@U2@@SAPAVAppSettings@2@XZ 10019362 f   U2Core:U2Core.dll
 0001:00018368       ?getIOAdapterRegistry@AppContext@U2@@SAPAVIOAdapterRegistry@2@XZ 10019368 f   U2Core:U2Core.dll
 0001:0001836e       ??0Logger@U2@@QAE@ABVQString@@@Z 1001936e f   U2Core:U2Core.dll
 0001:00018374       ??1Logger@U2@@UAE@XZ       10019374 f   U2Core:U2Core.dll
 0001:0001837a       ?details@Logger@U2@@QAEXABVQString@@@Z 1001937a f   U2Core:U2Core.dll
 0001:00018380       ?error@Logger@U2@@QAEXABVQString@@@Z 10019380 f   U2Core:U2Core.dll
 0001:00018386       ?addSubTask@Task@U2@@QAEXPAV12@@Z 10019386 f   U2Core:U2Core.dll
 0001:0001838c       ?hasError@Task@U2@@QBE_NXZ 1001938c f   U2Core:U2Core.dll
 0001:00018392       ?getError@Task@U2@@QBE?AVQString@@XZ 10019392 f   U2Core:U2Core.dll
 0001:00018398       ?setMaxParallelSubtasks@Task@U2@@QAEXH@Z 10019398 f   U2Core:U2Core.dll
 0001:0001839e       ?setError@Task@U2@@QAEXABVQString@@@Z 1001939e f   U2Core:U2Core.dll
 0001:000183a4       ?killProcessTree@CmdlineTaskRunner@U2@@SAHPAVQProcess@@@Z 100193a4 f   U2Core:U2Core.dll
 0001:000183aa       ??1GCounter@U2@@UAE@XZ     100193aa f   U2Core:U2Core.dll
 0001:000183b0       ??0GReportableCounter@U2@@QAE@ABVQString@@0N@Z 100193b0 f   U2Core:U2Core.dll
 0001:000183b6       ??1SimpleEventCounter@U2@@UAE@XZ 100193b6 f   U2Core:U2Core.dll
 0001:000183bc       ??0GUrl@U2@@QAE@ABVQString@@@Z 100193bc f   U2Core:U2Core.dll
 0001:000183c2       ??1GUrl@U2@@QAE@XZ         100193c2 f   U2Core:U2Core.dll
 0001:000183c8       ??0U2DbiRef@U2@@QAE@ABVQString@@0@Z 100193c8 f   U2Core:U2Core.dll
 0001:000183ce       ??1U2DbiRef@U2@@QAE@XZ     100193ce f   U2Core:U2Core.dll
 0001:000183d4       ??0U2DbiRef@U2@@QAE@ABV01@@Z 100193d4 f   U2Core:U2Core.dll
 0001:000183da       ??0GObjectReference@U2@@QAE@XZ 100193da f   U2Core:U2Core.dll
 0001:000183e0       ??1GObjectReference@U2@@QAE@XZ 100193e0 f   U2Core:U2Core.dll
 0001:000183e6       ?findGObjectByType@Document@U2@@QBE?AV?$QList@PAVGObject@U2@@@@VQString@@W4UnloadedObjectFilter@2@@Z 100193e6 f   U2Core:U2Core.dll
 0001:000183ec       ??1FormatDetectionResult@U2@@QAE@XZ 100193ec f   U2Core:U2Core.dll
 0001:000183f2       ??0FormatDetectionResult@U2@@QAE@ABV01@@Z 100193f2 f   U2Core:U2Core.dll
 0001:000183f8       ?detectFormat@DocumentUtils@U2@@SA?AV?$QList@VFormatDetectionResult@U2@@@@ABVGUrl@2@ABVFormatDetectionConfig@2@@Z 100193f8 f   U2Core:U2Core.dll
 0001:000183fe       ?prepareTmpFileLocation@GUrlUtils@U2@@SA?AVQString@@ABV3@00AAVU2OpStatus@2@@Z 100193fe f   U2Core:U2Core.dll
 0001:00018404       ?url2io@IOAdapterUtils@U2@@SA?AVQString@@ABVGUrl@2@@Z 10019404 f   U2Core:U2Core.dll
 0001:0001840a       ??0LoadDocumentTaskConfig@U2@@QAE@_NABVGObjectReference@1@PAVLDTObjectFactory@1@@Z 1001940a f   U2Core:U2Core.dll
 0001:00018410       ??1LoadDocumentTaskConfig@U2@@QAE@XZ 10019410 f   U2Core:U2Core.dll
 0001:00018416       ??0LoadDocumentTask@U2@@QAE@VQString@@ABVGUrl@1@PAVIOAdapterFactory@1@ABV?$QMap@VQString@@VQVariant@@@@ABVLoadDocumentTaskConfig@1@@Z 10019416 f   U2Core:U2Core.dll
 0001:0001841c       ??1LoadDocumentTask@U2@@UAE@XZ 1001941c f   U2Core:U2Core.dll
 0001:00018422       ?getCurrentProcessTemporaryDirPath@UserAppsSettings@U2@@QBE?AVQString@@ABV3@@Z 10019422 f   U2Core:U2Core.dll
 0001:00018428       ??1ProcessRun@U2@@QAE@XZ   10019428 f   U2Core:U2Core.dll
 0001:0001842e       ??0ExternalToolSupportTask@U2@@QAE@ABVQString@@V?$QFlags@W4TaskFlag@U2@@@@@Z 1001942e f   U2Core:U2Core.dll
 0001:00018434       ??1ExternalToolSupportTask@U2@@UAE@XZ 10019434 f   U2Core:U2Core.dll
 0001:0001843a       ?addListeners@ExternalToolSupportTask@U2@@QAEXABV?$QList@PAVExternalToolListener@U2@@@@@Z 1001943a f   U2Core:U2Core.dll
 0001:00018440       ?getListener@ExternalToolSupportTask@U2@@QAEPAVExternalToolListener@2@H@Z 10019440 f   U2Core:U2Core.dll
 0001:00018446       ??0ExternalToolRunTaskHelper@U2@@QAE@PAVQProcess@@PAVExternalToolLogParser@1@AAVU2OpStatus@1@@Z 10019446 f   U2Core:U2Core.dll
 0001:0001844c       ??1ExternalToolRunTaskHelper@U2@@UAE@XZ 1001944c f   U2Core:U2Core.dll
 0001:00018452       ?prepareProcess@ExternalToolSupportUtils@U2@@SA?AVProcessRun@2@ABVQString@@ABVQStringList@@01AAVU2OpStatus@2@PAVExternalToolListener@2@@Z 10019452 f   U2Core:U2Core.dll
 0001:00018458       ??0ExternalToolLogParser@U2@@QAE@_N@Z 10019458 f   U2Core:U2Core.dll
 0001:0001845e       ??1ExternalToolLogParser@U2@@UAE@XZ 1001945e f   U2Core:U2Core.dll
 0001:00018464       ?cleanup@DocumentProviderTask@U2@@UAEXXZ 10019464 f   U2Core:U2Core.dll
 0001:0001846a       ?cleanup@Task@U2@@UAEXXZ   1001946a f   U2Core:U2Core.dll
 0001:00018470       ?generateReport@Task@U2@@UBE?AVQString@@XZ 10019470 f   U2Core:U2Core.dll
 0001:00018476       ?getDocument@DocumentProviderTask@U2@@UAEPAVDocument@2@_N@Z 10019476 f   U2Core:U2Core.dll
 0001:0001847c       ?getDocumentDescription@DocumentProviderTask@U2@@UBE?AVQString@@XZ 1001947c f   U2Core:U2Core.dll
 0001:00018482       ?getNumParallelSubtasks@Task@U2@@UBEHXZ 10019482 f   U2Core:U2Core.dll
 0001:00018488       ?getParentTask@Task@U2@@UBEPAV12@XZ 10019488 f   U2Core:U2Core.dll
 0001:0001848e       ?getSubtaskWithErrors@Task@U2@@UBEPAV12@XZ 1001948e f   U2Core:U2Core.dll
 0001:00018494       ?getTaskId@Task@U2@@UBE_JXZ 10019494 f   U2Core:U2Core.dll
 0001:0001849a       ?getTopLevelParentTask@Task@U2@@UAEPAV12@XZ 1001949a f   U2Core:U2Core.dll
 0001:000184a0       ?getWarnings@Task@U2@@UBE?AVQStringList@@XZ 100194a0 f   U2Core:U2Core.dll
 0001:000184a6       ?hasSubtasksWithErrors@Task@U2@@UBE_NXZ 100194a6 f   U2Core:U2Core.dll
 0001:000184ac       ?hasWarning@Task@U2@@UBE_NXZ 100194ac f   U2Core:U2Core.dll
 0001:000184b2       ?isNotificationReport@Task@U2@@UBE_NXZ 100194b2 f   U2Core:U2Core.dll
 0001:000184b8       ?isReportingEnabled@Task@U2@@UBE_NXZ 100194b8 f   U2Core:U2Core.dll
 0001:000184be       ?isReportingSupported@Task@U2@@UBE_NXZ 100194be f   U2Core:U2Core.dll
 0001:000184c4       ?isTopLevelTask@Task@U2@@UBE_NXZ 100194c4 f   U2Core:U2Core.dll
 0001:000184ca       ?metaObject@LoadDocumentTask@U2@@UBEPBUQMetaObject@@XZ 100194ca f   U2Core:U2Core.dll
 0001:000184d0       ?onSubTaskFinished@Task@U2@@MAE?AV?$QList@PAVTask@U2@@@@PAV12@@Z 100194d0 f   U2Core:U2Core.dll
 0001:000184d6       ?prepare@LoadDocumentTask@U2@@UAEXXZ 100194d6 f   U2Core:U2Core.dll
 0001:000184dc       ?propagateSubtaskError@Task@U2@@UAE_NXZ 100194dc f   U2Core:U2Core.dll
 0001:000184e2       ?qt_metacall@LoadDocumentTask@U2@@UAEHW4Call@QMetaObject@@HPAPAX@Z 100194e2 f   U2Core:U2Core.dll
 0001:000184e8       ?qt_metacast@LoadDocumentTask@U2@@UAEPAXPBD@Z 100194e8 f   U2Core:U2Core.dll
 0001:000184ee       ?report@LoadDocumentTask@U2@@UAE?AW4ReportResult@Task@2@XZ 100194ee f   U2Core:U2Core.dll
 0001:000184f4       ?report@Task@U2@@UAE?AW4ReportResult@12@XZ 100194f4 f   U2Core:U2Core.dll
 0001:000184fa       ?run@LoadDocumentTask@U2@@UAEXXZ 100194fa f   U2Core:U2Core.dll
 0001:00018500       ?run@Task@U2@@UAEXXZ       10019500 f   U2Core:U2Core.dll
 0001:00018506       ?setCollectChildrensWarningsFlag@Task@U2@@UAEX_N@Z 10019506 f   U2Core:U2Core.dll
 0001:0001850c       ?setListenerForHelper@ExternalToolSupportTask@U2@@MAEXPAVExternalToolRunTaskHelper@2@H@Z 1001950c f   U2Core:U2Core.dll
 0001:00018512       ?setListenerForTask@ExternalToolSupportTask@U2@@MAEXPAVExternalToolRunTask@2@H@Z 10019512 f   U2Core:U2Core.dll
 0001:00018518       ?setNoAutoDelete@Task@U2@@UAEX_N@Z 10019518 f   U2Core:U2Core.dll
 0001:0001851e       ?setNotificationReport@Task@U2@@UAEX_N@Z 1001951e f   U2Core:U2Core.dll
 0001:00018524       ?setReportingEnabled@Task@U2@@UAEX_N@Z 10019524 f   U2Core:U2Core.dll
 0001:0001852a       ?setReportingSupported@Task@U2@@UAEX_N@Z 1001952a f   U2Core:U2Core.dll
 0001:00018530       ?takeDocument@DocumentProviderTask@U2@@UAEPAVDocument@2@_N@Z 10019530 f   U2Core:U2Core.dll
 0001:00018536       ?isCoR@U2OpStatus@U2@@UBE_NXZ 10019536 f   U2Core:U2Core.dll
 0001:0001853c       ??0TaskStateInfo@U2@@QAE@XZ 1001953c f   U2Core:U2Core.dll
 0001:00018542       ?getError@TaskStateInfo@U2@@UBE?AVQString@@XZ 10019542 f   U2Core:U2Core.dll
 0001:00018548       ?setError@TaskStateInfo@U2@@UAEXABVQString@@@Z 10019548 f   U2Core:U2Core.dll
 0001:0001854e       ??1TaskStateInfo@U2@@UAE@XZ 1001954e f   U2Core:U2Core.dll
 0001:00018554       ?rollFileName@GUrlUtils@U2@@SA?AVQString@@ABV3@0ABV?$QSet@VQString@@@@@Z 10019554 f   U2Core:U2Core.dll
 0001:0001855a       ??0U2OpStatus2Log@U2@@QAE@W4LogLevel@1@@Z 1001955a f   U2Core:U2Core.dll
 0001:00018560       ??1U2OpStatus2Log@U2@@UAE@XZ 10019560 f   U2Core:U2Core.dll
 0001:00018566       ?runScript@ScriptTask@U2@@SA?AVQScriptValue@@PAVQScriptEngine@@ABV?$QMap@VQString@@VQScriptValue@@@@ABVQString@@AAVTaskStateInfo@2@@Z 10019566 f   U2Core:U2Core.dll
 0001:0001856c       ?unpackMap@StrPackUtils@U2@@SA?AV?$QMap@VQString@@V1@@@ABVQString@@W4Options@12@@Z 1001956c f   U2Core:U2Core.dll
 0001:00018572       ??0Plugin@U2@@QAE@ABVQString@@0_NW4PluginState@1@@Z 10019572 f   U2Core:U2Core.dll
 0001:00018578       ??1Plugin@U2@@UAE@XZ       10019578 f   U2Core:U2Core.dll
 0001:0001857e       ?qt_metacast@Task@U2@@UAEPAXPBD@Z 1001957e f   U2Core:U2Core.dll
 0001:00018584       ?qt_metacall@Task@U2@@UAEHW4Call@QMetaObject@@HPAPAX@Z 10019584 f   U2Core:U2Core.dll
 0001:0001858a       ?qt_metacast@Plugin@U2@@UAEPAXPBD@Z 1001958a f   U2Core:U2Core.dll
 0001:00018590       ?qt_metacall@Plugin@U2@@UAEHW4Call@QMetaObject@@HPAPAX@Z 10019590 f   U2Core:U2Core.dll
 0001:00018596       ??1Descriptor@U2@@UAE@XZ   10019596 f   U2Lang:U2Lang.dll
 0001:0001859c       ?getId@Descriptor@U2@@QBE?AVQString@@XZ 1001959c f   U2Lang:U2Lang.dll
 0001:000185a2       ?URL_SLOT@BaseSlots@Workflow@U2@@SA?BVDescriptor@3@XZ 100195a2 f   U2Lang:U2Lang.dll
 0001:000185a8       ?VARIATION_TRACK_SLOT@BaseSlots@Workflow@U2@@SA?BVDescriptor@3@XZ 100195a8 f   U2Lang:U2Lang.dll
 0001:000185ae       ?getDbiRef@DbiDataStorage@Workflow@U2@@QAE?AVU2DbiRef@3@XZ 100195ae f   U2Lang:U2Lang.dll
 0001:000185b4       ??0VisibilityRelation@U2@@QAE@ABVQString@@ABV?$QList@VQVariant@@@@_N@Z 100195b4 f   U2Lang:U2Lang.dll
 0001:000185ba       ??1VisibilityRelation@U2@@UAE@XZ 100195ba f   U2Lang:U2Lang.dll
 0001:000185c0       ??0Descriptor@U2@@QAE@ABVQString@@00@Z 100195c0 f   U2Lang:U2Lang.dll
 0001:000185c6       ??0Descriptor@U2@@QAE@ABVQString@@@Z 100195c6 f   U2Lang:U2Lang.dll
 0001:000185cc       ??0Descriptor@U2@@QAE@PBD@Z 100195cc f   U2Lang:U2Lang.dll
 0001:000185d2       ?getDisplayName@Descriptor@U2@@QBE?AVQString@@XZ 100195d2 f   U2Lang:U2Lang.dll
 0001:000185d8       ??0Descriptor@U2@@QAE@ABV01@@Z 100195d8 f   U2Lang:U2Lang.dll
 0001:000185de       ?getDatatypeDescriptor@DataType@U2@@QBE?AVDescriptor@2@ABVQString@@@Z 100195de f   U2Lang:U2Lang.dll
 0001:000185e4       ??0MapDataType@U2@@QAE@ABVDescriptor@1@ABV?$QMap@VDescriptor@U2@@V?$QExplicitlySharedDataPointer@VDataType@U2@@@@@@@Z 100195e4 f   U2Lang:U2Lang.dll
 0001:000185ea       ??1MapDataType@U2@@UAE@XZ  100195ea f   U2Lang:U2Lang.dll
 0001:000185f0       ?initEngine@WorkflowScriptLibrary@U2@@SAXPAVWorkflowScriptEngine@2@@Z 100195f0 f   U2Lang:U2Lang.dll
 0001:000185f6       ??0WorkflowNotification@U2@@QAE@ABVQString@@00@Z 100195f6 f   U2Lang:U2Lang.dll
 0001:000185fc       ??1WorkflowNotification@U2@@QAE@XZ 100195fc f   U2Lang:U2Lang.dll
 0001:00018602       ??0WorkflowNotification@U2@@QAE@ABV01@@Z 10019602 f   U2Lang:U2Lang.dll
 0001:00018608       ?getDataStorage@WorkflowContext@Workflow@U2@@QAEPAVDbiDataStorage@23@XZ 10019608 f   U2Lang:U2Lang.dll
 0001:0001860e       ?absolutePath@WorkflowContext@Workflow@U2@@QBE?AVQString@@ABV4@@Z 1001960e f   U2Lang:U2Lang.dll
 0001:00018614       ??0WorkflowScriptEngine@U2@@QAE@PAVWorkflowContext@Workflow@1@@Z 10019614 f   U2Lang:U2Lang.dll
 0001:0001861a       ??1WorkflowScriptEngine@U2@@UAE@XZ 1001961a f   U2Lang:U2Lang.dll
 0001:00018620       ??0PortRelationDescriptor@U2@@QAE@ABVQString@@ABV?$QList@VQVariant@@@@@Z 10019620 f   U2Lang:U2Lang.dll
 0001:00018626       ??1PortRelationDescriptor@U2@@UAE@XZ 10019626 f   U2Lang:U2Lang.dll
 0001:0001862c       ?isEmpty@AttributeScript@U2@@QBE_NXZ 1001962c f   U2Lang:U2Lang.dll
 0001:00018632       ?getScriptText@AttributeScript@U2@@QBEABVQString@@XZ 10019632 f   U2Lang:U2Lang.dll
 0001:00018638       ?getScriptVars@AttributeScript@U2@@QBEABV?$QMap@VDescriptor@U2@@VQVariant@@@@XZ 10019638 f   U2Lang:U2Lang.dll
 0001:0001863e       ??0Attribute@U2@@QAE@ABVDescriptor@1@V?$QExplicitlySharedDataPointer@VDataType@U2@@@@_NABVQVariant@@@Z 1001963e f   U2Lang:U2Lang.dll
 0001:00018644       ??1Attribute@U2@@UAE@XZ    10019644 f   U2Lang:U2Lang.dll
 0001:0001864a       ?addRelation@Attribute@U2@@QAEXPBVAttributeRelation@2@@Z 1001964a f   U2Lang:U2Lang.dll
 0001:00018650       ?addPortRelation@Attribute@U2@@QAEXPAVPortRelationDescriptor@2@@Z 10019650 f   U2Lang:U2Lang.dll
 0001:00018656       ?isOutUrlAttribute@RFSUtils@U2@@SA_NPAVAttribute@2@PAVActor@Workflow@2@AA_N@Z 10019656 f   U2Lang:U2Lang.dll
 0001:0001865c       ??0PropertyWidget@U2@@QAE@PAVQWidget@@PAVDelegateTags@1@@Z 1001965c f   U2Lang:U2Lang.dll
 0001:00018662       ??1PropertyWidget@U2@@UAE@XZ 10019662 f   U2Lang:U2Lang.dll
 0001:00018668       ?addMainWidget@PropertyWidget@U2@@IAEXPAVQWidget@@@Z 10019668 f   U2Lang:U2Lang.dll
 0001:0001866e       ??0PropertyDelegate@U2@@QAE@PAVQObject@@@Z 1001966e f   U2Lang:U2Lang.dll
 0001:00018674       ??1PropertyDelegate@U2@@UAE@XZ 10019674 f   U2Lang:U2Lang.dll
 0001:0001867a       ??1ConfigurationValidator@U2@@UAE@XZ 1001967a f   U2Lang:U2Lang.dll
 0001:00018680       ?getId@Actor@Workflow@U2@@QBE?AVQString@@XZ 10019680 f   U2Lang:U2Lang.dll
 0001:00018686       ?getLabel@Actor@Workflow@U2@@QBE?AVQString@@XZ 10019686 f   U2Lang:U2Lang.dll
 0001:0001868c       ?getPort@Actor@Workflow@U2@@QBEPAVPort@23@ABVQString@@@Z 1001968c f   U2Lang:U2Lang.dll
 0001:00018692       ?getInputPorts@Actor@Workflow@U2@@QBE?AV?$QList@PAVPort@Workflow@U2@@@@XZ 10019692 f   U2Lang:U2Lang.dll
 0001:00018698       ?getOutputPorts@Actor@Workflow@U2@@QBE?AV?$QList@PAVPort@Workflow@U2@@@@XZ 10019698 f   U2Lang:U2Lang.dll
 0001:0001869e       ??0PortDescriptor@Workflow@U2@@QAE@ABVDescriptor@2@V?$QExplicitlySharedDataPointer@VDataType@U2@@@@_N2I@Z 1001969e f   U2Lang:U2Lang.dll
 0001:000186a4       ??1PortDescriptor@Workflow@U2@@UAE@XZ 100196a4 f   U2Lang:U2Lang.dll
 0001:000186aa       ??0ActorPrototype@Workflow@U2@@QAE@ABVDescriptor@2@ABV?$QList@PAVPortDescriptor@Workflow@U2@@@@ABV?$QList@PAVAttribute@U2@@@@@Z 100196aa f   U2Lang:U2Lang.dll
 0001:000186b0       ??1ActorPrototype@Workflow@U2@@UAE@XZ 100196b0 f   U2Lang:U2Lang.dll
 0001:000186b6       ?setEditor@ActorPrototype@Workflow@U2@@QAEXPAVConfigurationEditor@3@@Z 100196b6 f   U2Lang:U2Lang.dll
 0001:000186bc       ?setPrompter@ActorPrototype@Workflow@U2@@QAEXPAVPrompter@23@@Z 100196bc f   U2Lang:U2Lang.dll
 0001:000186c2       ?setPortValidator@ActorPrototype@Workflow@U2@@QAEXABVQString@@PAVConfigurationValidator@3@@Z 100196c2 f   U2Lang:U2Lang.dll
 0001:000186c8       ?addExternalTool@ActorPrototype@Workflow@U2@@QAEXABVQString@@0@Z 100196c8 f   U2Lang:U2Lang.dll
 0001:000186ce       ?registerProto@ActorPrototypeRegistry@Workflow@U2@@QAE_NABVDescriptor@3@PAVActorPrototype@23@@Z 100196ce f   U2Lang:U2Lang.dll
 0001:000186d4       ?CATEGORY_VARIATION_ANALYSIS@BaseActorCategories@Workflow@U2@@SA?BVDescriptor@3@XZ 100196d4 f   U2Lang:U2Lang.dll
 0001:000186da       ?IN_SEQ_PORT_ID@BasePorts@Workflow@U2@@SA?BVQString@@XZ 100196da f   U2Lang:U2Lang.dll
 0001:000186e0       ?OUT_VARIATION_TRACK_PORT_ID@BasePorts@Workflow@U2@@SA?BVQString@@XZ 100196e0 f   U2Lang:U2Lang.dll
 0001:000186e6       ?IN_ASSEMBLY_PORT_ID@BasePorts@Workflow@U2@@SA?BVQString@@XZ 100196e6 f   U2Lang:U2Lang.dll
 0001:000186ec       ?DATASET_SLOT@BaseSlots@Workflow@U2@@SA?BVDescriptor@3@XZ 100196ec f   U2Lang:U2Lang.dll
 0001:000186f2       ?VARIATION_TRACK_TYPE@BaseTypes@U2@@SA?AV?$QExplicitlySharedDataPointer@VDataType@U2@@@@XZ 100196f2 f   U2Lang:U2Lang.dll
 0001:000186f8       ?STRING_TYPE@BaseTypes@U2@@SA?AV?$QExplicitlySharedDataPointer@VDataType@U2@@@@XZ 100196f8 f   U2Lang:U2Lang.dll
 0001:000186fe       ?BOOL_TYPE@BaseTypes@U2@@SA?AV?$QExplicitlySharedDataPointer@VDataType@U2@@@@XZ 100196fe f   U2Lang:U2Lang.dll
 0001:00018704       ?NUM_TYPE@BaseTypes@U2@@SA?AV?$QExplicitlySharedDataPointer@VDataType@U2@@@@XZ 10019704 f   U2Lang:U2Lang.dll
 0001:0001870a       ?getProducer@IntegralBusPort@Workflow@U2@@QAEPAVActor@23@ABVQString@@@Z 1001970a f   U2Lang:U2Lang.dll
 0001:00018710       ?getProducers@IntegralBusPort@Workflow@U2@@QAE?AV?$QList@PAVActor@Workflow@U2@@@@ABVQString@@@Z 10019710 f   U2Lang:U2Lang.dll
 0001:00018716       ?getInstance@WorkflowEnv@Workflow@U2@@KAPAV123@XZ 10019716 f   U2Lang:U2Lang.dll
 0001:0001871c       ??0Message@Workflow@U2@@QAE@V?$QExplicitlySharedDataPointer@VDataType@U2@@@@ABVQVariant@@H@Z 1001971c f   U2Lang:U2Lang.dll
 0001:00018722       ?getData@Message@Workflow@U2@@QBE?AVQVariant@@XZ 10019722 f   U2Lang:U2Lang.dll
 0001:00018728       ?isEmpty@Message@Workflow@U2@@QBE_NXZ 10019728 f   U2Lang:U2Lang.dll
 0001:0001872e       ??1Message@Workflow@U2@@QAE@XZ 1001972e f   U2Lang:U2Lang.dll
 0001:00018734       ??0Message@Workflow@U2@@QAE@ABV012@@Z 10019734 f   U2Lang:U2Lang.dll
 0001:0001873a       ??0DomainFactory@Workflow@U2@@QAE@ABVQString@@@Z 1001973a f   U2Lang:U2Lang.dll
 0001:00018740       ??1DomainFactory@Workflow@U2@@UAE@XZ 10019740 f   U2Lang:U2Lang.dll
 0001:00018746       ?addOutputFile@WorkflowMonitor@Workflow@U2@@QAEXABVQString@@0_N@Z 10019746 f   U2Lang:U2Lang.dll
 0001:0001874c       ?addError@WorkflowMonitor@Workflow@U2@@QAEXABVQString@@00@Z 1001974c f   U2Lang:U2Lang.dll
 0001:00018752       ?getBusType@IntegralBus@Workflow@U2@@QBE?AV?$QExplicitlySharedDataPointer@VDataType@U2@@@@XZ 10019752 f   U2Lang:U2Lang.dll
 0001:00018758       ??0BaseWorker@LocalWorkflow@U2@@QAE@PAVActor@Workflow@2@_N@Z 10019758 f   U2Lang:U2Lang.dll
 0001:0001875e       ??1BaseWorker@LocalWorkflow@U2@@UAE@XZ 1001975e f   U2Lang:U2Lang.dll
 0001:00018764       ?createLogListeners@BaseWorker@LocalWorkflow@U2@@QBE?AV?$QList@PAVExternalToolListener@U2@@@@H@Z 10019764 f   U2Lang:U2Lang.dll
 0001:0001876a       ?monitor@BaseWorker@LocalWorkflow@U2@@IBEPAVWorkflowMonitor@Workflow@3@XZ 1001976a f   U2Lang:U2Lang.dll
 0001:00018770       ??0PrompterBaseImpl@U2@@QAE@PAVActor@Workflow@1@@Z 10019770 f   U2Lang:U2Lang.dll
 0001:00018776       ?getURL@PrompterBaseImpl@U2@@QAE?AVQString@@ABV3@PA_N00@Z 10019776 f   U2Lang:U2Lang.dll
 0001:0001877c       ?getHyperlink@PrompterBaseImpl@U2@@SA?AVQString@@ABV3@0@Z 1001977c f   U2Lang:U2Lang.dll
 0001:00018782       ??1PrompterBaseImpl@U2@@UAE@XZ 10019782 f   U2Lang:U2Lang.dll
 0001:00018788       ?activate@PropertyWidget@U2@@UAEXXZ 10019788 f   U2Lang:U2Lang.dll
 0001:0001878e       ?addCommunication@BaseWorker@LocalWorkflow@U2@@UAE_NABVQString@@PAVCommunicationChannel@Workflow@3@@Z 1001978e f   U2Lang:U2Lang.dll
 0001:00018794       ?canTaskBeCanceled@BaseWorker@LocalWorkflow@U2@@MBE_NPAVTask@3@@Z 10019794 f   U2Lang:U2Lang.dll
 0001:0001879a       ?clone@Attribute@U2@@UAEPAV12@XZ 1001979a f   U2Lang:U2Lang.dll
 0001:000187a0       ?clone@PortRelationDescriptor@U2@@UBEPAV12@XZ 100197a0 f   U2Lang:U2Lang.dll
 0001:000187a6       ?clone@VisibilityRelation@U2@@UBEPAV12@XZ 100197a6 f   U2Lang:U2Lang.dll
 0001:000187ac       ?createConnection@DomainFactory@Workflow@U2@@UAEPAVCommunicationChannel@23@PAVLink@23@@Z 100197ac f   U2Lang:U2Lang.dll
 0001:000187b2       ?createInstance@ActorPrototype@Workflow@U2@@UAEPAVActor@23@ABVQString@@PAVAttributeScript@3@ABV?$QMap@VQString@@VQVariant@@@@@Z 100197b2 f   U2Lang:U2Lang.dll
 0001:000187b8       ?createPort@IntegralBusActorPrototype@Workflow@U2@@UAEPAVPort@23@ABVPortDescriptor@23@PAVActor@23@@Z 100197b8 f   U2Lang:U2Lang.dll
 0001:000187be       ?createScheduler@DomainFactory@Workflow@U2@@UAEPAVScheduler@23@PAVSchema@23@@Z 100197be f   U2Lang:U2Lang.dll
 0001:000187c4       ?destroy@DomainFactory@Workflow@U2@@UAEXPAVScheduler@23@PAVSchema@23@@Z 100197c4 f   U2Lang:U2Lang.dll
 0001:000187ca       ?getActorId@BaseWorker@LocalWorkflow@U2@@UBE?AVQString@@XZ 100197ca f   U2Lang:U2Lang.dll
 0001:000187d0       ?getAffectResult@VisibilityRelation@U2@@UBE?AVQVariant@@ABV3@0PAVDelegateTags@2@1@Z 100197d0 f   U2Lang:U2Lang.dll
 0001:000187d6       ?getAllDescriptors@MapDataType@U2@@UBE?AV?$QList@VDescriptor@U2@@@@XZ 100197d6 f   U2Lang:U2Lang.dll
 0001:000187dc       ?getAllEntries@?$IdRegistry@VDomainFactory@Workflow@U2@@@U2@@UBE?AV?$QList@PAVDomainFactory@Workflow@U2@@@@XZ 100197dc f   U2Lang:U2Lang.dll
 0001:000187e2       ?getAllIds@?$IdRegistry@VDomainFactory@Workflow@U2@@@U2@@UBE?AV?$QList@VQString@@@@XZ 100197e2 f   U2Lang:U2Lang.dll
 0001:000187e8       ?getAttributePureValue@Attribute@U2@@UBEABVQVariant@@XZ 100197e8 f   U2Lang:U2Lang.dll
 0001:000187ee       ?getById@?$IdRegistry@VDomainFactory@Workflow@U2@@@U2@@UAEPAVDomainFactory@Workflow@2@ABVQString@@@Z 100197ee f   U2Lang:U2Lang.dll
 0001:000187f4       ?getCommunication@BaseWorker@LocalWorkflow@U2@@UAEPAVCommunicationChannel@Workflow@3@ABVQString@@@Z 100197f4 f   U2Lang:U2Lang.dll
 0001:000187fa       ?getDatatypeByDescriptor@MapDataType@U2@@UBE?AV?$QExplicitlySharedDataPointer@VDataType@U2@@@@ABVDescriptor@2@@Z 100197fa f   U2Lang:U2Lang.dll
 0001:00018800       ?getDatatypesMap@MapDataType@U2@@UBE?AV?$QMap@VDescriptor@U2@@V?$QExplicitlySharedDataPointer@VDataType@U2@@@@@@XZ 10019800 f   U2Lang:U2Lang.dll
 0001:00018806       ?getDefaultPureValue@Attribute@U2@@UBEABVQVariant@@XZ 10019806 f   U2Lang:U2Lang.dll
 0001:0001880c       ?getField@PropertyWidget@U2@@UAEPAVQWidget@@XZ 1001980c f   U2Lang:U2Lang.dll
 0001:00018812       ?getGroup@Attribute@U2@@UAE?AW4AttributeGroup@2@XZ 10019812 f   U2Lang:U2Lang.dll
 0001:00018818       ?getItems@PropertyDelegate@U2@@UBEXAAV?$QMap@VQString@@VQVariant@@@@@Z 10019818 f   U2Lang:U2Lang.dll
 0001:0001881e       ?getMessageAndSetupScriptValues@BaseWorker@LocalWorkflow@U2@@UAE?AVMessage@Workflow@3@PAVCommunicationChannel@53@@Z 1001981e f   U2Lang:U2Lang.dll
 0001:00018824       ?getOutputFiles@BaseWorker@LocalWorkflow@U2@@UAE?AVQStringList@@XZ 10019824 f   U2Lang:U2Lang.dll
 0001:0001882a       ?getType@PortDescriptor@Workflow@U2@@UBE?AV?$QExplicitlySharedDataPointer@VDataType@U2@@@@XZ 1001982a f   U2Lang:U2Lang.dll
 0001:00018830       ?getType@VisibilityRelation@U2@@UBE?AW4RelationType@2@XZ 10019830 f   U2Lang:U2Lang.dll
 0001:00018836       ?getWidget@ConfigurationEditor@U2@@UAEPAVQWidget@@XZ 10019836 f   U2Lang:U2Lang.dll
 0001:0001883c       ?isAcceptableDrop@ActorPrototype@Workflow@U2@@UBE_NPBVQMimeData@@PAV?$QMap@VQString@@VQVariant@@@@@Z 1001983c f   U2Lang:U2Lang.dll
 0001:00018842       ?isDefaultValue@Attribute@U2@@UBE_NXZ 10019842 f   U2Lang:U2Lang.dll
 0001:00018848       ?isDone@BaseWorker@LocalWorkflow@U2@@UBE_NXZ 10019848 f   U2Lang:U2Lang.dll
 0001:0001884e       ?isEmpty@Attribute@U2@@UBE_NXZ 1001984e f   U2Lang:U2Lang.dll
 0001:00018854       ?isEmpty@ConfigurationEditor@U2@@UBE_NXZ 10019854 f   U2Lang:U2Lang.dll
 0001:0001885a       ?isPortEnabled@PortRelationDescriptor@U2@@UBE_NABVQVariant@@@Z 1001985a f   U2Lang:U2Lang.dll
 0001:00018860       ?kind@MapDataType@U2@@UBE?AW4Kind@DataType@2@XZ 10019860 f   U2Lang:U2Lang.dll
 0001:00018866       ?metaObject@ActorPrototype@Workflow@U2@@UBEPBUQMetaObject@@XZ 10019866 f   U2Lang:U2Lang.dll
 0001:0001886c       ?metaObject@PrompterBaseImpl@U2@@UBEPBUQMetaObject@@XZ 1001986c f   U2Lang:U2Lang.dll
 0001:00018872       ?metaObject@PropertyDelegate@U2@@UBEPBUQMetaObject@@XZ 10019872 f   U2Lang:U2Lang.dll
 0001:00018878       ?processDelegateTags@PropertyWidget@U2@@UAEXXZ 10019878 f   U2Lang:U2Lang.dll
 0001:0001887e       ?qt_metacall@ActorPrototype@Workflow@U2@@UAEHW4Call@QMetaObject@@HPAPAX@Z 1001987e f   U2Lang:U2Lang.dll
 0001:00018884       ?qt_metacall@PrompterBaseImpl@U2@@UAEHW4Call@QMetaObject@@HPAPAX@Z 10019884 f   U2Lang:U2Lang.dll
 0001:0001888a       ?qt_metacall@PropertyDelegate@U2@@UAEHW4Call@QMetaObject@@HPAPAX@Z 1001988a f   U2Lang:U2Lang.dll
 0001:00018890       ?qt_metacast@ActorPrototype@Workflow@U2@@UAEPAXPBD@Z 10019890 f   U2Lang:U2Lang.dll
 0001:00018896       ?qt_metacast@PrompterBaseImpl@U2@@UAEPAXPBD@Z 10019896 f   U2Lang:U2Lang.dll
 0001:0001889c       ?qt_metacast@PropertyDelegate@U2@@UAEPAXPBD@Z 1001989c f   U2Lang:U2Lang.dll
 0001:000188a2       ?registerEntry@?$IdRegistry@VDomainFactory@Workflow@U2@@@U2@@UAE_NPAVDomainFactory@Workflow@2@@Z 100198a2 f   U2Lang:U2Lang.dll
 0001:000188a8       ?setAttributeValue@Attribute@U2@@UAEXABVQVariant@@@Z 100198a8 f   U2Lang:U2Lang.dll
 0001:000188ae       ?setDisplayName@ActorPrototype@Workflow@U2@@UAEXABVQString@@@Z 100198ae f   U2Lang:U2Lang.dll
 0001:000188b4       ?setDisplayName@Descriptor@U2@@UAEXABVQString@@@Z 100198b4 f   U2Lang:U2Lang.dll
 0001:000188ba       ?setDocumentation@ActorPrototype@Workflow@U2@@UAEXABVQString@@@Z 100198ba f   U2Lang:U2Lang.dll
 0001:000188c0       ?setDocumentation@Descriptor@U2@@UAEXABVQString@@@Z 100198c0 f   U2Lang:U2Lang.dll
 0001:000188c6       ?setDone@BaseWorker@LocalWorkflow@U2@@UAEXXZ 100198c6 f   U2Lang:U2Lang.dll
 0001:000188cc       ?setRequired@PropertyWidget@U2@@UAEXXZ 100198cc f   U2Lang:U2Lang.dll
 0001:000188d2       ?setVisibleSlot@PortDescriptor@Workflow@U2@@UAEXABVQString@@_N@Z 100198d2 f   U2Lang:U2Lang.dll
 0001:000188d8       ?sl_actorModified@PrompterBaseImpl@U2@@MAEXXZ 100198d8 f   U2Lang:U2Lang.dll
 0001:000188de       ?type@PropertyDelegate@U2@@UBE?AW4Type@12@XZ 100198de f   U2Lang:U2Lang.dll
 0001:000188e4       ?unregisterEntry@?$IdRegistry@VDomainFactory@Workflow@U2@@@U2@@UAEPAVDomainFactory@Workflow@2@ABVQString@@@Z 100198e4 f   U2Lang:U2Lang.dll
 0001:000188ea       ?update@PrompterBaseImpl@U2@@UAEXABV?$QMap@VQString@@VQVariant@@@@@Z 100198ea f   U2Lang:U2Lang.dll
 0001:000188f0       ?update@PropertyDelegate@U2@@UAEXXZ 100198f0 f   U2Lang:U2Lang.dll
 0001:000188f6       ?updateActorIds@Attribute@U2@@UAEXABV?$QMap@VQString@@V1@@@@Z 100198f6 f   U2Lang:U2Lang.dll
 0001:000188fc       ?updateDelegateTags@AttributeRelation@U2@@UBEXABVQVariant@@PAVDelegateTags@2@@Z 100198fc f   U2Lang:U2Lang.dll
 0001:00018902       ?validate@Attribute@U2@@UAE_NAAV?$QList@VWorkflowNotification@U2@@@@@Z 10019902 f   U2Lang:U2Lang.dll
 0001:00018908       ?valueChangingRelation@VisibilityRelation@U2@@UBE_NXZ 10019908 f   U2Lang:U2Lang.dll
 0001:0001890e       ?qt_metacast@PropertyWidget@U2@@UAEPAXPBD@Z 1001990e f   U2Lang:U2Lang.dll
 0001:00018914       ?qt_metacall@PropertyWidget@U2@@UAEHW4Call@QMetaObject@@HPAPAX@Z 10019914 f   U2Lang:U2Lang.dll
 0001:0001891a       ?qt_metacast@BaseWorker@LocalWorkflow@U2@@UAEPAXPBD@Z 1001991a f   U2Lang:U2Lang.dll
 0001:00018920       ?qt_metacall@BaseWorker@LocalWorkflow@U2@@UAEHW4Call@QMetaObject@@HPAPAX@Z 10019920 f   U2Lang:U2Lang.dll
 0001:00018926       ??0DelegateEditor@U2@@QAE@ABV?$QMap@VQString@@PAVPropertyDelegate@U2@@@@@Z 10019926 f   U2Designer:U2Designer.dll
 0001:0001892c       ??1DelegateEditor@U2@@UAE@XZ 1001992c f   U2Designer:U2Designer.dll
 0001:00018932       ??0URLDelegate@U2@@QAE@ABVQString@@0_N11PAVQObject@@011@Z 10019932 f   U2Designer:U2Designer.dll
 0001:00018938       ??1URLDelegate@U2@@UAE@XZ  10019938 f   U2Designer:U2Designer.dll
 0001:0001893e       ??0SpinBoxDelegate@U2@@QAE@ABV?$QMap@VQString@@VQVariant@@@@PAVQObject@@@Z 1001993e f   U2Designer:U2Designer.dll
 0001:00018944       ??1SpinBoxDelegate@U2@@UAE@XZ 10019944 f   U2Designer:U2Designer.dll
 0001:0001894a       ??0DoubleSpinBoxDelegate@U2@@QAE@ABV?$QMap@VQString@@VQVariant@@@@PAVQObject@@@Z 1001994a f   U2Designer:U2Designer.dll
 0001:00018950       ??1DoubleSpinBoxDelegate@U2@@UAE@XZ 10019950 f   U2Designer:U2Designer.dll
 0001:00018956       ??0ComboBoxDelegate@U2@@QAE@ABV?$QMap@VQString@@VQVariant@@@@PAVQObject@@@Z 10019956 f   U2Designer:U2Designer.dll
 0001:0001895c       ??1ComboBoxDelegate@U2@@UAE@XZ 1001995c f   U2Designer:U2Designer.dll
 0001:00018962       ?addDelegate@DelegateEditor@U2@@UAEXPAVPropertyDelegate@2@ABVQString@@@Z 10019962 f   U2Designer:U2Designer.dll
 0001:00018968       ?clone@ComboBoxDelegate@U2@@UAEPAVPropertyDelegate@2@XZ 10019968 f   U2Designer:U2Designer.dll
 0001:0001896e       ?clone@DelegateEditor@U2@@UAEPAVConfigurationEditor@2@XZ 1001996e f   U2Designer:U2Designer.dll
 0001:00018974       ?clone@DoubleSpinBoxDelegate@U2@@UAEPAVPropertyDelegate@2@XZ 10019974 f   U2Designer:U2Designer.dll
 0001:0001897a       ?clone@SpinBoxDelegate@U2@@UAEPAVPropertyDelegate@2@XZ 1001997a f   U2Designer:U2Designer.dll
 0001:00018980       ?clone@URLDelegate@U2@@UAEPAVPropertyDelegate@2@XZ 10019980 f   U2Designer:U2Designer.dll
 0001:00018986       ?commit@DelegateEditor@U2@@UAEXXZ 10019986 f   U2Designer:U2Designer.dll
 0001:0001898c       ?createEditor@ComboBoxDelegate@U2@@UBEPAVQWidget@@PAV3@ABVQStyleOptionViewItem@@ABVQModelIndex@@@Z 1001998c f   U2Designer:U2Designer.dll
 0001:00018992       ?createEditor@DoubleSpinBoxDelegate@U2@@UBEPAVQWidget@@PAV3@ABVQStyleOptionViewItem@@ABVQModelIndex@@@Z 10019992 f   U2Designer:U2Designer.dll
 0001:00018998       ?createEditor@SpinBoxDelegate@U2@@UBEPAVQWidget@@PAV3@ABVQStyleOptionViewItem@@ABVQModelIndex@@@Z 10019998 f   U2Designer:U2Designer.dll
 0001:0001899e       ?createEditor@URLDelegate@U2@@UBEPAVQWidget@@PAV3@ABVQStyleOptionViewItem@@ABVQModelIndex@@@Z 1001999e f   U2Designer:U2Designer.dll
 0001:000189a4       ?createWizardWidget@ComboBoxDelegate@U2@@UBEPAVPropertyWidget@2@AAVU2OpStatus@2@PAVQWidget@@@Z 100199a4 f   U2Designer:U2Designer.dll
 0001:000189aa       ?createWizardWidget@DoubleSpinBoxDelegate@U2@@UBEPAVPropertyWidget@2@AAVU2OpStatus@2@PAVQWidget@@@Z 100199aa f   U2Designer:U2Designer.dll
 0001:000189b0       ?createWizardWidget@SpinBoxDelegate@U2@@UBEPAVPropertyWidget@2@AAVU2OpStatus@2@PAVQWidget@@@Z 100199b0 f   U2Designer:U2Designer.dll
 0001:000189b6       ?createWizardWidget@URLDelegate@U2@@UBEPAVPropertyWidget@2@AAVU2OpStatus@2@PAVQWidget@@@Z 100199b6 f   U2Designer:U2Designer.dll
 0001:000189bc       ?getDelegate@DelegateEditor@U2@@UAEPAVPropertyDelegate@2@ABVQString@@@Z 100199bc f   U2Designer:U2Designer.dll
 0001:000189c2       ?getDisplayValue@ComboBoxDelegate@U2@@UBE?AVQVariant@@ABV3@@Z 100199c2 f   U2Designer:U2Designer.dll
 0001:000189c8       ?getDisplayValue@DoubleSpinBoxDelegate@U2@@UBE?AVQVariant@@ABV3@@Z 100199c8 f   U2Designer:U2Designer.dll
 0001:000189ce       ?getDisplayValue@SpinBoxDelegate@U2@@UBE?AVQVariant@@ABV3@@Z 100199ce f   U2Designer:U2Designer.dll
 0001:000189d4       ?getDisplayValue@URLDelegate@U2@@UBE?AVQVariant@@ABV3@@Z 100199d4 f   U2Designer:U2Designer.dll
 0001:000189da       ?getItems@ComboBoxDelegate@U2@@UBEXAAV?$QMap@VQString@@VQVariant@@@@@Z 100199da f   U2Designer:U2Designer.dll
 0001:000189e0       ?getItems@DoubleSpinBoxDelegate@U2@@UBEXAAV?$QMap@VQString@@VQVariant@@@@@Z 100199e0 f   U2Designer:U2Designer.dll
 0001:000189e6       ?getItems@SpinBoxDelegate@U2@@UBEXAAV?$QMap@VQString@@VQVariant@@@@@Z 100199e6 f   U2Designer:U2Designer.dll
 0001:000189ec       ?metaObject@ComboBoxDelegate@U2@@UBEPBUQMetaObject@@XZ 100199ec f   U2Designer:U2Designer.dll
 0001:000189f2       ?metaObject@DelegateEditor@U2@@UBEPBUQMetaObject@@XZ 100199f2 f   U2Designer:U2Designer.dll
 0001:000189f8       ?metaObject@DoubleSpinBoxDelegate@U2@@UBEPBUQMetaObject@@XZ 100199f8 f   U2Designer:U2Designer.dll
 0001:000189fe       ?metaObject@SpinBoxDelegate@U2@@UBEPBUQMetaObject@@XZ 100199fe f   U2Designer:U2Designer.dll
 0001:00018a04       ?metaObject@URLDelegate@U2@@UBEPBUQMetaObject@@XZ 10019a04 f   U2Designer:U2Designer.dll
 0001:00018a0a       ?qt_metacall@ComboBoxDelegate@U2@@UAEHW4Call@QMetaObject@@HPAPAX@Z 10019a0a f   U2Designer:U2Designer.dll
 0001:00018a10       ?qt_metacall@DelegateEditor@U2@@UAEHW4Call@QMetaObject@@HPAPAX@Z 10019a10 f   U2Designer:U2Designer.dll
 0001:00018a16       ?qt_metacall@DoubleSpinBoxDelegate@U2@@UAEHW4Call@QMetaObject@@HPAPAX@Z 10019a16 f   U2Designer:U2Designer.dll
 0001:00018a1c       ?qt_metacall@SpinBoxDelegate@U2@@UAEHW4Call@QMetaObject@@HPAPAX@Z 10019a1c f   U2Designer:U2Designer.dll
 0001:00018a22       ?qt_metacall@URLDelegate@U2@@UAEHW4Call@QMetaObject@@HPAPAX@Z 10019a22 f   U2Designer:U2Designer.dll
 0001:00018a28       ?qt_metacast@ComboBoxDelegate@U2@@UAEPAXPBD@Z 10019a28 f   U2Designer:U2Designer.dll
 0001:00018a2e       ?qt_metacast@DelegateEditor@U2@@UAEPAXPBD@Z 10019a2e f   U2Designer:U2Designer.dll
 0001:00018a34       ?qt_metacast@DoubleSpinBoxDelegate@U2@@UAEPAXPBD@Z 10019a34 f   U2Designer:U2Designer.dll
 0001:00018a3a       ?qt_metacast@SpinBoxDelegate@U2@@UAEPAXPBD@Z 10019a3a f   U2Designer:U2Designer.dll
 0001:00018a40       ?qt_metacast@URLDelegate@U2@@UAEPAXPBD@Z 10019a40 f   U2Designer:U2Designer.dll
 0001:00018a46       ?removeDelegate@DelegateEditor@U2@@UAEPAVPropertyDelegate@2@ABVQString@@@Z 10019a46 f   U2Designer:U2Designer.dll
 0001:00018a4c       ?setEditorData@ComboBoxDelegate@U2@@UBEXPAVQWidget@@ABVQModelIndex@@@Z 10019a4c f   U2Designer:U2Designer.dll
 0001:00018a52       ?setEditorData@DoubleSpinBoxDelegate@U2@@UBEXPAVQWidget@@ABVQModelIndex@@@Z 10019a52 f   U2Designer:U2Designer.dll
 0001:00018a58       ?setEditorData@SpinBoxDelegate@U2@@UBEXPAVQWidget@@ABVQModelIndex@@@Z 10019a58 f   U2Designer:U2Designer.dll
 0001:00018a5e       ?setEditorData@URLDelegate@U2@@UBEXPAVQWidget@@ABVQModelIndex@@@Z 10019a5e f   U2Designer:U2Designer.dll
 0001:00018a64       ?setModelData@ComboBoxDelegate@U2@@UBEXPAVQWidget@@PAVQAbstractItemModel@@ABVQModelIndex@@@Z 10019a64 f   U2Designer:U2Designer.dll
 0001:00018a6a       ?setModelData@DoubleSpinBoxDelegate@U2@@UBEXPAVQWidget@@PAVQAbstractItemModel@@ABVQModelIndex@@@Z 10019a6a f   U2Designer:U2Designer.dll
 0001:00018a70       ?setModelData@SpinBoxDelegate@U2@@UBEXPAVQWidget@@PAVQAbstractItemModel@@ABVQModelIndex@@@Z 10019a70 f   U2Designer:U2Designer.dll
 0001:00018a76       ?setModelData@URLDelegate@U2@@UBEXPAVQWidget@@PAVQAbstractItemModel@@ABVQModelIndex@@@Z 10019a76 f   U2Designer:U2Designer.dll
 0001:00018a7c       ?type@URLDelegate@U2@@UBE?AW4Type@PropertyDelegate@2@XZ 10019a7c f   U2Designer:U2Designer.dll
 0001:00018a82       ?updateDelegate@DelegateEditor@U2@@UAEXABVQString@@@Z 10019a82 f   U2Designer:U2Designer.dll
 0001:00018a88       ?updateDelegates@DelegateEditor@U2@@UAEXXZ 10019a88 f   U2Designer:U2Designer.dll
 0001:00018a8e       ??0QLineEdit@@QAE@PAVQWidget@@@Z 10019a8e f   Qt5Widgets:Qt5Widgets.dll
 0001:00018a94       ??1QLineEdit@@UAE@XZ       10019a94 f   Qt5Widgets:Qt5Widgets.dll
 0001:00018a9a       ?text@QLineEdit@@QBE?AVQString@@XZ 10019a9a f   Qt5Widgets:Qt5Widgets.dll
 0001:00018aa0       ?setValidator@QLineEdit@@QAEXPBVQValidator@@@Z 10019aa0 f   Qt5Widgets:Qt5Widgets.dll
 0001:00018aa6       ?setText@QLineEdit@@QAEXABVQString@@@Z 10019aa6 f   Qt5Widgets:Qt5Widgets.dll
 0001:00018aac       ?actionEvent@QWidget@@MAEXPAVQActionEvent@@@Z 10019aac f   Qt5Widgets:Qt5Widgets.dll
 0001:00018ab2       ?changeEvent@QLineEdit@@MAEXPAVQEvent@@@Z 10019ab2 f   Qt5Widgets:Qt5Widgets.dll
 0001:00018ab8       ?changeEvent@QWidget@@MAEXPAVQEvent@@@Z 10019ab8 f   Qt5Widgets:Qt5Widgets.dll
 0001:00018abe       ?closeEvent@QWidget@@MAEXPAVQCloseEvent@@@Z 10019abe f   Qt5Widgets:Qt5Widgets.dll
 0001:00018ac4       ?contextMenuEvent@QLineEdit@@MAEXPAVQContextMenuEvent@@@Z 10019ac4 f   Qt5Widgets:Qt5Widgets.dll
 0001:00018aca       ?contextMenuEvent@QWidget@@MAEXPAVQContextMenuEvent@@@Z 10019aca f   Qt5Widgets:Qt5Widgets.dll
 0001:00018ad0       ?destroyEditor@QAbstractItemDelegate@@UBEXPAVQWidget@@ABVQModelIndex@@@Z 10019ad0 f   Qt5Widgets:Qt5Widgets.dll
 0001:00018ad6       ?devType@QWidget@@UBEHXZ   10019ad6 f   Qt5Widgets:Qt5Widgets.dll
 0001:00018adc       ?dragEnterEvent@QLineEdit@@MAEXPAVQDragEnterEvent@@@Z 10019adc f   Qt5Widgets:Qt5Widgets.dll
 0001:00018ae2       ?dragEnterEvent@QWidget@@MAEXPAVQDragEnterEvent@@@Z 10019ae2 f   Qt5Widgets:Qt5Widgets.dll
 0001:00018ae8       ?dragLeaveEvent@QLineEdit@@MAEXPAVQDragLeaveEvent@@@Z 10019ae8 f   Qt5Widgets:Qt5Widgets.dll
 0001:00018aee       ?dragLeaveEvent@QWidget@@MAEXPAVQDragLeaveEvent@@@Z 10019aee f   Qt5Widgets:Qt5Widgets.dll
 0001:00018af4       ?dragMoveEvent@QLineEdit@@MAEXPAVQDragMoveEvent@@@Z 10019af4 f   Qt5Widgets:Qt5Widgets.dll
 0001:00018afa       ?dragMoveEvent@QWidget@@MAEXPAVQDragMoveEvent@@@Z 10019afa f   Qt5Widgets:Qt5Widgets.dll
 0001:00018b00       ?drawCheck@QItemDelegate@@MBEXPAVQPainter@@ABVQStyleOptionViewItem@@ABVQRect@@W4CheckState@Qt@@@Z 10019b00 f   Qt5Widgets:Qt5Widgets.dll
 0001:00018b06       ?drawDecoration@QItemDelegate@@MBEXPAVQPainter@@ABVQStyleOptionViewItem@@ABVQRect@@ABVQPixmap@@@Z 10019b06 f   Qt5Widgets:Qt5Widgets.dll
 0001:00018b0c       ?drawDisplay@QItemDelegate@@MBEXPAVQPainter@@ABVQStyleOptionViewItem@@ABVQRect@@ABVQString@@@Z 10019b0c f   Qt5Widgets:Qt5Widgets.dll
 0001:00018b12       ?drawFocus@QItemDelegate@@MBEXPAVQPainter@@ABVQStyleOptionViewItem@@ABVQRect@@@Z 10019b12 f   Qt5Widgets:Qt5Widgets.dll
 0001:00018b18       ?dropEvent@QLineEdit@@MAEXPAVQDropEvent@@@Z 10019b18 f   Qt5Widgets:Qt5Widgets.dll
 0001:00018b1e       ?dropEvent@QWidget@@MAEXPAVQDropEvent@@@Z 10019b1e f   Qt5Widgets:Qt5Widgets.dll
 0001:00018b24       ?editorEvent@QItemDelegate@@MAE_NPAVQEvent@@PAVQAbstractItemModel@@ABVQStyleOptionViewItem@@ABVQModelIndex@@@Z 10019b24 f   Qt5Widgets:Qt5Widgets.dll
 0001:00018b2a       ?enterEvent@QWidget@@MAEXPAVQEvent@@@Z 10019b2a f   Qt5Widgets:Qt5Widgets.dll
 0001:00018b30       ?event@QLineEdit@@UAE_NPAVQEvent@@@Z 10019b30 f   Qt5Widgets:Qt5Widgets.dll
 0001:00018b36       ?event@QWidget@@MAE_NPAVQEvent@@@Z 10019b36 f   Qt5Widgets:Qt5Widgets.dll
 0001:00018b3c       ?eventFilter@QItemDelegate@@MAE_NPAVQObject@@PAVQEvent@@@Z 10019b3c f   Qt5Widgets:Qt5Widgets.dll
 0001:00018b42       ?focusInEvent@QLineEdit@@MAEXPAVQFocusEvent@@@Z 10019b42 f   Qt5Widgets:Qt5Widgets.dll
 0001:00018b48       ?focusInEvent@QWidget@@MAEXPAVQFocusEvent@@@Z 10019b48 f   Qt5Widgets:Qt5Widgets.dll
 0001:00018b4e       ?focusNextPrevChild@QWidget@@MAE_N_N@Z 10019b4e f   Qt5Widgets:Qt5Widgets.dll
 0001:00018b54       ?focusOutEvent@QLineEdit@@MAEXPAVQFocusEvent@@@Z 10019b54 f   Qt5Widgets:Qt5Widgets.dll
 0001:00018b5a       ?focusOutEvent@QWidget@@MAEXPAVQFocusEvent@@@Z 10019b5a f   Qt5Widgets:Qt5Widgets.dll
 0001:00018b60       ?hasHeightForWidth@QWidget@@UBE_NXZ 10019b60 f   Qt5Widgets:Qt5Widgets.dll
 0001:00018b66       ?heightForWidth@QWidget@@UBEHH@Z 10019b66 f   Qt5Widgets:Qt5Widgets.dll
 0001:00018b6c       ?helpEvent@QAbstractItemDelegate@@UAE_NPAVQHelpEvent@@PAVQAbstractItemView@@ABVQStyleOptionViewItem@@ABVQModelIndex@@@Z 10019b6c f   Qt5Widgets:Qt5Widgets.dll
 0001:00018b72       ?hideEvent@QWidget@@MAEXPAVQHideEvent@@@Z 10019b72 f   Qt5Widgets:Qt5Widgets.dll
 0001:00018b78       ?initPainter@QWidget@@MBEXPAVQPainter@@@Z 10019b78 f   Qt5Widgets:Qt5Widgets.dll
 0001:00018b7e       ?inputMethodEvent@QLineEdit@@MAEXPAVQInputMethodEvent@@@Z 10019b7e f   Qt5Widgets:Qt5Widgets.dll
 0001:00018b84       ?inputMethodEvent@QWidget@@MAEXPAVQInputMethodEvent@@@Z 10019b84 f   Qt5Widgets:Qt5Widgets.dll
 0001:00018b8a       ?inputMethodQuery@QLineEdit@@UBE?AVQVariant@@W4InputMethodQuery@Qt@@@Z 10019b8a f   Qt5Widgets:Qt5Widgets.dll
 0001:00018b90       ?inputMethodQuery@QWidget@@UBE?AVQVariant@@W4InputMethodQuery@Qt@@@Z 10019b90 f   Qt5Widgets:Qt5Widgets.dll
 0001:00018b96       ?keyPressEvent@QLineEdit@@MAEXPAVQKeyEvent@@@Z 10019b96 f   Qt5Widgets:Qt5Widgets.dll
 0001:00018b9c       ?keyPressEvent@QWidget@@MAEXPAVQKeyEvent@@@Z 10019b9c f   Qt5Widgets:Qt5Widgets.dll
 0001:00018ba2       ?keyReleaseEvent@QWidget@@MAEXPAVQKeyEvent@@@Z 10019ba2 f   Qt5Widgets:Qt5Widgets.dll
 0001:00018ba8       ?leaveEvent@QWidget@@MAEXPAVQEvent@@@Z 10019ba8 f   Qt5Widgets:Qt5Widgets.dll
 0001:00018bae       ?metaObject@QLineEdit@@UBEPBUQMetaObject@@XZ 10019bae f   Qt5Widgets:Qt5Widgets.dll
 0001:00018bb4       ?metric@QWidget@@MBEHW4PaintDeviceMetric@QPaintDevice@@@Z 10019bb4 f   Qt5Widgets:Qt5Widgets.dll
 0001:00018bba       ?minimumSizeHint@QLineEdit@@UBE?AVQSize@@XZ 10019bba f   Qt5Widgets:Qt5Widgets.dll
 0001:00018bc0       ?minimumSizeHint@QWidget@@UBE?AVQSize@@XZ 10019bc0 f   Qt5Widgets:Qt5Widgets.dll
 0001:00018bc6       ?mouseDoubleClickEvent@QLineEdit@@MAEXPAVQMouseEvent@@@Z 10019bc6 f   Qt5Widgets:Qt5Widgets.dll
 0001:00018bcc       ?mouseDoubleClickEvent@QWidget@@MAEXPAVQMouseEvent@@@Z 10019bcc f   Qt5Widgets:Qt5Widgets.dll
 0001:00018bd2       ?mouseMoveEvent@QLineEdit@@MAEXPAVQMouseEvent@@@Z 10019bd2 f   Qt5Widgets:Qt5Widgets.dll
 0001:00018bd8       ?mouseMoveEvent@QWidget@@MAEXPAVQMouseEvent@@@Z 10019bd8 f   Qt5Widgets:Qt5Widgets.dll
 0001:00018bde       ?mousePressEvent@QLineEdit@@MAEXPAVQMouseEvent@@@Z 10019bde f   Qt5Widgets:Qt5Widgets.dll
 0001:00018be4       ?mousePressEvent@QWidget@@MAEXPAVQMouseEvent@@@Z 10019be4 f   Qt5Widgets:Qt5Widgets.dll
 0001:00018bea       ?mouseReleaseEvent@QLineEdit@@MAEXPAVQMouseEvent@@@Z 10019bea f   Qt5Widgets:Qt5Widgets.dll
 0001:00018bf0       ?mouseReleaseEvent@QWidget@@MAEXPAVQMouseEvent@@@Z 10019bf0 f   Qt5Widgets:Qt5Widgets.dll
 0001:00018bf6       ?moveEvent@QWidget@@MAEXPAVQMoveEvent@@@Z 10019bf6 f   Qt5Widgets:Qt5Widgets.dll
 0001:00018bfc       ?nativeEvent@QWidget@@MAE_NABVQByteArray@@PAXPAJ@Z 10019bfc f   Qt5Widgets:Qt5Widgets.dll
 0001:00018c02       ?paint@QItemDelegate@@UBEXPAVQPainter@@ABVQStyleOptionViewItem@@ABVQModelIndex@@@Z 10019c02 f   Qt5Widgets:Qt5Widgets.dll
 0001:00018c08       ?paintEngine@QWidget@@UBEPAVQPaintEngine@@XZ 10019c08 f   Qt5Widgets:Qt5Widgets.dll
 0001:00018c0e       ?paintEvent@QLineEdit@@MAEXPAVQPaintEvent@@@Z 10019c0e f   Qt5Widgets:Qt5Widgets.dll
 0001:00018c14       ?paintEvent@QWidget@@MAEXPAVQPaintEvent@@@Z 10019c14 f   Qt5Widgets:Qt5Widgets.dll
 0001:00018c1a       ?paintingRoles@QAbstractItemDelegate@@UBE?AV?$QVector@H@@XZ 10019c1a f   Qt5Widgets:Qt5Widgets.dll
 0001:00018c20       ?qt_metacall@QLineEdit@@UAEHW4Call@QMetaObject@@HPAPAX@Z 10019c20 f   Qt5Widgets:Qt5Widgets.dll
 0001:00018c26       ?qt_metacast@QLineEdit@@UAEPAXPBD@Z 10019c26 f   Qt5Widgets:Qt5Widgets.dll
 0001:00018c2c       ?redirected@QWidget@@MBEPAVQPaintDevice@@PAVQPoint@@@Z 10019c2c f   Qt5Widgets:Qt5Widgets.dll
 0001:00018c32       ?resizeEvent@QWidget@@MAEXPAVQResizeEvent@@@Z 10019c32 f   Qt5Widgets:Qt5Widgets.dll
 0001:00018c38       ?setVisible@QWidget@@UAEX_N@Z 10019c38 f   Qt5Widgets:Qt5Widgets.dll
 0001:00018c3e       ?sharedPainter@QWidget@@MBEPAVQPainter@@XZ 10019c3e f   Qt5Widgets:Qt5Widgets.dll
 0001:00018c44       ?showEvent@QWidget@@MAEXPAVQShowEvent@@@Z 10019c44 f   Qt5Widgets:Qt5Widgets.dll
 0001:00018c4a       ?sizeHint@QItemDelegate@@UBE?AVQSize@@ABVQStyleOptionViewItem@@ABVQModelIndex@@@Z 10019c4a f   Qt5Widgets:Qt5Widgets.dll
 0001:00018c50       ?sizeHint@QLineEdit@@UBE?AVQSize@@XZ 10019c50 f   Qt5Widgets:Qt5Widgets.dll
 0001:00018c56       ?sizeHint@QWidget@@UBE?AVQSize@@XZ 10019c56 f   Qt5Widgets:Qt5Widgets.dll
 0001:00018c5c       ?tabletEvent@QWidget@@MAEXPAVQTabletEvent@@@Z 10019c5c f   Qt5Widgets:Qt5Widgets.dll
 0001:00018c62       ?updateEditorGeometry@QItemDelegate@@UBEXPAVQWidget@@ABVQStyleOptionViewItem@@ABVQModelIndex@@@Z 10019c62 f   Qt5Widgets:Qt5Widgets.dll
 0001:00018c68       ?wheelEvent@QWidget@@MAEXPAVQWheelEvent@@@Z 10019c68 f   Qt5Widgets:Qt5Widgets.dll
 0001:00018c6e       ??0QDoubleValidator@@QAE@PAVQObject@@@Z 10019c6e f   Qt5Gui:Qt5Gui.dll
 0001:00018c74       ??1QDoubleValidator@@UAE@XZ 10019c74 f   Qt5Gui:Qt5Gui.dll
 0001:00018c7a       ?setNotation@QDoubleValidator@@QAEXW4Notation@1@@Z 10019c7a f   Qt5Gui:Qt5Gui.dll
 0001:00018c80       ?clear@QTextDocument@@UAEXXZ 10019c80 f   Qt5Gui:Qt5Gui.dll
 0001:00018c86       ?createObject@QTextDocument@@MAEPAVQTextObject@@ABVQTextFormat@@@Z 10019c86 f   Qt5Gui:Qt5Gui.dll
 0001:00018c8c       ?fixup@QValidator@@UBEXAAVQString@@@Z 10019c8c f   Qt5Gui:Qt5Gui.dll
 0001:00018c92       ?loadResource@QTextDocument@@MAE?AVQVariant@@HABVQUrl@@@Z 10019c92 f   Qt5Gui:Qt5Gui.dll
 0001:00018c98       ?metaObject@QDoubleValidator@@UBEPBUQMetaObject@@XZ 10019c98 f   Qt5Gui:Qt5Gui.dll
 0001:00018c9e       ?qt_metacall@QDoubleValidator@@UAEHW4Call@QMetaObject@@HPAPAX@Z 10019c9e f   Qt5Gui:Qt5Gui.dll
 0001:00018ca4       ?qt_metacast@QDoubleValidator@@UAEPAXPBD@Z 10019ca4 f   Qt5Gui:Qt5Gui.dll
 0001:00018caa       ?setRange@QDoubleValidator@@UAEXNNH@Z 10019caa f   Qt5Gui:Qt5Gui.dll
 0001:00018cb0       ?validate@QDoubleValidator@@UBE?AW4State@QValidator@@AAVQString@@AAH@Z 10019cb0 f   Qt5Gui:Qt5Gui.dll
 0001:00018cb6       ??0QScriptValue@@QAE@XZ    10019cb6 f   Qt5Script:Qt5Script.dll
 0001:00018cbc       ??1QScriptValue@@QAE@XZ    10019cbc f   Qt5Script:Qt5Script.dll
 0001:00018cc2       ??0QScriptValue@@QAE@ABV0@@Z 10019cc2 f   Qt5Script:Qt5Script.dll
 0001:00018cc8       ??4QScriptValue@@QAEAAV0@ABV0@@Z 10019cc8 f   Qt5Script:Qt5Script.dll
 0001:00018cce       ?isNumber@QScriptValue@@QBE_NXZ 10019cce f   Qt5Script:Qt5Script.dll
 0001:00018cd4       ?isString@QScriptValue@@QBE_NXZ 10019cd4 f   Qt5Script:Qt5Script.dll
 0001:00018cda       ?toString@QScriptValue@@QBE?AVQString@@XZ 10019cda f   Qt5Script:Qt5Script.dll
 0001:00018ce0       ?toInt32@QScriptValue@@QBEHXZ 10019ce0 f   Qt5Script:Qt5Script.dll
 0001:00018ce6       ??1QScriptEngine@@UAE@XZ   10019ce6 f   Qt5Script:Qt5Script.dll
 0001:00018cec       ?newVariant@QScriptEngine@@QAE?AVQScriptValue@@ABVQVariant@@@Z 10019cec f   Qt5Script:Qt5Script.dll
 0001:00018cf2       ??0QChar@@QAE@UQLatin1Char@@@Z 10019cf2 f   Qt5Core:Qt5Core.dll
 0001:00018cf8       ??0QByteArray@@QAE@ABV0@@Z 10019cf8 f   Qt5Core:Qt5Core.dll
 0001:00018cfe       ??1QByteArray@@QAE@XZ      10019cfe f   Qt5Core:Qt5Core.dll
 0001:00018d04       ??0QString@@QAE@XZ         10019d04 f   Qt5Core:Qt5Core.dll
 0001:00018d0a       ??0QString@@QAE@ABV0@@Z    10019d0a f   Qt5Core:Qt5Core.dll
 0001:00018d10       ??1QString@@QAE@XZ         10019d10 f   Qt5Core:Qt5Core.dll
 0001:00018d16       ?arg@QString@@QBE?AV1@HHHVQChar@@@Z 10019d16 f   Qt5Core:Qt5Core.dll
 0001:00018d1c       ?arg@QString@@QBE?AV1@ABV1@HVQChar@@@Z 10019d1c f   Qt5Core:Qt5Core.dll
 0001:00018d22       ?append@QString@@QAEAAV1@ABV1@@Z 10019d22 f   Qt5Core:Qt5Core.dll
 0001:00018d28       ?number@QString@@SA?AV1@HH@Z 10019d28 f   Qt5Core:Qt5Core.dll
 0001:00018d2e       ?number@QString@@SA?AV1@NDH@Z 10019d2e f   Qt5Core:Qt5Core.dll
 0001:00018d34       ??M@YA_NABVQString@@0@Z    10019d34 f   Qt5Core:Qt5Core.dll
 0001:00018d3a       ??0QString@@QAE@ABVQByteArray@@@Z 10019d3a f   Qt5Core:Qt5Core.dll
 0001:00018d40       ?fromAscii_helper@QString@@CAPAU?$QTypedArrayData@G@@PBDH@Z 10019d40 f   Qt5Core:Qt5Core.dll
 0001:00018d46       ?tr@QMetaObject@@QBE?AVQString@@PBD0H@Z 10019d46 f   Qt5Core:Qt5Core.dll
 0001:00018d4c       ?normalizedType@QMetaObject@@SA?AVQByteArray@@PBD@Z 10019d4c f   Qt5Core:Qt5Core.dll
 0001:00018d52       ?detach@QListData@@QAEPAUData@1@H@Z 10019d52 f   Qt5Core:Qt5Core.dll
 0001:00018d58       ?detach_grow@QListData@@QAEPAUData@1@PAHH@Z 10019d58 f   Qt5Core:Qt5Core.dll
 0001:00018d5e       ?dispose@QListData@@SAXPAUData@1@@Z 10019d5e f   Qt5Core:Qt5Core.dll
 0001:00018d64       ?append@QListData@@QAEPAPAXXZ 10019d64 f   Qt5Core:Qt5Core.dll
 0001:00018d6a       ?append@QListData@@QAEPAPAXABU1@@Z 10019d6a f   Qt5Core:Qt5Core.dll
 0001:00018d70       ?registerNormalizedType@QMetaType@@SAHABVQByteArray@@P6AXPAX@ZP6APAXPBX@Z2P6APAX13@ZHV?$QFlags@W4TypeFlag@QMetaType@@@@PBUQMetaObject@@@Z 10019d70 f   Qt5Core:Qt5Core.dll
 0001:00018d76       ?registerNormalizedTypedef@QMetaType@@SAHABVQByteArray@@H@Z 10019d76 f   Qt5Core:Qt5Core.dll
 0001:00018d7c       ?exists@QFile@@SA_NABVQString@@@Z 10019d7c f   Qt5Core:Qt5Core.dll
 0001:00018d82       ??0QFileInfo@@QAE@ABVQString@@@Z 10019d82 f   Qt5Core:Qt5Core.dll
 0001:00018d88       ??1QFileInfo@@QAE@XZ       10019d88 f   Qt5Core:Qt5Core.dll
 0001:00018d8e       ?absoluteDir@QFileInfo@@QBE?AVQDir@@XZ 10019d8e f   Qt5Core:Qt5Core.dll
 0001:00018d94       ??1QDir@@QAE@XZ            10019d94 f   Qt5Core:Qt5Core.dll
 0001:00018d9a       ?absolutePath@QDir@@QBE?AVQString@@XZ 10019d9a f   Qt5Core:Qt5Core.dll
 0001:00018da0       ?mkpath@QDir@@QBE_NABVQString@@@Z 10019da0 f   Qt5Core:Qt5Core.dll
 0001:00018da6       ?exists@QDir@@QBE_NXZ      10019da6 f   Qt5Core:Qt5Core.dll
 0001:00018dac       ?freeNodeAndRebalance@QMapDataBase@@QAEXPAUQMapNodeBase@@@Z 10019dac f   Qt5Core:Qt5Core.dll
 0001:00018db2       ?recalcMostLeftNode@QMapDataBase@@QAEXXZ 10019db2 f   Qt5Core:Qt5Core.dll
 0001:00018db8       ?createNode@QMapDataBase@@QAEPAUQMapNodeBase@@HHPAU2@_N@Z 10019db8 f   Qt5Core:Qt5Core.dll
 0001:00018dbe       ?freeTree@QMapDataBase@@QAEXPAUQMapNodeBase@@H@Z 10019dbe f   Qt5Core:Qt5Core.dll
 0001:00018dc4       ?createData@QMapDataBase@@SAPAU1@XZ 10019dc4 f   Qt5Core:Qt5Core.dll
 0001:00018dca       ?freeData@QMapDataBase@@SAXPAU1@@Z 10019dca f   Qt5Core:Qt5Core.dll
 0001:00018dd0       ??0QVariant@@QAE@XZ        10019dd0 f   Qt5Core:Qt5Core.dll
 0001:00018dd6       ??1QVariant@@QAE@XZ        10019dd6 f   Qt5Core:Qt5Core.dll
 0001:00018ddc       ??0QVariant@@QAE@HPBXI@Z   10019ddc f   Qt5Core:Qt5Core.dll
 0001:00018de2       ??0QVariant@@QAE@ABV0@@Z   10019de2 f   Qt5Core:Qt5Core.dll
 0001:00018de8       ??0QVariant@@QAE@ABVQString@@@Z 10019de8 f   Qt5Core:Qt5Core.dll
 0001:00018dee       ??4QVariant@@QAEAAV0@ABV0@@Z 10019dee f   Qt5Core:Qt5Core.dll
 0001:00018df4       ??4QVariant@@QAEAAV0@$$QAV0@@Z 10019df4 f   Qt5Core:Qt5Core.dll
 0001:00018dfa       ?start@QProcess@@QAEXABVQString@@ABVQStringList@@V?$QFlags@W4OpenModeFlag@QIODevice@@@@@Z 10019dfa f   Qt5Core:Qt5Core.dll
 0001:00018e00       ?setStandardOutputFile@QProcess@@QAEXABVQString@@V?$QFlags@W4OpenModeFlag@QIODevice@@@@@Z 10019e00 f   Qt5Core:Qt5Core.dll
 0001:00018e06       ?setStandardOutputProcess@QProcess@@QAEXPAV1@@Z 10019e06 f   Qt5Core:Qt5Core.dll
 0001:00018e0c       ?waitForStarted@QProcess@@QAE_NH@Z 10019e0c f   Qt5Core:Qt5Core.dll
 0001:00018e12       ?waitForFinished@QProcess@@QAE_NH@Z 10019e12 f   Qt5Core:Qt5Core.dll
 0001:00018e18       ?exitCode@QProcess@@QBEHXZ 10019e18 f   Qt5Core:Qt5Core.dll
 0001:00018e1e       ?childEvent@QObject@@MAEXPAVQChildEvent@@@Z 10019e1e f   Qt5Core:Qt5Core.dll
 0001:00018e24       ?connectNotify@QObject@@MAEXABVQMetaMethod@@@Z 10019e24 f   Qt5Core:Qt5Core.dll
 0001:00018e2a       ?customEvent@QObject@@MAEXPAVQEvent@@@Z 10019e2a f   Qt5Core:Qt5Core.dll
 0001:00018e30       ?disconnectNotify@QObject@@MAEXABVQMetaMethod@@@Z 10019e30 f   Qt5Core:Qt5Core.dll
 0001:00018e36       ?event@QObject@@UAE_NPAVQEvent@@@Z 10019e36 f   Qt5Core:Qt5Core.dll
 0001:00018e3c       ?eventFilter@QObject@@UAE_NPAV1@PAVQEvent@@@Z 10019e3c f   Qt5Core:Qt5Core.dll
 0001:00018e42       ?timerEvent@QObject@@MAEXPAVQTimerEvent@@@Z 10019e42 f   Qt5Core:Qt5Core.dll
 0001:00018e48       ?cast@QMetaObject@@QBEPAVQObject@@PAV2@@Z 10019e48 f   Qt5Core:Qt5Core.dll
 0001:00018e4e       ??1Connection@QMetaObject@@QAE@XZ 10019e4e f   Qt5Core:Qt5Core.dll
 0001:00018e54       ??0QByteArray@@QAE@XZ      10019e54 f   Qt5Core:Qt5Core.dll
 0001:00018e5a       ??4QByteArray@@QAEAAV0@ABV0@@Z 10019e5a f   Qt5Core:Qt5Core.dll
 0001:00018e60       ??4QByteArray@@QAEAAV0@$$QAV0@@Z 10019e60 f   Qt5Core:Qt5Core.dll
 0001:00018e66       ??4QString@@QAEAAV0@ABV0@@Z 10019e66 f   Qt5Core:Qt5Core.dll
 0001:00018e6c       ??0QString@@QAE@$$QAV0@@Z  10019e6c f   Qt5Core:Qt5Core.dll
 0001:00018e72       ??4QString@@QAEAAV0@$$QAV0@@Z 10019e72 f   Qt5Core:Qt5Core.dll
 0001:00018e78       ?clear@QString@@QAEXXZ     10019e78 f   Qt5Core:Qt5Core.dll
 0001:00018e7e       ?toLatin1@QString@@QBE?AVQByteArray@@XZ 10019e7e f   Qt5Core:Qt5Core.dll
 0001:00018e84       ?fromUtf8@QString@@SA?AV1@PBDH@Z 10019e84 f   Qt5Core:Qt5Core.dll
 0001:00018e8a       ?toDouble@QString@@QBENPA_N@Z 10019e8a f   Qt5Core:Qt5Core.dll
 0001:00018e90       ??8@YA_NABVQString@@0@Z    10019e90 f   Qt5Core:Qt5Core.dll
 0001:00018e96       ?realloc@QListData@@QAEXH@Z 10019e96 f   Qt5Core:Qt5Core.dll
 0001:00018e9c       ?erase@QListData@@QAEPAPAXPAPAX@Z 10019e9c f   Qt5Core:Qt5Core.dll
 0001:00018ea2       ?connect@QObject@@QBE?AVConnection@QMetaObject@@PBV1@PBD1W4ConnectionType@Qt@@@Z 10019ea2 f   Qt5Core:Qt5Core.dll
 0001:00018ea8       ?parent@QObject@@QBEPAV1@XZ 10019ea8 f   Qt5Core:Qt5Core.dll
 0001:00018eae       ?sender@QObject@@IBEPAV1@XZ 10019eae f   Qt5Core:Qt5Core.dll
 0001:00018eb4       ?nextNode@QMapNodeBase@@QBEPBU1@XZ 10019eb4 f   Qt5Core:Qt5Core.dll
 0001:00018eba       ?free_helper@QHashData@@QAEXP6AXPAUNode@1@@Z@Z 10019eba f   Qt5Core:Qt5Core.dll
 0001:00018ec0       ??0QVariant@@QAE@H@Z       10019ec0 f   Qt5Core:Qt5Core.dll
 0001:00018ec6       ??0QVariant@@QAE@_N@Z      10019ec6 f   Qt5Core:Qt5Core.dll
 0001:00018ecc       ??0QVariant@@QAE@N@Z       10019ecc f   Qt5Core:Qt5Core.dll
 0001:00018ed2       ??0QVariant@@QAE@PBD@Z     10019ed2 f   Qt5Core:Qt5Core.dll
 0001:00018ed8       ??0QVariant@@QAE@ABV?$QMap@VQString@@VQVariant@@@@@Z 10019ed8 f   Qt5Core:Qt5Core.dll
 0001:00018ede       ?userType@QVariant@@QBEHXZ 10019ede f   Qt5Core:Qt5Core.dll
 0001:00018ee4       ?toString@QVariant@@QBE?AVQString@@XZ 10019ee4 f   Qt5Core:Qt5Core.dll
 0001:00018eea       ?toMap@QVariant@@QBE?AV?$QMap@VQString@@VQVariant@@@@XZ 10019eea f   Qt5Core:Qt5Core.dll
 0001:00018ef0       ?constData@QVariant@@QBEPBXXZ 10019ef0 f   Qt5Core:Qt5Core.dll
 0001:00018ef6       ?convert@QVariant@@QBE_NHPAX@Z 10019ef6 f   Qt5Core:Qt5Core.dll
 0001:00018efc       ?dynamicMetaObject@QObjectData@@QBEPAUQMetaObject@@XZ 10019efc f   Qt5Core:Qt5Core.dll
 0001:00018f02       ?_Xbad_alloc@std@@YAXXZ    10019f02 f   msvcprt:MSVCP120.dll
 0001:00018f08       ?_Xlength_error@std@@YAXPBD@Z 10019f08 f   msvcprt:MSVCP120.dll
 0001:00018f0e       ?_Xout_of_range@std@@YAXPBD@Z 10019f0e f   msvcprt:MSVCP120.dll
 0001:00018f14       ?_Syserror_map@std@@YAPBDH@Z 10019f14 f   msvcprt:MSVCP120.dll
 0001:00018f1a       ?_Winerror_map@std@@YAPBDH@Z 10019f1a f   msvcprt:MSVCP120.dll
 0001:00018f20       __purecall                 10019f20 f   MSVCRT:MSVCR120.dll
 0001:00018f26       ??2@YAPAXI@Z               10019f26 f   MSVCRT:MSVCR120.dll
 0001:00018f2c       ??3@YAXPAX@Z               10019f2c f   MSVCRT:MSVCR120.dll
 0001:00018f32       ___atonexitinit            10019f32 f   MSVCRT:atonexit.obj
 0001:00018f6e       __onexit                   10019f6e f   MSVCRT:atonexit.obj
 0001:00019017       _atexit                    1001a017 f   MSVCRT:atonexit.obj
 0001:0001902c       _memmove                   1001a02c f   MSVCRT:MSVCR120.dll
 0001:00019032       __hypot                    1001a032 f   MSVCRT:MSVCR120.dll
 0001:00019038       @__security_check_cookie@4 1001a038 f   MSVCRT:secchk.obj
 0001:00019048       __CxxThrowException@8      1001a048 f   MSVCRT:MSVCR120.dll
 0001:0001904e       ___CxxFrameHandler3        1001a04e f   MSVCRT:MSVCR120.dll
 0001:00019054       ___RTDynamicCast           1001a054 f   MSVCRT:MSVCR120.dll
 0001:0001905a       _memcpy                    1001a05a f   MSVCRT:MSVCR120.dll
 0001:00019060       ??0type_info@@AAE@ABV0@@Z  1001a060 f   MSVCRT:ti_inst.obj
 0001:0001906b       ??4type_info@@AAEAAV0@ABV0@@Z 1001a06b f   MSVCRT:ti_inst.obj
 0001:00019070       ??_Etype_info@@UAEPAXI@Z   1001a070 f i MSVCRT:ti_inst.obj
 0001:0001910c       _NtCurrentTeb              1001a10c f i MSVCRT:crtdll.obj
 0001:00019113       __CRT_INIT@12              1001a113 f   MSVCRT:crtdll.obj
 0001:0001930a       __DllMainCRTStartup@12     1001a30a f   MSVCRT:crtdll.obj
 0001:00019460       __lock                     1001a460 f   MSVCRT:MSVCR120.dll
 0001:00019466       __unlock                   1001a466 f   MSVCRT:MSVCR120.dll
 0001:0001946c       __calloc_crt               1001a46c f   MSVCRT:MSVCR120.dll
 0001:00019472       ___dllonexit               1001a472 f   MSVCRT:MSVCR120.dll
 0001:00019480       __SEH_prolog4              1001a480 f   MSVCRT:sehprolg4.obj
 0001:000194c5       __SEH_epilog4              1001a4c5 f   MSVCRT:sehprolg4.obj
 0001:000194d9       __except_handler4          1001a4d9 f   MSVCRT:chandler4gs.obj
 0001:000194fc       ___raise_securityfailure   1001a4fc f   MSVCRT:gs_report.obj
 0001:00019539       ___report_gsfailure        1001a539 f   MSVCRT:gs_report.obj
 0001:00019634       ___report_rangecheckfailure 1001a634 f   MSVCRT:gs_report.obj
 0001:00019640       ___report_securityfailure  1001a640 f   MSVCRT:gs_report.obj
 0001:00019710       ___report_securityfailureEx 1001a710 f   MSVCRT:gs_report.obj
 0001:00019826       ??_M@YGXPAXIHP6EX0@Z@Z     1001a826 f   MSVCRT:ehvecdtr.obj
 0001:000198ae       ?__ArrayUnwind@@YGXPAXIHP6EX0@Z@Z 1001a8ae f   MSVCRT:ehvecdtr.obj
 0001:0001990c       ??1type_info@@UAE@XZ       1001a90c f   MSVCRT:MSVCR120.dll
 0001:00019912       ___CppXcptFilter           1001a912 f   MSVCRT:MSVCR120.dll
 0001:00019918       __amsg_exit                1001a918 f   MSVCRT:MSVCR120.dll
 0001:00019920       __FindPESection            1001a920 f   MSVCRT:pesect.obj
 0001:00019970       __IsNonwritableInCurrentImage 1001a970 f   MSVCRT:pesect.obj
 0001:00019a30       __ValidateImageBase        1001aa30 f   MSVCRT:pesect.obj
 0001:00019a62       _free                      1001aa62 f   MSVCRT:MSVCR120.dll
 0001:00019a68       ___security_init_cookie    1001aa68 f   MSVCRT:gs_support.obj
 0001:00019b04       _DllMain@12                1001ab04 f   MSVCRT:dllmain.obj
 0001:00019b26       __malloc_crt               1001ab26 f   MSVCRT:MSVCR120.dll
 0001:00019b2c       __RTC_Initialize           1001ab2c f   MSVCRT:initsect.obj
 0001:00019b4c       __RTC_Terminate            1001ab4c f   MSVCRT:initsect.obj
 0001:00019b6c       __initterm                 1001ab6c f   MSVCRT:MSVCR120.dll
 0001:00019b72       __initterm_e               1001ab72 f   MSVCRT:MSVCR120.dll
 0001:00019b78       ___clean_type_info_names   1001ab78 f   MSVCRT:tncleanup.obj
 0001:00019b84       __except_handler4_common   1001ab84 f   MSVCRT:MSVCR120.dll
 0001:00019b8a       __crt_debugger_hook        1001ab8a f   MSVCRT:MSVCR120.dll
 0001:00019b90       ___crtUnhandledException   1001ab90 f   MSVCRT:MSVCR120.dll
 0001:00019b96       ___crtTerminateProcess     1001ab96 f   MSVCRT:MSVCR120.dll
 0001:00019b9c       ?terminate@@YAXXZ          1001ab9c f   MSVCRT:MSVCR120.dll
 0001:00019ba2       ___clean_type_info_names_internal 1001aba2 f   MSVCRT:MSVCR120.dll
 0001:00019ba8       _EncodePointer@4           1001aba8 f   kernel32:KERNEL32.dll
 0001:00019bae       _DecodePointer@4           1001abae f   kernel32:KERNEL32.dll
 0001:00019bb4       _IsDebuggerPresent@0       1001abb4 f   kernel32:KERNEL32.dll
 0001:00019bba       _IsProcessorFeaturePresent@4 1001abba f   kernel32:KERNEL32.dll
 0001:00019bc0       _QueryPerformanceCounter@4 1001abc0 f   kernel32:KERNEL32.dll
 0001:00019bc6       _GetCurrentProcessId@0     1001abc6 f   kernel32:KERNEL32.dll
 0001:00019bcc       _GetCurrentThreadId@0      1001abcc f   kernel32:KERNEL32.dll
 0001:00019bd2       _GetSystemTimeAsFileTime@4 1001abd2 f   kernel32:KERNEL32.dll
 0001:00019bd8       _DisableThreadLibraryCalls@4 1001abd8 f   kernel32:KERNEL32.dll
 0002:00000000       __imp__DecodePointer@4     10020000     kernel32:KERNEL32.dll
 0002:00000004       __imp__IsDebuggerPresent@0 10020004     kernel32:KERNEL32.dll
 0002:00000008       __imp__IsProcessorFeaturePresent@4 10020008     kernel32:KERNEL32.dll
 0002:0000000c       __imp__QueryPerformanceCounter@4 1002000c     kernel32:KERNEL32.dll
 0002:00000010       __imp__GetCurrentProcessId@0 10020010     kernel32:KERNEL32.dll
 0002:00000014       __imp__DisableThreadLibraryCalls@4 10020014     kernel32:KERNEL32.dll
 0002:00000018       __imp__GetSystemTimeAsFileTime@4 10020018     kernel32:KERNEL32.dll
 0002:0000001c       __imp__GetCurrentThreadId@0 1002001c     kernel32:KERNEL32.dll
 0002:00000020       __imp__EncodePointer@4     10020020     kernel32:KERNEL32.dll
 0002:00000024       \177KERNEL32_NULL_THUNK_DATA 10020024     kernel32:KERNEL32.dll
 0002:00000028       __imp_?_Syserror_map@std@@YAPBDH@Z 10020028     msvcprt:MSVCP120.dll
 0002:0000002c       __imp_?_Xout_of_range@std@@YAXPBD@Z 1002002c     msvcprt:MSVCP120.dll
 0002:00000030       __imp_?_Xlength_error@std@@YAXPBD@Z 10020030     msvcprt:MSVCP120.dll
 0002:00000034       __imp_?_Winerror_map@std@@YAPBDH@Z 10020034     msvcprt:MSVCP120.dll
 0002:00000038       __imp_?_Xbad_alloc@std@@YAXXZ 10020038     msvcprt:MSVCP120.dll
 0002:0000003c       \177MSVCP120_NULL_THUNK_DATA 1002003c     msvcprt:MSVCP120.dll
 0002:00000040       __imp__free                10020040     MSVCRT:MSVCR120.dll
 0002:00000044       __imp___malloc_crt         10020044     MSVCRT:MSVCR120.dll
 0002:00000048       __imp___initterm           10020048     MSVCRT:MSVCR120.dll
 0002:0000004c       __imp___initterm_e         1002004c     MSVCRT:MSVCR120.dll
 0002:00000050       __imp___amsg_exit          10020050     MSVCRT:MSVCR120.dll
 0002:00000054       __imp___crt_debugger_hook  10020054     MSVCRT:MSVCR120.dll
 0002:00000058       __imp____crtUnhandledException 10020058     MSVCRT:MSVCR120.dll
 0002:0000005c       __imp____crtTerminateProcess 1002005c     MSVCRT:MSVCR120.dll
 0002:00000060       __imp_?terminate@@YAXXZ    10020060     MSVCRT:MSVCR120.dll
 0002:00000064       __imp____clean_type_info_names_internal 10020064     MSVCRT:MSVCR120.dll
 0002:00000068       __imp____CppXcptFilter     10020068     MSVCRT:MSVCR120.dll
 0002:0000006c       __imp_??1type_info@@UAE@XZ 1002006c     MSVCRT:MSVCR120.dll
 0002:00000070       __imp___onexit             10020070     MSVCRT:MSVCR120.dll
 0002:00000074       __imp____dllonexit         10020074     MSVCRT:MSVCR120.dll
 0002:00000078       __imp___calloc_crt         10020078     MSVCRT:MSVCR120.dll
 0002:0000007c       __imp___unlock             1002007c     MSVCRT:MSVCR120.dll
 0002:00000080       __imp___lock               10020080     MSVCRT:MSVCR120.dll
 0002:00000084       __imp__memcpy              10020084     MSVCRT:MSVCR120.dll
 0002:00000088       __imp____RTDynamicCast     10020088     MSVCRT:MSVCR120.dll
 0002:0000008c       __imp___purecall           1002008c     MSVCRT:MSVCR120.dll
 0002:00000090       __imp____CxxFrameHandler3  10020090     MSVCRT:MSVCR120.dll
 0002:00000094       __imp___CxxThrowException@8 10020094     MSVCRT:MSVCR120.dll
 0002:00000098       __imp___hypot              10020098     MSVCRT:MSVCR120.dll
 0002:0000009c       __imp__memmove             1002009c     MSVCRT:MSVCR120.dll
 0002:000000a0       __imp_??3@YAXPAX@Z         100200a0     MSVCRT:MSVCR120.dll
 0002:000000a4       __imp___except_handler4_common 100200a4     MSVCRT:MSVCR120.dll
 0002:000000a8       __imp_??2@YAPAXI@Z         100200a8     MSVCRT:MSVCR120.dll
 0002:000000ac       \177MSVCR120_NULL_THUNK_DATA 100200ac     MSVCRT:MSVCR120.dll
 0002:000000b0       __imp_??4QVariant@@QAEAAV0@$$QAV0@@Z 100200b0     Qt5Core:Qt5Core.dll
 0002:000000b4       __imp_?start@QProcess@@QAEXABVQString@@ABVQStringList@@V?$QFlags@W4OpenModeFlag@QIODevice@@@@@Z 100200b4     Qt5Core:Qt5Core.dll
 0002:000000b8       __imp_?setStandardOutputFile@QProcess@@QAEXABVQString@@V?$QFlags@W4OpenModeFlag@QIODevice@@@@@Z 100200b8     Qt5Core:Qt5Core.dll
 0002:000000bc       __imp_?setStandardOutputProcess@QProcess@@QAEXPAV1@@Z 100200bc     Qt5Core:Qt5Core.dll
 0002:000000c0       __imp_?waitForStarted@QProcess@@QAE_NH@Z 100200c0     Qt5Core:Qt5Core.dll
 0002:000000c4       __imp_?waitForFinished@QProcess@@QAE_NH@Z 100200c4     Qt5Core:Qt5Core.dll
 0002:000000c8       __imp_?exitCode@QProcess@@QBEHXZ 100200c8     Qt5Core:Qt5Core.dll
 0002:000000cc       __imp_?childEvent@QObject@@MAEXPAVQChildEvent@@@Z 100200cc     Qt5Core:Qt5Core.dll
 0002:000000d0       __imp_?connectNotify@QObject@@MAEXABVQMetaMethod@@@Z 100200d0     Qt5Core:Qt5Core.dll
 0002:000000d4       __imp_?customEvent@QObject@@MAEXPAVQEvent@@@Z 100200d4     Qt5Core:Qt5Core.dll
 0002:000000d8       __imp_?disconnectNotify@QObject@@MAEXABVQMetaMethod@@@Z 100200d8     Qt5Core:Qt5Core.dll
 0002:000000dc       __imp_?event@QObject@@UAE_NPAVQEvent@@@Z 100200dc     Qt5Core:Qt5Core.dll
 0002:000000e0       __imp_?eventFilter@QObject@@UAE_NPAV1@PAVQEvent@@@Z 100200e0     Qt5Core:Qt5Core.dll
 0002:000000e4       __imp_?timerEvent@QObject@@MAEXPAVQTimerEvent@@@Z 100200e4     Qt5Core:Qt5Core.dll
 0002:000000e8       __imp_?shared_null@QListData@@2UData@1@B 100200e8     Qt5Core:Qt5Core.dll
 0002:000000ec       __imp_?shared_null@QMapDataBase@@2U1@B 100200ec     Qt5Core:Qt5Core.dll
 0002:000000f0       __imp_?cast@QMetaObject@@QBEPAVQObject@@PAV2@@Z 100200f0     Qt5Core:Qt5Core.dll
 0002:000000f4       __imp_??1Connection@QMetaObject@@QAE@XZ 100200f4     Qt5Core:Qt5Core.dll
 0002:000000f8       __imp_??0QByteArray@@QAE@XZ 100200f8     Qt5Core:Qt5Core.dll
 0002:000000fc       __imp_??4QByteArray@@QAEAAV0@ABV0@@Z 100200fc     Qt5Core:Qt5Core.dll
 0002:00000100       __imp_??4QByteArray@@QAEAAV0@$$QAV0@@Z 10020100     Qt5Core:Qt5Core.dll
 0002:00000104       __imp_??4QString@@QAEAAV0@ABV0@@Z 10020104     Qt5Core:Qt5Core.dll
 0002:00000108       __imp_??0QString@@QAE@$$QAV0@@Z 10020108     Qt5Core:Qt5Core.dll
 0002:0000010c       __imp_??4QString@@QAEAAV0@$$QAV0@@Z 1002010c     Qt5Core:Qt5Core.dll
 0002:00000110       __imp_??4QVariant@@QAEAAV0@ABV0@@Z 10020110     Qt5Core:Qt5Core.dll
 0002:00000114       __imp_?toLatin1@QString@@QBE?AVQByteArray@@XZ 10020114     Qt5Core:Qt5Core.dll
 0002:00000118       __imp_?fromUtf8@QString@@SA?AV1@PBDH@Z 10020118     Qt5Core:Qt5Core.dll
 0002:0000011c       __imp_?toDouble@QString@@QBENPA_N@Z 1002011c     Qt5Core:Qt5Core.dll
 0002:00000120       __imp_??8@YA_NABVQString@@0@Z 10020120     Qt5Core:Qt5Core.dll
 0002:00000124       __imp_?realloc@QListData@@QAEXH@Z 10020124     Qt5Core:Qt5Core.dll
 0002:00000128       __imp_?erase@QListData@@QAEPAPAXPAPAX@Z 10020128     Qt5Core:Qt5Core.dll
 0002:0000012c       __imp_?connect@QObject@@QBE?AVConnection@QMetaObject@@PBV1@PBD1W4ConnectionType@Qt@@@Z 1002012c     Qt5Core:Qt5Core.dll
 0002:00000130       __imp_?parent@QObject@@QBEPAV1@XZ 10020130     Qt5Core:Qt5Core.dll
 0002:00000134       __imp_?sender@QObject@@IBEPAV1@XZ 10020134     Qt5Core:Qt5Core.dll
 0002:00000138       __imp_?nextNode@QMapNodeBase@@QBEPBU1@XZ 10020138     Qt5Core:Qt5Core.dll
 0002:0000013c       __imp_?free_helper@QHashData@@QAEXP6AXPAUNode@1@@Z@Z 1002013c     Qt5Core:Qt5Core.dll
 0002:00000140       __imp_??0QVariant@@QAE@H@Z 10020140     Qt5Core:Qt5Core.dll
 0002:00000144       __imp_??0QVariant@@QAE@_N@Z 10020144     Qt5Core:Qt5Core.dll
 0002:00000148       __imp_??0QVariant@@QAE@N@Z 10020148     Qt5Core:Qt5Core.dll
 0002:0000014c       __imp_??0QVariant@@QAE@PBD@Z 1002014c     Qt5Core:Qt5Core.dll
 0002:00000150       __imp_??0QVariant@@QAE@ABV?$QMap@VQString@@VQVariant@@@@@Z 10020150     Qt5Core:Qt5Core.dll
 0002:00000154       __imp_?userType@QVariant@@QBEHXZ 10020154     Qt5Core:Qt5Core.dll
 0002:00000158       __imp_?toString@QVariant@@QBE?AVQString@@XZ 10020158     Qt5Core:Qt5Core.dll
 0002:0000015c       __imp_?toMap@QVariant@@QBE?AV?$QMap@VQString@@VQVariant@@@@XZ 1002015c     Qt5Core:Qt5Core.dll
 0002:00000160       __imp_?constData@QVariant@@QBEPBXXZ 10020160     Qt5Core:Qt5Core.dll
 0002:00000164       __imp_?convert@QVariant@@QBE_NHPAX@Z 10020164     Qt5Core:Qt5Core.dll
 0002:00000168       __imp_?shared_null@QHashData@@2U1@B 10020168     Qt5Core:Qt5Core.dll
 0002:0000016c       __imp_?dynamicMetaObject@QObjectData@@QBEPAUQMetaObject@@XZ 1002016c     Qt5Core:Qt5Core.dll
 0002:00000170       __imp_??0QVariant@@QAE@ABVQString@@@Z 10020170     Qt5Core:Qt5Core.dll
 0002:00000174       __imp_??0QVariant@@QAE@ABV0@@Z 10020174     Qt5Core:Qt5Core.dll
 0002:00000178       __imp_??0QVariant@@QAE@HPBXI@Z 10020178     Qt5Core:Qt5Core.dll
 0002:0000017c       __imp_??1QVariant@@QAE@XZ  1002017c     Qt5Core:Qt5Core.dll
 0002:00000180       __imp_??0QVariant@@QAE@XZ  10020180     Qt5Core:Qt5Core.dll
 0002:00000184       __imp_?freeData@QMapDataBase@@SAXPAU1@@Z 10020184     Qt5Core:Qt5Core.dll
 0002:00000188       __imp_?createData@QMapDataBase@@SAPAU1@XZ 10020188     Qt5Core:Qt5Core.dll
 0002:0000018c       __imp_?freeTree@QMapDataBase@@QAEXPAUQMapNodeBase@@H@Z 1002018c     Qt5Core:Qt5Core.dll
 0002:00000190       __imp_?createNode@QMapDataBase@@QAEPAUQMapNodeBase@@HHPAU2@_N@Z 10020190     Qt5Core:Qt5Core.dll
 0002:00000194       __imp_?recalcMostLeftNode@QMapDataBase@@QAEXXZ 10020194     Qt5Core:Qt5Core.dll
 0002:00000198       __imp_?freeNodeAndRebalance@QMapDataBase@@QAEXPAUQMapNodeBase@@@Z 10020198     Qt5Core:Qt5Core.dll
 0002:0000019c       __imp_?exists@QDir@@QBE_NXZ 1002019c     Qt5Core:Qt5Core.dll
 0002:000001a0       __imp_?mkpath@QDir@@QBE_NABVQString@@@Z 100201a0     Qt5Core:Qt5Core.dll
 0002:000001a4       __imp_?absolutePath@QDir@@QBE?AVQString@@XZ 100201a4     Qt5Core:Qt5Core.dll
 0002:000001a8       __imp_??1QDir@@QAE@XZ      100201a8     Qt5Core:Qt5Core.dll
 0002:000001ac       __imp_?absoluteDir@QFileInfo@@QBE?AVQDir@@XZ 100201ac     Qt5Core:Qt5Core.dll
 0002:000001b0       __imp_??1QFileInfo@@QAE@XZ 100201b0     Qt5Core:Qt5Core.dll
 0002:000001b4       __imp_??0QFileInfo@@QAE@ABVQString@@@Z 100201b4     Qt5Core:Qt5Core.dll
 0002:000001b8       __imp_?exists@QFile@@SA_NABVQString@@@Z 100201b8     Qt5Core:Qt5Core.dll
 0002:000001bc       __imp_?registerNormalizedTypedef@QMetaType@@SAHABVQByteArray@@H@Z 100201bc     Qt5Core:Qt5Core.dll
 0002:000001c0       __imp_?registerNormalizedType@QMetaType@@SAHABVQByteArray@@P6AXPAX@ZP6APAXPBX@Z2P6APAX13@ZHV?$QFlags@W4TypeFlag@QMetaType@@@@PBUQMetaObject@@@Z 100201c0     Qt5Core:Qt5Core.dll
 0002:000001c4       __imp_?append@QListData@@QAEPAPAXABU1@@Z 100201c4     Qt5Core:Qt5Core.dll
 0002:000001c8       __imp_?append@QListData@@QAEPAPAXXZ 100201c8     Qt5Core:Qt5Core.dll
 0002:000001cc       __imp_?dispose@QListData@@SAXPAUData@1@@Z 100201cc     Qt5Core:Qt5Core.dll
 0002:000001d0       __imp_?detach_grow@QListData@@QAEPAUData@1@PAHH@Z 100201d0     Qt5Core:Qt5Core.dll
 0002:000001d4       __imp_?detach@QListData@@QAEPAUData@1@H@Z 100201d4     Qt5Core:Qt5Core.dll
 0002:000001d8       __imp_?normalizedType@QMetaObject@@SA?AVQByteArray@@PBD@Z 100201d8     Qt5Core:Qt5Core.dll
 0002:000001dc       __imp_?tr@QMetaObject@@QBE?AVQString@@PBD0H@Z 100201dc     Qt5Core:Qt5Core.dll
 0002:000001e0       __imp_?fromAscii_helper@QString@@CAPAU?$QTypedArrayData@G@@PBDH@Z 100201e0     Qt5Core:Qt5Core.dll
 0002:000001e4       __imp_??0QString@@QAE@ABVQByteArray@@@Z 100201e4     Qt5Core:Qt5Core.dll
 0002:000001e8       __imp_??M@YA_NABVQString@@0@Z 100201e8     Qt5Core:Qt5Core.dll
 0002:000001ec       __imp_?number@QString@@SA?AV1@NDH@Z 100201ec     Qt5Core:Qt5Core.dll
 0002:000001f0       __imp_?number@QString@@SA?AV1@HH@Z 100201f0     Qt5Core:Qt5Core.dll
 0002:000001f4       __imp_?append@QString@@QAEAAV1@ABV1@@Z 100201f4     Qt5Core:Qt5Core.dll
 0002:000001f8       __imp_?arg@QString@@QBE?AV1@ABV1@HVQChar@@@Z 100201f8     Qt5Core:Qt5Core.dll
 0002:000001fc       __imp_?arg@QString@@QBE?AV1@HHHVQChar@@@Z 100201fc     Qt5Core:Qt5Core.dll
 0002:00000200       __imp_??1QString@@QAE@XZ   10020200     Qt5Core:Qt5Core.dll
 0002:00000204       __imp_??0QString@@QAE@ABV0@@Z 10020204     Qt5Core:Qt5Core.dll
 0002:00000208       __imp_??0QString@@QAE@XZ   10020208     Qt5Core:Qt5Core.dll
 0002:0000020c       __imp_??1QByteArray@@QAE@XZ 1002020c     Qt5Core:Qt5Core.dll
 0002:00000210       __imp_??0QByteArray@@QAE@ABV0@@Z 10020210     Qt5Core:Qt5Core.dll
 0002:00000214       __imp_??0QChar@@QAE@UQLatin1Char@@@Z 10020214     Qt5Core:Qt5Core.dll
 0002:00000218       __imp_?clear@QString@@QAEXXZ 10020218     Qt5Core:Qt5Core.dll
 0002:0000021c       \177Qt5Core_NULL_THUNK_DATA 1002021c     Qt5Core:Qt5Core.dll
 0002:00000220       __imp_?validate@QDoubleValidator@@UBE?AW4State@QValidator@@AAVQString@@AAH@Z 10020220     Qt5Gui:Qt5Gui.dll
 0002:00000224       __imp_??1QDoubleValidator@@UAE@XZ 10020224     Qt5Gui:Qt5Gui.dll
 0002:00000228       __imp_?setNotation@QDoubleValidator@@QAEXW4Notation@1@@Z 10020228     Qt5Gui:Qt5Gui.dll
 0002:0000022c       __imp_?clear@QTextDocument@@UAEXXZ 1002022c     Qt5Gui:Qt5Gui.dll
 0002:00000230       __imp_?createObject@QTextDocument@@MAEPAVQTextObject@@ABVQTextFormat@@@Z 10020230     Qt5Gui:Qt5Gui.dll
 0002:00000234       __imp_?fixup@QValidator@@UBEXAAVQString@@@Z 10020234     Qt5Gui:Qt5Gui.dll
 0002:00000238       __imp_?loadResource@QTextDocument@@MAE?AVQVariant@@HABVQUrl@@@Z 10020238     Qt5Gui:Qt5Gui.dll
 0002:0000023c       __imp_?metaObject@QDoubleValidator@@UBEPBUQMetaObject@@XZ 1002023c     Qt5Gui:Qt5Gui.dll
 0002:00000240       __imp_?qt_metacall@QDoubleValidator@@UAEHW4Call@QMetaObject@@HPAPAX@Z 10020240     Qt5Gui:Qt5Gui.dll
 0002:00000244       __imp_?qt_metacast@QDoubleValidator@@UAEPAXPBD@Z 10020244     Qt5Gui:Qt5Gui.dll
 0002:00000248       __imp_??0QDoubleValidator@@QAE@PAVQObject@@@Z 10020248     Qt5Gui:Qt5Gui.dll
 0002:0000024c       __imp_?setRange@QDoubleValidator@@UAEXNNH@Z 1002024c     Qt5Gui:Qt5Gui.dll
 0002:00000250       \177Qt5Gui_NULL_THUNK_DATA 10020250     Qt5Gui:Qt5Gui.dll
 0002:00000254       __imp_??0QScriptValue@@QAE@XZ 10020254     Qt5Script:Qt5Script.dll
 0002:00000258       __imp_??1QScriptValue@@QAE@XZ 10020258     Qt5Script:Qt5Script.dll
 0002:0000025c       __imp_??0QScriptValue@@QAE@ABV0@@Z 1002025c     Qt5Script:Qt5Script.dll
 0002:00000260       __imp_??4QScriptValue@@QAEAAV0@ABV0@@Z 10020260     Qt5Script:Qt5Script.dll
 0002:00000264       __imp_?isNumber@QScriptValue@@QBE_NXZ 10020264     Qt5Script:Qt5Script.dll
 0002:00000268       __imp_?newVariant@QScriptEngine@@QAE?AVQScriptValue@@ABVQVariant@@@Z 10020268     Qt5Script:Qt5Script.dll
 0002:0000026c       __imp_??1QScriptEngine@@UAE@XZ 1002026c     Qt5Script:Qt5Script.dll
 0002:00000270       __imp_?toString@QScriptValue@@QBE?AVQString@@XZ 10020270     Qt5Script:Qt5Script.dll
 0002:00000274       __imp_?toInt32@QScriptValue@@QBEHXZ 10020274     Qt5Script:Qt5Script.dll
 0002:00000278       __imp_?isString@QScriptValue@@QBE_NXZ 10020278     Qt5Script:Qt5Script.dll
 0002:0000027c       \177Qt5Script_NULL_THUNK_DATA 1002027c     Qt5Script:Qt5Script.dll
 0002:00000280       __imp_?dropEvent@QWidget@@MAEXPAVQDropEvent@@@Z 10020280     Qt5Widgets:Qt5Widgets.dll
 0002:00000284       __imp_?editorEvent@QItemDelegate@@MAE_NPAVQEvent@@PAVQAbstractItemModel@@ABVQStyleOptionViewItem@@ABVQModelIndex@@@Z 10020284     Qt5Widgets:Qt5Widgets.dll
 0002:00000288       __imp_?enterEvent@QWidget@@MAEXPAVQEvent@@@Z 10020288     Qt5Widgets:Qt5Widgets.dll
 0002:0000028c       __imp_?event@QLineEdit@@UAE_NPAVQEvent@@@Z 1002028c     Qt5Widgets:Qt5Widgets.dll
 0002:00000290       __imp_?event@QWidget@@MAE_NPAVQEvent@@@Z 10020290     Qt5Widgets:Qt5Widgets.dll
 0002:00000294       __imp_?eventFilter@QItemDelegate@@MAE_NPAVQObject@@PAVQEvent@@@Z 10020294     Qt5Widgets:Qt5Widgets.dll
 0002:00000298       __imp_?focusInEvent@QLineEdit@@MAEXPAVQFocusEvent@@@Z 10020298     Qt5Widgets:Qt5Widgets.dll
 0002:0000029c       __imp_?focusInEvent@QWidget@@MAEXPAVQFocusEvent@@@Z 1002029c     Qt5Widgets:Qt5Widgets.dll
 0002:000002a0       __imp_?focusNextPrevChild@QWidget@@MAE_N_N@Z 100202a0     Qt5Widgets:Qt5Widgets.dll
 0002:000002a4       __imp_?focusOutEvent@QLineEdit@@MAEXPAVQFocusEvent@@@Z 100202a4     Qt5Widgets:Qt5Widgets.dll
 0002:000002a8       __imp_?focusOutEvent@QWidget@@MAEXPAVQFocusEvent@@@Z 100202a8     Qt5Widgets:Qt5Widgets.dll
 0002:000002ac       __imp_?hasHeightForWidth@QWidget@@UBE_NXZ 100202ac     Qt5Widgets:Qt5Widgets.dll
 0002:000002b0       __imp_?heightForWidth@QWidget@@UBEHH@Z 100202b0     Qt5Widgets:Qt5Widgets.dll
 0002:000002b4       __imp_?helpEvent@QAbstractItemDelegate@@UAE_NPAVQHelpEvent@@PAVQAbstractItemView@@ABVQStyleOptionViewItem@@ABVQModelIndex@@@Z 100202b4     Qt5Widgets:Qt5Widgets.dll
 0002:000002b8       __imp_?hideEvent@QWidget@@MAEXPAVQHideEvent@@@Z 100202b8     Qt5Widgets:Qt5Widgets.dll
 0002:000002bc       __imp_?initPainter@QWidget@@MBEXPAVQPainter@@@Z 100202bc     Qt5Widgets:Qt5Widgets.dll
 0002:000002c0       __imp_?inputMethodEvent@QLineEdit@@MAEXPAVQInputMethodEvent@@@Z 100202c0     Qt5Widgets:Qt5Widgets.dll
 0002:000002c4       __imp_?inputMethodEvent@QWidget@@MAEXPAVQInputMethodEvent@@@Z 100202c4     Qt5Widgets:Qt5Widgets.dll
 0002:000002c8       __imp_?inputMethodQuery@QLineEdit@@UBE?AVQVariant@@W4InputMethodQuery@Qt@@@Z 100202c8     Qt5Widgets:Qt5Widgets.dll
 0002:000002cc       __imp_?inputMethodQuery@QWidget@@UBE?AVQVariant@@W4InputMethodQuery@Qt@@@Z 100202cc     Qt5Widgets:Qt5Widgets.dll
 0002:000002d0       __imp_?keyPressEvent@QLineEdit@@MAEXPAVQKeyEvent@@@Z 100202d0     Qt5Widgets:Qt5Widgets.dll
 0002:000002d4       __imp_?keyPressEvent@QWidget@@MAEXPAVQKeyEvent@@@Z 100202d4     Qt5Widgets:Qt5Widgets.dll
 0002:000002d8       __imp_?keyReleaseEvent@QWidget@@MAEXPAVQKeyEvent@@@Z 100202d8     Qt5Widgets:Qt5Widgets.dll
 0002:000002dc       __imp_?leaveEvent@QWidget@@MAEXPAVQEvent@@@Z 100202dc     Qt5Widgets:Qt5Widgets.dll
 0002:000002e0       __imp_?metaObject@QLineEdit@@UBEPBUQMetaObject@@XZ 100202e0     Qt5Widgets:Qt5Widgets.dll
 0002:000002e4       __imp_?metric@QWidget@@MBEHW4PaintDeviceMetric@QPaintDevice@@@Z 100202e4     Qt5Widgets:Qt5Widgets.dll
 0002:000002e8       __imp_?minimumSizeHint@QLineEdit@@UBE?AVQSize@@XZ 100202e8     Qt5Widgets:Qt5Widgets.dll
 0002:000002ec       __imp_?minimumSizeHint@QWidget@@UBE?AVQSize@@XZ 100202ec     Qt5Widgets:Qt5Widgets.dll
 0002:000002f0       __imp_?dropEvent@QLineEdit@@MAEXPAVQDropEvent@@@Z 100202f0     Qt5Widgets:Qt5Widgets.dll
 0002:000002f4       __imp_?mouseDoubleClickEvent@QWidget@@MAEXPAVQMouseEvent@@@Z 100202f4     Qt5Widgets:Qt5Widgets.dll
 0002:000002f8       __imp_?mouseMoveEvent@QLineEdit@@MAEXPAVQMouseEvent@@@Z 100202f8     Qt5Widgets:Qt5Widgets.dll
 0002:000002fc       __imp_?mouseMoveEvent@QWidget@@MAEXPAVQMouseEvent@@@Z 100202fc     Qt5Widgets:Qt5Widgets.dll
 0002:00000300       __imp_?mousePressEvent@QLineEdit@@MAEXPAVQMouseEvent@@@Z 10020300     Qt5Widgets:Qt5Widgets.dll
 0002:00000304       __imp_?mousePressEvent@QWidget@@MAEXPAVQMouseEvent@@@Z 10020304     Qt5Widgets:Qt5Widgets.dll
 0002:00000308       __imp_?mouseReleaseEvent@QLineEdit@@MAEXPAVQMouseEvent@@@Z 10020308     Qt5Widgets:Qt5Widgets.dll
 0002:0000030c       __imp_?mouseReleaseEvent@QWidget@@MAEXPAVQMouseEvent@@@Z 1002030c     Qt5Widgets:Qt5Widgets.dll
 0002:00000310       __imp_?moveEvent@QWidget@@MAEXPAVQMoveEvent@@@Z 10020310     Qt5Widgets:Qt5Widgets.dll
 0002:00000314       __imp_?nativeEvent@QWidget@@MAE_NABVQByteArray@@PAXPAJ@Z 10020314     Qt5Widgets:Qt5Widgets.dll
 0002:00000318       __imp_?paint@QItemDelegate@@UBEXPAVQPainter@@ABVQStyleOptionViewItem@@ABVQModelIndex@@@Z 10020318     Qt5Widgets:Qt5Widgets.dll
 0002:0000031c       __imp_?paintEngine@QWidget@@UBEPAVQPaintEngine@@XZ 1002031c     Qt5Widgets:Qt5Widgets.dll
 0002:00000320       __imp_?paintEvent@QLineEdit@@MAEXPAVQPaintEvent@@@Z 10020320     Qt5Widgets:Qt5Widgets.dll
 0002:00000324       __imp_?paintEvent@QWidget@@MAEXPAVQPaintEvent@@@Z 10020324     Qt5Widgets:Qt5Widgets.dll
 0002:00000328       __imp_?paintingRoles@QAbstractItemDelegate@@UBE?AV?$QVector@H@@XZ 10020328     Qt5Widgets:Qt5Widgets.dll
 0002:0000032c       __imp_?qt_metacall@QLineEdit@@UAEHW4Call@QMetaObject@@HPAPAX@Z 1002032c     Qt5Widgets:Qt5Widgets.dll
 0002:00000330       __imp_?qt_metacast@QLineEdit@@UAEPAXPBD@Z 10020330     Qt5Widgets:Qt5Widgets.dll
 0002:00000334       __imp_?redirected@QWidget@@MBEPAVQPaintDevice@@PAVQPoint@@@Z 10020334     Qt5Widgets:Qt5Widgets.dll
 0002:00000338       __imp_?resizeEvent@QWidget@@MAEXPAVQResizeEvent@@@Z 10020338     Qt5Widgets:Qt5Widgets.dll
 0002:0000033c       __imp_?setVisible@QWidget@@UAEX_N@Z 1002033c     Qt5Widgets:Qt5Widgets.dll
 0002:00000340       __imp_?sharedPainter@QWidget@@MBEPAVQPainter@@XZ 10020340     Qt5Widgets:Qt5Widgets.dll
 0002:00000344       __imp_?showEvent@QWidget@@MAEXPAVQShowEvent@@@Z 10020344     Qt5Widgets:Qt5Widgets.dll
 0002:00000348       __imp_?sizeHint@QItemDelegate@@UBE?AVQSize@@ABVQStyleOptionViewItem@@ABVQModelIndex@@@Z 10020348     Qt5Widgets:Qt5Widgets.dll
 0002:0000034c       __imp_?sizeHint@QLineEdit@@UBE?AVQSize@@XZ 1002034c     Qt5Widgets:Qt5Widgets.dll
 0002:00000350       __imp_?sizeHint@QWidget@@UBE?AVQSize@@XZ 10020350     Qt5Widgets:Qt5Widgets.dll
 0002:00000354       __imp_?tabletEvent@QWidget@@MAEXPAVQTabletEvent@@@Z 10020354     Qt5Widgets:Qt5Widgets.dll
 0002:00000358       __imp_?updateEditorGeometry@QItemDelegate@@UBEXPAVQWidget@@ABVQStyleOptionViewItem@@ABVQModelIndex@@@Z 10020358     Qt5Widgets:Qt5Widgets.dll
 0002:0000035c       __imp_?wheelEvent@QWidget@@MAEXPAVQWheelEvent@@@Z 1002035c     Qt5Widgets:Qt5Widgets.dll
 0002:00000360       __imp_?drawFocus@QItemDelegate@@MBEXPAVQPainter@@ABVQStyleOptionViewItem@@ABVQRect@@@Z 10020360     Qt5Widgets:Qt5Widgets.dll
 0002:00000364       __imp_?drawDisplay@QItemDelegate@@MBEXPAVQPainter@@ABVQStyleOptionViewItem@@ABVQRect@@ABVQString@@@Z 10020364     Qt5Widgets:Qt5Widgets.dll
 0002:00000368       __imp_?drawDecoration@QItemDelegate@@MBEXPAVQPainter@@ABVQStyleOptionViewItem@@ABVQRect@@ABVQPixmap@@@Z 10020368     Qt5Widgets:Qt5Widgets.dll
 0002:0000036c       __imp_?drawCheck@QItemDelegate@@MBEXPAVQPainter@@ABVQStyleOptionViewItem@@ABVQRect@@W4CheckState@Qt@@@Z 1002036c     Qt5Widgets:Qt5Widgets.dll
 0002:00000370       __imp_??0QLineEdit@@QAE@PAVQWidget@@@Z 10020370     Qt5Widgets:Qt5Widgets.dll
 0002:00000374       __imp_??1QLineEdit@@UAE@XZ 10020374     Qt5Widgets:Qt5Widgets.dll
 0002:00000378       __imp_?text@QLineEdit@@QBE?AVQString@@XZ 10020378     Qt5Widgets:Qt5Widgets.dll
 0002:0000037c       __imp_?setValidator@QLineEdit@@QAEXPBVQValidator@@@Z 1002037c     Qt5Widgets:Qt5Widgets.dll
 0002:00000380       __imp_?setText@QLineEdit@@QAEXABVQString@@@Z 10020380     Qt5Widgets:Qt5Widgets.dll
 0002:00000384       __imp_?actionEvent@QWidget@@MAEXPAVQActionEvent@@@Z 10020384     Qt5Widgets:Qt5Widgets.dll
 0002:00000388       __imp_?changeEvent@QLineEdit@@MAEXPAVQEvent@@@Z 10020388     Qt5Widgets:Qt5Widgets.dll
 0002:0000038c       __imp_?changeEvent@QWidget@@MAEXPAVQEvent@@@Z 1002038c     Qt5Widgets:Qt5Widgets.dll
 0002:00000390       __imp_?closeEvent@QWidget@@MAEXPAVQCloseEvent@@@Z 10020390     Qt5Widgets:Qt5Widgets.dll
 0002:00000394       __imp_?contextMenuEvent@QLineEdit@@MAEXPAVQContextMenuEvent@@@Z 10020394     Qt5Widgets:Qt5Widgets.dll
 0002:00000398       __imp_?contextMenuEvent@QWidget@@MAEXPAVQContextMenuEvent@@@Z 10020398     Qt5Widgets:Qt5Widgets.dll
 0002:0000039c       __imp_?destroyEditor@QAbstractItemDelegate@@UBEXPAVQWidget@@ABVQModelIndex@@@Z 1002039c     Qt5Widgets:Qt5Widgets.dll
 0002:000003a0       __imp_?devType@QWidget@@UBEHXZ 100203a0     Qt5Widgets:Qt5Widgets.dll
 0002:000003a4       __imp_?dragEnterEvent@QLineEdit@@MAEXPAVQDragEnterEvent@@@Z 100203a4     Qt5Widgets:Qt5Widgets.dll
 0002:000003a8       __imp_?dragEnterEvent@QWidget@@MAEXPAVQDragEnterEvent@@@Z 100203a8     Qt5Widgets:Qt5Widgets.dll
 0002:000003ac       __imp_?dragLeaveEvent@QLineEdit@@MAEXPAVQDragLeaveEvent@@@Z 100203ac     Qt5Widgets:Qt5Widgets.dll
 0002:000003b0       __imp_?dragLeaveEvent@QWidget@@MAEXPAVQDragLeaveEvent@@@Z 100203b0     Qt5Widgets:Qt5Widgets.dll
 0002:000003b4       __imp_?dragMoveEvent@QWidget@@MAEXPAVQDragMoveEvent@@@Z 100203b4     Qt5Widgets:Qt5Widgets.dll
 0002:000003b8       __imp_?dragMoveEvent@QLineEdit@@MAEXPAVQDragMoveEvent@@@Z 100203b8     Qt5Widgets:Qt5Widgets.dll
 0002:000003bc       __imp_?mouseDoubleClickEvent@QLineEdit@@MAEXPAVQMouseEvent@@@Z 100203bc     Qt5Widgets:Qt5Widgets.dll
 0002:000003c0       \177Qt5Widgets_NULL_THUNK_DATA 100203c0     Qt5Widgets:Qt5Widgets.dll
 0002:000003c4       __imp_?getIOAdapterRegistry@AppContext@U2@@SAPAVIOAdapterRegistry@2@XZ 100203c4     U2Core:U2Core.dll
 0002:000003c8       __imp_??0Logger@U2@@QAE@ABVQString@@@Z 100203c8     U2Core:U2Core.dll
 0002:000003cc       __imp_??1Logger@U2@@UAE@XZ 100203cc     U2Core:U2Core.dll
 0002:000003d0       __imp_?details@Logger@U2@@QAEXABVQString@@@Z 100203d0     U2Core:U2Core.dll
 0002:000003d4       __imp_?error@Logger@U2@@QAEXABVQString@@@Z 100203d4     U2Core:U2Core.dll
 0002:000003d8       __imp_?addSubTask@Task@U2@@QAEXPAV12@@Z 100203d8     U2Core:U2Core.dll
 0002:000003dc       __imp_?hasError@Task@U2@@QBE_NXZ 100203dc     U2Core:U2Core.dll
 0002:000003e0       __imp_?getError@Task@U2@@QBE?AVQString@@XZ 100203e0     U2Core:U2Core.dll
 0002:000003e4       __imp_?setMaxParallelSubtasks@Task@U2@@QAEXH@Z 100203e4     U2Core:U2Core.dll
 0002:000003e8       __imp_?setError@Task@U2@@QAEXABVQString@@@Z 100203e8     U2Core:U2Core.dll
 0002:000003ec       __imp_?killProcessTree@CmdlineTaskRunner@U2@@SAHPAVQProcess@@@Z 100203ec     U2Core:U2Core.dll
 0002:000003f0       __imp_??1GCounter@U2@@UAE@XZ 100203f0     U2Core:U2Core.dll
 0002:000003f4       __imp_??0GReportableCounter@U2@@QAE@ABVQString@@0N@Z 100203f4     U2Core:U2Core.dll
 0002:000003f8       __imp_??1SimpleEventCounter@U2@@UAE@XZ 100203f8     U2Core:U2Core.dll
 0002:000003fc       __imp_??0GUrl@U2@@QAE@ABVQString@@@Z 100203fc     U2Core:U2Core.dll
 0002:00000400       __imp_??1GUrl@U2@@QAE@XZ   10020400     U2Core:U2Core.dll
 0002:00000404       __imp_??0U2DbiRef@U2@@QAE@ABVQString@@0@Z 10020404     U2Core:U2Core.dll
 0002:00000408       __imp_??1U2DbiRef@U2@@QAE@XZ 10020408     U2Core:U2Core.dll
 0002:0000040c       __imp_??0U2DbiRef@U2@@QAE@ABV01@@Z 1002040c     U2Core:U2Core.dll
 0002:00000410       __imp_??0GObjectReference@U2@@QAE@XZ 10020410     U2Core:U2Core.dll
 0002:00000414       __imp_??1GObjectReference@U2@@QAE@XZ 10020414     U2Core:U2Core.dll
 0002:00000418       __imp_?findGObjectByType@Document@U2@@QBE?AV?$QList@PAVGObject@U2@@@@VQString@@W4UnloadedObjectFilter@2@@Z 10020418     U2Core:U2Core.dll
 0002:0000041c       __imp_??1FormatDetectionResult@U2@@QAE@XZ 1002041c     U2Core:U2Core.dll
 0002:00000420       __imp_??0FormatDetectionResult@U2@@QAE@ABV01@@Z 10020420     U2Core:U2Core.dll
 0002:00000424       __imp_?detectFormat@DocumentUtils@U2@@SA?AV?$QList@VFormatDetectionResult@U2@@@@ABVGUrl@2@ABVFormatDetectionConfig@2@@Z 10020424     U2Core:U2Core.dll
 0002:00000428       __imp_?prepareTmpFileLocation@GUrlUtils@U2@@SA?AVQString@@ABV3@00AAVU2OpStatus@2@@Z 10020428     U2Core:U2Core.dll
 0002:0000042c       __imp_?url2io@IOAdapterUtils@U2@@SA?AVQString@@ABVGUrl@2@@Z 1002042c     U2Core:U2Core.dll
 0002:00000430       __imp_??0LoadDocumentTaskConfig@U2@@QAE@_NABVGObjectReference@1@PAVLDTObjectFactory@1@@Z 10020430     U2Core:U2Core.dll
 0002:00000434       __imp_??1LoadDocumentTaskConfig@U2@@QAE@XZ 10020434     U2Core:U2Core.dll
 0002:00000438       __imp_??0LoadDocumentTask@U2@@QAE@VQString@@ABVGUrl@1@PAVIOAdapterFactory@1@ABV?$QMap@VQString@@VQVariant@@@@ABVLoadDocumentTaskConfig@1@@Z 10020438     U2Core:U2Core.dll
 0002:0000043c       __imp_??1LoadDocumentTask@U2@@UAE@XZ 1002043c     U2Core:U2Core.dll
 0002:00000440       __imp_?getCurrentProcessTemporaryDirPath@UserAppsSettings@U2@@QBE?AVQString@@ABV3@@Z 10020440     U2Core:U2Core.dll
 0002:00000444       __imp_??1ProcessRun@U2@@QAE@XZ 10020444     U2Core:U2Core.dll
 0002:00000448       __imp_??0ExternalToolSupportTask@U2@@QAE@ABVQString@@V?$QFlags@W4TaskFlag@U2@@@@@Z 10020448     U2Core:U2Core.dll
 0002:0000044c       __imp_??1ExternalToolSupportTask@U2@@UAE@XZ 1002044c     U2Core:U2Core.dll
 0002:00000450       __imp_?addListeners@ExternalToolSupportTask@U2@@QAEXABV?$QList@PAVExternalToolListener@U2@@@@@Z 10020450     U2Core:U2Core.dll
 0002:00000454       __imp_?getListener@ExternalToolSupportTask@U2@@QAEPAVExternalToolListener@2@H@Z 10020454     U2Core:U2Core.dll
 0002:00000458       __imp_??0ExternalToolRunTaskHelper@U2@@QAE@PAVQProcess@@PAVExternalToolLogParser@1@AAVU2OpStatus@1@@Z 10020458     U2Core:U2Core.dll
 0002:0000045c       __imp_??1ExternalToolRunTaskHelper@U2@@UAE@XZ 1002045c     U2Core:U2Core.dll
 0002:00000460       __imp_?prepareProcess@ExternalToolSupportUtils@U2@@SA?AVProcessRun@2@ABVQString@@ABVQStringList@@01AAVU2OpStatus@2@PAVExternalToolListener@2@@Z 10020460     U2Core:U2Core.dll
 0002:00000464       __imp_?getAppSettings@AppContext@U2@@SAPAVAppSettings@2@XZ 10020464     U2Core:U2Core.dll
 0002:00000468       __imp_??0ExternalToolLogParser@U2@@QAE@_N@Z 10020468     U2Core:U2Core.dll
 0002:0000046c       __imp_??1ExternalToolLogParser@U2@@UAE@XZ 1002046c     U2Core:U2Core.dll
 0002:00000470       __imp_?cleanup@DocumentProviderTask@U2@@UAEXXZ 10020470     U2Core:U2Core.dll
 0002:00000474       __imp_?cleanup@Task@U2@@UAEXXZ 10020474     U2Core:U2Core.dll
 0002:00000478       __imp_?generateReport@Task@U2@@UBE?AVQString@@XZ 10020478     U2Core:U2Core.dll
 0002:0000047c       __imp_?getDocument@DocumentProviderTask@U2@@UAEPAVDocument@2@_N@Z 1002047c     U2Core:U2Core.dll
 0002:00000480       __imp_?getDocumentDescription@DocumentProviderTask@U2@@UBE?AVQString@@XZ 10020480     U2Core:U2Core.dll
 0002:00000484       __imp_?getNumParallelSubtasks@Task@U2@@UBEHXZ 10020484     U2Core:U2Core.dll
 0002:00000488       __imp_?getParentTask@Task@U2@@UBEPAV12@XZ 10020488     U2Core:U2Core.dll
 0002:0000048c       __imp_?getSubtaskWithErrors@Task@U2@@UBEPAV12@XZ 1002048c     U2Core:U2Core.dll
 0002:00000490       __imp_?getTaskId@Task@U2@@UBE_JXZ 10020490     U2Core:U2Core.dll
 0002:00000494       __imp_?getTopLevelParentTask@Task@U2@@UAEPAV12@XZ 10020494     U2Core:U2Core.dll
 0002:00000498       __imp_?getWarnings@Task@U2@@UBE?AVQStringList@@XZ 10020498     U2Core:U2Core.dll
 0002:0000049c       __imp_?hasSubtasksWithErrors@Task@U2@@UBE_NXZ 1002049c     U2Core:U2Core.dll
 0002:000004a0       __imp_?hasWarning@Task@U2@@UBE_NXZ 100204a0     U2Core:U2Core.dll
 0002:000004a4       __imp_?isNotificationReport@Task@U2@@UBE_NXZ 100204a4     U2Core:U2Core.dll
 0002:000004a8       __imp_?isReportingEnabled@Task@U2@@UBE_NXZ 100204a8     U2Core:U2Core.dll
 0002:000004ac       __imp_?isReportingSupported@Task@U2@@UBE_NXZ 100204ac     U2Core:U2Core.dll
 0002:000004b0       __imp_?isTopLevelTask@Task@U2@@UBE_NXZ 100204b0     U2Core:U2Core.dll
 0002:000004b4       __imp_?metaObject@LoadDocumentTask@U2@@UBEPBUQMetaObject@@XZ 100204b4     U2Core:U2Core.dll
 0002:000004b8       __imp_?onSubTaskFinished@Task@U2@@MAE?AV?$QList@PAVTask@U2@@@@PAV12@@Z 100204b8     U2Core:U2Core.dll
 0002:000004bc       __imp_?prepare@LoadDocumentTask@U2@@UAEXXZ 100204bc     U2Core:U2Core.dll
 0002:000004c0       __imp_?propagateSubtaskError@Task@U2@@UAE_NXZ 100204c0     U2Core:U2Core.dll
 0002:000004c4       __imp_?qt_metacall@LoadDocumentTask@U2@@UAEHW4Call@QMetaObject@@HPAPAX@Z 100204c4     U2Core:U2Core.dll
 0002:000004c8       __imp_?qt_metacast@LoadDocumentTask@U2@@UAEPAXPBD@Z 100204c8     U2Core:U2Core.dll
 0002:000004cc       __imp_?report@LoadDocumentTask@U2@@UAE?AW4ReportResult@Task@2@XZ 100204cc     U2Core:U2Core.dll
 0002:000004d0       __imp_?report@Task@U2@@UAE?AW4ReportResult@12@XZ 100204d0     U2Core:U2Core.dll
 0002:000004d4       __imp_?run@LoadDocumentTask@U2@@UAEXXZ 100204d4     U2Core:U2Core.dll
 0002:000004d8       __imp_?run@Task@U2@@UAEXXZ 100204d8     U2Core:U2Core.dll
 0002:000004dc       __imp_?setCollectChildrensWarningsFlag@Task@U2@@UAEX_N@Z 100204dc     U2Core:U2Core.dll
 0002:000004e0       __imp_?setListenerForHelper@ExternalToolSupportTask@U2@@MAEXPAVExternalToolRunTaskHelper@2@H@Z 100204e0     U2Core:U2Core.dll
 0002:000004e4       __imp_?setListenerForTask@ExternalToolSupportTask@U2@@MAEXPAVExternalToolRunTask@2@H@Z 100204e4     U2Core:U2Core.dll
 0002:000004e8       __imp_?setNoAutoDelete@Task@U2@@UAEX_N@Z 100204e8     U2Core:U2Core.dll
 0002:000004ec       __imp_?setNotificationReport@Task@U2@@UAEX_N@Z 100204ec     U2Core:U2Core.dll
 0002:000004f0       __imp_?setReportingEnabled@Task@U2@@UAEX_N@Z 100204f0     U2Core:U2Core.dll
 0002:000004f4       __imp_?setReportingSupported@Task@U2@@UAEX_N@Z 100204f4     U2Core:U2Core.dll
 0002:000004f8       __imp_?takeDocument@DocumentProviderTask@U2@@UAEPAVDocument@2@_N@Z 100204f8     U2Core:U2Core.dll
 0002:000004fc       __imp_??_7SimpleEventCounter@U2@@6B@ 100204fc     U2Core:U2Core.dll
 0002:00000500       __imp_?VARIANT_TRACK@GObjectTypes@U2@@2VQString@@B 10020500     U2Core:U2Core.dll
 0002:00000504       __imp_?DBI_REF_HINT@DocumentFormat@U2@@2VQString@@B 10020504     U2Core:U2Core.dll
 0002:00000508       __imp_?isCoR@U2OpStatus@U2@@UBE_NXZ 10020508     U2Core:U2Core.dll
 0002:0000050c       __imp_??0TaskStateInfo@U2@@QAE@XZ 1002050c     U2Core:U2Core.dll
 0002:00000510       __imp_?getError@TaskStateInfo@U2@@UBE?AVQString@@XZ 10020510     U2Core:U2Core.dll
 0002:00000514       __imp_?setError@TaskStateInfo@U2@@UAEXABVQString@@@Z 10020514     U2Core:U2Core.dll
 0002:00000518       __imp_??1TaskStateInfo@U2@@UAE@XZ 10020518     U2Core:U2Core.dll
 0002:0000051c       __imp_?rollFileName@GUrlUtils@U2@@SA?AVQString@@ABV3@0ABV?$QSet@VQString@@@@@Z 1002051c     U2Core:U2Core.dll
 0002:00000520       __imp_??0U2OpStatus2Log@U2@@QAE@W4LogLevel@1@@Z 10020520     U2Core:U2Core.dll
 0002:00000524       __imp_??1U2OpStatus2Log@U2@@UAE@XZ 10020524     U2Core:U2Core.dll
 0002:00000528       __imp_?runScript@ScriptTask@U2@@SA?AVQScriptValue@@PAVQScriptEngine@@ABV?$QMap@VQString@@VQScriptValue@@@@ABVQString@@AAVTaskStateInfo@2@@Z 10020528     U2Core:U2Core.dll
 0002:0000052c       __imp_?unpackMap@StrPackUtils@U2@@SA?AV?$QMap@VQString@@V1@@@ABVQString@@W4Options@12@@Z 1002052c     U2Core:U2Core.dll
 0002:00000530       __imp_??0Plugin@U2@@QAE@ABVQString@@0_NW4PluginState@1@@Z 10020530     U2Core:U2Core.dll
 0002:00000534       __imp_??1Plugin@U2@@UAE@XZ 10020534     U2Core:U2Core.dll
 0002:00000538       __imp_?qt_metacast@Task@U2@@UAEPAXPBD@Z 10020538     U2Core:U2Core.dll
 0002:0000053c       __imp_?qt_metacall@Task@U2@@UAEHW4Call@QMetaObject@@HPAPAX@Z 1002053c     U2Core:U2Core.dll
 0002:00000540       __imp_?staticMetaObject@Task@U2@@2UQMetaObject@@B 10020540     U2Core:U2Core.dll
 0002:00000544       __imp_?qt_metacast@Plugin@U2@@UAEPAXPBD@Z 10020544     U2Core:U2Core.dll
 0002:00000548       __imp_?qt_metacall@Plugin@U2@@UAEHW4Call@QMetaObject@@HPAPAX@Z 10020548     U2Core:U2Core.dll
 0002:0000054c       __imp_?staticMetaObject@Plugin@U2@@2UQMetaObject@@B 1002054c     U2Core:U2Core.dll
 0002:00000550       \177U2Core_NULL_THUNK_DATA 10020550     U2Core:U2Core.dll
 0002:00000554       __imp_?updateDelegates@DelegateEditor@U2@@UAEXXZ 10020554     U2Designer:U2Designer.dll
 0002:00000558       __imp_?updateDelegate@DelegateEditor@U2@@UAEXABVQString@@@Z 10020558     U2Designer:U2Designer.dll
 0002:0000055c       __imp_?type@URLDelegate@U2@@UBE?AW4Type@PropertyDelegate@2@XZ 1002055c     U2Designer:U2Designer.dll
 0002:00000560       __imp_?setModelData@URLDelegate@U2@@UBEXPAVQWidget@@PAVQAbstractItemModel@@ABVQModelIndex@@@Z 10020560     U2Designer:U2Designer.dll
 0002:00000564       __imp_?setModelData@SpinBoxDelegate@U2@@UBEXPAVQWidget@@PAVQAbstractItemModel@@ABVQModelIndex@@@Z 10020564     U2Designer:U2Designer.dll
 0002:00000568       __imp_?setModelData@DoubleSpinBoxDelegate@U2@@UBEXPAVQWidget@@PAVQAbstractItemModel@@ABVQModelIndex@@@Z 10020568     U2Designer:U2Designer.dll
 0002:0000056c       __imp_?setModelData@ComboBoxDelegate@U2@@UBEXPAVQWidget@@PAVQAbstractItemModel@@ABVQModelIndex@@@Z 1002056c     U2Designer:U2Designer.dll
 0002:00000570       __imp_?setEditorData@URLDelegate@U2@@UBEXPAVQWidget@@ABVQModelIndex@@@Z 10020570     U2Designer:U2Designer.dll
 0002:00000574       __imp_?setEditorData@SpinBoxDelegate@U2@@UBEXPAVQWidget@@ABVQModelIndex@@@Z 10020574     U2Designer:U2Designer.dll
 0002:00000578       __imp_?setEditorData@DoubleSpinBoxDelegate@U2@@UBEXPAVQWidget@@ABVQModelIndex@@@Z 10020578     U2Designer:U2Designer.dll
 0002:0000057c       __imp_?setEditorData@ComboBoxDelegate@U2@@UBEXPAVQWidget@@ABVQModelIndex@@@Z 1002057c     U2Designer:U2Designer.dll
 0002:00000580       __imp_?removeDelegate@DelegateEditor@U2@@UAEPAVPropertyDelegate@2@ABVQString@@@Z 10020580     U2Designer:U2Designer.dll
 0002:00000584       __imp_?qt_metacast@URLDelegate@U2@@UAEPAXPBD@Z 10020584     U2Designer:U2Designer.dll
 0002:00000588       __imp_?qt_metacast@SpinBoxDelegate@U2@@UAEPAXPBD@Z 10020588     U2Designer:U2Designer.dll
 0002:0000058c       __imp_?qt_metacast@DoubleSpinBoxDelegate@U2@@UAEPAXPBD@Z 1002058c     U2Designer:U2Designer.dll
 0002:00000590       __imp_?qt_metacast@DelegateEditor@U2@@UAEPAXPBD@Z 10020590     U2Designer:U2Designer.dll
 0002:00000594       __imp_?qt_metacast@ComboBoxDelegate@U2@@UAEPAXPBD@Z 10020594     U2Designer:U2Designer.dll
 0002:00000598       __imp_?qt_metacall@URLDelegate@U2@@UAEHW4Call@QMetaObject@@HPAPAX@Z 10020598     U2Designer:U2Designer.dll
 0002:0000059c       __imp_?qt_metacall@SpinBoxDelegate@U2@@UAEHW4Call@QMetaObject@@HPAPAX@Z 1002059c     U2Designer:U2Designer.dll
 0002:000005a0       __imp_?qt_metacall@DoubleSpinBoxDelegate@U2@@UAEHW4Call@QMetaObject@@HPAPAX@Z 100205a0     U2Designer:U2Designer.dll
 0002:000005a4       __imp_?qt_metacall@DelegateEditor@U2@@UAEHW4Call@QMetaObject@@HPAPAX@Z 100205a4     U2Designer:U2Designer.dll
 0002:000005a8       __imp_?qt_metacall@ComboBoxDelegate@U2@@UAEHW4Call@QMetaObject@@HPAPAX@Z 100205a8     U2Designer:U2Designer.dll
 0002:000005ac       __imp_?metaObject@URLDelegate@U2@@UBEPBUQMetaObject@@XZ 100205ac     U2Designer:U2Designer.dll
 0002:000005b0       __imp_?metaObject@SpinBoxDelegate@U2@@UBEPBUQMetaObject@@XZ 100205b0     U2Designer:U2Designer.dll
 0002:000005b4       __imp_?metaObject@DoubleSpinBoxDelegate@U2@@UBEPBUQMetaObject@@XZ 100205b4     U2Designer:U2Designer.dll
 0002:000005b8       __imp_?metaObject@DelegateEditor@U2@@UBEPBUQMetaObject@@XZ 100205b8     U2Designer:U2Designer.dll
 0002:000005bc       __imp_?metaObject@ComboBoxDelegate@U2@@UBEPBUQMetaObject@@XZ 100205bc     U2Designer:U2Designer.dll
 0002:000005c0       __imp_?getItems@SpinBoxDelegate@U2@@UBEXAAV?$QMap@VQString@@VQVariant@@@@@Z 100205c0     U2Designer:U2Designer.dll
 0002:000005c4       __imp_?getItems@DoubleSpinBoxDelegate@U2@@UBEXAAV?$QMap@VQString@@VQVariant@@@@@Z 100205c4     U2Designer:U2Designer.dll
 0002:000005c8       __imp_?getItems@ComboBoxDelegate@U2@@UBEXAAV?$QMap@VQString@@VQVariant@@@@@Z 100205c8     U2Designer:U2Designer.dll
 0002:000005cc       __imp_?getDisplayValue@URLDelegate@U2@@UBE?AVQVariant@@ABV3@@Z 100205cc     U2Designer:U2Designer.dll
 0002:000005d0       __imp_?getDisplayValue@SpinBoxDelegate@U2@@UBE?AVQVariant@@ABV3@@Z 100205d0     U2Designer:U2Designer.dll
 0002:000005d4       __imp_?getDisplayValue@DoubleSpinBoxDelegate@U2@@UBE?AVQVariant@@ABV3@@Z 100205d4     U2Designer:U2Designer.dll
 0002:000005d8       __imp_?getDisplayValue@ComboBoxDelegate@U2@@UBE?AVQVariant@@ABV3@@Z 100205d8     U2Designer:U2Designer.dll
 0002:000005dc       __imp_?getDelegate@DelegateEditor@U2@@UAEPAVPropertyDelegate@2@ABVQString@@@Z 100205dc     U2Designer:U2Designer.dll
 0002:000005e0       __imp_?createWizardWidget@URLDelegate@U2@@UBEPAVPropertyWidget@2@AAVU2OpStatus@2@PAVQWidget@@@Z 100205e0     U2Designer:U2Designer.dll
 0002:000005e4       __imp_?createWizardWidget@SpinBoxDelegate@U2@@UBEPAVPropertyWidget@2@AAVU2OpStatus@2@PAVQWidget@@@Z 100205e4     U2Designer:U2Designer.dll
 0002:000005e8       __imp_?createWizardWidget@DoubleSpinBoxDelegate@U2@@UBEPAVPropertyWidget@2@AAVU2OpStatus@2@PAVQWidget@@@Z 100205e8     U2Designer:U2Designer.dll
 0002:000005ec       __imp_?createWizardWidget@ComboBoxDelegate@U2@@UBEPAVPropertyWidget@2@AAVU2OpStatus@2@PAVQWidget@@@Z 100205ec     U2Designer:U2Designer.dll
 0002:000005f0       __imp_?createEditor@SpinBoxDelegate@U2@@UBEPAVQWidget@@PAV3@ABVQStyleOptionViewItem@@ABVQModelIndex@@@Z 100205f0     U2Designer:U2Designer.dll
 0002:000005f4       __imp_?createEditor@DoubleSpinBoxDelegate@U2@@UBEPAVQWidget@@PAV3@ABVQStyleOptionViewItem@@ABVQModelIndex@@@Z 100205f4     U2Designer:U2Designer.dll
 0002:000005f8       __imp_?createEditor@ComboBoxDelegate@U2@@UBEPAVQWidget@@PAV3@ABVQStyleOptionViewItem@@ABVQModelIndex@@@Z 100205f8     U2Designer:U2Designer.dll
 0002:000005fc       __imp_?commit@DelegateEditor@U2@@UAEXXZ 100205fc     U2Designer:U2Designer.dll
 0002:00000600       __imp_?clone@URLDelegate@U2@@UAEPAVPropertyDelegate@2@XZ 10020600     U2Designer:U2Designer.dll
 0002:00000604       __imp_?clone@SpinBoxDelegate@U2@@UAEPAVPropertyDelegate@2@XZ 10020604     U2Designer:U2Designer.dll
 0002:00000608       __imp_?clone@DoubleSpinBoxDelegate@U2@@UAEPAVPropertyDelegate@2@XZ 10020608     U2Designer:U2Designer.dll
 0002:0000060c       __imp_?clone@DelegateEditor@U2@@UAEPAVConfigurationEditor@2@XZ 1002060c     U2Designer:U2Designer.dll
 0002:00000610       __imp_?clone@ComboBoxDelegate@U2@@UAEPAVPropertyDelegate@2@XZ 10020610     U2Designer:U2Designer.dll
 0002:00000614       __imp_?addDelegate@DelegateEditor@U2@@UAEXPAVPropertyDelegate@2@ABVQString@@@Z 10020614     U2Designer:U2Designer.dll
 0002:00000618       __imp_??1ComboBoxDelegate@U2@@UAE@XZ 10020618     U2Designer:U2Designer.dll
 0002:0000061c       __imp_??0ComboBoxDelegate@U2@@QAE@ABV?$QMap@VQString@@VQVariant@@@@PAVQObject@@@Z 1002061c     U2Designer:U2Designer.dll
 0002:00000620       __imp_??1DoubleSpinBoxDelegate@U2@@UAE@XZ 10020620     U2Designer:U2Designer.dll
 0002:00000624       __imp_??0DoubleSpinBoxDelegate@U2@@QAE@ABV?$QMap@VQString@@VQVariant@@@@PAVQObject@@@Z 10020624     U2Designer:U2Designer.dll
 0002:00000628       __imp_??1SpinBoxDelegate@U2@@UAE@XZ 10020628     U2Designer:U2Designer.dll
 0002:0000062c       __imp_??0SpinBoxDelegate@U2@@QAE@ABV?$QMap@VQString@@VQVariant@@@@PAVQObject@@@Z 1002062c     U2Designer:U2Designer.dll
 0002:00000630       __imp_??1URLDelegate@U2@@UAE@XZ 10020630     U2Designer:U2Designer.dll
 0002:00000634       __imp_??0URLDelegate@U2@@QAE@ABVQString@@0_N11PAVQObject@@011@Z 10020634     U2Designer:U2Designer.dll
 0002:00000638       __imp_??1DelegateEditor@U2@@UAE@XZ 10020638     U2Designer:U2Designer.dll
 0002:0000063c       __imp_??0DelegateEditor@U2@@QAE@ABV?$QMap@VQString@@PAVPropertyDelegate@U2@@@@@Z 1002063c     U2Designer:U2Designer.dll
 0002:00000640       __imp_?createEditor@URLDelegate@U2@@UBEPAVQWidget@@PAV3@ABVQStyleOptionViewItem@@ABVQModelIndex@@@Z 10020640     U2Designer:U2Designer.dll
 0002:00000644       \177U2Designer_NULL_THUNK_DATA 10020644     U2Designer:U2Designer.dll
 0002:00000648       __imp_?staticMetaObject@PrompterBaseImpl@U2@@2UQMetaObject@@B 10020648     U2Lang:U2Lang.dll
 0002:0000064c       __imp_?staticMetaObject@BaseWorker@LocalWorkflow@U2@@2UQMetaObject@@B 1002064c     U2Lang:U2Lang.dll
 0002:00000650       __imp_?staticMetaObject@PropertyWidget@U2@@2UQMetaObject@@B 10020650     U2Lang:U2Lang.dll
 0002:00000654       __imp_?qt_metacall@BaseWorker@LocalWorkflow@U2@@UAEHW4Call@QMetaObject@@HPAPAX@Z 10020654     U2Lang:U2Lang.dll
 0002:00000658       __imp_?qt_metacast@BaseWorker@LocalWorkflow@U2@@UAEPAXPBD@Z 10020658     U2Lang:U2Lang.dll
 0002:0000065c       __imp_?qt_metacall@PropertyWidget@U2@@UAEHW4Call@QMetaObject@@HPAPAX@Z 1002065c     U2Lang:U2Lang.dll
 0002:00000660       __imp_?qt_metacast@PropertyWidget@U2@@UAEPAXPBD@Z 10020660     U2Lang:U2Lang.dll
 0002:00000664       __imp_?ID@LocalDomainFactory@LocalWorkflow@U2@@2VQString@@B 10020664     U2Lang:U2Lang.dll
 0002:00000668       __imp_?BUS_MAP_ATTR_ID@IntegralBusPort@Workflow@U2@@2VQString@@B 10020668     U2Lang:U2Lang.dll
 0002:0000066c       __imp_?staticMetaObject@IntegralBusPort@Workflow@U2@@2UQMetaObject@@B 1002066c     U2Lang:U2Lang.dll
 0002:00000670       __imp_??_7ConfigurationValidator@U2@@6B@ 10020670     U2Lang:U2Lang.dll
 0002:00000674       __imp_?U2_ERROR@WorkflowNotification@U2@@2VQString@@B 10020674     U2Lang:U2Lang.dll
 0002:00000678       __imp_?valueChangingRelation@VisibilityRelation@U2@@UBE_NXZ 10020678     U2Lang:U2Lang.dll
 0002:0000067c       __imp_?validate@Attribute@U2@@UAE_NAAV?$QList@VWorkflowNotification@U2@@@@@Z 1002067c     U2Lang:U2Lang.dll
 0002:00000680       __imp_?updateDelegateTags@AttributeRelation@U2@@UBEXABVQVariant@@PAVDelegateTags@2@@Z 10020680     U2Lang:U2Lang.dll
 0002:00000684       __imp_?updateActorIds@Attribute@U2@@UAEXABV?$QMap@VQString@@V1@@@@Z 10020684     U2Lang:U2Lang.dll
 0002:00000688       __imp_?update@PropertyDelegate@U2@@UAEXXZ 10020688     U2Lang:U2Lang.dll
 0002:0000068c       __imp_?update@PrompterBaseImpl@U2@@UAEXABV?$QMap@VQString@@VQVariant@@@@@Z 1002068c     U2Lang:U2Lang.dll
 0002:00000690       __imp_?unregisterEntry@?$IdRegistry@VDomainFactory@Workflow@U2@@@U2@@UAEPAVDomainFactory@Workflow@2@ABVQString@@@Z 10020690     U2Lang:U2Lang.dll
 0002:00000694       __imp_?type@PropertyDelegate@U2@@UBE?AW4Type@12@XZ 10020694     U2Lang:U2Lang.dll
 0002:00000698       __imp_?sl_actorModified@PrompterBaseImpl@U2@@MAEXXZ 10020698     U2Lang:U2Lang.dll
 0002:0000069c       __imp_?setVisibleSlot@PortDescriptor@Workflow@U2@@UAEXABVQString@@_N@Z 1002069c     U2Lang:U2Lang.dll
 0002:000006a0       __imp_?setRequired@PropertyWidget@U2@@UAEXXZ 100206a0     U2Lang:U2Lang.dll
 0002:000006a4       __imp_?setDone@BaseWorker@LocalWorkflow@U2@@UAEXXZ 100206a4     U2Lang:U2Lang.dll
 0002:000006a8       __imp_?setDocumentation@Descriptor@U2@@UAEXABVQString@@@Z 100206a8     U2Lang:U2Lang.dll
 0002:000006ac       __imp_?setDocumentation@ActorPrototype@Workflow@U2@@UAEXABVQString@@@Z 100206ac     U2Lang:U2Lang.dll
 0002:000006b0       __imp_?setDisplayName@Descriptor@U2@@UAEXABVQString@@@Z 100206b0     U2Lang:U2Lang.dll
 0002:000006b4       __imp_?setDisplayName@ActorPrototype@Workflow@U2@@UAEXABVQString@@@Z 100206b4     U2Lang:U2Lang.dll
 0002:000006b8       __imp_?setAttributeValue@Attribute@U2@@UAEXABVQVariant@@@Z 100206b8     U2Lang:U2Lang.dll
 0002:000006bc       __imp_?registerEntry@?$IdRegistry@VDomainFactory@Workflow@U2@@@U2@@UAE_NPAVDomainFactory@Workflow@2@@Z 100206bc     U2Lang:U2Lang.dll
 0002:000006c0       __imp_?qt_metacast@PropertyDelegate@U2@@UAEPAXPBD@Z 100206c0     U2Lang:U2Lang.dll
 0002:000006c4       __imp_?qt_metacast@PrompterBaseImpl@U2@@UAEPAXPBD@Z 100206c4     U2Lang:U2Lang.dll
 0002:000006c8       __imp_?qt_metacast@ActorPrototype@Workflow@U2@@UAEPAXPBD@Z 100206c8     U2Lang:U2Lang.dll
 0002:000006cc       __imp_?qt_metacall@PropertyDelegate@U2@@UAEHW4Call@QMetaObject@@HPAPAX@Z 100206cc     U2Lang:U2Lang.dll
 0002:000006d0       __imp_?qt_metacall@PrompterBaseImpl@U2@@UAEHW4Call@QMetaObject@@HPAPAX@Z 100206d0     U2Lang:U2Lang.dll
 0002:000006d4       __imp_?qt_metacall@ActorPrototype@Workflow@U2@@UAEHW4Call@QMetaObject@@HPAPAX@Z 100206d4     U2Lang:U2Lang.dll
 0002:000006d8       __imp_?processDelegateTags@PropertyWidget@U2@@UAEXXZ 100206d8     U2Lang:U2Lang.dll
 0002:000006dc       __imp_?metaObject@PropertyDelegate@U2@@UBEPBUQMetaObject@@XZ 100206dc     U2Lang:U2Lang.dll
 0002:000006e0       __imp_?metaObject@PrompterBaseImpl@U2@@UBEPBUQMetaObject@@XZ 100206e0     U2Lang:U2Lang.dll
 0002:000006e4       __imp_?metaObject@ActorPrototype@Workflow@U2@@UBEPBUQMetaObject@@XZ 100206e4     U2Lang:U2Lang.dll
 0002:000006e8       __imp_?kind@MapDataType@U2@@UBE?AW4Kind@DataType@2@XZ 100206e8     U2Lang:U2Lang.dll
 0002:000006ec       __imp_?isPortEnabled@PortRelationDescriptor@U2@@UBE_NABVQVariant@@@Z 100206ec     U2Lang:U2Lang.dll
 0002:000006f0       __imp_?isEmpty@ConfigurationEditor@U2@@UBE_NXZ 100206f0     U2Lang:U2Lang.dll
 0002:000006f4       __imp_?isEmpty@Attribute@U2@@UBE_NXZ 100206f4     U2Lang:U2Lang.dll
 0002:000006f8       __imp_?isDone@BaseWorker@LocalWorkflow@U2@@UBE_NXZ 100206f8     U2Lang:U2Lang.dll
 0002:000006fc       __imp_?isDefaultValue@Attribute@U2@@UBE_NXZ 100206fc     U2Lang:U2Lang.dll
 0002:00000700       __imp_?isAcceptableDrop@ActorPrototype@Workflow@U2@@UBE_NPBVQMimeData@@PAV?$QMap@VQString@@VQVariant@@@@@Z 10020700     U2Lang:U2Lang.dll
 0002:00000704       __imp_?getWidget@ConfigurationEditor@U2@@UAEPAVQWidget@@XZ 10020704     U2Lang:U2Lang.dll
 0002:00000708       __imp_?getType@VisibilityRelation@U2@@UBE?AW4RelationType@2@XZ 10020708     U2Lang:U2Lang.dll
 0002:0000070c       __imp_?getType@PortDescriptor@Workflow@U2@@UBE?AV?$QExplicitlySharedDataPointer@VDataType@U2@@@@XZ 1002070c     U2Lang:U2Lang.dll
 0002:00000710       __imp_?getMessageAndSetupScriptValues@BaseWorker@LocalWorkflow@U2@@UAE?AVMessage@Workflow@3@PAVCommunicationChannel@53@@Z 10020710     U2Lang:U2Lang.dll
 0002:00000714       __imp_?getItems@PropertyDelegate@U2@@UBEXAAV?$QMap@VQString@@VQVariant@@@@@Z 10020714     U2Lang:U2Lang.dll
 0002:00000718       __imp_?getGroup@Attribute@U2@@UAE?AW4AttributeGroup@2@XZ 10020718     U2Lang:U2Lang.dll
 0002:0000071c       __imp_?getField@PropertyWidget@U2@@UAEPAVQWidget@@XZ 1002071c     U2Lang:U2Lang.dll
 0002:00000720       __imp_?getDefaultPureValue@Attribute@U2@@UBEABVQVariant@@XZ 10020720     U2Lang:U2Lang.dll
 0002:00000724       __imp_?getDatatypesMap@MapDataType@U2@@UBE?AV?$QMap@VDescriptor@U2@@V?$QExplicitlySharedDataPointer@VDataType@U2@@@@@@XZ 10020724     U2Lang:U2Lang.dll
 0002:00000728       __imp_?getDatatypeByDescriptor@MapDataType@U2@@UBE?AV?$QExplicitlySharedDataPointer@VDataType@U2@@@@ABVDescriptor@2@@Z 10020728     U2Lang:U2Lang.dll
 0002:0000072c       __imp_?getCommunication@BaseWorker@LocalWorkflow@U2@@UAEPAVCommunicationChannel@Workflow@3@ABVQString@@@Z 1002072c     U2Lang:U2Lang.dll
 0002:00000730       __imp_?getById@?$IdRegistry@VDomainFactory@Workflow@U2@@@U2@@UAEPAVDomainFactory@Workflow@2@ABVQString@@@Z 10020730     U2Lang:U2Lang.dll
 0002:00000734       __imp_?getAttributePureValue@Attribute@U2@@UBEABVQVariant@@XZ 10020734     U2Lang:U2Lang.dll
 0002:00000738       __imp_?getAllIds@?$IdRegistry@VDomainFactory@Workflow@U2@@@U2@@UBE?AV?$QList@VQString@@@@XZ 10020738     U2Lang:U2Lang.dll
 0002:0000073c       __imp_?getAllEntries@?$IdRegistry@VDomainFactory@Workflow@U2@@@U2@@UBE?AV?$QList@PAVDomainFactory@Workflow@U2@@@@XZ 1002073c     U2Lang:U2Lang.dll
 0002:00000740       __imp_?getAllDescriptors@MapDataType@U2@@UBE?AV?$QList@VDescriptor@U2@@@@XZ 10020740     U2Lang:U2Lang.dll
 0002:00000744       __imp_?getAffectResult@VisibilityRelation@U2@@UBE?AVQVariant@@ABV3@0PAVDelegateTags@2@1@Z 10020744     U2Lang:U2Lang.dll
 0002:00000748       __imp_?getActorId@BaseWorker@LocalWorkflow@U2@@UBE?AVQString@@XZ 10020748     U2Lang:U2Lang.dll
 0002:0000074c       __imp_?destroy@DomainFactory@Workflow@U2@@UAEXPAVScheduler@23@PAVSchema@23@@Z 1002074c     U2Lang:U2Lang.dll
 0002:00000750       __imp_?createScheduler@DomainFactory@Workflow@U2@@UAEPAVScheduler@23@PAVSchema@23@@Z 10020750     U2Lang:U2Lang.dll
 0002:00000754       __imp_?createPort@IntegralBusActorPrototype@Workflow@U2@@UAEPAVPort@23@ABVPortDescriptor@23@PAVActor@23@@Z 10020754     U2Lang:U2Lang.dll
 0002:00000758       __imp_?createInstance@ActorPrototype@Workflow@U2@@UAEPAVActor@23@ABVQString@@PAVAttributeScript@3@ABV?$QMap@VQString@@VQVariant@@@@@Z 10020758     U2Lang:U2Lang.dll
 0002:0000075c       __imp_?createConnection@DomainFactory@Workflow@U2@@UAEPAVCommunicationChannel@23@PAVLink@23@@Z 1002075c     U2Lang:U2Lang.dll
 0002:00000760       __imp_?clone@VisibilityRelation@U2@@UBEPAV12@XZ 10020760     U2Lang:U2Lang.dll
 0002:00000764       __imp_?clone@PortRelationDescriptor@U2@@UBEPAV12@XZ 10020764     U2Lang:U2Lang.dll
 0002:00000768       __imp_?clone@Attribute@U2@@UAEPAV12@XZ 10020768     U2Lang:U2Lang.dll
 0002:0000076c       __imp_?canTaskBeCanceled@BaseWorker@LocalWorkflow@U2@@MBE_NPAVTask@3@@Z 1002076c     U2Lang:U2Lang.dll
 0002:00000770       __imp_?addCommunication@BaseWorker@LocalWorkflow@U2@@UAE_NABVQString@@PAVCommunicationChannel@Workflow@3@@Z 10020770     U2Lang:U2Lang.dll
 0002:00000774       __imp_?activate@PropertyWidget@U2@@UAEXXZ 10020774     U2Lang:U2Lang.dll
 0002:00000778       __imp_??1PrompterBaseImpl@U2@@UAE@XZ 10020778     U2Lang:U2Lang.dll
 0002:0000077c       __imp_?getHyperlink@PrompterBaseImpl@U2@@SA?AVQString@@ABV3@0@Z 1002077c     U2Lang:U2Lang.dll
 0002:00000780       __imp_?getURL@PrompterBaseImpl@U2@@QAE?AVQString@@ABV3@PA_N00@Z 10020780     U2Lang:U2Lang.dll
 0002:00000784       __imp_??0PrompterBaseImpl@U2@@QAE@PAVActor@Workflow@1@@Z 10020784     U2Lang:U2Lang.dll
 0002:00000788       __imp_?monitor@BaseWorker@LocalWorkflow@U2@@IBEPAVWorkflowMonitor@Workflow@3@XZ 10020788     U2Lang:U2Lang.dll
 0002:0000078c       __imp_?createLogListeners@BaseWorker@LocalWorkflow@U2@@QBE?AV?$QList@PAVExternalToolListener@U2@@@@H@Z 1002078c     U2Lang:U2Lang.dll
 0002:00000790       __imp_??1BaseWorker@LocalWorkflow@U2@@UAE@XZ 10020790     U2Lang:U2Lang.dll
 0002:00000794       __imp_??0BaseWorker@LocalWorkflow@U2@@QAE@PAVActor@Workflow@2@_N@Z 10020794     U2Lang:U2Lang.dll
 0002:00000798       __imp_?getBusType@IntegralBus@Workflow@U2@@QBE?AV?$QExplicitlySharedDataPointer@VDataType@U2@@@@XZ 10020798     U2Lang:U2Lang.dll
 0002:0000079c       __imp_?addError@WorkflowMonitor@Workflow@U2@@QAEXABVQString@@00@Z 1002079c     U2Lang:U2Lang.dll
 0002:000007a0       __imp_?addOutputFile@WorkflowMonitor@Workflow@U2@@QAEXABVQString@@0_N@Z 100207a0     U2Lang:U2Lang.dll
 0002:000007a4       __imp_??1DomainFactory@Workflow@U2@@UAE@XZ 100207a4     U2Lang:U2Lang.dll
 0002:000007a8       __imp_??0DomainFactory@Workflow@U2@@QAE@ABVQString@@@Z 100207a8     U2Lang:U2Lang.dll
 0002:000007ac       __imp_??0Message@Workflow@U2@@QAE@ABV012@@Z 100207ac     U2Lang:U2Lang.dll
 0002:000007b0       __imp_??1Message@Workflow@U2@@QAE@XZ 100207b0     U2Lang:U2Lang.dll
 0002:000007b4       __imp_?isEmpty@Message@Workflow@U2@@QBE_NXZ 100207b4     U2Lang:U2Lang.dll
 0002:000007b8       __imp_?getData@Message@Workflow@U2@@QBE?AVQVariant@@XZ 100207b8     U2Lang:U2Lang.dll
 0002:000007bc       __imp_??0Message@Workflow@U2@@QAE@V?$QExplicitlySharedDataPointer@VDataType@U2@@@@ABVQVariant@@H@Z 100207bc     U2Lang:U2Lang.dll
 0002:000007c0       __imp_?getInstance@WorkflowEnv@Workflow@U2@@KAPAV123@XZ 100207c0     U2Lang:U2Lang.dll
 0002:000007c4       __imp_?getProducers@IntegralBusPort@Workflow@U2@@QAE?AV?$QList@PAVActor@Workflow@U2@@@@ABVQString@@@Z 100207c4     U2Lang:U2Lang.dll
 0002:000007c8       __imp_?getProducer@IntegralBusPort@Workflow@U2@@QAEPAVActor@23@ABVQString@@@Z 100207c8     U2Lang:U2Lang.dll
 0002:000007cc       __imp_?NUM_TYPE@BaseTypes@U2@@SA?AV?$QExplicitlySharedDataPointer@VDataType@U2@@@@XZ 100207cc     U2Lang:U2Lang.dll
 0002:000007d0       __imp_?BOOL_TYPE@BaseTypes@U2@@SA?AV?$QExplicitlySharedDataPointer@VDataType@U2@@@@XZ 100207d0     U2Lang:U2Lang.dll
 0002:000007d4       __imp_?STRING_TYPE@BaseTypes@U2@@SA?AV?$QExplicitlySharedDataPointer@VDataType@U2@@@@XZ 100207d4     U2Lang:U2Lang.dll
 0002:000007d8       __imp_?VARIATION_TRACK_TYPE@BaseTypes@U2@@SA?AV?$QExplicitlySharedDataPointer@VDataType@U2@@@@XZ 100207d8     U2Lang:U2Lang.dll
 0002:000007dc       __imp_?DATASET_SLOT@BaseSlots@Workflow@U2@@SA?BVDescriptor@3@XZ 100207dc     U2Lang:U2Lang.dll
 0002:000007e0       __imp_?IN_ASSEMBLY_PORT_ID@BasePorts@Workflow@U2@@SA?BVQString@@XZ 100207e0     U2Lang:U2Lang.dll
 0002:000007e4       __imp_?OUT_VARIATION_TRACK_PORT_ID@BasePorts@Workflow@U2@@SA?BVQString@@XZ 100207e4     U2Lang:U2Lang.dll
 0002:000007e8       __imp_?IN_SEQ_PORT_ID@BasePorts@Workflow@U2@@SA?BVQString@@XZ 100207e8     U2Lang:U2Lang.dll
 0002:000007ec       __imp_?CATEGORY_VARIATION_ANALYSIS@BaseActorCategories@Workflow@U2@@SA?BVDescriptor@3@XZ 100207ec     U2Lang:U2Lang.dll
 0002:000007f0       __imp_?registerProto@ActorPrototypeRegistry@Workflow@U2@@QAE_NABVDescriptor@3@PAVActorPrototype@23@@Z 100207f0     U2Lang:U2Lang.dll
 0002:000007f4       __imp_?addExternalTool@ActorPrototype@Workflow@U2@@QAEXABVQString@@0@Z 100207f4     U2Lang:U2Lang.dll
 0002:000007f8       __imp_?setPortValidator@ActorPrototype@Workflow@U2@@QAEXABVQString@@PAVConfigurationValidator@3@@Z 100207f8     U2Lang:U2Lang.dll
 0002:000007fc       __imp_?setPrompter@ActorPrototype@Workflow@U2@@QAEXPAVPrompter@23@@Z 100207fc     U2Lang:U2Lang.dll
 0002:00000800       __imp_?setEditor@ActorPrototype@Workflow@U2@@QAEXPAVConfigurationEditor@3@@Z 10020800     U2Lang:U2Lang.dll
 0002:00000804       __imp_??1ActorPrototype@Workflow@U2@@UAE@XZ 10020804     U2Lang:U2Lang.dll
 0002:00000808       __imp_??0ActorPrototype@Workflow@U2@@QAE@ABVDescriptor@2@ABV?$QList@PAVPortDescriptor@Workflow@U2@@@@ABV?$QList@PAVAttribute@U2@@@@@Z 10020808     U2Lang:U2Lang.dll
 0002:0000080c       __imp_??1PortDescriptor@Workflow@U2@@UAE@XZ 1002080c     U2Lang:U2Lang.dll
 0002:00000810       __imp_??0PortDescriptor@Workflow@U2@@QAE@ABVDescriptor@2@V?$QExplicitlySharedDataPointer@VDataType@U2@@@@_N2I@Z 10020810     U2Lang:U2Lang.dll
 0002:00000814       __imp_?getOutputPorts@Actor@Workflow@U2@@QBE?AV?$QList@PAVPort@Workflow@U2@@@@XZ 10020814     U2Lang:U2Lang.dll
 0002:00000818       __imp_?getInputPorts@Actor@Workflow@U2@@QBE?AV?$QList@PAVPort@Workflow@U2@@@@XZ 10020818     U2Lang:U2Lang.dll
 0002:0000081c       __imp_?getPort@Actor@Workflow@U2@@QBEPAVPort@23@ABVQString@@@Z 1002081c     U2Lang:U2Lang.dll
 0002:00000820       __imp_?getLabel@Actor@Workflow@U2@@QBE?AVQString@@XZ 10020820     U2Lang:U2Lang.dll
 0002:00000824       __imp_?getId@Actor@Workflow@U2@@QBE?AVQString@@XZ 10020824     U2Lang:U2Lang.dll
 0002:00000828       __imp_??1ConfigurationValidator@U2@@UAE@XZ 10020828     U2Lang:U2Lang.dll
 0002:0000082c       __imp_??1PropertyDelegate@U2@@UAE@XZ 1002082c     U2Lang:U2Lang.dll
 0002:00000830       __imp_??0PropertyDelegate@U2@@QAE@PAVQObject@@@Z 10020830     U2Lang:U2Lang.dll
 0002:00000834       __imp_?addMainWidget@PropertyWidget@U2@@IAEXPAVQWidget@@@Z 10020834     U2Lang:U2Lang.dll
 0002:00000838       __imp_??1PropertyWidget@U2@@UAE@XZ 10020838     U2Lang:U2Lang.dll
 0002:0000083c       __imp_??0PropertyWidget@U2@@QAE@PAVQWidget@@PAVDelegateTags@1@@Z 1002083c     U2Lang:U2Lang.dll
 0002:00000840       __imp_?isOutUrlAttribute@RFSUtils@U2@@SA_NPAVAttribute@2@PAVActor@Workflow@2@AA_N@Z 10020840     U2Lang:U2Lang.dll
 0002:00000844       __imp_?addPortRelation@Attribute@U2@@QAEXPAVPortRelationDescriptor@2@@Z 10020844     U2Lang:U2Lang.dll
 0002:00000848       __imp_?addRelation@Attribute@U2@@QAEXPBVAttributeRelation@2@@Z 10020848     U2Lang:U2Lang.dll
 0002:0000084c       __imp_??1Attribute@U2@@UAE@XZ 1002084c     U2Lang:U2Lang.dll
 0002:00000850       __imp_??0Attribute@U2@@QAE@ABVDescriptor@1@V?$QExplicitlySharedDataPointer@VDataType@U2@@@@_NABVQVariant@@@Z 10020850     U2Lang:U2Lang.dll
 0002:00000854       __imp_?getScriptVars@AttributeScript@U2@@QBEABV?$QMap@VDescriptor@U2@@VQVariant@@@@XZ 10020854     U2Lang:U2Lang.dll
 0002:00000858       __imp_?getScriptText@AttributeScript@U2@@QBEABVQString@@XZ 10020858     U2Lang:U2Lang.dll
 0002:0000085c       __imp_?isEmpty@AttributeScript@U2@@QBE_NXZ 1002085c     U2Lang:U2Lang.dll
 0002:00000860       __imp_??1PortRelationDescriptor@U2@@UAE@XZ 10020860     U2Lang:U2Lang.dll
 0002:00000864       __imp_??0PortRelationDescriptor@U2@@QAE@ABVQString@@ABV?$QList@VQVariant@@@@@Z 10020864     U2Lang:U2Lang.dll
 0002:00000868       __imp_??1WorkflowScriptEngine@U2@@UAE@XZ 10020868     U2Lang:U2Lang.dll
 0002:0000086c       __imp_??0WorkflowScriptEngine@U2@@QAE@PAVWorkflowContext@Workflow@1@@Z 1002086c     U2Lang:U2Lang.dll
 0002:00000870       __imp_?absolutePath@WorkflowContext@Workflow@U2@@QBE?AVQString@@ABV4@@Z 10020870     U2Lang:U2Lang.dll
 0002:00000874       __imp_?getDataStorage@WorkflowContext@Workflow@U2@@QAEPAVDbiDataStorage@23@XZ 10020874     U2Lang:U2Lang.dll
 0002:00000878       __imp_??0WorkflowNotification@U2@@QAE@ABV01@@Z 10020878     U2Lang:U2Lang.dll
 0002:0000087c       __imp_??1WorkflowNotification@U2@@QAE@XZ 1002087c     U2Lang:U2Lang.dll
 0002:00000880       __imp_??0WorkflowNotification@U2@@QAE@ABVQString@@00@Z 10020880     U2Lang:U2Lang.dll
 0002:00000884       __imp_?initEngine@WorkflowScriptLibrary@U2@@SAXPAVWorkflowScriptEngine@2@@Z 10020884     U2Lang:U2Lang.dll
 0002:00000888       __imp_??1MapDataType@U2@@UAE@XZ 10020888     U2Lang:U2Lang.dll
 0002:0000088c       __imp_??0MapDataType@U2@@QAE@ABVDescriptor@1@ABV?$QMap@VDescriptor@U2@@V?$QExplicitlySharedDataPointer@VDataType@U2@@@@@@@Z 1002088c     U2Lang:U2Lang.dll
 0002:00000890       __imp_?getDatatypeDescriptor@DataType@U2@@QBE?AVDescriptor@2@ABVQString@@@Z 10020890     U2Lang:U2Lang.dll
 0002:00000894       __imp_??0Descriptor@U2@@QAE@ABV01@@Z 10020894     U2Lang:U2Lang.dll
 0002:00000898       __imp_?getDisplayName@Descriptor@U2@@QBE?AVQString@@XZ 10020898     U2Lang:U2Lang.dll
 0002:0000089c       __imp_??0Descriptor@U2@@QAE@PBD@Z 1002089c     U2Lang:U2Lang.dll
 0002:000008a0       __imp_??0Descriptor@U2@@QAE@ABVQString@@@Z 100208a0     U2Lang:U2Lang.dll
 0002:000008a4       __imp_??0Descriptor@U2@@QAE@ABVQString@@00@Z 100208a4     U2Lang:U2Lang.dll
 0002:000008a8       __imp_??1VisibilityRelation@U2@@UAE@XZ 100208a8     U2Lang:U2Lang.dll
 0002:000008ac       __imp_??0VisibilityRelation@U2@@QAE@ABVQString@@ABV?$QList@VQVariant@@@@_N@Z 100208ac     U2Lang:U2Lang.dll
 0002:000008b0       __imp_?getDbiRef@DbiDataStorage@Workflow@U2@@QAE?AVU2DbiRef@3@XZ 100208b0     U2Lang:U2Lang.dll
 0002:000008b4       __imp_?VARIATION_TRACK_SLOT@BaseSlots@Workflow@U2@@SA?BVDescriptor@3@XZ 100208b4     U2Lang:U2Lang.dll
 0002:000008b8       __imp_?URL_SLOT@BaseSlots@Workflow@U2@@SA?BVDescriptor@3@XZ 100208b8     U2Lang:U2Lang.dll
 0002:000008bc       __imp_?getId@Descriptor@U2@@QBE?AVQString@@XZ 100208bc     U2Lang:U2Lang.dll
 0002:000008c0       __imp_??1Descriptor@U2@@UAE@XZ 100208c0     U2Lang:U2Lang.dll
 0002:000008c4       __imp_?getOutputFiles@BaseWorker@LocalWorkflow@U2@@UAE?AVQStringList@@XZ 100208c4     U2Lang:U2Lang.dll
 0002:000008c8       \177U2Lang_NULL_THUNK_DATA 100208c8     U2Lang:U2Lang.dll
 0002:000008cc       ___xc_a                    100208cc     MSVCRT:cinitexe.obj
 0002:00000a88       ___xc_z                    10020a88     MSVCRT:cinitexe.obj
 0002:00000a8c       ___xi_a                    10020a8c     MSVCRT:cinitexe.obj
 0002:00000a98       ___xi_z                    10020a98     MSVCRT:cinitexe.obj
 0002:00000ad8       ??_C@_00CNPNBAHC@?$AA@     10020ad8     AssemblySamtoolsMpileup.obj
 0002:00000ae0       ??_7error_category@std@@6B@ 10020ae0     AssemblySamtoolsMpileup.obj
 0002:00000afc       ??_7_Generic_error_category@std@@6B@ 10020afc     AssemblySamtoolsMpileup.obj
 0002:00000b14       ??_C@_07DCLBNMLN@generic?$AA@ 10020b14     AssemblySamtoolsMpileup.obj
 0002:00000b1c       ??_C@_0O@BFJCFAAK@unknown?5error?$AA@ 10020b1c     AssemblySamtoolsMpileup.obj
 0002:00000b30       ??_7_Iostream_error_category@std@@6B@ 10020b30     AssemblySamtoolsMpileup.obj
 0002:00000b48       ??_C@_08LLGCOLLL@iostream?$AA@ 10020b48     AssemblySamtoolsMpileup.obj
 0002:00000b54       ??_C@_0BG@PADBLCHM@iostream?5stream?5error?$AA@ 10020b54     AssemblySamtoolsMpileup.obj
 0002:00000b70       ??_7_System_error_category@std@@6B@ 10020b70     AssemblySamtoolsMpileup.obj
 0002:00000b88       ??_C@_06FHFOAHML@system?$AA@ 10020b88     AssemblySamtoolsMpileup.obj
 0002:00000b90       ??_C@_0L@JLHNEGIN@Algorithms?$AA@ 10020b90     AssemblySamtoolsMpileup.obj
 0002:00000b9c       ??_C@_07PGLPGHFC@Console?$AA@ 10020b9c     AssemblySamtoolsMpileup.obj
 0002:00000ba4       ??_C@_0O@BOFHOPCF@Core?5Services?$AA@ 10020ba4     AssemblySamtoolsMpileup.obj
 0002:00000bb4       ??_C@_0N@PPADAKBM@Input?1Output?$AA@ 10020bb4     AssemblySamtoolsMpileup.obj
 0002:00000bc4       ??_C@_0M@KPPBKPKK@Performance?$AA@ 10020bc4     AssemblySamtoolsMpileup.obj
 0002:00000bd0       ??_C@_07BFDHHBBI@Scripts?$AA@ 10020bd0     AssemblySamtoolsMpileup.obj
 0002:00000bd8       ??_C@_05EEGKELMG@Tasks?$AA@ 10020bd8     AssemblySamtoolsMpileup.obj
 0002:00000be0       ??_C@_0P@NIIOBHGA@User?5Interface?$AA@ 10020be0     AssemblySamtoolsMpileup.obj
 0002:00000bf0       ??_C@_0N@JINCGGMN@User?5Actions?$AA@ 10020bf0     AssemblySamtoolsMpileup.obj
 0002:00000c00       ??_C@_0N@CLOACMBA@U2?3?3U2DbiRef?$AA@ 10020c00     AssemblySamtoolsMpileup.obj
 0002:00000c14       ??_SLoadDocumentTask@U2@@6B@ 10020c14     AssemblySamtoolsMpileup.obj
 0002:00000cac       ??_C@_0CD@LMLLOHBG@U2?3?3Workflow?3?3SharedDbiDataHandl@ 10020cac     AssemblySamtoolsMpileup.obj
 0002:00000cd4       ??_7SamtoolsMpileupTask@LocalWorkflow@U2@@6B@ 10020cd4     AssemblySamtoolsMpileup.obj
 0002:00000d6c       ??_7CallVariantsTask@LocalWorkflow@U2@@6B@ 10020d6c     AssemblySamtoolsMpileup.obj
 0002:00000e00       ??_C@_0BF@GEHGKKOL@Call?5variants?5for?5?$CF1?$AA@ 10020e00     AssemblySamtoolsMpileup.obj
 0002:00000e18       ??_C@_0BF@PNHIOAIL@NGS?3CallVariantsTask?$AA@ 10020e18     AssemblySamtoolsMpileup.obj
 0002:00000e30       ??_C@_09KJONPCOF@reference?$AA@ 10020e30     AssemblySamtoolsMpileup.obj
 0002:00000e3c       ??_C@_08LKDFMABF@assembly?$AA@ 10020e3c     AssemblySamtoolsMpileup.obj
 0002:00000e48       ??_C@_0CK@IGBIANDN@Trying?5to?5recover?5from?5error?3?5?$CF1@ 10020e48     AssemblySamtoolsMpileup.obj
 0002:00000e74       ??_C@_0BC@GPFGJGDI@Unknown?5file?5type?$AA@ 10020e74     AssemblySamtoolsMpileup.obj
 0002:00000e88       ??_C@_0CA@NFJGNOAM@src?2AssemblySamtoolsMpileup?4cpp?$AA@ 10020e88     AssemblySamtoolsMpileup.obj
 0002:00000ea8       ??_C@_0BP@IKHCENFC@The?5?$CF1?5file?5does?5not?5exist?3?5?$CF2?$AA@ 10020ea8     AssemblySamtoolsMpileup.obj
 0002:00000ec8       ??_C@_0BC@LKMOBCOB@No?5assembly?5files?$AA@ 10020ec8     AssemblySamtoolsMpileup.obj
 0002:00000edc       ??_C@_0P@HMLMIEOH@No?5dbi?5storage?$AA@ 10020edc     AssemblySamtoolsMpileup.obj
 0002:00000eec       ??_C@_0BA@GBHNBGFA@No?5sequence?5URL?$AA@ 10020eec     AssemblySamtoolsMpileup.obj
 0002:00000efc       ??_C@_0BD@IJHCCBPI@No?5document?5loaded?$AA@ 10020efc     AssemblySamtoolsMpileup.obj
 0002:00000f10       ??_C@_0CF@LEJBNDCK@Incorrect?5variant?5track?5object?5i@ 10020f10     AssemblySamtoolsMpileup.obj
 0002:00000f38       ??_C@_08PKEDFKMP@variants?$AA@ 10020f38     AssemblySamtoolsMpileup.obj
 0002:00000f44       ??_C@_0P@DLMOIKDA@USUPP_SAMTOOLS?$AA@ 10020f44     AssemblySamtoolsMpileup.obj
 0002:00000f54       ??_C@_0P@MAFHIPIF@USUPP_BCFTOOLS?$AA@ 10020f54     AssemblySamtoolsMpileup.obj
 0002:00000f64       ??_C@_0P@MIHMLGBC@USUPP_VCFUTILS?$AA@ 10020f64     AssemblySamtoolsMpileup.obj
 0002:00000f74       ??_C@_0BI@OFMEPBAM@Samtool?5mpileup?5for?5?$CF1?5?$AA@ 10020f74     AssemblySamtoolsMpileup.obj
 0002:00000f8c       ??_C@_0CH@IBLANLNA@No?5reference?5sequence?5URL?5to?5do?5@ 10020f8c     AssemblySamtoolsMpileup.obj
 0002:00000fb4       ??_C@_0BN@JDICDEAO@No?5assembly?5URL?5to?5do?5pileup?$AA@ 10020fb4     AssemblySamtoolsMpileup.obj
 0002:00000fd4       ??_C@_0CI@HIHDNNDB@There?5is?5an?5assembly?5with?5an?5emp@ 10020fd4     AssemblySamtoolsMpileup.obj
 0002:00000ffc       ??_C@_0BM@DJNLDNPA@Can?5not?5create?5the?5folder?3?5?$AA@ 10020ffc     AssemblySamtoolsMpileup.obj
 0002:00001018       ??_C@_08DPIJBAEH@SAMtools?$AA@ 10021018     AssemblySamtoolsMpileup.obj
 0002:00001024       ??_C@_08MEBABFPC@BCFtools?$AA@ 10021024     AssemblySamtoolsMpileup.obj
 0002:00001030       ??_C@_08HIABPFAM@vcfutils?$AA@ 10021030     AssemblySamtoolsMpileup.obj
 0002:0000103c       ??_C@_0BE@BOLJGIKE@Can?5not?5run?5?$CF1?5tool?$AA@ 1002103c     AssemblySamtoolsMpileup.obj
 0002:00001050       ??_C@_0BM@EKPABLJB@?$CF1?5tool?5exited?5with?5code?5?$CF2?$AA@ 10021050     AssemblySamtoolsMpileup.obj
 0002:0000106c       ??_C@_0BO@MBDPMDG@Tool?5?$CF1?5finished?5successfully?$AA@ 1002106c     AssemblySamtoolsMpileup.obj
 0002:0000108c       ??_C@_07DPJPFFHF@mpileup?$AA@ 1002108c     AssemblySamtoolsMpileup.obj
 0002:00001094       ??_C@_03ONHODBJK@?9uf?$AA@ 10021094     AssemblySamtoolsMpileup.obj
 0002:00001098       ??_C@_02OLHPOPJI@?9C?$AA@  10021098     AssemblySamtoolsMpileup.obj
 0002:0000109c       ??_C@_02DBLKFNPN@?9d?$AA@  1002109c     AssemblySamtoolsMpileup.obj
 0002:000010a0       ??_C@_02GAPLLOJ@?9q?$AA@   100210a0     AssemblySamtoolsMpileup.obj
 0002:000010a4       ??_C@_02JDILJPEL@?9Q?$AA@  100210a4     AssemblySamtoolsMpileup.obj
 0002:000010a8       ??_C@_02CIKBGMLM@?9e?$AA@  100210a8     AssemblySamtoolsMpileup.obj
 0002:000010ac       ??_C@_02JNAPBCPB@?9h?$AA@  100210ac     AssemblySamtoolsMpileup.obj
 0002:000010b0       ??_C@_02GMOHPDFH@?9L?$AA@  100210b0     AssemblySamtoolsMpileup.obj
 0002:000010b4       ??_C@_02NCEOIEDG@?9o?$AA@  100210b4     AssemblySamtoolsMpileup.obj
 0002:000010b8       ??_C@_02LJDHGCCL@?96?$AA@  100210b8     AssemblySamtoolsMpileup.obj
 0002:000010bc       ??_C@_02NJEJINBK@?9A?$AA@  100210bc     AssemblySamtoolsMpileup.obj
 0002:000010c0       ??_C@_02PCGENONJ@?9B?$AA@  100210c0     AssemblySamtoolsMpileup.obj
 0002:000010c4       ??_C@_02LNCFEIBO@?9E?$AA@  100210c4     AssemblySamtoolsMpileup.obj
 0002:000010c8       ??_C@_02PJGDNHPF@?9l?$AA@  100210c8     AssemblySamtoolsMpileup.obj
 0002:000010cc       ??_C@_02CNCCOICK@?9r?$AA@  100210cc     AssemblySamtoolsMpileup.obj
 0002:000010d0       ??_C@_02BBJAAHBC@?9I?$AA@  100210d0     AssemblySamtoolsMpileup.obj
 0002:000010d4       ??_C@_02IKJAKOAK@?9P?$AA@  100210d4     AssemblySamtoolsMpileup.obj
 0002:000010d8       ??_C@_04CHADEDPO@view?$AA@ 100210d8     AssemblySamtoolsMpileup.obj
 0002:000010e0       ??_C@_03JCEPHLIG@?9vc?$AA@ 100210e0     AssemblySamtoolsMpileup.obj
 0002:000010e4       ??_C@_02IEBECDLA@?9i?$AA@  100210e4     AssemblySamtoolsMpileup.obj
 0002:000010e8       ??_C@_02BPBEIKKI@?9p?$AA@  100210e8     AssemblySamtoolsMpileup.obj
 0002:000010ec       ??_C@_02HLHIEPKM@?9t?$AA@  100210ec     AssemblySamtoolsMpileup.obj
 0002:000010f0       ??_C@_02PGHGPEOM@?91?$AA@  100210f0     AssemblySamtoolsMpileup.obj
 0002:000010f4       ??_C@_02PHOHFKEP@?9U?$AA@  100210f4     AssemblySamtoolsMpileup.obj
 0002:000010f8       ??_C@_02ECEJCEAC@?9X?$AA@  100210f8     AssemblySamtoolsMpileup.obj
 0002:000010fc       ??_C@_02JGAIBLNN@?9F?$AA@  100210fc     AssemblySamtoolsMpileup.obj
 0002:00001100       ??_C@_02IPBDCKJM@?9G?$AA@  10021100     AssemblySamtoolsMpileup.obj
 0002:00001104       ??_C@_02FONBJBNF@?9N?$AA@  10021104     AssemblySamtoolsMpileup.obj
 0002:00001108       ??_C@_02DEDJNJGL@?9s?$AA@  10021108     AssemblySamtoolsMpileup.obj
 0002:0000110c       ??_C@_02BKJHAODO@?9g?$AA@  1002110c     AssemblySamtoolsMpileup.obj
 0002:00001110       ??_C@_02OOPMGLAO@?9T?$AA@  10021110     AssemblySamtoolsMpileup.obj
 0002:00001114       ??_C@_01JOAMLHOP@?9?$AA@   10021114     AssemblySamtoolsMpileup.obj
 0002:00001118       ??_C@_09KBOFMALF@varFilter?$AA@ 10021118     AssemblySamtoolsMpileup.obj
 0002:00001124       ??_C@_02KEDOHJFP@?9D?$AA@  10021124     AssemblySamtoolsMpileup.obj
 0002:00001128       ??_C@_02EMMNKJLI@?9a?$AA@  10021128     AssemblySamtoolsMpileup.obj
 0002:0000112c       ??_C@_02FAFFBMGP@?9w?$AA@  1002112c     AssemblySamtoolsMpileup.obj
 0002:00001130       ??_C@_02MFNBDIMN@?9W?$AA@  10021130     AssemblySamtoolsMpileup.obj
 0002:00001134       ??_C@_02NNFLKHCP@?92?$AA@  10021134     AssemblySamtoolsMpileup.obj
 0002:00001138       ??_C@_02MEEAJGGO@?93?$AA@  10021138     AssemblySamtoolsMpileup.obj
 0002:0000113c       ??_C@_02ILABAAKJ@?94?$AA@  1002113c     AssemblySamtoolsMpileup.obj
 0002:00001140       ??_C@_0BA@JFNIOLAK@string?5too?5long?$AA@ 10021140     AssemblySamtoolsMpileup.obj
 0002:00001150       ??_C@_0BI@CFPLBAOH@invalid?5string?5position?$AA@ 10021150     AssemblySamtoolsMpileup.obj
 0002:00001168       __real@3ff0000000000000    10021168     AssemblySamtoolsMpileup.obj
 0002:00001174       ??_SQDoubleValidator@@6B@  10021174     SamtoolMpileupWorker.obj
 0002:000011b4       ??_SQLineEdit@@6BQObject@@@ 100211b4     SamtoolMpileupWorker.obj
 0002:0000126c       ??_SQLineEdit@@6BQPaintDevice@@@ 1002126c     SamtoolMpileupWorker.obj
 0002:0000128c       ??_SVisibilityRelation@U2@@6B@ 1002128c     SamtoolMpileupWorker.obj
 0002:000012a8       ??_SDescriptor@U2@@6B@     100212a8     SamtoolMpileupWorker.obj
 0002:000012b8       ??_SMapDataType@U2@@6B@    100212b8     SamtoolMpileupWorker.obj
 0002:000012d8       ??_SPortRelationDescriptor@U2@@6B@ 100212d8     SamtoolMpileupWorker.obj
 0002:000012e8       ??_SAttribute@U2@@6B@      100212e8     SamtoolMpileupWorker.obj
 0002:00001318       ??_C@_0BF@COKBMJP@Script?5task?5canceled?$AA@ 10021318     SamtoolMpileupWorker.obj
 0002:00001334       ??_SDelegateEditor@U2@@6B@ 10021334     SamtoolMpileupWorker.obj
 0002:0000138c       ??_SURLDelegate@U2@@6B@    1002138c     SamtoolMpileupWorker.obj
 0002:0000140c       ??_SSpinBoxDelegate@U2@@6B@ 1002140c     SamtoolMpileupWorker.obj
 0002:0000148c       ??_SDoubleSpinBoxDelegate@U2@@6B@ 1002148c     SamtoolMpileupWorker.obj
 0002:0000150c       ??_SComboBoxDelegate@U2@@6B@ 1002150c     SamtoolMpileupWorker.obj
 0002:0000158c       ??_SPortDescriptor@Workflow@U2@@6B@ 1002158c     SamtoolMpileupWorker.obj
 0002:000015a4       ??_SIntegralBusActorPrototype@Workflow@U2@@6BQObject@@@ 100215a4     SamtoolMpileupWorker.obj
 0002:000015e0       ??_SIntegralBusActorPrototype@Workflow@U2@@6BVisualDescriptor@2@@ 100215e0     SamtoolMpileupWorker.obj
 0002:000015f0       ??_7?$PrompterBase@VCallVariantsPrompter@LocalWorkflow@U2@@@U2@@6BActorDocument@Workflow@1@@ 100215f0     SamtoolMpileupWorker.obj
 0002:00001638       ??_7?$PrompterBase@VCallVariantsPrompter@LocalWorkflow@U2@@@U2@@6BPrompter@Workflow@1@@ 10021638     SamtoolMpileupWorker.obj
 0002:00001644       ??_7CallVariantsPrompter@LocalWorkflow@U2@@6BActorDocument@Workflow@2@@ 10021644     SamtoolMpileupWorker.obj
 0002:0000168c       ??_7CallVariantsPrompter@LocalWorkflow@U2@@6BPrompter@Workflow@2@@ 1002168c     SamtoolMpileupWorker.obj
 0002:00001698       ??_7CallVariantsWorker@LocalWorkflow@U2@@6BQObject@@@ 10021698     SamtoolMpileupWorker.obj
 0002:000016dc       ??_7CallVariantsWorker@LocalWorkflow@U2@@6BWorker@Workflow@2@@ 100216dc     SamtoolMpileupWorker.obj
 0002:000016f8       ??_7CallVariantsWorker@LocalWorkflow@U2@@6BCommunicationSubject@Workflow@2@@ 100216f8     SamtoolMpileupWorker.obj
 0002:00001708       ??_7CallVariantsWorkerFactory@LocalWorkflow@U2@@6B?$IdRegistry@VDomainFactory@Workflow@U2@@@2@@ 10021708     SamtoolMpileupWorker.obj
 0002:00001734       ??_7CallVariantsWorkerFactory@LocalWorkflow@U2@@6BDescriptor@2@@ 10021734     SamtoolMpileupWorker.obj
 0002:00001744       ??_7ScientificDoubleWidget@LocalWorkflow@U2@@6BQObject@@@ 10021744     SamtoolMpileupWorker.obj
 0002:00001814       ??_7ScientificDoubleWidget@LocalWorkflow@U2@@6BQPaintDevice@@@ 10021814     SamtoolMpileupWorker.obj
 0002:00001834       ??_7ScientificDoubleDelegate@LocalWorkflow@U2@@6B@ 10021834     SamtoolMpileupWorker.obj
 0002:000018b0       ??_C@_0O@NBKBGGDM@call_variants?$AA@ 100218b0     SamtoolMpileupWorker.obj
 0002:000018c0       ??_C@_0BA@CNMNLKDG@ref?9seq?9port?9id?$AA@ 100218c0     SamtoolMpileupWorker.obj
 0002:000018d0       ??_C@_0BB@KOBCNCN@assembly?9port?9id?$AA@ 100218d0     SamtoolMpileupWorker.obj
 0002:000018e4       ??_C@_0N@DCLEHBHM@variants?9url?$AA@ 100218e4     SamtoolMpileupWorker.obj
 0002:000018f4       ??_C@_0BB@NKLIJMO@reference?9source?$AA@ 100218f4     SamtoolMpileupWorker.obj
 0002:00001908       ??_C@_04LPGMAPLE@port?$AA@ 10021908     SamtoolMpileupWorker.obj
 0002:00001910       ??_C@_04DAMGJPCA@file?$AA@ 10021910     SamtoolMpileupWorker.obj
 0002:00001918       ??_C@_0O@OILGKDNH@reference?9url?$AA@ 10021918     SamtoolMpileupWorker.obj
 0002:00001928       ??_C@_0BE@BDMBEII@illumina13?9encoding?$AA@ 10021928     SamtoolMpileupWorker.obj
 0002:0000193c       ??_C@_0L@BCLOODGD@use_orphan?$AA@ 1002193c     SamtoolMpileupWorker.obj
 0002:00001948       ??_C@_0M@DNPMKK@disable_baq?$AA@ 10021948     SamtoolMpileupWorker.obj
 0002:00001954       ??_C@_0L@JEGGCCFD@capq_thres?$AA@ 10021954     SamtoolMpileupWorker.obj
 0002:00001960       ??_C@_09IOAIKKBL@max_depth?$AA@ 10021960     SamtoolMpileupWorker.obj
 0002:0000196c       ??_C@_07BJLPNBOA@ext_baq?$AA@ 1002196c     SamtoolMpileupWorker.obj
 0002:00001974       ??_C@_03BJLIAD@bed?$AA@    10021974     SamtoolMpileupWorker.obj
 0002:00001978       ??_C@_03HLCNLMFP@reg?$AA@  10021978     SamtoolMpileupWorker.obj
 0002:0000197c       ??_C@_06GEEOJFCK@min_mq?$AA@ 1002197c     SamtoolMpileupWorker.obj
 0002:00001984       ??_C@_09DIIMLKMD@min_baseq?$AA@ 10021984     SamtoolMpileupWorker.obj
 0002:00001990       ??_C@_04DGNMNEDF@extQ?$AA@ 10021990     SamtoolMpileupWorker.obj
 0002:00001998       ??_C@_07COBNHEFN@tandemQ?$AA@ 10021998     SamtoolMpileupWorker.obj
 0002:000019a0       ??_C@_08GLOIEAKE@no_indel?$AA@ 100219a0     SamtoolMpileupWorker.obj
 0002:000019ac       ??_C@_0BA@FDGKDJGK@max_indel_depth?$AA@ 100219ac     SamtoolMpileupWorker.obj
 0002:000019bc       ??_C@_05KDFMIOBC@openQ?$AA@ 100219bc     SamtoolMpileupWorker.obj
 0002:000019c4       ??_C@_07IAELGFIL@pl_list?$AA@ 100219c4     SamtoolMpileupWorker.obj
 0002:000019cc       ??_C@_07OGDNJPMP@keepalt?$AA@ 100219cc     SamtoolMpileupWorker.obj
 0002:000019d4       ??_C@_06GCHLPPMN@fix_pl?$AA@ 100219d4     SamtoolMpileupWorker.obj
 0002:000019dc       ??_C@_07FIFMCJBP@no_geno?$AA@ 100219dc     SamtoolMpileupWorker.obj
 0002:000019e4       ??_C@_09HMEDCEJ@acgt_only?$AA@ 100219e4     SamtoolMpileupWorker.obj
 0002:000019f0       ??_C@_07IABPNJF@bcf_bed?$AA@ 100219f0     SamtoolMpileupWorker.obj
 0002:000019f8       ??_C@_05FLMOALCM@qcall?$AA@ 100219f8     SamtoolMpileupWorker.obj
 0002:00001a00       ??_C@_07ODIFGGLK@samples?$AA@ 10021a00     SamtoolMpileupWorker.obj
 0002:00001a08       ??_C@_0O@MLGNBJMK@min_smpl_frac?$AA@ 10021a08     SamtoolMpileupWorker.obj
 0002:00001a18       ??_C@_07FPCJOLFB@call_gt?$AA@ 10021a18     SamtoolMpileupWorker.obj
 0002:00001a20       ??_C@_0L@IIAEEDCA@indel_frac?$AA@ 10021a20     SamtoolMpileupWorker.obj
 0002:00001a2c       ??_C@_04HMICEFNA@pref?$AA@ 10021a2c     SamtoolMpileupWorker.obj
 0002:00001a34       ??_C@_05BDABANDG@ptype?$AA@ 10021a34     SamtoolMpileupWorker.obj
 0002:00001a3c       ??_C@_05FECKLAFM@theta?$AA@ 10021a3c     SamtoolMpileupWorker.obj
 0002:00001a44       ??_C@_05BFNAKILM@ccall?$AA@ 10021a44     SamtoolMpileupWorker.obj
 0002:00001a4c       ??_C@_02IEKKMHHF@n1?$AA@   10021a4c     SamtoolMpileupWorker.obj
 0002:00001a50       ??_C@_06DGMOODDB@n_perm?$AA@ 10021a50     SamtoolMpileupWorker.obj
 0002:00001a58       ??_C@_0L@IMLNMDAC@min_perm_p?$AA@ 10021a58     SamtoolMpileupWorker.obj
 0002:00001a64       ??_C@_08DMLALAP@min?9qual?$AA@ 10021a64     SamtoolMpileupWorker.obj
 0002:00001a70       ??_C@_07BBNFAJDM@min?9dep?$AA@ 10021a70     SamtoolMpileupWorker.obj
 0002:00001a78       ??_C@_07PHLFKGNN@max?9dep?$AA@ 10021a78     SamtoolMpileupWorker.obj
 0002:00001a80       ??_C@_0O@MAIGNCNC@min?9alt?9bases?$AA@ 10021a80     SamtoolMpileupWorker.obj
 0002:00001a90       ??_C@_08NDFPDBCI@gap?9size?$AA@ 10021a90     SamtoolMpileupWorker.obj
 0002:00001a9c       ??_C@_06NFBEFKOC@window?$AA@ 10021a9c     SamtoolMpileupWorker.obj
 0002:00001aa4       ??_C@_0L@NKHLHJAG@min?9strand?$AA@ 10021aa4     SamtoolMpileupWorker.obj
 0002:00001ab0       ??_C@_09NGPPFPGD@min?9baseQ?$AA@ 10021ab0     SamtoolMpileupWorker.obj
 0002:00001abc       ??_C@_08OKMDALN@min?9mapQ?$AA@ 10021abc     SamtoolMpileupWorker.obj
 0002:00001ac8       ??_C@_0BB@EABLENJM@min?9end?9distance?$AA@ 10021ac8     SamtoolMpileupWorker.obj
 0002:00001adc       ??_C@_07HDBECHIO@min?9hwe?$AA@ 10021adc     SamtoolMpileupWorker.obj
 0002:00001ae4       ??_C@_0P@HKDNIKFH@print?9filtered?$AA@ 10021ae4     SamtoolMpileupWorker.obj
 0002:00001af8       ??_7EmptySlotValidator@LocalWorkflow@U2@@6B@ 10021af8     SamtoolMpileupWorker.obj
 0002:00001b00       ??_C@_0BF@JCLBEAMA@Empty?5input?5slot?3?5?$CF1?$AA@ 10021b00     SamtoolMpileupWorker.obj
 0002:00001b18       ??_C@_0CB@GPADDDPB@A?5nucleotide?5reference?5sequence?4@ 10021b18     SamtoolMpileupWorker.obj
 0002:00001b3c       ??_C@_0BA@GLOOOALC@Input?5sequences?$AA@ 10021b3c     SamtoolMpileupWorker.obj
 0002:00001b4c       ??_C@_0BP@EIIBDCJL@Position?5sorted?5alignment?5file?$AA@ 10021b4c     SamtoolMpileupWorker.obj
 0002:00001b6c       ??_C@_0P@HHJLMJCG@Input?5assembly?$AA@ 10021b6c     SamtoolMpileupWorker.obj
 0002:00001b7c       ??_C@_0CJ@LMNJMNBP@Output?5tracks?5with?5SNPs?5and?5shor@ 10021b7c     SamtoolMpileupWorker.obj
 0002:00001ba8       ??_C@_0BC@HALKGCHI@Output?5variations?$AA@ 10021ba8     SamtoolMpileupWorker.obj
 0002:00001bbc       ??_C@_0DK@CJNLKJJG@Calls?5SNPs?5and?5INDELS?5with?5SAMto@ 10021bbc     SamtoolMpileupWorker.obj
 0002:00001bf8       ??_C@_0BM@FIOBACII@Call?5Variants?5with?5SAMtools?$AA@ 10021bf8     SamtoolMpileupWorker.obj
 0002:00001c14       ??_C@_0DD@EJLDGFGM@The?5url?5to?5the?5file?5with?5the?5ext@ 10021c14     SamtoolMpileupWorker.obj
 0002:00001c48       ??_C@_0BF@NKIIBGEB@Output?5variants?5file?$AA@ 10021c48     SamtoolMpileupWorker.obj
 0002:00001c60       ??_C@_0BGE@KEDGAAAM@?$DMp?$DOSpecify?5?$CCFile?$CC?5to?5set?5a?5singl@ 10021c60     SamtoolMpileupWorker.obj
 0002:00001dc4       ??_C@_0BD@IPBFLNCO@Use?5reference?5from?$AA@ 10021dc4     SamtoolMpileupWorker.obj
 0002:00001dd8       ??_C@_0IG@PJCEBIHI@?$DMp?$DOSpecify?5a?5file?5with?5the?5refer@ 10021dd8     SamtoolMpileupWorker.obj
 0002:00001e60       ??_C@_09OGLAPBDF@Reference?$AA@ 10021e60     SamtoolMpileupWorker.obj
 0002:00001e70       ??_C@_0ED@BNFCGLNF@Assume?5the?5quality?5is?5in?5the?5Ill@ 10021e70     SamtoolMpileupWorker.obj
 0002:00001eb4       ??_C@_0BH@LCFMEGPH@Illumina?91?43?$CL?5encoding?$AA@ 10021eb4     SamtoolMpileupWorker.obj
 0002:00001ed0       ??_C@_0EC@JHFFFOKB@Do?5not?5skip?5anomalous?5read?5pairs@ 10021ed0     SamtoolMpileupWorker.obj
 0002:00001f14       ??_C@_0BL@LEFBKFJ@Count?5anomalous?5read?5pairs?$AA@ 10021f14     SamtoolMpileupWorker.obj
 0002:00001f30       ??_C@_0PM@GNCNHGHL@Disable?5probabilistic?5realignmen@ 10021f30     SamtoolMpileupWorker.obj
 0002:0000202c       ??_C@_0BI@LEPJMGNK@Disable?5BAQ?5computation?$AA@ 1002202c     SamtoolMpileupWorker.obj
 0002:00002048       ??_C@_0BFI@KKILGLEG@Coefficient?5for?5downgrading?5mapp@ 10022048     SamtoolMpileupWorker.obj
 0002:000021a0       ??_C@_0CI@ONLHPOMC@Mapping?5quality?5downgrading?5coef@ 100221a0     SamtoolMpileupWorker.obj
 0002:000021c8       ??_C@_0EP@CIMOMODA@At?5a?5position?0?5read?5maximally?5th@ 100221c8     SamtoolMpileupWorker.obj
 0002:00002218       ??_C@_0CC@JDOMGLDO@Max?5number?5of?5reads?5per?5input?5BA@ 10022218     SamtoolMpileupWorker.obj
 0002:00002240       ??_C@_0IC@MFCBGFGA@Extended?5BAQ?5computation?4?5This?5o@ 10022240     SamtoolMpileupWorker.obj
 0002:000022c4       ??_C@_0BJ@JJJPMHPE@Extended?5BAQ?5computation?$AA@ 100222c4     SamtoolMpileupWorker.obj
 0002:000022e0       ??_C@_0HH@OCCLDHKI@BED?5or?5position?5list?5file?5contai@ 100222e0     SamtoolMpileupWorker.obj
 0002:00002358       ??_C@_0BK@BEPEMOBK@BED?5or?5position?5list?5file?$AA@ 10022358     SamtoolMpileupWorker.obj
 0002:00002374       ??_C@_0DC@GLHHIMFI@Only?5generate?5pileup?5in?5region?5S@ 10022374     SamtoolMpileupWorker.obj
 0002:000023a8       ??_C@_0O@GDEAOPLE@Pileup?5region?$AA@ 100223a8     SamtoolMpileupWorker.obj
 0002:000023b8       ??_C@_0ED@EECHBJNJ@Minimum?5mapping?5quality?5for?5an?5a@ 100223b8     SamtoolMpileupWorker.obj
 0002:000023fc       ??_C@_0BI@FOLEAOFM@Minimum?5mapping?5quality?$AA@ 100223fc     SamtoolMpileupWorker.obj
 0002:00002418       ??_C@_0EA@GMOJDIJK@Minimum?5base?5quality?5for?5a?5base?5@ 10022418     SamtoolMpileupWorker.obj
 0002:00002458       ??_C@_0BF@MHDGMJJA@Minimum?5base?5quality?$AA@ 10022458     SamtoolMpileupWorker.obj
 0002:00002470       ??_C@_0GM@MOMJMHND@Phred?9scaled?5gap?5extension?5seque@ 10022470     SamtoolMpileupWorker.obj
 0002:000024dc       ??_C@_0BE@FDCJHOIO@Gap?5extension?5error?$AA@ 100224dc     SamtoolMpileupWorker.obj
 0002:000024f0       ??_C@_0JO@BOJNDKDE@Coefficient?5for?5modeling?5homopol@ 100224f0     SamtoolMpileupWorker.obj
 0002:00002590       ??_C@_0BP@JJEDKKJK@Homopolymer?5errors?5coefficient?$AA@ 10022590     SamtoolMpileupWorker.obj
 0002:000025b0       ??_C@_0CM@IPHBKLIH@Do?5not?5perform?5INDEL?5calling?5?$CImp@ 100225b0     SamtoolMpileupWorker.obj
 0002:000025dc       ??_C@_09HOEANPBI@No?5INDELs?$AA@ 100225dc     SamtoolMpileupWorker.obj
 0002:000025e8       ??_C@_0EP@BCJJCING@Skip?5INDEL?5calling?5if?5the?5averag@ 100225e8     SamtoolMpileupWorker.obj
 0002:00002638       ??_C@_0BA@GJIGPMGO@Max?5INDEL?5depth?$AA@ 10022638     SamtoolMpileupWorker.obj
 0002:00002648       ??_C@_0GK@KLBAHAIM@Phred?9scaled?5gap?5open?5sequencing@ 10022648     SamtoolMpileupWorker.obj
 0002:000026b4       ??_C@_0P@KHBDDLPM@Gap?5open?5error?$AA@ 100226b4     SamtoolMpileupWorker.obj
 0002:000026c8       ??_C@_0OM@DHBAHLFF@Comma?5dilimited?5list?5of?5platform@ 100226c8     SamtoolMpileupWorker.obj
 0002:000027b4       ??_C@_0BN@IGIBPLD@List?5of?5platforms?5for?5indels?$AA@ 100227b4     SamtoolMpileupWorker.obj
 0002:000027d8       ??_C@_0HP@BONHBFIG@Retain?5all?5possible?5alternate?5al@ 100227d8     SamtoolMpileupWorker.obj
 0002:00002858       ??_C@_0BO@PNOJMPOK@Retain?5all?5possible?5alternate?$AA@ 10022858     SamtoolMpileupWorker.obj
 0002:00002878       ??_C@_0FD@HBENNNHH@Indicate?5PL?5is?5generated?5by?5r921@ 10022878     SamtoolMpileupWorker.obj
 0002:000028cc       ??_C@_0M@CBAIEMFO@Indicate?5PL?$AA@ 100228cc     SamtoolMpileupWorker.obj
 0002:000028d8       ??_C@_0DN@NAENGOBF@Suppress?5all?5individual?5genotype@ 100228d8     SamtoolMpileupWorker.obj
 0002:00002918       ??_C@_0BI@HENFHFIA@No?5genotype?5information?$AA@ 10022918     SamtoolMpileupWorker.obj
 0002:00002930       ??_C@_0DO@BDKMNKHL@Skip?5sites?5where?5the?5REF?5field?5i@ 10022930     SamtoolMpileupWorker.obj
 0002:00002970       ??_C@_0N@DOPBNEJI@A?1C?1G?1T?5only?$AA@ 10022970     SamtoolMpileupWorker.obj
 0002:00002980       ??_C@_0EB@PHOIOBKH@List?5of?5sites?5at?5which?5informati@ 10022980     SamtoolMpileupWorker.obj
 0002:000029c4       ??_C@_0O@HDDIOBEE@List?5of?5sites?$AA@ 100229c4     SamtoolMpileupWorker.obj
 0002:000029d4       ??_C@_0DD@FMNAOPEC@Output?5the?5QCALL?5likelihood?5form@ 100229d4     SamtoolMpileupWorker.obj
 0002:00002a08       ??_C@_0BB@BKMFFOG@QCALL?5likelihood?$AA@ 10022a08     SamtoolMpileupWorker.obj
 0002:00002a20       ??_C@_0BCJ@CBFFPHFC@List?5of?5samples?5to?5use?4?5The?5firs@ 10022a20     SamtoolMpileupWorker.obj
 0002:00002b4c       ??_C@_0BA@LOFKEKCG@List?5of?5samples?$AA@ 10022b4c     SamtoolMpileupWorker.obj
 0002:00002b60       ??_C@_0FI@IHCNOBGL@skip?5loci?5where?5the?5fraction?5of?5@ 10022b60     SamtoolMpileupWorker.obj
 0002:00002bb8       ??_C@_0BF@PPJNPCKF@Min?5samples?5fraction?$AA@ 10022bb8     SamtoolMpileupWorker.obj
 0002:00002bd0       ??_C@_0DL@LDIHOMFJ@Call?5per?9sample?5genotypes?5at?5var@ 10022bd0     SamtoolMpileupWorker.obj
 0002:00002c0c       ??_C@_0BF@CJILHEDK@Per?9sample?5genotypes?$AA@ 10022c0c     SamtoolMpileupWorker.obj
 0002:00002c24       ??_C@_0DE@HGKPFEIN@Ratio?5of?5INDEL?9to?9SNP?5mutation?5r@ 10022c24     SamtoolMpileupWorker.obj
 0002:00002c58       ??_C@_0BD@INKENJHD@INDEL?9to?9SNP?5Ratio?$AA@ 10022c58     SamtoolMpileupWorker.obj
 0002:00002c70       ??_C@_0EH@NPAGBJGL@A?5site?5is?5considered?5to?5be?5a?5var@ 10022c70     SamtoolMpileupWorker.obj
 0002:00002cb8       ??_C@_0N@MNCAJIOJ@Max?5P?$CIref?$HMD?$CJ?$AA@ 10022cb8     SamtoolMpileupWorker.obj
 0002:00002cc8       ??_C@_0HL@MGPGBPAE@If?5STR?5can?5be?5full?0?5cond2?0?5flat?5@ 10022cc8     SamtoolMpileupWorker.obj
 0002:00002d44       ??_C@_0CA@LKAMKJIF@Prior?5allele?5frequency?5spectrum?$AA@ 10022d44     SamtoolMpileupWorker.obj
 0002:00002d64       ??_C@_0DJ@LNFODJCF@Scaled?5mutation?5rate?5for?5variant@ 10022d64     SamtoolMpileupWorker.obj
 0002:00002da0       ??_C@_0O@FILMNDFF@Mutation?5rate?$AA@ 10022da0     SamtoolMpileupWorker.obj
 0002:00002db0       ??_C@_0CCK@FCBIAMIB@Enable?5pair?1trio?5calling?4?5For?5tr@ 10022db0     SamtoolMpileupWorker.obj
 0002:00002fdc       ??_C@_0BC@GMKLMOPA@Pair?1trio?5calling?$AA@ 10022fdc     SamtoolMpileupWorker.obj
 0002:00002ff0       ??_C@_0PA@DAFECLCP@Number?5of?5group?91?5samples?4?5This?5@ 10022ff0     SamtoolMpileupWorker.obj
 0002:000030e0       ??_C@_0BC@BHMNOEIL@N?5group?91?5samples?$AA@ 100230e0     SamtoolMpileupWorker.obj
 0002:000030f8       ??_C@_0FF@PADFJFGD@Number?5of?5permutations?5for?5assoc@ 100230f8     SamtoolMpileupWorker.obj
 0002:00003150       ??_C@_0P@NEPCMLKG@N?5permutations?$AA@ 10023150     SamtoolMpileupWorker.obj
 0002:00003160       ??_C@_0EO@KMNONEHO@Only?5perform?5permutations?5for?5P?$CI@ 10023160     SamtoolMpileupWorker.obj
 0002:000031b0       ??_C@_0N@GIAAPIML@Max?5P?$CIchi?$FO2?$CJ?$AA@ 100231b0     SamtoolMpileupWorker.obj
 0002:000031c0       ??_C@_0DH@LEFODLOE@Minimum?5RMS?5mapping?5quality?5for?5@ 100231c0     SamtoolMpileupWorker.obj
 0002:000031f8       ??_C@_0BE@BANFGOEE@Minimum?5RMS?5quality?$AA@ 100231f8     SamtoolMpileupWorker.obj
 0002:0000320c       ??_C@_0CF@EDFDICDP@Minimum?5read?5depth?5?$CIvarFilter?$CJ?5?$CI@ 1002320c     SamtoolMpileupWorker.obj
 0002:00003234       ??_C@_0BD@BCFCPBG@Minimum?5read?5depth?$AA@ 10023234     SamtoolMpileupWorker.obj
 0002:00003248       ??_C@_0CF@BAOMKCBH@Maximum?5read?5depth?5?$CIvarFilter?$CJ?5?$CI@ 10023248     SamtoolMpileupWorker.obj
 0002:00003270       ??_C@_0BD@KGBBKPGP@Maximum?5read?5depth?$AA@ 10023270     SamtoolMpileupWorker.obj
 0002:00003284       ??_C@_0DE@FFEGNOLP@Minimum?5number?5of?5alternate?5base@ 10023284     SamtoolMpileupWorker.obj
 0002:000032b8       ??_C@_0BA@KIGDHOHE@Alternate?5bases?$AA@ 100232b8     SamtoolMpileupWorker.obj
 0002:000032c8       ??_C@_0EA@OKKHKCEG@SNP?5within?5INT?5bp?5around?5a?5gap?5t@ 100232c8     SamtoolMpileupWorker.obj
 0002:00003308       ??_C@_08ONDAKAFF@Gap?5size?$AA@ 10023308     SamtoolMpileupWorker.obj
 0002:00003314       ??_C@_0DK@NJBALMLE@Window?5size?5for?5filtering?5adjace@ 10023314     SamtoolMpileupWorker.obj
 0002:00003350       ??_C@_0M@LHOJMPLD@Window?5size?$AA@ 10023350     SamtoolMpileupWorker.obj
 0002:0000335c       ??_C@_0DO@BENOKJOD@Minimum?5P?9value?5for?5strand?5bias?5@ 1002335c     SamtoolMpileupWorker.obj
 0002:0000339c       ??_C@_0M@GNHPJIJA@Strand?5bias?$AA@ 1002339c     SamtoolMpileupWorker.obj
 0002:000033a8       ??_C@_0DB@LAJFGODH@Minimum?5P?9value?5for?5baseQ?5bias?5?$CI@ 100233a8     SamtoolMpileupWorker.obj
 0002:000033dc       ??_C@_0L@BPIJCAAP@BaseQ?5bias?$AA@ 100233dc     SamtoolMpileupWorker.obj
 0002:000033e8       ??_C@_0DA@GDIPBBFC@Minimum?5P?9value?5for?5mapQ?5bias?5?$CIv@ 100233e8     SamtoolMpileupWorker.obj
 0002:00003418       ??_C@_09PKKMOPFN@MapQ?5bias?$AA@ 10023418     SamtoolMpileupWorker.obj
 0002:00003424       ??_C@_0DI@ONNGCCCD@Minimum?5P?9value?5for?5end?5distance@ 10023424     SamtoolMpileupWorker.obj
 0002:0000345c       ??_C@_0BC@FCMGDABA@End?5distance?5bias?$AA@ 1002345c     SamtoolMpileupWorker.obj
 0002:00003470       ??_C@_0DF@LOHJHLLE@Minimum?5P?9value?5for?5HWE?5?$CIplus?5F?$DM@ 10023470     SamtoolMpileupWorker.obj
 0002:000034a8       ??_C@_03GEOGNDEE@HWE?$AA@  100234a8     SamtoolMpileupWorker.obj
 0002:000034ac       ??_C@_0DH@KAEIANBE@Print?5filtered?5variants?5into?5the@ 100234ac     SamtoolMpileupWorker.obj
 0002:000034e4       ??_C@_0N@FINJPPIF@Log?5filtered?$AA@ 100234e4     SamtoolMpileupWorker.obj
 0002:000034f4       ??_C@_04PLMLMMEO@full?$AA@ 100234f4     SamtoolMpileupWorker.obj
 0002:000034fc       ??_C@_06LOFFLHJM@1e?9100?$AA@ 100234fc     SamtoolMpileupWorker.obj
 0002:00003504       ??_C@_07CCOEHHFD@minimum?$AA@ 10023504     SamtoolMpileupWorker.obj
 0002:0000350c       ??_C@_07MEIENILC@maximum?$AA@ 1002350c     SamtoolMpileupWorker.obj
 0002:00003514       ??_C@_0L@HOCHOMFK@singleStep?$AA@ 10023514     SamtoolMpileupWorker.obj
 0002:00003520       ??_C@_05KCGIHEIJ@cond2?$AA@ 10023520     SamtoolMpileupWorker.obj
 0002:00003528       ??_C@_04FMBJNPFB@flat?$AA@ 10023528     SamtoolMpileupWorker.obj
 0002:00003530       ??_C@_04BJJKJDJA@pair?$AA@ 10023530     SamtoolMpileupWorker.obj
 0002:00003538       ??_C@_08PEGOOCGL@trioauto?$AA@ 10023538     SamtoolMpileupWorker.obj
 0002:00003544       ??_C@_06JAEKBNFB@trioxd?$AA@ 10023544     SamtoolMpileupWorker.obj
 0002:0000354c       ??_C@_06JFMJJJMH@trioxs?$AA@ 1002354c     SamtoolMpileupWorker.obj
 0002:00003554       ??_C@_0L@HLHKPHMD@Input?5port?$AA@ 10023554     SamtoolMpileupWorker.obj
 0002:00003560       ??_C@_04PBAHLACE@File?$AA@ 10023560     SamtoolMpileupWorker.obj
 0002:00003568       ??_C@_03OJNJGGPL@vcf?$AA@  10023568     SamtoolMpileupWorker.obj
 0002:0000356c       ??_C@_0L@NLHBDLEH@USUPP_PERL?$AA@ 1002356c     SamtoolMpileupWorker.obj
 0002:00003578       ??_C@_0BE@PABMJKED@USUPP_VCF_CONSENSUS?$AA@ 10023578     SamtoolMpileupWorker.obj
 0002:0000358c       ??_C@_07HNEBHIML@?$DM?1font?$DO?$AA@ 1002358c     SamtoolMpileupWorker.obj
 0002:00003594       ??_C@_05EPBFLBEJ@unset?$AA@ 10023594     SamtoolMpileupWorker.obj
 0002:0000359c       ??_C@_0BD@HCEOAMGB@?$DMfont?5color?$DN?8red?8?$DO?$AA@ 1002359c     SamtoolMpileupWorker.obj
 0002:000035b0       ??_C@_0CH@BEHGADJN@For?5reference?5sequence?5from?5?$DMu?$DO?$CF@ 100235b0     SamtoolMpileupWorker.obj
 0002:000035d8       ??_C@_0CJ@JDMMMCJE@with?5assembly?5data?5provided?5by?5?$DM@ 100235d8     SamtoolMpileupWorker.obj
 0002:00003604       ??_C@_0BF@PDHMMOEP@?$CF1?5call?5variants?5?$CF2?4?$AA@ 10023604     SamtoolMpileupWorker.obj
 0002:00003620       ??_C@_0EO@IAOCGHDB@Internal?5error?5during?5CallVarian@ 10023620     SamtoolMpileupWorker.obj
 0002:00003670       ??_C@_0BN@PPIPDGA@src?2SamtoolMpileupWorker?4cpp?$AA@ 10023670     SamtoolMpileupWorker.obj
 0002:00003690       ??_C@_0EN@NNJHKLOG@Internal?5error?5during?5CallVarian@ 10023690     SamtoolMpileupWorker.obj
 0002:000036e0       ??_C@_01IDAFKMJL@_?$AA@    100236e0     SamtoolMpileupWorker.obj
 0002:000036e4       ??_C@_0BD@GBNMGBMK@1sl_taskFinished?$CI?$CJ?$AA@ 100236e4     SamtoolMpileupWorker.obj
 0002:000036f8       ??_C@_0BD@PFECGAMD@2si_stateChanged?$CI?$CJ?$AA@ 100236f8     SamtoolMpileupWorker.obj
 0002:0000370c       ??_C@_0DJ@CKAOFNMM@Assembly?5URL?5slot?5is?5empty?4?5Plea@ 1002370c     SamtoolMpileupWorker.obj
 0002:00003748       ??_C@_0DN@JMKDFMP@Ref?5sequence?5URL?5slot?5is?5empty?4?5@ 10023748     SamtoolMpileupWorker.obj
 0002:00003788       ??_C@_0BG@IIEPNAJO@Not?5enough?5references?$AA@ 10023788     SamtoolMpileupWorker.obj
 0002:000037a0       ??_C@_0GI@CFNDPGNA@The?5dataset?5slot?5is?5not?5binded?0?5@ 100237a0     SamtoolMpileupWorker.obj
 0002:00003808       ??_C@_0BG@OKFCOLFO@Not?5enough?5assemblies?$AA@ 10023808     SamtoolMpileupWorker.obj
 0002:00003820       ??_C@_0CD@ELGHHDAM@1sl_valueChanged?$CIconst?5QVariant?5@ 10023820     SamtoolMpileupWorker.obj
 0002:00003844       ??_C@_0BO@JONBIMPD@2textChanged?$CIconst?5QString?5?$CG?$CJ?$AA@ 10023844     SamtoolMpileupWorker.obj
 0002:00003864       ??_C@_0BE@LGBLLFOL@1sl_actorModified?$CI?$CJ?$AA@ 10023864     SamtoolMpileupWorker.obj
 0002:00003878       ??_C@_0BD@FGIDJNMI@2si_labelChanged?$CI?$CJ?$AA@ 10023878     SamtoolMpileupWorker.obj
 0002:0000388c       ??_C@_0P@DIBOLHGA@2si_modified?$CI?$CJ?$AA@ 1002388c     SamtoolMpileupWorker.obj
 0002:0000389c       ??_C@_0BC@HBGBGNIM@2bindingChanged?$CI?$CJ?$AA@ 1002389c     SamtoolMpileupWorker.obj
 0002:000038b0       __real@00000000            100238b0     SamtoolMpileupWorker.obj
 0002:000038b8       __real@3f1a36e2eb1c432d    100238b8     SamtoolMpileupWorker.obj
 0002:000038c0       __real@3f50624dd2f1a9fc    100238c0     SamtoolMpileupWorker.obj
 0002:000038c8       __real@3f847ae147ae147b    100238c8     SamtoolMpileupWorker.obj
 0002:000038d0       __real@3fb999999999999a    100238d0     SamtoolMpileupWorker.obj
 0002:000038d8       __real@3fe0000000000000    100238d8     SamtoolMpileupWorker.obj
 0002:000038e0       __real@bff0000000000000    100238e0     SamtoolMpileupWorker.obj
 0002:000038ec       ??_7SamtoolsPlugin@U2@@6B@ 100238ec     SamtoolsPlugin.obj
 0002:00003918       ??_C@_0CG@IPPFMNCL@Samtools?5plugin?5for?5NGS?5data?5ana@ 10023918     SamtoolsPlugin.obj
 0002:00003940       ??_C@_0BA@JCPGFOOB@Samtools?5plugin?$AA@ 10023940     SamtoolsPlugin.obj
 0002:00003cac       ?value@?$integral_constant@_N$0A@@std@@2_NB 10023cac     MSVCRT:ti_inst.obj
 0002:00003cad       ?value@?$integral_constant@_N$00@std@@2_NB 10023cad     MSVCRT:ti_inst.obj
 0002:00003cb4       ??_7type_info@@6B@         10023cb4     MSVCRT:ti_inst.obj
 0002:00003cb8       __pRawDllMain              10023cb8     MSVCRT:crtdll.obj
 0002:00003cb8       __pDefaultRawDllMain       10023cb8     MSVCRT:crtdll.obj
 0002:00003cc4       ?ProcessDetach@NativeDll@<CrtImplementationDetails>@@0IB 10023cc4     MSVCRT:initsect.obj
 0002:00003cc8       ?ProcessAttach@NativeDll@<CrtImplementationDetails>@@0IB 10023cc8     MSVCRT:initsect.obj
 0002:00003ccc       ?ThreadAttach@NativeDll@<CrtImplementationDetails>@@0IB 10023ccc     MSVCRT:initsect.obj
 0002:00003cd0       ?ThreadDetach@NativeDll@<CrtImplementationDetails>@@0IB 10023cd0     MSVCRT:initsect.obj
 0002:00003cd4       ?ProcessVerifier@NativeDll@<CrtImplementationDetails>@@0IB 10023cd4     MSVCRT:initsect.obj
 0002:00003cd8       __load_config_used         10023cd8     MSVCRT:loadcfg.obj
 0002:00003d90       ??_R4error_category@std@@6B@ 10023d90     AssemblySamtoolsMpileup.obj
 0002:00003da4       ??_R3error_category@std@@8 10023da4     AssemblySamtoolsMpileup.obj
 0002:00003db4       ??_R2error_category@std@@8 10023db4     AssemblySamtoolsMpileup.obj
 0002:00003dbc       ??_R1A@?0A@EA@error_category@std@@8 10023dbc     AssemblySamtoolsMpileup.obj
 0002:00003dd8       ??_R4_Generic_error_category@std@@6B@ 10023dd8     AssemblySamtoolsMpileup.obj
 0002:00003dec       ??_R3_Generic_error_category@std@@8 10023dec     AssemblySamtoolsMpileup.obj
 0002:00003dfc       ??_R2_Generic_error_category@std@@8 10023dfc     AssemblySamtoolsMpileup.obj
 0002:00003e08       ??_R1A@?0A@EA@_Generic_error_category@std@@8 10023e08     AssemblySamtoolsMpileup.obj
 0002:00003e24       ??_R4_Iostream_error_category@std@@6B@ 10023e24     AssemblySamtoolsMpileup.obj
 0002:00003e38       ??_R3_Iostream_error_category@std@@8 10023e38     AssemblySamtoolsMpileup.obj
 0002:00003e48       ??_R2_Iostream_error_category@std@@8 10023e48     AssemblySamtoolsMpileup.obj
 0002:00003e58       ??_R1A@?0A@EA@_Iostream_error_category@std@@8 10023e58     AssemblySamtoolsMpileup.obj
 0002:00003e74       ??_R4_System_error_category@std@@6B@ 10023e74     AssemblySamtoolsMpileup.obj
 0002:00003e88       ??_R3_System_error_category@std@@8 10023e88     AssemblySamtoolsMpileup.obj
 0002:00003e98       ??_R2_System_error_category@std@@8 10023e98     AssemblySamtoolsMpileup.obj
 0002:00003ea8       ??_R1A@?0A@EA@_System_error_category@std@@8 10023ea8     AssemblySamtoolsMpileup.obj
 0002:00003ec4       ??_R1A@?0A@EA@QObject@@8   10023ec4     AssemblySamtoolsMpileup.obj
 0002:00003ee0       ??_R3QObject@@8            10023ee0     AssemblySamtoolsMpileup.obj
 0002:00003ef0       ??_R2QObject@@8            10023ef0     AssemblySamtoolsMpileup.obj
 0002:00003ef8       ??_R4LoadDocumentTask@U2@@6B@ 10023ef8     AssemblySamtoolsMpileup.obj
 0002:00003f0c       ??_R3LoadDocumentTask@U2@@8 10023f0c     AssemblySamtoolsMpileup.obj
 0002:00003f1c       ??_R2LoadDocumentTask@U2@@8 10023f1c     AssemblySamtoolsMpileup.obj
 0002:00003f30       ??_R1A@?0A@EA@LoadDocumentTask@U2@@8 10023f30     AssemblySamtoolsMpileup.obj
 0002:00003f4c       ??_R1A@?0A@EA@DocumentProviderTask@U2@@8 10023f4c     AssemblySamtoolsMpileup.obj
 0002:00003f68       ??_R3DocumentProviderTask@U2@@8 10023f68     AssemblySamtoolsMpileup.obj
 0002:00003f78       ??_R2DocumentProviderTask@U2@@8 10023f78     AssemblySamtoolsMpileup.obj
 0002:00003f88       ??_R1A@?0A@EA@Task@U2@@8   10023f88     AssemblySamtoolsMpileup.obj
 0002:00003fa4       ??_R3Task@U2@@8            10023fa4     AssemblySamtoolsMpileup.obj
 0002:00003fb4       ??_R2Task@U2@@8            10023fb4     AssemblySamtoolsMpileup.obj
 0002:00003fc0       ??_R4SamtoolsMpileupTask@LocalWorkflow@U2@@6B@ 10023fc0     AssemblySamtoolsMpileup.obj
 0002:00003fd4       ??_R3SamtoolsMpileupTask@LocalWorkflow@U2@@8 10023fd4     AssemblySamtoolsMpileup.obj
 0002:00003fe4       ??_R2SamtoolsMpileupTask@LocalWorkflow@U2@@8 10023fe4     AssemblySamtoolsMpileup.obj
 0002:00003ff8       ??_R1A@?0A@EA@SamtoolsMpileupTask@LocalWorkflow@U2@@8 10023ff8     AssemblySamtoolsMpileup.obj
 0002:00004014       ??_R1A@?0A@EA@ExternalToolSupportTask@U2@@8 10024014     AssemblySamtoolsMpileup.obj
 0002:00004030       ??_R3ExternalToolSupportTask@U2@@8 10024030     AssemblySamtoolsMpileup.obj
 0002:00004040       ??_R2ExternalToolSupportTask@U2@@8 10024040     AssemblySamtoolsMpileup.obj
 0002:00004050       ??_R4CallVariantsTask@LocalWorkflow@U2@@6B@ 10024050     AssemblySamtoolsMpileup.obj
 0002:00004064       ??_R3CallVariantsTask@LocalWorkflow@U2@@8 10024064     AssemblySamtoolsMpileup.obj
 0002:00004074       ??_R2CallVariantsTask@LocalWorkflow@U2@@8 10024074     AssemblySamtoolsMpileup.obj
 0002:00004088       ??_R1A@?0A@EA@CallVariantsTask@LocalWorkflow@U2@@8 10024088     AssemblySamtoolsMpileup.obj
 0002:000040a4       ??_R4QDoubleValidator@@6B@ 100240a4     SamtoolMpileupWorker.obj
 0002:000040b8       ??_R3QDoubleValidator@@8   100240b8     SamtoolMpileupWorker.obj
 0002:000040c8       ??_R2QDoubleValidator@@8   100240c8     SamtoolMpileupWorker.obj
 0002:000040d8       ??_R1A@?0A@EA@QDoubleValidator@@8 100240d8     SamtoolMpileupWorker.obj
 0002:000040f4       ??_R1A@?0A@EA@QValidator@@8 100240f4     SamtoolMpileupWorker.obj
 0002:00004110       ??_R3QValidator@@8         10024110     SamtoolMpileupWorker.obj
 0002:00004120       ??_R2QValidator@@8         10024120     SamtoolMpileupWorker.obj
 0002:0000412c       ??_R4QLineEdit@@6BQObject@@@ 1002412c     SamtoolMpileupWorker.obj
 0002:00004140       ??_R3QLineEdit@@8          10024140     SamtoolMpileupWorker.obj
 0002:00004150       ??_R2QLineEdit@@8          10024150     SamtoolMpileupWorker.obj
 0002:00004164       ??_R1A@?0A@EA@QLineEdit@@8 10024164     SamtoolMpileupWorker.obj
 0002:00004180       ??_R1A@?0A@EA@QWidget@@8   10024180     SamtoolMpileupWorker.obj
 0002:0000419c       ??_R3QWidget@@8            1002419c     SamtoolMpileupWorker.obj
 0002:000041ac       ??_R2QWidget@@8            100241ac     SamtoolMpileupWorker.obj
 0002:000041bc       ??_R17?0A@EA@QPaintDevice@@8 100241bc     SamtoolMpileupWorker.obj
 0002:000041d8       ??_R3QPaintDevice@@8       100241d8     SamtoolMpileupWorker.obj
 0002:000041e8       ??_R2QPaintDevice@@8       100241e8     SamtoolMpileupWorker.obj
 0002:000041f0       ??_R1A@?0A@EA@QPaintDevice@@8 100241f0     SamtoolMpileupWorker.obj
 0002:0000420c       ??_R4QLineEdit@@6BQPaintDevice@@@ 1002420c     SamtoolMpileupWorker.obj
 0002:00004220       ??_R4VisibilityRelation@U2@@6B@ 10024220     SamtoolMpileupWorker.obj
 0002:00004234       ??_R3VisibilityRelation@U2@@8 10024234     SamtoolMpileupWorker.obj
 0002:00004244       ??_R2VisibilityRelation@U2@@8 10024244     SamtoolMpileupWorker.obj
 0002:00004250       ??_R1A@?0A@EA@VisibilityRelation@U2@@8 10024250     SamtoolMpileupWorker.obj
 0002:0000426c       ??_R1A@?0A@EA@AttributeRelation@U2@@8 1002426c     SamtoolMpileupWorker.obj
 0002:00004288       ??_R3AttributeRelation@U2@@8 10024288     SamtoolMpileupWorker.obj
 0002:00004298       ??_R2AttributeRelation@U2@@8 10024298     SamtoolMpileupWorker.obj
 0002:000042a0       ??_R4Descriptor@U2@@6B@    100242a0     SamtoolMpileupWorker.obj
 0002:000042b4       ??_R3Descriptor@U2@@8      100242b4     SamtoolMpileupWorker.obj
 0002:000042c4       ??_R2Descriptor@U2@@8      100242c4     SamtoolMpileupWorker.obj
 0002:000042cc       ??_R1A@?0A@EA@Descriptor@U2@@8 100242cc     SamtoolMpileupWorker.obj
 0002:000042e8       ??_R4MapDataType@U2@@6B@   100242e8     SamtoolMpileupWorker.obj
 0002:000042fc       ??_R3MapDataType@U2@@8     100242fc     SamtoolMpileupWorker.obj
 0002:0000430c       ??_R2MapDataType@U2@@8     1002430c     SamtoolMpileupWorker.obj
 0002:00004320       ??_R1A@?0A@EA@MapDataType@U2@@8 10024320     SamtoolMpileupWorker.obj
 0002:0000433c       ??_R1A@?0A@EA@DataType@U2@@8 1002433c     SamtoolMpileupWorker.obj
 0002:00004358       ??_R3DataType@U2@@8        10024358     SamtoolMpileupWorker.obj
 0002:00004368       ??_R2DataType@U2@@8        10024368     SamtoolMpileupWorker.obj
 0002:00004378       ??_R1BA@?0A@EA@QSharedData@@8 10024378     SamtoolMpileupWorker.obj
 0002:00004394       ??_R3QSharedData@@8        10024394     SamtoolMpileupWorker.obj
 0002:000043a4       ??_R2QSharedData@@8        100243a4     SamtoolMpileupWorker.obj
 0002:000043ac       ??_R1A@?0A@EA@QSharedData@@8 100243ac     SamtoolMpileupWorker.obj
 0002:000043c8       ??_R4PortRelationDescriptor@U2@@6B@ 100243c8     SamtoolMpileupWorker.obj
 0002:000043dc       ??_R3PortRelationDescriptor@U2@@8 100243dc     SamtoolMpileupWorker.obj
 0002:000043ec       ??_R2PortRelationDescriptor@U2@@8 100243ec     SamtoolMpileupWorker.obj
 0002:000043f4       ??_R1A@?0A@EA@PortRelationDescriptor@U2@@8 100243f4     SamtoolMpileupWorker.obj
 0002:00004410       ??_R4Attribute@U2@@6B@     10024410     SamtoolMpileupWorker.obj
 0002:00004424       ??_R3Attribute@U2@@8       10024424     SamtoolMpileupWorker.obj
 0002:00004434       ??_R2Attribute@U2@@8       10024434     SamtoolMpileupWorker.obj
 0002:00004440       ??_R1A@?0A@EA@Attribute@U2@@8 10024440     SamtoolMpileupWorker.obj
 0002:0000445c       ??_R3ConfigurationEditor@U2@@8 1002445c     SamtoolMpileupWorker.obj
 0002:0000446c       ??_R2ConfigurationEditor@U2@@8 1002446c     SamtoolMpileupWorker.obj
 0002:00004478       ??_R1A@?0A@EA@ConfigurationEditor@U2@@8 10024478     SamtoolMpileupWorker.obj
 0002:00004494       ??_R4DelegateEditor@U2@@6B@ 10024494     SamtoolMpileupWorker.obj
 0002:000044a8       ??_R3DelegateEditor@U2@@8  100244a8     SamtoolMpileupWorker.obj
 0002:000044b8       ??_R2DelegateEditor@U2@@8  100244b8     SamtoolMpileupWorker.obj
 0002:000044c8       ??_R1A@?0A@EA@DelegateEditor@U2@@8 100244c8     SamtoolMpileupWorker.obj
 0002:000044e4       ??_R4URLDelegate@U2@@6B@   100244e4     SamtoolMpileupWorker.obj
 0002:000044f8       ??_R3URLDelegate@U2@@8     100244f8     SamtoolMpileupWorker.obj
 0002:00004508       ??_R2URLDelegate@U2@@8     10024508     SamtoolMpileupWorker.obj
 0002:00004520       ??_R1A@?0A@EA@URLDelegate@U2@@8 10024520     SamtoolMpileupWorker.obj
 0002:0000453c       ??_R1A@?0A@EA@PropertyDelegate@U2@@8 1002453c     SamtoolMpileupWorker.obj
 0002:00004558       ??_R3PropertyDelegate@U2@@8 10024558     SamtoolMpileupWorker.obj
 0002:00004568       ??_R2PropertyDelegate@U2@@8 10024568     SamtoolMpileupWorker.obj
 0002:0000457c       ??_R1A@?0A@EA@QItemDelegate@@8 1002457c     SamtoolMpileupWorker.obj
 0002:00004598       ??_R3QItemDelegate@@8      10024598     SamtoolMpileupWorker.obj
 0002:000045a8       ??_R2QItemDelegate@@8      100245a8     SamtoolMpileupWorker.obj
 0002:000045b8       ??_R1A@?0A@EA@QAbstractItemDelegate@@8 100245b8     SamtoolMpileupWorker.obj
 0002:000045d4       ??_R3QAbstractItemDelegate@@8 100245d4     SamtoolMpileupWorker.obj
 0002:000045e4       ??_R2QAbstractItemDelegate@@8 100245e4     SamtoolMpileupWorker.obj
 0002:000045f0       ??_R4SpinBoxDelegate@U2@@6B@ 100245f0     SamtoolMpileupWorker.obj
 0002:00004604       ??_R3SpinBoxDelegate@U2@@8 10024604     SamtoolMpileupWorker.obj
 0002:00004614       ??_R2SpinBoxDelegate@U2@@8 10024614     SamtoolMpileupWorker.obj
 0002:0000462c       ??_R1A@?0A@EA@SpinBoxDelegate@U2@@8 1002462c     SamtoolMpileupWorker.obj
 0002:00004648       ??_R4DoubleSpinBoxDelegate@U2@@6B@ 10024648     SamtoolMpileupWorker.obj
 0002:0000465c       ??_R3DoubleSpinBoxDelegate@U2@@8 1002465c     SamtoolMpileupWorker.obj
 0002:0000466c       ??_R2DoubleSpinBoxDelegate@U2@@8 1002466c     SamtoolMpileupWorker.obj
 0002:00004684       ??_R1A@?0A@EA@DoubleSpinBoxDelegate@U2@@8 10024684     SamtoolMpileupWorker.obj
 0002:000046a0       ??_R4ComboBoxDelegate@U2@@6B@ 100246a0     SamtoolMpileupWorker.obj
 0002:000046b4       ??_R3ComboBoxDelegate@U2@@8 100246b4     SamtoolMpileupWorker.obj
 0002:000046c4       ??_R2ComboBoxDelegate@U2@@8 100246c4     SamtoolMpileupWorker.obj
 0002:000046dc       ??_R1A@?0A@EA@ComboBoxDelegate@U2@@8 100246dc     SamtoolMpileupWorker.obj
 0002:000046f8       ??_R4PortDescriptor@Workflow@U2@@6B@ 100246f8     SamtoolMpileupWorker.obj
 0002:0000470c       ??_R3PortDescriptor@Workflow@U2@@8 1002470c     SamtoolMpileupWorker.obj
 0002:0000471c       ??_R2PortDescriptor@Workflow@U2@@8 1002471c     SamtoolMpileupWorker.obj
 0002:00004728       ??_R1A@?0A@EA@PortDescriptor@Workflow@U2@@8 10024728     SamtoolMpileupWorker.obj
 0002:00004744       ??_R17?0A@EA@Descriptor@U2@@8 10024744     SamtoolMpileupWorker.obj
 0002:00004760       ??_R4IntegralBusActorPrototype@Workflow@U2@@6BQObject@@@ 10024760     SamtoolMpileupWorker.obj
 0002:00004774       ??_R3IntegralBusActorPrototype@Workflow@U2@@8 10024774     SamtoolMpileupWorker.obj
 0002:00004784       ??_R2IntegralBusActorPrototype@Workflow@U2@@8 10024784     SamtoolMpileupWorker.obj
 0002:0000479c       ??_R1A@?0A@EA@IntegralBusActorPrototype@Workflow@U2@@8 1002479c     SamtoolMpileupWorker.obj
 0002:000047b8       ??_R1A@?0A@EA@ActorPrototype@Workflow@U2@@8 100247b8     SamtoolMpileupWorker.obj
 0002:000047d4       ??_R3ActorPrototype@Workflow@U2@@8 100247d4     SamtoolMpileupWorker.obj
 0002:000047e4       ??_R2ActorPrototype@Workflow@U2@@8 100247e4     SamtoolMpileupWorker.obj
 0002:000047f8       ??_R17?0A@EA@VisualDescriptor@U2@@8 100247f8     SamtoolMpileupWorker.obj
 0002:00004814       ??_R3VisualDescriptor@U2@@8 10024814     SamtoolMpileupWorker.obj
 0002:00004824       ??_R2VisualDescriptor@U2@@8 10024824     SamtoolMpileupWorker.obj
 0002:00004830       ??_R1A@?0A@EA@VisualDescriptor@U2@@8 10024830     SamtoolMpileupWorker.obj
 0002:0000484c       ??_R4IntegralBusActorPrototype@Workflow@U2@@6BVisualDescriptor@2@@ 1002484c     SamtoolMpileupWorker.obj
 0002:00004860       ??_R4CallVariantsPrompter@LocalWorkflow@U2@@6BActorDocument@Workflow@2@@ 10024860     SamtoolMpileupWorker.obj
 0002:00004874       ??_R3CallVariantsPrompter@LocalWorkflow@U2@@8 10024874     SamtoolMpileupWorker.obj
 0002:00004884       ??_R2CallVariantsPrompter@LocalWorkflow@U2@@8 10024884     SamtoolMpileupWorker.obj
 0002:000048a4       ??_R1A@?0A@EA@CallVariantsPrompter@LocalWorkflow@U2@@8 100248a4     SamtoolMpileupWorker.obj
 0002:000048c0       ??_R1A@?0A@EA@?$PrompterBase@VCallVariantsPrompter@LocalWorkflow@U2@@@U2@@8 100248c0     SamtoolMpileupWorker.obj
 0002:000048dc       ??_R3?$PrompterBase@VCallVariantsPrompter@LocalWorkflow@U2@@@U2@@8 100248dc     SamtoolMpileupWorker.obj
 0002:000048ec       ??_R2?$PrompterBase@VCallVariantsPrompter@LocalWorkflow@U2@@@U2@@8 100248ec     SamtoolMpileupWorker.obj
 0002:00004908       ??_R1A@?0A@EA@PrompterBaseImpl@U2@@8 10024908     SamtoolMpileupWorker.obj
 0002:00004924       ??_R3PrompterBaseImpl@U2@@8 10024924     SamtoolMpileupWorker.obj
 0002:00004934       ??_R2PrompterBaseImpl@U2@@8 10024934     SamtoolMpileupWorker.obj
 0002:0000494c       ??_R1A@?0A@EA@ActorDocument@Workflow@U2@@8 1002494c     SamtoolMpileupWorker.obj
 0002:00004968       ??_R3ActorDocument@Workflow@U2@@8 10024968     SamtoolMpileupWorker.obj
 0002:00004978       ??_R2ActorDocument@Workflow@U2@@8 10024978     SamtoolMpileupWorker.obj
 0002:00004988       ??_R1A@?0A@EA@QTextDocument@@8 10024988     SamtoolMpileupWorker.obj
 0002:000049a4       ??_R3QTextDocument@@8      100249a4     SamtoolMpileupWorker.obj
 0002:000049b4       ??_R2QTextDocument@@8      100249b4     SamtoolMpileupWorker.obj
 0002:000049c0       ??_R1M@?0A@EA@Prompter@Workflow@U2@@8 100249c0     SamtoolMpileupWorker.obj
 0002:000049dc       ??_R3Prompter@Workflow@U2@@8 100249dc     SamtoolMpileupWorker.obj
 0002:000049ec       ??_R2Prompter@Workflow@U2@@8 100249ec     SamtoolMpileupWorker.obj
 0002:000049f4       ??_R1A@?0A@EA@Prompter@Workflow@U2@@8 100249f4     SamtoolMpileupWorker.obj
 0002:00004a10       ??_R4CallVariantsPrompter@LocalWorkflow@U2@@6BPrompter@Workflow@2@@ 10024a10     SamtoolMpileupWorker.obj
 0002:00004a24       ??_R4?$PrompterBase@VCallVariantsPrompter@LocalWorkflow@U2@@@U2@@6BActorDocument@Workflow@1@@ 10024a24     SamtoolMpileupWorker.obj
 0002:00004a38       ??_R4?$PrompterBase@VCallVariantsPrompter@LocalWorkflow@U2@@@U2@@6BPrompter@Workflow@1@@ 10024a38     SamtoolMpileupWorker.obj
 0002:00004a4c       ??_R4CallVariantsWorker@LocalWorkflow@U2@@6BQObject@@@ 10024a4c     SamtoolMpileupWorker.obj
 0002:00004a60       ??_R3CallVariantsWorker@LocalWorkflow@U2@@8 10024a60     SamtoolMpileupWorker.obj
 0002:00004a70       ??_R2CallVariantsWorker@LocalWorkflow@U2@@8 10024a70     SamtoolMpileupWorker.obj
 0002:00004a88       ??_R1A@?0A@EA@CallVariantsWorker@LocalWorkflow@U2@@8 10024a88     SamtoolMpileupWorker.obj
 0002:00004aa4       ??_R1A@?0A@EA@BaseWorker@LocalWorkflow@U2@@8 10024aa4     SamtoolMpileupWorker.obj
 0002:00004ac0       ??_R3BaseWorker@LocalWorkflow@U2@@8 10024ac0     SamtoolMpileupWorker.obj
 0002:00004ad0       ??_R2BaseWorker@LocalWorkflow@U2@@8 10024ad0     SamtoolMpileupWorker.obj
 0002:00004ae4       ??_R17?0A@EA@Worker@Workflow@U2@@8 10024ae4     SamtoolMpileupWorker.obj
 0002:00004b00       ??_R3Worker@Workflow@U2@@8 10024b00     SamtoolMpileupWorker.obj
 0002:00004b10       ??_R2Worker@Workflow@U2@@8 10024b10     SamtoolMpileupWorker.obj
 0002:00004b18       ??_R1A@?0A@EA@Worker@Workflow@U2@@8 10024b18     SamtoolMpileupWorker.obj
 0002:00004b34       ??_R1BA@?0A@EA@CommunicationSubject@Workflow@U2@@8 10024b34     SamtoolMpileupWorker.obj
 0002:00004b50       ??_R3CommunicationSubject@Workflow@U2@@8 10024b50     SamtoolMpileupWorker.obj
 0002:00004b60       ??_R2CommunicationSubject@Workflow@U2@@8 10024b60     SamtoolMpileupWorker.obj
 0002:00004b68       ??_R1A@?0A@EA@CommunicationSubject@Workflow@U2@@8 10024b68     SamtoolMpileupWorker.obj
 0002:00004b84       ??_R4CallVariantsWorker@LocalWorkflow@U2@@6BWorker@Workflow@2@@ 10024b84     SamtoolMpileupWorker.obj
 0002:00004b98       ??_R4CallVariantsWorker@LocalWorkflow@U2@@6BCommunicationSubject@Workflow@2@@ 10024b98     SamtoolMpileupWorker.obj
 0002:00004bac       ??_R4CallVariantsWorkerFactory@LocalWorkflow@U2@@6B?$IdRegistry@VDomainFactory@Workflow@U2@@@2@@ 10024bac     SamtoolMpileupWorker.obj
 0002:00004bc0       ??_R3CallVariantsWorkerFactory@LocalWorkflow@U2@@8 10024bc0     SamtoolMpileupWorker.obj
 0002:00004bd0       ??_R2CallVariantsWorkerFactory@LocalWorkflow@U2@@8 10024bd0     SamtoolMpileupWorker.obj
 0002:00004be4       ??_R1A@?0A@EA@CallVariantsWorkerFactory@LocalWorkflow@U2@@8 10024be4     SamtoolMpileupWorker.obj
 0002:00004c00       ??_R1A@?0A@EA@DomainFactory@Workflow@U2@@8 10024c00     SamtoolMpileupWorker.obj
 0002:00004c1c       ??_R3DomainFactory@Workflow@U2@@8 10024c1c     SamtoolMpileupWorker.obj
 0002:00004c2c       ??_R2DomainFactory@Workflow@U2@@8 10024c2c     SamtoolMpileupWorker.obj
 0002:00004c3c       ??_R1A@?0A@EA@?$IdRegistry@VDomainFactory@Workflow@U2@@@U2@@8 10024c3c     SamtoolMpileupWorker.obj
 0002:00004c58       ??_R3?$IdRegistry@VDomainFactory@Workflow@U2@@@U2@@8 10024c58     SamtoolMpileupWorker.obj
 0002:00004c68       ??_R2?$IdRegistry@VDomainFactory@Workflow@U2@@@U2@@8 10024c68     SamtoolMpileupWorker.obj
 0002:00004c70       ??_R4CallVariantsWorkerFactory@LocalWorkflow@U2@@6BDescriptor@2@@ 10024c70     SamtoolMpileupWorker.obj
 0002:00004c84       ??_R4ScientificDoubleWidget@LocalWorkflow@U2@@6BQObject@@@ 10024c84     SamtoolMpileupWorker.obj
 0002:00004c98       ??_R3ScientificDoubleWidget@LocalWorkflow@U2@@8 10024c98     SamtoolMpileupWorker.obj
 0002:00004ca8       ??_R2ScientificDoubleWidget@LocalWorkflow@U2@@8 10024ca8     SamtoolMpileupWorker.obj
 0002:00004cc0       ??_R1A@?0A@EA@ScientificDoubleWidget@LocalWorkflow@U2@@8 10024cc0     SamtoolMpileupWorker.obj
 0002:00004cdc       ??_R1A@?0A@EA@PropertyWidget@U2@@8 10024cdc     SamtoolMpileupWorker.obj
 0002:00004cf8       ??_R3PropertyWidget@U2@@8  10024cf8     SamtoolMpileupWorker.obj
 0002:00004d08       ??_R2PropertyWidget@U2@@8  10024d08     SamtoolMpileupWorker.obj
 0002:00004d1c       ??_R4ScientificDoubleWidget@LocalWorkflow@U2@@6BQPaintDevice@@@ 10024d1c     SamtoolMpileupWorker.obj
 0002:00004d30       ??_R4ScientificDoubleDelegate@LocalWorkflow@U2@@6B@ 10024d30     SamtoolMpileupWorker.obj
 0002:00004d44       ??_R3ScientificDoubleDelegate@LocalWorkflow@U2@@8 10024d44     SamtoolMpileupWorker.obj
 0002:00004d54       ??_R2ScientificDoubleDelegate@LocalWorkflow@U2@@8 10024d54     SamtoolMpileupWorker.obj
 0002:00004d6c       ??_R1A@?0A@EA@ScientificDoubleDelegate@LocalWorkflow@U2@@8 10024d6c     SamtoolMpileupWorker.obj
 0002:00004d88       ??_R4EmptySlotValidator@LocalWorkflow@U2@@6B@ 10024d88     SamtoolMpileupWorker.obj
 0002:00004d9c       ??_R3EmptySlotValidator@LocalWorkflow@U2@@8 10024d9c     SamtoolMpileupWorker.obj
 0002:00004dac       ??_R2EmptySlotValidator@LocalWorkflow@U2@@8 10024dac     SamtoolMpileupWorker.obj
 0002:00004db8       ??_R1A@?0A@EA@EmptySlotValidator@LocalWorkflow@U2@@8 10024db8     SamtoolMpileupWorker.obj
 0002:00004dd4       ??_R1A@?0A@EA@ConfigurationValidator@U2@@8 10024dd4     SamtoolMpileupWorker.obj
 0002:00004df0       ??_R3ConfigurationValidator@U2@@8 10024df0     SamtoolMpileupWorker.obj
 0002:00004e00       ??_R2ConfigurationValidator@U2@@8 10024e00     SamtoolMpileupWorker.obj
 0002:00004e08       ??_R4SamtoolsPlugin@U2@@6B@ 10024e08     SamtoolsPlugin.obj
 0002:00004e1c       ??_R3SamtoolsPlugin@U2@@8  10024e1c     SamtoolsPlugin.obj
 0002:00004e2c       ??_R2SamtoolsPlugin@U2@@8  10024e2c     SamtoolsPlugin.obj
 0002:00004e3c       ??_R1A@?0A@EA@SamtoolsPlugin@U2@@8 10024e3c     SamtoolsPlugin.obj
 0002:00004e58       ??_R1A@?0A@EA@Plugin@U2@@8 10024e58     SamtoolsPlugin.obj
 0002:00004e74       ??_R3Plugin@U2@@8          10024e74     SamtoolsPlugin.obj
 0002:00004e84       ??_R2Plugin@U2@@8          10024e84     SamtoolsPlugin.obj
 0002:00004e90       ??_R4type_info@@6B@        10024e90     MSVCRT:ti_inst.obj
 0002:00004ea4       ??_R3type_info@@8          10024ea4     MSVCRT:ti_inst.obj
 0002:00004eb4       ??_R2type_info@@8          10024eb4     MSVCRT:ti_inst.obj
 0002:00004ebc       ??_R1A@?0A@EA@type_info@@8 10024ebc     MSVCRT:ti_inst.obj
 0002:00004ee0       ___safe_se_handler_table   10024ee0     <linker-defined>
 0002:0000515c       ___rtc_iaa                 1002515c     MSVCRT:initsect.obj
 0002:00005160       ___rtc_izz                 10025160     MSVCRT:initsect.obj
 0002:00005164       ___rtc_taa                 10025164     MSVCRT:initsect.obj
 0002:00005168       ___rtc_tzz                 10025168     MSVCRT:initsect.obj
 0002:00009ee4       __IMPORT_DESCRIPTOR_U2Core 10029ee4     U2Core:U2Core.dll
 0002:00009ef8       __IMPORT_DESCRIPTOR_U2Lang 10029ef8     U2Lang:U2Lang.dll
 0002:00009f0c       __IMPORT_DESCRIPTOR_U2Designer 10029f0c     U2Designer:U2Designer.dll
 0002:00009f20       __IMPORT_DESCRIPTOR_Qt5Widgets 10029f20     Qt5Widgets:Qt5Widgets.dll
 0002:00009f34       __IMPORT_DESCRIPTOR_Qt5Gui 10029f34     Qt5Gui:Qt5Gui.dll
 0002:00009f48       __IMPORT_DESCRIPTOR_Qt5Script 10029f48     Qt5Script:Qt5Script.dll
 0002:00009f5c       __IMPORT_DESCRIPTOR_Qt5Core 10029f5c     Qt5Core:Qt5Core.dll
 0002:00009f70       __IMPORT_DESCRIPTOR_MSVCP120 10029f70     msvcprt:MSVCP120.dll
 0002:00009f84       __IMPORT_DESCRIPTOR_MSVCR120 10029f84     MSVCRT:MSVCR120.dll
 0002:00009f98       __IMPORT_DESCRIPTOR_KERNEL32 10029f98     kernel32:KERNEL32.dll
 0002:00009fac       __NULL_IMPORT_DESCRIPTOR   10029fac     U2Core:U2Core.dll
 0003:00000000       ?_Generic_object@?$_Error_objects@H@std@@2V_Generic_error_category@2@A 10032000     AssemblySamtoolsMpileup.obj
 0003:00000004       ?_Iostream_object@?$_Error_objects@H@std@@2V_Iostream_error_category@2@A 10032004     AssemblySamtoolsMpileup.obj
 0003:00000008       ?_System_object@?$_Error_objects@H@std@@2V_System_error_category@2@A 10032008     AssemblySamtoolsMpileup.obj
 0003:0000000c       ?staticMetaObject@SamtoolsMpileupTask@LocalWorkflow@U2@@2UQMetaObject@@B 1003200c     moc_AssemblySamtoolsMpileup.obj
 0003:00000024       ?staticMetaObject@CallVariantsTask@LocalWorkflow@U2@@2UQMetaObject@@B 10032024     moc_AssemblySamtoolsMpileup.obj
 0003:0000003c       ?staticMetaObject@CallVariantsPrompter@LocalWorkflow@U2@@2UQMetaObject@@B 1003203c     moc_SamtoolMpileupWorker.obj
 0003:00000054       ?staticMetaObject@CallVariantsWorker@LocalWorkflow@U2@@2UQMetaObject@@B 10032054     moc_SamtoolMpileupWorker.obj
 0003:0000006c       ?staticMetaObject@ScientificDoubleWidget@LocalWorkflow@U2@@2UQMetaObject@@B 1003206c     moc_SamtoolMpileupWorker.obj
 0003:00000084       ?staticMetaObject@SamtoolsPlugin@U2@@2UQMetaObject@@B 10032084     moc_SamtoolsPlugin.obj
 0003:0000009c       ___security_cookie         1003209c     MSVCRT:gs_cookie.obj
 0003:000000a0       ___security_cookie_complement 100320a0     MSVCRT:gs_cookie.obj
 0003:000000b0       ___native_dllmain_reason   100320b0     MSVCRT:natstart.obj
 0003:000000b8       ??_R0?AVGObject@U2@@@8     100320b8     AssemblySamtoolsMpileup.obj
 0003:000000d4       ??_R0?AVVariantTrackObject@U2@@@8 100320d4     AssemblySamtoolsMpileup.obj
 0003:000000f8       ??_R0?AVerror_category@std@@@8 100320f8     AssemblySamtoolsMpileup.obj
 0003:0000011c       ??_R0?AV_Generic_error_category@std@@@8 1003211c     AssemblySamtoolsMpileup.obj
 0003:00000148       ??_R0?AV_Iostream_error_category@std@@@8 10032148     AssemblySamtoolsMpileup.obj
 0003:00000174       ??_R0?AV_System_error_category@std@@@8 10032174     AssemblySamtoolsMpileup.obj
 0003:000001a0       ??_R0?AVQObject@@@8        100321a0     AssemblySamtoolsMpileup.obj
 0003:000001b8       ??_R0?AVLoadDocumentTask@U2@@@8 100321b8     AssemblySamtoolsMpileup.obj
 0003:000001dc       ??_R0?AVDocumentProviderTask@U2@@@8 100321dc     AssemblySamtoolsMpileup.obj
 0003:00000204       ??_R0?AVTask@U2@@@8        10032204     AssemblySamtoolsMpileup.obj
 0003:0000021c       ??_R0?AVSamtoolsMpileupTask@LocalWorkflow@U2@@@8 1003221c     AssemblySamtoolsMpileup.obj
 0003:00000250       ??_R0?AVExternalToolSupportTask@U2@@@8 10032250     AssemblySamtoolsMpileup.obj
 0003:0000027c       ??_R0?AVCallVariantsTask@LocalWorkflow@U2@@@8 1003227c     AssemblySamtoolsMpileup.obj
 0003:000002ac       ??_R0?AVPort@Workflow@U2@@@8 100322ac     SamtoolMpileupWorker.obj
 0003:000002cc       ??_R0?AVIntegralBusPort@Workflow@U2@@@8 100322cc     SamtoolMpileupWorker.obj
 0003:000002f8       ??_R0?AVQDoubleValidator@@@8 100322f8     SamtoolMpileupWorker.obj
 0003:00000318       ??_R0?AVQValidator@@@8     10032318     SamtoolMpileupWorker.obj
 0003:00000334       ??_R0?AVQLineEdit@@@8      10032334     SamtoolMpileupWorker.obj
 0003:0000034c       ??_R0?AVQWidget@@@8        1003234c     SamtoolMpileupWorker.obj
 0003:00000364       ??_R0?AVQPaintDevice@@@8   10032364     SamtoolMpileupWorker.obj
 0003:00000380       ??_R0?AVVisibilityRelation@U2@@@8 10032380     SamtoolMpileupWorker.obj
 0003:000003a4       ??_R0?AVAttributeRelation@U2@@@8 100323a4     SamtoolMpileupWorker.obj
 0003:000003c8       ??_R0?AVDescriptor@U2@@@8  100323c8     SamtoolMpileupWorker.obj
 0003:000003e4       ??_R0?AVMapDataType@U2@@@8 100323e4     SamtoolMpileupWorker.obj
 0003:00000404       ??_R0?AVDataType@U2@@@8    10032404     SamtoolMpileupWorker.obj
 0003:00000420       ??_R0?AVQSharedData@@@8    10032420     SamtoolMpileupWorker.obj
 0003:0000043c       ??_R0?AVPortRelationDescriptor@U2@@@8 1003243c     SamtoolMpileupWorker.obj
 0003:00000464       ??_R0?AVAttribute@U2@@@8   10032464     SamtoolMpileupWorker.obj
 0003:00000480       ??_R0?AVConfigurationEditor@U2@@@8 10032480     SamtoolMpileupWorker.obj
 0003:000004a8       ??_R0?AVDelegateEditor@U2@@@8 100324a8     SamtoolMpileupWorker.obj
 0003:000004c8       ??_R0?AVURLDelegate@U2@@@8 100324c8     SamtoolMpileupWorker.obj
 0003:000004e8       ??_R0?AVPropertyDelegate@U2@@@8 100324e8     SamtoolMpileupWorker.obj
 0003:0000050c       ??_R0?AVQItemDelegate@@@8  1003250c     SamtoolMpileupWorker.obj
 0003:00000528       ??_R0?AVQAbstractItemDelegate@@@8 10032528     SamtoolMpileupWorker.obj
 0003:0000054c       ??_R0?AVSpinBoxDelegate@U2@@@8 1003254c     SamtoolMpileupWorker.obj
 0003:00000570       ??_R0?AVDoubleSpinBoxDelegate@U2@@@8 10032570     SamtoolMpileupWorker.obj
 0003:00000598       ??_R0?AVComboBoxDelegate@U2@@@8 10032598     SamtoolMpileupWorker.obj
 0003:000005bc       ??_R0?AVPortDescriptor@Workflow@U2@@@8 100325bc     SamtoolMpileupWorker.obj
 0003:000005e8       ??_R0?AVIntegralBusActorPrototype@Workflow@U2@@@8 100325e8     SamtoolMpileupWorker.obj
 0003:0000061c       ??_R0?AVActorPrototype@Workflow@U2@@@8 1003261c     SamtoolMpileupWorker.obj
 0003:00000648       ??_R0?AVVisualDescriptor@U2@@@8 10032648     SamtoolMpileupWorker.obj
 0003:0000066c       ??_R0?AVCallVariantsPrompter@LocalWorkflow@U2@@@8 1003266c     SamtoolMpileupWorker.obj
 0003:000006a0       ??_R0?AV?$PrompterBase@VCallVariantsPrompter@LocalWorkflow@U2@@@U2@@@8 100326a0     SamtoolMpileupWorker.obj
 0003:000006ec       ??_R0?AVPrompterBaseImpl@U2@@@8 100326ec     SamtoolMpileupWorker.obj
 0003:00000710       ??_R0?AVActorDocument@Workflow@U2@@@8 10032710     SamtoolMpileupWorker.obj
 0003:00000738       ??_R0?AVQTextDocument@@@8  10032738     SamtoolMpileupWorker.obj
 0003:00000754       ??_R0?AVPrompter@Workflow@U2@@@8 10032754     SamtoolMpileupWorker.obj
 0003:00000778       ??_R0?AVCallVariantsWorker@LocalWorkflow@U2@@@8 10032778     SamtoolMpileupWorker.obj
 0003:000007ac       ??_R0?AVBaseWorker@LocalWorkflow@U2@@@8 100327ac     SamtoolMpileupWorker.obj
 0003:000007d8       ??_R0?AVWorker@Workflow@U2@@@8 100327d8     SamtoolMpileupWorker.obj
 0003:000007fc       ??_R0?AVCommunicationSubject@Workflow@U2@@@8 100327fc     SamtoolMpileupWorker.obj
 0003:0000082c       ??_R0?AVCallVariantsWorkerFactory@LocalWorkflow@U2@@@8 1003282c     SamtoolMpileupWorker.obj
 0003:00000868       ??_R0?AVDomainFactory@Workflow@U2@@@8 10032868     SamtoolMpileupWorker.obj
 0003:00000890       ??_R0?AV?$IdRegistry@VDomainFactory@Workflow@U2@@@U2@@@8 10032890     SamtoolMpileupWorker.obj
 0003:000008cc       ??_R0?AVScientificDoubleWidget@LocalWorkflow@U2@@@8 100328cc     SamtoolMpileupWorker.obj
 0003:00000904       ??_R0?AVPropertyWidget@U2@@@8 10032904     SamtoolMpileupWorker.obj
 0003:00000924       ??_R0?AVScientificDoubleDelegate@LocalWorkflow@U2@@@8 10032924     SamtoolMpileupWorker.obj
 0003:0000095c       ??_R0?AVEmptySlotValidator@LocalWorkflow@U2@@@8 1003295c     SamtoolMpileupWorker.obj
 0003:00000990       ??_R0?AVConfigurationValidator@U2@@@8 10032990     SamtoolMpileupWorker.obj
 0003:000009b8       ??_R0?AVSamtoolsPlugin@U2@@@8 100329b8     SamtoolsPlugin.obj
 0003:000009d8       ??_R0?AVPlugin@U2@@@8      100329d8     SamtoolsPlugin.obj
 0003:000009f0       ??_R0?AVtype_info@@@8      100329f0     MSVCRT:ti_inst.obj
 0003:00000a0c       ?VCFUTILS_ID@SamtoolsMpileupTask@LocalWorkflow@U2@@0VQString@@B 10032a0c     AssemblySamtoolsMpileup.obj
 0003:00000a38       ?BCFTOOLS_ID@SamtoolsMpileupTask@LocalWorkflow@U2@@0VQString@@B 10032a38     AssemblySamtoolsMpileup.obj
 0003:00000a5c       ?SAMTOOLS_ID@SamtoolsMpileupTask@LocalWorkflow@U2@@0VQString@@B 10032a5c     AssemblySamtoolsMpileup.obj
 0003:00000a60       ?id@?$num_put@DV?$back_insert_iterator@V?$basic_string@DU?$char_traits@D@std@@V?$allocator@D@2@@std@@@std@@@std@@2V0locale@2@A 10032a60     AssemblySamtoolsMpileup.obj
 0003:00000a64       ?id@?$num_put@_WV?$back_insert_iterator@V?$basic_string@_WU?$char_traits@_W@std@@V?$allocator@_W@2@@std@@@std@@@std@@2V0locale@2@A 10032a64     AssemblySamtoolsMpileup.obj
 0003:00000a68       ?metatype_id@?1??qt_metatype_id@?$QMetaTypeId@VU2DbiRef@U2@@@@SAHXZ@4V?$QBasicAtomicInteger@H@@A 10032a68     AssemblySamtoolsMpileup.obj
 0003:00000a6c       ?metatype_id@?1??qt_metatype_id@?$QMetaTypeId@V?$QSharedDataPointer@VDbiDataHandler@Workflow@U2@@@@@@SAHXZ@4V?$QBasicAtomicInteger@H@@A 10032a6c     AssemblySamtoolsMpileup.obj
 0003:00000acc       ?ACTOR_ID@CallVariantsWorkerFactory@LocalWorkflow@U2@@2VQString@@B 10032acc     SamtoolMpileupWorker.obj
 0003:00000fc8       ?__type_info_root_node@@3U__type_info_node@@A 10032fc8     MSVCRT:tncleanup.obj
 0003:00000fd0       ___native_startup_lock     10032fd0     <common>
 0003:00000fd4       ___native_startup_state    10032fd4     <common>
 0003:00000fd8       ___dyn_tls_init_callback   10032fd8     <common>
 0003:00000fdc       ___onexitend               10032fdc     <common>
 0003:00000fe0       ___onexitbegin             10032fe0     <common>

 entry point at        0001:0001930a

 Static symbols

 0000:fffc7000       .debug$S                   10000000     MSVCRT:MSVCR120.dll
 0000:fffc7000       .debug$S                   10000000     MSVCRT:MSVCR120.dll
 0000:fffc7000       .debug$S                   10000000     MSVCRT:MSVCR120.dll
 0000:fffc7000       .debug$S                   10000000     MSVCRT:MSVCR120.dll
 0000:fffc7000       .debug$S                   10000000     MSVCRT:MSVCR120.dll
 0000:fffc7000       .debug$S                   10000000     MSVCRT:MSVCR120.dll
 0000:fffc7000       .debug$S                   10000000     MSVCRT:MSVCR120.dll
 0000:fffc7000       .debug$S                   10000000     U2Lang:U2Lang.dll
 0000:fffc7000       .debug$S                   10000000     U2Lang:U2Lang.dll
 0000:fffc7000       .debug$S                   10000000     U2Lang:U2Lang.dll
 0000:fffc7000       .debug$S                   10000000     U2Lang:U2Lang.dll
 0000:fffc7000       .debug$S                   10000000     U2Lang:U2Lang.dll
 0000:fffc7000       .debug$S                   10000000     U2Lang:U2Lang.dll
 0000:fffc7000       .debug$S                   10000000     U2Lang:U2Lang.dll
 0000:fffc7000       .debug$S                   10000000     U2Lang:U2Lang.dll
 0000:fffc7000       .debug$S                   10000000     U2Lang:U2Lang.dll
 0001:fffff000       __ehhandler$?_Copy@?$basic_string@DU?$char_traits@D@std@@V?$allocator@D@2@@std@@QAEXII@Z 10000000 f   moc_SamtoolsPlugin.obj
 0000:fffc7000       .debug$S                   10000000     U2Lang:U2Lang.dll
 0000:fffc7000       .debug$S                   10000000     U2Lang:U2Lang.dll
 0000:fffc7000       .debug$S                   10000000     U2Lang:U2Lang.dll
 0000:fffc7000       .debug$S                   10000000     U2Lang:U2Lang.dll
 0000:fffc7000       .debug$S                   10000000     U2Lang:U2Lang.dll
 0000:fffc7000       .debug$S                   10000000     U2Lang:U2Lang.dll
 0002:fffe0000       __catchsym$?_Copy@?$basic_string@DU?$char_traits@D@std@@V?$allocator@D@2@@std@@QAEXII@Z$5 10000000     moc_SamtoolsPlugin.obj
 0000:fffc7000       .debug$S                   10000000     MSVCRT:MSVCR120.dll
 0000:fffc7000       .debug$S                   10000000     MSVCRT:MSVCR120.dll
 0000:fffc7000       .debug$S                   10000000     MSVCRT:MSVCR120.dll
 0000:fffc7000       .debug$S                   10000000     MSVCRT:MSVCR120.dll
 0000:fffc7000       .debug$S                   10000000     U2Lang:U2Lang.dll
 0002:fffe0000       ?_Generic_object$initializer$@?$_Error_objects@H@std@@2P6AXXZA 10000000     moc_SamtoolsPlugin.obj
 0002:fffe0000       ?_Iostream_object$initializer$@?$_Error_objects@H@std@@2P6AXXZA 10000000     moc_SamtoolsPlugin.obj
 0002:fffe0000       ?_System_object$initializer$@?$_Error_objects@H@std@@2P6AXXZA 10000000     moc_SamtoolsPlugin.obj
 0000:fffc7000       .debug$S                   10000000     U2Lang:U2Lang.dll
 0000:fffc7000       .debug$S                   10000000     U2Lang:U2Lang.dll
 0000:fffc7000       .debug$S                   10000000     U2Lang:U2Lang.dll
 0000:fffc7000       .debug$S                   10000000     U2Lang:U2Lang.dll
 0000:fffc7000       .debug$S                   10000000     U2Lang:U2Lang.dll
 0000:fffc7000       .debug$S                   10000000     U2Lang:U2Lang.dll
 0000:fffc7000       .debug$S                   10000000     U2Lang:U2Lang.dll
 0000:fffc7000       .debug$S                   10000000     U2Lang:U2Lang.dll
 0000:fffc7000       .debug$S                   10000000     U2Lang:U2Lang.dll
 0000:fffc7000       .debug$S                   10000000     U2Lang:U2Lang.dll
 0000:fffc7000       .debug$S                   10000000     U2Lang:U2Lang.dll
 0000:fffc7000       .debug$S                   10000000     U2Lang:U2Lang.dll
 0000:fffc7000       .debug$S                   10000000     U2Lang:U2Lang.dll
 0000:fffc7000       .debug$S                   10000000     U2Lang:U2Lang.dll
 0000:fffc7000       .debug$S                   10000000     U2Lang:U2Lang.dll
 0000:fffc7000       .debug$S                   10000000     U2Lang:U2Lang.dll
 0000:fffc7000       .debug$S                   10000000     U2Lang:U2Lang.dll
 0000:fffc7000       .debug$S                   10000000     U2Lang:U2Lang.dll
 0000:fffc7000       .debug$S                   10000000     U2Lang:U2Lang.dll
 0000:fffc7000       .debug$S                   10000000     U2Lang:U2Lang.dll
 0000:fffc7000       .debug$S                   10000000     U2Lang:U2Lang.dll
 0000:fffc7000       .debug$S                   10000000     U2Lang:U2Lang.dll
 0000:fffc7000       .debug$S                   10000000     U2Lang:U2Lang.dll
 0000:fffc7000       .debug$S                   10000000     U2Lang:U2Lang.dll
 0000:fffc7000       .debug$S                   10000000     U2Lang:U2Lang.dll
 0000:fffc7000       .debug$S                   10000000     U2Lang:U2Lang.dll
 0000:fffc7000       .debug$S                   10000000     U2Lang:U2Lang.dll
 0000:fffc7000       .debug$S                   10000000     U2Lang:U2Lang.dll
 0000:fffc7000       .debug$S                   10000000     U2Lang:U2Lang.dll
 0000:fffc7000       .debug$S                   10000000     U2Lang:U2Lang.dll
 0000:fffc7000       .debug$S                   10000000     U2Lang:U2Lang.dll
 0000:fffc7000       .debug$S                   10000000     U2Lang:U2Lang.dll
 0000:fffc7000       .debug$S                   10000000     U2Lang:U2Lang.dll
 0001:fffff000       __ehhandler$?_Copy@?$basic_string@DU?$char_traits@D@std@@V?$allocator@D@2@@std@@QAEXII@Z 10000000 f   moc_SamtoolMpileupWorker.obj
 0000:fffc7000       .debug$S                   10000000     U2Lang:U2Lang.dll
 0000:fffc7000       .debug$S                   10000000     U2Lang:U2Lang.dll
 0000:fffc7000       .debug$S                   10000000     U2Lang:U2Lang.dll
 0000:fffc7000       .debug$S                   10000000     U2Lang:U2Lang.dll
 0000:fffc7000       .debug$S                   10000000     U2Lang:U2Lang.dll
 0000:fffc7000       .debug$S                   10000000     U2Lang:U2Lang.dll
 0000:fffc7000       .debug$S                   10000000     U2Lang:U2Lang.dll
 0000:fffc7000       .debug$S                   10000000     U2Lang:U2Lang.dll
 0000:fffc7000       .debug$S                   10000000     U2Lang:U2Lang.dll
 0000:fffc7000       .debug$S                   10000000     U2Lang:U2Lang.dll
 0000:fffc7000       .debug$S                   10000000     U2Lang:U2Lang.dll
 0000:fffc7000       .debug$S                   10000000     U2Lang:U2Lang.dll
 0000:fffc7000       .debug$S                   10000000     U2Lang:U2Lang.dll
 0000:fffc7000       .debug$S                   10000000     U2Lang:U2Lang.dll
 0000:fffc7000       .debug$S                   10000000     U2Lang:U2Lang.dll
 0000:fffc7000       .debug$S                   10000000     U2Lang:U2Lang.dll
 0000:fffc7000       .debug$S                   10000000     U2Lang:U2Lang.dll
 0000:fffc7000       .debug$S                   10000000     U2Lang:U2Lang.dll
 0000:fffc7000       .debug$S                   10000000     U2Lang:U2Lang.dll
 0000:fffc7000       .debug$S                   10000000     U2Core:U2Core.dll
 0000:fffc7000       .debug$S                   10000000     U2Core:U2Core.dll
 0000:fffc7000       .debug$S                   10000000     U2Core:U2Core.dll
 0000:fffc7000       .debug$S                   10000000     U2Core:U2Core.dll
 0000:fffc7000       .debug$S                   10000000     U2Core:U2Core.dll
 0002:fffe0000       __catchsym$?_Copy@?$basic_string@DU?$char_traits@D@std@@V?$allocator@D@2@@std@@QAEXII@Z$5 10000000     moc_SamtoolMpileupWorker.obj
 0000:fffc7000       .debug$S                   10000000     MSVCRT:MSVCR120.dll
 0000:fffc7000       .debug$S                   10000000     MSVCRT:MSVCR120.dll
 0000:fffc7000       .debug$S                   10000000     MSVCRT:MSVCR120.dll
 0000:fffc7000       .debug$S                   10000000     MSVCRT:MSVCR120.dll
 0000:fffc7000       .debug$S                   10000000     MSVCRT:MSVCR120.dll
 0000:fffc7000       .debug$S                   10000000     MSVCRT:MSVCR120.dll
 0000:fffc7000       .debug$S                   10000000     MSVCRT:MSVCR120.dll
 0000:fffc7000       .debug$S                   10000000     MSVCRT:MSVCR120.dll
 0000:fffc7000       .debug$S                   10000000     MSVCRT:MSVCR120.dll
 0000:fffc7000       .debug$S                   10000000     MSVCRT:MSVCR120.dll
 0000:fffc7000       .debug$S                   10000000     MSVCRT:MSVCR120.dll
 0000:fffc7000       .debug$S                   10000000     MSVCRT:MSVCR120.dll
 0000:fffc7000       .debug$S                   10000000     MSVCRT:MSVCR120.dll
 0000:fffc7000       .debug$S                   10000000     MSVCRT:MSVCR120.dll
 0000:fffc7000       .debug$S                   10000000     MSVCRT:MSVCR120.dll
 0000:fffc7000       .debug$S                   10000000     MSVCRT:MSVCR120.dll
 0000:fffc7000       .debug$S                   10000000     U2Core:U2Core.dll
 0000:fffc7000       .debug$S                   10000000     U2Core:U2Core.dll
 0000:fffc7000       .debug$S                   10000000     U2Core:U2Core.dll
 0000:fffc7000       .debug$S                   10000000     U2Core:U2Core.dll
 0000:fffc7000       .debug$S                   10000000     U2Core:U2Core.dll
 0000:fffc7000       .debug$S                   10000000     U2Core:U2Core.dll
 0000:fffc7000       .debug$S                   10000000     U2Core:U2Core.dll
 0000:fffc7000       .debug$S                   10000000     msvcprt:MSVCP120.dll
 0000:fffc7000       .debug$S                   10000000     msvcprt:MSVCP120.dll
 0000:fffc7000       .debug$S                   10000000     msvcprt:MSVCP120.dll
 0000:fffc7000       .debug$S                   10000000     msvcprt:MSVCP120.dll
 0000:fffc7000       .debug$S                   10000000     msvcprt:MSVCP120.dll
 0000:fffc7000       .debug$S                   10000000     kernel32:KERNEL32.dll
 0000:fffc7000       .debug$S                   10000000     kernel32:KERNEL32.dll
 0000:fffc7000       .debug$S                   10000000     kernel32:KERNEL32.dll
 0000:fffc7000       .debug$S                   10000000     U2Core:U2Core.dll
 0000:fffc7000       .debug$S                   10000000     U2Core:U2Core.dll
 0000:fffc7000       .debug$S                   10000000     U2Core:U2Core.dll
 0000:fffc7000       .debug$S                   10000000     U2Core:U2Core.dll
 0000:fffc7000       .debug$S                   10000000     U2Core:U2Core.dll
 0000:fffc7000       .debug$S                   10000000     U2Core:U2Core.dll
 0000:fffc7000       .debug$S                   10000000     U2Core:U2Core.dll
 0000:fffc7000       .debug$S                   10000000     U2Core:U2Core.dll
 0000:fffc7000       .debug$S                   10000000     U2Core:U2Core.dll
 0000:fffc7000       .debug$S                   10000000     U2Core:U2Core.dll
 0000:fffc7000       .debug$S                   10000000     U2Core:U2Core.dll
 0000:fffc7000       .debug$S                   10000000     U2Core:U2Core.dll
 0002:fffe0000       ?_Generic_object$initializer$@?$_Error_objects@H@std@@2P6AXXZA 10000000     moc_SamtoolMpileupWorker.obj
 0002:fffe0000       ?_Iostream_object$initializer$@?$_Error_objects@H@std@@2P6AXXZA 10000000     moc_SamtoolMpileupWorker.obj
 0002:fffe0000       ?_System_object$initializer$@?$_Error_objects@H@std@@2P6AXXZA 10000000     moc_SamtoolMpileupWorker.obj
 0000:fffc7000       .debug$S                   10000000     U2Core:U2Core.dll
 0000:fffc7000       .debug$S                   10000000     U2Core:U2Core.dll
 0000:fffc7000       .debug$S                   10000000     U2Core:U2Core.dll
 0000:fffc7000       .debug$S                   10000000     U2Core:U2Core.dll
 0000:fffc7000       .debug$S                   10000000     U2Core:U2Core.dll
 0000:fffc7000       .debug$S                   10000000     U2Core:U2Core.dll
 0000:fffc7000       .debug$S                   10000000     U2Core:U2Core.dll
 0000:fffc7000       .debug$S                   10000000     U2Core:U2Core.dll
 0000:fffc7000       .debug$S                   10000000     U2Core:U2Core.dll
 0000:fffc7000       .debug$S                   10000000     U2Core:U2Core.dll
 0000:fffc7000       .debug$S                   10000000     U2Core:U2Core.dll
 0000:fffc7000       .debug$S                   10000000     U2Core:U2Core.dll
 0000:fffc7000       .debug$S                   10000000     U2Core:U2Core.dll
 0000:fffc7000       .debug$S                   10000000     U2Core:U2Core.dll
 0000:fffc7000       .debug$S                   10000000     U2Core:U2Core.dll
 0000:fffc7000       .debug$S                   10000000     U2Core:U2Core.dll
 0000:fffc7000       .debug$S                   10000000     U2Core:U2Core.dll
 0000:fffc7000       .debug$S                   10000000     U2Core:U2Core.dll
 0000:fffc7000       .debug$S                   10000000     U2Core:U2Core.dll
 0000:fffc7000       .debug$S                   10000000     U2Core:U2Core.dll
 0000:fffc7000       .debug$S                   10000000     U2Core:U2Core.dll
 0000:fffc7000       .debug$S                   10000000     U2Core:U2Core.dll
 0000:fffc7000       .debug$S                   10000000     U2Core:U2Core.dll
 0000:fffc7000       .debug$S                   10000000     U2Core:U2Core.dll
 0000:fffc7000       .debug$S                   10000000     U2Core:U2Core.dll
 0000:fffc7000       .debug$S                   10000000     U2Core:U2Core.dll
 0000:fffc7000       .debug$S                   10000000     U2Core:U2Core.dll
 0000:fffc7000       .debug$S                   10000000     U2Core:U2Core.dll
 0000:fffc7000       .debug$S                   10000000     U2Core:U2Core.dll
 0000:fffc7000       .debug$S                   10000000     U2Core:U2Core.dll
 0001:fffff000       __ehhandler$?_Copy@?$basic_string@DU?$char_traits@D@std@@V?$allocator@D@2@@std@@QAEXII@Z 10000000 f   moc_AssemblySamtoolsMpileup.obj
 0000:fffc7000       .debug$S                   10000000     U2Core:U2Core.dll
 0000:fffc7000       .debug$S                   10000000     U2Core:U2Core.dll
 0000:fffc7000       .debug$S                   10000000     U2Core:U2Core.dll
 0000:fffc7000       .debug$S                   10000000     U2Core:U2Core.dll
 0000:fffc7000       .debug$S                   10000000     U2Core:U2Core.dll
 0000:fffc7000       .debug$S                   10000000     U2Core:U2Core.dll
 0000:fffc7000       .debug$S                   10000000     U2Core:U2Core.dll
 0000:fffc7000       .debug$S                   10000000     U2Core:U2Core.dll
 0000:fffc7000       .debug$S                   10000000     U2Core:U2Core.dll
 0000:fffc7000       .debug$S                   10000000     U2Core:U2Core.dll
 0000:fffc7000       .debug$S                   10000000     U2Core:U2Core.dll
 0000:fffc7000       .debug$S                   10000000     U2Core:U2Core.dll
 0000:fffc7000       .debug$S                   10000000     U2Core:U2Core.dll
 0000:fffc7000       .debug$S                   10000000     U2Core:U2Core.dll
 0000:fffc7000       .debug$S                   10000000     U2Core:U2Core.dll
 0000:fffc7000       .debug$S                   10000000     U2Core:U2Core.dll
 0000:fffc7000       .debug$S                   10000000     U2Core:U2Core.dll
 0000:fffc7000       .debug$S                   10000000     U2Core:U2Core.dll
 0000:fffc7000       .debug$S                   10000000     U2Core:U2Core.dll
 0000:fffc7000       .debug$S                   10000000     U2Core:U2Core.dll
 0000:fffc7000       .debug$S                   10000000     U2Core:U2Core.dll
 0000:fffc7000       .debug$S                   10000000     U2Core:U2Core.dll
 0000:fffc7000       .debug$S                   10000000     U2Core:U2Core.dll
 0000:fffc7000       .debug$S                   10000000     U2Core:U2Core.dll
 0002:fffe0000       __catchsym$?_Copy@?$basic_string@DU?$char_traits@D@std@@V?$allocator@D@2@@std@@QAEXII@Z$5 10000000     moc_AssemblySamtoolsMpileup.obj
 0000:fffc7000       .debug$S                   10000000     kernel32:KERNEL32.dll
 0000:fffc7000       .debug$S                   10000000     kernel32:KERNEL32.dll
 0000:fffc7000       .debug$S                   10000000     kernel32:KERNEL32.dll
 0000:fffc7000       .debug$S                   10000000     kernel32:KERNEL32.dll
 0000:fffc7000       .debug$S                   10000000     kernel32:KERNEL32.dll
 0000:fffc7000       .debug$S                   10000000     kernel32:KERNEL32.dll
 0000:fffc7000       .debug$S                   10000000     Qt5Core:Qt5Core.dll
 0000:fffc7000       .debug$S                   10000000     Qt5Core:Qt5Core.dll
 0000:fffc7000       .debug$S                   10000000     Qt5Core:Qt5Core.dll
 0000:fffc7000       .debug$S                   10000000     Qt5Core:Qt5Core.dll
 0000:fffc7000       .debug$S                   10000000     Qt5Core:Qt5Core.dll
 0000:fffc7000       .debug$S                   10000000     Qt5Core:Qt5Core.dll
 0000:fffc7000       .debug$S                   10000000     Qt5Core:Qt5Core.dll
 0000:fffc7000       .debug$S                   10000000     Qt5Core:Qt5Core.dll
 0000:fffc7000       .debug$S                   10000000     Qt5Core:Qt5Core.dll
 0000:fffc7000       .debug$S                   10000000     Qt5Core:Qt5Core.dll
 0000:fffc7000       .debug$S                   10000000     Qt5Core:Qt5Core.dll
 0000:fffc7000       .debug$S                   10000000     Qt5Core:Qt5Core.dll
 0000:fffc7000       .debug$S                   10000000     Qt5Core:Qt5Core.dll
 0000:fffc7000       .debug$S                   10000000     Qt5Core:Qt5Core.dll
 0000:fffc7000       .debug$S                   10000000     Qt5Core:Qt5Core.dll
 0000:fffc7000       .debug$S                   10000000     Qt5Core:Qt5Core.dll
 0000:fffc7000       .debug$S                   10000000     Qt5Core:Qt5Core.dll
 0000:fffc7000       .debug$S                   10000000     Qt5Core:Qt5Core.dll
 0000:fffc7000       .debug$S                   10000000     Qt5Core:Qt5Core.dll
 0000:fffc7000       .debug$S                   10000000     Qt5Core:Qt5Core.dll
 0000:fffc7000       .debug$S                   10000000     Qt5Core:Qt5Core.dll
 0000:fffc7000       .debug$S                   10000000     Qt5Core:Qt5Core.dll
 0000:fffc7000       .debug$S                   10000000     Qt5Core:Qt5Core.dll
 0000:fffc7000       .debug$S                   10000000     Qt5Core:Qt5Core.dll
 0000:fffc7000       .debug$S                   10000000     Qt5Core:Qt5Core.dll
 0000:fffc7000       .debug$S                   10000000     U2Core:U2Core.dll
 0000:fffc7000       .debug$S                   10000000     U2Core:U2Core.dll
 0000:fffc7000       .debug$S                   10000000     U2Core:U2Core.dll
 0000:fffc7000       .debug$S                   10000000     U2Core:U2Core.dll
 0000:fffc7000       .debug$S                   10000000     U2Core:U2Core.dll
 0000:fffc7000       .debug$S                   10000000     U2Core:U2Core.dll
 0000:fffc7000       .debug$S                   10000000     U2Core:U2Core.dll
 0000:fffc7000       .debug$S                   10000000     U2Core:U2Core.dll
 0000:fffc7000       .debug$S                   10000000     U2Core:U2Core.dll
 0000:fffc7000       .debug$S                   10000000     U2Core:U2Core.dll
 0000:fffc7000       .debug$S                   10000000     U2Core:U2Core.dll
 0002:fffe0000       ?_Generic_object$initializer$@?$_Error_objects@H@std@@2P6AXXZA 10000000     moc_AssemblySamtoolsMpileup.obj
 0002:fffe0000       ?_Iostream_object$initializer$@?$_Error_objects@H@std@@2P6AXXZA 10000000     moc_AssemblySamtoolsMpileup.obj
 0002:fffe0000       ?_System_object$initializer$@?$_Error_objects@H@std@@2P6AXXZA 10000000     moc_AssemblySamtoolsMpileup.obj
 0000:fffc7000       .debug$S                   10000000     U2Core:U2Core.dll
 0000:fffc7000       .debug$S                   10000000     U2Core:U2Core.dll
 0000:fffc7000       .debug$S                   10000000     U2Core:U2Core.dll
 0000:fffc7000       .debug$S                   10000000     U2Core:U2Core.dll
 0000:fffc7000       .debug$S                   10000000     U2Core:U2Core.dll
 0000:fffc7000       .debug$S                   10000000     U2Core:U2Core.dll
 0000:fffc7000       .debug$S                   10000000     U2Core:U2Core.dll
 0000:fffc7000       .debug$S                   10000000     U2Core:U2Core.dll
 0000:fffc7000       .debug$S                   10000000     U2Core:U2Core.dll
 0000:fffc7000       .debug$S                   10000000     U2Core:U2Core.dll
 0000:fffc7000       .debug$S                   10000000     U2Lang:U2Lang.dll
 0000:fffc7000       .debug$S                   10000000     U2Lang:U2Lang.dll
 0000:fffc7000       .debug$S                   10000000     U2Lang:U2Lang.dll
 0000:fffc7000       .debug$S                   10000000     U2Lang:U2Lang.dll
 0000:fffc7000       .debug$S                   10000000     U2Lang:U2Lang.dll
 0000:fffc7000       .debug$S                   10000000     U2Lang:U2Lang.dll
 0000:fffc7000       .debug$S                   10000000     U2Lang:U2Lang.dll
 0000:fffc7000       .debug$S                   10000000     U2Lang:U2Lang.dll
 0000:fffc7000       .debug$S                   10000000     U2Lang:U2Lang.dll
 0000:fffc7000       .debug$S                   10000000     U2Lang:U2Lang.dll
 0000:fffc7000       .debug$S                   10000000     U2Lang:U2Lang.dll
 0000:fffc7000       .debug$S                   10000000     U2Lang:U2Lang.dll
 0000:fffc7000       .debug$S                   10000000     U2Lang:U2Lang.dll
 0000:fffc7000       .debug$S                   10000000     U2Lang:U2Lang.dll
 0001:fffff000       __ehhandler$?_Copy@?$basic_string@DU?$char_traits@D@std@@V?$allocator@D@2@@std@@QAEXII@Z 10000000 f   SamtoolsPlugin.obj
 0000:fffc7000       .debug$S                   10000000     U2Lang:U2Lang.dll
 0002:fffe0000       ?_System_object$initializer$@?$_Error_objects@H@std@@2P6AXXZA 10000000     SamtoolMpileupWorker.obj
 0002:fffe0000       ?_Iostream_object$initializer$@?$_Error_objects@H@std@@2P6AXXZA 10000000     SamtoolMpileupWorker.obj
 0002:fffe0000       ?_Generic_object$initializer$@?$_Error_objects@H@std@@2P6AXXZA 10000000     SamtoolMpileupWorker.obj
 0000:fffc7000       .debug$S                   10000000     U2Lang:U2Lang.dll
 0000:fffc7000       .debug$S                   10000000     U2Lang:U2Lang.dll
 0000:fffc7000       .debug$S                   10000000     U2Lang:U2Lang.dll
 0000:fffc7000       .debug$S                   10000000     U2Lang:U2Lang.dll
 0000:fffc7000       .debug$S                   10000000     U2Lang:U2Lang.dll
 0000:fffc7000       .debug$S                   10000000     U2Lang:U2Lang.dll
 0000:fffc7000       .debug$S                   10000000     U2Lang:U2Lang.dll
 0000:fffc7000       .debug$S                   10000000     U2Lang:U2Lang.dll
 0000:fffc7000       .debug$S                   10000000     U2Lang:U2Lang.dll
 0000:fffc7000       .debug$S                   10000000     U2Lang:U2Lang.dll
 0000:fffc7000       .debug$S                   10000000     U2Lang:U2Lang.dll
 0000:fffc7000       .debug$S                   10000000     U2Lang:U2Lang.dll
 0000:fffc7000       .debug$S                   10000000     U2Lang:U2Lang.dll
 0000:fffc7000       .debug$S                   10000000     U2Lang:U2Lang.dll
 0000:fffc7000       .debug$S                   10000000     U2Lang:U2Lang.dll
 0000:fffc7000       .debug$S                   10000000     U2Lang:U2Lang.dll
 0000:fffc7000       .debug$S                   10000000     U2Lang:U2Lang.dll
 0000:fffc7000       .debug$S                   10000000     U2Lang:U2Lang.dll
 0000:fffc7000       .debug$S                   10000000     U2Lang:U2Lang.dll
 0000:fffc7000       .debug$S                   10000000     U2Lang:U2Lang.dll
 0000:fffc7000       .debug$S                   10000000     U2Lang:U2Lang.dll
 0000:fffc7000       .debug$S                   10000000     U2Lang:U2Lang.dll
 0000:fffc7000       .debug$S                   10000000     U2Lang:U2Lang.dll
 0000:fffc7000       .debug$S                   10000000     U2Lang:U2Lang.dll
 0002:fffe0000       __catchsym$?_Copy@?$basic_string@DU?$char_traits@D@std@@V?$allocator@D@2@@std@@QAEXII@Z$5 10000000     SamtoolsPlugin.obj
 0000:fffc7000       .debug$S                   10000000     Qt5Core:Qt5Core.dll
 0000:fffc7000       .debug$S                   10000000     Qt5Core:Qt5Core.dll
 0000:fffc7000       .debug$S                   10000000     Qt5Core:Qt5Core.dll
 0000:fffc7000       .debug$S                   10000000     Qt5Core:Qt5Core.dll
 0000:fffc7000       .debug$S                   10000000     Qt5Core:Qt5Core.dll
 0000:fffc7000       .debug$S                   10000000     Qt5Core:Qt5Core.dll
 0000:fffc7000       .debug$S                   10000000     Qt5Core:Qt5Core.dll
 0000:fffc7000       .debug$S                   10000000     Qt5Core:Qt5Core.dll
 0000:fffc7000       .debug$S                   10000000     Qt5Core:Qt5Core.dll
 0000:fffc7000       .debug$S                   10000000     Qt5Core:Qt5Core.dll
 0000:fffc7000       .debug$S                   10000000     Qt5Core:Qt5Core.dll
 0000:fffc7000       .debug$S                   10000000     Qt5Core:Qt5Core.dll
 0000:fffc7000       .debug$S                   10000000     Qt5Core:Qt5Core.dll
 0000:fffc7000       .debug$S                   10000000     Qt5Core:Qt5Core.dll
 0000:fffc7000       .debug$S                   10000000     Qt5Core:Qt5Core.dll
 0000:fffc7000       .debug$S                   10000000     Qt5Core:Qt5Core.dll
 0000:fffc7000       .debug$S                   10000000     Qt5Core:Qt5Core.dll
 0000:fffc7000       .debug$S                   10000000     Qt5Core:Qt5Core.dll
 0000:fffc7000       .debug$S                   10000000     Qt5Core:Qt5Core.dll
 0000:fffc7000       .debug$S                   10000000     Qt5Core:Qt5Core.dll
 0000:fffc7000       .debug$S                   10000000     Qt5Core:Qt5Core.dll
 0000:fffc7000       .debug$S                   10000000     Qt5Core:Qt5Core.dll
 0000:fffc7000       .debug$S                   10000000     Qt5Core:Qt5Core.dll
 0000:fffc7000       .debug$S                   10000000     Qt5Core:Qt5Core.dll
 0000:fffc7000       .debug$S                   10000000     Qt5Core:Qt5Core.dll
 0000:fffc7000       .debug$S                   10000000     Qt5Core:Qt5Core.dll
 0000:fffc7000       .debug$S                   10000000     Qt5Core:Qt5Core.dll
 0000:fffc7000       .debug$S                   10000000     Qt5Core:Qt5Core.dll
 0000:fffc7000       .debug$S                   10000000     Qt5Core:Qt5Core.dll
 0000:fffc7000       .debug$S                   10000000     Qt5Core:Qt5Core.dll
 0000:fffc7000       .debug$S                   10000000     Qt5Core:Qt5Core.dll
 0000:fffc7000       .debug$S                   10000000     Qt5Core:Qt5Core.dll
 0000:fffc7000       .debug$S                   10000000     Qt5Core:Qt5Core.dll
 0000:fffc7000       .debug$S                   10000000     U2Lang:U2Lang.dll
 0000:fffc7000       .debug$S                   10000000     U2Lang:U2Lang.dll
 0000:fffc7000       .debug$S                   10000000     U2Lang:U2Lang.dll
 0000:fffc7000       .debug$S                   10000000     U2Lang:U2Lang.dll
 0000:fffc7000       .debug$S                   10000000     U2Lang:U2Lang.dll
 0000:fffc7000       .debug$S                   10000000     U2Lang:U2Lang.dll
 0000:fffc7000       .debug$S                   10000000     U2Lang:U2Lang.dll
 0000:fffc7000       .debug$S                   10000000     U2Lang:U2Lang.dll
 0000:fffc7000       .debug$S                   10000000     U2Lang:U2Lang.dll
 0002:fffe0000       ?_Generic_object$initializer$@?$_Error_objects@H@std@@2P6AXXZA 10000000     SamtoolsPlugin.obj
 0002:fffe0000       ?_Iostream_object$initializer$@?$_Error_objects@H@std@@2P6AXXZA 10000000     SamtoolsPlugin.obj
 0002:fffe0000       ?_System_object$initializer$@?$_Error_objects@H@std@@2P6AXXZA 10000000     SamtoolsPlugin.obj
 0000:fffc7000       .debug$S                   10000000     U2Lang:U2Lang.dll
 0000:fffc7000       .debug$S                   10000000     U2Lang:U2Lang.dll
 0000:fffc7000       .debug$S                   10000000     U2Lang:U2Lang.dll
 0000:fffc7000       .debug$S                   10000000     U2Lang:U2Lang.dll
 0000:fffc7000       .debug$S                   10000000     U2Lang:U2Lang.dll
 0000:fffc7000       .debug$S                   10000000     U2Lang:U2Lang.dll
 0000:fffc7000       .debug$S                   10000000     U2Lang:U2Lang.dll
 0000:fffc7000       .debug$S                   10000000     U2Lang:U2Lang.dll
 0000:fffc7000       .debug$S                   10000000     U2Lang:U2Lang.dll
 0000:fffc7000       .debug$S                   10000000     U2Lang:U2Lang.dll
 0000:fffc7000       .debug$S                   10000000     U2Lang:U2Lang.dll
 0000:fffc7000       .debug$S                   10000000     U2Lang:U2Lang.dll
 0000:fffc7000       .debug$S                   10000000     U2Lang:U2Lang.dll
 0000:fffc7000       .debug$S                   10000000     U2Lang:U2Lang.dll
 0000:fffc7000       .debug$S                   10000000     U2Lang:U2Lang.dll
 0000:fffc7000       .debug$S                   10000000     U2Lang:U2Lang.dll
 0000:fffc7000       .debug$S                   10000000     U2Lang:U2Lang.dll
 0000:fffc7000       .debug$S                   10000000     U2Lang:U2Lang.dll
 0000:fffc7000       .debug$S                   10000000     U2Lang:U2Lang.dll
 0000:fffc7000       .debug$S                   10000000     U2Lang:U2Lang.dll
 0000:fffc7000       .debug$S                   10000000     U2Lang:U2Lang.dll
 0000:fffc7000       .debug$S                   10000000     U2Lang:U2Lang.dll
 0000:fffc7000       .debug$S                   10000000     U2Lang:U2Lang.dll
 0000:fffc7000       .debug$S                   10000000     U2Lang:U2Lang.dll
 0000:fffc7000       .debug$S                   10000000     U2Lang:U2Lang.dll
 0000:fffc7000       .debug$S                   10000000     U2Lang:U2Lang.dll
 0000:fffc7000       .debug$S                   10000000     U2Lang:U2Lang.dll
 0000:fffc7000       .debug$S                   10000000     U2Lang:U2Lang.dll
 0000:fffc7000       .debug$S                   10000000     U2Lang:U2Lang.dll
 0000:fffc7000       .debug$S                   10000000     U2Lang:U2Lang.dll
 0000:fffc7000       .debug$S                   10000000     U2Lang:U2Lang.dll
 0000:fffc7000       .debug$S                   10000000     U2Lang:U2Lang.dll
 0000:fffc7000       .debug$S                   10000000     U2Lang:U2Lang.dll
 0000:fffc7000       .debug$S                   10000000     U2Lang:U2Lang.dll
 0000:fffc7000       .debug$S                   10000000     U2Lang:U2Lang.dll
 0000:fffc7000       .debug$S                   10000000     U2Lang:U2Lang.dll
 0000:fffc7000       .debug$S                   10000000     U2Lang:U2Lang.dll
 0000:fffc7000       .debug$S                   10000000     U2Lang:U2Lang.dll
 0000:fffc7000       .debug$S                   10000000     U2Lang:U2Lang.dll
 0000:fffc7000       .debug$S                   10000000     U2Lang:U2Lang.dll
 0000:fffc7000       .debug$S                   10000000     U2Lang:U2Lang.dll
 0000:fffc7000       .debug$S                   10000000     U2Lang:U2Lang.dll
 0000:fffc7000       .debug$S                   10000000     U2Lang:U2Lang.dll
 0000:fffc7000       .debug$S                   10000000     U2Designer:U2Designer.dll
 0000:fffc7000       .debug$S                   10000000     U2Designer:U2Designer.dll
 0000:fffc7000       .debug$S                   10000000     U2Designer:U2Designer.dll
 0000:fffc7000       .debug$S                   10000000     U2Designer:U2Designer.dll
 0000:fffc7000       .debug$S                   10000000     U2Designer:U2Designer.dll
 0000:fffc7000       .debug$S                   10000000     U2Designer:U2Designer.dll
 0000:fffc7000       .debug$S                   10000000     U2Designer:U2Designer.dll
 0000:fffc7000       .debug$S                   10000000     U2Designer:U2Designer.dll
 0000:fffc7000       .debug$S                   10000000     U2Designer:U2Designer.dll
 0000:fffc7000       .debug$S                   10000000     U2Designer:U2Designer.dll
 0000:fffc7000       .debug$S                   10000000     U2Designer:U2Designer.dll
 0000:fffc7000       .debug$S                   10000000     U2Designer:U2Designer.dll
 0000:fffc7000       .debug$S                   10000000     U2Designer:U2Designer.dll
 0002:fffe0000       __catchsym$?createNode@?$QMapData@VQString@@VQVariant@@@@QAEPAU?$QMapNode@VQString@@VQVariant@@@@ABVQString@@ABVQVariant@@PAU2@_N@Z$7 10000000     SamtoolMpileupWorker.obj
 0000:fffc7000       .debug$S                   10000000     U2Designer:U2Designer.dll
 0000:fffc7000       .debug$S                   10000000     U2Designer:U2Designer.dll
 0000:fffc7000       .debug$S                   10000000     U2Designer:U2Designer.dll
 0000:fffc7000       .debug$S                   10000000     U2Designer:U2Designer.dll
 0000:fffc7000       .debug$S                   10000000     U2Designer:U2Designer.dll
 0000:fffc7000       .debug$S                   10000000     U2Designer:U2Designer.dll
 0000:fffc7000       .debug$S                   10000000     U2Designer:U2Designer.dll
 0000:fffc7000       .debug$S                   10000000     U2Designer:U2Designer.dll
 0000:fffc7000       .debug$S                   10000000     U2Designer:U2Designer.dll
 0000:fffc7000       .debug$S                   10000000     U2Designer:U2Designer.dll
 0000:fffc7000       .debug$S                   10000000     U2Designer:U2Designer.dll
 0000:fffc7000       .debug$S                   10000000     U2Designer:U2Designer.dll
 0000:fffc7000       .debug$S                   10000000     U2Designer:U2Designer.dll
 0000:fffc7000       .debug$S                   10000000     U2Designer:U2Designer.dll
 0000:fffc7000       .debug$S                   10000000     U2Designer:U2Designer.dll
 0000:fffc7000       .debug$S                   10000000     U2Designer:U2Designer.dll
 0000:fffc7000       .debug$S                   10000000     U2Designer:U2Designer.dll
 0000:fffc7000       .debug$S                   10000000     U2Designer:U2Designer.dll
 0000:fffc7000       .debug$S                   10000000     U2Designer:U2Designer.dll
 0000:fffc7000       .debug$S                   10000000     U2Designer:U2Designer.dll
 0000:fffc7000       .debug$S                   10000000     U2Designer:U2Designer.dll
 0000:fffc7000       .debug$S                   10000000     U2Designer:U2Designer.dll
 0000:fffc7000       .debug$S                   10000000     U2Designer:U2Designer.dll
 0000:fffc7000       .debug$S                   10000000     U2Designer:U2Designer.dll
 0000:fffc7000       .debug$S                   10000000     U2Designer:U2Designer.dll
 0000:fffc7000       .debug$S                   10000000     U2Designer:U2Designer.dll
 0000:fffc7000       .debug$S                   10000000     U2Designer:U2Designer.dll
 0000:fffc7000       .debug$S                   10000000     U2Designer:U2Designer.dll
 0000:fffc7000       .debug$S                   10000000     U2Designer:U2Designer.dll
 0000:fffc7000       .debug$S                   10000000     U2Designer:U2Designer.dll
 0000:fffc7000       .debug$S                   10000000     U2Designer:U2Designer.dll
 0000:fffc7000       .debug$S                   10000000     U2Designer:U2Designer.dll
 0000:fffc7000       .debug$S                   10000000     U2Designer:U2Designer.dll
 0000:fffc7000       .debug$S                   10000000     U2Designer:U2Designer.dll
 0000:fffc7000       .debug$S                   10000000     U2Designer:U2Designer.dll
 0000:fffc7000       .debug$S                   10000000     U2Designer:U2Designer.dll
 0000:fffc7000       .debug$S                   10000000     U2Designer:U2Designer.dll
 0000:fffc7000       .debug$S                   10000000     U2Designer:U2Designer.dll
 0000:fffc7000       .debug$S                   10000000     U2Designer:U2Designer.dll
 0000:fffc7000       .debug$S                   10000000     U2Designer:U2Designer.dll
 0000:fffc7000       .debug$S                   10000000     U2Designer:U2Designer.dll
 0000:fffc7000       .debug$S                   10000000     U2Designer:U2Designer.dll
 0000:fffc7000       .debug$S                   10000000     U2Designer:U2Designer.dll
 0000:fffc7000       .debug$S                   10000000     U2Designer:U2Designer.dll
 0000:fffc7000       .debug$S                   10000000     U2Designer:U2Designer.dll
 0000:fffc7000       .debug$S                   10000000     U2Designer:U2Designer.dll
 0000:fffc7000       .debug$S                   10000000     U2Designer:U2Designer.dll
 0000:fffc7000       .debug$S                   10000000     Qt5Widgets:Qt5Widgets.dll
 0000:fffc7000       .debug$S                   10000000     Qt5Widgets:Qt5Widgets.dll
 0000:fffc7000       .debug$S                   10000000     Qt5Widgets:Qt5Widgets.dll
 0000:fffc7000       .debug$S                   10000000     Qt5Widgets:Qt5Widgets.dll
 0000:fffc7000       .debug$S                   10000000     Qt5Widgets:Qt5Widgets.dll
 0000:fffc7000       .debug$S                   10000000     Qt5Widgets:Qt5Widgets.dll
 0000:fffc7000       .debug$S                   10000000     Qt5Widgets:Qt5Widgets.dll
 0002:fffe0000       __catchsym$?node_copy@?$QList@V?$QMap@VQString@@VQVariant@@@@@@AAEXPAUNode@1@00@Z$6 10000000     SamtoolMpileupWorker.obj
 0000:fffc7000       .debug$S                   10000000     Qt5Widgets:Qt5Widgets.dll
 0000:fffc7000       .debug$S                   10000000     Qt5Widgets:Qt5Widgets.dll
 0000:fffc7000       .debug$S                   10000000     Qt5Widgets:Qt5Widgets.dll
 0000:fffc7000       .debug$S                   10000000     Qt5Widgets:Qt5Widgets.dll
 0002:fffe0000       __ehfuncinfo$??0CallVariantsTaskSettings@LocalWorkflow@U2@@QAE@ABV012@@Z 10000000     SamtoolMpileupWorker.obj
 0002:fffe0000       __ehfuncinfo$??1CallVariantsTaskSettings@LocalWorkflow@U2@@QAE@XZ 10000000     SamtoolMpileupWorker.obj
 0000:fffc7000       .debug$S                   10000000     Qt5Widgets:Qt5Widgets.dll
 0000:fffc7000       .debug$S                   10000000     Qt5Widgets:Qt5Widgets.dll
 0000:fffc7000       .debug$S                   10000000     Qt5Widgets:Qt5Widgets.dll
 0000:fffc7000       .debug$S                   10000000     Qt5Widgets:Qt5Widgets.dll
 0000:fffc7000       .debug$S                   10000000     Qt5Widgets:Qt5Widgets.dll
 0000:fffc7000       .debug$S                   10000000     Qt5Widgets:Qt5Widgets.dll
 0000:fffc7000       .debug$S                   10000000     Qt5Widgets:Qt5Widgets.dll
 0000:fffc7000       .debug$S                   10000000     Qt5Widgets:Qt5Widgets.dll
 0000:fffc7000       .debug$S                   10000000     Qt5Widgets:Qt5Widgets.dll
 0000:fffc7000       .debug$S                   10000000     Qt5Widgets:Qt5Widgets.dll
 0000:fffc7000       .debug$S                   10000000     Qt5Widgets:Qt5Widgets.dll
 0000:fffc7000       .debug$S                   10000000     Qt5Widgets:Qt5Widgets.dll
 0001:fffff000       __ehhandler$?_Copy@?$basic_string@DU?$char_traits@D@std@@V?$allocator@D@2@@std@@QAEXII@Z 10000000 f   SamtoolMpileupWorker.obj
 0000:fffc7000       .debug$S                   10000000     Qt5Widgets:Qt5Widgets.dll
 0000:fffc7000       .debug$S                   10000000     Qt5Widgets:Qt5Widgets.dll
 0000:fffc7000       .debug$S                   10000000     Qt5Widgets:Qt5Widgets.dll
 0000:fffc7000       .debug$S                   10000000     Qt5Widgets:Qt5Widgets.dll
 0000:fffc7000       .debug$S                   10000000     Qt5Widgets:Qt5Widgets.dll
 0000:fffc7000       .debug$S                   10000000     Qt5Widgets:Qt5Widgets.dll
 0000:fffc7000       .debug$S                   10000000     Qt5Widgets:Qt5Widgets.dll
 0001:fffff000       __ehhandler$??0?$QList@VQString@@@@QAE@ABV0@@Z 10000000 f   SamtoolMpileupWorker.obj
 0000:fffc7000       .debug$S                   10000000     Qt5Widgets:Qt5Widgets.dll
 0000:fffc7000       .debug$S                   10000000     Qt5Widgets:Qt5Widgets.dll
 0000:fffc7000       .debug$S                   10000000     Qt5Widgets:Qt5Widgets.dll
 0000:fffc7000       .debug$S                   10000000     Qt5Widgets:Qt5Widgets.dll
 0001:fffff000       __unwindfunclet$?append@?$QList@VQString@@@@QAEXABVQString@@@Z$7 10000000 f   SamtoolMpileupWorker.obj
 0000:fffc7000       .debug$S                   10000000     Qt5Widgets:Qt5Widgets.dll
 0001:fffff000       __ehhandler$?detach_helper_grow@?$QList@VQString@@@@AAEPAUNode@1@HH@Z 10000000 f   SamtoolMpileupWorker.obj
 0000:fffc7000       .debug$S                   10000000     Qt5Widgets:Qt5Widgets.dll
 0000:fffc7000       .debug$S                   10000000     Qt5Widgets:Qt5Widgets.dll
 0000:fffc7000       .debug$S                   10000000     Qt5Widgets:Qt5Widgets.dll
 0001:fffff000       __unwindfunclet$?node_construct@?$QList@VQString@@@@AAEXPAUNode@1@ABVQString@@@Z$1 10000000 f   SamtoolMpileupWorker.obj
 0000:fffc7000       .debug$S                   10000000     Qt5Widgets:Qt5Widgets.dll
 0000:fffc7000       .debug$S                   10000000     Qt5Widgets:Qt5Widgets.dll
 0001:fffff000       __unwindfunclet$?node_copy@?$QList@VQString@@@@AAEXPAUNode@1@00@Z$5 10000000 f   SamtoolMpileupWorker.obj
 0000:fffc7000       .debug$S                   10000000     Qt5Widgets:Qt5Widgets.dll
 0001:fffff000       __unwindfunclet$??A?$QMap@VQString@@VQVariant@@@@QAEAAVQVariant@@ABVQString@@@Z$0 10000000 f   SamtoolMpileupWorker.obj
 0000:fffc7000       .debug$S                   10000000     Qt5Widgets:Qt5Widgets.dll
 0000:fffc7000       .debug$S                   10000000     Qt5Widgets:Qt5Widgets.dll
 0000:fffc7000       .debug$S                   10000000     Qt5Widgets:Qt5Widgets.dll
 0000:fffc7000       .debug$S                   10000000     Qt5Widgets:Qt5Widgets.dll
 0000:fffc7000       .debug$S                   10000000     Qt5Widgets:Qt5Widgets.dll
 0000:fffc7000       .debug$S                   10000000     Qt5Widgets:Qt5Widgets.dll
 0000:fffc7000       .debug$S                   10000000     Qt5Widgets:Qt5Widgets.dll
 0000:fffc7000       .debug$S                   10000000     Qt5Widgets:Qt5Widgets.dll
 0000:fffc7000       .debug$S                   10000000     Qt5Widgets:Qt5Widgets.dll
 0000:fffc7000       .debug$S                   10000000     Qt5Widgets:Qt5Widgets.dll
 0000:fffc7000       .debug$S                   10000000     Qt5Widgets:Qt5Widgets.dll
 0000:fffc7000       .debug$S                   10000000     Qt5Widgets:Qt5Widgets.dll
 0000:fffc7000       .debug$S                   10000000     Qt5Widgets:Qt5Widgets.dll
 0000:fffc7000       .debug$S                   10000000     Qt5Widgets:Qt5Widgets.dll
 0000:fffc7000       .debug$S                   10000000     Qt5Widgets:Qt5Widgets.dll
 0000:fffc7000       .debug$S                   10000000     Qt5Widgets:Qt5Widgets.dll
 0000:fffc7000       .debug$S                   10000000     Qt5Widgets:Qt5Widgets.dll
 0000:fffc7000       .debug$S                   10000000     Qt5Widgets:Qt5Widgets.dll
 0000:fffc7000       .debug$S                   10000000     Qt5Widgets:Qt5Widgets.dll
 0000:fffc7000       .debug$S                   10000000     Qt5Widgets:Qt5Widgets.dll
 0000:fffc7000       .debug$S                   10000000     Qt5Widgets:Qt5Widgets.dll
 0000:fffc7000       .debug$S                   10000000     Qt5Widgets:Qt5Widgets.dll
 0000:fffc7000       .debug$S                   10000000     Qt5Widgets:Qt5Widgets.dll
 0000:fffc7000       .debug$S                   10000000     Qt5Widgets:Qt5Widgets.dll
 0000:fffc7000       .debug$S                   10000000     Qt5Widgets:Qt5Widgets.dll
 0000:fffc7000       .debug$S                   10000000     Qt5Widgets:Qt5Widgets.dll
 0000:fffc7000       .debug$S                   10000000     Qt5Widgets:Qt5Widgets.dll
 0000:fffc7000       .debug$S                   10000000     Qt5Widgets:Qt5Widgets.dll
 0000:fffc7000       .debug$S                   10000000     Qt5Widgets:Qt5Widgets.dll
 0000:fffc7000       .debug$S                   10000000     Qt5Widgets:Qt5Widgets.dll
 0000:fffc7000       .debug$S                   10000000     Qt5Widgets:Qt5Widgets.dll
 0000:fffc7000       .debug$S                   10000000     Qt5Widgets:Qt5Widgets.dll
 0000:fffc7000       .debug$S                   10000000     Qt5Widgets:Qt5Widgets.dll
 0000:fffc7000       .debug$S                   10000000     Qt5Widgets:Qt5Widgets.dll
 0000:fffc7000       .debug$S                   10000000     Qt5Widgets:Qt5Widgets.dll
 0000:fffc7000       .debug$S                   10000000     Qt5Widgets:Qt5Widgets.dll
 0000:fffc7000       .debug$S                   10000000     Qt5Widgets:Qt5Widgets.dll
 0000:fffc7000       .debug$S                   10000000     Qt5Widgets:Qt5Widgets.dll
 0000:fffc7000       .debug$S                   10000000     Qt5Widgets:Qt5Widgets.dll
 0000:fffc7000       .debug$S                   10000000     Qt5Gui:Qt5Gui.dll
 0000:fffc7000       .debug$S                   10000000     Qt5Gui:Qt5Gui.dll
 0000:fffc7000       .debug$S                   10000000     Qt5Gui:Qt5Gui.dll
 0000:fffc7000       .debug$S                   10000000     Qt5Gui:Qt5Gui.dll
 0000:fffc7000       .debug$S                   10000000     Qt5Gui:Qt5Gui.dll
 0000:fffc7000       .debug$S                   10000000     Qt5Gui:Qt5Gui.dll
 0000:fffc7000       .debug$S                   10000000     Qt5Gui:Qt5Gui.dll
 0000:fffc7000       .debug$S                   10000000     Qt5Gui:Qt5Gui.dll
 0000:fffc7000       .debug$S                   10000000     Qt5Gui:Qt5Gui.dll
 0000:fffc7000       .debug$S                   10000000     Qt5Gui:Qt5Gui.dll
 0000:fffc7000       .debug$S                   10000000     Qt5Gui:Qt5Gui.dll
 0000:fffc7000       .debug$S                   10000000     Qt5Gui:Qt5Gui.dll
 0000:fffc7000       .debug$S                   10000000     Qt5Script:Qt5Script.dll
 0000:fffc7000       .debug$S                   10000000     Qt5Script:Qt5Script.dll
 0000:fffc7000       .debug$S                   10000000     Qt5Script:Qt5Script.dll
 0000:fffc7000       .debug$S                   10000000     Qt5Script:Qt5Script.dll
 0000:fffc7000       .debug$S                   10000000     Qt5Script:Qt5Script.dll
 0000:fffc7000       .debug$S                   10000000     Qt5Script:Qt5Script.dll
 0000:fffc7000       .debug$S                   10000000     Qt5Script:Qt5Script.dll
 0000:fffc7000       .debug$S                   10000000     Qt5Script:Qt5Script.dll
 0000:fffc7000       .debug$S                   10000000     Qt5Script:Qt5Script.dll
 0000:fffc7000       .debug$S                   10000000     Qt5Script:Qt5Script.dll
 0000:fffc7000       .debug$S                   10000000     Qt5Core:Qt5Core.dll
 0000:fffc7000       .debug$S                   10000000     Qt5Core:Qt5Core.dll
 0000:fffc7000       .debug$S                   10000000     Qt5Core:Qt5Core.dll
 0000:fffc7000       .debug$S                   10000000     Qt5Core:Qt5Core.dll
 0000:fffc7000       .debug$S                   10000000     Qt5Core:Qt5Core.dll
 0000:fffc7000       .debug$S                   10000000     Qt5Core:Qt5Core.dll
 0000:fffc7000       .debug$S                   10000000     Qt5Core:Qt5Core.dll
 0000:fffc7000       .debug$S                   10000000     Qt5Core:Qt5Core.dll
 0000:fffc7000       .debug$S                   10000000     Qt5Core:Qt5Core.dll
 0000:fffc7000       .debug$S                   10000000     Qt5Core:Qt5Core.dll
 0000:fffc7000       .debug$S                   10000000     Qt5Core:Qt5Core.dll
 0000:fffc7000       .debug$S                   10000000     Qt5Core:Qt5Core.dll
 0000:fffc7000       .debug$S                   10000000     Qt5Core:Qt5Core.dll
 0000:fffc7000       .debug$S                   10000000     Qt5Core:Qt5Core.dll
 0000:fffc7000       .debug$S                   10000000     Qt5Core:Qt5Core.dll
 0000:fffc7000       .debug$S                   10000000     Qt5Core:Qt5Core.dll
 0000:fffc7000       .debug$S                   10000000     Qt5Core:Qt5Core.dll
 0000:fffc7000       .debug$S                   10000000     Qt5Core:Qt5Core.dll
 0000:fffc7000       .debug$S                   10000000     Qt5Core:Qt5Core.dll
 0000:fffc7000       .debug$S                   10000000     Qt5Core:Qt5Core.dll
 0000:fffc7000       .debug$S                   10000000     Qt5Core:Qt5Core.dll
 0000:fffc7000       .debug$S                   10000000     Qt5Core:Qt5Core.dll
 0000:fffc7000       .debug$S                   10000000     Qt5Core:Qt5Core.dll
 0000:fffc7000       .debug$S                   10000000     Qt5Core:Qt5Core.dll
 0000:fffc7000       .debug$S                   10000000     Qt5Core:Qt5Core.dll
 0000:fffc7000       .debug$S                   10000000     Qt5Core:Qt5Core.dll
 0000:fffc7000       .debug$S                   10000000     Qt5Core:Qt5Core.dll
 0000:fffc7000       .debug$S                   10000000     Qt5Core:Qt5Core.dll
 0000:fffc7000       .debug$S                   10000000     Qt5Core:Qt5Core.dll
 0000:fffc7000       .debug$S                   10000000     Qt5Core:Qt5Core.dll
 0000:fffc7000       .debug$S                   10000000     Qt5Core:Qt5Core.dll
 0000:fffc7000       .debug$S                   10000000     Qt5Core:Qt5Core.dll
 0000:fffc7000       .debug$S                   10000000     Qt5Core:Qt5Core.dll
 0002:fffe0000       __unwindtable$??A?$QMap@VQString@@VQVariant@@@@QAEAAVQVariant@@ABVQString@@@Z 10000000     SamtoolMpileupWorker.obj
 0002:fffe0000       __catchsym$?node_copy@?$QList@VQString@@@@AAEXPAUNode@1@00@Z$6 10000000     SamtoolMpileupWorker.obj
 0002:fffe0000       __unwindtable$?node_construct@?$QList@VQString@@@@AAEXPAUNode@1@ABVQString@@@Z 10000000     SamtoolMpileupWorker.obj
 0002:fffe0000       __catchsym$?detach_helper_grow@?$QList@VQString@@@@AAEPAUNode@1@HH@Z$5 10000000     SamtoolMpileupWorker.obj
 0002:fffe0000       __catchsym$?append@?$QList@VQString@@@@QAEXABVQString@@@Z$13 10000000     SamtoolMpileupWorker.obj
 0002:fffe0000       __catchsym$??0?$QList@VQString@@@@QAE@ABV0@@Z$2 10000000     SamtoolMpileupWorker.obj
 0002:fffe0000       __catchsym$?_Copy@?$basic_string@DU?$char_traits@D@std@@V?$allocator@D@2@@std@@QAEXII@Z$5 10000000     SamtoolMpileupWorker.obj
 0001:fffff000       __unwindfunclet$?createNode@?$QMapData@VQString@@VQVariant@@@@QAEPAU?$QMapNode@VQString@@VQVariant@@@@ABVQString@@ABVQVariant@@PAU2@_N@Z$4 10000000 f   SamtoolMpileupWorker.obj
 0000:fffc7000       .debug$S                   10000000     U2Lang:U2Lang.dll
 0001:fffff000       __unwindfunclet$?node_copy@?$QList@V?$QMap@VQString@@VQVariant@@@@@@AAEXPAUNode@1@00@Z$4 10000000 f   SamtoolMpileupWorker.obj
 0001:fffff000       __unwindfunclet$??0CallVariantsTaskSettings@LocalWorkflow@U2@@QAE@ABV012@@Z$0 10000000 f   SamtoolMpileupWorker.obj
 0001:fffff000       __unwindfunclet$??1CallVariantsTaskSettings@LocalWorkflow@U2@@QAE@XZ$0 10000000 f   SamtoolMpileupWorker.obj
 0002:fffe0008       __ehfuncinfo$??A?$QMap@VQString@@VQVariant@@@@QAEAAVQVariant@@ABVQString@@@Z 10000008     SamtoolMpileupWorker.obj
 0001:fffff009       __ehhandler$??A?$QMap@VQString@@VQVariant@@@@QAEAAVQVariant@@ABVQString@@@Z 10000009 f   SamtoolMpileupWorker.obj
 0001:fffff009       __unwindfunclet$??1CallVariantsTaskSettings@LocalWorkflow@U2@@QAE@XZ$1 10000009 f   SamtoolMpileupWorker.obj
 0001:fffff009       __unwindfunclet$??0CallVariantsTaskSettings@LocalWorkflow@U2@@QAE@ABV012@@Z$1 10000009 f   SamtoolMpileupWorker.obj
 0001:fffff00b       __ehhandler$?node_copy@?$QList@V?$QMap@VQString@@VQVariant@@@@@@AAEXPAUNode@1@00@Z 1000000b f   SamtoolMpileupWorker.obj
 0002:fffe0010       __catchsym$?detach_helper_grow@?$QList@VQString@@@@AAEPAUNode@1@HH@Z$4 10000010     SamtoolMpileupWorker.obj
 0002:fffe0010       __catchsym$?append@?$QList@VQString@@@@QAEXABVQString@@@Z$12 10000010     SamtoolMpileupWorker.obj
 0002:fffe0010       __catchsym$?createNode@?$QMapData@VQString@@VQVariant@@@@QAEPAU?$QMapNode@VQString@@VQVariant@@@@ABVQString@@ABVQVariant@@PAU2@_N@Z$6 10000010     SamtoolMpileupWorker.obj
 0002:fffe0010       __catchsym$?_Copy@?$basic_string@DU?$char_traits@D@std@@V?$allocator@D@2@@std@@QAEXII@Z$4 10000010     SamtoolsPlugin.obj
 0002:fffe0010       __tryblocktable$?node_copy@?$QList@V?$QMap@VQString@@VQVariant@@@@@@AAEXPAUNode@1@00@Z 10000010     SamtoolMpileupWorker.obj
 0002:fffe0010       __tryblocktable$?node_copy@?$QList@VQString@@@@AAEXPAUNode@1@00@Z 10000010     SamtoolMpileupWorker.obj
 0002:fffe0010       __ehfuncinfo$?node_construct@?$QList@VQString@@@@AAEXPAUNode@1@ABVQString@@@Z 10000010     SamtoolMpileupWorker.obj
 0002:fffe0010       __catchsym$?_Copy@?$basic_string@DU?$char_traits@D@std@@V?$allocator@D@2@@std@@QAEXII@Z$4 10000010     moc_AssemblySamtoolsMpileup.obj
 0002:fffe0010       __catchsym$?_Copy@?$basic_string@DU?$char_traits@D@std@@V?$allocator@D@2@@std@@QAEXII@Z$4 10000010     moc_SamtoolMpileupWorker.obj
 0002:fffe0010       __catchsym$?_Copy@?$basic_string@DU?$char_traits@D@std@@V?$allocator@D@2@@std@@QAEXII@Z$4 10000010     SamtoolMpileupWorker.obj
 0002:fffe0010       __catchsym$?_Copy@?$basic_string@DU?$char_traits@D@std@@V?$allocator@D@2@@std@@QAEXII@Z$4 10000010     moc_SamtoolsPlugin.obj
 0002:fffe0010       __unwindtable$??0?$QList@VQString@@@@QAE@ABV0@@Z 10000010     SamtoolMpileupWorker.obj
 0001:fffff011       __unwindfunclet$?append@?$QList@VQString@@@@QAEXABVQString@@@Z$11 10000011 f   SamtoolMpileupWorker.obj
 0001:fffff011       __ehhandler$?node_copy@?$QList@VQString@@@@AAEXPAUNode@1@00@Z 10000011 f   SamtoolMpileupWorker.obj
 0001:fffff011       __ehhandler$?node_construct@?$QList@VQString@@@@AAEXPAUNode@1@ABVQString@@@Z 10000011 f   SamtoolMpileupWorker.obj
 0001:fffff014       __unwindfunclet$??1CallVariantsTaskSettings@LocalWorkflow@U2@@QAE@XZ$2 10000014 f   SamtoolMpileupWorker.obj
 0001:fffff014       __unwindfunclet$??0CallVariantsTaskSettings@LocalWorkflow@U2@@QAE@ABV012@@Z$2 10000014 f   SamtoolMpileupWorker.obj
 0001:fffff014       __unwindfunclet$?createNode@?$QMapData@VQString@@VQVariant@@@@QAEPAU?$QMapNode@VQString@@VQVariant@@@@ABVQString@@ABVQVariant@@PAU2@_N@Z$5 10000014 f   SamtoolMpileupWorker.obj
 0002:fffe0020       __unwindtable$?detach_helper_grow@?$QList@VQString@@@@AAEPAUNode@1@HH@Z 10000020     SamtoolMpileupWorker.obj
 0002:fffe0020       __tryblocktable$??0?$QList@VQString@@@@QAE@ABV0@@Z 10000020     SamtoolMpileupWorker.obj
 0002:fffe0020       __unwindtable$?_Copy@?$basic_string@DU?$char_traits@D@std@@V?$allocator@D@2@@std@@QAEXII@Z 10000020     moc_AssemblySamtoolsMpileup.obj
 0002:fffe0020       __unwindtable$?_Copy@?$basic_string@DU?$char_traits@D@std@@V?$allocator@D@2@@std@@QAEXII@Z 10000020     SamtoolMpileupWorker.obj
 0001:fffff020       __unwindfunclet$??0CallVariantsTaskSettings@LocalWorkflow@U2@@QAE@ABV012@@Z$3 10000020 f   SamtoolMpileupWorker.obj
 0002:fffe0020       __unwindtable$?_Copy@?$basic_string@DU?$char_traits@D@std@@V?$allocator@D@2@@std@@QAEXII@Z 10000020     SamtoolsPlugin.obj
 0002:fffe0020       __unwindtable$?_Copy@?$basic_string@DU?$char_traits@D@std@@V?$allocator@D@2@@std@@QAEXII@Z 10000020     moc_SamtoolsPlugin.obj
 0002:fffe0020       __ehfuncinfo$?createNode@?$QMapData@VQString@@VQVariant@@@@QAEPAU?$QMapNode@VQString@@VQVariant@@@@ABVQString@@ABVQVariant@@PAU2@_N@Z 10000020     SamtoolMpileupWorker.obj
 0001:fffff020       __unwindfunclet$??1CallVariantsTaskSettings@LocalWorkflow@U2@@QAE@XZ$3 10000020 f   SamtoolMpileupWorker.obj
 0002:fffe0020       __unwindtable$?_Copy@?$basic_string@DU?$char_traits@D@std@@V?$allocator@D@2@@std@@QAEXII@Z 10000020     moc_SamtoolMpileupWorker.obj
 0002:fffe0020       __ehfuncinfo$?append@?$QList@VQString@@@@QAEXABVQString@@@Z 10000020     SamtoolMpileupWorker.obj
 0001:fffff022       __ehhandler$?append@?$QList@VQString@@@@QAEXABVQString@@@Z 10000022 f   SamtoolMpileupWorker.obj
 0002:fffe0024       __unwindtable$??0CallVariantsTaskSettings@LocalWorkflow@U2@@QAE@ABV012@@Z 10000024     SamtoolMpileupWorker.obj
 0002:fffe0024       __ehfuncinfo$?node_copy@?$QList@V?$QMap@VQString@@VQVariant@@@@@@AAEXPAUNode@1@00@Z 10000024     SamtoolMpileupWorker.obj
 0002:fffe0024       __unwindtable$??1CallVariantsTaskSettings@LocalWorkflow@U2@@QAE@XZ 10000024     SamtoolMpileupWorker.obj
 0002:fffe0024       __ehfuncinfo$?node_copy@?$QList@VQString@@@@AAEXPAUNode@1@00@Z 10000024     SamtoolMpileupWorker.obj
 0001:fffff028       __ehhandler$?createNode@?$QMapData@VQString@@VQVariant@@@@QAEPAU?$QMapNode@VQString@@VQVariant@@@@ABVQString@@ABVQVariant@@PAU2@_N@Z 10000028 f   SamtoolMpileupWorker.obj
 0001:fffff02c       __unwindfunclet$??0CallVariantsTaskSettings@LocalWorkflow@U2@@QAE@ABV012@@Z$4 1000002c f   SamtoolMpileupWorker.obj
 0001:fffff02c       __unwindfunclet$??1CallVariantsTaskSettings@LocalWorkflow@U2@@QAE@XZ$4 1000002c f   SamtoolMpileupWorker.obj
 0002:fffe0034       __ehfuncinfo$??0?$QList@VQString@@@@QAE@ABV0@@Z 10000034     SamtoolMpileupWorker.obj
 0001:fffff038       __unwindfunclet$??0CallVariantsTaskSettings@LocalWorkflow@U2@@QAE@ABV012@@Z$5 10000038 f   SamtoolMpileupWorker.obj
 0001:fffff038       __unwindfunclet$??1CallVariantsTaskSettings@LocalWorkflow@U2@@QAE@XZ$5 10000038 f   SamtoolMpileupWorker.obj
 0002:fffe0040       __ehfuncinfo$?_Copy@?$basic_string@DU?$char_traits@D@std@@V?$allocator@D@2@@std@@QAEXII@Z 10000040     moc_SamtoolMpileupWorker.obj
 0002:fffe0040       __ehfuncinfo$?detach_helper_grow@?$QList@VQString@@@@AAEPAUNode@1@HH@Z 10000040     SamtoolMpileupWorker.obj
 0002:fffe0040       __ehfuncinfo$?_Copy@?$basic_string@DU?$char_traits@D@std@@V?$allocator@D@2@@std@@QAEXII@Z 10000040     moc_SamtoolsPlugin.obj
 0002:fffe0040       __ehfuncinfo$?_Copy@?$basic_string@DU?$char_traits@D@std@@V?$allocator@D@2@@std@@QAEXII@Z 10000040     SamtoolsPlugin.obj
 0002:fffe0040       __ehfuncinfo$?_Copy@?$basic_string@DU?$char_traits@D@std@@V?$allocator@D@2@@std@@QAEXII@Z 10000040     moc_AssemblySamtoolsMpileup.obj
 0002:fffe0040       __ehfuncinfo$?_Copy@?$basic_string@DU?$char_traits@D@std@@V?$allocator@D@2@@std@@QAEXII@Z 10000040     SamtoolMpileupWorker.obj
 0001:fffff044       __unwindfunclet$??0CallVariantsTaskSettings@LocalWorkflow@U2@@QAE@ABV012@@Z$6 10000044 f   SamtoolMpileupWorker.obj
 0002:fffe0044       __tryblocktable$?createNode@?$QMapData@VQString@@VQVariant@@@@QAEPAU?$QMapNode@VQString@@VQVariant@@@@ABVQString@@ABVQVariant@@PAU2@_N@Z 10000044     SamtoolMpileupWorker.obj
 0001:fffff044       __unwindfunclet$??1CallVariantsTaskSettings@LocalWorkflow@U2@@QAE@XZ$6 10000044 f   SamtoolMpileupWorker.obj
 0002:fffe0044       __tryblocktable$?append@?$QList@VQString@@@@QAEXABVQString@@@Z 10000044     SamtoolMpileupWorker.obj
 0002:fffe0048       __unwindtable$?node_copy@?$QList@VQString@@@@AAEXPAUNode@1@00@Z 10000048     SamtoolMpileupWorker.obj
 0002:fffe0048       __unwindtable$?node_copy@?$QList@V?$QMap@VQString@@VQVariant@@@@@@AAEXPAUNode@1@00@Z 10000048     SamtoolMpileupWorker.obj
 0001:fffff050       __unwindfunclet$??1CallVariantsTaskSettings@LocalWorkflow@U2@@QAE@XZ$7 10000050 f   SamtoolMpileupWorker.obj
 0001:fffff050       __unwindfunclet$??0CallVariantsTaskSettings@LocalWorkflow@U2@@QAE@ABV012@@Z$7 10000050 f   SamtoolMpileupWorker.obj
 0001:fffff05c       __unwindfunclet$??0CallVariantsTaskSettings@LocalWorkflow@U2@@QAE@ABV012@@Z$8 1000005c f   SamtoolMpileupWorker.obj
 0001:fffff05c       __unwindfunclet$??1CallVariantsTaskSettings@LocalWorkflow@U2@@QAE@XZ$8 1000005c f   SamtoolMpileupWorker.obj
 0001:fffff062       __catch$?node_copy@?$QList@VQString@@@@AAEXPAUNode@1@00@Z$2 10000062 f   SamtoolMpileupWorker.obj
 0002:fffe0064       __tryblocktable$?_Copy@?$basic_string@DU?$char_traits@D@std@@V?$allocator@D@2@@std@@QAEXII@Z 10000064     SamtoolMpileupWorker.obj
 0002:fffe0064       __tryblocktable$?_Copy@?$basic_string@DU?$char_traits@D@std@@V?$allocator@D@2@@std@@QAEXII@Z 10000064     moc_SamtoolsPlugin.obj
 0002:fffe0064       __tryblocktable$?_Copy@?$basic_string@DU?$char_traits@D@std@@V?$allocator@D@2@@std@@QAEXII@Z 10000064     SamtoolsPlugin.obj
 0002:fffe0064       __tryblocktable$?detach_helper_grow@?$QList@VQString@@@@AAEPAUNode@1@HH@Z 10000064     SamtoolMpileupWorker.obj
 0002:fffe0064       __tryblocktable$?_Copy@?$basic_string@DU?$char_traits@D@std@@V?$allocator@D@2@@std@@QAEXII@Z 10000064     moc_AssemblySamtoolsMpileup.obj
 0002:fffe0064       __tryblocktable$?_Copy@?$basic_string@DU?$char_traits@D@std@@V?$allocator@D@2@@std@@QAEXII@Z 10000064     moc_SamtoolMpileupWorker.obj
 0001:fffff068       __ehhandler$??0CallVariantsTaskSettings@LocalWorkflow@U2@@QAE@ABV012@@Z 10000068 f   SamtoolMpileupWorker.obj
 0001:fffff068       __ehhandler$??1CallVariantsTaskSettings@LocalWorkflow@U2@@QAE@XZ 10000068 f   SamtoolMpileupWorker.obj
 0002:fffe006c       __unwindtable$?createNode@?$QMapData@VQString@@VQVariant@@@@QAEPAU?$QMapNode@VQString@@VQVariant@@@@ABVQString@@ABVQVariant@@PAU2@_N@Z 1000006c     SamtoolMpileupWorker.obj
 0002:fffe006c       __unwindtable$?append@?$QList@VQString@@@@QAEXABVQString@@@Z 1000006c     SamtoolMpileupWorker.obj
 0001:fffff07d       __catch$?append@?$QList@VQString@@@@QAEXABVQString@@@Z$0 1000007d f   SamtoolMpileupWorker.obj
 0001:fffff08e       __catch$?createNode@?$QMapData@VQString@@VQVariant@@@@QAEPAU?$QMapNode@VQString@@VQVariant@@@@ABVQString@@ABVQVariant@@PAU2@_N@Z$0 1000008e f   SamtoolMpileupWorker.obj
 0001:fffff096       __catch$?_Copy@?$basic_string@DU?$char_traits@D@std@@V?$allocator@D@2@@std@@QAEXII@Z$0 10000096 f   moc_SamtoolsPlugin.obj
 0001:fffff096       __catch$?_Copy@?$basic_string@DU?$char_traits@D@std@@V?$allocator@D@2@@std@@QAEXII@Z$0 10000096 f   moc_SamtoolMpileupWorker.obj
 0001:fffff096       __catch$?_Copy@?$basic_string@DU?$char_traits@D@std@@V?$allocator@D@2@@std@@QAEXII@Z$0 10000096 f   SamtoolMpileupWorker.obj
 0001:fffff096       __catch$?_Copy@?$basic_string@DU?$char_traits@D@std@@V?$allocator@D@2@@std@@QAEXII@Z$0 10000096 f   SamtoolsPlugin.obj
 0001:fffff096       __catch$?_Copy@?$basic_string@DU?$char_traits@D@std@@V?$allocator@D@2@@std@@QAEXII@Z$0 10000096 f   moc_AssemblySamtoolsMpileup.obj
 0001:fffff09e       __catch$??0?$QList@VQString@@@@QAE@ABV0@@Z$0 1000009e f   SamtoolMpileupWorker.obj
 0001:fffff0a3       __catch$?createNode@?$QMapData@VQString@@VQVariant@@@@QAEPAU?$QMapNode@VQString@@VQVariant@@@@ABVQString@@ABVQVariant@@PAU2@_N@Z$2 100000a3 f   SamtoolMpileupWorker.obj
 0001:fffff0ce       __catch$?append@?$QList@VQString@@@@QAEXABVQString@@@Z$4 100000ce f   SamtoolMpileupWorker.obj
 0001:fffff0d3       __catch$?_Copy@?$basic_string@DU?$char_traits@D@std@@V?$allocator@D@2@@std@@QAEXII@Z$1 100000d3 f   SamtoolsPlugin.obj
 0001:fffff0d3       __catch$?_Copy@?$basic_string@DU?$char_traits@D@std@@V?$allocator@D@2@@std@@QAEXII@Z$1 100000d3 f   moc_AssemblySamtoolsMpileup.obj
 0001:fffff0d3       __catch$?_Copy@?$basic_string@DU?$char_traits@D@std@@V?$allocator@D@2@@std@@QAEXII@Z$1 100000d3 f   SamtoolMpileupWorker.obj
 0001:fffff0d3       __catch$?_Copy@?$basic_string@DU?$char_traits@D@std@@V?$allocator@D@2@@std@@QAEXII@Z$1 100000d3 f   moc_SamtoolMpileupWorker.obj
 0001:fffff0d3       __catch$?_Copy@?$basic_string@DU?$char_traits@D@std@@V?$allocator@D@2@@std@@QAEXII@Z$1 100000d3 f   moc_SamtoolsPlugin.obj
 0001:fffff0e1       __catch$?node_copy@?$QList@V?$QMap@VQString@@VQVariant@@@@@@AAEXPAUNode@1@00@Z$0 100000e1 f   SamtoolMpileupWorker.obj
 0001:fffff11e       __catch$?detach_helper_grow@?$QList@VQString@@@@AAEPAUNode@1@HH@Z$2 1000011e f   SamtoolMpileupWorker.obj
 0001:fffff159       __catch$?detach_helper_grow@?$QList@VQString@@@@AAEPAUNode@1@HH@Z$0 10000159 f   SamtoolMpileupWorker.obj
 0001:00000000       ??__E?BCFTOOLS_ID@SamtoolsMpileupTask@LocalWorkflow@U2@@0VQString@@B@@YAXXZ 10001000 f   AssemblySamtoolsMpileup.obj
 0001:00000020       ??__E?SAMTOOLS_ID@SamtoolsMpileupTask@LocalWorkflow@U2@@0VQString@@B@@YAXXZ 10001020 f   AssemblySamtoolsMpileup.obj
 0001:00000040       ??__E?VCFUTILS_ID@SamtoolsMpileupTask@LocalWorkflow@U2@@0VQString@@B@@YAXXZ 10001040 f   AssemblySamtoolsMpileup.obj
 0001:00000060       ??__E?_Generic_object@?$_Error_objects@H@std@@2V_Generic_error_category@2@A@@YAXXZ 10001060 f   AssemblySamtoolsMpileup.obj
 0001:00000070       ??__E?_Iostream_object@?$_Error_objects@H@std@@2V_Iostream_error_category@2@A@@YAXXZ 10001070 f   AssemblySamtoolsMpileup.obj
 0001:00000080       ??__E?_System_object@?$_Error_objects@H@std@@2V_System_error_category@2@A@@YAXXZ 10001080 f   AssemblySamtoolsMpileup.obj
 0001:00000090       ??__EalgoLog@U2@@YAXXZ     10001090 f   AssemblySamtoolsMpileup.obj
 0001:00000110       ??__EcmdLog@U2@@YAXXZ      10001110 f   AssemblySamtoolsMpileup.obj
 0001:00000190       ??__EcoreLog@U2@@YAXXZ     10001190 f   AssemblySamtoolsMpileup.obj
 0001:00000210       ??__EioLog@U2@@YAXXZ       10001210 f   AssemblySamtoolsMpileup.obj
 0001:00000290       ??__EperfLog@U2@@YAXXZ     10001290 f   AssemblySamtoolsMpileup.obj
 0001:00000310       ??__EscriptLog@U2@@YAXXZ   10001310 f   AssemblySamtoolsMpileup.obj
 0001:00000390       ??__EtaskLog@U2@@YAXXZ     10001390 f   AssemblySamtoolsMpileup.obj
 0001:00000410       ??__EuiLog@U2@@YAXXZ       10001410 f   AssemblySamtoolsMpileup.obj
 0001:00000490       ??__EuserActLog@U2@@YAXXZ  10001490 f   AssemblySamtoolsMpileup.obj
 0001:00000510       ??__E?ACTOR_ID@CallVariantsWorkerFactory@LocalWorkflow@U2@@2VQString@@B@@YAXXZ 10001510 f   SamtoolMpileupWorker.obj
 0001:00000530       ??__E?_Generic_object@?$_Error_objects@H@std@@2V_Generic_error_category@2@A@@YAXXZ 10001530 f   SamtoolMpileupWorker.obj
 0001:00000540       ??__E?_Iostream_object@?$_Error_objects@H@std@@2V_Iostream_error_category@2@A@@YAXXZ 10001540 f   SamtoolMpileupWorker.obj
 0001:00000550       ??__E?_System_object@?$_Error_objects@H@std@@2V_System_error_category@2@A@@YAXXZ 10001550 f   SamtoolMpileupWorker.obj
 0001:00000560       ??__EACGT_ONLY@LocalWorkflow@U2@@YAXXZ 10001560 f   SamtoolMpileupWorker.obj
 0001:00000580       ??__EASSEMBLY_PORT_ID@LocalWorkflow@U2@@YAXXZ 10001580 f   SamtoolMpileupWorker.obj
 0001:000005a0       ??__EBCF_BED@LocalWorkflow@U2@@YAXXZ 100015a0 f   SamtoolMpileupWorker.obj
 0001:000005c0       ??__EBED@LocalWorkflow@U2@@YAXXZ 100015c0 f   SamtoolMpileupWorker.obj
 0001:000005e0       ??__ECALL_GT@LocalWorkflow@U2@@YAXXZ 100015e0 f   SamtoolMpileupWorker.obj
 0001:00000600       ??__ECAPQ_THRES@LocalWorkflow@U2@@YAXXZ 10001600 f   SamtoolMpileupWorker.obj
 0001:00000620       ??__ECCALL@LocalWorkflow@U2@@YAXXZ 10001620 f   SamtoolMpileupWorker.obj
 0001:00000640       ??__EDISABLE_BAQ@LocalWorkflow@U2@@YAXXZ 10001640 f   SamtoolMpileupWorker.obj
 0001:00000660       ??__EEXTQ@LocalWorkflow@U2@@YAXXZ 10001660 f   SamtoolMpileupWorker.obj
 0001:00000680       ??__EEXT_BAQ@LocalWorkflow@U2@@YAXXZ 10001680 f   SamtoolMpileupWorker.obj
 0001:000006a0       ??__EFIX_PL@LocalWorkflow@U2@@YAXXZ 100016a0 f   SamtoolMpileupWorker.obj
 0001:000006c0       ??__EGAP_SIZE@LocalWorkflow@U2@@YAXXZ 100016c0 f   SamtoolMpileupWorker.obj
 0001:000006e0       ??__EILLUMINA13@LocalWorkflow@U2@@YAXXZ 100016e0 f   SamtoolMpileupWorker.obj
 0001:00000700       ??__EINDEL_FRAC@LocalWorkflow@U2@@YAXXZ 10001700 f   SamtoolMpileupWorker.obj
 0001:00000720       ??__EKEEPALT@LocalWorkflow@U2@@YAXXZ 10001720 f   SamtoolMpileupWorker.obj
 0001:00000740       ??__EMAX_DEP@LocalWorkflow@U2@@YAXXZ 10001740 f   SamtoolMpileupWorker.obj
 0001:00000760       ??__EMAX_DEPTH@LocalWorkflow@U2@@YAXXZ 10001760 f   SamtoolMpileupWorker.obj
 0001:00000780       ??__EMAX_INDEL_DEPTH@LocalWorkflow@U2@@YAXXZ 10001780 f   SamtoolMpileupWorker.obj
 0001:000007a0       ??__EMIN_ALT@LocalWorkflow@U2@@YAXXZ 100017a0 f   SamtoolMpileupWorker.obj
 0001:000007c0       ??__EMIN_BASEQ@LocalWorkflow@U2@@YAXXZ 100017c0 f   SamtoolMpileupWorker.obj
 0001:000007e0       ??__EMIN_DEP@LocalWorkflow@U2@@YAXXZ 100017e0 f   SamtoolMpileupWorker.obj
 0001:00000800       ??__EMIN_MQ@LocalWorkflow@U2@@YAXXZ 10001800 f   SamtoolMpileupWorker.obj
 0001:00000820       ??__EMIN_PERM_P@LocalWorkflow@U2@@YAXXZ 10001820 f   SamtoolMpileupWorker.obj
 0001:00000840       ??__EMIN_QUAL@LocalWorkflow@U2@@YAXXZ 10001840 f   SamtoolMpileupWorker.obj
 0001:00000860       ??__EMIN_SMPL_FRAC@LocalWorkflow@U2@@YAXXZ 10001860 f   SamtoolMpileupWorker.obj
 0001:00000880       ??__EN1@LocalWorkflow@U2@@YAXXZ 10001880 f   SamtoolMpileupWorker.obj
 0001:000008a0       ??__ENO_GENO@LocalWorkflow@U2@@YAXXZ 100018a0 f   SamtoolMpileupWorker.obj
 0001:000008c0       ??__ENO_INDEL@LocalWorkflow@U2@@YAXXZ 100018c0 f   SamtoolMpileupWorker.obj
 0001:000008e0       ??__EN_PERM@LocalWorkflow@U2@@YAXXZ 100018e0 f   SamtoolMpileupWorker.obj
 0001:00000900       ??__EOPENQ@LocalWorkflow@U2@@YAXXZ 10001900 f   SamtoolMpileupWorker.obj
 0001:00000920       ??__EOUT_URL@LocalWorkflow@U2@@YAXXZ 10001920 f   SamtoolMpileupWorker.obj
 0001:00000940       ??__EPL_LIST@LocalWorkflow@U2@@YAXXZ 10001940 f   SamtoolMpileupWorker.obj
 0001:00000960       ??__EPREF@LocalWorkflow@U2@@YAXXZ 10001960 f   SamtoolMpileupWorker.obj
 0001:00000980       ??__EPRINT@LocalWorkflow@U2@@YAXXZ 10001980 f   SamtoolMpileupWorker.obj
 0001:000009a0       ??__EPTYPE@LocalWorkflow@U2@@YAXXZ 100019a0 f   SamtoolMpileupWorker.obj
 0001:000009c0       ??__EPVALUE1@LocalWorkflow@U2@@YAXXZ 100019c0 f   SamtoolMpileupWorker.obj
 0001:000009e0       ??__EPVALUE2@LocalWorkflow@U2@@YAXXZ 100019e0 f   SamtoolMpileupWorker.obj
 0001:00000a00       ??__EPVALUE3@LocalWorkflow@U2@@YAXXZ 10001a00 f   SamtoolMpileupWorker.obj
 0001:00000a20       ??__EPVALUE4@LocalWorkflow@U2@@YAXXZ 10001a20 f   SamtoolMpileupWorker.obj
 0001:00000a40       ??__EPVALUE_HWE@LocalWorkflow@U2@@YAXXZ 10001a40 f   SamtoolMpileupWorker.obj
 0001:00000a60       ??__EQCALL@LocalWorkflow@U2@@YAXXZ 10001a60 f   SamtoolMpileupWorker.obj
 0001:00000a80       ??__EREF_SEQ_PORT_ID@LocalWorkflow@U2@@YAXXZ 10001a80 f   SamtoolMpileupWorker.obj
 0001:00000aa0       ??__EREF_SOURCE@LocalWorkflow@U2@@YAXXZ 10001aa0 f   SamtoolMpileupWorker.obj
 0001:00000ac0       ??__EREF_SOURCE_FILE@LocalWorkflow@U2@@YAXXZ 10001ac0 f   SamtoolMpileupWorker.obj
 0001:00000ae0       ??__EREF_SOURCE_PORT@LocalWorkflow@U2@@YAXXZ 10001ae0 f   SamtoolMpileupWorker.obj
 0001:00000b00       ??__EREF_URL@LocalWorkflow@U2@@YAXXZ 10001b00 f   SamtoolMpileupWorker.obj
 0001:00000b20       ??__EREG@LocalWorkflow@U2@@YAXXZ 10001b20 f   SamtoolMpileupWorker.obj
 0001:00000b40       ??__ESAMPLES@LocalWorkflow@U2@@YAXXZ 10001b40 f   SamtoolMpileupWorker.obj
 0001:00000b60       ??__ETANDEMQ@LocalWorkflow@U2@@YAXXZ 10001b60 f   SamtoolMpileupWorker.obj
 0001:00000b80       ??__ETHETA@LocalWorkflow@U2@@YAXXZ 10001b80 f   SamtoolMpileupWorker.obj
 0001:00000ba0       ??__EUSE_ORPHAN@LocalWorkflow@U2@@YAXXZ 10001ba0 f   SamtoolMpileupWorker.obj
 0001:00000bc0       ??__EWINDOW@LocalWorkflow@U2@@YAXXZ 10001bc0 f   SamtoolMpileupWorker.obj
 0001:00000be0       ??__EalgoLog@U2@@YAXXZ     10001be0 f   SamtoolMpileupWorker.obj
 0001:00000c60       ??__EcmdLog@U2@@YAXXZ      10001c60 f   SamtoolMpileupWorker.obj
 0001:00000ce0       ??__EcoreLog@U2@@YAXXZ     10001ce0 f   SamtoolMpileupWorker.obj
 0001:00000d60       ??__EioLog@U2@@YAXXZ       10001d60 f   SamtoolMpileupWorker.obj
 0001:00000de0       ??__EperfLog@U2@@YAXXZ     10001de0 f   SamtoolMpileupWorker.obj
 0001:00000e60       ??__EscriptLog@U2@@YAXXZ   10001e60 f   SamtoolMpileupWorker.obj
 0001:00000ee0       ??__EtaskLog@U2@@YAXXZ     10001ee0 f   SamtoolMpileupWorker.obj
 0001:00000f60       ??__EuiLog@U2@@YAXXZ       10001f60 f   SamtoolMpileupWorker.obj
 0001:00000fe0       ??__EuserActLog@U2@@YAXXZ  10001fe0 f   SamtoolMpileupWorker.obj
 0001:00001060       ??__E?_Generic_object@?$_Error_objects@H@std@@2V_Generic_error_category@2@A@@YAXXZ 10002060 f   SamtoolsPlugin.obj
 0001:00001070       ??__E?_Iostream_object@?$_Error_objects@H@std@@2V_Iostream_error_category@2@A@@YAXXZ 10002070 f   SamtoolsPlugin.obj
 0001:00001080       ??__E?_System_object@?$_Error_objects@H@std@@2V_System_error_category@2@A@@YAXXZ 10002080 f   SamtoolsPlugin.obj
 0001:00001090       ??__EalgoLog@U2@@YAXXZ     10002090 f   SamtoolsPlugin.obj
 0001:00001110       ??__EcmdLog@U2@@YAXXZ      10002110 f   SamtoolsPlugin.obj
 0001:00001190       ??__EcoreLog@U2@@YAXXZ     10002190 f   SamtoolsPlugin.obj
 0001:00001210       ??__EioLog@U2@@YAXXZ       10002210 f   SamtoolsPlugin.obj
 0001:00001290       ??__EperfLog@U2@@YAXXZ     10002290 f   SamtoolsPlugin.obj
 0001:00001310       ??__EscriptLog@U2@@YAXXZ   10002310 f   SamtoolsPlugin.obj
 0001:00001390       ??__EtaskLog@U2@@YAXXZ     10002390 f   SamtoolsPlugin.obj
 0001:00001410       ??__EuiLog@U2@@YAXXZ       10002410 f   SamtoolsPlugin.obj
 0001:00001490       ??__EuserActLog@U2@@YAXXZ  10002490 f   SamtoolsPlugin.obj
 0001:00001510       ??__E?_Generic_object@?$_Error_objects@H@std@@2V_Generic_error_category@2@A@@YAXXZ 10002510 f   moc_AssemblySamtoolsMpileup.obj
 0001:00001520       ??__E?_Iostream_object@?$_Error_objects@H@std@@2V_Iostream_error_category@2@A@@YAXXZ 10002520 f   moc_AssemblySamtoolsMpileup.obj
 0001:00001530       ??__E?_System_object@?$_Error_objects@H@std@@2V_System_error_category@2@A@@YAXXZ 10002530 f   moc_AssemblySamtoolsMpileup.obj
 0001:00001540       ??__E?staticMetaObject@CallVariantsTask@LocalWorkflow@U2@@2UQMetaObject@@B@@YAXXZ 10002540 f   moc_AssemblySamtoolsMpileup.obj
 0001:00001550       ??__E?staticMetaObject@SamtoolsMpileupTask@LocalWorkflow@U2@@2UQMetaObject@@B@@YAXXZ 10002550 f   moc_AssemblySamtoolsMpileup.obj
 0001:00001560       ??__EalgoLog@U2@@YAXXZ     10002560 f   moc_AssemblySamtoolsMpileup.obj
 0001:000015e0       ??__EcmdLog@U2@@YAXXZ      100025e0 f   moc_AssemblySamtoolsMpileup.obj
 0001:00001660       ??__EcoreLog@U2@@YAXXZ     10002660 f   moc_AssemblySamtoolsMpileup.obj
 0001:000016e0       ??__EioLog@U2@@YAXXZ       100026e0 f   moc_AssemblySamtoolsMpileup.obj
 0001:00001760       ??__EperfLog@U2@@YAXXZ     10002760 f   moc_AssemblySamtoolsMpileup.obj
 0001:000017e0       ??__EscriptLog@U2@@YAXXZ   100027e0 f   moc_AssemblySamtoolsMpileup.obj
 0001:00001860       ??__EtaskLog@U2@@YAXXZ     10002860 f   moc_AssemblySamtoolsMpileup.obj
 0001:000018e0       ??__EuiLog@U2@@YAXXZ       100028e0 f   moc_AssemblySamtoolsMpileup.obj
 0001:00001960       ??__EuserActLog@U2@@YAXXZ  10002960 f   moc_AssemblySamtoolsMpileup.obj
 0001:000019e0       ??__E?_Generic_object@?$_Error_objects@H@std@@2V_Generic_error_category@2@A@@YAXXZ 100029e0 f   moc_SamtoolMpileupWorker.obj
 0001:000019f0       ??__E?_Iostream_object@?$_Error_objects@H@std@@2V_Iostream_error_category@2@A@@YAXXZ 100029f0 f   moc_SamtoolMpileupWorker.obj
 0001:00001a00       ??__E?_System_object@?$_Error_objects@H@std@@2V_System_error_category@2@A@@YAXXZ 10002a00 f   moc_SamtoolMpileupWorker.obj
 0001:00001a10       ??__E?staticMetaObject@CallVariantsPrompter@LocalWorkflow@U2@@2UQMetaObject@@B@@YAXXZ 10002a10 f   moc_SamtoolMpileupWorker.obj
 0001:00001a20       ??__E?staticMetaObject@CallVariantsWorker@LocalWorkflow@U2@@2UQMetaObject@@B@@YAXXZ 10002a20 f   moc_SamtoolMpileupWorker.obj
 0001:00001a30       ??__E?staticMetaObject@ScientificDoubleWidget@LocalWorkflow@U2@@2UQMetaObject@@B@@YAXXZ 10002a30 f   moc_SamtoolMpileupWorker.obj
 0001:00001a40       ??__EalgoLog@U2@@YAXXZ     10002a40 f   moc_SamtoolMpileupWorker.obj
 0001:00001ac0       ??__EcmdLog@U2@@YAXXZ      10002ac0 f   moc_SamtoolMpileupWorker.obj
 0001:00001b40       ??__EcoreLog@U2@@YAXXZ     10002b40 f   moc_SamtoolMpileupWorker.obj
 0001:00001bc0       ??__EioLog@U2@@YAXXZ       10002bc0 f   moc_SamtoolMpileupWorker.obj
 0001:00001c40       ??__EperfLog@U2@@YAXXZ     10002c40 f   moc_SamtoolMpileupWorker.obj
 0001:00001cc0       ??__EscriptLog@U2@@YAXXZ   10002cc0 f   moc_SamtoolMpileupWorker.obj
 0001:00001d40       ??__EtaskLog@U2@@YAXXZ     10002d40 f   moc_SamtoolMpileupWorker.obj
 0001:00001dc0       ??__EuiLog@U2@@YAXXZ       10002dc0 f   moc_SamtoolMpileupWorker.obj
 0001:00001e40       ??__EuserActLog@U2@@YAXXZ  10002e40 f   moc_SamtoolMpileupWorker.obj
 0001:00001ec0       ??__E?_Generic_object@?$_Error_objects@H@std@@2V_Generic_error_category@2@A@@YAXXZ 10002ec0 f   moc_SamtoolsPlugin.obj
 0001:00001ed0       ??__E?_Iostream_object@?$_Error_objects@H@std@@2V_Iostream_error_category@2@A@@YAXXZ 10002ed0 f   moc_SamtoolsPlugin.obj
 0001:00001ee0       ??__E?_System_object@?$_Error_objects@H@std@@2V_System_error_category@2@A@@YAXXZ 10002ee0 f   moc_SamtoolsPlugin.obj
 0001:00001ef0       ??__E?staticMetaObject@SamtoolsPlugin@U2@@2UQMetaObject@@B@@YAXXZ 10002ef0 f   moc_SamtoolsPlugin.obj
 0001:000024fe       __catch$??0?$QList@PAVGObject@U2@@@@QAE@ABV0@@Z$0 100034fe f i AssemblySamtoolsMpileup.obj
 0001:000025fe       __catch$??0?$QList@VQString@@@@QAE@ABV0@@Z$0 100035fe f i AssemblySamtoolsMpileup.obj
 0001:0000356a       __catch$??Y?$QList@VQString@@@@QAEAAV0@ABV0@@Z$0 1000456a f i AssemblySamtoolsMpileup.obj
 0001:00003c86       __catch$?_Copy@?$basic_string@DU?$char_traits@D@std@@V?$allocator@D@2@@std@@QAEXII@Z$0 10004c86 f i AssemblySamtoolsMpileup.obj
 0001:00003cc3       __catch$?_Copy@?$basic_string@DU?$char_traits@D@std@@V?$allocator@D@2@@std@@QAEXII@Z$1 10004cc3 f i AssemblySamtoolsMpileup.obj
 0001:00003fe5       __catch$?append@?$QList@PAVTask@U2@@@@QAEXABQAVTask@U2@@@Z$4 10004fe5 f i AssemblySamtoolsMpileup.obj
 0001:0000408f       __catch$?append@?$QList@V?$QMap@VQString@@VQVariant@@@@@@QAEXABV?$QMap@VQString@@VQVariant@@@@@Z$0 1000508f f i AssemblySamtoolsMpileup.obj
 0001:0000408f       __catch$?append@?$QList@V?$QMap@VQString@@VQVariant@@@@@@QAEXABV?$QMap@VQString@@VQVariant@@@@@Z$2 1000508f f i AssemblySamtoolsMpileup.obj
 0001:0000414d       __catch$?append@?$QList@VQString@@@@QAEXABVQString@@@Z$0 1000514d f i AssemblySamtoolsMpileup.obj
 0001:0000419e       __catch$?append@?$QList@VQString@@@@QAEXABVQString@@@Z$4 1000519e f i AssemblySamtoolsMpileup.obj
 0001:000047be       __catch$?createNode@?$QMapData@VQString@@VQVariant@@@@QAEPAU?$QMapNode@VQString@@VQVariant@@@@ABVQString@@ABVQVariant@@PAU2@_N@Z$0 100057be f i AssemblySamtoolsMpileup.obj
 0001:000047d3       __catch$?createNode@?$QMapData@VQString@@VQVariant@@@@QAEPAU?$QMapNode@VQString@@VQVariant@@@@ABVQString@@ABVQVariant@@PAU2@_N@Z$2 100057d3 f i AssemblySamtoolsMpileup.obj
 0001:00004b2a       __catch$?detach_helper@?$QList@VFormatDetectionResult@U2@@@@AAEXH@Z$0 10005b2a f i AssemblySamtoolsMpileup.obj
 0001:00004cd1       __catch$?detach_helper_grow@?$QList@PAVTask@U2@@@@AAEPAUNode@1@HH@Z$0 10005cd1 f i AssemblySamtoolsMpileup.obj
 0001:00004cd1       __catch$?detach_helper_grow@?$QList@PAVTask@U2@@@@AAEPAUNode@1@HH@Z$2 10005cd1 f i AssemblySamtoolsMpileup.obj
 0001:00004dfc       __catch$?detach_helper_grow@?$QList@V?$QMap@VQString@@VQVariant@@@@@@AAEPAUNode@1@HH@Z$2 10005dfc f i AssemblySamtoolsMpileup.obj
 0001:00004e37       __catch$?detach_helper_grow@?$QList@V?$QMap@VQString@@VQVariant@@@@@@AAEPAUNode@1@HH@Z$0 10005e37 f i AssemblySamtoolsMpileup.obj
 0001:00004f7e       __catch$?detach_helper_grow@?$QList@VQString@@@@AAEPAUNode@1@HH@Z$2 10005f7e f i AssemblySamtoolsMpileup.obj
 0001:00004fb9       __catch$?detach_helper_grow@?$QList@VQString@@@@AAEPAUNode@1@HH@Z$0 10005fb9 f i AssemblySamtoolsMpileup.obj
 0001:000069c1       __catch$?node_copy@?$QList@V?$QMap@VQString@@VQVariant@@@@@@AAEXPAUNode@1@00@Z$0 100079c1 f i AssemblySamtoolsMpileup.obj
 0001:00006a8e       __catch$?node_copy@?$QList@VFormatDetectionResult@U2@@@@AAEXPAUNode@1@00@Z$0 10007a8e f i AssemblySamtoolsMpileup.obj
 0001:00006b42       __catch$?node_copy@?$QList@VQString@@@@AAEXPAUNode@1@00@Z$2 10007b42 f i AssemblySamtoolsMpileup.obj
 0001:000097ce       __catch$??0?$QList@PAVPort@Workflow@U2@@@@QAE@ABV0@@Z$0 1000a7ce f i SamtoolMpileupWorker.obj
 0001:0000989e       __catch$??0?$QList@V?$QMap@VQString@@VQVariant@@@@@@QAE@ABV0@@Z$0 1000a89e f i SamtoolMpileupWorker.obj
 0001:0000997e       __catch$??0?$QList@VDescriptor@U2@@@@QAE@ABV0@@Z$0 1000a97e f i SamtoolMpileupWorker.obj
 0001:0000b285       __catch$?append@?$QList@PAVAttribute@U2@@@@QAEXABQAVAttribute@U2@@@Z$4 1000c285 f i SamtoolMpileupWorker.obj
 0001:0000b315       __catch$?append@?$QList@PAVPortDescriptor@Workflow@U2@@@@QAEXABQAVPortDescriptor@Workflow@U2@@@Z$4 1000c315 f i SamtoolMpileupWorker.obj
 0001:0000b3cc       __catch$?append@?$QList@VDescriptor@U2@@@@QAEXABVDescriptor@U2@@@Z$0 1000c3cc f i SamtoolMpileupWorker.obj
 0001:0000b3cc       __catch$?append@?$QList@VDescriptor@U2@@@@QAEXABVDescriptor@U2@@@Z$2 1000c3cc f i SamtoolMpileupWorker.obj
 0001:0000b4b0       __catch$?append@?$QList@VMessage@Workflow@U2@@@@QAEXABVMessage@Workflow@U2@@@Z$2 1000c4b0 f i SamtoolMpileupWorker.obj
 0001:0000b4b0       __catch$?append@?$QList@VMessage@Workflow@U2@@@@QAEXABVMessage@Workflow@U2@@@Z$0 1000c4b0 f i SamtoolMpileupWorker.obj
 0001:0000b590       __catch$?append@?$QList@VQVariant@@@@QAEXABVQVariant@@@Z$2 1000c590 f i SamtoolMpileupWorker.obj
 0001:0000b590       __catch$?append@?$QList@VQVariant@@@@QAEXABVQVariant@@@Z$0 1000c590 f i SamtoolMpileupWorker.obj
 0001:0000b670       __catch$?append@?$QList@VWorkflowNotification@U2@@@@QAEXABVWorkflowNotification@U2@@@Z$2 1000c670 f i SamtoolMpileupWorker.obj
 0001:0000b670       __catch$?append@?$QList@VWorkflowNotification@U2@@@@QAEXABVWorkflowNotification@U2@@@Z$0 1000c670 f i SamtoolMpileupWorker.obj
 0001:0000c69d       __catch$?createNode@?$QMapData@VDescriptor@U2@@V?$QExplicitlySharedDataPointer@VDataType@U2@@@@@@QAEPAU?$QMapNode@VDescriptor@U2@@V?$QExplicitlySharedDataPointer@VDataType@U2@@@@@@ABVDescriptor@U2@@ABV?$QExplicitlySharedDataPointer@VDataType@U2@@@@PAU2@_N@Z$2 1000d69d f i SamtoolMpileupWorker.obj
 0001:0000c745       __catch$?createNode@?$QMapData@VQString@@PAVPropertyDelegate@U2@@@@QAEPAU?$QMapNode@VQString@@PAVPropertyDelegate@U2@@@@ABVQString@@ABQAVPropertyDelegate@U2@@PAU2@_N@Z$2 1000d745 f i SamtoolMpileupWorker.obj
 0001:0000c7ee       __catch$?createNode@?$QMapData@VQString@@V1@@@QAEPAU?$QMapNode@VQString@@V1@@@ABVQString@@0PAU2@_N@Z$0 1000d7ee f i SamtoolMpileupWorker.obj
 0001:0000c803       __catch$?createNode@?$QMapData@VQString@@V1@@@QAEPAU?$QMapNode@VQString@@V1@@@ABVQString@@0PAU2@_N@Z$2 1000d803 f i SamtoolMpileupWorker.obj
 0001:0000c8ae       __catch$?createNode@?$QMapData@VQString@@VQScriptValue@@@@QAEPAU?$QMapNode@VQString@@VQScriptValue@@@@ABVQString@@ABVQScriptValue@@PAU2@_N@Z$0 1000d8ae f i SamtoolMpileupWorker.obj
 0001:0000c8c3       __catch$?createNode@?$QMapData@VQString@@VQScriptValue@@@@QAEPAU?$QMapNode@VQString@@VQScriptValue@@@@ABVQString@@ABVQScriptValue@@PAU2@_N@Z$2 1000d8c3 f i SamtoolMpileupWorker.obj
 0001:0000ceea       __catch$?detach_helper@?$QList@VDescriptor@U2@@@@AAEXH@Z$0 1000deea f i SamtoolMpileupWorker.obj
 0001:0000cfba       __catch$?detach_helper@?$QList@VMessage@Workflow@U2@@@@AAEXH@Z$0 1000dfba f i SamtoolMpileupWorker.obj
 0001:0000d291       __catch$?detach_helper_grow@?$QList@PAVAttribute@U2@@@@AAEPAUNode@1@HH@Z$0 1000e291 f i SamtoolMpileupWorker.obj
 0001:0000d291       __catch$?detach_helper_grow@?$QList@PAVAttribute@U2@@@@AAEPAUNode@1@HH@Z$2 1000e291 f i SamtoolMpileupWorker.obj
 0001:0000d3a1       __catch$?detach_helper_grow@?$QList@PAVPortDescriptor@Workflow@U2@@@@AAEPAUNode@1@HH@Z$2 1000e3a1 f i SamtoolMpileupWorker.obj
 0001:0000d3a1       __catch$?detach_helper_grow@?$QList@PAVPortDescriptor@Workflow@U2@@@@AAEPAUNode@1@HH@Z$0 1000e3a1 f i SamtoolMpileupWorker.obj
 0001:0000d4af       __catch$?detach_helper_grow@?$QList@VDescriptor@U2@@@@AAEPAUNode@1@HH@Z$2 1000e4af f i SamtoolMpileupWorker.obj
 0001:0000d4ea       __catch$?detach_helper_grow@?$QList@VDescriptor@U2@@@@AAEPAUNode@1@HH@Z$0 1000e4ea f i SamtoolMpileupWorker.obj
 0001:0000d5ff       __catch$?detach_helper_grow@?$QList@VMessage@Workflow@U2@@@@AAEPAUNode@1@HH@Z$2 1000e5ff f i SamtoolMpileupWorker.obj
 0001:0000d63a       __catch$?detach_helper_grow@?$QList@VMessage@Workflow@U2@@@@AAEPAUNode@1@HH@Z$0 1000e63a f i SamtoolMpileupWorker.obj
 0001:0000d74f       __catch$?detach_helper_grow@?$QList@VQVariant@@@@AAEPAUNode@1@HH@Z$2 1000e74f f i SamtoolMpileupWorker.obj
 0001:0000d78a       __catch$?detach_helper_grow@?$QList@VQVariant@@@@AAEPAUNode@1@HH@Z$0 1000e78a f i SamtoolMpileupWorker.obj
 0001:0000d89f       __catch$?detach_helper_grow@?$QList@VWorkflowNotification@U2@@@@AAEPAUNode@1@HH@Z$2 1000e89f f i SamtoolMpileupWorker.obj
 0001:0000d8da       __catch$?detach_helper_grow@?$QList@VWorkflowNotification@U2@@@@AAEPAUNode@1@HH@Z$0 1000e8da f i SamtoolMpileupWorker.obj
 0001:00016325       __catch$?node_copy@?$QList@VDescriptor@U2@@@@AAEXPAUNode@1@00@Z$0 10017325 f i SamtoolMpileupWorker.obj
 0001:000163ee       __catch$?node_copy@?$QList@VMessage@Workflow@U2@@@@AAEXPAUNode@1@00@Z$0 100173ee f i SamtoolMpileupWorker.obj
 0001:000164be       __catch$?node_copy@?$QList@VQVariant@@@@AAEXPAUNode@1@00@Z$0 100174be f i SamtoolMpileupWorker.obj
 0001:0001658e       __catch$?node_copy@?$QList@VWorkflowNotification@U2@@@@AAEXPAUNode@1@00@Z$0 1001758e f i SamtoolMpileupWorker.obj
 0001:000190c0       _pre_c_init                1001a0c0 f   MSVCRT:crtdll.obj
 0001:0001932d       ___DllMainCRTStartup       1001a32d f   MSVCRT:crtdll.obj
 0001:00019480       $$000000                   1001a480     MSVCRT:sehprolg4.obj
 0001:00019895       ?ArrayUnwindFilter@@YAHPAU_EXCEPTION_POINTERS@@@Z 1001a895 f   MSVCRT:ehvecdtr.obj
 0001:00019be0       __unwindfunclet$??$qRegisterMetaType@V?$QSharedDataPointer@VDbiDataHandler@Workflow@U2@@@@@@YAHPBDPAV?$QSharedDataPointer@VDbiDataHandler@Workflow@U2@@@@W4DefinedType@?$MetaTypeDefinedHelper@V?$QSharedDataPointer@VDbiDataHandler@Workflow@U2@@@@$00@QtPrivate@@@Z$0 1001abe0 f   AssemblySamtoolsMpileup.obj
 0001:00019be9       __ehhandler$??$qRegisterMetaType@V?$QSharedDataPointer@VDbiDataHandler@Workflow@U2@@@@@@YAHPBDPAV?$QSharedDataPointer@VDbiDataHandler@Workflow@U2@@@@W4DefinedType@?$MetaTypeDefinedHelper@V?$QSharedDataPointer@VDbiDataHandler@Workflow@U2@@@@$00@QtPrivate@@@Z 1001abe9 f   AssemblySamtoolsMpileup.obj
 0001:00019c10       __unwindfunclet$??$qRegisterMetaType@VU2DbiRef@U2@@@@YAHPBDPAVU2DbiRef@U2@@W4DefinedType@?$MetaTypeDefinedHelper@VU2DbiRef@U2@@$00@QtPrivate@@@Z$0 1001ac10 f   AssemblySamtoolsMpileup.obj
 0001:00019c19       __ehhandler$??$qRegisterMetaType@VU2DbiRef@U2@@@@YAHPBDPAVU2DbiRef@U2@@W4DefinedType@?$MetaTypeDefinedHelper@VU2DbiRef@U2@@$00@QtPrivate@@@Z 1001ac19 f   AssemblySamtoolsMpileup.obj
 0001:00019c40       __ehhandler$??0?$QList@PAVGObject@U2@@@@QAE@ABV0@@Z 1001ac40 f   AssemblySamtoolsMpileup.obj
 0001:00019c60       __ehhandler$??0?$QList@VQString@@@@QAE@ABV0@@Z 1001ac60 f   AssemblySamtoolsMpileup.obj
 0001:00019c80       __unwindfunclet$??0CallVariantsTask@LocalWorkflow@U2@@QAE@ABVCallVariantsTaskSettings@12@PAVDbiDataStorage@Workflow@2@@Z$0 1001ac80 f   AssemblySamtoolsMpileup.obj
 0001:00019c89       __unwindfunclet$??0CallVariantsTask@LocalWorkflow@U2@@QAE@ABVCallVariantsTaskSettings@12@PAVDbiDataStorage@Workflow@2@@Z$1 1001ac89 f   AssemblySamtoolsMpileup.obj
 0001:00019c92       __unwindfunclet$??0CallVariantsTask@LocalWorkflow@U2@@QAE@ABVCallVariantsTaskSettings@12@PAVDbiDataStorage@Workflow@2@@Z$2 1001ac92 f   AssemblySamtoolsMpileup.obj
 0001:00019c9b       __unwindfunclet$??0CallVariantsTask@LocalWorkflow@U2@@QAE@ABVCallVariantsTaskSettings@12@PAVDbiDataStorage@Workflow@2@@Z$3 1001ac9b f   AssemblySamtoolsMpileup.obj
 0001:00019ca9       __unwindfunclet$??0CallVariantsTask@LocalWorkflow@U2@@QAE@ABVCallVariantsTaskSettings@12@PAVDbiDataStorage@Workflow@2@@Z$4 1001aca9 f   AssemblySamtoolsMpileup.obj
 0001:00019cb7       __unwindfunclet$??0CallVariantsTask@LocalWorkflow@U2@@QAE@ABVCallVariantsTaskSettings@12@PAVDbiDataStorage@Workflow@2@@Z$5 1001acb7 f   AssemblySamtoolsMpileup.obj
 0001:00019cc5       __unwindfunclet$??0CallVariantsTask@LocalWorkflow@U2@@QAE@ABVCallVariantsTaskSettings@12@PAVDbiDataStorage@Workflow@2@@Z$6 1001acc5 f   AssemblySamtoolsMpileup.obj
 0001:00019cce       __unwindfunclet$??0CallVariantsTask@LocalWorkflow@U2@@QAE@ABVCallVariantsTaskSettings@12@PAVDbiDataStorage@Workflow@2@@Z$7 1001acce f   AssemblySamtoolsMpileup.obj
 0001:00019cd7       __unwindfunclet$??0CallVariantsTask@LocalWorkflow@U2@@QAE@ABVCallVariantsTaskSettings@12@PAVDbiDataStorage@Workflow@2@@Z$8 1001acd7 f   AssemblySamtoolsMpileup.obj
 0001:00019ce0       __ehhandler$??0CallVariantsTask@LocalWorkflow@U2@@QAE@ABVCallVariantsTaskSettings@12@PAVDbiDataStorage@Workflow@2@@Z 1001ace0 f   AssemblySamtoolsMpileup.obj
 0001:00019d00       __unwindfunclet$??0CallVariantsTaskSettings@LocalWorkflow@U2@@QAE@ABV012@@Z$0 1001ad00 f   AssemblySamtoolsMpileup.obj
 0001:00019d09       __unwindfunclet$??0CallVariantsTaskSettings@LocalWorkflow@U2@@QAE@ABV012@@Z$1 1001ad09 f   AssemblySamtoolsMpileup.obj
 0001:00019d14       __unwindfunclet$??0CallVariantsTaskSettings@LocalWorkflow@U2@@QAE@ABV012@@Z$2 1001ad14 f   AssemblySamtoolsMpileup.obj
 0001:00019d20       __unwindfunclet$??0CallVariantsTaskSettings@LocalWorkflow@U2@@QAE@ABV012@@Z$3 1001ad20 f   AssemblySamtoolsMpileup.obj
 0001:00019d2c       __unwindfunclet$??0CallVariantsTaskSettings@LocalWorkflow@U2@@QAE@ABV012@@Z$4 1001ad2c f   AssemblySamtoolsMpileup.obj
 0001:00019d38       __unwindfunclet$??0CallVariantsTaskSettings@LocalWorkflow@U2@@QAE@ABV012@@Z$5 1001ad38 f   AssemblySamtoolsMpileup.obj
 0001:00019d44       __unwindfunclet$??0CallVariantsTaskSettings@LocalWorkflow@U2@@QAE@ABV012@@Z$6 1001ad44 f   AssemblySamtoolsMpileup.obj
 0001:00019d50       __unwindfunclet$??0CallVariantsTaskSettings@LocalWorkflow@U2@@QAE@ABV012@@Z$7 1001ad50 f   AssemblySamtoolsMpileup.obj
 0001:00019d5c       __unwindfunclet$??0CallVariantsTaskSettings@LocalWorkflow@U2@@QAE@ABV012@@Z$8 1001ad5c f   AssemblySamtoolsMpileup.obj
 0001:00019d68       __ehhandler$??0CallVariantsTaskSettings@LocalWorkflow@U2@@QAE@ABV012@@Z 1001ad68 f   AssemblySamtoolsMpileup.obj
 0001:00019d90       __unwindfunclet$??0SamtoolsMpileupTask@LocalWorkflow@U2@@QAE@ABVCallVariantsTaskSettings@12@@Z$0 1001ad90 f   AssemblySamtoolsMpileup.obj
 0001:00019d99       __unwindfunclet$??0SamtoolsMpileupTask@LocalWorkflow@U2@@QAE@ABVCallVariantsTaskSettings@12@@Z$1 1001ad99 f   AssemblySamtoolsMpileup.obj
 0001:00019da2       __unwindfunclet$??0SamtoolsMpileupTask@LocalWorkflow@U2@@QAE@ABVCallVariantsTaskSettings@12@@Z$2 1001ada2 f   AssemblySamtoolsMpileup.obj
 0001:00019dab       __ehhandler$??0SamtoolsMpileupTask@LocalWorkflow@U2@@QAE@ABVCallVariantsTaskSettings@12@@Z 1001adab f   AssemblySamtoolsMpileup.obj
 0001:00019dd0       __unwindfunclet$??1CallVariantsTask@LocalWorkflow@U2@@UAE@XZ$0 1001add0 f   AssemblySamtoolsMpileup.obj
 0001:00019dd9       __unwindfunclet$??1CallVariantsTask@LocalWorkflow@U2@@UAE@XZ$1 1001add9 f   AssemblySamtoolsMpileup.obj
 0001:00019de7       __ehhandler$??1CallVariantsTask@LocalWorkflow@U2@@UAE@XZ 1001ade7 f   AssemblySamtoolsMpileup.obj
 0001:00019e10       __unwindfunclet$??1CallVariantsTaskSettings@LocalWorkflow@U2@@QAE@XZ$0 1001ae10 f   AssemblySamtoolsMpileup.obj
 0001:00019e19       __unwindfunclet$??1CallVariantsTaskSettings@LocalWorkflow@U2@@QAE@XZ$1 1001ae19 f   AssemblySamtoolsMpileup.obj
 0001:00019e24       __unwindfunclet$??1CallVariantsTaskSettings@LocalWorkflow@U2@@QAE@XZ$2 1001ae24 f   AssemblySamtoolsMpileup.obj
 0001:00019e30       __unwindfunclet$??1CallVariantsTaskSettings@LocalWorkflow@U2@@QAE@XZ$3 1001ae30 f   AssemblySamtoolsMpileup.obj
 0001:00019e3c       __unwindfunclet$??1CallVariantsTaskSettings@LocalWorkflow@U2@@QAE@XZ$4 1001ae3c f   AssemblySamtoolsMpileup.obj
 0001:00019e48       __unwindfunclet$??1CallVariantsTaskSettings@LocalWorkflow@U2@@QAE@XZ$5 1001ae48 f   AssemblySamtoolsMpileup.obj
 0001:00019e54       __unwindfunclet$??1CallVariantsTaskSettings@LocalWorkflow@U2@@QAE@XZ$6 1001ae54 f   AssemblySamtoolsMpileup.obj
 0001:00019e60       __unwindfunclet$??1CallVariantsTaskSettings@LocalWorkflow@U2@@QAE@XZ$7 1001ae60 f   AssemblySamtoolsMpileup.obj
 0001:00019e6c       __unwindfunclet$??1CallVariantsTaskSettings@LocalWorkflow@U2@@QAE@XZ$8 1001ae6c f   AssemblySamtoolsMpileup.obj
 0001:00019e78       __ehhandler$??1CallVariantsTaskSettings@LocalWorkflow@U2@@QAE@XZ 1001ae78 f   AssemblySamtoolsMpileup.obj
 0001:00019ea0       __unwindfunclet$??1SamtoolsMpileupTask@LocalWorkflow@U2@@UAE@XZ$0 1001aea0 f   AssemblySamtoolsMpileup.obj
 0001:00019ea9       __ehhandler$??1SamtoolsMpileupTask@LocalWorkflow@U2@@UAE@XZ 1001aea9 f   AssemblySamtoolsMpileup.obj
 0001:00019ed0       __unwindfunclet$??A?$QMap@VQString@@VQVariant@@@@QAEAAVQVariant@@ABVQString@@@Z$0 1001aed0 f   AssemblySamtoolsMpileup.obj
 0001:00019ed9       __ehhandler$??A?$QMap@VQString@@VQVariant@@@@QAEAAVQVariant@@ABVQString@@@Z 1001aed9 f   AssemblySamtoolsMpileup.obj
 0001:00019f00       __unwindfunclet$??H@YA?BVQString@@ABV0@0@Z$0 1001af00 f   AssemblySamtoolsMpileup.obj
 0001:00019f1a       __ehhandler$??H@YA?BVQString@@ABV0@0@Z 1001af1a f   AssemblySamtoolsMpileup.obj
 0001:00019f40       __ehhandler$??Y?$QList@VQString@@@@QAEAAV0@ABV0@@Z 1001af40 f   AssemblySamtoolsMpileup.obj
 0001:00019f60       __unwindfunclet$??_GSamtoolsMpileupTask@LocalWorkflow@U2@@UAEPAXI@Z$0 1001af60 f   AssemblySamtoolsMpileup.obj
 0001:00019f69       __ehhandler$??_GSamtoolsMpileupTask@LocalWorkflow@U2@@UAEPAXI@Z 1001af69 f   AssemblySamtoolsMpileup.obj
 0001:00019f90       __unwindfunclet$??__EalgoLog@U2@@YAXXZ$0 1001af90 f   AssemblySamtoolsMpileup.obj
 0001:00019f99       __ehhandler$??__EalgoLog@U2@@YAXXZ 1001af99 f   AssemblySamtoolsMpileup.obj
 0001:00019fc0       __unwindfunclet$??__EcmdLog@U2@@YAXXZ$0 1001afc0 f   AssemblySamtoolsMpileup.obj
 0001:00019fc9       __ehhandler$??__EcmdLog@U2@@YAXXZ 1001afc9 f   AssemblySamtoolsMpileup.obj
 0001:00019ff0       __unwindfunclet$??__EcoreLog@U2@@YAXXZ$0 1001aff0 f   AssemblySamtoolsMpileup.obj
 0001:00019ff9       __ehhandler$??__EcoreLog@U2@@YAXXZ 1001aff9 f   AssemblySamtoolsMpileup.obj
 0001:0001a020       __unwindfunclet$??__EioLog@U2@@YAXXZ$0 1001b020 f   AssemblySamtoolsMpileup.obj
 0001:0001a029       __ehhandler$??__EioLog@U2@@YAXXZ 1001b029 f   AssemblySamtoolsMpileup.obj
 0001:0001a050       __unwindfunclet$??__EperfLog@U2@@YAXXZ$0 1001b050 f   AssemblySamtoolsMpileup.obj
 0001:0001a059       __ehhandler$??__EperfLog@U2@@YAXXZ 1001b059 f   AssemblySamtoolsMpileup.obj
 0001:0001a080       __unwindfunclet$??__EscriptLog@U2@@YAXXZ$0 1001b080 f   AssemblySamtoolsMpileup.obj
 0001:0001a089       __ehhandler$??__EscriptLog@U2@@YAXXZ 1001b089 f   AssemblySamtoolsMpileup.obj
 0001:0001a0b0       __unwindfunclet$??__EtaskLog@U2@@YAXXZ$0 1001b0b0 f   AssemblySamtoolsMpileup.obj
 0001:0001a0b9       __ehhandler$??__EtaskLog@U2@@YAXXZ 1001b0b9 f   AssemblySamtoolsMpileup.obj
 0001:0001a0e0       __unwindfunclet$??__EuiLog@U2@@YAXXZ$0 1001b0e0 f   AssemblySamtoolsMpileup.obj
 0001:0001a0e9       __ehhandler$??__EuiLog@U2@@YAXXZ 1001b0e9 f   AssemblySamtoolsMpileup.obj
 0001:0001a110       __unwindfunclet$??__EuserActLog@U2@@YAXXZ$0 1001b110 f   AssemblySamtoolsMpileup.obj
 0001:0001a119       __ehhandler$??__EuserActLog@U2@@YAXXZ 1001b119 f   AssemblySamtoolsMpileup.obj
 0001:0001a140       __unwindfunclet$?Construct@?$QMetaTypeFunctionHelper@VU2DbiRef@U2@@$00@QtMetaTypePrivate@@SAPAXPAXPBX@Z$0 1001b140 f   AssemblySamtoolsMpileup.obj
 0001:0001a151       __unwindfunclet$?Construct@?$QMetaTypeFunctionHelper@VU2DbiRef@U2@@$00@QtMetaTypePrivate@@SAPAXPAXPBX@Z$1 1001b151 f   AssemblySamtoolsMpileup.obj
 0001:0001a162       __unwindfunclet$?Construct@?$QMetaTypeFunctionHelper@VU2DbiRef@U2@@$00@QtMetaTypePrivate@@SAPAXPAXPBX@Z$2 1001b162 f   AssemblySamtoolsMpileup.obj
 0001:0001a17c       __unwindfunclet$?Construct@?$QMetaTypeFunctionHelper@VU2DbiRef@U2@@$00@QtMetaTypePrivate@@SAPAXPAXPBX@Z$3 1001b17c f   AssemblySamtoolsMpileup.obj
 0001:0001a196       __ehhandler$?Construct@?$QMetaTypeFunctionHelper@VU2DbiRef@U2@@$00@QtMetaTypePrivate@@SAPAXPAXPBX@Z 1001b196 f   AssemblySamtoolsMpileup.obj
 0001:0001a1c0       __unwindfunclet$?Create@?$QMetaTypeFunctionHelper@VU2DbiRef@U2@@$00@QtMetaTypePrivate@@SAPAXPBX@Z$0 1001b1c0 f   AssemblySamtoolsMpileup.obj
 0001:0001a1cb       __unwindfunclet$?Create@?$QMetaTypeFunctionHelper@VU2DbiRef@U2@@$00@QtMetaTypePrivate@@SAPAXPBX@Z$1 1001b1cb f   AssemblySamtoolsMpileup.obj
 0001:0001a1d6       __unwindfunclet$?Create@?$QMetaTypeFunctionHelper@VU2DbiRef@U2@@$00@QtMetaTypePrivate@@SAPAXPBX@Z$2 1001b1d6 f   AssemblySamtoolsMpileup.obj
 0001:0001a1f0       __unwindfunclet$?Create@?$QMetaTypeFunctionHelper@VU2DbiRef@U2@@$00@QtMetaTypePrivate@@SAPAXPBX@Z$3 1001b1f0 f   AssemblySamtoolsMpileup.obj
 0001:0001a20a       __ehhandler$?Create@?$QMetaTypeFunctionHelper@VU2DbiRef@U2@@$00@QtMetaTypePrivate@@SAPAXPBX@Z 1001b20a f   AssemblySamtoolsMpileup.obj
 0001:0001a230       __ehhandler$?_Copy@?$basic_string@DU?$char_traits@D@std@@V?$allocator@D@2@@std@@QAEXII@Z 1001b230 f   AssemblySamtoolsMpileup.obj
 0001:0001a250       __ehhandler$?append@?$QList@PAVTask@U2@@@@QAEXABQAVTask@U2@@@Z 1001b250 f   AssemblySamtoolsMpileup.obj
 0001:0001a270       __unwindfunclet$?append@?$QList@V?$QMap@VQString@@VQVariant@@@@@@QAEXABV?$QMap@VQString@@VQVariant@@@@@Z$6 1001b270 f   AssemblySamtoolsMpileup.obj
 0001:0001a27b       __ehhandler$?append@?$QList@V?$QMap@VQString@@VQVariant@@@@@@QAEXABV?$QMap@VQString@@VQVariant@@@@@Z 1001b27b f   AssemblySamtoolsMpileup.obj
 0001:0001a2a0       __unwindfunclet$?append@?$QList@VQString@@@@QAEXABVQString@@@Z$7 1001b2a0 f   AssemblySamtoolsMpileup.obj
 0001:0001a2b1       __unwindfunclet$?append@?$QList@VQString@@@@QAEXABVQString@@@Z$11 1001b2b1 f   AssemblySamtoolsMpileup.obj
 0001:0001a2c2       __ehhandler$?append@?$QList@VQString@@@@QAEXABVQString@@@Z 1001b2c2 f   AssemblySamtoolsMpileup.obj
 0001:0001a2e0       __unwindfunclet$?checkExitCode@SamtoolsMpileupTask@LocalWorkflow@U2@@AAEXPAVQProcess@@ABVQString@@@Z$0 1001b2e0 f   AssemblySamtoolsMpileup.obj
 0001:0001a2e9       __unwindfunclet$?checkExitCode@SamtoolsMpileupTask@LocalWorkflow@U2@@AAEXPAVQProcess@@ABVQString@@@Z$1 1001b2e9 f   AssemblySamtoolsMpileup.obj
 0001:0001a2f2       __unwindfunclet$?checkExitCode@SamtoolsMpileupTask@LocalWorkflow@U2@@AAEXPAVQProcess@@ABVQString@@@Z$2 1001b2f2 f   AssemblySamtoolsMpileup.obj
 0001:0001a2fb       __unwindfunclet$?checkExitCode@SamtoolsMpileupTask@LocalWorkflow@U2@@AAEXPAVQProcess@@ABVQString@@@Z$3 1001b2fb f   AssemblySamtoolsMpileup.obj
 0001:0001a304       __unwindfunclet$?checkExitCode@SamtoolsMpileupTask@LocalWorkflow@U2@@AAEXPAVQProcess@@ABVQString@@@Z$4 1001b304 f   AssemblySamtoolsMpileup.obj
 0001:0001a30d       __ehhandler$?checkExitCode@SamtoolsMpileupTask@LocalWorkflow@U2@@AAEXPAVQProcess@@ABVQString@@@Z 1001b30d f   AssemblySamtoolsMpileup.obj
 0001:0001a330       __unwindfunclet$?createNode@?$QMapData@VQString@@VQVariant@@@@QAEPAU?$QMapNode@VQString@@VQVariant@@@@ABVQString@@ABVQVariant@@PAU2@_N@Z$4 1001b330 f   AssemblySamtoolsMpileup.obj
 0001:0001a344       __unwindfunclet$?createNode@?$QMapData@VQString@@VQVariant@@@@QAEPAU?$QMapNode@VQString@@VQVariant@@@@ABVQString@@ABVQVariant@@PAU2@_N@Z$5 1001b344 f   AssemblySamtoolsMpileup.obj
 0001:0001a358       __ehhandler$?createNode@?$QMapData@VQString@@VQVariant@@@@QAEPAU?$QMapNode@VQString@@VQVariant@@@@ABVQString@@ABVQVariant@@PAU2@_N@Z 1001b358 f   AssemblySamtoolsMpileup.obj
 0001:0001a380       __ehhandler$?detach_helper@?$QList@VFormatDetectionResult@U2@@@@AAEXH@Z 1001b380 f   AssemblySamtoolsMpileup.obj
 0001:0001a3a0       __ehhandler$?detach_helper_grow@?$QList@PAVTask@U2@@@@AAEPAUNode@1@HH@Z 1001b3a0 f   AssemblySamtoolsMpileup.obj
 0001:0001a3c0       __ehhandler$?detach_helper_grow@?$QList@V?$QMap@VQString@@VQVariant@@@@@@AAEPAUNode@1@HH@Z 1001b3c0 f   AssemblySamtoolsMpileup.obj
 0001:0001a3e0       __ehhandler$?detach_helper_grow@?$QList@VQString@@@@AAEPAUNode@1@HH@Z 1001b3e0 f   AssemblySamtoolsMpileup.obj
 0001:0001a400       __unwindfunclet$?ensureFileExists@CallVariantsTask@LocalWorkflow@U2@@AAE_NABVQString@@W4FileType@123@@Z$0 1001b400 f   AssemblySamtoolsMpileup.obj
 0001:0001a409       __unwindfunclet$?ensureFileExists@CallVariantsTask@LocalWorkflow@U2@@AAE_NABVQString@@W4FileType@123@@Z$1 1001b409 f   AssemblySamtoolsMpileup.obj
 0001:0001a412       __unwindfunclet$?ensureFileExists@CallVariantsTask@LocalWorkflow@U2@@AAE_NABVQString@@W4FileType@123@@Z$2 1001b412 f   AssemblySamtoolsMpileup.obj
 0001:0001a41b       __unwindfunclet$?ensureFileExists@CallVariantsTask@LocalWorkflow@U2@@AAE_NABVQString@@W4FileType@123@@Z$3 1001b41b f   AssemblySamtoolsMpileup.obj
 0001:0001a424       __ehhandler$?ensureFileExists@CallVariantsTask@LocalWorkflow@U2@@AAE_NABVQString@@W4FileType@123@@Z 1001b424 f   AssemblySamtoolsMpileup.obj
 0001:0001a440       __unwindfunclet$?getBcfViewArgs@CallVariantsTaskSettings@LocalWorkflow@U2@@QBE?AVQStringList@@XZ$0 1001b440 f   AssemblySamtoolsMpileup.obj
 0001:0001a459       __unwindfunclet$?getBcfViewArgs@CallVariantsTaskSettings@LocalWorkflow@U2@@QBE?AVQStringList@@XZ$1 1001b459 f   AssemblySamtoolsMpileup.obj
 0001:0001a462       __unwindfunclet$?getBcfViewArgs@CallVariantsTaskSettings@LocalWorkflow@U2@@QBE?AVQStringList@@XZ$2 1001b462 f   AssemblySamtoolsMpileup.obj
 0001:0001a46b       __unwindfunclet$?getBcfViewArgs@CallVariantsTaskSettings@LocalWorkflow@U2@@QBE?AVQStringList@@XZ$3 1001b46b f   AssemblySamtoolsMpileup.obj
 0001:0001a474       __unwindfunclet$?getBcfViewArgs@CallVariantsTaskSettings@LocalWorkflow@U2@@QBE?AVQStringList@@XZ$4 1001b474 f   AssemblySamtoolsMpileup.obj
 0001:0001a47d       __unwindfunclet$?getBcfViewArgs@CallVariantsTaskSettings@LocalWorkflow@U2@@QBE?AVQStringList@@XZ$5 1001b47d f   AssemblySamtoolsMpileup.obj
 0001:0001a486       __unwindfunclet$?getBcfViewArgs@CallVariantsTaskSettings@LocalWorkflow@U2@@QBE?AVQStringList@@XZ$6 1001b486 f   AssemblySamtoolsMpileup.obj
 0001:0001a48f       __unwindfunclet$?getBcfViewArgs@CallVariantsTaskSettings@LocalWorkflow@U2@@QBE?AVQStringList@@XZ$7 1001b48f f   AssemblySamtoolsMpileup.obj
 0001:0001a498       __unwindfunclet$?getBcfViewArgs@CallVariantsTaskSettings@LocalWorkflow@U2@@QBE?AVQStringList@@XZ$8 1001b498 f   AssemblySamtoolsMpileup.obj
 0001:0001a4a1       __unwindfunclet$?getBcfViewArgs@CallVariantsTaskSettings@LocalWorkflow@U2@@QBE?AVQStringList@@XZ$9 1001b4a1 f   AssemblySamtoolsMpileup.obj
 0001:0001a4aa       __unwindfunclet$?getBcfViewArgs@CallVariantsTaskSettings@LocalWorkflow@U2@@QBE?AVQStringList@@XZ$10 1001b4aa f   AssemblySamtoolsMpileup.obj
 0001:0001a4b3       __unwindfunclet$?getBcfViewArgs@CallVariantsTaskSettings@LocalWorkflow@U2@@QBE?AVQStringList@@XZ$11 1001b4b3 f   AssemblySamtoolsMpileup.obj
 0001:0001a4bc       __unwindfunclet$?getBcfViewArgs@CallVariantsTaskSettings@LocalWorkflow@U2@@QBE?AVQStringList@@XZ$12 1001b4bc f   AssemblySamtoolsMpileup.obj
 0001:0001a4c5       __unwindfunclet$?getBcfViewArgs@CallVariantsTaskSettings@LocalWorkflow@U2@@QBE?AVQStringList@@XZ$13 1001b4c5 f   AssemblySamtoolsMpileup.obj
 0001:0001a4ce       __unwindfunclet$?getBcfViewArgs@CallVariantsTaskSettings@LocalWorkflow@U2@@QBE?AVQStringList@@XZ$14 1001b4ce f   AssemblySamtoolsMpileup.obj
 0001:0001a4d7       __unwindfunclet$?getBcfViewArgs@CallVariantsTaskSettings@LocalWorkflow@U2@@QBE?AVQStringList@@XZ$15 1001b4d7 f   AssemblySamtoolsMpileup.obj
 0001:0001a4e0       __unwindfunclet$?getBcfViewArgs@CallVariantsTaskSettings@LocalWorkflow@U2@@QBE?AVQStringList@@XZ$16 1001b4e0 f   AssemblySamtoolsMpileup.obj
 0001:0001a4e9       __unwindfunclet$?getBcfViewArgs@CallVariantsTaskSettings@LocalWorkflow@U2@@QBE?AVQStringList@@XZ$17 1001b4e9 f   AssemblySamtoolsMpileup.obj
 0001:0001a4f2       __unwindfunclet$?getBcfViewArgs@CallVariantsTaskSettings@LocalWorkflow@U2@@QBE?AVQStringList@@XZ$18 1001b4f2 f   AssemblySamtoolsMpileup.obj
 0001:0001a4fb       __unwindfunclet$?getBcfViewArgs@CallVariantsTaskSettings@LocalWorkflow@U2@@QBE?AVQStringList@@XZ$19 1001b4fb f   AssemblySamtoolsMpileup.obj
 0001:0001a504       __unwindfunclet$?getBcfViewArgs@CallVariantsTaskSettings@LocalWorkflow@U2@@QBE?AVQStringList@@XZ$20 1001b504 f   AssemblySamtoolsMpileup.obj
 0001:0001a50d       __unwindfunclet$?getBcfViewArgs@CallVariantsTaskSettings@LocalWorkflow@U2@@QBE?AVQStringList@@XZ$21 1001b50d f   AssemblySamtoolsMpileup.obj
 0001:0001a516       __unwindfunclet$?getBcfViewArgs@CallVariantsTaskSettings@LocalWorkflow@U2@@QBE?AVQStringList@@XZ$22 1001b516 f   AssemblySamtoolsMpileup.obj
 0001:0001a51f       __unwindfunclet$?getBcfViewArgs@CallVariantsTaskSettings@LocalWorkflow@U2@@QBE?AVQStringList@@XZ$23 1001b51f f   AssemblySamtoolsMpileup.obj
 0001:0001a528       __unwindfunclet$?getBcfViewArgs@CallVariantsTaskSettings@LocalWorkflow@U2@@QBE?AVQStringList@@XZ$24 1001b528 f   AssemblySamtoolsMpileup.obj
 0001:0001a531       __unwindfunclet$?getBcfViewArgs@CallVariantsTaskSettings@LocalWorkflow@U2@@QBE?AVQStringList@@XZ$25 1001b531 f   AssemblySamtoolsMpileup.obj
 0001:0001a53a       __unwindfunclet$?getBcfViewArgs@CallVariantsTaskSettings@LocalWorkflow@U2@@QBE?AVQStringList@@XZ$26 1001b53a f   AssemblySamtoolsMpileup.obj
 0001:0001a543       __unwindfunclet$?getBcfViewArgs@CallVariantsTaskSettings@LocalWorkflow@U2@@QBE?AVQStringList@@XZ$27 1001b543 f   AssemblySamtoolsMpileup.obj
 0001:0001a54c       __unwindfunclet$?getBcfViewArgs@CallVariantsTaskSettings@LocalWorkflow@U2@@QBE?AVQStringList@@XZ$28 1001b54c f   AssemblySamtoolsMpileup.obj
 0001:0001a555       __unwindfunclet$?getBcfViewArgs@CallVariantsTaskSettings@LocalWorkflow@U2@@QBE?AVQStringList@@XZ$29 1001b555 f   AssemblySamtoolsMpileup.obj
 0001:0001a55e       __unwindfunclet$?getBcfViewArgs@CallVariantsTaskSettings@LocalWorkflow@U2@@QBE?AVQStringList@@XZ$30 1001b55e f   AssemblySamtoolsMpileup.obj
 0001:0001a567       __unwindfunclet$?getBcfViewArgs@CallVariantsTaskSettings@LocalWorkflow@U2@@QBE?AVQStringList@@XZ$31 1001b567 f   AssemblySamtoolsMpileup.obj
 0001:0001a570       __ehhandler$?getBcfViewArgs@CallVariantsTaskSettings@LocalWorkflow@U2@@QBE?AVQStringList@@XZ 1001b570 f   AssemblySamtoolsMpileup.obj
 0001:0001a590       __unwindfunclet$?getMpiliupArgs@CallVariantsTaskSettings@LocalWorkflow@U2@@QBE?AVQStringList@@XZ$0 1001b590 f   AssemblySamtoolsMpileup.obj
 0001:0001a5a9       __unwindfunclet$?getMpiliupArgs@CallVariantsTaskSettings@LocalWorkflow@U2@@QBE?AVQStringList@@XZ$1 1001b5a9 f   AssemblySamtoolsMpileup.obj
 0001:0001a5b2       __unwindfunclet$?getMpiliupArgs@CallVariantsTaskSettings@LocalWorkflow@U2@@QBE?AVQStringList@@XZ$2 1001b5b2 f   AssemblySamtoolsMpileup.obj
 0001:0001a5bb       __unwindfunclet$?getMpiliupArgs@CallVariantsTaskSettings@LocalWorkflow@U2@@QBE?AVQStringList@@XZ$3 1001b5bb f   AssemblySamtoolsMpileup.obj
 0001:0001a5c4       __unwindfunclet$?getMpiliupArgs@CallVariantsTaskSettings@LocalWorkflow@U2@@QBE?AVQStringList@@XZ$4 1001b5c4 f   AssemblySamtoolsMpileup.obj
 0001:0001a5cd       __unwindfunclet$?getMpiliupArgs@CallVariantsTaskSettings@LocalWorkflow@U2@@QBE?AVQStringList@@XZ$5 1001b5cd f   AssemblySamtoolsMpileup.obj
 0001:0001a5d6       __unwindfunclet$?getMpiliupArgs@CallVariantsTaskSettings@LocalWorkflow@U2@@QBE?AVQStringList@@XZ$6 1001b5d6 f   AssemblySamtoolsMpileup.obj
 0001:0001a5df       __unwindfunclet$?getMpiliupArgs@CallVariantsTaskSettings@LocalWorkflow@U2@@QBE?AVQStringList@@XZ$7 1001b5df f   AssemblySamtoolsMpileup.obj
 0001:0001a5e8       __unwindfunclet$?getMpiliupArgs@CallVariantsTaskSettings@LocalWorkflow@U2@@QBE?AVQStringList@@XZ$8 1001b5e8 f   AssemblySamtoolsMpileup.obj
 0001:0001a5f1       __unwindfunclet$?getMpiliupArgs@CallVariantsTaskSettings@LocalWorkflow@U2@@QBE?AVQStringList@@XZ$9 1001b5f1 f   AssemblySamtoolsMpileup.obj
 0001:0001a5fa       __unwindfunclet$?getMpiliupArgs@CallVariantsTaskSettings@LocalWorkflow@U2@@QBE?AVQStringList@@XZ$10 1001b5fa f   AssemblySamtoolsMpileup.obj
 0001:0001a603       __unwindfunclet$?getMpiliupArgs@CallVariantsTaskSettings@LocalWorkflow@U2@@QBE?AVQStringList@@XZ$11 1001b603 f   AssemblySamtoolsMpileup.obj
 0001:0001a60c       __unwindfunclet$?getMpiliupArgs@CallVariantsTaskSettings@LocalWorkflow@U2@@QBE?AVQStringList@@XZ$12 1001b60c f   AssemblySamtoolsMpileup.obj
 0001:0001a615       __unwindfunclet$?getMpiliupArgs@CallVariantsTaskSettings@LocalWorkflow@U2@@QBE?AVQStringList@@XZ$13 1001b615 f   AssemblySamtoolsMpileup.obj
 0001:0001a61e       __unwindfunclet$?getMpiliupArgs@CallVariantsTaskSettings@LocalWorkflow@U2@@QBE?AVQStringList@@XZ$14 1001b61e f   AssemblySamtoolsMpileup.obj
 0001:0001a627       __unwindfunclet$?getMpiliupArgs@CallVariantsTaskSettings@LocalWorkflow@U2@@QBE?AVQStringList@@XZ$15 1001b627 f   AssemblySamtoolsMpileup.obj
 0001:0001a630       __unwindfunclet$?getMpiliupArgs@CallVariantsTaskSettings@LocalWorkflow@U2@@QBE?AVQStringList@@XZ$16 1001b630 f   AssemblySamtoolsMpileup.obj
 0001:0001a639       __unwindfunclet$?getMpiliupArgs@CallVariantsTaskSettings@LocalWorkflow@U2@@QBE?AVQStringList@@XZ$17 1001b639 f   AssemblySamtoolsMpileup.obj
 0001:0001a642       __unwindfunclet$?getMpiliupArgs@CallVariantsTaskSettings@LocalWorkflow@U2@@QBE?AVQStringList@@XZ$18 1001b642 f   AssemblySamtoolsMpileup.obj
 0001:0001a64b       __unwindfunclet$?getMpiliupArgs@CallVariantsTaskSettings@LocalWorkflow@U2@@QBE?AVQStringList@@XZ$19 1001b64b f   AssemblySamtoolsMpileup.obj
 0001:0001a654       __unwindfunclet$?getMpiliupArgs@CallVariantsTaskSettings@LocalWorkflow@U2@@QBE?AVQStringList@@XZ$20 1001b654 f   AssemblySamtoolsMpileup.obj
 0001:0001a65d       __unwindfunclet$?getMpiliupArgs@CallVariantsTaskSettings@LocalWorkflow@U2@@QBE?AVQStringList@@XZ$21 1001b65d f   AssemblySamtoolsMpileup.obj
 0001:0001a666       __unwindfunclet$?getMpiliupArgs@CallVariantsTaskSettings@LocalWorkflow@U2@@QBE?AVQStringList@@XZ$22 1001b666 f   AssemblySamtoolsMpileup.obj
 0001:0001a66f       __unwindfunclet$?getMpiliupArgs@CallVariantsTaskSettings@LocalWorkflow@U2@@QBE?AVQStringList@@XZ$23 1001b66f f   AssemblySamtoolsMpileup.obj
 0001:0001a678       __unwindfunclet$?getMpiliupArgs@CallVariantsTaskSettings@LocalWorkflow@U2@@QBE?AVQStringList@@XZ$24 1001b678 f   AssemblySamtoolsMpileup.obj
 0001:0001a681       __unwindfunclet$?getMpiliupArgs@CallVariantsTaskSettings@LocalWorkflow@U2@@QBE?AVQStringList@@XZ$25 1001b681 f   AssemblySamtoolsMpileup.obj
 0001:0001a68a       __unwindfunclet$?getMpiliupArgs@CallVariantsTaskSettings@LocalWorkflow@U2@@QBE?AVQStringList@@XZ$26 1001b68a f   AssemblySamtoolsMpileup.obj
 0001:0001a693       __unwindfunclet$?getMpiliupArgs@CallVariantsTaskSettings@LocalWorkflow@U2@@QBE?AVQStringList@@XZ$27 1001b693 f   AssemblySamtoolsMpileup.obj
 0001:0001a69c       __unwindfunclet$?getMpiliupArgs@CallVariantsTaskSettings@LocalWorkflow@U2@@QBE?AVQStringList@@XZ$28 1001b69c f   AssemblySamtoolsMpileup.obj
 0001:0001a6a5       __unwindfunclet$?getMpiliupArgs@CallVariantsTaskSettings@LocalWorkflow@U2@@QBE?AVQStringList@@XZ$29 1001b6a5 f   AssemblySamtoolsMpileup.obj
 0001:0001a6ae       __ehhandler$?getMpiliupArgs@CallVariantsTaskSettings@LocalWorkflow@U2@@QBE?AVQStringList@@XZ 1001b6ae f   AssemblySamtoolsMpileup.obj
 0001:0001a6d0       __unwindfunclet$?getVarFilterArgs@CallVariantsTaskSettings@LocalWorkflow@U2@@QBE?AVQStringList@@XZ$0 1001b6d0 f   AssemblySamtoolsMpileup.obj
 0001:0001a6e9       __unwindfunclet$?getVarFilterArgs@CallVariantsTaskSettings@LocalWorkflow@U2@@QBE?AVQStringList@@XZ$1 1001b6e9 f   AssemblySamtoolsMpileup.obj
 0001:0001a6f2       __unwindfunclet$?getVarFilterArgs@CallVariantsTaskSettings@LocalWorkflow@U2@@QBE?AVQStringList@@XZ$2 1001b6f2 f   AssemblySamtoolsMpileup.obj
 0001:0001a6fb       __unwindfunclet$?getVarFilterArgs@CallVariantsTaskSettings@LocalWorkflow@U2@@QBE?AVQStringList@@XZ$3 1001b6fb f   AssemblySamtoolsMpileup.obj
 0001:0001a704       __unwindfunclet$?getVarFilterArgs@CallVariantsTaskSettings@LocalWorkflow@U2@@QBE?AVQStringList@@XZ$4 1001b704 f   AssemblySamtoolsMpileup.obj
 0001:0001a70d       __unwindfunclet$?getVarFilterArgs@CallVariantsTaskSettings@LocalWorkflow@U2@@QBE?AVQStringList@@XZ$5 1001b70d f   AssemblySamtoolsMpileup.obj
 0001:0001a716       __unwindfunclet$?getVarFilterArgs@CallVariantsTaskSettings@LocalWorkflow@U2@@QBE?AVQStringList@@XZ$6 1001b716 f   AssemblySamtoolsMpileup.obj
 0001:0001a71f       __unwindfunclet$?getVarFilterArgs@CallVariantsTaskSettings@LocalWorkflow@U2@@QBE?AVQStringList@@XZ$7 1001b71f f   AssemblySamtoolsMpileup.obj
 0001:0001a728       __unwindfunclet$?getVarFilterArgs@CallVariantsTaskSettings@LocalWorkflow@U2@@QBE?AVQStringList@@XZ$8 1001b728 f   AssemblySamtoolsMpileup.obj
 0001:0001a731       __unwindfunclet$?getVarFilterArgs@CallVariantsTaskSettings@LocalWorkflow@U2@@QBE?AVQStringList@@XZ$9 1001b731 f   AssemblySamtoolsMpileup.obj
 0001:0001a73a       __unwindfunclet$?getVarFilterArgs@CallVariantsTaskSettings@LocalWorkflow@U2@@QBE?AVQStringList@@XZ$10 1001b73a f   AssemblySamtoolsMpileup.obj
 0001:0001a743       __unwindfunclet$?getVarFilterArgs@CallVariantsTaskSettings@LocalWorkflow@U2@@QBE?AVQStringList@@XZ$11 1001b743 f   AssemblySamtoolsMpileup.obj
 0001:0001a74c       __unwindfunclet$?getVarFilterArgs@CallVariantsTaskSettings@LocalWorkflow@U2@@QBE?AVQStringList@@XZ$12 1001b74c f   AssemblySamtoolsMpileup.obj
 0001:0001a755       __unwindfunclet$?getVarFilterArgs@CallVariantsTaskSettings@LocalWorkflow@U2@@QBE?AVQStringList@@XZ$13 1001b755 f   AssemblySamtoolsMpileup.obj
 0001:0001a761       __unwindfunclet$?getVarFilterArgs@CallVariantsTaskSettings@LocalWorkflow@U2@@QBE?AVQStringList@@XZ$14 1001b761 f   AssemblySamtoolsMpileup.obj
 0001:0001a76d       __unwindfunclet$?getVarFilterArgs@CallVariantsTaskSettings@LocalWorkflow@U2@@QBE?AVQStringList@@XZ$15 1001b76d f   AssemblySamtoolsMpileup.obj
 0001:0001a776       __unwindfunclet$?getVarFilterArgs@CallVariantsTaskSettings@LocalWorkflow@U2@@QBE?AVQStringList@@XZ$16 1001b776 f   AssemblySamtoolsMpileup.obj
 0001:0001a77f       __unwindfunclet$?getVarFilterArgs@CallVariantsTaskSettings@LocalWorkflow@U2@@QBE?AVQStringList@@XZ$17 1001b77f f   AssemblySamtoolsMpileup.obj
 0001:0001a788       __unwindfunclet$?getVarFilterArgs@CallVariantsTaskSettings@LocalWorkflow@U2@@QBE?AVQStringList@@XZ$18 1001b788 f   AssemblySamtoolsMpileup.obj
 0001:0001a791       __unwindfunclet$?getVarFilterArgs@CallVariantsTaskSettings@LocalWorkflow@U2@@QBE?AVQStringList@@XZ$19 1001b791 f   AssemblySamtoolsMpileup.obj
 0001:0001a79a       __unwindfunclet$?getVarFilterArgs@CallVariantsTaskSettings@LocalWorkflow@U2@@QBE?AVQStringList@@XZ$20 1001b79a f   AssemblySamtoolsMpileup.obj
 0001:0001a7a3       __unwindfunclet$?getVarFilterArgs@CallVariantsTaskSettings@LocalWorkflow@U2@@QBE?AVQStringList@@XZ$21 1001b7a3 f   AssemblySamtoolsMpileup.obj
 0001:0001a7ac       __unwindfunclet$?getVarFilterArgs@CallVariantsTaskSettings@LocalWorkflow@U2@@QBE?AVQStringList@@XZ$22 1001b7ac f   AssemblySamtoolsMpileup.obj
 0001:0001a7b5       __unwindfunclet$?getVarFilterArgs@CallVariantsTaskSettings@LocalWorkflow@U2@@QBE?AVQStringList@@XZ$23 1001b7b5 f   AssemblySamtoolsMpileup.obj
 0001:0001a7be       __unwindfunclet$?getVarFilterArgs@CallVariantsTaskSettings@LocalWorkflow@U2@@QBE?AVQStringList@@XZ$24 1001b7be f   AssemblySamtoolsMpileup.obj
 0001:0001a7c7       __ehhandler$?getVarFilterArgs@CallVariantsTaskSettings@LocalWorkflow@U2@@QBE?AVQStringList@@XZ 1001b7c7 f   AssemblySamtoolsMpileup.obj
 0001:0001a7f0       __unwindfunclet$?node_construct@?$QList@V?$QMap@VQString@@VQVariant@@@@@@AAEXPAUNode@1@ABV?$QMap@VQString@@VQVariant@@@@@Z$0 1001b7f0 f   AssemblySamtoolsMpileup.obj
 0001:0001a7fb       __ehhandler$?node_construct@?$QList@V?$QMap@VQString@@VQVariant@@@@@@AAEXPAUNode@1@ABV?$QMap@VQString@@VQVariant@@@@@Z 1001b7fb f   AssemblySamtoolsMpileup.obj
 0001:0001a820       __unwindfunclet$?node_construct@?$QList@VQString@@@@AAEXPAUNode@1@ABVQString@@@Z$1 1001b820 f   AssemblySamtoolsMpileup.obj
 0001:0001a831       __ehhandler$?node_construct@?$QList@VQString@@@@AAEXPAUNode@1@ABVQString@@@Z 1001b831 f   AssemblySamtoolsMpileup.obj
 0001:0001a850       __unwindfunclet$?node_copy@?$QList@V?$QMap@VQString@@VQVariant@@@@@@AAEXPAUNode@1@00@Z$4 1001b850 f   AssemblySamtoolsMpileup.obj
 0001:0001a85b       __ehhandler$?node_copy@?$QList@V?$QMap@VQString@@VQVariant@@@@@@AAEXPAUNode@1@00@Z 1001b85b f   AssemblySamtoolsMpileup.obj
 0001:0001a880       __unwindfunclet$?node_copy@?$QList@VFormatDetectionResult@U2@@@@AAEXPAUNode@1@00@Z$4 1001b880 f   AssemblySamtoolsMpileup.obj
 0001:0001a88b       __ehhandler$?node_copy@?$QList@VFormatDetectionResult@U2@@@@AAEXPAUNode@1@00@Z 1001b88b f   AssemblySamtoolsMpileup.obj
 0001:0001a8b0       __unwindfunclet$?node_copy@?$QList@VQString@@@@AAEXPAUNode@1@00@Z$5 1001b8b0 f   AssemblySamtoolsMpileup.obj
 0001:0001a8c1       __ehhandler$?node_copy@?$QList@VQString@@@@AAEXPAUNode@1@00@Z 1001b8c1 f   AssemblySamtoolsMpileup.obj
 0001:0001a8e0       __unwindfunclet$?onSubTaskFinished@CallVariantsTask@LocalWorkflow@U2@@UAE?AV?$QList@PAVTask@U2@@@@PAVTask@3@@Z$0 1001b8e0 f   AssemblySamtoolsMpileup.obj
 0001:0001a8e8       __unwindfunclet$?onSubTaskFinished@CallVariantsTask@LocalWorkflow@U2@@UAE?AV?$QList@PAVTask@U2@@@@PAVTask@3@@Z$1 1001b8e8 f   AssemblySamtoolsMpileup.obj
 0001:0001a8f1       __unwindfunclet$?onSubTaskFinished@CallVariantsTask@LocalWorkflow@U2@@UAE?AV?$QList@PAVTask@U2@@@@PAVTask@3@@Z$2 1001b8f1 f   AssemblySamtoolsMpileup.obj
 0001:0001a90a       __unwindfunclet$?onSubTaskFinished@CallVariantsTask@LocalWorkflow@U2@@UAE?AV?$QList@PAVTask@U2@@@@PAVTask@3@@Z$3 1001b90a f   AssemblySamtoolsMpileup.obj
 0001:0001a913       __unwindfunclet$?onSubTaskFinished@CallVariantsTask@LocalWorkflow@U2@@UAE?AV?$QList@PAVTask@U2@@@@PAVTask@3@@Z$5 1001b913 f   AssemblySamtoolsMpileup.obj
 0001:0001a91b       __unwindfunclet$?onSubTaskFinished@CallVariantsTask@LocalWorkflow@U2@@UAE?AV?$QList@PAVTask@U2@@@@PAVTask@3@@Z$6 1001b91b f   AssemblySamtoolsMpileup.obj
 0001:0001a923       __unwindfunclet$?onSubTaskFinished@CallVariantsTask@LocalWorkflow@U2@@UAE?AV?$QList@PAVTask@U2@@@@PAVTask@3@@Z$7 1001b923 f   AssemblySamtoolsMpileup.obj
 0001:0001a92c       __unwindfunclet$?onSubTaskFinished@CallVariantsTask@LocalWorkflow@U2@@UAE?AV?$QList@PAVTask@U2@@@@PAVTask@3@@Z$8 1001b92c f   AssemblySamtoolsMpileup.obj
 0001:0001a935       __unwindfunclet$?onSubTaskFinished@CallVariantsTask@LocalWorkflow@U2@@UAE?AV?$QList@PAVTask@U2@@@@PAVTask@3@@Z$9 1001b935 f   AssemblySamtoolsMpileup.obj
 0001:0001a940       __unwindfunclet$?onSubTaskFinished@CallVariantsTask@LocalWorkflow@U2@@UAE?AV?$QList@PAVTask@U2@@@@PAVTask@3@@Z$10 1001b940 f   AssemblySamtoolsMpileup.obj
 0001:0001a95d       __unwindfunclet$?onSubTaskFinished@CallVariantsTask@LocalWorkflow@U2@@UAE?AV?$QList@PAVTask@U2@@@@PAVTask@3@@Z$11 1001b95d f   AssemblySamtoolsMpileup.obj
 0001:0001a97a       __unwindfunclet$?onSubTaskFinished@CallVariantsTask@LocalWorkflow@U2@@UAE?AV?$QList@PAVTask@U2@@@@PAVTask@3@@Z$13 1001b97a f   AssemblySamtoolsMpileup.obj
 0001:0001a982       __unwindfunclet$?onSubTaskFinished@CallVariantsTask@LocalWorkflow@U2@@UAE?AV?$QList@PAVTask@U2@@@@PAVTask@3@@Z$14 1001b982 f   AssemblySamtoolsMpileup.obj
 0001:0001a98b       __unwindfunclet$?onSubTaskFinished@CallVariantsTask@LocalWorkflow@U2@@UAE?AV?$QList@PAVTask@U2@@@@PAVTask@3@@Z$15 1001b98b f   AssemblySamtoolsMpileup.obj
 0001:0001a994       __unwindfunclet$?onSubTaskFinished@CallVariantsTask@LocalWorkflow@U2@@UAE?AV?$QList@PAVTask@U2@@@@PAVTask@3@@Z$16 1001b994 f   AssemblySamtoolsMpileup.obj
 0001:0001a99d       __unwindfunclet$?onSubTaskFinished@CallVariantsTask@LocalWorkflow@U2@@UAE?AV?$QList@PAVTask@U2@@@@PAVTask@3@@Z$17 1001b99d f   AssemblySamtoolsMpileup.obj
 0001:0001a9a6       __unwindfunclet$?onSubTaskFinished@CallVariantsTask@LocalWorkflow@U2@@UAE?AV?$QList@PAVTask@U2@@@@PAVTask@3@@Z$18 1001b9a6 f   AssemblySamtoolsMpileup.obj
 0001:0001a9af       __unwindfunclet$?onSubTaskFinished@CallVariantsTask@LocalWorkflow@U2@@UAE?AV?$QList@PAVTask@U2@@@@PAVTask@3@@Z$19 1001b9af f   AssemblySamtoolsMpileup.obj
 0001:0001a9b8       __unwindfunclet$?onSubTaskFinished@CallVariantsTask@LocalWorkflow@U2@@UAE?AV?$QList@PAVTask@U2@@@@PAVTask@3@@Z$21 1001b9b8 f   AssemblySamtoolsMpileup.obj
 0001:0001a9c0       __unwindfunclet$?onSubTaskFinished@CallVariantsTask@LocalWorkflow@U2@@UAE?AV?$QList@PAVTask@U2@@@@PAVTask@3@@Z$22 1001b9c0 f   AssemblySamtoolsMpileup.obj
 0001:0001a9c8       __unwindfunclet$?onSubTaskFinished@CallVariantsTask@LocalWorkflow@U2@@UAE?AV?$QList@PAVTask@U2@@@@PAVTask@3@@Z$25 1001b9c8 f   AssemblySamtoolsMpileup.obj
 0001:0001a9d0       __unwindfunclet$?onSubTaskFinished@CallVariantsTask@LocalWorkflow@U2@@UAE?AV?$QList@PAVTask@U2@@@@PAVTask@3@@Z$26 1001b9d0 f   AssemblySamtoolsMpileup.obj
 0001:0001a9d8       __unwindfunclet$?onSubTaskFinished@CallVariantsTask@LocalWorkflow@U2@@UAE?AV?$QList@PAVTask@U2@@@@PAVTask@3@@Z$27 1001b9d8 f   AssemblySamtoolsMpileup.obj
 0001:0001a9e4       __unwindfunclet$?onSubTaskFinished@CallVariantsTask@LocalWorkflow@U2@@UAE?AV?$QList@PAVTask@U2@@@@PAVTask@3@@Z$28 1001b9e4 f   AssemblySamtoolsMpileup.obj
 0001:0001a9ed       __unwindfunclet$?onSubTaskFinished@CallVariantsTask@LocalWorkflow@U2@@UAE?AV?$QList@PAVTask@U2@@@@PAVTask@3@@Z$29 1001b9ed f   AssemblySamtoolsMpileup.obj
 0001:0001a9f6       __unwindfunclet$?onSubTaskFinished@CallVariantsTask@LocalWorkflow@U2@@UAE?AV?$QList@PAVTask@U2@@@@PAVTask@3@@Z$30 1001b9f6 f   AssemblySamtoolsMpileup.obj
 0001:0001a9ff       __unwindfunclet$?onSubTaskFinished@CallVariantsTask@LocalWorkflow@U2@@UAE?AV?$QList@PAVTask@U2@@@@PAVTask@3@@Z$31 1001b9ff f   AssemblySamtoolsMpileup.obj
 0001:0001aa08       __unwindfunclet$?onSubTaskFinished@CallVariantsTask@LocalWorkflow@U2@@UAE?AV?$QList@PAVTask@U2@@@@PAVTask@3@@Z$32 1001ba08 f   AssemblySamtoolsMpileup.obj
 0001:0001aa11       __unwindfunclet$?onSubTaskFinished@CallVariantsTask@LocalWorkflow@U2@@UAE?AV?$QList@PAVTask@U2@@@@PAVTask@3@@Z$23 1001ba11 f   AssemblySamtoolsMpileup.obj
 0001:0001aa1a       __unwindfunclet$?onSubTaskFinished@CallVariantsTask@LocalWorkflow@U2@@UAE?AV?$QList@PAVTask@U2@@@@PAVTask@3@@Z$24 1001ba1a f   AssemblySamtoolsMpileup.obj
 0001:0001aa23       __ehhandler$?onSubTaskFinished@CallVariantsTask@LocalWorkflow@U2@@UAE?AV?$QList@PAVTask@U2@@@@PAVTask@3@@Z 1001ba23 f   AssemblySamtoolsMpileup.obj
 0001:0001aa50       __unwindfunclet$?prepare@CallVariantsTask@LocalWorkflow@U2@@UAEXXZ$0 1001ba50 f   AssemblySamtoolsMpileup.obj
 0001:0001aa58       __unwindfunclet$?prepare@CallVariantsTask@LocalWorkflow@U2@@UAEXXZ$1 1001ba58 f   AssemblySamtoolsMpileup.obj
 0001:0001aa61       __unwindfunclet$?prepare@CallVariantsTask@LocalWorkflow@U2@@UAEXXZ$2 1001ba61 f   AssemblySamtoolsMpileup.obj
 0001:0001aa6a       __unwindfunclet$?prepare@CallVariantsTask@LocalWorkflow@U2@@UAEXXZ$3 1001ba6a f   AssemblySamtoolsMpileup.obj
 0001:0001aa73       __unwindfunclet$?prepare@CallVariantsTask@LocalWorkflow@U2@@UAEXXZ$4 1001ba73 f   AssemblySamtoolsMpileup.obj
 0001:0001aa7e       __ehhandler$?prepare@CallVariantsTask@LocalWorkflow@U2@@UAEXXZ 1001ba7e f   AssemblySamtoolsMpileup.obj
 0001:0001aaa0       __unwindfunclet$?prepare@SamtoolsMpileupTask@LocalWorkflow@U2@@UAEXXZ$0 1001baa0 f   AssemblySamtoolsMpileup.obj
 0001:0001aaa9       __unwindfunclet$?prepare@SamtoolsMpileupTask@LocalWorkflow@U2@@UAEXXZ$1 1001baa9 f   AssemblySamtoolsMpileup.obj
 0001:0001aab2       __unwindfunclet$?prepare@SamtoolsMpileupTask@LocalWorkflow@U2@@UAEXXZ$2 1001bab2 f   AssemblySamtoolsMpileup.obj
 0001:0001aaba       __unwindfunclet$?prepare@SamtoolsMpileupTask@LocalWorkflow@U2@@UAEXXZ$4 1001baba f   AssemblySamtoolsMpileup.obj
 0001:0001aac3       __unwindfunclet$?prepare@SamtoolsMpileupTask@LocalWorkflow@U2@@UAEXXZ$5 1001bac3 f   AssemblySamtoolsMpileup.obj
 0001:0001aacc       __unwindfunclet$?prepare@SamtoolsMpileupTask@LocalWorkflow@U2@@UAEXXZ$6 1001bacc f   AssemblySamtoolsMpileup.obj
 0001:0001aad5       __unwindfunclet$?prepare@SamtoolsMpileupTask@LocalWorkflow@U2@@UAEXXZ$7 1001bad5 f   AssemblySamtoolsMpileup.obj
 0001:0001aade       __unwindfunclet$?prepare@SamtoolsMpileupTask@LocalWorkflow@U2@@UAEXXZ$8 1001bade f   AssemblySamtoolsMpileup.obj
 0001:0001aae7       __unwindfunclet$?prepare@SamtoolsMpileupTask@LocalWorkflow@U2@@UAEXXZ$9 1001bae7 f   AssemblySamtoolsMpileup.obj
 0001:0001aaf0       __unwindfunclet$?prepare@SamtoolsMpileupTask@LocalWorkflow@U2@@UAEXXZ$3 1001baf0 f   AssemblySamtoolsMpileup.obj
 0001:0001aaf9       __ehhandler$?prepare@SamtoolsMpileupTask@LocalWorkflow@U2@@UAEXXZ 1001baf9 f   AssemblySamtoolsMpileup.obj
 0001:0001ab20       __unwindfunclet$?qt_metatype_id@?$QMetaTypeId@V?$QSharedDataPointer@VDbiDataHandler@Workflow@U2@@@@@@SAHXZ$0 1001bb20 f   AssemblySamtoolsMpileup.obj
 0001:0001ab29       __ehhandler$?qt_metatype_id@?$QMetaTypeId@V?$QSharedDataPointer@VDbiDataHandler@Workflow@U2@@@@@@SAHXZ 1001bb29 f   AssemblySamtoolsMpileup.obj
 0001:0001ab50       __unwindfunclet$?qt_metatype_id@?$QMetaTypeId@VU2DbiRef@U2@@@@SAHXZ$0 1001bb50 f   AssemblySamtoolsMpileup.obj
 0001:0001ab59       __ehhandler$?qt_metatype_id@?$QMetaTypeId@VU2DbiRef@U2@@@@SAHXZ 1001bb59 f   AssemblySamtoolsMpileup.obj
 0001:0001ab80       __unwindfunclet$?run@SamtoolsMpileupTask@LocalWorkflow@U2@@UAEXXZ$0 1001bb80 f   AssemblySamtoolsMpileup.obj
 0001:0001ab89       __unwindfunclet$?run@SamtoolsMpileupTask@LocalWorkflow@U2@@UAEXXZ$1 1001bb89 f   AssemblySamtoolsMpileup.obj
 0001:0001ab91       __unwindfunclet$?run@SamtoolsMpileupTask@LocalWorkflow@U2@@UAEXXZ$2 1001bb91 f   AssemblySamtoolsMpileup.obj
 0001:0001ab99       __unwindfunclet$?run@SamtoolsMpileupTask@LocalWorkflow@U2@@UAEXXZ$3 1001bb99 f   AssemblySamtoolsMpileup.obj
 0001:0001aba2       __unwindfunclet$?run@SamtoolsMpileupTask@LocalWorkflow@U2@@UAEXXZ$4 1001bba2 f   AssemblySamtoolsMpileup.obj
 0001:0001abaa       __unwindfunclet$?run@SamtoolsMpileupTask@LocalWorkflow@U2@@UAEXXZ$5 1001bbaa f   AssemblySamtoolsMpileup.obj
 0001:0001abb6       __unwindfunclet$?run@SamtoolsMpileupTask@LocalWorkflow@U2@@UAEXXZ$6 1001bbb6 f   AssemblySamtoolsMpileup.obj
 0001:0001abc2       __unwindfunclet$?run@SamtoolsMpileupTask@LocalWorkflow@U2@@UAEXXZ$7 1001bbc2 f   AssemblySamtoolsMpileup.obj
 0001:0001abcb       __unwindfunclet$?run@SamtoolsMpileupTask@LocalWorkflow@U2@@UAEXXZ$8 1001bbcb f   AssemblySamtoolsMpileup.obj
 0001:0001abd3       __unwindfunclet$?run@SamtoolsMpileupTask@LocalWorkflow@U2@@UAEXXZ$9 1001bbd3 f   AssemblySamtoolsMpileup.obj
 0001:0001abdb       __unwindfunclet$?run@SamtoolsMpileupTask@LocalWorkflow@U2@@UAEXXZ$10 1001bbdb f   AssemblySamtoolsMpileup.obj
 0001:0001abe4       __unwindfunclet$?run@SamtoolsMpileupTask@LocalWorkflow@U2@@UAEXXZ$11 1001bbe4 f   AssemblySamtoolsMpileup.obj
 0001:0001abec       __unwindfunclet$?run@SamtoolsMpileupTask@LocalWorkflow@U2@@UAEXXZ$12 1001bbec f   AssemblySamtoolsMpileup.obj
 0001:0001abf8       __unwindfunclet$?run@SamtoolsMpileupTask@LocalWorkflow@U2@@UAEXXZ$13 1001bbf8 f   AssemblySamtoolsMpileup.obj
 0001:0001ac04       __unwindfunclet$?run@SamtoolsMpileupTask@LocalWorkflow@U2@@UAEXXZ$14 1001bc04 f   AssemblySamtoolsMpileup.obj
 0001:0001ac0d       __unwindfunclet$?run@SamtoolsMpileupTask@LocalWorkflow@U2@@UAEXXZ$15 1001bc0d f   AssemblySamtoolsMpileup.obj
 0001:0001ac15       __unwindfunclet$?run@SamtoolsMpileupTask@LocalWorkflow@U2@@UAEXXZ$16 1001bc15 f   AssemblySamtoolsMpileup.obj
 0001:0001ac1d       __unwindfunclet$?run@SamtoolsMpileupTask@LocalWorkflow@U2@@UAEXXZ$17 1001bc1d f   AssemblySamtoolsMpileup.obj
 0001:0001ac26       __unwindfunclet$?run@SamtoolsMpileupTask@LocalWorkflow@U2@@UAEXXZ$18 1001bc26 f   AssemblySamtoolsMpileup.obj
 0001:0001ac2e       __unwindfunclet$?run@SamtoolsMpileupTask@LocalWorkflow@U2@@UAEXXZ$19 1001bc2e f   AssemblySamtoolsMpileup.obj
 0001:0001ac3a       __unwindfunclet$?run@SamtoolsMpileupTask@LocalWorkflow@U2@@UAEXXZ$20 1001bc3a f   AssemblySamtoolsMpileup.obj
 0001:0001ac46       __unwindfunclet$?run@SamtoolsMpileupTask@LocalWorkflow@U2@@UAEXXZ$21 1001bc46 f   AssemblySamtoolsMpileup.obj
 0001:0001ac4f       __unwindfunclet$?run@SamtoolsMpileupTask@LocalWorkflow@U2@@UAEXXZ$22 1001bc4f f   AssemblySamtoolsMpileup.obj
 0001:0001ac58       __unwindfunclet$?run@SamtoolsMpileupTask@LocalWorkflow@U2@@UAEXXZ$23 1001bc58 f   AssemblySamtoolsMpileup.obj
 0001:0001ac61       __unwindfunclet$?run@SamtoolsMpileupTask@LocalWorkflow@U2@@UAEXXZ$24 1001bc61 f   AssemblySamtoolsMpileup.obj
 0001:0001ac6a       __unwindfunclet$?run@SamtoolsMpileupTask@LocalWorkflow@U2@@UAEXXZ$25 1001bc6a f   AssemblySamtoolsMpileup.obj
 0001:0001ac73       __unwindfunclet$?run@SamtoolsMpileupTask@LocalWorkflow@U2@@UAEXXZ$26 1001bc73 f   AssemblySamtoolsMpileup.obj
 0001:0001ac7c       __ehhandler$?run@SamtoolsMpileupTask@LocalWorkflow@U2@@UAEXXZ 1001bc7c f   AssemblySamtoolsMpileup.obj
 0001:0001aca0       __unwindfunclet$?start@SamtoolsMpileupTask@LocalWorkflow@U2@@AAEXABVProcessRun@3@ABVQString@@@Z$0 1001bca0 f   AssemblySamtoolsMpileup.obj
 0001:0001aca9       __unwindfunclet$?start@SamtoolsMpileupTask@LocalWorkflow@U2@@AAEXABVProcessRun@3@ABVQString@@@Z$1 1001bca9 f   AssemblySamtoolsMpileup.obj
 0001:0001acb2       __ehhandler$?start@SamtoolsMpileupTask@LocalWorkflow@U2@@AAEXABVProcessRun@3@ABVQString@@@Z 1001bcb2 f   AssemblySamtoolsMpileup.obj
 0001:0001acd0       __unwindfunclet$?tmpFilePath@CallVariantsTask@LocalWorkflow@U2@@SA?AVQString@@ABV4@0AAVU2OpStatus@3@@Z$0 1001bcd0 f   AssemblySamtoolsMpileup.obj
 0001:0001acd9       __unwindfunclet$?tmpFilePath@CallVariantsTask@LocalWorkflow@U2@@SA?AVQString@@ABV4@0AAVU2OpStatus@3@@Z$1 1001bcd9 f   AssemblySamtoolsMpileup.obj
 0001:0001ace2       __unwindfunclet$?tmpFilePath@CallVariantsTask@LocalWorkflow@U2@@SA?AVQString@@ABV4@0AAVU2OpStatus@3@@Z$2 1001bce2 f   AssemblySamtoolsMpileup.obj
 0001:0001acfc       __ehhandler$?tmpFilePath@CallVariantsTask@LocalWorkflow@U2@@SA?AVQString@@ABV4@0AAVU2OpStatus@3@@Z 1001bcfc f   AssemblySamtoolsMpileup.obj
 0001:0001ad20       __unwindfunclet$?toString@CallVariantsTask@LocalWorkflow@U2@@CA?AVQString@@W4FileType@123@@Z$1 1001bd20 f   AssemblySamtoolsMpileup.obj
 0001:0001ad29       __unwindfunclet$?toString@CallVariantsTask@LocalWorkflow@U2@@CA?AVQString@@W4FileType@123@@Z$2 1001bd29 f   AssemblySamtoolsMpileup.obj
 0001:0001ad32       __unwindfunclet$?toString@CallVariantsTask@LocalWorkflow@U2@@CA?AVQString@@W4FileType@123@@Z$3 1001bd32 f   AssemblySamtoolsMpileup.obj
 0001:0001ad3b       __unwindfunclet$?toString@CallVariantsTask@LocalWorkflow@U2@@CA?AVQString@@W4FileType@123@@Z$4 1001bd3b f   AssemblySamtoolsMpileup.obj
 0001:0001ad44       __unwindfunclet$?toString@CallVariantsTask@LocalWorkflow@U2@@CA?AVQString@@W4FileType@123@@Z$5 1001bd44 f   AssemblySamtoolsMpileup.obj
 0001:0001ad4d       __unwindfunclet$?toString@CallVariantsTask@LocalWorkflow@U2@@CA?AVQString@@W4FileType@123@@Z$6 1001bd4d f   AssemblySamtoolsMpileup.obj
 0001:0001ad56       __ehhandler$?toString@CallVariantsTask@LocalWorkflow@U2@@CA?AVQString@@W4FileType@123@@Z 1001bd56 f   AssemblySamtoolsMpileup.obj
 0001:0001ad80       __unwindfunclet$??$getAttributeValue@H@Attribute@U2@@QBEHPAVWorkflowContext@Workflow@1@@Z$0 1001bd80 f   SamtoolMpileupWorker.obj
 0001:0001ad89       __unwindfunclet$??$getAttributeValue@H@Attribute@U2@@QBEHPAVWorkflowContext@Workflow@1@@Z$1 1001bd89 f   SamtoolMpileupWorker.obj
 0001:0001ad91       __unwindfunclet$??$getAttributeValue@H@Attribute@U2@@QBEHPAVWorkflowContext@Workflow@1@@Z$2 1001bd91 f   SamtoolMpileupWorker.obj
 0001:0001ad99       __unwindfunclet$??$getAttributeValue@H@Attribute@U2@@QBEHPAVWorkflowContext@Workflow@1@@Z$3 1001bd99 f   SamtoolMpileupWorker.obj
 0001:0001ada1       __unwindfunclet$??$getAttributeValue@H@Attribute@U2@@QBEHPAVWorkflowContext@Workflow@1@@Z$4 1001bda1 f   SamtoolMpileupWorker.obj
 0001:0001adaa       __unwindfunclet$??$getAttributeValue@H@Attribute@U2@@QBEHPAVWorkflowContext@Workflow@1@@Z$5 1001bdaa f   SamtoolMpileupWorker.obj
 0001:0001adb3       __unwindfunclet$??$getAttributeValue@H@Attribute@U2@@QBEHPAVWorkflowContext@Workflow@1@@Z$6 1001bdb3 f   SamtoolMpileupWorker.obj
 0001:0001adbc       __unwindfunclet$??$getAttributeValue@H@Attribute@U2@@QBEHPAVWorkflowContext@Workflow@1@@Z$7 1001bdbc f   SamtoolMpileupWorker.obj
 0001:0001adc5       __unwindfunclet$??$getAttributeValue@H@Attribute@U2@@QBEHPAVWorkflowContext@Workflow@1@@Z$8 1001bdc5 f   SamtoolMpileupWorker.obj
 0001:0001adce       __unwindfunclet$??$getAttributeValue@H@Attribute@U2@@QBEHPAVWorkflowContext@Workflow@1@@Z$9 1001bdce f   SamtoolMpileupWorker.obj
 0001:0001add7       __unwindfunclet$??$getAttributeValue@H@Attribute@U2@@QBEHPAVWorkflowContext@Workflow@1@@Z$10 1001bdd7 f   SamtoolMpileupWorker.obj
 0001:0001ade0       __unwindfunclet$??$getAttributeValue@H@Attribute@U2@@QBEHPAVWorkflowContext@Workflow@1@@Z$11 1001bde0 f   SamtoolMpileupWorker.obj
 0001:0001ade9       __ehhandler$??$getAttributeValue@H@Attribute@U2@@QBEHPAVWorkflowContext@Workflow@1@@Z 1001bde9 f   SamtoolMpileupWorker.obj
 0001:0001ae10       __unwindfunclet$??$getAttributeValue@VQString@@@Attribute@U2@@QBE?AVQString@@PAVWorkflowContext@Workflow@1@@Z$0 1001be10 f   SamtoolMpileupWorker.obj
 0001:0001ae2a       __unwindfunclet$??$getAttributeValue@VQString@@@Attribute@U2@@QBE?AVQString@@PAVWorkflowContext@Workflow@1@@Z$1 1001be2a f   SamtoolMpileupWorker.obj
 0001:0001ae33       __unwindfunclet$??$getAttributeValue@VQString@@@Attribute@U2@@QBE?AVQString@@PAVWorkflowContext@Workflow@1@@Z$2 1001be33 f   SamtoolMpileupWorker.obj
 0001:0001ae3b       __unwindfunclet$??$getAttributeValue@VQString@@@Attribute@U2@@QBE?AVQString@@PAVWorkflowContext@Workflow@1@@Z$3 1001be3b f   SamtoolMpileupWorker.obj
 0001:0001ae43       __unwindfunclet$??$getAttributeValue@VQString@@@Attribute@U2@@QBE?AVQString@@PAVWorkflowContext@Workflow@1@@Z$4 1001be43 f   SamtoolMpileupWorker.obj
 0001:0001ae4b       __unwindfunclet$??$getAttributeValue@VQString@@@Attribute@U2@@QBE?AVQString@@PAVWorkflowContext@Workflow@1@@Z$5 1001be4b f   SamtoolMpileupWorker.obj
 0001:0001ae54       __unwindfunclet$??$getAttributeValue@VQString@@@Attribute@U2@@QBE?AVQString@@PAVWorkflowContext@Workflow@1@@Z$6 1001be54 f   SamtoolMpileupWorker.obj
 0001:0001ae5d       __unwindfunclet$??$getAttributeValue@VQString@@@Attribute@U2@@QBE?AVQString@@PAVWorkflowContext@Workflow@1@@Z$7 1001be5d f   SamtoolMpileupWorker.obj
 0001:0001ae66       __unwindfunclet$??$getAttributeValue@VQString@@@Attribute@U2@@QBE?AVQString@@PAVWorkflowContext@Workflow@1@@Z$8 1001be66 f   SamtoolMpileupWorker.obj
 0001:0001ae6f       __unwindfunclet$??$getAttributeValue@VQString@@@Attribute@U2@@QBE?AVQString@@PAVWorkflowContext@Workflow@1@@Z$9 1001be6f f   SamtoolMpileupWorker.obj
 0001:0001ae78       __unwindfunclet$??$getAttributeValue@VQString@@@Attribute@U2@@QBE?AVQString@@PAVWorkflowContext@Workflow@1@@Z$10 1001be78 f   SamtoolMpileupWorker.obj
 0001:0001ae81       __unwindfunclet$??$getAttributeValue@VQString@@@Attribute@U2@@QBE?AVQString@@PAVWorkflowContext@Workflow@1@@Z$11 1001be81 f   SamtoolMpileupWorker.obj
 0001:0001ae8a       __unwindfunclet$??$getAttributeValue@VQString@@@Attribute@U2@@QBE?AVQString@@PAVWorkflowContext@Workflow@1@@Z$12 1001be8a f   SamtoolMpileupWorker.obj
 0001:0001ae93       __ehhandler$??$getAttributeValue@VQString@@@Attribute@U2@@QBE?AVQString@@PAVWorkflowContext@Workflow@1@@Z 1001be93 f   SamtoolMpileupWorker.obj
 0001:0001aec0       __unwindfunclet$??$getValue@VQString@@@BaseWorker@LocalWorkflow@U2@@IBE?AVQString@@ABV3@@Z$0 1001bec0 f   SamtoolMpileupWorker.obj
 0001:0001aeda       __unwindfunclet$??$getValue@VQString@@@BaseWorker@LocalWorkflow@U2@@IBE?AVQString@@ABV3@@Z$1 1001beda f   SamtoolMpileupWorker.obj
 0001:0001aee3       __ehhandler$??$getValue@VQString@@@BaseWorker@LocalWorkflow@U2@@IBE?AVQString@@ABV3@@Z 1001bee3 f   SamtoolMpileupWorker.obj
 0001:0001af00       __unwindfunclet$??$qvariant_cast@V?$QMap@VQString@@V1@@@@@YA?AV?$QMap@VQString@@V1@@@ABVQVariant@@@Z$0 1001bf00 f   SamtoolMpileupWorker.obj
 0001:0001af09       __unwindfunclet$??$qvariant_cast@V?$QMap@VQString@@V1@@@@@YA?AV?$QMap@VQString@@V1@@@ABVQVariant@@@Z$1 1001bf09 f   SamtoolMpileupWorker.obj
 0001:0001af22       __ehhandler$??$qvariant_cast@V?$QMap@VQString@@V1@@@@@YA?AV?$QMap@VQString@@V1@@@ABVQVariant@@@Z 1001bf22 f   SamtoolMpileupWorker.obj
 0001:0001af40       __ehhandler$??0?$QList@PAVPort@Workflow@U2@@@@QAE@ABV0@@Z 1001bf40 f   SamtoolMpileupWorker.obj
 0001:0001af60       __ehhandler$??0?$QList@V?$QMap@VQString@@VQVariant@@@@@@QAE@ABV0@@Z 1001bf60 f   SamtoolMpileupWorker.obj
 0001:0001af80       __ehhandler$??0?$QList@VDescriptor@U2@@@@QAE@ABV0@@Z 1001bf80 f   SamtoolMpileupWorker.obj
 0001:0001afa0       __unwindfunclet$??0CallVariantsTaskSettings@LocalWorkflow@U2@@QAE@XZ$0 1001bfa0 f   SamtoolMpileupWorker.obj
 0001:0001afa9       __unwindfunclet$??0CallVariantsTaskSettings@LocalWorkflow@U2@@QAE@XZ$1 1001bfa9 f   SamtoolMpileupWorker.obj
 0001:0001afb4       __unwindfunclet$??0CallVariantsTaskSettings@LocalWorkflow@U2@@QAE@XZ$2 1001bfb4 f   SamtoolMpileupWorker.obj
 0001:0001afc0       __unwindfunclet$??0CallVariantsTaskSettings@LocalWorkflow@U2@@QAE@XZ$3 1001bfc0 f   SamtoolMpileupWorker.obj
 0001:0001afcc       __unwindfunclet$??0CallVariantsTaskSettings@LocalWorkflow@U2@@QAE@XZ$4 1001bfcc f   SamtoolMpileupWorker.obj
 0001:0001afd8       __unwindfunclet$??0CallVariantsTaskSettings@LocalWorkflow@U2@@QAE@XZ$5 1001bfd8 f   SamtoolMpileupWorker.obj
 0001:0001afe4       __unwindfunclet$??0CallVariantsTaskSettings@LocalWorkflow@U2@@QAE@XZ$6 1001bfe4 f   SamtoolMpileupWorker.obj
 0001:0001aff0       __unwindfunclet$??0CallVariantsTaskSettings@LocalWorkflow@U2@@QAE@XZ$7 1001bff0 f   SamtoolMpileupWorker.obj
 0001:0001affc       __unwindfunclet$??0CallVariantsTaskSettings@LocalWorkflow@U2@@QAE@XZ$8 1001bffc f   SamtoolMpileupWorker.obj
 0001:0001b008       __ehhandler$??0CallVariantsTaskSettings@LocalWorkflow@U2@@QAE@XZ 1001c008 f   SamtoolMpileupWorker.obj
 0001:0001b030       __unwindfunclet$??0CallVariantsWorker@LocalWorkflow@U2@@QAE@PAVActor@Workflow@2@@Z$0 1001c030 f   SamtoolMpileupWorker.obj
 0001:0001b039       __unwindfunclet$??0CallVariantsWorker@LocalWorkflow@U2@@QAE@PAVActor@Workflow@2@@Z$1 1001c039 f   SamtoolMpileupWorker.obj
 0001:0001b044       __unwindfunclet$??0CallVariantsWorker@LocalWorkflow@U2@@QAE@PAVActor@Workflow@2@@Z$2 1001c044 f   SamtoolMpileupWorker.obj
 0001:0001b052       __unwindfunclet$??0CallVariantsWorker@LocalWorkflow@U2@@QAE@PAVActor@Workflow@2@@Z$3 1001c052 f   SamtoolMpileupWorker.obj
 0001:0001b060       __ehhandler$??0CallVariantsWorker@LocalWorkflow@U2@@QAE@PAVActor@Workflow@2@@Z 1001c060 f   SamtoolMpileupWorker.obj
 0001:0001b080       __unwindfunclet$??0EmptySlotValidator@LocalWorkflow@U2@@QAE@ABVQString@@@Z$0 1001c080 f   SamtoolMpileupWorker.obj
 0001:0001b089       __ehhandler$??0EmptySlotValidator@LocalWorkflow@U2@@QAE@ABVQString@@@Z 1001c089 f   SamtoolMpileupWorker.obj
 0001:0001b0b0       __unwindfunclet$??0ScientificDoubleWidget@LocalWorkflow@U2@@QAE@PAVQWidget@@@Z$0 1001c0b0 f   SamtoolMpileupWorker.obj
 0001:0001b0b9       __unwindfunclet$??0ScientificDoubleWidget@LocalWorkflow@U2@@QAE@PAVQWidget@@@Z$1 1001c0b9 f   SamtoolMpileupWorker.obj
 0001:0001b0c4       __unwindfunclet$??0ScientificDoubleWidget@LocalWorkflow@U2@@QAE@PAVQWidget@@@Z$2 1001c0c4 f   SamtoolMpileupWorker.obj
 0001:0001b0cf       __ehhandler$??0ScientificDoubleWidget@LocalWorkflow@U2@@QAE@PAVQWidget@@@Z 1001c0cf f   SamtoolMpileupWorker.obj
 0001:0001b0f0       __unwindfunclet$??1CallVariantsWorker@LocalWorkflow@U2@@UAE@XZ$0 1001c0f0 f   SamtoolMpileupWorker.obj
 0001:0001b0f9       __unwindfunclet$??1CallVariantsWorker@LocalWorkflow@U2@@UAE@XZ$1 1001c0f9 f   SamtoolMpileupWorker.obj
 0001:0001b104       __unwindfunclet$??1CallVariantsWorker@LocalWorkflow@U2@@UAE@XZ$2 1001c104 f   SamtoolMpileupWorker.obj
 0001:0001b112       __unwindfunclet$??1CallVariantsWorker@LocalWorkflow@U2@@UAE@XZ$3 1001c112 f   SamtoolMpileupWorker.obj
 0001:0001b120       __ehhandler$??1CallVariantsWorker@LocalWorkflow@U2@@UAE@XZ 1001c120 f   SamtoolMpileupWorker.obj
 0001:0001b140       __unwindfunclet$??1EmptySlotValidator@LocalWorkflow@U2@@UAE@XZ$0 1001c140 f   SamtoolMpileupWorker.obj
 0001:0001b149       __ehhandler$??1EmptySlotValidator@LocalWorkflow@U2@@UAE@XZ 1001c149 f   SamtoolMpileupWorker.obj
 0001:0001b170       __unwindfunclet$??A?$QMap@VDescriptor@U2@@V?$QExplicitlySharedDataPointer@VDataType@U2@@@@@@QAEAAV?$QExplicitlySharedDataPointer@VDataType@U2@@@@ABVDescriptor@U2@@@Z$0 1001c170 f   SamtoolMpileupWorker.obj
 0001:0001b178       __ehhandler$??A?$QMap@VDescriptor@U2@@V?$QExplicitlySharedDataPointer@VDataType@U2@@@@@@QAEAAV?$QExplicitlySharedDataPointer@VDataType@U2@@@@ABVDescriptor@U2@@@Z 1001c178 f   SamtoolMpileupWorker.obj
 0001:0001b1a0       __unwindfunclet$??A?$QMap@VQString@@VQScriptValue@@@@QAEAAVQScriptValue@@ABVQString@@@Z$0 1001c1a0 f   SamtoolMpileupWorker.obj
 0001:0001b1a9       __ehhandler$??A?$QMap@VQString@@VQScriptValue@@@@QAEAAVQScriptValue@@ABVQString@@@Z 1001c1a9 f   SamtoolMpileupWorker.obj
 0001:0001b1d0       __unwindfunclet$??H@YA?BVQString@@ABV0@PBD@Z$0 1001c1d0 f   SamtoolMpileupWorker.obj
 0001:0001b1ea       __unwindfunclet$??H@YA?BVQString@@ABV0@PBD@Z$1 1001c1ea f   SamtoolMpileupWorker.obj
 0001:0001b1f3       __ehhandler$??H@YA?BVQString@@ABV0@PBD@Z 1001c1f3 f   SamtoolMpileupWorker.obj
 0001:0001b210       __unwindfunclet$??H@YA?BVQString@@PBDABV0@@Z$0 1001c210 f   SamtoolMpileupWorker.obj
 0001:0001b22a       __ehhandler$??H@YA?BVQString@@PBDABV0@@Z 1001c22a f   SamtoolMpileupWorker.obj
 0001:0001b250       __unwindfunclet$??_GEmptySlotValidator@LocalWorkflow@U2@@UAEPAXI@Z$0 1001c250 f   SamtoolMpileupWorker.obj
 0001:0001b259       __ehhandler$??_GEmptySlotValidator@LocalWorkflow@U2@@UAEPAXI@Z 1001c259 f   SamtoolMpileupWorker.obj
 0001:0001b280       __unwindfunclet$??__EalgoLog@U2@@YAXXZ$0 1001c280 f   SamtoolMpileupWorker.obj
 0001:0001b289       __ehhandler$??__EalgoLog@U2@@YAXXZ 1001c289 f   SamtoolMpileupWorker.obj
 0001:0001b2b0       __unwindfunclet$??__EcmdLog@U2@@YAXXZ$0 1001c2b0 f   SamtoolMpileupWorker.obj
 0001:0001b2b9       __ehhandler$??__EcmdLog@U2@@YAXXZ 1001c2b9 f   SamtoolMpileupWorker.obj
 0001:0001b2e0       __unwindfunclet$??__EcoreLog@U2@@YAXXZ$0 1001c2e0 f   SamtoolMpileupWorker.obj
 0001:0001b2e9       __ehhandler$??__EcoreLog@U2@@YAXXZ 1001c2e9 f   SamtoolMpileupWorker.obj
 0001:0001b310       __unwindfunclet$??__EioLog@U2@@YAXXZ$0 1001c310 f   SamtoolMpileupWorker.obj
 0001:0001b319       __ehhandler$??__EioLog@U2@@YAXXZ 1001c319 f   SamtoolMpileupWorker.obj
 0001:0001b340       __unwindfunclet$??__EperfLog@U2@@YAXXZ$0 1001c340 f   SamtoolMpileupWorker.obj
 0001:0001b349       __ehhandler$??__EperfLog@U2@@YAXXZ 1001c349 f   SamtoolMpileupWorker.obj
 0001:0001b370       __unwindfunclet$??__EscriptLog@U2@@YAXXZ$0 1001c370 f   SamtoolMpileupWorker.obj
 0001:0001b379       __ehhandler$??__EscriptLog@U2@@YAXXZ 1001c379 f   SamtoolMpileupWorker.obj
 0001:0001b3a0       __unwindfunclet$??__EtaskLog@U2@@YAXXZ$0 1001c3a0 f   SamtoolMpileupWorker.obj
 0001:0001b3a9       __ehhandler$??__EtaskLog@U2@@YAXXZ 1001c3a9 f   SamtoolMpileupWorker.obj
 0001:0001b3d0       __unwindfunclet$??__EuiLog@U2@@YAXXZ$0 1001c3d0 f   SamtoolMpileupWorker.obj
 0001:0001b3d9       __ehhandler$??__EuiLog@U2@@YAXXZ 1001c3d9 f   SamtoolMpileupWorker.obj
 0001:0001b400       __unwindfunclet$??__EuserActLog@U2@@YAXXZ$0 1001c400 f   SamtoolMpileupWorker.obj
 0001:0001b409       __ehhandler$??__EuserActLog@U2@@YAXXZ 1001c409 f   SamtoolMpileupWorker.obj
 0001:0001b430       __ehhandler$?append@?$QList@PAVAttribute@U2@@@@QAEXABQAVAttribute@U2@@@Z 1001c430 f   SamtoolMpileupWorker.obj
 0001:0001b450       __ehhandler$?append@?$QList@PAVPortDescriptor@Workflow@U2@@@@QAEXABQAVPortDescriptor@Workflow@U2@@@Z 1001c450 f   SamtoolMpileupWorker.obj
 0001:0001b470       __unwindfunclet$?append@?$QList@VDescriptor@U2@@@@QAEXABVDescriptor@U2@@@Z$6 1001c470 f   SamtoolMpileupWorker.obj
 0001:0001b47b       __ehhandler$?append@?$QList@VDescriptor@U2@@@@QAEXABVDescriptor@U2@@@Z 1001c47b f   SamtoolMpileupWorker.obj
 0001:0001b4a0       __unwindfunclet$?append@?$QList@VMessage@Workflow@U2@@@@QAEXABVMessage@Workflow@U2@@@Z$6 1001c4a0 f   SamtoolMpileupWorker.obj
 0001:0001b4ab       __ehhandler$?append@?$QList@VMessage@Workflow@U2@@@@QAEXABVMessage@Workflow@U2@@@Z 1001c4ab f   SamtoolMpileupWorker.obj
 0001:0001b4d0       __unwindfunclet$?append@?$QList@VQVariant@@@@QAEXABVQVariant@@@Z$6 1001c4d0 f   SamtoolMpileupWorker.obj
 0001:0001b4db       __ehhandler$?append@?$QList@VQVariant@@@@QAEXABVQVariant@@@Z 1001c4db f   SamtoolMpileupWorker.obj
 0001:0001b500       __unwindfunclet$?append@?$QList@VWorkflowNotification@U2@@@@QAEXABVWorkflowNotification@U2@@@Z$6 1001c500 f   SamtoolMpileupWorker.obj
 0001:0001b50b       __ehhandler$?append@?$QList@VWorkflowNotification@U2@@@@QAEXABVWorkflowNotification@U2@@@Z 1001c50b f   SamtoolMpileupWorker.obj
 0001:0001b530       __unwindfunclet$?checkState@CallVariantsWorker@LocalWorkflow@U2@@AAEXAAVU2OpStatus@3@@Z$0 1001c530 f   SamtoolMpileupWorker.obj
 0001:0001b539       __unwindfunclet$?checkState@CallVariantsWorker@LocalWorkflow@U2@@AAEXAAVU2OpStatus@3@@Z$1 1001c539 f   SamtoolMpileupWorker.obj
 0001:0001b542       __unwindfunclet$?checkState@CallVariantsWorker@LocalWorkflow@U2@@AAEXAAVU2OpStatus@3@@Z$2 1001c542 f   SamtoolMpileupWorker.obj
 0001:0001b54b       __ehhandler$?checkState@CallVariantsWorker@LocalWorkflow@U2@@AAEXAAVU2OpStatus@3@@Z 1001c54b f   SamtoolMpileupWorker.obj
 0001:0001b570       __unwindfunclet$?clone@ScientificDoubleDelegate@LocalWorkflow@U2@@UAEPAVPropertyDelegate@3@XZ$0 1001c570 f   SamtoolMpileupWorker.obj
 0001:0001b57b       __ehhandler$?clone@ScientificDoubleDelegate@LocalWorkflow@U2@@UAEPAVPropertyDelegate@3@XZ 1001c57b f   SamtoolMpileupWorker.obj
 0001:0001b5a0       __unwindfunclet$?composeRichDoc@CallVariantsPrompter@LocalWorkflow@U2@@MAE?AVQString@@XZ$0 1001c5a0 f   SamtoolMpileupWorker.obj
 0001:0001b5a9       __unwindfunclet$?composeRichDoc@CallVariantsPrompter@LocalWorkflow@U2@@MAE?AVQString@@XZ$1 1001c5a9 f   SamtoolMpileupWorker.obj
 0001:0001b5b2       __unwindfunclet$?composeRichDoc@CallVariantsPrompter@LocalWorkflow@U2@@MAE?AVQString@@XZ$2 1001c5b2 f   SamtoolMpileupWorker.obj
 0001:0001b5bb       __unwindfunclet$?composeRichDoc@CallVariantsPrompter@LocalWorkflow@U2@@MAE?AVQString@@XZ$3 1001c5bb f   SamtoolMpileupWorker.obj
 0001:0001b5c4       __unwindfunclet$?composeRichDoc@CallVariantsPrompter@LocalWorkflow@U2@@MAE?AVQString@@XZ$4 1001c5c4 f   SamtoolMpileupWorker.obj
 0001:0001b5cd       __unwindfunclet$?composeRichDoc@CallVariantsPrompter@LocalWorkflow@U2@@MAE?AVQString@@XZ$5 1001c5cd f   SamtoolMpileupWorker.obj
 0001:0001b5d6       __unwindfunclet$?composeRichDoc@CallVariantsPrompter@LocalWorkflow@U2@@MAE?AVQString@@XZ$6 1001c5d6 f   SamtoolMpileupWorker.obj
 0001:0001b5df       __unwindfunclet$?composeRichDoc@CallVariantsPrompter@LocalWorkflow@U2@@MAE?AVQString@@XZ$7 1001c5df f   SamtoolMpileupWorker.obj
 0001:0001b5f9       __unwindfunclet$?composeRichDoc@CallVariantsPrompter@LocalWorkflow@U2@@MAE?AVQString@@XZ$8 1001c5f9 f   SamtoolMpileupWorker.obj
 0001:0001b613       __unwindfunclet$?composeRichDoc@CallVariantsPrompter@LocalWorkflow@U2@@MAE?AVQString@@XZ$9 1001c613 f   SamtoolMpileupWorker.obj
 0001:0001b61c       __unwindfunclet$?composeRichDoc@CallVariantsPrompter@LocalWorkflow@U2@@MAE?AVQString@@XZ$10 1001c61c f   SamtoolMpileupWorker.obj
 0001:0001b625       __unwindfunclet$?composeRichDoc@CallVariantsPrompter@LocalWorkflow@U2@@MAE?AVQString@@XZ$11 1001c625 f   SamtoolMpileupWorker.obj
 0001:0001b62e       __unwindfunclet$?composeRichDoc@CallVariantsPrompter@LocalWorkflow@U2@@MAE?AVQString@@XZ$12 1001c62e f   SamtoolMpileupWorker.obj
 0001:0001b637       __unwindfunclet$?composeRichDoc@CallVariantsPrompter@LocalWorkflow@U2@@MAE?AVQString@@XZ$13 1001c637 f   SamtoolMpileupWorker.obj
 0001:0001b640       __unwindfunclet$?composeRichDoc@CallVariantsPrompter@LocalWorkflow@U2@@MAE?AVQString@@XZ$14 1001c640 f   SamtoolMpileupWorker.obj
 0001:0001b649       __unwindfunclet$?composeRichDoc@CallVariantsPrompter@LocalWorkflow@U2@@MAE?AVQString@@XZ$15 1001c649 f   SamtoolMpileupWorker.obj
 0001:0001b652       __unwindfunclet$?composeRichDoc@CallVariantsPrompter@LocalWorkflow@U2@@MAE?AVQString@@XZ$16 1001c652 f   SamtoolMpileupWorker.obj
 0001:0001b65b       __unwindfunclet$?composeRichDoc@CallVariantsPrompter@LocalWorkflow@U2@@MAE?AVQString@@XZ$17 1001c65b f   SamtoolMpileupWorker.obj
 0001:0001b664       __unwindfunclet$?composeRichDoc@CallVariantsPrompter@LocalWorkflow@U2@@MAE?AVQString@@XZ$18 1001c664 f   SamtoolMpileupWorker.obj
 0001:0001b67e       __unwindfunclet$?composeRichDoc@CallVariantsPrompter@LocalWorkflow@U2@@MAE?AVQString@@XZ$19 1001c67e f   SamtoolMpileupWorker.obj
 0001:0001b698       __unwindfunclet$?composeRichDoc@CallVariantsPrompter@LocalWorkflow@U2@@MAE?AVQString@@XZ$20 1001c698 f   SamtoolMpileupWorker.obj
 0001:0001b6a1       __unwindfunclet$?composeRichDoc@CallVariantsPrompter@LocalWorkflow@U2@@MAE?AVQString@@XZ$21 1001c6a1 f   SamtoolMpileupWorker.obj
 0001:0001b6aa       __unwindfunclet$?composeRichDoc@CallVariantsPrompter@LocalWorkflow@U2@@MAE?AVQString@@XZ$22 1001c6aa f   SamtoolMpileupWorker.obj
 0001:0001b6b3       __unwindfunclet$?composeRichDoc@CallVariantsPrompter@LocalWorkflow@U2@@MAE?AVQString@@XZ$23 1001c6b3 f   SamtoolMpileupWorker.obj
 0001:0001b6bc       __unwindfunclet$?composeRichDoc@CallVariantsPrompter@LocalWorkflow@U2@@MAE?AVQString@@XZ$24 1001c6bc f   SamtoolMpileupWorker.obj
 0001:0001b6d6       __ehhandler$?composeRichDoc@CallVariantsPrompter@LocalWorkflow@U2@@MAE?AVQString@@XZ 1001c6d6 f   SamtoolMpileupWorker.obj
 0001:0001b700       __unwindfunclet$?createDescription@?$PrompterBase@VCallVariantsPrompter@LocalWorkflow@U2@@@U2@@UAEPAVActorDocument@Workflow@2@PAVActor@42@@Z$0 1001c700 f   SamtoolMpileupWorker.obj
 0001:0001b70b       __unwindfunclet$?createDescription@?$PrompterBase@VCallVariantsPrompter@LocalWorkflow@U2@@@U2@@UAEPAVActorDocument@Workflow@2@PAVActor@42@@Z$3 1001c70b f   SamtoolMpileupWorker.obj
 0001:0001b713       __unwindfunclet$?createDescription@?$PrompterBase@VCallVariantsPrompter@LocalWorkflow@U2@@@U2@@UAEPAVActorDocument@Workflow@2@PAVActor@42@@Z$4 1001c713 f   SamtoolMpileupWorker.obj
 0001:0001b71b       __unwindfunclet$?createDescription@?$PrompterBase@VCallVariantsPrompter@LocalWorkflow@U2@@@U2@@UAEPAVActorDocument@Workflow@2@PAVActor@42@@Z$6 1001c71b f   SamtoolMpileupWorker.obj
 0001:0001b723       __unwindfunclet$?createDescription@?$PrompterBase@VCallVariantsPrompter@LocalWorkflow@U2@@@U2@@UAEPAVActorDocument@Workflow@2@PAVActor@42@@Z$7 1001c723 f   SamtoolMpileupWorker.obj
 0001:0001b72b       __ehhandler$?createDescription@?$PrompterBase@VCallVariantsPrompter@LocalWorkflow@U2@@@U2@@UAEPAVActorDocument@Workflow@2@PAVActor@42@@Z 1001c72b f   SamtoolMpileupWorker.obj
 0001:0001b750       __unwindfunclet$?createEditor@ScientificDoubleDelegate@LocalWorkflow@U2@@UBEPAVQWidget@@PAV4@ABVQStyleOptionViewItem@@ABVQModelIndex@@@Z$0 1001c750 f   SamtoolMpileupWorker.obj
 0001:0001b75b       __ehhandler$?createEditor@ScientificDoubleDelegate@LocalWorkflow@U2@@UBEPAVQWidget@@PAV4@ABVQStyleOptionViewItem@@ABVQModelIndex@@@Z 1001c75b f   SamtoolMpileupWorker.obj
 0001:0001b780       __unwindfunclet$?createNode@?$QMapData@VDescriptor@U2@@V?$QExplicitlySharedDataPointer@VDataType@U2@@@@@@QAEPAU?$QMapNode@VDescriptor@U2@@V?$QExplicitlySharedDataPointer@VDataType@U2@@@@@@ABVDescriptor@U2@@ABV?$QExplicitlySharedDataPointer@VDataType@U2@@@@PAU2@_N@Z$4 1001c780 f   SamtoolMpileupWorker.obj
 0001:0001b794       __ehhandler$?createNode@?$QMapData@VDescriptor@U2@@V?$QExplicitlySharedDataPointer@VDataType@U2@@@@@@QAEPAU?$QMapNode@VDescriptor@U2@@V?$QExplicitlySharedDataPointer@VDataType@U2@@@@@@ABVDescriptor@U2@@ABV?$QExplicitlySharedDataPointer@VDataType@U2@@@@PAU2@_N@Z 1001c794 f   SamtoolMpileupWorker.obj
 0001:0001b7b0       __unwindfunclet$?createNode@?$QMapData@VQString@@PAVPropertyDelegate@U2@@@@QAEPAU?$QMapNode@VQString@@PAVPropertyDelegate@U2@@@@ABVQString@@ABQAVPropertyDelegate@U2@@PAU2@_N@Z$4 1001c7b0 f   SamtoolMpileupWorker.obj
 0001:0001b7c4       __ehhandler$?createNode@?$QMapData@VQString@@PAVPropertyDelegate@U2@@@@QAEPAU?$QMapNode@VQString@@PAVPropertyDelegate@U2@@@@ABVQString@@ABQAVPropertyDelegate@U2@@PAU2@_N@Z 1001c7c4 f   SamtoolMpileupWorker.obj
 0001:0001b7e0       __unwindfunclet$?createNode@?$QMapData@VQString@@V1@@@QAEPAU?$QMapNode@VQString@@V1@@@ABVQString@@0PAU2@_N@Z$4 1001c7e0 f   SamtoolMpileupWorker.obj
 0001:0001b7f4       __unwindfunclet$?createNode@?$QMapData@VQString@@V1@@@QAEPAU?$QMapNode@VQString@@V1@@@ABVQString@@0PAU2@_N@Z$5 1001c7f4 f   SamtoolMpileupWorker.obj
 0001:0001b808       __ehhandler$?createNode@?$QMapData@VQString@@V1@@@QAEPAU?$QMapNode@VQString@@V1@@@ABVQString@@0PAU2@_N@Z 1001c808 f   SamtoolMpileupWorker.obj
 0001:0001b830       __unwindfunclet$?createNode@?$QMapData@VQString@@VQScriptValue@@@@QAEPAU?$QMapNode@VQString@@VQScriptValue@@@@ABVQString@@ABVQScriptValue@@PAU2@_N@Z$4 1001c830 f   SamtoolMpileupWorker.obj
 0001:0001b844       __unwindfunclet$?createNode@?$QMapData@VQString@@VQScriptValue@@@@QAEPAU?$QMapNode@VQString@@VQScriptValue@@@@ABVQString@@ABVQScriptValue@@PAU2@_N@Z$5 1001c844 f   SamtoolMpileupWorker.obj
 0001:0001b858       __ehhandler$?createNode@?$QMapData@VQString@@VQScriptValue@@@@QAEPAU?$QMapNode@VQString@@VQScriptValue@@@@ABVQString@@ABVQScriptValue@@PAU2@_N@Z 1001c858 f   SamtoolMpileupWorker.obj
 0001:0001b880       __unwindfunclet$?createWizardWidget@ScientificDoubleDelegate@LocalWorkflow@U2@@UBEPAVPropertyWidget@3@AAVU2OpStatus@3@PAVQWidget@@@Z$0 1001c880 f   SamtoolMpileupWorker.obj
 0001:0001b88b       __ehhandler$?createWizardWidget@ScientificDoubleDelegate@LocalWorkflow@U2@@UBEPAVPropertyWidget@3@AAVU2OpStatus@3@PAVQWidget@@@Z 1001c88b f   SamtoolMpileupWorker.obj
 0001:0001b8b0       __unwindfunclet$?createWorker@CallVariantsWorkerFactory@LocalWorkflow@U2@@UAEPAVWorker@Workflow@3@PAVActor@53@@Z$0 1001c8b0 f   SamtoolMpileupWorker.obj
 0001:0001b8bb       __ehhandler$?createWorker@CallVariantsWorkerFactory@LocalWorkflow@U2@@UAEPAVWorker@Workflow@3@PAVActor@53@@Z 1001c8bb f   SamtoolMpileupWorker.obj
 0001:0001b8e0       __ehhandler$?detach_helper@?$QList@VDescriptor@U2@@@@AAEXH@Z 1001c8e0 f   SamtoolMpileupWorker.obj
 0001:0001b900       __ehhandler$?detach_helper@?$QList@VMessage@Workflow@U2@@@@AAEXH@Z 1001c900 f   SamtoolMpileupWorker.obj
 0001:0001b920       __ehhandler$?detach_helper_grow@?$QList@PAVAttribute@U2@@@@AAEPAUNode@1@HH@Z 1001c920 f   SamtoolMpileupWorker.obj
 0001:0001b940       __ehhandler$?detach_helper_grow@?$QList@PAVPortDescriptor@Workflow@U2@@@@AAEPAUNode@1@HH@Z 1001c940 f   SamtoolMpileupWorker.obj
 0001:0001b960       __ehhandler$?detach_helper_grow@?$QList@VDescriptor@U2@@@@AAEPAUNode@1@HH@Z 1001c960 f   SamtoolMpileupWorker.obj
 0001:0001b980       __ehhandler$?detach_helper_grow@?$QList@VMessage@Workflow@U2@@@@AAEPAUNode@1@HH@Z 1001c980 f   SamtoolMpileupWorker.obj
 0001:0001b9a0       __ehhandler$?detach_helper_grow@?$QList@VQVariant@@@@AAEPAUNode@1@HH@Z 1001c9a0 f   SamtoolMpileupWorker.obj
 0001:0001b9c0       __ehhandler$?detach_helper_grow@?$QList@VWorkflowNotification@U2@@@@AAEPAUNode@1@HH@Z 1001c9c0 f   SamtoolMpileupWorker.obj
 0001:0001b9e0       __unwindfunclet$?getSettings@CallVariantsWorker@LocalWorkflow@U2@@AAE?AVCallVariantsTaskSettings@23@XZ$0 1001c9e0 f   SamtoolMpileupWorker.obj
 0001:0001b9f9       __unwindfunclet$?getSettings@CallVariantsWorker@LocalWorkflow@U2@@AAE?AVCallVariantsTaskSettings@23@XZ$1 1001c9f9 f   SamtoolMpileupWorker.obj
 0001:0001ba02       __unwindfunclet$?getSettings@CallVariantsWorker@LocalWorkflow@U2@@AAE?AVCallVariantsTaskSettings@23@XZ$2 1001ca02 f   SamtoolMpileupWorker.obj
 0001:0001ba0b       __unwindfunclet$?getSettings@CallVariantsWorker@LocalWorkflow@U2@@AAE?AVCallVariantsTaskSettings@23@XZ$3 1001ca0b f   SamtoolMpileupWorker.obj
 0001:0001ba14       __unwindfunclet$?getSettings@CallVariantsWorker@LocalWorkflow@U2@@AAE?AVCallVariantsTaskSettings@23@XZ$4 1001ca14 f   SamtoolMpileupWorker.obj
 0001:0001ba1d       __unwindfunclet$?getSettings@CallVariantsWorker@LocalWorkflow@U2@@AAE?AVCallVariantsTaskSettings@23@XZ$5 1001ca1d f   SamtoolMpileupWorker.obj
 0001:0001ba26       __unwindfunclet$?getSettings@CallVariantsWorker@LocalWorkflow@U2@@AAE?AVCallVariantsTaskSettings@23@XZ$6 1001ca26 f   SamtoolMpileupWorker.obj
 0001:0001ba2f       __unwindfunclet$?getSettings@CallVariantsWorker@LocalWorkflow@U2@@AAE?AVCallVariantsTaskSettings@23@XZ$7 1001ca2f f   SamtoolMpileupWorker.obj
 0001:0001ba38       __unwindfunclet$?getSettings@CallVariantsWorker@LocalWorkflow@U2@@AAE?AVCallVariantsTaskSettings@23@XZ$8 1001ca38 f   SamtoolMpileupWorker.obj
 0001:0001ba41       __unwindfunclet$?getSettings@CallVariantsWorker@LocalWorkflow@U2@@AAE?AVCallVariantsTaskSettings@23@XZ$9 1001ca41 f   SamtoolMpileupWorker.obj
 0001:0001ba4a       __unwindfunclet$?getSettings@CallVariantsWorker@LocalWorkflow@U2@@AAE?AVCallVariantsTaskSettings@23@XZ$10 1001ca4a f   SamtoolMpileupWorker.obj
 0001:0001ba53       __unwindfunclet$?getSettings@CallVariantsWorker@LocalWorkflow@U2@@AAE?AVCallVariantsTaskSettings@23@XZ$11 1001ca53 f   SamtoolMpileupWorker.obj
 0001:0001ba5c       __unwindfunclet$?getSettings@CallVariantsWorker@LocalWorkflow@U2@@AAE?AVCallVariantsTaskSettings@23@XZ$12 1001ca5c f   SamtoolMpileupWorker.obj
 0001:0001ba65       __unwindfunclet$?getSettings@CallVariantsWorker@LocalWorkflow@U2@@AAE?AVCallVariantsTaskSettings@23@XZ$13 1001ca65 f   SamtoolMpileupWorker.obj
 0001:0001ba6e       __unwindfunclet$?getSettings@CallVariantsWorker@LocalWorkflow@U2@@AAE?AVCallVariantsTaskSettings@23@XZ$14 1001ca6e f   SamtoolMpileupWorker.obj
 0001:0001ba77       __unwindfunclet$?getSettings@CallVariantsWorker@LocalWorkflow@U2@@AAE?AVCallVariantsTaskSettings@23@XZ$15 1001ca77 f   SamtoolMpileupWorker.obj
 0001:0001ba80       __ehhandler$?getSettings@CallVariantsWorker@LocalWorkflow@U2@@AAE?AVCallVariantsTaskSettings@23@XZ 1001ca80 f   SamtoolMpileupWorker.obj
 0001:0001baa0       __unwindfunclet$?init@CallVariantsWorker@LocalWorkflow@U2@@UAEXXZ$0 1001caa0 f   SamtoolMpileupWorker.obj
 0001:0001baa9       __unwindfunclet$?init@CallVariantsWorker@LocalWorkflow@U2@@UAEXXZ$1 1001caa9 f   SamtoolMpileupWorker.obj
 0001:0001bab2       __unwindfunclet$?init@CallVariantsWorker@LocalWorkflow@U2@@UAEXXZ$2 1001cab2 f   SamtoolMpileupWorker.obj
 0001:0001babb       __unwindfunclet$?init@CallVariantsWorker@LocalWorkflow@U2@@UAEXXZ$3 1001cabb f   SamtoolMpileupWorker.obj
 0001:0001bac4       __unwindfunclet$?init@CallVariantsWorker@LocalWorkflow@U2@@UAEXXZ$4 1001cac4 f   SamtoolMpileupWorker.obj
 0001:0001bacf       __ehhandler$?init@CallVariantsWorker@LocalWorkflow@U2@@UAEXXZ 1001cacf f   SamtoolMpileupWorker.obj
 0001:0001bb20       __unwindfunclet$?init@CallVariantsWorkerFactory@LocalWorkflow@U2@@SAXXZ$0 1001cb20 f   SamtoolMpileupWorker.obj
 0001:0001bb28       __unwindfunclet$?init@CallVariantsWorkerFactory@LocalWorkflow@U2@@SAXXZ$1 1001cb28 f   SamtoolMpileupWorker.obj
 0001:0001bb30       __unwindfunclet$?init@CallVariantsWorkerFactory@LocalWorkflow@U2@@SAXXZ$2 1001cb30 f   SamtoolMpileupWorker.obj
 0001:0001bb38       __unwindfunclet$?init@CallVariantsWorkerFactory@LocalWorkflow@U2@@SAXXZ$3 1001cb38 f   SamtoolMpileupWorker.obj
 0001:0001bb44       __unwindfunclet$?init@CallVariantsWorkerFactory@LocalWorkflow@U2@@SAXXZ$4 1001cb44 f   SamtoolMpileupWorker.obj
 0001:0001bb52       __unwindfunclet$?init@CallVariantsWorkerFactory@LocalWorkflow@U2@@SAXXZ$5 1001cb52 f   SamtoolMpileupWorker.obj
 0001:0001bb6f       __unwindfunclet$?init@CallVariantsWorkerFactory@LocalWorkflow@U2@@SAXXZ$6 1001cb6f f   SamtoolMpileupWorker.obj
 0001:0001bb7a       __unwindfunclet$?init@CallVariantsWorkerFactory@LocalWorkflow@U2@@SAXXZ$7 1001cb7a f   SamtoolMpileupWorker.obj
 0001:0001bb86       __unwindfunclet$?init@CallVariantsWorkerFactory@LocalWorkflow@U2@@SAXXZ$8 1001cb86 f   SamtoolMpileupWorker.obj
 0001:0001bb92       __unwindfunclet$?init@CallVariantsWorkerFactory@LocalWorkflow@U2@@SAXXZ$9 1001cb92 f   SamtoolMpileupWorker.obj
 0001:0001bb9e       __unwindfunclet$?init@CallVariantsWorkerFactory@LocalWorkflow@U2@@SAXXZ$10 1001cb9e f   SamtoolMpileupWorker.obj
 0001:0001bba7       __unwindfunclet$?init@CallVariantsWorkerFactory@LocalWorkflow@U2@@SAXXZ$11 1001cba7 f   SamtoolMpileupWorker.obj
 0001:0001bbb2       __unwindfunclet$?init@CallVariantsWorkerFactory@LocalWorkflow@U2@@SAXXZ$13 1001cbb2 f   SamtoolMpileupWorker.obj
 0001:0001bbba       __unwindfunclet$?init@CallVariantsWorkerFactory@LocalWorkflow@U2@@SAXXZ$14 1001cbba f   SamtoolMpileupWorker.obj
 0001:0001bbc2       __unwindfunclet$?init@CallVariantsWorkerFactory@LocalWorkflow@U2@@SAXXZ$15 1001cbc2 f   SamtoolMpileupWorker.obj
 0001:0001bbce       __unwindfunclet$?init@CallVariantsWorkerFactory@LocalWorkflow@U2@@SAXXZ$16 1001cbce f   SamtoolMpileupWorker.obj
 0001:0001bbd6       __unwindfunclet$?init@CallVariantsWorkerFactory@LocalWorkflow@U2@@SAXXZ$17 1001cbd6 f   SamtoolMpileupWorker.obj
 0001:0001bbe2       __unwindfunclet$?init@CallVariantsWorkerFactory@LocalWorkflow@U2@@SAXXZ$18 1001cbe2 f   SamtoolMpileupWorker.obj
 0001:0001bbed       __unwindfunclet$?init@CallVariantsWorkerFactory@LocalWorkflow@U2@@SAXXZ$19 1001cbed f   SamtoolMpileupWorker.obj
 0001:0001bc0a       __unwindfunclet$?init@CallVariantsWorkerFactory@LocalWorkflow@U2@@SAXXZ$20 1001cc0a f   SamtoolMpileupWorker.obj
 0001:0001bc12       __unwindfunclet$?init@CallVariantsWorkerFactory@LocalWorkflow@U2@@SAXXZ$21 1001cc12 f   SamtoolMpileupWorker.obj
 0001:0001bc1e       __unwindfunclet$?init@CallVariantsWorkerFactory@LocalWorkflow@U2@@SAXXZ$22 1001cc1e f   SamtoolMpileupWorker.obj
 0001:0001bc2a       __unwindfunclet$?init@CallVariantsWorkerFactory@LocalWorkflow@U2@@SAXXZ$23 1001cc2a f   SamtoolMpileupWorker.obj
 0001:0001bc36       __unwindfunclet$?init@CallVariantsWorkerFactory@LocalWorkflow@U2@@SAXXZ$24 1001cc36 f   SamtoolMpileupWorker.obj
 0001:0001bc3f       __unwindfunclet$?init@CallVariantsWorkerFactory@LocalWorkflow@U2@@SAXXZ$25 1001cc3f f   SamtoolMpileupWorker.obj
 0001:0001bc4a       __unwindfunclet$?init@CallVariantsWorkerFactory@LocalWorkflow@U2@@SAXXZ$27 1001cc4a f   SamtoolMpileupWorker.obj
 0001:0001bc52       __unwindfunclet$?init@CallVariantsWorkerFactory@LocalWorkflow@U2@@SAXXZ$28 1001cc52 f   SamtoolMpileupWorker.obj
 0001:0001bc5a       __unwindfunclet$?init@CallVariantsWorkerFactory@LocalWorkflow@U2@@SAXXZ$29 1001cc5a f   SamtoolMpileupWorker.obj
 0001:0001bc66       __unwindfunclet$?init@CallVariantsWorkerFactory@LocalWorkflow@U2@@SAXXZ$30 1001cc66 f   SamtoolMpileupWorker.obj
 0001:0001bc6e       __unwindfunclet$?init@CallVariantsWorkerFactory@LocalWorkflow@U2@@SAXXZ$31 1001cc6e f   SamtoolMpileupWorker.obj
 0001:0001bc7a       __unwindfunclet$?init@CallVariantsWorkerFactory@LocalWorkflow@U2@@SAXXZ$32 1001cc7a f   SamtoolMpileupWorker.obj
 0001:0001bc85       __unwindfunclet$?init@CallVariantsWorkerFactory@LocalWorkflow@U2@@SAXXZ$33 1001cc85 f   SamtoolMpileupWorker.obj
 0001:0001bca2       __unwindfunclet$?init@CallVariantsWorkerFactory@LocalWorkflow@U2@@SAXXZ$34 1001cca2 f   SamtoolMpileupWorker.obj
 0001:0001bcaa       __unwindfunclet$?init@CallVariantsWorkerFactory@LocalWorkflow@U2@@SAXXZ$35 1001ccaa f   SamtoolMpileupWorker.obj
 0001:0001bcb6       __unwindfunclet$?init@CallVariantsWorkerFactory@LocalWorkflow@U2@@SAXXZ$36 1001ccb6 f   SamtoolMpileupWorker.obj
 0001:0001bcc2       __unwindfunclet$?init@CallVariantsWorkerFactory@LocalWorkflow@U2@@SAXXZ$37 1001ccc2 f   SamtoolMpileupWorker.obj
 0001:0001bcce       __unwindfunclet$?init@CallVariantsWorkerFactory@LocalWorkflow@U2@@SAXXZ$38 1001ccce f   SamtoolMpileupWorker.obj
 0001:0001bcd7       __unwindfunclet$?init@CallVariantsWorkerFactory@LocalWorkflow@U2@@SAXXZ$39 1001ccd7 f   SamtoolMpileupWorker.obj
 0001:0001bce5       __unwindfunclet$?init@CallVariantsWorkerFactory@LocalWorkflow@U2@@SAXXZ$41 1001cce5 f   SamtoolMpileupWorker.obj
 0001:0001bcf1       __unwindfunclet$?init@CallVariantsWorkerFactory@LocalWorkflow@U2@@SAXXZ$42 1001ccf1 f   SamtoolMpileupWorker.obj
 0001:0001bcfd       __unwindfunclet$?init@CallVariantsWorkerFactory@LocalWorkflow@U2@@SAXXZ$43 1001ccfd f   SamtoolMpileupWorker.obj
 0001:0001bd09       __unwindfunclet$?init@CallVariantsWorkerFactory@LocalWorkflow@U2@@SAXXZ$44 1001cd09 f   SamtoolMpileupWorker.obj
 0001:0001bd11       __unwindfunclet$?init@CallVariantsWorkerFactory@LocalWorkflow@U2@@SAXXZ$45 1001cd11 f   SamtoolMpileupWorker.obj
 0001:0001bd1d       __unwindfunclet$?init@CallVariantsWorkerFactory@LocalWorkflow@U2@@SAXXZ$46 1001cd1d f   SamtoolMpileupWorker.obj
 0001:0001bd29       __unwindfunclet$?init@CallVariantsWorkerFactory@LocalWorkflow@U2@@SAXXZ$47 1001cd29 f   SamtoolMpileupWorker.obj
 0001:0001bd35       __unwindfunclet$?init@CallVariantsWorkerFactory@LocalWorkflow@U2@@SAXXZ$48 1001cd35 f   SamtoolMpileupWorker.obj
 0001:0001bd41       __unwindfunclet$?init@CallVariantsWorkerFactory@LocalWorkflow@U2@@SAXXZ$49 1001cd41 f   SamtoolMpileupWorker.obj
 0001:0001bd4d       __unwindfunclet$?init@CallVariantsWorkerFactory@LocalWorkflow@U2@@SAXXZ$50 1001cd4d f   SamtoolMpileupWorker.obj
 0001:0001bd59       __unwindfunclet$?init@CallVariantsWorkerFactory@LocalWorkflow@U2@@SAXXZ$51 1001cd59 f   SamtoolMpileupWorker.obj
 0001:0001bd65       __unwindfunclet$?init@CallVariantsWorkerFactory@LocalWorkflow@U2@@SAXXZ$52 1001cd65 f   SamtoolMpileupWorker.obj
 0001:0001bd71       __unwindfunclet$?init@CallVariantsWorkerFactory@LocalWorkflow@U2@@SAXXZ$53 1001cd71 f   SamtoolMpileupWorker.obj
 0001:0001bd7d       __unwindfunclet$?init@CallVariantsWorkerFactory@LocalWorkflow@U2@@SAXXZ$54 1001cd7d f   SamtoolMpileupWorker.obj
 0001:0001bd89       __unwindfunclet$?init@CallVariantsWorkerFactory@LocalWorkflow@U2@@SAXXZ$55 1001cd89 f   SamtoolMpileupWorker.obj
 0001:0001bd95       __unwindfunclet$?init@CallVariantsWorkerFactory@LocalWorkflow@U2@@SAXXZ$56 1001cd95 f   SamtoolMpileupWorker.obj
 0001:0001bda1       __unwindfunclet$?init@CallVariantsWorkerFactory@LocalWorkflow@U2@@SAXXZ$57 1001cda1 f   SamtoolMpileupWorker.obj
 0001:0001bdad       __unwindfunclet$?init@CallVariantsWorkerFactory@LocalWorkflow@U2@@SAXXZ$58 1001cdad f   SamtoolMpileupWorker.obj
 0001:0001bdb9       __unwindfunclet$?init@CallVariantsWorkerFactory@LocalWorkflow@U2@@SAXXZ$59 1001cdb9 f   SamtoolMpileupWorker.obj
 0001:0001bdc5       __unwindfunclet$?init@CallVariantsWorkerFactory@LocalWorkflow@U2@@SAXXZ$60 1001cdc5 f   SamtoolMpileupWorker.obj
 0001:0001bdd1       __unwindfunclet$?init@CallVariantsWorkerFactory@LocalWorkflow@U2@@SAXXZ$61 1001cdd1 f   SamtoolMpileupWorker.obj
 0001:0001bddd       __unwindfunclet$?init@CallVariantsWorkerFactory@LocalWorkflow@U2@@SAXXZ$62 1001cddd f   SamtoolMpileupWorker.obj
 0001:0001bde9       __unwindfunclet$?init@CallVariantsWorkerFactory@LocalWorkflow@U2@@SAXXZ$63 1001cde9 f   SamtoolMpileupWorker.obj
 0001:0001bdf5       __unwindfunclet$?init@CallVariantsWorkerFactory@LocalWorkflow@U2@@SAXXZ$64 1001cdf5 f   SamtoolMpileupWorker.obj
 0001:0001be01       __unwindfunclet$?init@CallVariantsWorkerFactory@LocalWorkflow@U2@@SAXXZ$65 1001ce01 f   SamtoolMpileupWorker.obj
 0001:0001be0d       __unwindfunclet$?init@CallVariantsWorkerFactory@LocalWorkflow@U2@@SAXXZ$66 1001ce0d f   SamtoolMpileupWorker.obj
 0001:0001be19       __unwindfunclet$?init@CallVariantsWorkerFactory@LocalWorkflow@U2@@SAXXZ$67 1001ce19 f   SamtoolMpileupWorker.obj
 0001:0001be25       __unwindfunclet$?init@CallVariantsWorkerFactory@LocalWorkflow@U2@@SAXXZ$68 1001ce25 f   SamtoolMpileupWorker.obj
 0001:0001be31       __unwindfunclet$?init@CallVariantsWorkerFactory@LocalWorkflow@U2@@SAXXZ$69 1001ce31 f   SamtoolMpileupWorker.obj
 0001:0001be3d       __unwindfunclet$?init@CallVariantsWorkerFactory@LocalWorkflow@U2@@SAXXZ$70 1001ce3d f   SamtoolMpileupWorker.obj
 0001:0001be49       __unwindfunclet$?init@CallVariantsWorkerFactory@LocalWorkflow@U2@@SAXXZ$71 1001ce49 f   SamtoolMpileupWorker.obj
 0001:0001be55       __unwindfunclet$?init@CallVariantsWorkerFactory@LocalWorkflow@U2@@SAXXZ$72 1001ce55 f   SamtoolMpileupWorker.obj
 0001:0001be61       __unwindfunclet$?init@CallVariantsWorkerFactory@LocalWorkflow@U2@@SAXXZ$73 1001ce61 f   SamtoolMpileupWorker.obj
 0001:0001be6d       __unwindfunclet$?init@CallVariantsWorkerFactory@LocalWorkflow@U2@@SAXXZ$74 1001ce6d f   SamtoolMpileupWorker.obj
 0001:0001be79       __unwindfunclet$?init@CallVariantsWorkerFactory@LocalWorkflow@U2@@SAXXZ$75 1001ce79 f   SamtoolMpileupWorker.obj
 0001:0001be85       __unwindfunclet$?init@CallVariantsWorkerFactory@LocalWorkflow@U2@@SAXXZ$76 1001ce85 f   SamtoolMpileupWorker.obj
 0001:0001be91       __unwindfunclet$?init@CallVariantsWorkerFactory@LocalWorkflow@U2@@SAXXZ$77 1001ce91 f   SamtoolMpileupWorker.obj
 0001:0001be9d       __unwindfunclet$?init@CallVariantsWorkerFactory@LocalWorkflow@U2@@SAXXZ$78 1001ce9d f   SamtoolMpileupWorker.obj
 0001:0001bea9       __unwindfunclet$?init@CallVariantsWorkerFactory@LocalWorkflow@U2@@SAXXZ$79 1001cea9 f   SamtoolMpileupWorker.obj
 0001:0001beb5       __unwindfunclet$?init@CallVariantsWorkerFactory@LocalWorkflow@U2@@SAXXZ$80 1001ceb5 f   SamtoolMpileupWorker.obj
 0001:0001bec1       __unwindfunclet$?init@CallVariantsWorkerFactory@LocalWorkflow@U2@@SAXXZ$81 1001cec1 f   SamtoolMpileupWorker.obj
 0001:0001becd       __unwindfunclet$?init@CallVariantsWorkerFactory@LocalWorkflow@U2@@SAXXZ$82 1001cecd f   SamtoolMpileupWorker.obj
 0001:0001bed9       __unwindfunclet$?init@CallVariantsWorkerFactory@LocalWorkflow@U2@@SAXXZ$83 1001ced9 f   SamtoolMpileupWorker.obj
 0001:0001bee5       __unwindfunclet$?init@CallVariantsWorkerFactory@LocalWorkflow@U2@@SAXXZ$84 1001cee5 f   SamtoolMpileupWorker.obj
 0001:0001bef1       __unwindfunclet$?init@CallVariantsWorkerFactory@LocalWorkflow@U2@@SAXXZ$85 1001cef1 f   SamtoolMpileupWorker.obj
 0001:0001befd       __unwindfunclet$?init@CallVariantsWorkerFactory@LocalWorkflow@U2@@SAXXZ$86 1001cefd f   SamtoolMpileupWorker.obj
 0001:0001bf09       __unwindfunclet$?init@CallVariantsWorkerFactory@LocalWorkflow@U2@@SAXXZ$87 1001cf09 f   SamtoolMpileupWorker.obj
 0001:0001bf15       __unwindfunclet$?init@CallVariantsWorkerFactory@LocalWorkflow@U2@@SAXXZ$88 1001cf15 f   SamtoolMpileupWorker.obj
 0001:0001bf21       __unwindfunclet$?init@CallVariantsWorkerFactory@LocalWorkflow@U2@@SAXXZ$89 1001cf21 f   SamtoolMpileupWorker.obj
 0001:0001bf2d       __unwindfunclet$?init@CallVariantsWorkerFactory@LocalWorkflow@U2@@SAXXZ$90 1001cf2d f   SamtoolMpileupWorker.obj
 0001:0001bf39       __unwindfunclet$?init@CallVariantsWorkerFactory@LocalWorkflow@U2@@SAXXZ$91 1001cf39 f   SamtoolMpileupWorker.obj
 0001:0001bf45       __unwindfunclet$?init@CallVariantsWorkerFactory@LocalWorkflow@U2@@SAXXZ$92 1001cf45 f   SamtoolMpileupWorker.obj
 0001:0001bf51       __unwindfunclet$?init@CallVariantsWorkerFactory@LocalWorkflow@U2@@SAXXZ$93 1001cf51 f   SamtoolMpileupWorker.obj
 0001:0001bf5d       __unwindfunclet$?init@CallVariantsWorkerFactory@LocalWorkflow@U2@@SAXXZ$94 1001cf5d f   SamtoolMpileupWorker.obj
 0001:0001bf69       __unwindfunclet$?init@CallVariantsWorkerFactory@LocalWorkflow@U2@@SAXXZ$95 1001cf69 f   SamtoolMpileupWorker.obj
 0001:0001bf75       __unwindfunclet$?init@CallVariantsWorkerFactory@LocalWorkflow@U2@@SAXXZ$96 1001cf75 f   SamtoolMpileupWorker.obj
 0001:0001bf81       __unwindfunclet$?init@CallVariantsWorkerFactory@LocalWorkflow@U2@@SAXXZ$97 1001cf81 f   SamtoolMpileupWorker.obj
 0001:0001bf8d       __unwindfunclet$?init@CallVariantsWorkerFactory@LocalWorkflow@U2@@SAXXZ$98 1001cf8d f   SamtoolMpileupWorker.obj
 0001:0001bf99       __unwindfunclet$?init@CallVariantsWorkerFactory@LocalWorkflow@U2@@SAXXZ$99 1001cf99 f   SamtoolMpileupWorker.obj
 0001:0001bfa5       __unwindfunclet$?init@CallVariantsWorkerFactory@LocalWorkflow@U2@@SAXXZ$100 1001cfa5 f   SamtoolMpileupWorker.obj
 0001:0001bfb1       __unwindfunclet$?init@CallVariantsWorkerFactory@LocalWorkflow@U2@@SAXXZ$101 1001cfb1 f   SamtoolMpileupWorker.obj
 0001:0001bfbd       __unwindfunclet$?init@CallVariantsWorkerFactory@LocalWorkflow@U2@@SAXXZ$102 1001cfbd f   SamtoolMpileupWorker.obj
 0001:0001bfc9       __unwindfunclet$?init@CallVariantsWorkerFactory@LocalWorkflow@U2@@SAXXZ$103 1001cfc9 f   SamtoolMpileupWorker.obj
 0001:0001bfd5       __unwindfunclet$?init@CallVariantsWorkerFactory@LocalWorkflow@U2@@SAXXZ$104 1001cfd5 f   SamtoolMpileupWorker.obj
 0001:0001bfe1       __unwindfunclet$?init@CallVariantsWorkerFactory@LocalWorkflow@U2@@SAXXZ$105 1001cfe1 f   SamtoolMpileupWorker.obj
 0001:0001bfed       __unwindfunclet$?init@CallVariantsWorkerFactory@LocalWorkflow@U2@@SAXXZ$106 1001cfed f   SamtoolMpileupWorker.obj
 0001:0001bff9       __unwindfunclet$?init@CallVariantsWorkerFactory@LocalWorkflow@U2@@SAXXZ$107 1001cff9 f   SamtoolMpileupWorker.obj
 0001:0001c005       __unwindfunclet$?init@CallVariantsWorkerFactory@LocalWorkflow@U2@@SAXXZ$108 1001d005 f   SamtoolMpileupWorker.obj
 0001:0001c011       __unwindfunclet$?init@CallVariantsWorkerFactory@LocalWorkflow@U2@@SAXXZ$109 1001d011 f   SamtoolMpileupWorker.obj
 0001:0001c01d       __unwindfunclet$?init@CallVariantsWorkerFactory@LocalWorkflow@U2@@SAXXZ$110 1001d01d f   SamtoolMpileupWorker.obj
 0001:0001c029       __unwindfunclet$?init@CallVariantsWorkerFactory@LocalWorkflow@U2@@SAXXZ$111 1001d029 f   SamtoolMpileupWorker.obj
 0001:0001c035       __unwindfunclet$?init@CallVariantsWorkerFactory@LocalWorkflow@U2@@SAXXZ$112 1001d035 f   SamtoolMpileupWorker.obj
 0001:0001c041       __unwindfunclet$?init@CallVariantsWorkerFactory@LocalWorkflow@U2@@SAXXZ$113 1001d041 f   SamtoolMpileupWorker.obj
 0001:0001c04d       __unwindfunclet$?init@CallVariantsWorkerFactory@LocalWorkflow@U2@@SAXXZ$114 1001d04d f   SamtoolMpileupWorker.obj
 0001:0001c059       __unwindfunclet$?init@CallVariantsWorkerFactory@LocalWorkflow@U2@@SAXXZ$115 1001d059 f   SamtoolMpileupWorker.obj
 0001:0001c065       __unwindfunclet$?init@CallVariantsWorkerFactory@LocalWorkflow@U2@@SAXXZ$116 1001d065 f   SamtoolMpileupWorker.obj
 0001:0001c071       __unwindfunclet$?init@CallVariantsWorkerFactory@LocalWorkflow@U2@@SAXXZ$117 1001d071 f   SamtoolMpileupWorker.obj
 0001:0001c07d       __unwindfunclet$?init@CallVariantsWorkerFactory@LocalWorkflow@U2@@SAXXZ$118 1001d07d f   SamtoolMpileupWorker.obj
 0001:0001c089       __unwindfunclet$?init@CallVariantsWorkerFactory@LocalWorkflow@U2@@SAXXZ$119 1001d089 f   SamtoolMpileupWorker.obj
 0001:0001c095       __unwindfunclet$?init@CallVariantsWorkerFactory@LocalWorkflow@U2@@SAXXZ$120 1001d095 f   SamtoolMpileupWorker.obj
 0001:0001c0a1       __unwindfunclet$?init@CallVariantsWorkerFactory@LocalWorkflow@U2@@SAXXZ$121 1001d0a1 f   SamtoolMpileupWorker.obj
 0001:0001c0ad       __unwindfunclet$?init@CallVariantsWorkerFactory@LocalWorkflow@U2@@SAXXZ$122 1001d0ad f   SamtoolMpileupWorker.obj
 0001:0001c0b9       __unwindfunclet$?init@CallVariantsWorkerFactory@LocalWorkflow@U2@@SAXXZ$123 1001d0b9 f   SamtoolMpileupWorker.obj
 0001:0001c0c5       __unwindfunclet$?init@CallVariantsWorkerFactory@LocalWorkflow@U2@@SAXXZ$124 1001d0c5 f   SamtoolMpileupWorker.obj
 0001:0001c0d1       __unwindfunclet$?init@CallVariantsWorkerFactory@LocalWorkflow@U2@@SAXXZ$125 1001d0d1 f   SamtoolMpileupWorker.obj
 0001:0001c0dd       __unwindfunclet$?init@CallVariantsWorkerFactory@LocalWorkflow@U2@@SAXXZ$126 1001d0dd f   SamtoolMpileupWorker.obj
 0001:0001c0e9       __unwindfunclet$?init@CallVariantsWorkerFactory@LocalWorkflow@U2@@SAXXZ$127 1001d0e9 f   SamtoolMpileupWorker.obj
 0001:0001c0f5       __unwindfunclet$?init@CallVariantsWorkerFactory@LocalWorkflow@U2@@SAXXZ$128 1001d0f5 f   SamtoolMpileupWorker.obj
 0001:0001c101       __unwindfunclet$?init@CallVariantsWorkerFactory@LocalWorkflow@U2@@SAXXZ$129 1001d101 f   SamtoolMpileupWorker.obj
 0001:0001c10d       __unwindfunclet$?init@CallVariantsWorkerFactory@LocalWorkflow@U2@@SAXXZ$130 1001d10d f   SamtoolMpileupWorker.obj
 0001:0001c119       __unwindfunclet$?init@CallVariantsWorkerFactory@LocalWorkflow@U2@@SAXXZ$131 1001d119 f   SamtoolMpileupWorker.obj
 0001:0001c125       __unwindfunclet$?init@CallVariantsWorkerFactory@LocalWorkflow@U2@@SAXXZ$132 1001d125 f   SamtoolMpileupWorker.obj
 0001:0001c131       __unwindfunclet$?init@CallVariantsWorkerFactory@LocalWorkflow@U2@@SAXXZ$133 1001d131 f   SamtoolMpileupWorker.obj
 0001:0001c13d       __unwindfunclet$?init@CallVariantsWorkerFactory@LocalWorkflow@U2@@SAXXZ$134 1001d13d f   SamtoolMpileupWorker.obj
 0001:0001c149       __unwindfunclet$?init@CallVariantsWorkerFactory@LocalWorkflow@U2@@SAXXZ$135 1001d149 f   SamtoolMpileupWorker.obj
 0001:0001c155       __unwindfunclet$?init@CallVariantsWorkerFactory@LocalWorkflow@U2@@SAXXZ$136 1001d155 f   SamtoolMpileupWorker.obj
 0001:0001c161       __unwindfunclet$?init@CallVariantsWorkerFactory@LocalWorkflow@U2@@SAXXZ$137 1001d161 f   SamtoolMpileupWorker.obj
 0001:0001c16d       __unwindfunclet$?init@CallVariantsWorkerFactory@LocalWorkflow@U2@@SAXXZ$138 1001d16d f   SamtoolMpileupWorker.obj
 0001:0001c179       __unwindfunclet$?init@CallVariantsWorkerFactory@LocalWorkflow@U2@@SAXXZ$139 1001d179 f   SamtoolMpileupWorker.obj
 0001:0001c185       __unwindfunclet$?init@CallVariantsWorkerFactory@LocalWorkflow@U2@@SAXXZ$140 1001d185 f   SamtoolMpileupWorker.obj
 0001:0001c191       __unwindfunclet$?init@CallVariantsWorkerFactory@LocalWorkflow@U2@@SAXXZ$141 1001d191 f   SamtoolMpileupWorker.obj
 0001:0001c19d       __unwindfunclet$?init@CallVariantsWorkerFactory@LocalWorkflow@U2@@SAXXZ$142 1001d19d f   SamtoolMpileupWorker.obj
 0001:0001c1a9       __unwindfunclet$?init@CallVariantsWorkerFactory@LocalWorkflow@U2@@SAXXZ$143 1001d1a9 f   SamtoolMpileupWorker.obj
 0001:0001c1b5       __unwindfunclet$?init@CallVariantsWorkerFactory@LocalWorkflow@U2@@SAXXZ$144 1001d1b5 f   SamtoolMpileupWorker.obj
 0001:0001c1c1       __unwindfunclet$?init@CallVariantsWorkerFactory@LocalWorkflow@U2@@SAXXZ$145 1001d1c1 f   SamtoolMpileupWorker.obj
 0001:0001c1cd       __unwindfunclet$?init@CallVariantsWorkerFactory@LocalWorkflow@U2@@SAXXZ$146 1001d1cd f   SamtoolMpileupWorker.obj
 0001:0001c1d9       __unwindfunclet$?init@CallVariantsWorkerFactory@LocalWorkflow@U2@@SAXXZ$147 1001d1d9 f   SamtoolMpileupWorker.obj
 0001:0001c1e5       __unwindfunclet$?init@CallVariantsWorkerFactory@LocalWorkflow@U2@@SAXXZ$148 1001d1e5 f   SamtoolMpileupWorker.obj
 0001:0001c1f1       __unwindfunclet$?init@CallVariantsWorkerFactory@LocalWorkflow@U2@@SAXXZ$149 1001d1f1 f   SamtoolMpileupWorker.obj
 0001:0001c1fd       __unwindfunclet$?init@CallVariantsWorkerFactory@LocalWorkflow@U2@@SAXXZ$150 1001d1fd f   SamtoolMpileupWorker.obj
 0001:0001c209       __unwindfunclet$?init@CallVariantsWorkerFactory@LocalWorkflow@U2@@SAXXZ$151 1001d209 f   SamtoolMpileupWorker.obj
 0001:0001c215       __unwindfunclet$?init@CallVariantsWorkerFactory@LocalWorkflow@U2@@SAXXZ$152 1001d215 f   SamtoolMpileupWorker.obj
 0001:0001c221       __unwindfunclet$?init@CallVariantsWorkerFactory@LocalWorkflow@U2@@SAXXZ$153 1001d221 f   SamtoolMpileupWorker.obj
 0001:0001c22d       __unwindfunclet$?init@CallVariantsWorkerFactory@LocalWorkflow@U2@@SAXXZ$154 1001d22d f   SamtoolMpileupWorker.obj
 0001:0001c239       __unwindfunclet$?init@CallVariantsWorkerFactory@LocalWorkflow@U2@@SAXXZ$155 1001d239 f   SamtoolMpileupWorker.obj
 0001:0001c245       __unwindfunclet$?init@CallVariantsWorkerFactory@LocalWorkflow@U2@@SAXXZ$156 1001d245 f   SamtoolMpileupWorker.obj
 0001:0001c251       __unwindfunclet$?init@CallVariantsWorkerFactory@LocalWorkflow@U2@@SAXXZ$157 1001d251 f   SamtoolMpileupWorker.obj
 0001:0001c25d       __unwindfunclet$?init@CallVariantsWorkerFactory@LocalWorkflow@U2@@SAXXZ$158 1001d25d f   SamtoolMpileupWorker.obj
 0001:0001c269       __unwindfunclet$?init@CallVariantsWorkerFactory@LocalWorkflow@U2@@SAXXZ$159 1001d269 f   SamtoolMpileupWorker.obj
 0001:0001c275       __unwindfunclet$?init@CallVariantsWorkerFactory@LocalWorkflow@U2@@SAXXZ$160 1001d275 f   SamtoolMpileupWorker.obj
 0001:0001c281       __unwindfunclet$?init@CallVariantsWorkerFactory@LocalWorkflow@U2@@SAXXZ$161 1001d281 f   SamtoolMpileupWorker.obj
 0001:0001c28d       __unwindfunclet$?init@CallVariantsWorkerFactory@LocalWorkflow@U2@@SAXXZ$162 1001d28d f   SamtoolMpileupWorker.obj
 0001:0001c299       __unwindfunclet$?init@CallVariantsWorkerFactory@LocalWorkflow@U2@@SAXXZ$163 1001d299 f   SamtoolMpileupWorker.obj
 0001:0001c2a5       __unwindfunclet$?init@CallVariantsWorkerFactory@LocalWorkflow@U2@@SAXXZ$164 1001d2a5 f   SamtoolMpileupWorker.obj
 0001:0001c2b1       __unwindfunclet$?init@CallVariantsWorkerFactory@LocalWorkflow@U2@@SAXXZ$165 1001d2b1 f   SamtoolMpileupWorker.obj
 0001:0001c2bd       __unwindfunclet$?init@CallVariantsWorkerFactory@LocalWorkflow@U2@@SAXXZ$166 1001d2bd f   SamtoolMpileupWorker.obj
 0001:0001c2c9       __unwindfunclet$?init@CallVariantsWorkerFactory@LocalWorkflow@U2@@SAXXZ$167 1001d2c9 f   SamtoolMpileupWorker.obj
 0001:0001c2d5       __unwindfunclet$?init@CallVariantsWorkerFactory@LocalWorkflow@U2@@SAXXZ$168 1001d2d5 f   SamtoolMpileupWorker.obj
 0001:0001c2e1       __unwindfunclet$?init@CallVariantsWorkerFactory@LocalWorkflow@U2@@SAXXZ$169 1001d2e1 f   SamtoolMpileupWorker.obj
 0001:0001c2ed       __unwindfunclet$?init@CallVariantsWorkerFactory@LocalWorkflow@U2@@SAXXZ$170 1001d2ed f   SamtoolMpileupWorker.obj
 0001:0001c2f9       __unwindfunclet$?init@CallVariantsWorkerFactory@LocalWorkflow@U2@@SAXXZ$171 1001d2f9 f   SamtoolMpileupWorker.obj
 0001:0001c305       __unwindfunclet$?init@CallVariantsWorkerFactory@LocalWorkflow@U2@@SAXXZ$172 1001d305 f   SamtoolMpileupWorker.obj
 0001:0001c311       __unwindfunclet$?init@CallVariantsWorkerFactory@LocalWorkflow@U2@@SAXXZ$173 1001d311 f   SamtoolMpileupWorker.obj
 0001:0001c31d       __unwindfunclet$?init@CallVariantsWorkerFactory@LocalWorkflow@U2@@SAXXZ$174 1001d31d f   SamtoolMpileupWorker.obj
 0001:0001c329       __unwindfunclet$?init@CallVariantsWorkerFactory@LocalWorkflow@U2@@SAXXZ$175 1001d329 f   SamtoolMpileupWorker.obj
 0001:0001c335       __unwindfunclet$?init@CallVariantsWorkerFactory@LocalWorkflow@U2@@SAXXZ$176 1001d335 f   SamtoolMpileupWorker.obj
 0001:0001c341       __unwindfunclet$?init@CallVariantsWorkerFactory@LocalWorkflow@U2@@SAXXZ$177 1001d341 f   SamtoolMpileupWorker.obj
 0001:0001c34d       __unwindfunclet$?init@CallVariantsWorkerFactory@LocalWorkflow@U2@@SAXXZ$178 1001d34d f   SamtoolMpileupWorker.obj
 0001:0001c359       __unwindfunclet$?init@CallVariantsWorkerFactory@LocalWorkflow@U2@@SAXXZ$179 1001d359 f   SamtoolMpileupWorker.obj
 0001:0001c365       __unwindfunclet$?init@CallVariantsWorkerFactory@LocalWorkflow@U2@@SAXXZ$180 1001d365 f   SamtoolMpileupWorker.obj
 0001:0001c371       __unwindfunclet$?init@CallVariantsWorkerFactory@LocalWorkflow@U2@@SAXXZ$181 1001d371 f   SamtoolMpileupWorker.obj
 0001:0001c37d       __unwindfunclet$?init@CallVariantsWorkerFactory@LocalWorkflow@U2@@SAXXZ$182 1001d37d f   SamtoolMpileupWorker.obj
 0001:0001c389       __unwindfunclet$?init@CallVariantsWorkerFactory@LocalWorkflow@U2@@SAXXZ$183 1001d389 f   SamtoolMpileupWorker.obj
 0001:0001c392       __unwindfunclet$?init@CallVariantsWorkerFactory@LocalWorkflow@U2@@SAXXZ$184 1001d392 f   SamtoolMpileupWorker.obj
 0001:0001c39e       __unwindfunclet$?init@CallVariantsWorkerFactory@LocalWorkflow@U2@@SAXXZ$185 1001d39e f   SamtoolMpileupWorker.obj
 0001:0001c3aa       __unwindfunclet$?init@CallVariantsWorkerFactory@LocalWorkflow@U2@@SAXXZ$186 1001d3aa f   SamtoolMpileupWorker.obj
 0001:0001c3b6       __unwindfunclet$?init@CallVariantsWorkerFactory@LocalWorkflow@U2@@SAXXZ$187 1001d3b6 f   SamtoolMpileupWorker.obj
 0001:0001c3bf       __unwindfunclet$?init@CallVariantsWorkerFactory@LocalWorkflow@U2@@SAXXZ$188 1001d3bf f   SamtoolMpileupWorker.obj
 0001:0001c3cb       __unwindfunclet$?init@CallVariantsWorkerFactory@LocalWorkflow@U2@@SAXXZ$189 1001d3cb f   SamtoolMpileupWorker.obj
 0001:0001c3d6       __unwindfunclet$?init@CallVariantsWorkerFactory@LocalWorkflow@U2@@SAXXZ$190 1001d3d6 f   SamtoolMpileupWorker.obj
 0001:0001c3f0       __unwindfunclet$?init@CallVariantsWorkerFactory@LocalWorkflow@U2@@SAXXZ$192 1001d3f0 f   SamtoolMpileupWorker.obj
 0001:0001c3fb       __unwindfunclet$?init@CallVariantsWorkerFactory@LocalWorkflow@U2@@SAXXZ$193 1001d3fb f   SamtoolMpileupWorker.obj
 0001:0001c415       __unwindfunclet$?init@CallVariantsWorkerFactory@LocalWorkflow@U2@@SAXXZ$195 1001d415 f   SamtoolMpileupWorker.obj
 0001:0001c41d       __unwindfunclet$?init@CallVariantsWorkerFactory@LocalWorkflow@U2@@SAXXZ$196 1001d41d f   SamtoolMpileupWorker.obj
 0001:0001c426       __unwindfunclet$?init@CallVariantsWorkerFactory@LocalWorkflow@U2@@SAXXZ$197 1001d426 f   SamtoolMpileupWorker.obj
 0001:0001c431       __unwindfunclet$?init@CallVariantsWorkerFactory@LocalWorkflow@U2@@SAXXZ$198 1001d431 f   SamtoolMpileupWorker.obj
 0001:0001c43c       __unwindfunclet$?init@CallVariantsWorkerFactory@LocalWorkflow@U2@@SAXXZ$199 1001d43c f   SamtoolMpileupWorker.obj
 0001:0001c456       __unwindfunclet$?init@CallVariantsWorkerFactory@LocalWorkflow@U2@@SAXXZ$201 1001d456 f   SamtoolMpileupWorker.obj
 0001:0001c45e       __unwindfunclet$?init@CallVariantsWorkerFactory@LocalWorkflow@U2@@SAXXZ$202 1001d45e f   SamtoolMpileupWorker.obj
 0001:0001c467       __unwindfunclet$?init@CallVariantsWorkerFactory@LocalWorkflow@U2@@SAXXZ$203 1001d467 f   SamtoolMpileupWorker.obj
 0001:0001c472       __unwindfunclet$?init@CallVariantsWorkerFactory@LocalWorkflow@U2@@SAXXZ$204 1001d472 f   SamtoolMpileupWorker.obj
 0001:0001c48c       __unwindfunclet$?init@CallVariantsWorkerFactory@LocalWorkflow@U2@@SAXXZ$205 1001d48c f   SamtoolMpileupWorker.obj
 0001:0001c497       __unwindfunclet$?init@CallVariantsWorkerFactory@LocalWorkflow@U2@@SAXXZ$206 1001d497 f   SamtoolMpileupWorker.obj
 0001:0001c4b6       __unwindfunclet$?init@CallVariantsWorkerFactory@LocalWorkflow@U2@@SAXXZ$208 1001d4b6 f   SamtoolMpileupWorker.obj
 0001:0001c4c1       __unwindfunclet$?init@CallVariantsWorkerFactory@LocalWorkflow@U2@@SAXXZ$209 1001d4c1 f   SamtoolMpileupWorker.obj
 0001:0001c4e0       __unwindfunclet$?init@CallVariantsWorkerFactory@LocalWorkflow@U2@@SAXXZ$211 1001d4e0 f   SamtoolMpileupWorker.obj
 0001:0001c4eb       __unwindfunclet$?init@CallVariantsWorkerFactory@LocalWorkflow@U2@@SAXXZ$212 1001d4eb f   SamtoolMpileupWorker.obj
 0001:0001c50a       __unwindfunclet$?init@CallVariantsWorkerFactory@LocalWorkflow@U2@@SAXXZ$214 1001d50a f   SamtoolMpileupWorker.obj
 0001:0001c515       __unwindfunclet$?init@CallVariantsWorkerFactory@LocalWorkflow@U2@@SAXXZ$215 1001d515 f   SamtoolMpileupWorker.obj
 0001:0001c534       __unwindfunclet$?init@CallVariantsWorkerFactory@LocalWorkflow@U2@@SAXXZ$217 1001d534 f   SamtoolMpileupWorker.obj
 0001:0001c53f       __unwindfunclet$?init@CallVariantsWorkerFactory@LocalWorkflow@U2@@SAXXZ$218 1001d53f f   SamtoolMpileupWorker.obj
 0001:0001c55e       __unwindfunclet$?init@CallVariantsWorkerFactory@LocalWorkflow@U2@@SAXXZ$220 1001d55e f   SamtoolMpileupWorker.obj
 0001:0001c569       __unwindfunclet$?init@CallVariantsWorkerFactory@LocalWorkflow@U2@@SAXXZ$221 1001d569 f   SamtoolMpileupWorker.obj
 0001:0001c588       __unwindfunclet$?init@CallVariantsWorkerFactory@LocalWorkflow@U2@@SAXXZ$223 1001d588 f   SamtoolMpileupWorker.obj
 0001:0001c593       __unwindfunclet$?init@CallVariantsWorkerFactory@LocalWorkflow@U2@@SAXXZ$224 1001d593 f   SamtoolMpileupWorker.obj
 0001:0001c5b2       __unwindfunclet$?init@CallVariantsWorkerFactory@LocalWorkflow@U2@@SAXXZ$226 1001d5b2 f   SamtoolMpileupWorker.obj
 0001:0001c5bd       __unwindfunclet$?init@CallVariantsWorkerFactory@LocalWorkflow@U2@@SAXXZ$227 1001d5bd f   SamtoolMpileupWorker.obj
 0001:0001c5dc       __unwindfunclet$?init@CallVariantsWorkerFactory@LocalWorkflow@U2@@SAXXZ$229 1001d5dc f   SamtoolMpileupWorker.obj
 0001:0001c5e7       __unwindfunclet$?init@CallVariantsWorkerFactory@LocalWorkflow@U2@@SAXXZ$230 1001d5e7 f   SamtoolMpileupWorker.obj
 0001:0001c606       __unwindfunclet$?init@CallVariantsWorkerFactory@LocalWorkflow@U2@@SAXXZ$232 1001d606 f   SamtoolMpileupWorker.obj
 0001:0001c611       __unwindfunclet$?init@CallVariantsWorkerFactory@LocalWorkflow@U2@@SAXXZ$233 1001d611 f   SamtoolMpileupWorker.obj
 0001:0001c630       __unwindfunclet$?init@CallVariantsWorkerFactory@LocalWorkflow@U2@@SAXXZ$235 1001d630 f   SamtoolMpileupWorker.obj
 0001:0001c63b       __unwindfunclet$?init@CallVariantsWorkerFactory@LocalWorkflow@U2@@SAXXZ$236 1001d63b f   SamtoolMpileupWorker.obj
 0001:0001c65a       __unwindfunclet$?init@CallVariantsWorkerFactory@LocalWorkflow@U2@@SAXXZ$238 1001d65a f   SamtoolMpileupWorker.obj
 0001:0001c665       __unwindfunclet$?init@CallVariantsWorkerFactory@LocalWorkflow@U2@@SAXXZ$239 1001d665 f   SamtoolMpileupWorker.obj
 0001:0001c684       __unwindfunclet$?init@CallVariantsWorkerFactory@LocalWorkflow@U2@@SAXXZ$241 1001d684 f   SamtoolMpileupWorker.obj
 0001:0001c68f       __unwindfunclet$?init@CallVariantsWorkerFactory@LocalWorkflow@U2@@SAXXZ$242 1001d68f f   SamtoolMpileupWorker.obj
 0001:0001c6ae       __unwindfunclet$?init@CallVariantsWorkerFactory@LocalWorkflow@U2@@SAXXZ$244 1001d6ae f   SamtoolMpileupWorker.obj
 0001:0001c6b9       __unwindfunclet$?init@CallVariantsWorkerFactory@LocalWorkflow@U2@@SAXXZ$245 1001d6b9 f   SamtoolMpileupWorker.obj
 0001:0001c6d8       __unwindfunclet$?init@CallVariantsWorkerFactory@LocalWorkflow@U2@@SAXXZ$247 1001d6d8 f   SamtoolMpileupWorker.obj
 0001:0001c6e3       __unwindfunclet$?init@CallVariantsWorkerFactory@LocalWorkflow@U2@@SAXXZ$248 1001d6e3 f   SamtoolMpileupWorker.obj
 0001:0001c702       __unwindfunclet$?init@CallVariantsWorkerFactory@LocalWorkflow@U2@@SAXXZ$250 1001d702 f   SamtoolMpileupWorker.obj
 0001:0001c70d       __unwindfunclet$?init@CallVariantsWorkerFactory@LocalWorkflow@U2@@SAXXZ$251 1001d70d f   SamtoolMpileupWorker.obj
 0001:0001c72c       __unwindfunclet$?init@CallVariantsWorkerFactory@LocalWorkflow@U2@@SAXXZ$253 1001d72c f   SamtoolMpileupWorker.obj
 0001:0001c737       __unwindfunclet$?init@CallVariantsWorkerFactory@LocalWorkflow@U2@@SAXXZ$254 1001d737 f   SamtoolMpileupWorker.obj
 0001:0001c756       __unwindfunclet$?init@CallVariantsWorkerFactory@LocalWorkflow@U2@@SAXXZ$256 1001d756 f   SamtoolMpileupWorker.obj
 0001:0001c761       __unwindfunclet$?init@CallVariantsWorkerFactory@LocalWorkflow@U2@@SAXXZ$257 1001d761 f   SamtoolMpileupWorker.obj
 0001:0001c780       __unwindfunclet$?init@CallVariantsWorkerFactory@LocalWorkflow@U2@@SAXXZ$259 1001d780 f   SamtoolMpileupWorker.obj
 0001:0001c78b       __unwindfunclet$?init@CallVariantsWorkerFactory@LocalWorkflow@U2@@SAXXZ$260 1001d78b f   SamtoolMpileupWorker.obj
 0001:0001c7aa       __unwindfunclet$?init@CallVariantsWorkerFactory@LocalWorkflow@U2@@SAXXZ$262 1001d7aa f   SamtoolMpileupWorker.obj
 0001:0001c7b5       __unwindfunclet$?init@CallVariantsWorkerFactory@LocalWorkflow@U2@@SAXXZ$263 1001d7b5 f   SamtoolMpileupWorker.obj
 0001:0001c7d4       __unwindfunclet$?init@CallVariantsWorkerFactory@LocalWorkflow@U2@@SAXXZ$265 1001d7d4 f   SamtoolMpileupWorker.obj
 0001:0001c7df       __unwindfunclet$?init@CallVariantsWorkerFactory@LocalWorkflow@U2@@SAXXZ$266 1001d7df f   SamtoolMpileupWorker.obj
 0001:0001c7fe       __unwindfunclet$?init@CallVariantsWorkerFactory@LocalWorkflow@U2@@SAXXZ$268 1001d7fe f   SamtoolMpileupWorker.obj
 0001:0001c809       __unwindfunclet$?init@CallVariantsWorkerFactory@LocalWorkflow@U2@@SAXXZ$269 1001d809 f   SamtoolMpileupWorker.obj
 0001:0001c828       __unwindfunclet$?init@CallVariantsWorkerFactory@LocalWorkflow@U2@@SAXXZ$271 1001d828 f   SamtoolMpileupWorker.obj
 0001:0001c833       __unwindfunclet$?init@CallVariantsWorkerFactory@LocalWorkflow@U2@@SAXXZ$272 1001d833 f   SamtoolMpileupWorker.obj
 0001:0001c852       __unwindfunclet$?init@CallVariantsWorkerFactory@LocalWorkflow@U2@@SAXXZ$274 1001d852 f   SamtoolMpileupWorker.obj
 0001:0001c85d       __unwindfunclet$?init@CallVariantsWorkerFactory@LocalWorkflow@U2@@SAXXZ$275 1001d85d f   SamtoolMpileupWorker.obj
 0001:0001c87c       __unwindfunclet$?init@CallVariantsWorkerFactory@LocalWorkflow@U2@@SAXXZ$277 1001d87c f   SamtoolMpileupWorker.obj
 0001:0001c887       __unwindfunclet$?init@CallVariantsWorkerFactory@LocalWorkflow@U2@@SAXXZ$278 1001d887 f   SamtoolMpileupWorker.obj
 0001:0001c8a6       __unwindfunclet$?init@CallVariantsWorkerFactory@LocalWorkflow@U2@@SAXXZ$280 1001d8a6 f   SamtoolMpileupWorker.obj
 0001:0001c8b1       __unwindfunclet$?init@CallVariantsWorkerFactory@LocalWorkflow@U2@@SAXXZ$281 1001d8b1 f   SamtoolMpileupWorker.obj
 0001:0001c8cb       __unwindfunclet$?init@CallVariantsWorkerFactory@LocalWorkflow@U2@@SAXXZ$283 1001d8cb f   SamtoolMpileupWorker.obj
 0001:0001c8d6       __unwindfunclet$?init@CallVariantsWorkerFactory@LocalWorkflow@U2@@SAXXZ$284 1001d8d6 f   SamtoolMpileupWorker.obj
 0001:0001c8f0       __unwindfunclet$?init@CallVariantsWorkerFactory@LocalWorkflow@U2@@SAXXZ$286 1001d8f0 f   SamtoolMpileupWorker.obj
 0001:0001c8fb       __unwindfunclet$?init@CallVariantsWorkerFactory@LocalWorkflow@U2@@SAXXZ$287 1001d8fb f   SamtoolMpileupWorker.obj
 0001:0001c915       __unwindfunclet$?init@CallVariantsWorkerFactory@LocalWorkflow@U2@@SAXXZ$289 1001d915 f   SamtoolMpileupWorker.obj
 0001:0001c920       __unwindfunclet$?init@CallVariantsWorkerFactory@LocalWorkflow@U2@@SAXXZ$290 1001d920 f   SamtoolMpileupWorker.obj
 0001:0001c93a       __unwindfunclet$?init@CallVariantsWorkerFactory@LocalWorkflow@U2@@SAXXZ$292 1001d93a f   SamtoolMpileupWorker.obj
 0001:0001c945       __unwindfunclet$?init@CallVariantsWorkerFactory@LocalWorkflow@U2@@SAXXZ$293 1001d945 f   SamtoolMpileupWorker.obj
 0001:0001c95f       __unwindfunclet$?init@CallVariantsWorkerFactory@LocalWorkflow@U2@@SAXXZ$295 1001d95f f   SamtoolMpileupWorker.obj
 0001:0001c96a       __unwindfunclet$?init@CallVariantsWorkerFactory@LocalWorkflow@U2@@SAXXZ$296 1001d96a f   SamtoolMpileupWorker.obj
 0001:0001c984       __unwindfunclet$?init@CallVariantsWorkerFactory@LocalWorkflow@U2@@SAXXZ$298 1001d984 f   SamtoolMpileupWorker.obj
 0001:0001c98f       __unwindfunclet$?init@CallVariantsWorkerFactory@LocalWorkflow@U2@@SAXXZ$299 1001d98f f   SamtoolMpileupWorker.obj
 0001:0001c9a9       __unwindfunclet$?init@CallVariantsWorkerFactory@LocalWorkflow@U2@@SAXXZ$301 1001d9a9 f   SamtoolMpileupWorker.obj
 0001:0001c9b4       __unwindfunclet$?init@CallVariantsWorkerFactory@LocalWorkflow@U2@@SAXXZ$302 1001d9b4 f   SamtoolMpileupWorker.obj
 0001:0001c9d3       __unwindfunclet$?init@CallVariantsWorkerFactory@LocalWorkflow@U2@@SAXXZ$304 1001d9d3 f   SamtoolMpileupWorker.obj
 0001:0001c9de       __unwindfunclet$?init@CallVariantsWorkerFactory@LocalWorkflow@U2@@SAXXZ$305 1001d9de f   SamtoolMpileupWorker.obj
 0001:0001c9fd       __unwindfunclet$?init@CallVariantsWorkerFactory@LocalWorkflow@U2@@SAXXZ$307 1001d9fd f   SamtoolMpileupWorker.obj
 0001:0001ca08       __unwindfunclet$?init@CallVariantsWorkerFactory@LocalWorkflow@U2@@SAXXZ$308 1001da08 f   SamtoolMpileupWorker.obj
 0001:0001ca27       __unwindfunclet$?init@CallVariantsWorkerFactory@LocalWorkflow@U2@@SAXXZ$310 1001da27 f   SamtoolMpileupWorker.obj
 0001:0001ca32       __unwindfunclet$?init@CallVariantsWorkerFactory@LocalWorkflow@U2@@SAXXZ$311 1001da32 f   SamtoolMpileupWorker.obj
 0001:0001ca51       __unwindfunclet$?init@CallVariantsWorkerFactory@LocalWorkflow@U2@@SAXXZ$313 1001da51 f   SamtoolMpileupWorker.obj
 0001:0001ca5c       __unwindfunclet$?init@CallVariantsWorkerFactory@LocalWorkflow@U2@@SAXXZ$314 1001da5c f   SamtoolMpileupWorker.obj
 0001:0001ca7b       __unwindfunclet$?init@CallVariantsWorkerFactory@LocalWorkflow@U2@@SAXXZ$316 1001da7b f   SamtoolMpileupWorker.obj
 0001:0001ca86       __unwindfunclet$?init@CallVariantsWorkerFactory@LocalWorkflow@U2@@SAXXZ$317 1001da86 f   SamtoolMpileupWorker.obj
 0001:0001caa5       __unwindfunclet$?init@CallVariantsWorkerFactory@LocalWorkflow@U2@@SAXXZ$319 1001daa5 f   SamtoolMpileupWorker.obj
 0001:0001cab0       __unwindfunclet$?init@CallVariantsWorkerFactory@LocalWorkflow@U2@@SAXXZ$320 1001dab0 f   SamtoolMpileupWorker.obj
 0001:0001cacf       __unwindfunclet$?init@CallVariantsWorkerFactory@LocalWorkflow@U2@@SAXXZ$322 1001dacf f   SamtoolMpileupWorker.obj
 0001:0001cada       __unwindfunclet$?init@CallVariantsWorkerFactory@LocalWorkflow@U2@@SAXXZ$323 1001dada f   SamtoolMpileupWorker.obj
 0001:0001caf9       __unwindfunclet$?init@CallVariantsWorkerFactory@LocalWorkflow@U2@@SAXXZ$325 1001daf9 f   SamtoolMpileupWorker.obj
 0001:0001cb04       __unwindfunclet$?init@CallVariantsWorkerFactory@LocalWorkflow@U2@@SAXXZ$326 1001db04 f   SamtoolMpileupWorker.obj
 0001:0001cb23       __unwindfunclet$?init@CallVariantsWorkerFactory@LocalWorkflow@U2@@SAXXZ$328 1001db23 f   SamtoolMpileupWorker.obj
 0001:0001cb2e       __unwindfunclet$?init@CallVariantsWorkerFactory@LocalWorkflow@U2@@SAXXZ$329 1001db2e f   SamtoolMpileupWorker.obj
 0001:0001cb4d       __unwindfunclet$?init@CallVariantsWorkerFactory@LocalWorkflow@U2@@SAXXZ$331 1001db4d f   SamtoolMpileupWorker.obj
 0001:0001cb58       __unwindfunclet$?init@CallVariantsWorkerFactory@LocalWorkflow@U2@@SAXXZ$332 1001db58 f   SamtoolMpileupWorker.obj
 0001:0001cb77       __unwindfunclet$?init@CallVariantsWorkerFactory@LocalWorkflow@U2@@SAXXZ$334 1001db77 f   SamtoolMpileupWorker.obj
 0001:0001cb82       __unwindfunclet$?init@CallVariantsWorkerFactory@LocalWorkflow@U2@@SAXXZ$335 1001db82 f   SamtoolMpileupWorker.obj
 0001:0001cba1       __unwindfunclet$?init@CallVariantsWorkerFactory@LocalWorkflow@U2@@SAXXZ$337 1001dba1 f   SamtoolMpileupWorker.obj
 0001:0001cbac       __unwindfunclet$?init@CallVariantsWorkerFactory@LocalWorkflow@U2@@SAXXZ$338 1001dbac f   SamtoolMpileupWorker.obj
 0001:0001cbcb       __unwindfunclet$?init@CallVariantsWorkerFactory@LocalWorkflow@U2@@SAXXZ$340 1001dbcb f   SamtoolMpileupWorker.obj
 0001:0001cbd6       __unwindfunclet$?init@CallVariantsWorkerFactory@LocalWorkflow@U2@@SAXXZ$341 1001dbd6 f   SamtoolMpileupWorker.obj
 0001:0001cbde       __unwindfunclet$?init@CallVariantsWorkerFactory@LocalWorkflow@U2@@SAXXZ$342 1001dbde f   SamtoolMpileupWorker.obj
 0001:0001cbe6       __unwindfunclet$?init@CallVariantsWorkerFactory@LocalWorkflow@U2@@SAXXZ$343 1001dbe6 f   SamtoolMpileupWorker.obj
 0001:0001cbef       __unwindfunclet$?init@CallVariantsWorkerFactory@LocalWorkflow@U2@@SAXXZ$344 1001dbef f   SamtoolMpileupWorker.obj
 0001:0001cbf8       __unwindfunclet$?init@CallVariantsWorkerFactory@LocalWorkflow@U2@@SAXXZ$345 1001dbf8 f   SamtoolMpileupWorker.obj
 0001:0001cc01       __unwindfunclet$?init@CallVariantsWorkerFactory@LocalWorkflow@U2@@SAXXZ$346 1001dc01 f   SamtoolMpileupWorker.obj
 0001:0001cc0a       __unwindfunclet$?init@CallVariantsWorkerFactory@LocalWorkflow@U2@@SAXXZ$347 1001dc0a f   SamtoolMpileupWorker.obj
 0001:0001cc13       __unwindfunclet$?init@CallVariantsWorkerFactory@LocalWorkflow@U2@@SAXXZ$348 1001dc13 f   SamtoolMpileupWorker.obj
 0001:0001cc1c       __unwindfunclet$?init@CallVariantsWorkerFactory@LocalWorkflow@U2@@SAXXZ$349 1001dc1c f   SamtoolMpileupWorker.obj
 0001:0001cc27       __unwindfunclet$?init@CallVariantsWorkerFactory@LocalWorkflow@U2@@SAXXZ$350 1001dc27 f   SamtoolMpileupWorker.obj
 0001:0001cc2f       __unwindfunclet$?init@CallVariantsWorkerFactory@LocalWorkflow@U2@@SAXXZ$351 1001dc2f f   SamtoolMpileupWorker.obj
 0001:0001cc38       __unwindfunclet$?init@CallVariantsWorkerFactory@LocalWorkflow@U2@@SAXXZ$352 1001dc38 f   SamtoolMpileupWorker.obj
 0001:0001cc41       __unwindfunclet$?init@CallVariantsWorkerFactory@LocalWorkflow@U2@@SAXXZ$353 1001dc41 f   SamtoolMpileupWorker.obj
 0001:0001cc4a       __unwindfunclet$?init@CallVariantsWorkerFactory@LocalWorkflow@U2@@SAXXZ$354 1001dc4a f   SamtoolMpileupWorker.obj
 0001:0001cc53       __unwindfunclet$?init@CallVariantsWorkerFactory@LocalWorkflow@U2@@SAXXZ$355 1001dc53 f   SamtoolMpileupWorker.obj
 0001:0001cc5c       __unwindfunclet$?init@CallVariantsWorkerFactory@LocalWorkflow@U2@@SAXXZ$356 1001dc5c f   SamtoolMpileupWorker.obj
 0001:0001cc65       __unwindfunclet$?init@CallVariantsWorkerFactory@LocalWorkflow@U2@@SAXXZ$357 1001dc65 f   SamtoolMpileupWorker.obj
 0001:0001cc70       __unwindfunclet$?init@CallVariantsWorkerFactory@LocalWorkflow@U2@@SAXXZ$358 1001dc70 f   SamtoolMpileupWorker.obj
 0001:0001cc78       __unwindfunclet$?init@CallVariantsWorkerFactory@LocalWorkflow@U2@@SAXXZ$359 1001dc78 f   SamtoolMpileupWorker.obj
 0001:0001cc81       __unwindfunclet$?init@CallVariantsWorkerFactory@LocalWorkflow@U2@@SAXXZ$360 1001dc81 f   SamtoolMpileupWorker.obj
 0001:0001cc8a       __unwindfunclet$?init@CallVariantsWorkerFactory@LocalWorkflow@U2@@SAXXZ$361 1001dc8a f   SamtoolMpileupWorker.obj
 0001:0001cc93       __unwindfunclet$?init@CallVariantsWorkerFactory@LocalWorkflow@U2@@SAXXZ$362 1001dc93 f   SamtoolMpileupWorker.obj
 0001:0001cc9c       __unwindfunclet$?init@CallVariantsWorkerFactory@LocalWorkflow@U2@@SAXXZ$363 1001dc9c f   SamtoolMpileupWorker.obj
 0001:0001cca5       __unwindfunclet$?init@CallVariantsWorkerFactory@LocalWorkflow@U2@@SAXXZ$364 1001dca5 f   SamtoolMpileupWorker.obj
 0001:0001ccae       __unwindfunclet$?init@CallVariantsWorkerFactory@LocalWorkflow@U2@@SAXXZ$365 1001dcae f   SamtoolMpileupWorker.obj
 0001:0001ccb9       __unwindfunclet$?init@CallVariantsWorkerFactory@LocalWorkflow@U2@@SAXXZ$366 1001dcb9 f   SamtoolMpileupWorker.obj
 0001:0001ccc1       __unwindfunclet$?init@CallVariantsWorkerFactory@LocalWorkflow@U2@@SAXXZ$367 1001dcc1 f   SamtoolMpileupWorker.obj
 0001:0001ccca       __unwindfunclet$?init@CallVariantsWorkerFactory@LocalWorkflow@U2@@SAXXZ$368 1001dcca f   SamtoolMpileupWorker.obj
 0001:0001ccd3       __unwindfunclet$?init@CallVariantsWorkerFactory@LocalWorkflow@U2@@SAXXZ$369 1001dcd3 f   SamtoolMpileupWorker.obj
 0001:0001ccdc       __unwindfunclet$?init@CallVariantsWorkerFactory@LocalWorkflow@U2@@SAXXZ$370 1001dcdc f   SamtoolMpileupWorker.obj
 0001:0001cce5       __unwindfunclet$?init@CallVariantsWorkerFactory@LocalWorkflow@U2@@SAXXZ$371 1001dce5 f   SamtoolMpileupWorker.obj
 0001:0001ccee       __unwindfunclet$?init@CallVariantsWorkerFactory@LocalWorkflow@U2@@SAXXZ$372 1001dcee f   SamtoolMpileupWorker.obj
 0001:0001ccf7       __unwindfunclet$?init@CallVariantsWorkerFactory@LocalWorkflow@U2@@SAXXZ$373 1001dcf7 f   SamtoolMpileupWorker.obj
 0001:0001cd02       __unwindfunclet$?init@CallVariantsWorkerFactory@LocalWorkflow@U2@@SAXXZ$374 1001dd02 f   SamtoolMpileupWorker.obj
 0001:0001cd0a       __unwindfunclet$?init@CallVariantsWorkerFactory@LocalWorkflow@U2@@SAXXZ$375 1001dd0a f   SamtoolMpileupWorker.obj
 0001:0001cd13       __unwindfunclet$?init@CallVariantsWorkerFactory@LocalWorkflow@U2@@SAXXZ$376 1001dd13 f   SamtoolMpileupWorker.obj
 0001:0001cd1c       __unwindfunclet$?init@CallVariantsWorkerFactory@LocalWorkflow@U2@@SAXXZ$377 1001dd1c f   SamtoolMpileupWorker.obj
 0001:0001cd25       __unwindfunclet$?init@CallVariantsWorkerFactory@LocalWorkflow@U2@@SAXXZ$378 1001dd25 f   SamtoolMpileupWorker.obj
 0001:0001cd2e       __unwindfunclet$?init@CallVariantsWorkerFactory@LocalWorkflow@U2@@SAXXZ$379 1001dd2e f   SamtoolMpileupWorker.obj
 0001:0001cd37       __unwindfunclet$?init@CallVariantsWorkerFactory@LocalWorkflow@U2@@SAXXZ$380 1001dd37 f   SamtoolMpileupWorker.obj
 0001:0001cd40       __unwindfunclet$?init@CallVariantsWorkerFactory@LocalWorkflow@U2@@SAXXZ$381 1001dd40 f   SamtoolMpileupWorker.obj
 0001:0001cd4b       __unwindfunclet$?init@CallVariantsWorkerFactory@LocalWorkflow@U2@@SAXXZ$382 1001dd4b f   SamtoolMpileupWorker.obj
 0001:0001cd53       __unwindfunclet$?init@CallVariantsWorkerFactory@LocalWorkflow@U2@@SAXXZ$383 1001dd53 f   SamtoolMpileupWorker.obj
 0001:0001cd5c       __unwindfunclet$?init@CallVariantsWorkerFactory@LocalWorkflow@U2@@SAXXZ$384 1001dd5c f   SamtoolMpileupWorker.obj
 0001:0001cd65       __unwindfunclet$?init@CallVariantsWorkerFactory@LocalWorkflow@U2@@SAXXZ$385 1001dd65 f   SamtoolMpileupWorker.obj
 0001:0001cd6e       __unwindfunclet$?init@CallVariantsWorkerFactory@LocalWorkflow@U2@@SAXXZ$386 1001dd6e f   SamtoolMpileupWorker.obj
 0001:0001cd77       __unwindfunclet$?init@CallVariantsWorkerFactory@LocalWorkflow@U2@@SAXXZ$387 1001dd77 f   SamtoolMpileupWorker.obj
 0001:0001cd80       __unwindfunclet$?init@CallVariantsWorkerFactory@LocalWorkflow@U2@@SAXXZ$388 1001dd80 f   SamtoolMpileupWorker.obj
 0001:0001cd89       __unwindfunclet$?init@CallVariantsWorkerFactory@LocalWorkflow@U2@@SAXXZ$389 1001dd89 f   SamtoolMpileupWorker.obj
 0001:0001cd94       __unwindfunclet$?init@CallVariantsWorkerFactory@LocalWorkflow@U2@@SAXXZ$390 1001dd94 f   SamtoolMpileupWorker.obj
 0001:0001cd9c       __unwindfunclet$?init@CallVariantsWorkerFactory@LocalWorkflow@U2@@SAXXZ$391 1001dd9c f   SamtoolMpileupWorker.obj
 0001:0001cda5       __unwindfunclet$?init@CallVariantsWorkerFactory@LocalWorkflow@U2@@SAXXZ$392 1001dda5 f   SamtoolMpileupWorker.obj
 0001:0001cdae       __unwindfunclet$?init@CallVariantsWorkerFactory@LocalWorkflow@U2@@SAXXZ$393 1001ddae f   SamtoolMpileupWorker.obj
 0001:0001cdb7       __unwindfunclet$?init@CallVariantsWorkerFactory@LocalWorkflow@U2@@SAXXZ$394 1001ddb7 f   SamtoolMpileupWorker.obj
 0001:0001cdc0       __unwindfunclet$?init@CallVariantsWorkerFactory@LocalWorkflow@U2@@SAXXZ$395 1001ddc0 f   SamtoolMpileupWorker.obj
 0001:0001cdc9       __unwindfunclet$?init@CallVariantsWorkerFactory@LocalWorkflow@U2@@SAXXZ$396 1001ddc9 f   SamtoolMpileupWorker.obj
 0001:0001cdd2       __unwindfunclet$?init@CallVariantsWorkerFactory@LocalWorkflow@U2@@SAXXZ$397 1001ddd2 f   SamtoolMpileupWorker.obj
 0001:0001cddd       __unwindfunclet$?init@CallVariantsWorkerFactory@LocalWorkflow@U2@@SAXXZ$398 1001dddd f   SamtoolMpileupWorker.obj
 0001:0001cde5       __unwindfunclet$?init@CallVariantsWorkerFactory@LocalWorkflow@U2@@SAXXZ$399 1001dde5 f   SamtoolMpileupWorker.obj
 0001:0001cdee       __unwindfunclet$?init@CallVariantsWorkerFactory@LocalWorkflow@U2@@SAXXZ$400 1001ddee f   SamtoolMpileupWorker.obj
 0001:0001cdf7       __unwindfunclet$?init@CallVariantsWorkerFactory@LocalWorkflow@U2@@SAXXZ$401 1001ddf7 f   SamtoolMpileupWorker.obj
 0001:0001ce00       __unwindfunclet$?init@CallVariantsWorkerFactory@LocalWorkflow@U2@@SAXXZ$402 1001de00 f   SamtoolMpileupWorker.obj
 0001:0001ce09       __unwindfunclet$?init@CallVariantsWorkerFactory@LocalWorkflow@U2@@SAXXZ$403 1001de09 f   SamtoolMpileupWorker.obj
 0001:0001ce12       __unwindfunclet$?init@CallVariantsWorkerFactory@LocalWorkflow@U2@@SAXXZ$404 1001de12 f   SamtoolMpileupWorker.obj
 0001:0001ce1b       __unwindfunclet$?init@CallVariantsWorkerFactory@LocalWorkflow@U2@@SAXXZ$405 1001de1b f   SamtoolMpileupWorker.obj
 0001:0001ce26       __unwindfunclet$?init@CallVariantsWorkerFactory@LocalWorkflow@U2@@SAXXZ$406 1001de26 f   SamtoolMpileupWorker.obj
 0001:0001ce31       __unwindfunclet$?init@CallVariantsWorkerFactory@LocalWorkflow@U2@@SAXXZ$407 1001de31 f   SamtoolMpileupWorker.obj
 0001:0001ce50       __unwindfunclet$?init@CallVariantsWorkerFactory@LocalWorkflow@U2@@SAXXZ$408 1001de50 f   SamtoolMpileupWorker.obj
 0001:0001ce6f       __unwindfunclet$?init@CallVariantsWorkerFactory@LocalWorkflow@U2@@SAXXZ$409 1001de6f f   SamtoolMpileupWorker.obj
 0001:0001ce8e       __unwindfunclet$?init@CallVariantsWorkerFactory@LocalWorkflow@U2@@SAXXZ$410 1001de8e f   SamtoolMpileupWorker.obj
 0001:0001ce96       __unwindfunclet$?init@CallVariantsWorkerFactory@LocalWorkflow@U2@@SAXXZ$411 1001de96 f   SamtoolMpileupWorker.obj
 0001:0001ce9f       __unwindfunclet$?init@CallVariantsWorkerFactory@LocalWorkflow@U2@@SAXXZ$412 1001de9f f   SamtoolMpileupWorker.obj
 0001:0001cea8       __unwindfunclet$?init@CallVariantsWorkerFactory@LocalWorkflow@U2@@SAXXZ$413 1001dea8 f   SamtoolMpileupWorker.obj
 0001:0001ceb1       __unwindfunclet$?init@CallVariantsWorkerFactory@LocalWorkflow@U2@@SAXXZ$414 1001deb1 f   SamtoolMpileupWorker.obj
 0001:0001ceba       __unwindfunclet$?init@CallVariantsWorkerFactory@LocalWorkflow@U2@@SAXXZ$415 1001deba f   SamtoolMpileupWorker.obj
 0001:0001cec3       __unwindfunclet$?init@CallVariantsWorkerFactory@LocalWorkflow@U2@@SAXXZ$416 1001dec3 f   SamtoolMpileupWorker.obj
 0001:0001cecc       __unwindfunclet$?init@CallVariantsWorkerFactory@LocalWorkflow@U2@@SAXXZ$417 1001decc f   SamtoolMpileupWorker.obj
 0001:0001ced7       __unwindfunclet$?init@CallVariantsWorkerFactory@LocalWorkflow@U2@@SAXXZ$418 1001ded7 f   SamtoolMpileupWorker.obj
 0001:0001cedf       __unwindfunclet$?init@CallVariantsWorkerFactory@LocalWorkflow@U2@@SAXXZ$419 1001dedf f   SamtoolMpileupWorker.obj
 0001:0001cee8       __unwindfunclet$?init@CallVariantsWorkerFactory@LocalWorkflow@U2@@SAXXZ$420 1001dee8 f   SamtoolMpileupWorker.obj
 0001:0001cef1       __unwindfunclet$?init@CallVariantsWorkerFactory@LocalWorkflow@U2@@SAXXZ$421 1001def1 f   SamtoolMpileupWorker.obj
 0001:0001cefa       __unwindfunclet$?init@CallVariantsWorkerFactory@LocalWorkflow@U2@@SAXXZ$422 1001defa f   SamtoolMpileupWorker.obj
 0001:0001cf03       __unwindfunclet$?init@CallVariantsWorkerFactory@LocalWorkflow@U2@@SAXXZ$423 1001df03 f   SamtoolMpileupWorker.obj
 0001:0001cf0c       __unwindfunclet$?init@CallVariantsWorkerFactory@LocalWorkflow@U2@@SAXXZ$424 1001df0c f   SamtoolMpileupWorker.obj
 0001:0001cf15       __unwindfunclet$?init@CallVariantsWorkerFactory@LocalWorkflow@U2@@SAXXZ$425 1001df15 f   SamtoolMpileupWorker.obj
 0001:0001cf20       __unwindfunclet$?init@CallVariantsWorkerFactory@LocalWorkflow@U2@@SAXXZ$426 1001df20 f   SamtoolMpileupWorker.obj
 0001:0001cf28       __unwindfunclet$?init@CallVariantsWorkerFactory@LocalWorkflow@U2@@SAXXZ$427 1001df28 f   SamtoolMpileupWorker.obj
 0001:0001cf31       __unwindfunclet$?init@CallVariantsWorkerFactory@LocalWorkflow@U2@@SAXXZ$428 1001df31 f   SamtoolMpileupWorker.obj
 0001:0001cf3a       __unwindfunclet$?init@CallVariantsWorkerFactory@LocalWorkflow@U2@@SAXXZ$429 1001df3a f   SamtoolMpileupWorker.obj
 0001:0001cf43       __unwindfunclet$?init@CallVariantsWorkerFactory@LocalWorkflow@U2@@SAXXZ$430 1001df43 f   SamtoolMpileupWorker.obj
 0001:0001cf4c       __unwindfunclet$?init@CallVariantsWorkerFactory@LocalWorkflow@U2@@SAXXZ$431 1001df4c f   SamtoolMpileupWorker.obj
 0001:0001cf55       __unwindfunclet$?init@CallVariantsWorkerFactory@LocalWorkflow@U2@@SAXXZ$432 1001df55 f   SamtoolMpileupWorker.obj
 0001:0001cf5e       __unwindfunclet$?init@CallVariantsWorkerFactory@LocalWorkflow@U2@@SAXXZ$433 1001df5e f   SamtoolMpileupWorker.obj
 0001:0001cf69       __unwindfunclet$?init@CallVariantsWorkerFactory@LocalWorkflow@U2@@SAXXZ$434 1001df69 f   SamtoolMpileupWorker.obj
 0001:0001cf71       __unwindfunclet$?init@CallVariantsWorkerFactory@LocalWorkflow@U2@@SAXXZ$435 1001df71 f   SamtoolMpileupWorker.obj
 0001:0001cf7a       __unwindfunclet$?init@CallVariantsWorkerFactory@LocalWorkflow@U2@@SAXXZ$436 1001df7a f   SamtoolMpileupWorker.obj
 0001:0001cf83       __unwindfunclet$?init@CallVariantsWorkerFactory@LocalWorkflow@U2@@SAXXZ$437 1001df83 f   SamtoolMpileupWorker.obj
 0001:0001cf8c       __unwindfunclet$?init@CallVariantsWorkerFactory@LocalWorkflow@U2@@SAXXZ$438 1001df8c f   SamtoolMpileupWorker.obj
 0001:0001cf95       __unwindfunclet$?init@CallVariantsWorkerFactory@LocalWorkflow@U2@@SAXXZ$439 1001df95 f   SamtoolMpileupWorker.obj
 0001:0001cf9e       __unwindfunclet$?init@CallVariantsWorkerFactory@LocalWorkflow@U2@@SAXXZ$440 1001df9e f   SamtoolMpileupWorker.obj
 0001:0001cfa7       __unwindfunclet$?init@CallVariantsWorkerFactory@LocalWorkflow@U2@@SAXXZ$441 1001dfa7 f   SamtoolMpileupWorker.obj
 0001:0001cfb3       __unwindfunclet$?init@CallVariantsWorkerFactory@LocalWorkflow@U2@@SAXXZ$442 1001dfb3 f   SamtoolMpileupWorker.obj
 0001:0001cfbc       __unwindfunclet$?init@CallVariantsWorkerFactory@LocalWorkflow@U2@@SAXXZ$443 1001dfbc f   SamtoolMpileupWorker.obj
 0001:0001cfc7       __unwindfunclet$?init@CallVariantsWorkerFactory@LocalWorkflow@U2@@SAXXZ$444 1001dfc7 f   SamtoolMpileupWorker.obj
 0001:0001cfcf       __unwindfunclet$?init@CallVariantsWorkerFactory@LocalWorkflow@U2@@SAXXZ$445 1001dfcf f   SamtoolMpileupWorker.obj
 0001:0001cfd8       __unwindfunclet$?init@CallVariantsWorkerFactory@LocalWorkflow@U2@@SAXXZ$446 1001dfd8 f   SamtoolMpileupWorker.obj
 0001:0001cfe1       __unwindfunclet$?init@CallVariantsWorkerFactory@LocalWorkflow@U2@@SAXXZ$447 1001dfe1 f   SamtoolMpileupWorker.obj
 0001:0001cfea       __unwindfunclet$?init@CallVariantsWorkerFactory@LocalWorkflow@U2@@SAXXZ$448 1001dfea f   SamtoolMpileupWorker.obj
 0001:0001cff3       __unwindfunclet$?init@CallVariantsWorkerFactory@LocalWorkflow@U2@@SAXXZ$449 1001dff3 f   SamtoolMpileupWorker.obj
 0001:0001cffc       __unwindfunclet$?init@CallVariantsWorkerFactory@LocalWorkflow@U2@@SAXXZ$450 1001dffc f   SamtoolMpileupWorker.obj
 0001:0001d005       __unwindfunclet$?init@CallVariantsWorkerFactory@LocalWorkflow@U2@@SAXXZ$451 1001e005 f   SamtoolMpileupWorker.obj
 0001:0001d010       __unwindfunclet$?init@CallVariantsWorkerFactory@LocalWorkflow@U2@@SAXXZ$452 1001e010 f   SamtoolMpileupWorker.obj
 0001:0001d018       __unwindfunclet$?init@CallVariantsWorkerFactory@LocalWorkflow@U2@@SAXXZ$453 1001e018 f   SamtoolMpileupWorker.obj
 0001:0001d021       __unwindfunclet$?init@CallVariantsWorkerFactory@LocalWorkflow@U2@@SAXXZ$454 1001e021 f   SamtoolMpileupWorker.obj
 0001:0001d02a       __unwindfunclet$?init@CallVariantsWorkerFactory@LocalWorkflow@U2@@SAXXZ$455 1001e02a f   SamtoolMpileupWorker.obj
 0001:0001d033       __unwindfunclet$?init@CallVariantsWorkerFactory@LocalWorkflow@U2@@SAXXZ$456 1001e033 f   SamtoolMpileupWorker.obj
 0001:0001d03c       __unwindfunclet$?init@CallVariantsWorkerFactory@LocalWorkflow@U2@@SAXXZ$457 1001e03c f   SamtoolMpileupWorker.obj
 0001:0001d045       __unwindfunclet$?init@CallVariantsWorkerFactory@LocalWorkflow@U2@@SAXXZ$458 1001e045 f   SamtoolMpileupWorker.obj
 0001:0001d04e       __unwindfunclet$?init@CallVariantsWorkerFactory@LocalWorkflow@U2@@SAXXZ$459 1001e04e f   SamtoolMpileupWorker.obj
 0001:0001d05a       __unwindfunclet$?init@CallVariantsWorkerFactory@LocalWorkflow@U2@@SAXXZ$460 1001e05a f   SamtoolMpileupWorker.obj
 0001:0001d063       __unwindfunclet$?init@CallVariantsWorkerFactory@LocalWorkflow@U2@@SAXXZ$461 1001e063 f   SamtoolMpileupWorker.obj
 0001:0001d06f       __unwindfunclet$?init@CallVariantsWorkerFactory@LocalWorkflow@U2@@SAXXZ$462 1001e06f f   SamtoolMpileupWorker.obj
 0001:0001d078       __unwindfunclet$?init@CallVariantsWorkerFactory@LocalWorkflow@U2@@SAXXZ$463 1001e078 f   SamtoolMpileupWorker.obj
 0001:0001d083       __unwindfunclet$?init@CallVariantsWorkerFactory@LocalWorkflow@U2@@SAXXZ$464 1001e083 f   SamtoolMpileupWorker.obj
 0001:0001d08b       __unwindfunclet$?init@CallVariantsWorkerFactory@LocalWorkflow@U2@@SAXXZ$465 1001e08b f   SamtoolMpileupWorker.obj
 0001:0001d094       __unwindfunclet$?init@CallVariantsWorkerFactory@LocalWorkflow@U2@@SAXXZ$466 1001e094 f   SamtoolMpileupWorker.obj
 0001:0001d09d       __unwindfunclet$?init@CallVariantsWorkerFactory@LocalWorkflow@U2@@SAXXZ$467 1001e09d f   SamtoolMpileupWorker.obj
 0001:0001d0a6       __unwindfunclet$?init@CallVariantsWorkerFactory@LocalWorkflow@U2@@SAXXZ$468 1001e0a6 f   SamtoolMpileupWorker.obj
 0001:0001d0af       __unwindfunclet$?init@CallVariantsWorkerFactory@LocalWorkflow@U2@@SAXXZ$469 1001e0af f   SamtoolMpileupWorker.obj
 0001:0001d0b8       __unwindfunclet$?init@CallVariantsWorkerFactory@LocalWorkflow@U2@@SAXXZ$470 1001e0b8 f   SamtoolMpileupWorker.obj
 0001:0001d0c1       __unwindfunclet$?init@CallVariantsWorkerFactory@LocalWorkflow@U2@@SAXXZ$471 1001e0c1 f   SamtoolMpileupWorker.obj
 0001:0001d0cc       __unwindfunclet$?init@CallVariantsWorkerFactory@LocalWorkflow@U2@@SAXXZ$472 1001e0cc f   SamtoolMpileupWorker.obj
 0001:0001d0d4       __unwindfunclet$?init@CallVariantsWorkerFactory@LocalWorkflow@U2@@SAXXZ$473 1001e0d4 f   SamtoolMpileupWorker.obj
 0001:0001d0dd       __unwindfunclet$?init@CallVariantsWorkerFactory@LocalWorkflow@U2@@SAXXZ$474 1001e0dd f   SamtoolMpileupWorker.obj
 0001:0001d0e6       __unwindfunclet$?init@CallVariantsWorkerFactory@LocalWorkflow@U2@@SAXXZ$475 1001e0e6 f   SamtoolMpileupWorker.obj
 0001:0001d0ef       __unwindfunclet$?init@CallVariantsWorkerFactory@LocalWorkflow@U2@@SAXXZ$476 1001e0ef f   SamtoolMpileupWorker.obj
 0001:0001d0f8       __unwindfunclet$?init@CallVariantsWorkerFactory@LocalWorkflow@U2@@SAXXZ$477 1001e0f8 f   SamtoolMpileupWorker.obj
 0001:0001d101       __unwindfunclet$?init@CallVariantsWorkerFactory@LocalWorkflow@U2@@SAXXZ$478 1001e101 f   SamtoolMpileupWorker.obj
 0001:0001d10a       __unwindfunclet$?init@CallVariantsWorkerFactory@LocalWorkflow@U2@@SAXXZ$479 1001e10a f   SamtoolMpileupWorker.obj
 0001:0001d115       __unwindfunclet$?init@CallVariantsWorkerFactory@LocalWorkflow@U2@@SAXXZ$480 1001e115 f   SamtoolMpileupWorker.obj
 0001:0001d11d       __unwindfunclet$?init@CallVariantsWorkerFactory@LocalWorkflow@U2@@SAXXZ$481 1001e11d f   SamtoolMpileupWorker.obj
 0001:0001d126       __unwindfunclet$?init@CallVariantsWorkerFactory@LocalWorkflow@U2@@SAXXZ$482 1001e126 f   SamtoolMpileupWorker.obj
 0001:0001d12f       __unwindfunclet$?init@CallVariantsWorkerFactory@LocalWorkflow@U2@@SAXXZ$483 1001e12f f   SamtoolMpileupWorker.obj
 0001:0001d138       __unwindfunclet$?init@CallVariantsWorkerFactory@LocalWorkflow@U2@@SAXXZ$484 1001e138 f   SamtoolMpileupWorker.obj
 0001:0001d141       __unwindfunclet$?init@CallVariantsWorkerFactory@LocalWorkflow@U2@@SAXXZ$485 1001e141 f   SamtoolMpileupWorker.obj
 0001:0001d14a       __unwindfunclet$?init@CallVariantsWorkerFactory@LocalWorkflow@U2@@SAXXZ$486 1001e14a f   SamtoolMpileupWorker.obj
 0001:0001d153       __unwindfunclet$?init@CallVariantsWorkerFactory@LocalWorkflow@U2@@SAXXZ$487 1001e153 f   SamtoolMpileupWorker.obj
 0001:0001d15e       __unwindfunclet$?init@CallVariantsWorkerFactory@LocalWorkflow@U2@@SAXXZ$488 1001e15e f   SamtoolMpileupWorker.obj
 0001:0001d166       __unwindfunclet$?init@CallVariantsWorkerFactory@LocalWorkflow@U2@@SAXXZ$489 1001e166 f   SamtoolMpileupWorker.obj
 0001:0001d16f       __unwindfunclet$?init@CallVariantsWorkerFactory@LocalWorkflow@U2@@SAXXZ$490 1001e16f f   SamtoolMpileupWorker.obj
 0001:0001d178       __unwindfunclet$?init@CallVariantsWorkerFactory@LocalWorkflow@U2@@SAXXZ$491 1001e178 f   SamtoolMpileupWorker.obj
 0001:0001d181       __unwindfunclet$?init@CallVariantsWorkerFactory@LocalWorkflow@U2@@SAXXZ$492 1001e181 f   SamtoolMpileupWorker.obj
 0001:0001d18a       __unwindfunclet$?init@CallVariantsWorkerFactory@LocalWorkflow@U2@@SAXXZ$493 1001e18a f   SamtoolMpileupWorker.obj
 0001:0001d193       __unwindfunclet$?init@CallVariantsWorkerFactory@LocalWorkflow@U2@@SAXXZ$494 1001e193 f   SamtoolMpileupWorker.obj
 0001:0001d19c       __unwindfunclet$?init@CallVariantsWorkerFactory@LocalWorkflow@U2@@SAXXZ$495 1001e19c f   SamtoolMpileupWorker.obj
 0001:0001d1a7       __unwindfunclet$?init@CallVariantsWorkerFactory@LocalWorkflow@U2@@SAXXZ$496 1001e1a7 f   SamtoolMpileupWorker.obj
 0001:0001d1af       __unwindfunclet$?init@CallVariantsWorkerFactory@LocalWorkflow@U2@@SAXXZ$497 1001e1af f   SamtoolMpileupWorker.obj
 0001:0001d1b8       __unwindfunclet$?init@CallVariantsWorkerFactory@LocalWorkflow@U2@@SAXXZ$498 1001e1b8 f   SamtoolMpileupWorker.obj
 0001:0001d1c1       __unwindfunclet$?init@CallVariantsWorkerFactory@LocalWorkflow@U2@@SAXXZ$499 1001e1c1 f   SamtoolMpileupWorker.obj
 0001:0001d1ca       __unwindfunclet$?init@CallVariantsWorkerFactory@LocalWorkflow@U2@@SAXXZ$500 1001e1ca f   SamtoolMpileupWorker.obj
 0001:0001d1d3       __unwindfunclet$?init@CallVariantsWorkerFactory@LocalWorkflow@U2@@SAXXZ$501 1001e1d3 f   SamtoolMpileupWorker.obj
 0001:0001d1dc       __unwindfunclet$?init@CallVariantsWorkerFactory@LocalWorkflow@U2@@SAXXZ$502 1001e1dc f   SamtoolMpileupWorker.obj
 0001:0001d1e5       __unwindfunclet$?init@CallVariantsWorkerFactory@LocalWorkflow@U2@@SAXXZ$503 1001e1e5 f   SamtoolMpileupWorker.obj
 0001:0001d1f0       __unwindfunclet$?init@CallVariantsWorkerFactory@LocalWorkflow@U2@@SAXXZ$504 1001e1f0 f   SamtoolMpileupWorker.obj
 0001:0001d1f8       __unwindfunclet$?init@CallVariantsWorkerFactory@LocalWorkflow@U2@@SAXXZ$505 1001e1f8 f   SamtoolMpileupWorker.obj
 0001:0001d201       __unwindfunclet$?init@CallVariantsWorkerFactory@LocalWorkflow@U2@@SAXXZ$506 1001e201 f   SamtoolMpileupWorker.obj
 0001:0001d20a       __unwindfunclet$?init@CallVariantsWorkerFactory@LocalWorkflow@U2@@SAXXZ$507 1001e20a f   SamtoolMpileupWorker.obj
 0001:0001d213       __unwindfunclet$?init@CallVariantsWorkerFactory@LocalWorkflow@U2@@SAXXZ$508 1001e213 f   SamtoolMpileupWorker.obj
 0001:0001d21c       __unwindfunclet$?init@CallVariantsWorkerFactory@LocalWorkflow@U2@@SAXXZ$509 1001e21c f   SamtoolMpileupWorker.obj
 0001:0001d225       __unwindfunclet$?init@CallVariantsWorkerFactory@LocalWorkflow@U2@@SAXXZ$510 1001e225 f   SamtoolMpileupWorker.obj
 0001:0001d22e       __unwindfunclet$?init@CallVariantsWorkerFactory@LocalWorkflow@U2@@SAXXZ$511 1001e22e f   SamtoolMpileupWorker.obj
 0001:0001d239       __unwindfunclet$?init@CallVariantsWorkerFactory@LocalWorkflow@U2@@SAXXZ$512 1001e239 f   SamtoolMpileupWorker.obj
 0001:0001d241       __unwindfunclet$?init@CallVariantsWorkerFactory@LocalWorkflow@U2@@SAXXZ$513 1001e241 f   SamtoolMpileupWorker.obj
 0001:0001d24a       __unwindfunclet$?init@CallVariantsWorkerFactory@LocalWorkflow@U2@@SAXXZ$514 1001e24a f   SamtoolMpileupWorker.obj
 0001:0001d253       __unwindfunclet$?init@CallVariantsWorkerFactory@LocalWorkflow@U2@@SAXXZ$515 1001e253 f   SamtoolMpileupWorker.obj
 0001:0001d25c       __unwindfunclet$?init@CallVariantsWorkerFactory@LocalWorkflow@U2@@SAXXZ$516 1001e25c f   SamtoolMpileupWorker.obj
 0001:0001d265       __unwindfunclet$?init@CallVariantsWorkerFactory@LocalWorkflow@U2@@SAXXZ$517 1001e265 f   SamtoolMpileupWorker.obj
 0001:0001d26e       __unwindfunclet$?init@CallVariantsWorkerFactory@LocalWorkflow@U2@@SAXXZ$518 1001e26e f   SamtoolMpileupWorker.obj
 0001:0001d277       __unwindfunclet$?init@CallVariantsWorkerFactory@LocalWorkflow@U2@@SAXXZ$519 1001e277 f   SamtoolMpileupWorker.obj
 0001:0001d282       __unwindfunclet$?init@CallVariantsWorkerFactory@LocalWorkflow@U2@@SAXXZ$520 1001e282 f   SamtoolMpileupWorker.obj
 0001:0001d28a       __unwindfunclet$?init@CallVariantsWorkerFactory@LocalWorkflow@U2@@SAXXZ$521 1001e28a f   SamtoolMpileupWorker.obj
 0001:0001d293       __unwindfunclet$?init@CallVariantsWorkerFactory@LocalWorkflow@U2@@SAXXZ$522 1001e293 f   SamtoolMpileupWorker.obj
 0001:0001d29c       __unwindfunclet$?init@CallVariantsWorkerFactory@LocalWorkflow@U2@@SAXXZ$523 1001e29c f   SamtoolMpileupWorker.obj
 0001:0001d2a5       __unwindfunclet$?init@CallVariantsWorkerFactory@LocalWorkflow@U2@@SAXXZ$524 1001e2a5 f   SamtoolMpileupWorker.obj
 0001:0001d2ae       __unwindfunclet$?init@CallVariantsWorkerFactory@LocalWorkflow@U2@@SAXXZ$525 1001e2ae f   SamtoolMpileupWorker.obj
 0001:0001d2b7       __unwindfunclet$?init@CallVariantsWorkerFactory@LocalWorkflow@U2@@SAXXZ$526 1001e2b7 f   SamtoolMpileupWorker.obj
 0001:0001d2c0       __unwindfunclet$?init@CallVariantsWorkerFactory@LocalWorkflow@U2@@SAXXZ$527 1001e2c0 f   SamtoolMpileupWorker.obj
 0001:0001d2cb       __unwindfunclet$?init@CallVariantsWorkerFactory@LocalWorkflow@U2@@SAXXZ$528 1001e2cb f   SamtoolMpileupWorker.obj
 0001:0001d2d3       __unwindfunclet$?init@CallVariantsWorkerFactory@LocalWorkflow@U2@@SAXXZ$529 1001e2d3 f   SamtoolMpileupWorker.obj
 0001:0001d2dc       __unwindfunclet$?init@CallVariantsWorkerFactory@LocalWorkflow@U2@@SAXXZ$530 1001e2dc f   SamtoolMpileupWorker.obj
 0001:0001d2e5       __unwindfunclet$?init@CallVariantsWorkerFactory@LocalWorkflow@U2@@SAXXZ$531 1001e2e5 f   SamtoolMpileupWorker.obj
 0001:0001d2ee       __unwindfunclet$?init@CallVariantsWorkerFactory@LocalWorkflow@U2@@SAXXZ$532 1001e2ee f   SamtoolMpileupWorker.obj
 0001:0001d2f7       __unwindfunclet$?init@CallVariantsWorkerFactory@LocalWorkflow@U2@@SAXXZ$533 1001e2f7 f   SamtoolMpileupWorker.obj
 0001:0001d300       __unwindfunclet$?init@CallVariantsWorkerFactory@LocalWorkflow@U2@@SAXXZ$534 1001e300 f   SamtoolMpileupWorker.obj
 0001:0001d309       __unwindfunclet$?init@CallVariantsWorkerFactory@LocalWorkflow@U2@@SAXXZ$535 1001e309 f   SamtoolMpileupWorker.obj
 0001:0001d314       __unwindfunclet$?init@CallVariantsWorkerFactory@LocalWorkflow@U2@@SAXXZ$536 1001e314 f   SamtoolMpileupWorker.obj
 0001:0001d31c       __unwindfunclet$?init@CallVariantsWorkerFactory@LocalWorkflow@U2@@SAXXZ$537 1001e31c f   SamtoolMpileupWorker.obj
 0001:0001d325       __unwindfunclet$?init@CallVariantsWorkerFactory@LocalWorkflow@U2@@SAXXZ$538 1001e325 f   SamtoolMpileupWorker.obj
 0001:0001d32e       __unwindfunclet$?init@CallVariantsWorkerFactory@LocalWorkflow@U2@@SAXXZ$539 1001e32e f   SamtoolMpileupWorker.obj
 0001:0001d337       __unwindfunclet$?init@CallVariantsWorkerFactory@LocalWorkflow@U2@@SAXXZ$540 1001e337 f   SamtoolMpileupWorker.obj
 0001:0001d340       __unwindfunclet$?init@CallVariantsWorkerFactory@LocalWorkflow@U2@@SAXXZ$541 1001e340 f   SamtoolMpileupWorker.obj
 0001:0001d349       __unwindfunclet$?init@CallVariantsWorkerFactory@LocalWorkflow@U2@@SAXXZ$542 1001e349 f   SamtoolMpileupWorker.obj
 0001:0001d352       __unwindfunclet$?init@CallVariantsWorkerFactory@LocalWorkflow@U2@@SAXXZ$543 1001e352 f   SamtoolMpileupWorker.obj
 0001:0001d35d       __unwindfunclet$?init@CallVariantsWorkerFactory@LocalWorkflow@U2@@SAXXZ$544 1001e35d f   SamtoolMpileupWorker.obj
 0001:0001d368       __unwindfunclet$?init@CallVariantsWorkerFactory@LocalWorkflow@U2@@SAXXZ$545 1001e368 f   SamtoolMpileupWorker.obj
 0001:0001d370       __unwindfunclet$?init@CallVariantsWorkerFactory@LocalWorkflow@U2@@SAXXZ$546 1001e370 f   SamtoolMpileupWorker.obj
 0001:0001d379       __unwindfunclet$?init@CallVariantsWorkerFactory@LocalWorkflow@U2@@SAXXZ$547 1001e379 f   SamtoolMpileupWorker.obj
 0001:0001d382       __unwindfunclet$?init@CallVariantsWorkerFactory@LocalWorkflow@U2@@SAXXZ$548 1001e382 f   SamtoolMpileupWorker.obj
 0001:0001d38b       __unwindfunclet$?init@CallVariantsWorkerFactory@LocalWorkflow@U2@@SAXXZ$549 1001e38b f   SamtoolMpileupWorker.obj
 0001:0001d394       __unwindfunclet$?init@CallVariantsWorkerFactory@LocalWorkflow@U2@@SAXXZ$550 1001e394 f   SamtoolMpileupWorker.obj
 0001:0001d39d       __unwindfunclet$?init@CallVariantsWorkerFactory@LocalWorkflow@U2@@SAXXZ$551 1001e39d f   SamtoolMpileupWorker.obj
 0001:0001d3a6       __unwindfunclet$?init@CallVariantsWorkerFactory@LocalWorkflow@U2@@SAXXZ$552 1001e3a6 f   SamtoolMpileupWorker.obj
 0001:0001d3b1       __unwindfunclet$?init@CallVariantsWorkerFactory@LocalWorkflow@U2@@SAXXZ$553 1001e3b1 f   SamtoolMpileupWorker.obj
 0001:0001d3b9       __unwindfunclet$?init@CallVariantsWorkerFactory@LocalWorkflow@U2@@SAXXZ$554 1001e3b9 f   SamtoolMpileupWorker.obj
 0001:0001d3c2       __unwindfunclet$?init@CallVariantsWorkerFactory@LocalWorkflow@U2@@SAXXZ$555 1001e3c2 f   SamtoolMpileupWorker.obj
 0001:0001d3cb       __unwindfunclet$?init@CallVariantsWorkerFactory@LocalWorkflow@U2@@SAXXZ$556 1001e3cb f   SamtoolMpileupWorker.obj
 0001:0001d3d4       __unwindfunclet$?init@CallVariantsWorkerFactory@LocalWorkflow@U2@@SAXXZ$557 1001e3d4 f   SamtoolMpileupWorker.obj
 0001:0001d3dd       __unwindfunclet$?init@CallVariantsWorkerFactory@LocalWorkflow@U2@@SAXXZ$558 1001e3dd f   SamtoolMpileupWorker.obj
 0001:0001d3e6       __unwindfunclet$?init@CallVariantsWorkerFactory@LocalWorkflow@U2@@SAXXZ$559 1001e3e6 f   SamtoolMpileupWorker.obj
 0001:0001d3ef       __unwindfunclet$?init@CallVariantsWorkerFactory@LocalWorkflow@U2@@SAXXZ$560 1001e3ef f   SamtoolMpileupWorker.obj
 0001:0001d3fa       __unwindfunclet$?init@CallVariantsWorkerFactory@LocalWorkflow@U2@@SAXXZ$561 1001e3fa f   SamtoolMpileupWorker.obj
 0001:0001d402       __unwindfunclet$?init@CallVariantsWorkerFactory@LocalWorkflow@U2@@SAXXZ$562 1001e402 f   SamtoolMpileupWorker.obj
 0001:0001d40b       __unwindfunclet$?init@CallVariantsWorkerFactory@LocalWorkflow@U2@@SAXXZ$563 1001e40b f   SamtoolMpileupWorker.obj
 0001:0001d414       __unwindfunclet$?init@CallVariantsWorkerFactory@LocalWorkflow@U2@@SAXXZ$564 1001e414 f   SamtoolMpileupWorker.obj
 0001:0001d41d       __unwindfunclet$?init@CallVariantsWorkerFactory@LocalWorkflow@U2@@SAXXZ$565 1001e41d f   SamtoolMpileupWorker.obj
 0001:0001d426       __unwindfunclet$?init@CallVariantsWorkerFactory@LocalWorkflow@U2@@SAXXZ$566 1001e426 f   SamtoolMpileupWorker.obj
 0001:0001d42f       __unwindfunclet$?init@CallVariantsWorkerFactory@LocalWorkflow@U2@@SAXXZ$567 1001e42f f   SamtoolMpileupWorker.obj
 0001:0001d438       __unwindfunclet$?init@CallVariantsWorkerFactory@LocalWorkflow@U2@@SAXXZ$568 1001e438 f   SamtoolMpileupWorker.obj
 0001:0001d443       __unwindfunclet$?init@CallVariantsWorkerFactory@LocalWorkflow@U2@@SAXXZ$569 1001e443 f   SamtoolMpileupWorker.obj
 0001:0001d44b       __unwindfunclet$?init@CallVariantsWorkerFactory@LocalWorkflow@U2@@SAXXZ$570 1001e44b f   SamtoolMpileupWorker.obj
 0001:0001d454       __unwindfunclet$?init@CallVariantsWorkerFactory@LocalWorkflow@U2@@SAXXZ$571 1001e454 f   SamtoolMpileupWorker.obj
 0001:0001d45d       __unwindfunclet$?init@CallVariantsWorkerFactory@LocalWorkflow@U2@@SAXXZ$572 1001e45d f   SamtoolMpileupWorker.obj
 0001:0001d466       __unwindfunclet$?init@CallVariantsWorkerFactory@LocalWorkflow@U2@@SAXXZ$573 1001e466 f   SamtoolMpileupWorker.obj
 0001:0001d46f       __unwindfunclet$?init@CallVariantsWorkerFactory@LocalWorkflow@U2@@SAXXZ$574 1001e46f f   SamtoolMpileupWorker.obj
 0001:0001d47a       __unwindfunclet$?init@CallVariantsWorkerFactory@LocalWorkflow@U2@@SAXXZ$575 1001e47a f   SamtoolMpileupWorker.obj
 0001:0001d485       __unwindfunclet$?init@CallVariantsWorkerFactory@LocalWorkflow@U2@@SAXXZ$576 1001e485 f   SamtoolMpileupWorker.obj
 0001:0001d4a4       __unwindfunclet$?init@CallVariantsWorkerFactory@LocalWorkflow@U2@@SAXXZ$577 1001e4a4 f   SamtoolMpileupWorker.obj
 0001:0001d4c3       __unwindfunclet$?init@CallVariantsWorkerFactory@LocalWorkflow@U2@@SAXXZ$578 1001e4c3 f   SamtoolMpileupWorker.obj
 0001:0001d4e2       __unwindfunclet$?init@CallVariantsWorkerFactory@LocalWorkflow@U2@@SAXXZ$579 1001e4e2 f   SamtoolMpileupWorker.obj
 0001:0001d4ed       __unwindfunclet$?init@CallVariantsWorkerFactory@LocalWorkflow@U2@@SAXXZ$580 1001e4ed f   SamtoolMpileupWorker.obj
 0001:0001d50c       __unwindfunclet$?init@CallVariantsWorkerFactory@LocalWorkflow@U2@@SAXXZ$581 1001e50c f   SamtoolMpileupWorker.obj
 0001:0001d52b       __unwindfunclet$?init@CallVariantsWorkerFactory@LocalWorkflow@U2@@SAXXZ$582 1001e52b f   SamtoolMpileupWorker.obj
 0001:0001d54a       __unwindfunclet$?init@CallVariantsWorkerFactory@LocalWorkflow@U2@@SAXXZ$583 1001e54a f   SamtoolMpileupWorker.obj
 0001:0001d555       __unwindfunclet$?init@CallVariantsWorkerFactory@LocalWorkflow@U2@@SAXXZ$584 1001e555 f   SamtoolMpileupWorker.obj
 0001:0001d574       __unwindfunclet$?init@CallVariantsWorkerFactory@LocalWorkflow@U2@@SAXXZ$585 1001e574 f   SamtoolMpileupWorker.obj
 0001:0001d593       __unwindfunclet$?init@CallVariantsWorkerFactory@LocalWorkflow@U2@@SAXXZ$586 1001e593 f   SamtoolMpileupWorker.obj
 0001:0001d5b2       __unwindfunclet$?init@CallVariantsWorkerFactory@LocalWorkflow@U2@@SAXXZ$587 1001e5b2 f   SamtoolMpileupWorker.obj
 0001:0001d5bd       __unwindfunclet$?init@CallVariantsWorkerFactory@LocalWorkflow@U2@@SAXXZ$588 1001e5bd f   SamtoolMpileupWorker.obj
 0001:0001d5d7       __unwindfunclet$?init@CallVariantsWorkerFactory@LocalWorkflow@U2@@SAXXZ$589 1001e5d7 f   SamtoolMpileupWorker.obj
 0001:0001d5f1       __unwindfunclet$?init@CallVariantsWorkerFactory@LocalWorkflow@U2@@SAXXZ$590 1001e5f1 f   SamtoolMpileupWorker.obj
 0001:0001d60b       __unwindfunclet$?init@CallVariantsWorkerFactory@LocalWorkflow@U2@@SAXXZ$591 1001e60b f   SamtoolMpileupWorker.obj
 0001:0001d616       __unwindfunclet$?init@CallVariantsWorkerFactory@LocalWorkflow@U2@@SAXXZ$592 1001e616 f   SamtoolMpileupWorker.obj
 0001:0001d621       __unwindfunclet$?init@CallVariantsWorkerFactory@LocalWorkflow@U2@@SAXXZ$593 1001e621 f   SamtoolMpileupWorker.obj
 0001:0001d62c       __unwindfunclet$?init@CallVariantsWorkerFactory@LocalWorkflow@U2@@SAXXZ$594 1001e62c f   SamtoolMpileupWorker.obj
 0001:0001d646       __unwindfunclet$?init@CallVariantsWorkerFactory@LocalWorkflow@U2@@SAXXZ$595 1001e646 f   SamtoolMpileupWorker.obj
 0001:0001d660       __unwindfunclet$?init@CallVariantsWorkerFactory@LocalWorkflow@U2@@SAXXZ$615 1001e660 f   SamtoolMpileupWorker.obj
 0001:0001d669       __unwindfunclet$?init@CallVariantsWorkerFactory@LocalWorkflow@U2@@SAXXZ$596 1001e669 f   SamtoolMpileupWorker.obj
 0001:0001d672       __unwindfunclet$?init@CallVariantsWorkerFactory@LocalWorkflow@U2@@SAXXZ$597 1001e672 f   SamtoolMpileupWorker.obj
 0001:0001d67d       __unwindfunclet$?init@CallVariantsWorkerFactory@LocalWorkflow@U2@@SAXXZ$598 1001e67d f   SamtoolMpileupWorker.obj
 0001:0001d697       __unwindfunclet$?init@CallVariantsWorkerFactory@LocalWorkflow@U2@@SAXXZ$599 1001e697 f   SamtoolMpileupWorker.obj
 0001:0001d6b1       __unwindfunclet$?init@CallVariantsWorkerFactory@LocalWorkflow@U2@@SAXXZ$617 1001e6b1 f   SamtoolMpileupWorker.obj
 0001:0001d6ba       __unwindfunclet$?init@CallVariantsWorkerFactory@LocalWorkflow@U2@@SAXXZ$600 1001e6ba f   SamtoolMpileupWorker.obj
 0001:0001d6c3       __unwindfunclet$?init@CallVariantsWorkerFactory@LocalWorkflow@U2@@SAXXZ$601 1001e6c3 f   SamtoolMpileupWorker.obj
 0001:0001d6cc       __unwindfunclet$?init@CallVariantsWorkerFactory@LocalWorkflow@U2@@SAXXZ$602 1001e6cc f   SamtoolMpileupWorker.obj
 0001:0001d6d5       __unwindfunclet$?init@CallVariantsWorkerFactory@LocalWorkflow@U2@@SAXXZ$603 1001e6d5 f   SamtoolMpileupWorker.obj
 0001:0001d6de       __unwindfunclet$?init@CallVariantsWorkerFactory@LocalWorkflow@U2@@SAXXZ$604 1001e6de f   SamtoolMpileupWorker.obj
 0001:0001d6e7       __unwindfunclet$?init@CallVariantsWorkerFactory@LocalWorkflow@U2@@SAXXZ$605 1001e6e7 f   SamtoolMpileupWorker.obj
 0001:0001d6f0       __unwindfunclet$?init@CallVariantsWorkerFactory@LocalWorkflow@U2@@SAXXZ$606 1001e6f0 f   SamtoolMpileupWorker.obj
 0001:0001d6f9       __unwindfunclet$?init@CallVariantsWorkerFactory@LocalWorkflow@U2@@SAXXZ$607 1001e6f9 f   SamtoolMpileupWorker.obj
 0001:0001d702       __unwindfunclet$?init@CallVariantsWorkerFactory@LocalWorkflow@U2@@SAXXZ$608 1001e702 f   SamtoolMpileupWorker.obj
 0001:0001d70b       __unwindfunclet$?init@CallVariantsWorkerFactory@LocalWorkflow@U2@@SAXXZ$609 1001e70b f   SamtoolMpileupWorker.obj
 0001:0001d714       __unwindfunclet$?init@CallVariantsWorkerFactory@LocalWorkflow@U2@@SAXXZ$610 1001e714 f   SamtoolMpileupWorker.obj
 0001:0001d71f       __ehhandler$?init@CallVariantsWorkerFactory@LocalWorkflow@U2@@SAXXZ 1001e71f f   SamtoolMpileupWorker.obj
 0001:0001d740       __unwindfunclet$?initDatasetMode@CallVariantsWorker@LocalWorkflow@U2@@AAEXXZ$0 1001e740 f   SamtoolMpileupWorker.obj
 0001:0001d749       __unwindfunclet$?initDatasetMode@CallVariantsWorker@LocalWorkflow@U2@@AAEXXZ$1 1001e749 f   SamtoolMpileupWorker.obj
 0001:0001d752       __unwindfunclet$?initDatasetMode@CallVariantsWorker@LocalWorkflow@U2@@AAEXXZ$2 1001e752 f   SamtoolMpileupWorker.obj
 0001:0001d75b       __unwindfunclet$?initDatasetMode@CallVariantsWorker@LocalWorkflow@U2@@AAEXXZ$3 1001e75b f   SamtoolMpileupWorker.obj
 0001:0001d764       __unwindfunclet$?initDatasetMode@CallVariantsWorker@LocalWorkflow@U2@@AAEXXZ$4 1001e764 f   SamtoolMpileupWorker.obj
 0001:0001d76d       __unwindfunclet$?initDatasetMode@CallVariantsWorker@LocalWorkflow@U2@@AAEXXZ$5 1001e76d f   SamtoolMpileupWorker.obj
 0001:0001d776       __unwindfunclet$?initDatasetMode@CallVariantsWorker@LocalWorkflow@U2@@AAEXXZ$6 1001e776 f   SamtoolMpileupWorker.obj
 0001:0001d77f       __unwindfunclet$?initDatasetMode@CallVariantsWorker@LocalWorkflow@U2@@AAEXXZ$7 1001e77f f   SamtoolMpileupWorker.obj
 0001:0001d788       __unwindfunclet$?initDatasetMode@CallVariantsWorker@LocalWorkflow@U2@@AAEXXZ$8 1001e788 f   SamtoolMpileupWorker.obj
 0001:0001d791       __unwindfunclet$?initDatasetMode@CallVariantsWorker@LocalWorkflow@U2@@AAEXXZ$9 1001e791 f   SamtoolMpileupWorker.obj
 0001:0001d79a       __unwindfunclet$?initDatasetMode@CallVariantsWorker@LocalWorkflow@U2@@AAEXXZ$10 1001e79a f   SamtoolMpileupWorker.obj
 0001:0001d7a3       __unwindfunclet$?initDatasetMode@CallVariantsWorker@LocalWorkflow@U2@@AAEXXZ$11 1001e7a3 f   SamtoolMpileupWorker.obj
 0001:0001d7ac       __unwindfunclet$?initDatasetMode@CallVariantsWorker@LocalWorkflow@U2@@AAEXXZ$12 1001e7ac f   SamtoolMpileupWorker.obj
 0001:0001d7b5       __unwindfunclet$?initDatasetMode@CallVariantsWorker@LocalWorkflow@U2@@AAEXXZ$13 1001e7b5 f   SamtoolMpileupWorker.obj
 0001:0001d7be       __unwindfunclet$?initDatasetMode@CallVariantsWorker@LocalWorkflow@U2@@AAEXXZ$14 1001e7be f   SamtoolMpileupWorker.obj
 0001:0001d7c7       __unwindfunclet$?initDatasetMode@CallVariantsWorker@LocalWorkflow@U2@@AAEXXZ$15 1001e7c7 f   SamtoolMpileupWorker.obj
 0001:0001d7cf       __ehhandler$?initDatasetMode@CallVariantsWorker@LocalWorkflow@U2@@AAEXXZ 1001e7cf f   SamtoolMpileupWorker.obj
 0001:0001d7f0       __unwindfunclet$?metaType@?$QVariantValueHelper@VQString@@@QtPrivate@@SA?AVQString@@ABVQVariant@@@Z$0 1001e7f0 f   SamtoolMpileupWorker.obj
 0001:0001d80a       __unwindfunclet$?metaType@?$QVariantValueHelper@VQString@@@QtPrivate@@SA?AVQString@@ABVQVariant@@@Z$1 1001e80a f   SamtoolMpileupWorker.obj
 0001:0001d813       __ehhandler$?metaType@?$QVariantValueHelper@VQString@@@QtPrivate@@SA?AVQString@@ABVQVariant@@@Z 1001e813 f   SamtoolMpileupWorker.obj
 0001:0001d830       __unwindfunclet$?node_construct@?$QList@VDescriptor@U2@@@@AAEXPAUNode@1@ABVDescriptor@U2@@@Z$0 1001e830 f   SamtoolMpileupWorker.obj
 0001:0001d83b       __ehhandler$?node_construct@?$QList@VDescriptor@U2@@@@AAEXPAUNode@1@ABVDescriptor@U2@@@Z 1001e83b f   SamtoolMpileupWorker.obj
 0001:0001d860       __unwindfunclet$?node_construct@?$QList@VMessage@Workflow@U2@@@@AAEXPAUNode@1@ABVMessage@Workflow@U2@@@Z$0 1001e860 f   SamtoolMpileupWorker.obj
 0001:0001d86b       __ehhandler$?node_construct@?$QList@VMessage@Workflow@U2@@@@AAEXPAUNode@1@ABVMessage@Workflow@U2@@@Z 1001e86b f   SamtoolMpileupWorker.obj
 0001:0001d890       __unwindfunclet$?node_construct@?$QList@VQVariant@@@@AAEXPAUNode@1@ABVQVariant@@@Z$0 1001e890 f   SamtoolMpileupWorker.obj
 0001:0001d89b       __ehhandler$?node_construct@?$QList@VQVariant@@@@AAEXPAUNode@1@ABVQVariant@@@Z 1001e89b f   SamtoolMpileupWorker.obj
 0001:0001d8c0       __unwindfunclet$?node_construct@?$QList@VWorkflowNotification@U2@@@@AAEXPAUNode@1@ABVWorkflowNotification@U2@@@Z$0 1001e8c0 f   SamtoolMpileupWorker.obj
 0001:0001d8cb       __ehhandler$?node_construct@?$QList@VWorkflowNotification@U2@@@@AAEXPAUNode@1@ABVWorkflowNotification@U2@@@Z 1001e8cb f   SamtoolMpileupWorker.obj
 0001:0001d8f0       __unwindfunclet$?node_copy@?$QList@VDescriptor@U2@@@@AAEXPAUNode@1@00@Z$4 1001e8f0 f   SamtoolMpileupWorker.obj
 0001:0001d8fb       __ehhandler$?node_copy@?$QList@VDescriptor@U2@@@@AAEXPAUNode@1@00@Z 1001e8fb f   SamtoolMpileupWorker.obj
 0001:0001d920       __unwindfunclet$?node_copy@?$QList@VMessage@Workflow@U2@@@@AAEXPAUNode@1@00@Z$4 1001e920 f   SamtoolMpileupWorker.obj
 0001:0001d92b       __ehhandler$?node_copy@?$QList@VMessage@Workflow@U2@@@@AAEXPAUNode@1@00@Z 1001e92b f   SamtoolMpileupWorker.obj
 0001:0001d950       __unwindfunclet$?node_copy@?$QList@VQVariant@@@@AAEXPAUNode@1@00@Z$4 1001e950 f   SamtoolMpileupWorker.obj
 0001:0001d95b       __ehhandler$?node_copy@?$QList@VQVariant@@@@AAEXPAUNode@1@00@Z 1001e95b f   SamtoolMpileupWorker.obj
 0001:0001d980       __unwindfunclet$?node_copy@?$QList@VWorkflowNotification@U2@@@@AAEXPAUNode@1@00@Z$4 1001e980 f   SamtoolMpileupWorker.obj
 0001:0001d98b       __ehhandler$?node_copy@?$QList@VWorkflowNotification@U2@@@@AAEXPAUNode@1@00@Z 1001e98b f   SamtoolMpileupWorker.obj
 0001:0001d9b0       __unwindfunclet$?processError@CallVariantsWorker@LocalWorkflow@U2@@AAEXABVU2OpStatus@3@@Z$0 1001e9b0 f   SamtoolMpileupWorker.obj
 0001:0001d9b9       __unwindfunclet$?processError@CallVariantsWorker@LocalWorkflow@U2@@AAEXABVU2OpStatus@3@@Z$1 1001e9b9 f   SamtoolMpileupWorker.obj
 0001:0001d9c2       __ehhandler$?processError@CallVariantsWorker@LocalWorkflow@U2@@AAEXABVU2OpStatus@3@@Z 1001e9c2 f   SamtoolMpileupWorker.obj
 0001:0001d9e0       __unwindfunclet$?setEditorData@ScientificDoubleDelegate@LocalWorkflow@U2@@UBEXPAVQWidget@@ABVQModelIndex@@@Z$0 1001e9e0 f   SamtoolMpileupWorker.obj
 0001:0001d9e9       __ehhandler$?setEditorData@ScientificDoubleDelegate@LocalWorkflow@U2@@UBEXPAVQWidget@@ABVQModelIndex@@@Z 1001e9e9 f   SamtoolMpileupWorker.obj
 0001:0001da10       __unwindfunclet$?setModelData@ScientificDoubleDelegate@LocalWorkflow@U2@@UBEXPAVQWidget@@PAVQAbstractItemModel@@ABVQModelIndex@@@Z$0 1001ea10 f   SamtoolMpileupWorker.obj
 0001:0001da19       __ehhandler$?setModelData@ScientificDoubleDelegate@LocalWorkflow@U2@@UBEXPAVQWidget@@PAVQAbstractItemModel@@ABVQModelIndex@@@Z 1001ea19 f   SamtoolMpileupWorker.obj
 0001:0001da40       __unwindfunclet$?setValue@ScientificDoubleWidget@LocalWorkflow@U2@@UAEXABVQVariant@@@Z$0 1001ea40 f   SamtoolMpileupWorker.obj
 0001:0001da49       __ehhandler$?setValue@ScientificDoubleWidget@LocalWorkflow@U2@@UAEXABVQVariant@@@Z 1001ea49 f   SamtoolMpileupWorker.obj
 0001:0001da70       __unwindfunclet$?sl_taskFinished@CallVariantsWorker@LocalWorkflow@U2@@AAEXXZ$0 1001ea70 f   SamtoolMpileupWorker.obj
 0001:0001da78       __unwindfunclet$?sl_taskFinished@CallVariantsWorker@LocalWorkflow@U2@@AAEXXZ$1 1001ea78 f   SamtoolMpileupWorker.obj
 0001:0001da80       __unwindfunclet$?sl_taskFinished@CallVariantsWorker@LocalWorkflow@U2@@AAEXXZ$2 1001ea80 f   SamtoolMpileupWorker.obj
 0001:0001da89       __unwindfunclet$?sl_taskFinished@CallVariantsWorker@LocalWorkflow@U2@@AAEXXZ$4 1001ea89 f   SamtoolMpileupWorker.obj
 0001:0001da92       __unwindfunclet$?sl_taskFinished@CallVariantsWorker@LocalWorkflow@U2@@AAEXXZ$5 1001ea92 f   SamtoolMpileupWorker.obj
 0001:0001da9b       __unwindfunclet$?sl_taskFinished@CallVariantsWorker@LocalWorkflow@U2@@AAEXXZ$6 1001ea9b f   SamtoolMpileupWorker.obj
 0001:0001daa4       __ehhandler$?sl_taskFinished@CallVariantsWorker@LocalWorkflow@U2@@AAEXXZ 1001eaa4 f   SamtoolMpileupWorker.obj
 0001:0001dac0       __unwindfunclet$?takeAssembly@CallVariantsWorker@LocalWorkflow@U2@@AAEXAAVU2OpStatus@3@@Z$0 1001eac0 f   SamtoolMpileupWorker.obj
 0001:0001dacc       __unwindfunclet$?takeAssembly@CallVariantsWorker@LocalWorkflow@U2@@AAEXAAVU2OpStatus@3@@Z$1 1001eacc f   SamtoolMpileupWorker.obj
 0001:0001dad5       __unwindfunclet$?takeAssembly@CallVariantsWorker@LocalWorkflow@U2@@AAEXAAVU2OpStatus@3@@Z$2 1001ead5 f   SamtoolMpileupWorker.obj
 0001:0001dadd       __unwindfunclet$?takeAssembly@CallVariantsWorker@LocalWorkflow@U2@@AAEXAAVU2OpStatus@3@@Z$3 1001eadd f   SamtoolMpileupWorker.obj
 0001:0001dae6       __unwindfunclet$?takeAssembly@CallVariantsWorker@LocalWorkflow@U2@@AAEXAAVU2OpStatus@3@@Z$4 1001eae6 f   SamtoolMpileupWorker.obj
 0001:0001daef       __unwindfunclet$?takeAssembly@CallVariantsWorker@LocalWorkflow@U2@@AAEXAAVU2OpStatus@3@@Z$5 1001eaef f   SamtoolMpileupWorker.obj
 0001:0001daf8       __unwindfunclet$?takeAssembly@CallVariantsWorker@LocalWorkflow@U2@@AAEXAAVU2OpStatus@3@@Z$6 1001eaf8 f   SamtoolMpileupWorker.obj
 0001:0001db01       __unwindfunclet$?takeAssembly@CallVariantsWorker@LocalWorkflow@U2@@AAEXAAVU2OpStatus@3@@Z$7 1001eb01 f   SamtoolMpileupWorker.obj
 0001:0001db0a       __unwindfunclet$?takeAssembly@CallVariantsWorker@LocalWorkflow@U2@@AAEXAAVU2OpStatus@3@@Z$8 1001eb0a f   SamtoolMpileupWorker.obj
 0001:0001db13       __unwindfunclet$?takeAssembly@CallVariantsWorker@LocalWorkflow@U2@@AAEXAAVU2OpStatus@3@@Z$9 1001eb13 f   SamtoolMpileupWorker.obj
 0001:0001db1c       __unwindfunclet$?takeAssembly@CallVariantsWorker@LocalWorkflow@U2@@AAEXAAVU2OpStatus@3@@Z$10 1001eb1c f   SamtoolMpileupWorker.obj
 0001:0001db25       __unwindfunclet$?takeAssembly@CallVariantsWorker@LocalWorkflow@U2@@AAEXAAVU2OpStatus@3@@Z$11 1001eb25 f   SamtoolMpileupWorker.obj
 0001:0001db2e       __unwindfunclet$?takeAssembly@CallVariantsWorker@LocalWorkflow@U2@@AAEXAAVU2OpStatus@3@@Z$12 1001eb2e f   SamtoolMpileupWorker.obj
 0001:0001db37       __unwindfunclet$?takeAssembly@CallVariantsWorker@LocalWorkflow@U2@@AAEXAAVU2OpStatus@3@@Z$13 1001eb37 f   SamtoolMpileupWorker.obj
 0001:0001db40       __ehhandler$?takeAssembly@CallVariantsWorker@LocalWorkflow@U2@@AAEXAAVU2OpStatus@3@@Z 1001eb40 f   SamtoolMpileupWorker.obj
 0001:0001db60       __unwindfunclet$?takeFirst@?$QList@VMessage@Workflow@U2@@@@QAE?AVMessage@Workflow@U2@@XZ$0 1001eb60 f   SamtoolMpileupWorker.obj
 0001:0001db7a       __ehhandler$?takeFirst@?$QList@VMessage@Workflow@U2@@@@QAE?AVMessage@Workflow@U2@@XZ 1001eb7a f   SamtoolMpileupWorker.obj
 0001:0001dba0       __unwindfunclet$?takeReference@CallVariantsWorker@LocalWorkflow@U2@@AAEXAAVU2OpStatus@3@@Z$0 1001eba0 f   SamtoolMpileupWorker.obj
 0001:0001dba9       __unwindfunclet$?takeReference@CallVariantsWorker@LocalWorkflow@U2@@AAEXAAVU2OpStatus@3@@Z$1 1001eba9 f   SamtoolMpileupWorker.obj
 0001:0001dbb2       __unwindfunclet$?takeReference@CallVariantsWorker@LocalWorkflow@U2@@AAEXAAVU2OpStatus@3@@Z$2 1001ebb2 f   SamtoolMpileupWorker.obj
 0001:0001dbba       __unwindfunclet$?takeReference@CallVariantsWorker@LocalWorkflow@U2@@AAEXAAVU2OpStatus@3@@Z$3 1001ebba f   SamtoolMpileupWorker.obj
 0001:0001dbc3       __unwindfunclet$?takeReference@CallVariantsWorker@LocalWorkflow@U2@@AAEXAAVU2OpStatus@3@@Z$4 1001ebc3 f   SamtoolMpileupWorker.obj
 0001:0001dbcc       __unwindfunclet$?takeReference@CallVariantsWorker@LocalWorkflow@U2@@AAEXAAVU2OpStatus@3@@Z$5 1001ebcc f   SamtoolMpileupWorker.obj
 0001:0001dbd5       __unwindfunclet$?takeReference@CallVariantsWorker@LocalWorkflow@U2@@AAEXAAVU2OpStatus@3@@Z$6 1001ebd5 f   SamtoolMpileupWorker.obj
 0001:0001dbde       __unwindfunclet$?takeReference@CallVariantsWorker@LocalWorkflow@U2@@AAEXAAVU2OpStatus@3@@Z$7 1001ebde f   SamtoolMpileupWorker.obj
 0001:0001dbe7       __unwindfunclet$?takeReference@CallVariantsWorker@LocalWorkflow@U2@@AAEXAAVU2OpStatus@3@@Z$8 1001ebe7 f   SamtoolMpileupWorker.obj
 0001:0001dbf0       __unwindfunclet$?takeReference@CallVariantsWorker@LocalWorkflow@U2@@AAEXAAVU2OpStatus@3@@Z$9 1001ebf0 f   SamtoolMpileupWorker.obj
 0001:0001dbf9       __unwindfunclet$?takeReference@CallVariantsWorker@LocalWorkflow@U2@@AAEXAAVU2OpStatus@3@@Z$10 1001ebf9 f   SamtoolMpileupWorker.obj
 0001:0001dc02       __ehhandler$?takeReference@CallVariantsWorker@LocalWorkflow@U2@@AAEXAAVU2OpStatus@3@@Z 1001ec02 f   SamtoolMpileupWorker.obj
 0001:0001dc20       __unwindfunclet$?tick@CallVariantsWorker@LocalWorkflow@U2@@UAEPAVTask@3@XZ$0 1001ec20 f   SamtoolMpileupWorker.obj
 0001:0001dc29       __unwindfunclet$?tick@CallVariantsWorker@LocalWorkflow@U2@@UAEPAVTask@3@XZ$1 1001ec29 f   SamtoolMpileupWorker.obj
 0001:0001dc32       __unwindfunclet$?tick@CallVariantsWorker@LocalWorkflow@U2@@UAEPAVTask@3@XZ$2 1001ec32 f   SamtoolMpileupWorker.obj
 0001:0001dc3b       __unwindfunclet$?tick@CallVariantsWorker@LocalWorkflow@U2@@UAEPAVTask@3@XZ$3 1001ec3b f   SamtoolMpileupWorker.obj
 0001:0001dc44       __unwindfunclet$?tick@CallVariantsWorker@LocalWorkflow@U2@@UAEPAVTask@3@XZ$4 1001ec44 f   SamtoolMpileupWorker.obj
 0001:0001dc4c       __unwindfunclet$?tick@CallVariantsWorker@LocalWorkflow@U2@@UAEPAVTask@3@XZ$5 1001ec4c f   SamtoolMpileupWorker.obj
 0001:0001dc55       __unwindfunclet$?tick@CallVariantsWorker@LocalWorkflow@U2@@UAEPAVTask@3@XZ$6 1001ec55 f   SamtoolMpileupWorker.obj
 0001:0001dc5e       __unwindfunclet$?tick@CallVariantsWorker@LocalWorkflow@U2@@UAEPAVTask@3@XZ$7 1001ec5e f   SamtoolMpileupWorker.obj
 0001:0001dc69       __unwindfunclet$?tick@CallVariantsWorker@LocalWorkflow@U2@@UAEPAVTask@3@XZ$8 1001ec69 f   SamtoolMpileupWorker.obj
 0001:0001dc71       __ehhandler$?tick@CallVariantsWorker@LocalWorkflow@U2@@UAEPAVTask@3@XZ 1001ec71 f   SamtoolMpileupWorker.obj
 0001:0001dc90       __unwindfunclet$?uniqueKeys@?$QMap@VDescriptor@U2@@VQVariant@@@@QBE?AV?$QList@VDescriptor@U2@@@@XZ$1 1001ec90 f   SamtoolMpileupWorker.obj
 0001:0001dca9       __ehhandler$?uniqueKeys@?$QMap@VDescriptor@U2@@VQVariant@@@@QBE?AV?$QList@VDescriptor@U2@@@@XZ 1001eca9 f   SamtoolMpileupWorker.obj
 0001:0001dcd0       __unwindfunclet$?validate@EmptySlotValidator@LocalWorkflow@U2@@UBE_NPBVConfiguration@3@AAV?$QList@VWorkflowNotification@U2@@@@@Z$0 1001ecd0 f   SamtoolMpileupWorker.obj
 0001:0001dcd8       __unwindfunclet$?validate@EmptySlotValidator@LocalWorkflow@U2@@UBE_NPBVConfiguration@3@AAV?$QList@VWorkflowNotification@U2@@@@@Z$1 1001ecd8 f   SamtoolMpileupWorker.obj
 0001:0001dce0       __unwindfunclet$?validate@EmptySlotValidator@LocalWorkflow@U2@@UBE_NPBVConfiguration@3@AAV?$QList@VWorkflowNotification@U2@@@@@Z$2 1001ece0 f   SamtoolMpileupWorker.obj
 0001:0001dce8       __unwindfunclet$?validate@EmptySlotValidator@LocalWorkflow@U2@@UBE_NPBVConfiguration@3@AAV?$QList@VWorkflowNotification@U2@@@@@Z$3 1001ece8 f   SamtoolMpileupWorker.obj
 0001:0001dcf1       __unwindfunclet$?validate@EmptySlotValidator@LocalWorkflow@U2@@UBE_NPBVConfiguration@3@AAV?$QList@VWorkflowNotification@U2@@@@@Z$4 1001ecf1 f   SamtoolMpileupWorker.obj
 0001:0001dcfa       __unwindfunclet$?validate@EmptySlotValidator@LocalWorkflow@U2@@UBE_NPBVConfiguration@3@AAV?$QList@VWorkflowNotification@U2@@@@@Z$5 1001ecfa f   SamtoolMpileupWorker.obj
 0001:0001dd03       __unwindfunclet$?validate@EmptySlotValidator@LocalWorkflow@U2@@UBE_NPBVConfiguration@3@AAV?$QList@VWorkflowNotification@U2@@@@@Z$6 1001ed03 f   SamtoolMpileupWorker.obj
 0001:0001dd0c       __unwindfunclet$?validate@EmptySlotValidator@LocalWorkflow@U2@@UBE_NPBVConfiguration@3@AAV?$QList@VWorkflowNotification@U2@@@@@Z$7 1001ed0c f   SamtoolMpileupWorker.obj
 0001:0001dd15       __unwindfunclet$?validate@EmptySlotValidator@LocalWorkflow@U2@@UBE_NPBVConfiguration@3@AAV?$QList@VWorkflowNotification@U2@@@@@Z$8 1001ed15 f   SamtoolMpileupWorker.obj
 0001:0001dd1e       __ehhandler$?validate@EmptySlotValidator@LocalWorkflow@U2@@UBE_NPBVConfiguration@3@AAV?$QList@VWorkflowNotification@U2@@@@@Z 1001ed1e f   SamtoolMpileupWorker.obj
 0001:0001dd40       __unwindfunclet$?value@ScientificDoubleWidget@LocalWorkflow@U2@@UAE?AVQVariant@@XZ$0 1001ed40 f   SamtoolMpileupWorker.obj
 0001:0001dd49       __unwindfunclet$?value@ScientificDoubleWidget@LocalWorkflow@U2@@UAE?AVQVariant@@XZ$1 1001ed49 f   SamtoolMpileupWorker.obj
 0001:0001dd63       __ehhandler$?value@ScientificDoubleWidget@LocalWorkflow@U2@@UAE?AVQVariant@@XZ 1001ed63 f   SamtoolMpileupWorker.obj
 0001:0001dd80       __unwindfunclet$??0SamtoolsPlugin@U2@@QAE@XZ$0 1001ed80 f   SamtoolsPlugin.obj
 0001:0001dd89       __unwindfunclet$??0SamtoolsPlugin@U2@@QAE@XZ$1 1001ed89 f   SamtoolsPlugin.obj
 0001:0001dd92       __unwindfunclet$??0SamtoolsPlugin@U2@@QAE@XZ$2 1001ed92 f   SamtoolsPlugin.obj
 0001:0001dd9b       __ehhandler$??0SamtoolsPlugin@U2@@QAE@XZ 1001ed9b f   SamtoolsPlugin.obj
 0001:0001ddc0       __unwindfunclet$??__EalgoLog@U2@@YAXXZ$0 1001edc0 f   SamtoolsPlugin.obj
 0001:0001ddc9       __ehhandler$??__EalgoLog@U2@@YAXXZ 1001edc9 f   SamtoolsPlugin.obj
 0001:0001ddf0       __unwindfunclet$??__EcmdLog@U2@@YAXXZ$0 1001edf0 f   SamtoolsPlugin.obj
 0001:0001ddf9       __ehhandler$??__EcmdLog@U2@@YAXXZ 1001edf9 f   SamtoolsPlugin.obj
 0001:0001de20       __unwindfunclet$??__EcoreLog@U2@@YAXXZ$0 1001ee20 f   SamtoolsPlugin.obj
 0001:0001de29       __ehhandler$??__EcoreLog@U2@@YAXXZ 1001ee29 f   SamtoolsPlugin.obj
 0001:0001de50       __unwindfunclet$??__EioLog@U2@@YAXXZ$0 1001ee50 f   SamtoolsPlugin.obj
 0001:0001de59       __ehhandler$??__EioLog@U2@@YAXXZ 1001ee59 f   SamtoolsPlugin.obj
 0001:0001de80       __unwindfunclet$??__EperfLog@U2@@YAXXZ$0 1001ee80 f   SamtoolsPlugin.obj
 0001:0001de89       __ehhandler$??__EperfLog@U2@@YAXXZ 1001ee89 f   SamtoolsPlugin.obj
 0001:0001deb0       __unwindfunclet$??__EscriptLog@U2@@YAXXZ$0 1001eeb0 f   SamtoolsPlugin.obj
 0001:0001deb9       __ehhandler$??__EscriptLog@U2@@YAXXZ 1001eeb9 f   SamtoolsPlugin.obj
 0001:0001dee0       __unwindfunclet$??__EtaskLog@U2@@YAXXZ$0 1001eee0 f   SamtoolsPlugin.obj
 0001:0001dee9       __ehhandler$??__EtaskLog@U2@@YAXXZ 1001eee9 f   SamtoolsPlugin.obj
 0001:0001df10       __unwindfunclet$??__EuiLog@U2@@YAXXZ$0 1001ef10 f   SamtoolsPlugin.obj
 0001:0001df19       __ehhandler$??__EuiLog@U2@@YAXXZ 1001ef19 f   SamtoolsPlugin.obj
 0001:0001df40       __unwindfunclet$??__EuserActLog@U2@@YAXXZ$0 1001ef40 f   SamtoolsPlugin.obj
 0001:0001df49       __ehhandler$??__EuserActLog@U2@@YAXXZ 1001ef49 f   SamtoolsPlugin.obj
 0001:0001df70       __unwindfunclet$??__EalgoLog@U2@@YAXXZ$0 1001ef70 f   moc_AssemblySamtoolsMpileup.obj
 0001:0001df79       __ehhandler$??__EalgoLog@U2@@YAXXZ 1001ef79 f   moc_AssemblySamtoolsMpileup.obj
 0001:0001dfa0       __unwindfunclet$??__EcmdLog@U2@@YAXXZ$0 1001efa0 f   moc_AssemblySamtoolsMpileup.obj
 0001:0001dfa9       __ehhandler$??__EcmdLog@U2@@YAXXZ 1001efa9 f   moc_AssemblySamtoolsMpileup.obj
 0001:0001dfd0       __unwindfunclet$??__EcoreLog@U2@@YAXXZ$0 1001efd0 f   moc_AssemblySamtoolsMpileup.obj
 0001:0001dfd9       __ehhandler$??__EcoreLog@U2@@YAXXZ 1001efd9 f   moc_AssemblySamtoolsMpileup.obj
 0001:0001e000       __unwindfunclet$??__EioLog@U2@@YAXXZ$0 1001f000 f   moc_AssemblySamtoolsMpileup.obj
 0001:0001e009       __ehhandler$??__EioLog@U2@@YAXXZ 1001f009 f   moc_AssemblySamtoolsMpileup.obj
 0001:0001e030       __unwindfunclet$??__EperfLog@U2@@YAXXZ$0 1001f030 f   moc_AssemblySamtoolsMpileup.obj
 0001:0001e039       __ehhandler$??__EperfLog@U2@@YAXXZ 1001f039 f   moc_AssemblySamtoolsMpileup.obj
 0001:0001e060       __unwindfunclet$??__EscriptLog@U2@@YAXXZ$0 1001f060 f   moc_AssemblySamtoolsMpileup.obj
 0001:0001e069       __ehhandler$??__EscriptLog@U2@@YAXXZ 1001f069 f   moc_AssemblySamtoolsMpileup.obj
 0001:0001e090       __unwindfunclet$??__EtaskLog@U2@@YAXXZ$0 1001f090 f   moc_AssemblySamtoolsMpileup.obj
 0001:0001e099       __ehhandler$??__EtaskLog@U2@@YAXXZ 1001f099 f   moc_AssemblySamtoolsMpileup.obj
 0001:0001e0c0       __unwindfunclet$??__EuiLog@U2@@YAXXZ$0 1001f0c0 f   moc_AssemblySamtoolsMpileup.obj
 0001:0001e0c9       __ehhandler$??__EuiLog@U2@@YAXXZ 1001f0c9 f   moc_AssemblySamtoolsMpileup.obj
 0001:0001e0f0       __unwindfunclet$??__EuserActLog@U2@@YAXXZ$0 1001f0f0 f   moc_AssemblySamtoolsMpileup.obj
 0001:0001e0f9       __ehhandler$??__EuserActLog@U2@@YAXXZ 1001f0f9 f   moc_AssemblySamtoolsMpileup.obj
 0001:0001e120       __unwindfunclet$??__EalgoLog@U2@@YAXXZ$0 1001f120 f   moc_SamtoolMpileupWorker.obj
 0001:0001e129       __ehhandler$??__EalgoLog@U2@@YAXXZ 1001f129 f   moc_SamtoolMpileupWorker.obj
 0001:0001e150       __unwindfunclet$??__EcmdLog@U2@@YAXXZ$0 1001f150 f   moc_SamtoolMpileupWorker.obj
 0001:0001e159       __ehhandler$??__EcmdLog@U2@@YAXXZ 1001f159 f   moc_SamtoolMpileupWorker.obj
 0001:0001e180       __unwindfunclet$??__EcoreLog@U2@@YAXXZ$0 1001f180 f   moc_SamtoolMpileupWorker.obj
 0001:0001e189       __ehhandler$??__EcoreLog@U2@@YAXXZ 1001f189 f   moc_SamtoolMpileupWorker.obj
 0001:0001e1b0       __unwindfunclet$??__EioLog@U2@@YAXXZ$0 1001f1b0 f   moc_SamtoolMpileupWorker.obj
 0001:0001e1b9       __ehhandler$??__EioLog@U2@@YAXXZ 1001f1b9 f   moc_SamtoolMpileupWorker.obj
 0001:0001e1e0       __unwindfunclet$??__EperfLog@U2@@YAXXZ$0 1001f1e0 f   moc_SamtoolMpileupWorker.obj
 0001:0001e1e9       __ehhandler$??__EperfLog@U2@@YAXXZ 1001f1e9 f   moc_SamtoolMpileupWorker.obj
 0001:0001e210       __unwindfunclet$??__EscriptLog@U2@@YAXXZ$0 1001f210 f   moc_SamtoolMpileupWorker.obj
 0001:0001e219       __ehhandler$??__EscriptLog@U2@@YAXXZ 1001f219 f   moc_SamtoolMpileupWorker.obj
 0001:0001e240       __unwindfunclet$??__EtaskLog@U2@@YAXXZ$0 1001f240 f   moc_SamtoolMpileupWorker.obj
 0001:0001e249       __ehhandler$??__EtaskLog@U2@@YAXXZ 1001f249 f   moc_SamtoolMpileupWorker.obj
 0001:0001e270       __unwindfunclet$??__EuiLog@U2@@YAXXZ$0 1001f270 f   moc_SamtoolMpileupWorker.obj
 0001:0001e279       __ehhandler$??__EuiLog@U2@@YAXXZ 1001f279 f   moc_SamtoolMpileupWorker.obj
 0001:0001e2a0       __unwindfunclet$??__EuserActLog@U2@@YAXXZ$0 1001f2a0 f   moc_SamtoolMpileupWorker.obj
 0001:0001e2a9       __ehhandler$??__EuserActLog@U2@@YAXXZ 1001f2a9 f   moc_SamtoolMpileupWorker.obj
 0001:0001e2d0       ??__F?BCFTOOLS_ID@SamtoolsMpileupTask@LocalWorkflow@U2@@0VQString@@B@@YAXXZ 1001f2d0 f   AssemblySamtoolsMpileup.obj
 0001:0001e2e0       ??__F?SAMTOOLS_ID@SamtoolsMpileupTask@LocalWorkflow@U2@@0VQString@@B@@YAXXZ 1001f2e0 f   AssemblySamtoolsMpileup.obj
 0001:0001e2f0       ??__F?VCFUTILS_ID@SamtoolsMpileupTask@LocalWorkflow@U2@@0VQString@@B@@YAXXZ 1001f2f0 f   AssemblySamtoolsMpileup.obj
 0001:0001e300       ??__F?_Generic_object@?$_Error_objects@H@std@@2V_Generic_error_category@2@A@@YAXXZ 1001f300 f   AssemblySamtoolsMpileup.obj
 0001:0001e310       ??__F?_Iostream_object@?$_Error_objects@H@std@@2V_Iostream_error_category@2@A@@YAXXZ 1001f310 f   AssemblySamtoolsMpileup.obj
 0001:0001e320       ??__F?_System_object@?$_Error_objects@H@std@@2V_System_error_category@2@A@@YAXXZ 1001f320 f   AssemblySamtoolsMpileup.obj
 0001:0001e330       ??__FalgoLog@U2@@YAXXZ     1001f330 f   AssemblySamtoolsMpileup.obj
 0001:0001e340       ??__FcmdLog@U2@@YAXXZ      1001f340 f   AssemblySamtoolsMpileup.obj
 0001:0001e350       ??__FcoreLog@U2@@YAXXZ     1001f350 f   AssemblySamtoolsMpileup.obj
 0001:0001e360       ??__Fcvar@?1???0CallVariantsTask@LocalWorkflow@U2@@QAE@ABVCallVariantsTaskSettings@12@PAVDbiDataStorage@Workflow@2@@Z@YAXXZ 1001f360 f   AssemblySamtoolsMpileup.obj
 0001:0001e370       ??__FioLog@U2@@YAXXZ       1001f370 f   AssemblySamtoolsMpileup.obj
 0001:0001e380       ??__FperfLog@U2@@YAXXZ     1001f380 f   AssemblySamtoolsMpileup.obj
 0001:0001e390       ??__FscriptLog@U2@@YAXXZ   1001f390 f   AssemblySamtoolsMpileup.obj
 0001:0001e3a0       ??__FtaskLog@U2@@YAXXZ     1001f3a0 f   AssemblySamtoolsMpileup.obj
 0001:0001e3b0       ??__FuiLog@U2@@YAXXZ       1001f3b0 f   AssemblySamtoolsMpileup.obj
 0001:0001e3c0       ??__FuserActLog@U2@@YAXXZ  1001f3c0 f   AssemblySamtoolsMpileup.obj
 0001:0001e3d0       ??__F?ACTOR_ID@CallVariantsWorkerFactory@LocalWorkflow@U2@@2VQString@@B@@YAXXZ 1001f3d0 f   SamtoolMpileupWorker.obj
 0001:0001e3e0       ??__F?_Generic_object@?$_Error_objects@H@std@@2V_Generic_error_category@2@A@@YAXXZ 1001f3e0 f   SamtoolMpileupWorker.obj
 0001:0001e3f0       ??__F?_Iostream_object@?$_Error_objects@H@std@@2V_Iostream_error_category@2@A@@YAXXZ 1001f3f0 f   SamtoolMpileupWorker.obj
 0001:0001e400       ??__F?_System_object@?$_Error_objects@H@std@@2V_System_error_category@2@A@@YAXXZ 1001f400 f   SamtoolMpileupWorker.obj
 0001:0001e410       ??__FACGT_ONLY@LocalWorkflow@U2@@YAXXZ 1001f410 f   SamtoolMpileupWorker.obj
 0001:0001e420       ??__FASSEMBLY_PORT_ID@LocalWorkflow@U2@@YAXXZ 1001f420 f   SamtoolMpileupWorker.obj
 0001:0001e430       ??__FBCF_BED@LocalWorkflow@U2@@YAXXZ 1001f430 f   SamtoolMpileupWorker.obj
 0001:0001e440       ??__FBED@LocalWorkflow@U2@@YAXXZ 1001f440 f   SamtoolMpileupWorker.obj
 0001:0001e450       ??__FCALL_GT@LocalWorkflow@U2@@YAXXZ 1001f450 f   SamtoolMpileupWorker.obj
 0001:0001e460       ??__FCAPQ_THRES@LocalWorkflow@U2@@YAXXZ 1001f460 f   SamtoolMpileupWorker.obj
 0001:0001e470       ??__FCCALL@LocalWorkflow@U2@@YAXXZ 1001f470 f   SamtoolMpileupWorker.obj
 0001:0001e480       ??__FDISABLE_BAQ@LocalWorkflow@U2@@YAXXZ 1001f480 f   SamtoolMpileupWorker.obj
 0001:0001e490       ??__FEXTQ@LocalWorkflow@U2@@YAXXZ 1001f490 f   SamtoolMpileupWorker.obj
 0001:0001e4a0       ??__FEXT_BAQ@LocalWorkflow@U2@@YAXXZ 1001f4a0 f   SamtoolMpileupWorker.obj
 0001:0001e4b0       ??__FFIX_PL@LocalWorkflow@U2@@YAXXZ 1001f4b0 f   SamtoolMpileupWorker.obj
 0001:0001e4c0       ??__FGAP_SIZE@LocalWorkflow@U2@@YAXXZ 1001f4c0 f   SamtoolMpileupWorker.obj
 0001:0001e4d0       ??__FILLUMINA13@LocalWorkflow@U2@@YAXXZ 1001f4d0 f   SamtoolMpileupWorker.obj
 0001:0001e4e0       ??__FINDEL_FRAC@LocalWorkflow@U2@@YAXXZ 1001f4e0 f   SamtoolMpileupWorker.obj
 0001:0001e4f0       ??__FKEEPALT@LocalWorkflow@U2@@YAXXZ 1001f4f0 f   SamtoolMpileupWorker.obj
 0001:0001e500       ??__FMAX_DEP@LocalWorkflow@U2@@YAXXZ 1001f500 f   SamtoolMpileupWorker.obj
 0001:0001e510       ??__FMAX_DEPTH@LocalWorkflow@U2@@YAXXZ 1001f510 f   SamtoolMpileupWorker.obj
 0001:0001e520       ??__FMAX_INDEL_DEPTH@LocalWorkflow@U2@@YAXXZ 1001f520 f   SamtoolMpileupWorker.obj
 0001:0001e530       ??__FMIN_ALT@LocalWorkflow@U2@@YAXXZ 1001f530 f   SamtoolMpileupWorker.obj
 0001:0001e540       ??__FMIN_BASEQ@LocalWorkflow@U2@@YAXXZ 1001f540 f   SamtoolMpileupWorker.obj
 0001:0001e550       ??__FMIN_DEP@LocalWorkflow@U2@@YAXXZ 1001f550 f   SamtoolMpileupWorker.obj
 0001:0001e560       ??__FMIN_MQ@LocalWorkflow@U2@@YAXXZ 1001f560 f   SamtoolMpileupWorker.obj
 0001:0001e570       ??__FMIN_PERM_P@LocalWorkflow@U2@@YAXXZ 1001f570 f   SamtoolMpileupWorker.obj
 0001:0001e580       ??__FMIN_QUAL@LocalWorkflow@U2@@YAXXZ 1001f580 f   SamtoolMpileupWorker.obj
 0001:0001e590       ??__FMIN_SMPL_FRAC@LocalWorkflow@U2@@YAXXZ 1001f590 f   SamtoolMpileupWorker.obj
 0001:0001e5a0       ??__FN1@LocalWorkflow@U2@@YAXXZ 1001f5a0 f   SamtoolMpileupWorker.obj
 0001:0001e5b0       ??__FNO_GENO@LocalWorkflow@U2@@YAXXZ 1001f5b0 f   SamtoolMpileupWorker.obj
 0001:0001e5c0       ??__FNO_INDEL@LocalWorkflow@U2@@YAXXZ 1001f5c0 f   SamtoolMpileupWorker.obj
 0001:0001e5d0       ??__FN_PERM@LocalWorkflow@U2@@YAXXZ 1001f5d0 f   SamtoolMpileupWorker.obj
 0001:0001e5e0       ??__FOPENQ@LocalWorkflow@U2@@YAXXZ 1001f5e0 f   SamtoolMpileupWorker.obj
 0001:0001e5f0       ??__FOUT_URL@LocalWorkflow@U2@@YAXXZ 1001f5f0 f   SamtoolMpileupWorker.obj
 0001:0001e600       ??__FPL_LIST@LocalWorkflow@U2@@YAXXZ 1001f600 f   SamtoolMpileupWorker.obj
 0001:0001e610       ??__FPREF@LocalWorkflow@U2@@YAXXZ 1001f610 f   SamtoolMpileupWorker.obj
 0001:0001e620       ??__FPRINT@LocalWorkflow@U2@@YAXXZ 1001f620 f   SamtoolMpileupWorker.obj
 0001:0001e630       ??__FPTYPE@LocalWorkflow@U2@@YAXXZ 1001f630 f   SamtoolMpileupWorker.obj
 0001:0001e640       ??__FPVALUE1@LocalWorkflow@U2@@YAXXZ 1001f640 f   SamtoolMpileupWorker.obj
 0001:0001e650       ??__FPVALUE2@LocalWorkflow@U2@@YAXXZ 1001f650 f   SamtoolMpileupWorker.obj
 0001:0001e660       ??__FPVALUE3@LocalWorkflow@U2@@YAXXZ 1001f660 f   SamtoolMpileupWorker.obj
 0001:0001e670       ??__FPVALUE4@LocalWorkflow@U2@@YAXXZ 1001f670 f   SamtoolMpileupWorker.obj
 0001:0001e680       ??__FPVALUE_HWE@LocalWorkflow@U2@@YAXXZ 1001f680 f   SamtoolMpileupWorker.obj
 0001:0001e690       ??__FQCALL@LocalWorkflow@U2@@YAXXZ 1001f690 f   SamtoolMpileupWorker.obj
 0001:0001e6a0       ??__FREF_SEQ_PORT_ID@LocalWorkflow@U2@@YAXXZ 1001f6a0 f   SamtoolMpileupWorker.obj
 0001:0001e6b0       ??__FREF_SOURCE@LocalWorkflow@U2@@YAXXZ 1001f6b0 f   SamtoolMpileupWorker.obj
 0001:0001e6c0       ??__FREF_SOURCE_FILE@LocalWorkflow@U2@@YAXXZ 1001f6c0 f   SamtoolMpileupWorker.obj
 0001:0001e6d0       ??__FREF_SOURCE_PORT@LocalWorkflow@U2@@YAXXZ 1001f6d0 f   SamtoolMpileupWorker.obj
 0001:0001e6e0       ??__FREF_URL@LocalWorkflow@U2@@YAXXZ 1001f6e0 f   SamtoolMpileupWorker.obj
 0001:0001e6f0       ??__FREG@LocalWorkflow@U2@@YAXXZ 1001f6f0 f   SamtoolMpileupWorker.obj
 0001:0001e700       ??__FSAMPLES@LocalWorkflow@U2@@YAXXZ 1001f700 f   SamtoolMpileupWorker.obj
 0001:0001e710       ??__FTANDEMQ@LocalWorkflow@U2@@YAXXZ 1001f710 f   SamtoolMpileupWorker.obj
 0001:0001e720       ??__FTHETA@LocalWorkflow@U2@@YAXXZ 1001f720 f   SamtoolMpileupWorker.obj
 0001:0001e730       ??__FUSE_ORPHAN@LocalWorkflow@U2@@YAXXZ 1001f730 f   SamtoolMpileupWorker.obj
 0001:0001e740       ??__FWINDOW@LocalWorkflow@U2@@YAXXZ 1001f740 f   SamtoolMpileupWorker.obj
 0001:0001e750       ??__FalgoLog@U2@@YAXXZ     1001f750 f   SamtoolMpileupWorker.obj
 0001:0001e760       ??__FcmdLog@U2@@YAXXZ      1001f760 f   SamtoolMpileupWorker.obj
 0001:0001e770       ??__FcoreLog@U2@@YAXXZ     1001f770 f   SamtoolMpileupWorker.obj
 0001:0001e780       ??__FioLog@U2@@YAXXZ       1001f780 f   SamtoolMpileupWorker.obj
 0001:0001e790       ??__FperfLog@U2@@YAXXZ     1001f790 f   SamtoolMpileupWorker.obj
 0001:0001e7a0       ??__FscriptLog@U2@@YAXXZ   1001f7a0 f   SamtoolMpileupWorker.obj
 0001:0001e7b0       ??__FtaskLog@U2@@YAXXZ     1001f7b0 f   SamtoolMpileupWorker.obj
 0001:0001e7c0       ??__FuiLog@U2@@YAXXZ       1001f7c0 f   SamtoolMpileupWorker.obj
 0001:0001e7d0       ??__FuserActLog@U2@@YAXXZ  1001f7d0 f   SamtoolMpileupWorker.obj
 0001:0001e7e0       ??__F?_Generic_object@?$_Error_objects@H@std@@2V_Generic_error_category@2@A@@YAXXZ 1001f7e0 f   SamtoolsPlugin.obj
 0001:0001e7f0       ??__F?_Iostream_object@?$_Error_objects@H@std@@2V_Iostream_error_category@2@A@@YAXXZ 1001f7f0 f   SamtoolsPlugin.obj
 0001:0001e800       ??__F?_System_object@?$_Error_objects@H@std@@2V_System_error_category@2@A@@YAXXZ 1001f800 f   SamtoolsPlugin.obj
 0001:0001e810       ??__FalgoLog@U2@@YAXXZ     1001f810 f   SamtoolsPlugin.obj
 0001:0001e820       ??__FcmdLog@U2@@YAXXZ      1001f820 f   SamtoolsPlugin.obj
 0001:0001e830       ??__FcoreLog@U2@@YAXXZ     1001f830 f   SamtoolsPlugin.obj
 0001:0001e840       ??__FioLog@U2@@YAXXZ       1001f840 f   SamtoolsPlugin.obj
 0001:0001e850       ??__FperfLog@U2@@YAXXZ     1001f850 f   SamtoolsPlugin.obj
 0001:0001e860       ??__FscriptLog@U2@@YAXXZ   1001f860 f   SamtoolsPlugin.obj
 0001:0001e870       ??__FtaskLog@U2@@YAXXZ     1001f870 f   SamtoolsPlugin.obj
 0001:0001e880       ??__FuiLog@U2@@YAXXZ       1001f880 f   SamtoolsPlugin.obj
 0001:0001e890       ??__FuserActLog@U2@@YAXXZ  1001f890 f   SamtoolsPlugin.obj
 0001:0001e8a0       ??__F?_Generic_object@?$_Error_objects@H@std@@2V_Generic_error_category@2@A@@YAXXZ 1001f8a0 f   moc_AssemblySamtoolsMpileup.obj
 0001:0001e8b0       ??__F?_Iostream_object@?$_Error_objects@H@std@@2V_Iostream_error_category@2@A@@YAXXZ 1001f8b0 f   moc_AssemblySamtoolsMpileup.obj
 0001:0001e8c0       ??__F?_System_object@?$_Error_objects@H@std@@2V_System_error_category@2@A@@YAXXZ 1001f8c0 f   moc_AssemblySamtoolsMpileup.obj
 0001:0001e8d0       ??__FalgoLog@U2@@YAXXZ     1001f8d0 f   moc_AssemblySamtoolsMpileup.obj
 0001:0001e8e0       ??__FcmdLog@U2@@YAXXZ      1001f8e0 f   moc_AssemblySamtoolsMpileup.obj
 0001:0001e8f0       ??__FcoreLog@U2@@YAXXZ     1001f8f0 f   moc_AssemblySamtoolsMpileup.obj
 0001:0001e900       ??__FioLog@U2@@YAXXZ       1001f900 f   moc_AssemblySamtoolsMpileup.obj
 0001:0001e910       ??__FperfLog@U2@@YAXXZ     1001f910 f   moc_AssemblySamtoolsMpileup.obj
 0001:0001e920       ??__FscriptLog@U2@@YAXXZ   1001f920 f   moc_AssemblySamtoolsMpileup.obj
 0001:0001e930       ??__FtaskLog@U2@@YAXXZ     1001f930 f   moc_AssemblySamtoolsMpileup.obj
 0001:0001e940       ??__FuiLog@U2@@YAXXZ       1001f940 f   moc_AssemblySamtoolsMpileup.obj
 0001:0001e950       ??__FuserActLog@U2@@YAXXZ  1001f950 f   moc_AssemblySamtoolsMpileup.obj
 0001:0001e960       ??__F?_Generic_object@?$_Error_objects@H@std@@2V_Generic_error_category@2@A@@YAXXZ 1001f960 f   moc_SamtoolMpileupWorker.obj
 0001:0001e970       ??__F?_Iostream_object@?$_Error_objects@H@std@@2V_Iostream_error_category@2@A@@YAXXZ 1001f970 f   moc_SamtoolMpileupWorker.obj
 0001:0001e980       ??__F?_System_object@?$_Error_objects@H@std@@2V_System_error_category@2@A@@YAXXZ 1001f980 f   moc_SamtoolMpileupWorker.obj
 0001:0001e990       ??__FalgoLog@U2@@YAXXZ     1001f990 f   moc_SamtoolMpileupWorker.obj
 0001:0001e9a0       ??__FcmdLog@U2@@YAXXZ      1001f9a0 f   moc_SamtoolMpileupWorker.obj
 0001:0001e9b0       ??__FcoreLog@U2@@YAXXZ     1001f9b0 f   moc_SamtoolMpileupWorker.obj
 0001:0001e9c0       ??__FioLog@U2@@YAXXZ       1001f9c0 f   moc_SamtoolMpileupWorker.obj
 0001:0001e9d0       ??__FperfLog@U2@@YAXXZ     1001f9d0 f   moc_SamtoolMpileupWorker.obj
 0001:0001e9e0       ??__FscriptLog@U2@@YAXXZ   1001f9e0 f   moc_SamtoolMpileupWorker.obj
 0001:0001e9f0       ??__FtaskLog@U2@@YAXXZ     1001f9f0 f   moc_SamtoolMpileupWorker.obj
 0001:0001ea00       ??__FuiLog@U2@@YAXXZ       1001fa00 f   moc_SamtoolMpileupWorker.obj
 0001:0001ea10       ??__FuserActLog@U2@@YAXXZ  1001fa10 f   moc_SamtoolMpileupWorker.obj
 0001:0001ea20       ??__F?_Generic_object@?$_Error_objects@H@std@@2V_Generic_error_category@2@A@@YAXXZ 1001fa20 f   moc_SamtoolsPlugin.obj
 0001:0001ea30       ??__F?_Iostream_object@?$_Error_objects@H@std@@2V_Iostream_error_category@2@A@@YAXXZ 1001fa30 f   moc_SamtoolsPlugin.obj
 0001:0001ea40       ??__F?_System_object@?$_Error_objects@H@std@@2V_System_error_category@2@A@@YAXXZ 1001fa40 f   moc_SamtoolsPlugin.obj
 0002:000008d0       _algoLog$initializer$      100208d0     AssemblySamtoolsMpileup.obj
 0002:000008d4       _cmdLog$initializer$       100208d4     AssemblySamtoolsMpileup.obj
 0002:000008d8       _coreLog$initializer$      100208d8     AssemblySamtoolsMpileup.obj
 0002:000008dc       _ioLog$initializer$        100208dc     AssemblySamtoolsMpileup.obj
 0002:000008e0       _perfLog$initializer$      100208e0     AssemblySamtoolsMpileup.obj
 0002:000008e4       _scriptLog$initializer$    100208e4     AssemblySamtoolsMpileup.obj
 0002:000008e8       _taskLog$initializer$      100208e8     AssemblySamtoolsMpileup.obj
 0002:000008ec       _uiLog$initializer$        100208ec     AssemblySamtoolsMpileup.obj
 0002:000008f0       _userActLog$initializer$   100208f0     AssemblySamtoolsMpileup.obj
 0002:000008f4       ?SAMTOOLS_ID$initializer$@SamtoolsMpileupTask@LocalWorkflow@U2@@0P6AXXZA 100208f4     AssemblySamtoolsMpileup.obj
 0002:000008f8       ?BCFTOOLS_ID$initializer$@SamtoolsMpileupTask@LocalWorkflow@U2@@0P6AXXZA 100208f8     AssemblySamtoolsMpileup.obj
 0002:000008fc       ?VCFUTILS_ID$initializer$@SamtoolsMpileupTask@LocalWorkflow@U2@@0P6AXXZA 100208fc     AssemblySamtoolsMpileup.obj
 0002:00000900       ?_Generic_object$initializer$@?$_Error_objects@H@std@@2P6AXXZA 10020900     AssemblySamtoolsMpileup.obj
 0002:00000904       ?_Iostream_object$initializer$@?$_Error_objects@H@std@@2P6AXXZA 10020904     AssemblySamtoolsMpileup.obj
 0002:00000908       ?_System_object$initializer$@?$_Error_objects@H@std@@2P6AXXZA 10020908     AssemblySamtoolsMpileup.obj
 0002:0000090c       _algoLog$initializer$      1002090c     SamtoolMpileupWorker.obj
 0002:00000910       _cmdLog$initializer$       10020910     SamtoolMpileupWorker.obj
 0002:00000914       _coreLog$initializer$      10020914     SamtoolMpileupWorker.obj
 0002:00000918       _ioLog$initializer$        10020918     SamtoolMpileupWorker.obj
 0002:0000091c       _perfLog$initializer$      1002091c     SamtoolMpileupWorker.obj
 0002:00000920       _scriptLog$initializer$    10020920     SamtoolMpileupWorker.obj
 0002:00000924       _taskLog$initializer$      10020924     SamtoolMpileupWorker.obj
 0002:00000928       _uiLog$initializer$        10020928     SamtoolMpileupWorker.obj
 0002:0000092c       _userActLog$initializer$   1002092c     SamtoolMpileupWorker.obj
 0002:00000930       ?ACTOR_ID$initializer$@CallVariantsWorkerFactory@LocalWorkflow@U2@@2P6AXXZA 10020930     SamtoolMpileupWorker.obj
 0002:00000934       _REF_SEQ_PORT_ID$initializer$ 10020934     SamtoolMpileupWorker.obj
 0002:00000938       _ASSEMBLY_PORT_ID$initializer$ 10020938     SamtoolMpileupWorker.obj
 0002:0000093c       _OUT_URL$initializer$      1002093c     SamtoolMpileupWorker.obj
 0002:00000940       _REF_SOURCE$initializer$   10020940     SamtoolMpileupWorker.obj
 0002:00000944       _REF_SOURCE_PORT$initializer$ 10020944     SamtoolMpileupWorker.obj
 0002:00000948       _REF_SOURCE_FILE$initializer$ 10020948     SamtoolMpileupWorker.obj
 0002:0000094c       _REF_URL$initializer$      1002094c     SamtoolMpileupWorker.obj
 0002:00000950       _ILLUMINA13$initializer$   10020950     SamtoolMpileupWorker.obj
 0002:00000954       _USE_ORPHAN$initializer$   10020954     SamtoolMpileupWorker.obj
 0002:00000958       _DISABLE_BAQ$initializer$  10020958     SamtoolMpileupWorker.obj
 0002:0000095c       _CAPQ_THRES$initializer$   1002095c     SamtoolMpileupWorker.obj
 0002:00000960       _MAX_DEPTH$initializer$    10020960     SamtoolMpileupWorker.obj
 0002:00000964       _EXT_BAQ$initializer$      10020964     SamtoolMpileupWorker.obj
 0002:00000968       _BED$initializer$          10020968     SamtoolMpileupWorker.obj
 0002:0000096c       _REG$initializer$          1002096c     SamtoolMpileupWorker.obj
 0002:00000970       _MIN_MQ$initializer$       10020970     SamtoolMpileupWorker.obj
 0002:00000974       _MIN_BASEQ$initializer$    10020974     SamtoolMpileupWorker.obj
 0002:00000978       _EXTQ$initializer$         10020978     SamtoolMpileupWorker.obj
 0002:0000097c       _TANDEMQ$initializer$      1002097c     SamtoolMpileupWorker.obj
 0002:00000980       _NO_INDEL$initializer$     10020980     SamtoolMpileupWorker.obj
 0002:00000984       _MAX_INDEL_DEPTH$initializer$ 10020984     SamtoolMpileupWorker.obj
 0002:00000988       _OPENQ$initializer$        10020988     SamtoolMpileupWorker.obj
 0002:0000098c       _PL_LIST$initializer$      1002098c     SamtoolMpileupWorker.obj
 0002:00000990       _KEEPALT$initializer$      10020990     SamtoolMpileupWorker.obj
 0002:00000994       _FIX_PL$initializer$       10020994     SamtoolMpileupWorker.obj
 0002:00000998       _NO_GENO$initializer$      10020998     SamtoolMpileupWorker.obj
 0002:0000099c       _ACGT_ONLY$initializer$    1002099c     SamtoolMpileupWorker.obj
 0002:000009a0       _BCF_BED$initializer$      100209a0     SamtoolMpileupWorker.obj
 0002:000009a4       _QCALL$initializer$        100209a4     SamtoolMpileupWorker.obj
 0002:000009a8       _SAMPLES$initializer$      100209a8     SamtoolMpileupWorker.obj
 0002:000009ac       _MIN_SMPL_FRAC$initializer$ 100209ac     SamtoolMpileupWorker.obj
 0002:000009b0       _CALL_GT$initializer$      100209b0     SamtoolMpileupWorker.obj
 0002:000009b4       _INDEL_FRAC$initializer$   100209b4     SamtoolMpileupWorker.obj
 0002:000009b8       _PREF$initializer$         100209b8     SamtoolMpileupWorker.obj
 0002:000009bc       _PTYPE$initializer$        100209bc     SamtoolMpileupWorker.obj
 0002:000009c0       _THETA$initializer$        100209c0     SamtoolMpileupWorker.obj
 0002:000009c4       _CCALL$initializer$        100209c4     SamtoolMpileupWorker.obj
 0002:000009c8       _N1$initializer$           100209c8     SamtoolMpileupWorker.obj
 0002:000009cc       _N_PERM$initializer$       100209cc     SamtoolMpileupWorker.obj
 0002:000009d0       _MIN_PERM_P$initializer$   100209d0     SamtoolMpileupWorker.obj
 0002:000009d4       _MIN_QUAL$initializer$     100209d4     SamtoolMpileupWorker.obj
 0002:000009d8       _MIN_DEP$initializer$      100209d8     SamtoolMpileupWorker.obj
 0002:000009dc       _MAX_DEP$initializer$      100209dc     SamtoolMpileupWorker.obj
 0002:000009e0       _MIN_ALT$initializer$      100209e0     SamtoolMpileupWorker.obj
 0002:000009e4       _GAP_SIZE$initializer$     100209e4     SamtoolMpileupWorker.obj
 0002:000009e8       _WINDOW$initializer$       100209e8     SamtoolMpileupWorker.obj
 0002:000009ec       _PVALUE1$initializer$      100209ec     SamtoolMpileupWorker.obj
 0002:000009f0       _PVALUE2$initializer$      100209f0     SamtoolMpileupWorker.obj
 0002:000009f4       _PVALUE3$initializer$      100209f4     SamtoolMpileupWorker.obj
 0002:000009f8       _PVALUE4$initializer$      100209f8     SamtoolMpileupWorker.obj
 0002:000009fc       _PVALUE_HWE$initializer$   100209fc     SamtoolMpileupWorker.obj
 0002:00000a00       _PRINT$initializer$        10020a00     SamtoolMpileupWorker.obj
 0002:00000a04       _algoLog$initializer$      10020a04     SamtoolsPlugin.obj
 0002:00000a08       _cmdLog$initializer$       10020a08     SamtoolsPlugin.obj
 0002:00000a0c       _coreLog$initializer$      10020a0c     SamtoolsPlugin.obj
 0002:00000a10       _ioLog$initializer$        10020a10     SamtoolsPlugin.obj
 0002:00000a14       _perfLog$initializer$      10020a14     SamtoolsPlugin.obj
 0002:00000a18       _scriptLog$initializer$    10020a18     SamtoolsPlugin.obj
 0002:00000a1c       _taskLog$initializer$      10020a1c     SamtoolsPlugin.obj
 0002:00000a20       _uiLog$initializer$        10020a20     SamtoolsPlugin.obj
 0002:00000a24       _userActLog$initializer$   10020a24     SamtoolsPlugin.obj
 0002:00000a28       _algoLog$initializer$      10020a28     moc_AssemblySamtoolsMpileup.obj
 0002:00000a2c       _cmdLog$initializer$       10020a2c     moc_AssemblySamtoolsMpileup.obj
 0002:00000a30       _coreLog$initializer$      10020a30     moc_AssemblySamtoolsMpileup.obj
 0002:00000a34       _ioLog$initializer$        10020a34     moc_AssemblySamtoolsMpileup.obj
 0002:00000a38       _perfLog$initializer$      10020a38     moc_AssemblySamtoolsMpileup.obj
 0002:00000a3c       _scriptLog$initializer$    10020a3c     moc_AssemblySamtoolsMpileup.obj
 0002:00000a40       _taskLog$initializer$      10020a40     moc_AssemblySamtoolsMpileup.obj
 0002:00000a44       _uiLog$initializer$        10020a44     moc_AssemblySamtoolsMpileup.obj
 0002:00000a48       _userActLog$initializer$   10020a48     moc_AssemblySamtoolsMpileup.obj
 0002:00000a4c       ?staticMetaObject$initializer$@SamtoolsMpileupTask@LocalWorkflow@U2@@2P6AXXZA 10020a4c     moc_AssemblySamtoolsMpileup.obj
 0002:00000a50       ?staticMetaObject$initializer$@CallVariantsTask@LocalWorkflow@U2@@2P6AXXZA 10020a50     moc_AssemblySamtoolsMpileup.obj
 0002:00000a54       _algoLog$initializer$      10020a54     moc_SamtoolMpileupWorker.obj
 0002:00000a58       _cmdLog$initializer$       10020a58     moc_SamtoolMpileupWorker.obj
 0002:00000a5c       _coreLog$initializer$      10020a5c     moc_SamtoolMpileupWorker.obj
 0002:00000a60       _ioLog$initializer$        10020a60     moc_SamtoolMpileupWorker.obj
 0002:00000a64       _perfLog$initializer$      10020a64     moc_SamtoolMpileupWorker.obj
 0002:00000a68       _scriptLog$initializer$    10020a68     moc_SamtoolMpileupWorker.obj
 0002:00000a6c       _taskLog$initializer$      10020a6c     moc_SamtoolMpileupWorker.obj
 0002:00000a70       _uiLog$initializer$        10020a70     moc_SamtoolMpileupWorker.obj
 0002:00000a74       _userActLog$initializer$   10020a74     moc_SamtoolMpileupWorker.obj
 0002:00000a78       ?staticMetaObject$initializer$@CallVariantsPrompter@LocalWorkflow@U2@@2P6AXXZA 10020a78     moc_SamtoolMpileupWorker.obj
 0002:00000a7c       ?staticMetaObject$initializer$@CallVariantsWorker@LocalWorkflow@U2@@2P6AXXZA 10020a7c     moc_SamtoolMpileupWorker.obj
 0002:00000a80       ?staticMetaObject$initializer$@ScientificDoubleWidget@LocalWorkflow@U2@@2P6AXXZA 10020a80     moc_SamtoolMpileupWorker.obj
 0002:00000a84       ?staticMetaObject$initializer$@SamtoolsPlugin@U2@@2P6AXXZA 10020a84     moc_SamtoolsPlugin.obj
 0002:00000a90       _pcinit                    10020a90     MSVCRT:crtdll.obj
 0002:00000a94       _pinit                     10020a94     MSVCRT:atonexit.obj
 0002:00003950       _qt_meta_stringdata_U2__LocalWorkflow__SamtoolsMpileupTask 10023950     moc_AssemblySamtoolsMpileup.obj
 0002:00003988       _qt_meta_data_U2__LocalWorkflow__SamtoolsMpileupTask 10023988     moc_AssemblySamtoolsMpileup.obj
 0002:000039c4       _qt_meta_stringdata_U2__LocalWorkflow__CallVariantsTask 100239c4     moc_AssemblySamtoolsMpileup.obj
 0002:000039f8       _qt_meta_data_U2__LocalWorkflow__CallVariantsTask 100239f8     moc_AssemblySamtoolsMpileup.obj
 0002:00003a38       _qt_meta_stringdata_U2__LocalWorkflow__CallVariantsPrompter 10023a38     moc_SamtoolMpileupWorker.obj
 0002:00003a70       _qt_meta_data_U2__LocalWorkflow__CallVariantsPrompter 10023a70     moc_SamtoolMpileupWorker.obj
 0002:00003ab0       _qt_meta_stringdata_U2__LocalWorkflow__CallVariantsWorker 10023ab0     moc_SamtoolMpileupWorker.obj
 0002:00003b18       _qt_meta_data_U2__LocalWorkflow__CallVariantsWorker 10023b18     moc_SamtoolMpileupWorker.obj
 0002:00003b70       _qt_meta_stringdata_U2__LocalWorkflow__ScientificDoubleWidget 10023b70     moc_SamtoolMpileupWorker.obj
 0002:00003bf0       _qt_meta_data_U2__LocalWorkflow__ScientificDoubleWidget 10023bf0     moc_SamtoolMpileupWorker.obj
 0002:00003c4c       _qt_meta_stringdata_U2__SamtoolsPlugin 10023c4c     moc_SamtoolsPlugin.obj
 0002:00003c70       _qt_meta_data_U2__SamtoolsPlugin 10023c70     moc_SamtoolsPlugin.obj
 0002:00003cbc       _GS_ExceptionPointers      10023cbc     MSVCRT:gs_report.obj
 0002:00005170       __catchsym$?_Copy@?$basic_string@DU?$char_traits@D@std@@V?$allocator@D@2@@std@@QAEXII@Z$5 10025170     AssemblySamtoolsMpileup.obj
 0002:00005180       __catchsym$?_Copy@?$basic_string@DU?$char_traits@D@std@@V?$allocator@D@2@@std@@QAEXII@Z$4 10025180     AssemblySamtoolsMpileup.obj
 0002:00005190       __unwindtable$?_Copy@?$basic_string@DU?$char_traits@D@std@@V?$allocator@D@2@@std@@QAEXII@Z 10025190     AssemblySamtoolsMpileup.obj
 0002:000051b0       __ehfuncinfo$?_Copy@?$basic_string@DU?$char_traits@D@std@@V?$allocator@D@2@@std@@QAEXII@Z 100251b0     AssemblySamtoolsMpileup.obj
 0002:000051d4       __tryblocktable$?_Copy@?$basic_string@DU?$char_traits@D@std@@V?$allocator@D@2@@std@@QAEXII@Z 100251d4     AssemblySamtoolsMpileup.obj
 0002:000051fc       __unwindtable$??H@YA?BVQString@@ABV0@0@Z 100251fc     AssemblySamtoolsMpileup.obj
 0002:00005204       __ehfuncinfo$??H@YA?BVQString@@ABV0@0@Z 10025204     AssemblySamtoolsMpileup.obj
 0002:00005228       __catchsym$??0?$QList@VQString@@@@QAE@ABV0@@Z$2 10025228     AssemblySamtoolsMpileup.obj
 0002:00005238       __unwindtable$??0?$QList@VQString@@@@QAE@ABV0@@Z 10025238     AssemblySamtoolsMpileup.obj
 0002:00005248       __tryblocktable$??0?$QList@VQString@@@@QAE@ABV0@@Z 10025248     AssemblySamtoolsMpileup.obj
 0002:0000525c       __ehfuncinfo$??0?$QList@VQString@@@@QAE@ABV0@@Z 1002525c     AssemblySamtoolsMpileup.obj
 0002:00005280       __catchsym$?append@?$QList@VQString@@@@QAEXABVQString@@@Z$13 10025280     AssemblySamtoolsMpileup.obj
 0002:00005290       __catchsym$?append@?$QList@VQString@@@@QAEXABVQString@@@Z$12 10025290     AssemblySamtoolsMpileup.obj
 0002:000052a0       __ehfuncinfo$?append@?$QList@VQString@@@@QAEXABVQString@@@Z 100252a0     AssemblySamtoolsMpileup.obj
 0002:000052c4       __tryblocktable$?append@?$QList@VQString@@@@QAEXABVQString@@@Z 100252c4     AssemblySamtoolsMpileup.obj
 0002:000052ec       __unwindtable$?append@?$QList@VQString@@@@QAEXABVQString@@@Z 100252ec     AssemblySamtoolsMpileup.obj
 0002:0000534c       __catchsym$??Y?$QList@VQString@@@@QAEAAV0@ABV0@@Z$3 1002534c     AssemblySamtoolsMpileup.obj
 0002:0000535c       __unwindtable$??Y?$QList@VQString@@@@QAEAAV0@ABV0@@Z 1002535c     AssemblySamtoolsMpileup.obj
 0002:0000536c       __tryblocktable$??Y?$QList@VQString@@@@QAEAAV0@ABV0@@Z 1002536c     AssemblySamtoolsMpileup.obj
 0002:00005380       __ehfuncinfo$??Y?$QList@VQString@@@@QAEAAV0@ABV0@@Z 10025380     AssemblySamtoolsMpileup.obj
 0002:000053a4       __catchsym$?detach_helper_grow@?$QList@VQString@@@@AAEPAUNode@1@HH@Z$5 100253a4     AssemblySamtoolsMpileup.obj
 0002:000053b4       __catchsym$?detach_helper_grow@?$QList@VQString@@@@AAEPAUNode@1@HH@Z$4 100253b4     AssemblySamtoolsMpileup.obj
 0002:000053c4       __unwindtable$?detach_helper_grow@?$QList@VQString@@@@AAEPAUNode@1@HH@Z 100253c4     AssemblySamtoolsMpileup.obj
 0002:000053e4       __ehfuncinfo$?detach_helper_grow@?$QList@VQString@@@@AAEPAUNode@1@HH@Z 100253e4     AssemblySamtoolsMpileup.obj
 0002:00005408       __tryblocktable$?detach_helper_grow@?$QList@VQString@@@@AAEPAUNode@1@HH@Z 10025408     AssemblySamtoolsMpileup.obj
 0002:00005430       __unwindtable$?node_construct@?$QList@VQString@@@@AAEXPAUNode@1@ABVQString@@@Z 10025430     AssemblySamtoolsMpileup.obj
 0002:00005440       __ehfuncinfo$?node_construct@?$QList@VQString@@@@AAEXPAUNode@1@ABVQString@@@Z 10025440     AssemblySamtoolsMpileup.obj
 0002:00005464       __catchsym$?node_copy@?$QList@VQString@@@@AAEXPAUNode@1@00@Z$6 10025464     AssemblySamtoolsMpileup.obj
 0002:00005474       __tryblocktable$?node_copy@?$QList@VQString@@@@AAEXPAUNode@1@00@Z 10025474     AssemblySamtoolsMpileup.obj
 0002:00005488       __ehfuncinfo$?node_copy@?$QList@VQString@@@@AAEXPAUNode@1@00@Z 10025488     AssemblySamtoolsMpileup.obj
 0002:000054ac       __unwindtable$?node_copy@?$QList@VQString@@@@AAEXPAUNode@1@00@Z 100254ac     AssemblySamtoolsMpileup.obj
 0002:000054dc       __unwindtable$??A?$QMap@VQString@@VQVariant@@@@QAEAAVQVariant@@ABVQString@@@Z 100254dc     AssemblySamtoolsMpileup.obj
 0002:000054e4       __ehfuncinfo$??A?$QMap@VQString@@VQVariant@@@@QAEAAVQVariant@@ABVQString@@@Z 100254e4     AssemblySamtoolsMpileup.obj
 0002:00005508       __unwindtable$??__EalgoLog@U2@@YAXXZ 10025508     AssemblySamtoolsMpileup.obj
 0002:00005510       __ehfuncinfo$??__EalgoLog@U2@@YAXXZ 10025510     AssemblySamtoolsMpileup.obj
 0002:00005534       __unwindtable$??__EcmdLog@U2@@YAXXZ 10025534     AssemblySamtoolsMpileup.obj
 0002:0000553c       __ehfuncinfo$??__EcmdLog@U2@@YAXXZ 1002553c     AssemblySamtoolsMpileup.obj
 0002:00005560       __unwindtable$??__EcoreLog@U2@@YAXXZ 10025560     AssemblySamtoolsMpileup.obj
 0002:00005568       __ehfuncinfo$??__EcoreLog@U2@@YAXXZ 10025568     AssemblySamtoolsMpileup.obj
 0002:0000558c       __unwindtable$??__EioLog@U2@@YAXXZ 1002558c     AssemblySamtoolsMpileup.obj
 0002:00005594       __ehfuncinfo$??__EioLog@U2@@YAXXZ 10025594     AssemblySamtoolsMpileup.obj
 0002:000055b8       __unwindtable$??__EperfLog@U2@@YAXXZ 100255b8     AssemblySamtoolsMpileup.obj
 0002:000055c0       __ehfuncinfo$??__EperfLog@U2@@YAXXZ 100255c0     AssemblySamtoolsMpileup.obj
 0002:000055e4       __unwindtable$??__EscriptLog@U2@@YAXXZ 100255e4     AssemblySamtoolsMpileup.obj
 0002:000055ec       __ehfuncinfo$??__EscriptLog@U2@@YAXXZ 100255ec     AssemblySamtoolsMpileup.obj
 0002:00005610       __unwindtable$??__EtaskLog@U2@@YAXXZ 10025610     AssemblySamtoolsMpileup.obj
 0002:00005618       __ehfuncinfo$??__EtaskLog@U2@@YAXXZ 10025618     AssemblySamtoolsMpileup.obj
 0002:0000563c       __unwindtable$??__EuiLog@U2@@YAXXZ 1002563c     AssemblySamtoolsMpileup.obj
 0002:00005644       __ehfuncinfo$??__EuiLog@U2@@YAXXZ 10025644     AssemblySamtoolsMpileup.obj
 0002:00005668       __unwindtable$??__EuserActLog@U2@@YAXXZ 10025668     AssemblySamtoolsMpileup.obj
 0002:00005670       __ehfuncinfo$??__EuserActLog@U2@@YAXXZ 10025670     AssemblySamtoolsMpileup.obj
 0002:00005694       __catchsym$?append@?$QList@PAVTask@U2@@@@QAEXABQAVTask@U2@@@Z$6 10025694     AssemblySamtoolsMpileup.obj
 0002:000056a4       __tryblocktable$?append@?$QList@PAVTask@U2@@@@QAEXABQAVTask@U2@@@Z 100256a4     AssemblySamtoolsMpileup.obj
 0002:000056b8       __ehfuncinfo$?append@?$QList@PAVTask@U2@@@@QAEXABQAVTask@U2@@@Z 100256b8     AssemblySamtoolsMpileup.obj
 0002:000056dc       __unwindtable$?append@?$QList@PAVTask@U2@@@@QAEXABQAVTask@U2@@@Z 100256dc     AssemblySamtoolsMpileup.obj
 0002:0000570c       __catchsym$?detach_helper_grow@?$QList@PAVTask@U2@@@@AAEPAUNode@1@HH@Z$5 1002570c     AssemblySamtoolsMpileup.obj
 0002:0000571c       __catchsym$?detach_helper_grow@?$QList@PAVTask@U2@@@@AAEPAUNode@1@HH@Z$4 1002571c     AssemblySamtoolsMpileup.obj
 0002:0000572c       __unwindtable$?detach_helper_grow@?$QList@PAVTask@U2@@@@AAEPAUNode@1@HH@Z 1002572c     AssemblySamtoolsMpileup.obj
 0002:0000574c       __ehfuncinfo$?detach_helper_grow@?$QList@PAVTask@U2@@@@AAEPAUNode@1@HH@Z 1002574c     AssemblySamtoolsMpileup.obj
 0002:00005770       __tryblocktable$?detach_helper_grow@?$QList@PAVTask@U2@@@@AAEPAUNode@1@HH@Z 10025770     AssemblySamtoolsMpileup.obj
 0002:00005798       __unwindtable$?qt_metatype_id@?$QMetaTypeId@VU2DbiRef@U2@@@@SAHXZ 10025798     AssemblySamtoolsMpileup.obj
 0002:000057a0       __ehfuncinfo$?qt_metatype_id@?$QMetaTypeId@VU2DbiRef@U2@@@@SAHXZ 100257a0     AssemblySamtoolsMpileup.obj
 0002:000057c4       __unwindtable$??$qRegisterMetaType@VU2DbiRef@U2@@@@YAHPBDPAVU2DbiRef@U2@@W4DefinedType@?$MetaTypeDefinedHelper@VU2DbiRef@U2@@$00@QtPrivate@@@Z 100257c4     AssemblySamtoolsMpileup.obj
 0002:000057cc       __ehfuncinfo$??$qRegisterMetaType@VU2DbiRef@U2@@@@YAHPBDPAVU2DbiRef@U2@@W4DefinedType@?$MetaTypeDefinedHelper@VU2DbiRef@U2@@$00@QtPrivate@@@Z 100257cc     AssemblySamtoolsMpileup.obj
 0002:000057f0       __catchsym$??0?$QList@PAVGObject@U2@@@@QAE@ABV0@@Z$2 100257f0     AssemblySamtoolsMpileup.obj
 0002:00005800       __unwindtable$??0?$QList@PAVGObject@U2@@@@QAE@ABV0@@Z 10025800     AssemblySamtoolsMpileup.obj
 0002:00005810       __tryblocktable$??0?$QList@PAVGObject@U2@@@@QAE@ABV0@@Z 10025810     AssemblySamtoolsMpileup.obj
 0002:00005824       __ehfuncinfo$??0?$QList@PAVGObject@U2@@@@QAE@ABV0@@Z 10025824     AssemblySamtoolsMpileup.obj
 0002:00005848       __unwindtable$?qt_metatype_id@?$QMetaTypeId@V?$QSharedDataPointer@VDbiDataHandler@Workflow@U2@@@@@@SAHXZ 10025848     AssemblySamtoolsMpileup.obj
 0002:00005850       __ehfuncinfo$?qt_metatype_id@?$QMetaTypeId@V?$QSharedDataPointer@VDbiDataHandler@Workflow@U2@@@@@@SAHXZ 10025850     AssemblySamtoolsMpileup.obj
 0002:00005874       __unwindtable$??$qRegisterMetaType@V?$QSharedDataPointer@VDbiDataHandler@Workflow@U2@@@@@@YAHPBDPAV?$QSharedDataPointer@VDbiDataHandler@Workflow@U2@@@@W4DefinedType@?$MetaTypeDefinedHelper@V?$QSharedDataPointer@VDbiDataHandler@Workflow@U2@@@@$00@QtPrivate@@@Z 10025874     AssemblySamtoolsMpileup.obj
 0002:0000587c       __ehfuncinfo$??$qRegisterMetaType@V?$QSharedDataPointer@VDbiDataHandler@Workflow@U2@@@@@@YAHPBDPAV?$QSharedDataPointer@VDbiDataHandler@Workflow@U2@@@@W4DefinedType@?$MetaTypeDefinedHelper@V?$QSharedDataPointer@VDbiDataHandler@Workflow@U2@@@@$00@QtPrivate@@@Z 1002587c     AssemblySamtoolsMpileup.obj
 0002:000058a0       __ehfuncinfo$?getMpiliupArgs@CallVariantsTaskSettings@LocalWorkflow@U2@@QBE?AVQStringList@@XZ 100258a0     AssemblySamtoolsMpileup.obj
 0002:000058c4       __unwindtable$?getMpiliupArgs@CallVariantsTaskSettings@LocalWorkflow@U2@@QBE?AVQStringList@@XZ 100258c4     AssemblySamtoolsMpileup.obj
 0002:000059b4       __ehfuncinfo$?getBcfViewArgs@CallVariantsTaskSettings@LocalWorkflow@U2@@QBE?AVQStringList@@XZ 100259b4     AssemblySamtoolsMpileup.obj
 0002:000059d8       __unwindtable$?getBcfViewArgs@CallVariantsTaskSettings@LocalWorkflow@U2@@QBE?AVQStringList@@XZ 100259d8     AssemblySamtoolsMpileup.obj
 0002:00005ad8       __ehfuncinfo$?getVarFilterArgs@CallVariantsTaskSettings@LocalWorkflow@U2@@QBE?AVQStringList@@XZ 10025ad8     AssemblySamtoolsMpileup.obj
 0002:00005afc       __unwindtable$?getVarFilterArgs@CallVariantsTaskSettings@LocalWorkflow@U2@@QBE?AVQStringList@@XZ 10025afc     AssemblySamtoolsMpileup.obj
 0002:00005bc4       __ehfuncinfo$??1CallVariantsTaskSettings@LocalWorkflow@U2@@QAE@XZ 10025bc4     AssemblySamtoolsMpileup.obj
 0002:00005be8       __unwindtable$??1CallVariantsTaskSettings@LocalWorkflow@U2@@QAE@XZ 10025be8     AssemblySamtoolsMpileup.obj
 0002:00005c30       __ehfuncinfo$??0CallVariantsTaskSettings@LocalWorkflow@U2@@QAE@ABV012@@Z 10025c30     AssemblySamtoolsMpileup.obj
 0002:00005c54       __unwindtable$??0CallVariantsTaskSettings@LocalWorkflow@U2@@QAE@ABV012@@Z 10025c54     AssemblySamtoolsMpileup.obj
 0002:00005c9c       __ehfuncinfo$??0SamtoolsMpileupTask@LocalWorkflow@U2@@QAE@ABVCallVariantsTaskSettings@12@@Z 10025c9c     AssemblySamtoolsMpileup.obj
 0002:00005cc0       __unwindtable$??0SamtoolsMpileupTask@LocalWorkflow@U2@@QAE@ABVCallVariantsTaskSettings@12@@Z 10025cc0     AssemblySamtoolsMpileup.obj
 0002:00005ce8       __ehfuncinfo$?prepare@SamtoolsMpileupTask@LocalWorkflow@U2@@UAEXXZ 10025ce8     AssemblySamtoolsMpileup.obj
 0002:00005d0c       __unwindtable$?prepare@SamtoolsMpileupTask@LocalWorkflow@U2@@UAEXXZ 10025d0c     AssemblySamtoolsMpileup.obj
 0002:00005d64       __ehfuncinfo$?run@SamtoolsMpileupTask@LocalWorkflow@U2@@UAEXXZ 10025d64     AssemblySamtoolsMpileup.obj
 0002:00005d88       __unwindtable$?run@SamtoolsMpileupTask@LocalWorkflow@U2@@UAEXXZ 10025d88     AssemblySamtoolsMpileup.obj
 0002:00005ea8       __unwindtable$?start@SamtoolsMpileupTask@LocalWorkflow@U2@@AAEXABVProcessRun@3@ABVQString@@@Z 10025ea8     AssemblySamtoolsMpileup.obj
 0002:00005eb8       __ehfuncinfo$?start@SamtoolsMpileupTask@LocalWorkflow@U2@@AAEXABVProcessRun@3@ABVQString@@@Z 10025eb8     AssemblySamtoolsMpileup.obj
 0002:00005edc       __ehfuncinfo$?checkExitCode@SamtoolsMpileupTask@LocalWorkflow@U2@@AAEXPAVQProcess@@ABVQString@@@Z 10025edc     AssemblySamtoolsMpileup.obj
 0002:00005f00       __unwindtable$?checkExitCode@SamtoolsMpileupTask@LocalWorkflow@U2@@AAEXPAVQProcess@@ABVQString@@@Z 10025f00     AssemblySamtoolsMpileup.obj
 0002:00005f28       __unwindtable$??1SamtoolsMpileupTask@LocalWorkflow@U2@@UAE@XZ 10025f28     AssemblySamtoolsMpileup.obj
 0002:00005f30       __ehfuncinfo$??1SamtoolsMpileupTask@LocalWorkflow@U2@@UAE@XZ 10025f30     AssemblySamtoolsMpileup.obj
 0002:00005f54       __unwindtable$??_GSamtoolsMpileupTask@LocalWorkflow@U2@@UAEPAXI@Z 10025f54     AssemblySamtoolsMpileup.obj
 0002:00005f5c       __ehfuncinfo$??_GSamtoolsMpileupTask@LocalWorkflow@U2@@UAEPAXI@Z 10025f5c     AssemblySamtoolsMpileup.obj
 0002:00005f80       __ehfuncinfo$??0CallVariantsTask@LocalWorkflow@U2@@QAE@ABVCallVariantsTaskSettings@12@PAVDbiDataStorage@Workflow@2@@Z 10025f80     AssemblySamtoolsMpileup.obj
 0002:00005fa4       __unwindtable$??0CallVariantsTask@LocalWorkflow@U2@@QAE@ABVCallVariantsTaskSettings@12@PAVDbiDataStorage@Workflow@2@@Z 10025fa4     AssemblySamtoolsMpileup.obj
 0002:00005ffc       __ehfuncinfo$?prepare@CallVariantsTask@LocalWorkflow@U2@@UAEXXZ 10025ffc     AssemblySamtoolsMpileup.obj
 0002:00006020       __unwindtable$?prepare@CallVariantsTask@LocalWorkflow@U2@@UAEXXZ 10026020     AssemblySamtoolsMpileup.obj
 0002:00006048       __ehfuncinfo$?onSubTaskFinished@CallVariantsTask@LocalWorkflow@U2@@UAE?AV?$QList@PAVTask@U2@@@@PAVTask@3@@Z 10026048     AssemblySamtoolsMpileup.obj
 0002:0000606c       __unwindtable$?onSubTaskFinished@CallVariantsTask@LocalWorkflow@U2@@UAE?AV?$QList@PAVTask@U2@@@@PAVTask@3@@Z 1002606c     AssemblySamtoolsMpileup.obj
 0002:00006174       __unwindtable$?tmpFilePath@CallVariantsTask@LocalWorkflow@U2@@SA?AVQString@@ABV4@0AAVU2OpStatus@3@@Z 10026174     AssemblySamtoolsMpileup.obj
 0002:00006194       __ehfuncinfo$?tmpFilePath@CallVariantsTask@LocalWorkflow@U2@@SA?AVQString@@ABV4@0AAVU2OpStatus@3@@Z 10026194     AssemblySamtoolsMpileup.obj
 0002:000061b8       __ehfuncinfo$?toString@CallVariantsTask@LocalWorkflow@U2@@CA?AVQString@@W4FileType@123@@Z 100261b8     AssemblySamtoolsMpileup.obj
 0002:000061dc       __unwindtable$?toString@CallVariantsTask@LocalWorkflow@U2@@CA?AVQString@@W4FileType@123@@Z 100261dc     AssemblySamtoolsMpileup.obj
 0002:0000620c       __unwindtable$?ensureFileExists@CallVariantsTask@LocalWorkflow@U2@@AAE_NABVQString@@W4FileType@123@@Z 1002620c     AssemblySamtoolsMpileup.obj
 0002:0000622c       __ehfuncinfo$?ensureFileExists@CallVariantsTask@LocalWorkflow@U2@@AAE_NABVQString@@W4FileType@123@@Z 1002622c     AssemblySamtoolsMpileup.obj
 0002:00006250       __catchsym$?append@?$QList@V?$QMap@VQString@@VQVariant@@@@@@QAEXABV?$QMap@VQString@@VQVariant@@@@@Z$11 10026250     AssemblySamtoolsMpileup.obj
 0002:00006260       __catchsym$?append@?$QList@V?$QMap@VQString@@VQVariant@@@@@@QAEXABV?$QMap@VQString@@VQVariant@@@@@Z$10 10026260     AssemblySamtoolsMpileup.obj
 0002:00006270       __ehfuncinfo$?append@?$QList@V?$QMap@VQString@@VQVariant@@@@@@QAEXABV?$QMap@VQString@@VQVariant@@@@@Z 10026270     AssemblySamtoolsMpileup.obj
 0002:00006294       __tryblocktable$?append@?$QList@V?$QMap@VQString@@VQVariant@@@@@@QAEXABV?$QMap@VQString@@VQVariant@@@@@Z 10026294     AssemblySamtoolsMpileup.obj
 0002:000062bc       __unwindtable$?append@?$QList@V?$QMap@VQString@@VQVariant@@@@@@QAEXABV?$QMap@VQString@@VQVariant@@@@@Z 100262bc     AssemblySamtoolsMpileup.obj
 0002:0000630c       __catchsym$?detach_helper_grow@?$QList@V?$QMap@VQString@@VQVariant@@@@@@AAEPAUNode@1@HH@Z$5 1002630c     AssemblySamtoolsMpileup.obj
 0002:0000631c       __catchsym$?detach_helper_grow@?$QList@V?$QMap@VQString@@VQVariant@@@@@@AAEPAUNode@1@HH@Z$4 1002631c     AssemblySamtoolsMpileup.obj
 0002:0000632c       __unwindtable$?detach_helper_grow@?$QList@V?$QMap@VQString@@VQVariant@@@@@@AAEPAUNode@1@HH@Z 1002632c     AssemblySamtoolsMpileup.obj
 0002:0000634c       __ehfuncinfo$?detach_helper_grow@?$QList@V?$QMap@VQString@@VQVariant@@@@@@AAEPAUNode@1@HH@Z 1002634c     AssemblySamtoolsMpileup.obj
 0002:00006370       __tryblocktable$?detach_helper_grow@?$QList@V?$QMap@VQString@@VQVariant@@@@@@AAEPAUNode@1@HH@Z 10026370     AssemblySamtoolsMpileup.obj
 0002:00006398       __unwindtable$?node_construct@?$QList@V?$QMap@VQString@@VQVariant@@@@@@AAEXPAUNode@1@ABV?$QMap@VQString@@VQVariant@@@@@Z 10026398     AssemblySamtoolsMpileup.obj
 0002:000063a8       __ehfuncinfo$?node_construct@?$QList@V?$QMap@VQString@@VQVariant@@@@@@AAEXPAUNode@1@ABV?$QMap@VQString@@VQVariant@@@@@Z 100263a8     AssemblySamtoolsMpileup.obj
 0002:000063cc       __catchsym$?node_copy@?$QList@V?$QMap@VQString@@VQVariant@@@@@@AAEXPAUNode@1@00@Z$6 100263cc     AssemblySamtoolsMpileup.obj
 0002:000063dc       __tryblocktable$?node_copy@?$QList@V?$QMap@VQString@@VQVariant@@@@@@AAEXPAUNode@1@00@Z 100263dc     AssemblySamtoolsMpileup.obj
 0002:000063f0       __ehfuncinfo$?node_copy@?$QList@V?$QMap@VQString@@VQVariant@@@@@@AAEXPAUNode@1@00@Z 100263f0     AssemblySamtoolsMpileup.obj
 0002:00006414       __unwindtable$?node_copy@?$QList@V?$QMap@VQString@@VQVariant@@@@@@AAEXPAUNode@1@00@Z 10026414     AssemblySamtoolsMpileup.obj
 0002:00006444       __unwindtable$??1CallVariantsTask@LocalWorkflow@U2@@UAE@XZ 10026444     AssemblySamtoolsMpileup.obj
 0002:00006454       __ehfuncinfo$??1CallVariantsTask@LocalWorkflow@U2@@UAE@XZ 10026454     AssemblySamtoolsMpileup.obj
 0002:00006478       __catchsym$?detach_helper@?$QList@VFormatDetectionResult@U2@@@@AAEXH@Z$2 10026478     AssemblySamtoolsMpileup.obj
 0002:00006488       __unwindtable$?detach_helper@?$QList@VFormatDetectionResult@U2@@@@AAEXH@Z 10026488     AssemblySamtoolsMpileup.obj
 0002:00006498       __tryblocktable$?detach_helper@?$QList@VFormatDetectionResult@U2@@@@AAEXH@Z 10026498     AssemblySamtoolsMpileup.obj
 0002:000064ac       __ehfuncinfo$?detach_helper@?$QList@VFormatDetectionResult@U2@@@@AAEXH@Z 100264ac     AssemblySamtoolsMpileup.obj
 0002:000064d0       __catchsym$?node_copy@?$QList@VFormatDetectionResult@U2@@@@AAEXPAUNode@1@00@Z$6 100264d0     AssemblySamtoolsMpileup.obj
 0002:000064e0       __tryblocktable$?node_copy@?$QList@VFormatDetectionResult@U2@@@@AAEXPAUNode@1@00@Z 100264e0     AssemblySamtoolsMpileup.obj
 0002:000064f4       __ehfuncinfo$?node_copy@?$QList@VFormatDetectionResult@U2@@@@AAEXPAUNode@1@00@Z 100264f4     AssemblySamtoolsMpileup.obj
 0002:00006518       __unwindtable$?node_copy@?$QList@VFormatDetectionResult@U2@@@@AAEXPAUNode@1@00@Z 10026518     AssemblySamtoolsMpileup.obj
 0002:00006548       __catchsym$?createNode@?$QMapData@VQString@@VQVariant@@@@QAEPAU?$QMapNode@VQString@@VQVariant@@@@ABVQString@@ABVQVariant@@PAU2@_N@Z$7 10026548     AssemblySamtoolsMpileup.obj
 0002:00006558       __catchsym$?createNode@?$QMapData@VQString@@VQVariant@@@@QAEPAU?$QMapNode@VQString@@VQVariant@@@@ABVQString@@ABVQVariant@@PAU2@_N@Z$6 10026558     AssemblySamtoolsMpileup.obj
 0002:00006568       __ehfuncinfo$?createNode@?$QMapData@VQString@@VQVariant@@@@QAEPAU?$QMapNode@VQString@@VQVariant@@@@ABVQString@@ABVQVariant@@PAU2@_N@Z 10026568     AssemblySamtoolsMpileup.obj
 0002:0000658c       __tryblocktable$?createNode@?$QMapData@VQString@@VQVariant@@@@QAEPAU?$QMapNode@VQString@@VQVariant@@@@ABVQString@@ABVQVariant@@PAU2@_N@Z 1002658c     AssemblySamtoolsMpileup.obj
 0002:000065b4       __unwindtable$?createNode@?$QMapData@VQString@@VQVariant@@@@QAEPAU?$QMapNode@VQString@@VQVariant@@@@ABVQString@@ABVQVariant@@PAU2@_N@Z 100265b4     AssemblySamtoolsMpileup.obj
 0002:000065e4       __ehfuncinfo$?Create@?$QMetaTypeFunctionHelper@VU2DbiRef@U2@@$00@QtMetaTypePrivate@@SAPAXPBX@Z 100265e4     AssemblySamtoolsMpileup.obj
 0002:00006608       __unwindtable$?Create@?$QMetaTypeFunctionHelper@VU2DbiRef@U2@@$00@QtMetaTypePrivate@@SAPAXPBX@Z 10026608     AssemblySamtoolsMpileup.obj
 0002:00006638       __ehfuncinfo$?Construct@?$QMetaTypeFunctionHelper@VU2DbiRef@U2@@$00@QtMetaTypePrivate@@SAPAXPAXPBX@Z 10026638     AssemblySamtoolsMpileup.obj
 0002:0000665c       __unwindtable$?Construct@?$QMetaTypeFunctionHelper@VU2DbiRef@U2@@$00@QtMetaTypePrivate@@SAPAXPAXPBX@Z 1002665c     AssemblySamtoolsMpileup.obj
 0002:0000668c       __unwindtable$??H@YA?BVQString@@ABV0@PBD@Z 1002668c     SamtoolMpileupWorker.obj
 0002:0000669c       __ehfuncinfo$??H@YA?BVQString@@ABV0@PBD@Z 1002669c     SamtoolMpileupWorker.obj
 0002:000066c0       __unwindtable$??H@YA?BVQString@@PBDABV0@@Z 100266c0     SamtoolMpileupWorker.obj
 0002:000066c8       __ehfuncinfo$??H@YA?BVQString@@PBDABV0@@Z 100266c8     SamtoolMpileupWorker.obj
 0002:000066ec       __catchsym$?append@?$QList@VQVariant@@@@QAEXABVQVariant@@@Z$11 100266ec     SamtoolMpileupWorker.obj
 0002:000066fc       __catchsym$?append@?$QList@VQVariant@@@@QAEXABVQVariant@@@Z$10 100266fc     SamtoolMpileupWorker.obj
 0002:0000670c       __ehfuncinfo$?append@?$QList@VQVariant@@@@QAEXABVQVariant@@@Z 1002670c     SamtoolMpileupWorker.obj
 0002:00006730       __tryblocktable$?append@?$QList@VQVariant@@@@QAEXABVQVariant@@@Z 10026730     SamtoolMpileupWorker.obj
 0002:00006758       __unwindtable$?append@?$QList@VQVariant@@@@QAEXABVQVariant@@@Z 10026758     SamtoolMpileupWorker.obj
 0002:000067a8       __catchsym$?detach_helper_grow@?$QList@VQVariant@@@@AAEPAUNode@1@HH@Z$5 100267a8     SamtoolMpileupWorker.obj
 0002:000067b8       __catchsym$?detach_helper_grow@?$QList@VQVariant@@@@AAEPAUNode@1@HH@Z$4 100267b8     SamtoolMpileupWorker.obj
 0002:000067c8       __unwindtable$?detach_helper_grow@?$QList@VQVariant@@@@AAEPAUNode@1@HH@Z 100267c8     SamtoolMpileupWorker.obj
 0002:000067e8       __ehfuncinfo$?detach_helper_grow@?$QList@VQVariant@@@@AAEPAUNode@1@HH@Z 100267e8     SamtoolMpileupWorker.obj
 0002:0000680c       __tryblocktable$?detach_helper_grow@?$QList@VQVariant@@@@AAEPAUNode@1@HH@Z 1002680c     SamtoolMpileupWorker.obj
 0002:00006834       __unwindtable$?node_construct@?$QList@VQVariant@@@@AAEXPAUNode@1@ABVQVariant@@@Z 10026834     SamtoolMpileupWorker.obj
 0002:00006844       __ehfuncinfo$?node_construct@?$QList@VQVariant@@@@AAEXPAUNode@1@ABVQVariant@@@Z 10026844     SamtoolMpileupWorker.obj
 0002:00006868       __catchsym$?node_copy@?$QList@VQVariant@@@@AAEXPAUNode@1@00@Z$6 10026868     SamtoolMpileupWorker.obj
 0002:00006878       __tryblocktable$?node_copy@?$QList@VQVariant@@@@AAEXPAUNode@1@00@Z 10026878     SamtoolMpileupWorker.obj
 0002:0000688c       __ehfuncinfo$?node_copy@?$QList@VQVariant@@@@AAEXPAUNode@1@00@Z 1002688c     SamtoolMpileupWorker.obj
 0002:000068b0       __unwindtable$?node_copy@?$QList@VQVariant@@@@AAEXPAUNode@1@00@Z 100268b0     SamtoolMpileupWorker.obj
 0002:000068e0       __unwindtable$??__EalgoLog@U2@@YAXXZ 100268e0     SamtoolMpileupWorker.obj
 0002:000068e8       __ehfuncinfo$??__EalgoLog@U2@@YAXXZ 100268e8     SamtoolMpileupWorker.obj
 0002:0000690c       __unwindtable$??__EcmdLog@U2@@YAXXZ 1002690c     SamtoolMpileupWorker.obj
 0002:00006914       __ehfuncinfo$??__EcmdLog@U2@@YAXXZ 10026914     SamtoolMpileupWorker.obj
 0002:00006938       __unwindtable$??__EcoreLog@U2@@YAXXZ 10026938     SamtoolMpileupWorker.obj
 0002:00006940       __ehfuncinfo$??__EcoreLog@U2@@YAXXZ 10026940     SamtoolMpileupWorker.obj
 0002:00006964       __unwindtable$??__EioLog@U2@@YAXXZ 10026964     SamtoolMpileupWorker.obj
 0002:0000696c       __ehfuncinfo$??__EioLog@U2@@YAXXZ 1002696c     SamtoolMpileupWorker.obj
 0002:00006990       __unwindtable$??__EperfLog@U2@@YAXXZ 10026990     SamtoolMpileupWorker.obj
 0002:00006998       __ehfuncinfo$??__EperfLog@U2@@YAXXZ 10026998     SamtoolMpileupWorker.obj
 0002:000069bc       __unwindtable$??__EscriptLog@U2@@YAXXZ 100269bc     SamtoolMpileupWorker.obj
 0002:000069c4       __ehfuncinfo$??__EscriptLog@U2@@YAXXZ 100269c4     SamtoolMpileupWorker.obj
 0002:000069e8       __unwindtable$??__EtaskLog@U2@@YAXXZ 100269e8     SamtoolMpileupWorker.obj
 0002:000069f0       __ehfuncinfo$??__EtaskLog@U2@@YAXXZ 100269f0     SamtoolMpileupWorker.obj
 0002:00006a14       __unwindtable$??__EuiLog@U2@@YAXXZ 10026a14     SamtoolMpileupWorker.obj
 0002:00006a1c       __ehfuncinfo$??__EuiLog@U2@@YAXXZ 10026a1c     SamtoolMpileupWorker.obj
 0002:00006a40       __unwindtable$??__EuserActLog@U2@@YAXXZ 10026a40     SamtoolMpileupWorker.obj
 0002:00006a48       __ehfuncinfo$??__EuserActLog@U2@@YAXXZ 10026a48     SamtoolMpileupWorker.obj
 0002:00006a6c       __unwindtable$??A?$QMap@VQString@@VQScriptValue@@@@QAEAAVQScriptValue@@ABVQString@@@Z 10026a6c     SamtoolMpileupWorker.obj
 0002:00006a74       __ehfuncinfo$??A?$QMap@VQString@@VQScriptValue@@@@QAEAAVQScriptValue@@ABVQString@@@Z 10026a74     SamtoolMpileupWorker.obj
 0002:00006a98       __catchsym$??0?$QList@VDescriptor@U2@@@@QAE@ABV0@@Z$2 10026a98     SamtoolMpileupWorker.obj
 0002:00006aa8       __unwindtable$??0?$QList@VDescriptor@U2@@@@QAE@ABV0@@Z 10026aa8     SamtoolMpileupWorker.obj
 0002:00006ab8       __tryblocktable$??0?$QList@VDescriptor@U2@@@@QAE@ABV0@@Z 10026ab8     SamtoolMpileupWorker.obj
 0002:00006acc       __ehfuncinfo$??0?$QList@VDescriptor@U2@@@@QAE@ABV0@@Z 10026acc     SamtoolMpileupWorker.obj
 0002:00006af0       __catchsym$?append@?$QList@VDescriptor@U2@@@@QAEXABVDescriptor@U2@@@Z$9 10026af0     SamtoolMpileupWorker.obj
 0002:00006b00       __catchsym$?append@?$QList@VDescriptor@U2@@@@QAEXABVDescriptor@U2@@@Z$8 10026b00     SamtoolMpileupWorker.obj
 0002:00006b10       __ehfuncinfo$?append@?$QList@VDescriptor@U2@@@@QAEXABVDescriptor@U2@@@Z 10026b10     SamtoolMpileupWorker.obj
 0002:00006b34       __tryblocktable$?append@?$QList@VDescriptor@U2@@@@QAEXABVDescriptor@U2@@@Z 10026b34     SamtoolMpileupWorker.obj
 0002:00006b5c       __unwindtable$?append@?$QList@VDescriptor@U2@@@@QAEXABVDescriptor@U2@@@Z 10026b5c     SamtoolMpileupWorker.obj
 0002:00006b9c       __catchsym$?detach_helper_grow@?$QList@VDescriptor@U2@@@@AAEPAUNode@1@HH@Z$5 10026b9c     SamtoolMpileupWorker.obj
 0002:00006bac       __catchsym$?detach_helper_grow@?$QList@VDescriptor@U2@@@@AAEPAUNode@1@HH@Z$4 10026bac     SamtoolMpileupWorker.obj
 0002:00006bbc       __unwindtable$?detach_helper_grow@?$QList@VDescriptor@U2@@@@AAEPAUNode@1@HH@Z 10026bbc     SamtoolMpileupWorker.obj
 0002:00006bdc       __ehfuncinfo$?detach_helper_grow@?$QList@VDescriptor@U2@@@@AAEPAUNode@1@HH@Z 10026bdc     SamtoolMpileupWorker.obj
 0002:00006c00       __tryblocktable$?detach_helper_grow@?$QList@VDescriptor@U2@@@@AAEPAUNode@1@HH@Z 10026c00     SamtoolMpileupWorker.obj
 0002:00006c28       __catchsym$?detach_helper@?$QList@VDescriptor@U2@@@@AAEXH@Z$2 10026c28     SamtoolMpileupWorker.obj
 0002:00006c38       __unwindtable$?detach_helper@?$QList@VDescriptor@U2@@@@AAEXH@Z 10026c38     SamtoolMpileupWorker.obj
 0002:00006c48       __tryblocktable$?detach_helper@?$QList@VDescriptor@U2@@@@AAEXH@Z 10026c48     SamtoolMpileupWorker.obj
 0002:00006c5c       __ehfuncinfo$?detach_helper@?$QList@VDescriptor@U2@@@@AAEXH@Z 10026c5c     SamtoolMpileupWorker.obj
 0002:00006c80       __unwindtable$?node_construct@?$QList@VDescriptor@U2@@@@AAEXPAUNode@1@ABVDescriptor@U2@@@Z 10026c80     SamtoolMpileupWorker.obj
 0002:00006c90       __ehfuncinfo$?node_construct@?$QList@VDescriptor@U2@@@@AAEXPAUNode@1@ABVDescriptor@U2@@@Z 10026c90     SamtoolMpileupWorker.obj
 0002:00006cb4       __catchsym$?node_copy@?$QList@VDescriptor@U2@@@@AAEXPAUNode@1@00@Z$6 10026cb4     SamtoolMpileupWorker.obj
 0002:00006cc4       __tryblocktable$?node_copy@?$QList@VDescriptor@U2@@@@AAEXPAUNode@1@00@Z 10026cc4     SamtoolMpileupWorker.obj
 0002:00006cd8       __ehfuncinfo$?node_copy@?$QList@VDescriptor@U2@@@@AAEXPAUNode@1@00@Z 10026cd8     SamtoolMpileupWorker.obj
 0002:00006cfc       __unwindtable$?node_copy@?$QList@VDescriptor@U2@@@@AAEXPAUNode@1@00@Z 10026cfc     SamtoolMpileupWorker.obj
 0002:00006d2c       __unwindtable$??A?$QMap@VDescriptor@U2@@V?$QExplicitlySharedDataPointer@VDataType@U2@@@@@@QAEAAV?$QExplicitlySharedDataPointer@VDataType@U2@@@@ABVDescriptor@U2@@@Z 10026d2c     SamtoolMpileupWorker.obj
 0002:00006d34       __ehfuncinfo$??A?$QMap@VDescriptor@U2@@V?$QExplicitlySharedDataPointer@VDataType@U2@@@@@@QAEAAV?$QExplicitlySharedDataPointer@VDataType@U2@@@@ABVDescriptor@U2@@@Z 10026d34     SamtoolMpileupWorker.obj
 0002:00006d58       __unwindtable$??$qvariant_cast@V?$QMap@VQString@@V1@@@@@YA?AV?$QMap@VQString@@V1@@@ABVQVariant@@@Z 10026d58     SamtoolMpileupWorker.obj
 0002:00006d68       __ehfuncinfo$??$qvariant_cast@V?$QMap@VQString@@V1@@@@@YA?AV?$QMap@VQString@@V1@@@ABVQVariant@@@Z 10026d68     SamtoolMpileupWorker.obj
 0002:00006d8c       __unwindtable$?uniqueKeys@?$QMap@VDescriptor@U2@@VQVariant@@@@QBE?AV?$QList@VDescriptor@U2@@@@XZ 10026d8c     SamtoolMpileupWorker.obj
 0002:00006d94       __ehfuncinfo$?uniqueKeys@?$QMap@VDescriptor@U2@@VQVariant@@@@QBE?AV?$QList@VDescriptor@U2@@@@XZ 10026d94     SamtoolMpileupWorker.obj
 0002:00006db8       __ehfuncinfo$??$getAttributeValue@VQString@@@Attribute@U2@@QBE?AVQString@@PAVWorkflowContext@Workflow@1@@Z 10026db8     SamtoolMpileupWorker.obj
 0002:00006ddc       __unwindtable$??$getAttributeValue@VQString@@@Attribute@U2@@QBE?AVQString@@PAVWorkflowContext@Workflow@1@@Z 10026ddc     SamtoolMpileupWorker.obj
 0002:00006e4c       __ehfuncinfo$??$getAttributeValue@H@Attribute@U2@@QBEHPAVWorkflowContext@Workflow@1@@Z 10026e4c     SamtoolMpileupWorker.obj
 0002:00006e70       __unwindtable$??$getAttributeValue@H@Attribute@U2@@QBEHPAVWorkflowContext@Workflow@1@@Z 10026e70     SamtoolMpileupWorker.obj
 0002:00006ed8       __catchsym$?append@?$QList@PAVAttribute@U2@@@@QAEXABQAVAttribute@U2@@@Z$6 10026ed8     SamtoolMpileupWorker.obj
 0002:00006ee8       __tryblocktable$?append@?$QList@PAVAttribute@U2@@@@QAEXABQAVAttribute@U2@@@Z 10026ee8     SamtoolMpileupWorker.obj
 0002:00006efc       __ehfuncinfo$?append@?$QList@PAVAttribute@U2@@@@QAEXABQAVAttribute@U2@@@Z 10026efc     SamtoolMpileupWorker.obj
 0002:00006f20       __unwindtable$?append@?$QList@PAVAttribute@U2@@@@QAEXABQAVAttribute@U2@@@Z 10026f20     SamtoolMpileupWorker.obj
 0002:00006f50       __catchsym$?detach_helper_grow@?$QList@PAVAttribute@U2@@@@AAEPAUNode@1@HH@Z$5 10026f50     SamtoolMpileupWorker.obj
 0002:00006f60       __catchsym$?detach_helper_grow@?$QList@PAVAttribute@U2@@@@AAEPAUNode@1@HH@Z$4 10026f60     SamtoolMpileupWorker.obj
 0002:00006f70       __unwindtable$?detach_helper_grow@?$QList@PAVAttribute@U2@@@@AAEPAUNode@1@HH@Z 10026f70     SamtoolMpileupWorker.obj
 0002:00006f90       __ehfuncinfo$?detach_helper_grow@?$QList@PAVAttribute@U2@@@@AAEPAUNode@1@HH@Z 10026f90     SamtoolMpileupWorker.obj
 0002:00006fb4       __tryblocktable$?detach_helper_grow@?$QList@PAVAttribute@U2@@@@AAEPAUNode@1@HH@Z 10026fb4     SamtoolMpileupWorker.obj
 0002:00006fdc       __catchsym$?append@?$QList@PAVPortDescriptor@Workflow@U2@@@@QAEXABQAVPortDescriptor@Workflow@U2@@@Z$6 10026fdc     SamtoolMpileupWorker.obj
 0002:00006fec       __tryblocktable$?append@?$QList@PAVPortDescriptor@Workflow@U2@@@@QAEXABQAVPortDescriptor@Workflow@U2@@@Z 10026fec     SamtoolMpileupWorker.obj
 0002:00007000       __ehfuncinfo$?append@?$QList@PAVPortDescriptor@Workflow@U2@@@@QAEXABQAVPortDescriptor@Workflow@U2@@@Z 10027000     SamtoolMpileupWorker.obj
 0002:00007024       __unwindtable$?append@?$QList@PAVPortDescriptor@Workflow@U2@@@@QAEXABQAVPortDescriptor@Workflow@U2@@@Z 10027024     SamtoolMpileupWorker.obj
 0002:00007054       __catchsym$?detach_helper_grow@?$QList@PAVPortDescriptor@Workflow@U2@@@@AAEPAUNode@1@HH@Z$5 10027054     SamtoolMpileupWorker.obj
 0002:00007064       __catchsym$?detach_helper_grow@?$QList@PAVPortDescriptor@Workflow@U2@@@@AAEPAUNode@1@HH@Z$4 10027064     SamtoolMpileupWorker.obj
 0002:00007074       __unwindtable$?detach_helper_grow@?$QList@PAVPortDescriptor@Workflow@U2@@@@AAEPAUNode@1@HH@Z 10027074     SamtoolMpileupWorker.obj
 0002:00007094       __ehfuncinfo$?detach_helper_grow@?$QList@PAVPortDescriptor@Workflow@U2@@@@AAEPAUNode@1@HH@Z 10027094     SamtoolMpileupWorker.obj
 0002:000070b8       __tryblocktable$?detach_helper_grow@?$QList@PAVPortDescriptor@Workflow@U2@@@@AAEPAUNode@1@HH@Z 100270b8     SamtoolMpileupWorker.obj
 0002:000070e0       __catchsym$?append@?$QList@VWorkflowNotification@U2@@@@QAEXABVWorkflowNotification@U2@@@Z$11 100270e0     SamtoolMpileupWorker.obj
 0002:000070f0       __catchsym$?append@?$QList@VWorkflowNotification@U2@@@@QAEXABVWorkflowNotification@U2@@@Z$10 100270f0     SamtoolMpileupWorker.obj
 0002:00007100       __ehfuncinfo$?append@?$QList@VWorkflowNotification@U2@@@@QAEXABVWorkflowNotification@U2@@@Z 10027100     SamtoolMpileupWorker.obj
 0002:00007124       __tryblocktable$?append@?$QList@VWorkflowNotification@U2@@@@QAEXABVWorkflowNotification@U2@@@Z 10027124     SamtoolMpileupWorker.obj
 0002:0000714c       __unwindtable$?append@?$QList@VWorkflowNotification@U2@@@@QAEXABVWorkflowNotification@U2@@@Z 1002714c     SamtoolMpileupWorker.obj
 0002:0000719c       __catchsym$?detach_helper_grow@?$QList@VWorkflowNotification@U2@@@@AAEPAUNode@1@HH@Z$5 1002719c     SamtoolMpileupWorker.obj
 0002:000071ac       __catchsym$?detach_helper_grow@?$QList@VWorkflowNotification@U2@@@@AAEPAUNode@1@HH@Z$4 100271ac     SamtoolMpileupWorker.obj
 0002:000071bc       __unwindtable$?detach_helper_grow@?$QList@VWorkflowNotification@U2@@@@AAEPAUNode@1@HH@Z 100271bc     SamtoolMpileupWorker.obj
 0002:000071dc       __ehfuncinfo$?detach_helper_grow@?$QList@VWorkflowNotification@U2@@@@AAEPAUNode@1@HH@Z 100271dc     SamtoolMpileupWorker.obj
 0002:00007200       __tryblocktable$?detach_helper_grow@?$QList@VWorkflowNotification@U2@@@@AAEPAUNode@1@HH@Z 10027200     SamtoolMpileupWorker.obj
 0002:00007228       __unwindtable$?node_construct@?$QList@VWorkflowNotification@U2@@@@AAEXPAUNode@1@ABVWorkflowNotification@U2@@@Z 10027228     SamtoolMpileupWorker.obj
 0002:00007238       __ehfuncinfo$?node_construct@?$QList@VWorkflowNotification@U2@@@@AAEXPAUNode@1@ABVWorkflowNotification@U2@@@Z 10027238     SamtoolMpileupWorker.obj
 0002:0000725c       __catchsym$?node_copy@?$QList@VWorkflowNotification@U2@@@@AAEXPAUNode@1@00@Z$6 1002725c     SamtoolMpileupWorker.obj
 0002:0000726c       __tryblocktable$?node_copy@?$QList@VWorkflowNotification@U2@@@@AAEXPAUNode@1@00@Z 1002726c     SamtoolMpileupWorker.obj
 0002:00007280       __ehfuncinfo$?node_copy@?$QList@VWorkflowNotification@U2@@@@AAEXPAUNode@1@00@Z 10027280     SamtoolMpileupWorker.obj
 0002:000072a4       __unwindtable$?node_copy@?$QList@VWorkflowNotification@U2@@@@AAEXPAUNode@1@00@Z 100272a4     SamtoolMpileupWorker.obj
 0002:000072d4       __catchsym$?append@?$QList@VMessage@Workflow@U2@@@@QAEXABVMessage@Workflow@U2@@@Z$11 100272d4     SamtoolMpileupWorker.obj
 0002:000072e4       __catchsym$?append@?$QList@VMessage@Workflow@U2@@@@QAEXABVMessage@Workflow@U2@@@Z$10 100272e4     SamtoolMpileupWorker.obj
 0002:000072f4       __ehfuncinfo$?append@?$QList@VMessage@Workflow@U2@@@@QAEXABVMessage@Workflow@U2@@@Z 100272f4     SamtoolMpileupWorker.obj
 0002:00007318       __tryblocktable$?append@?$QList@VMessage@Workflow@U2@@@@QAEXABVMessage@Workflow@U2@@@Z 10027318     SamtoolMpileupWorker.obj
 0002:00007340       __unwindtable$?append@?$QList@VMessage@Workflow@U2@@@@QAEXABVMessage@Workflow@U2@@@Z 10027340     SamtoolMpileupWorker.obj
 0002:00007390       __unwindtable$?takeFirst@?$QList@VMessage@Workflow@U2@@@@QAE?AVMessage@Workflow@U2@@XZ 10027390     SamtoolMpileupWorker.obj
 0002:00007398       __ehfuncinfo$?takeFirst@?$QList@VMessage@Workflow@U2@@@@QAE?AVMessage@Workflow@U2@@XZ 10027398     SamtoolMpileupWorker.obj
 0002:000073bc       __catchsym$?detach_helper_grow@?$QList@VMessage@Workflow@U2@@@@AAEPAUNode@1@HH@Z$5 100273bc     SamtoolMpileupWorker.obj
 0002:000073cc       __catchsym$?detach_helper_grow@?$QList@VMessage@Workflow@U2@@@@AAEPAUNode@1@HH@Z$4 100273cc     SamtoolMpileupWorker.obj
 0002:000073dc       __unwindtable$?detach_helper_grow@?$QList@VMessage@Workflow@U2@@@@AAEPAUNode@1@HH@Z 100273dc     SamtoolMpileupWorker.obj
 0002:000073fc       __ehfuncinfo$?detach_helper_grow@?$QList@VMessage@Workflow@U2@@@@AAEPAUNode@1@HH@Z 100273fc     SamtoolMpileupWorker.obj
 0002:00007420       __tryblocktable$?detach_helper_grow@?$QList@VMessage@Workflow@U2@@@@AAEPAUNode@1@HH@Z 10027420     SamtoolMpileupWorker.obj
 0002:00007448       __catchsym$?detach_helper@?$QList@VMessage@Workflow@U2@@@@AAEXH@Z$2 10027448     SamtoolMpileupWorker.obj
 0002:00007458       __unwindtable$?detach_helper@?$QList@VMessage@Workflow@U2@@@@AAEXH@Z 10027458     SamtoolMpileupWorker.obj
 0002:00007468       __tryblocktable$?detach_helper@?$QList@VMessage@Workflow@U2@@@@AAEXH@Z 10027468     SamtoolMpileupWorker.obj
 0002:0000747c       __ehfuncinfo$?detach_helper@?$QList@VMessage@Workflow@U2@@@@AAEXH@Z 1002747c     SamtoolMpileupWorker.obj
 0002:000074a0       __unwindtable$?node_construct@?$QList@VMessage@Workflow@U2@@@@AAEXPAUNode@1@ABVMessage@Workflow@U2@@@Z 100274a0     SamtoolMpileupWorker.obj
 0002:000074b0       __ehfuncinfo$?node_construct@?$QList@VMessage@Workflow@U2@@@@AAEXPAUNode@1@ABVMessage@Workflow@U2@@@Z 100274b0     SamtoolMpileupWorker.obj
 0002:000074d4       __catchsym$?node_copy@?$QList@VMessage@Workflow@U2@@@@AAEXPAUNode@1@00@Z$6 100274d4     SamtoolMpileupWorker.obj
 0002:000074e4       __tryblocktable$?node_copy@?$QList@VMessage@Workflow@U2@@@@AAEXPAUNode@1@00@Z 100274e4     SamtoolMpileupWorker.obj
 0002:000074f8       __ehfuncinfo$?node_copy@?$QList@VMessage@Workflow@U2@@@@AAEXPAUNode@1@00@Z 100274f8     SamtoolMpileupWorker.obj
 0002:0000751c       __unwindtable$?node_copy@?$QList@VMessage@Workflow@U2@@@@AAEXPAUNode@1@00@Z 1002751c     SamtoolMpileupWorker.obj
 0002:0000754c       __unwindtable$??$getValue@VQString@@@BaseWorker@LocalWorkflow@U2@@IBE?AVQString@@ABV3@@Z 1002754c     SamtoolMpileupWorker.obj
 0002:0000755c       __ehfuncinfo$??$getValue@VQString@@@BaseWorker@LocalWorkflow@U2@@IBE?AVQString@@ABV3@@Z 1002755c     SamtoolMpileupWorker.obj
 0002:00007580       __ehfuncinfo$??0CallVariantsTaskSettings@LocalWorkflow@U2@@QAE@XZ 10027580     SamtoolMpileupWorker.obj
 0002:000075a4       __unwindtable$??0CallVariantsTaskSettings@LocalWorkflow@U2@@QAE@XZ 100275a4     SamtoolMpileupWorker.obj
 0002:000075ec       __catchsym$??0?$QList@V?$QMap@VQString@@VQVariant@@@@@@QAE@ABV0@@Z$2 100275ec     SamtoolMpileupWorker.obj
 0002:000075fc       __unwindtable$??0?$QList@V?$QMap@VQString@@VQVariant@@@@@@QAE@ABV0@@Z 100275fc     SamtoolMpileupWorker.obj
 0002:0000760c       __tryblocktable$??0?$QList@V?$QMap@VQString@@VQVariant@@@@@@QAE@ABV0@@Z 1002760c     SamtoolMpileupWorker.obj
 0002:00007620       __ehfuncinfo$??0?$QList@V?$QMap@VQString@@VQVariant@@@@@@QAE@ABV0@@Z 10027620     SamtoolMpileupWorker.obj
 0002:00007644       __ehfuncinfo$?createDescription@?$PrompterBase@VCallVariantsPrompter@LocalWorkflow@U2@@@U2@@UAEPAVActorDocument@Workflow@2@PAVActor@42@@Z 10027644     SamtoolMpileupWorker.obj
 0002:00007668       __unwindtable$?createDescription@?$PrompterBase@VCallVariantsPrompter@LocalWorkflow@U2@@@U2@@UAEPAVActorDocument@Workflow@2@PAVActor@42@@Z 10027668     SamtoolMpileupWorker.obj
 0002:000076a0       __ehfuncinfo$?composeRichDoc@CallVariantsPrompter@LocalWorkflow@U2@@MAE?AVQString@@XZ 100276a0     SamtoolMpileupWorker.obj
 0002:000076c4       __unwindtable$?composeRichDoc@CallVariantsPrompter@LocalWorkflow@U2@@MAE?AVQString@@XZ 100276c4     SamtoolMpileupWorker.obj
 0002:000077bc       __unwindtable$??0CallVariantsWorker@LocalWorkflow@U2@@QAE@PAVActor@Workflow@2@@Z 100277bc     SamtoolMpileupWorker.obj
 0002:000077dc       __ehfuncinfo$??0CallVariantsWorker@LocalWorkflow@U2@@QAE@PAVActor@Workflow@2@@Z 100277dc     SamtoolMpileupWorker.obj
 0002:00007800       __ehfuncinfo$?init@CallVariantsWorker@LocalWorkflow@U2@@UAEXXZ 10027800     SamtoolMpileupWorker.obj
 0002:00007824       __unwindtable$?init@CallVariantsWorker@LocalWorkflow@U2@@UAEXXZ 10027824     SamtoolMpileupWorker.obj
 0002:0000784c       __ehfuncinfo$?tick@CallVariantsWorker@LocalWorkflow@U2@@UAEPAVTask@3@XZ 1002784c     SamtoolMpileupWorker.obj
 0002:00007870       __unwindtable$?tick@CallVariantsWorker@LocalWorkflow@U2@@UAEPAVTask@3@XZ 10027870     SamtoolMpileupWorker.obj
 0002:000078b8       __ehfuncinfo$?sl_taskFinished@CallVariantsWorker@LocalWorkflow@U2@@AAEXXZ 100278b8     SamtoolMpileupWorker.obj
 0002:000078dc       __unwindtable$?sl_taskFinished@CallVariantsWorker@LocalWorkflow@U2@@AAEXXZ 100278dc     SamtoolMpileupWorker.obj
 0002:0000790c       __ehfuncinfo$?initDatasetMode@CallVariantsWorker@LocalWorkflow@U2@@AAEXXZ 1002790c     SamtoolMpileupWorker.obj
 0002:00007930       __unwindtable$?initDatasetMode@CallVariantsWorker@LocalWorkflow@U2@@AAEXXZ 10027930     SamtoolMpileupWorker.obj
 0002:000079c0       __ehfuncinfo$?takeAssembly@CallVariantsWorker@LocalWorkflow@U2@@AAEXAAVU2OpStatus@3@@Z 100279c0     SamtoolMpileupWorker.obj
 0002:000079e4       __unwindtable$?takeAssembly@CallVariantsWorker@LocalWorkflow@U2@@AAEXAAVU2OpStatus@3@@Z 100279e4     SamtoolMpileupWorker.obj
 0002:00007a6c       __ehfuncinfo$?takeReference@CallVariantsWorker@LocalWorkflow@U2@@AAEXAAVU2OpStatus@3@@Z 10027a6c     SamtoolMpileupWorker.obj
 0002:00007a90       __unwindtable$?takeReference@CallVariantsWorker@LocalWorkflow@U2@@AAEXAAVU2OpStatus@3@@Z 10027a90     SamtoolMpileupWorker.obj
 0002:00007af0       __ehfuncinfo$?getSettings@CallVariantsWorker@LocalWorkflow@U2@@AAE?AVCallVariantsTaskSettings@23@XZ 10027af0     SamtoolMpileupWorker.obj
 0002:00007b14       __unwindtable$?getSettings@CallVariantsWorker@LocalWorkflow@U2@@AAE?AVCallVariantsTaskSettings@23@XZ 10027b14     SamtoolMpileupWorker.obj
 0002:00007b94       __unwindtable$?processError@CallVariantsWorker@LocalWorkflow@U2@@AAEXABVU2OpStatus@3@@Z 10027b94     SamtoolMpileupWorker.obj
 0002:00007ba4       __ehfuncinfo$?processError@CallVariantsWorker@LocalWorkflow@U2@@AAEXABVU2OpStatus@3@@Z 10027ba4     SamtoolMpileupWorker.obj
 0002:00007bc8       __unwindtable$?checkState@CallVariantsWorker@LocalWorkflow@U2@@AAEXAAVU2OpStatus@3@@Z 10027bc8     SamtoolMpileupWorker.obj
 0002:00007be0       __ehfuncinfo$?checkState@CallVariantsWorker@LocalWorkflow@U2@@AAEXAAVU2OpStatus@3@@Z 10027be0     SamtoolMpileupWorker.obj
 0002:00007c04       __unwindtable$??1CallVariantsWorker@LocalWorkflow@U2@@UAE@XZ 10027c04     SamtoolMpileupWorker.obj
 0002:00007c24       __ehfuncinfo$??1CallVariantsWorker@LocalWorkflow@U2@@UAE@XZ 10027c24     SamtoolMpileupWorker.obj
 0002:00007c48       __ehfuncinfo$?init@CallVariantsWorkerFactory@LocalWorkflow@U2@@SAXXZ 10027c48     SamtoolMpileupWorker.obj
 0002:00007c6c       __unwindtable$?init@CallVariantsWorkerFactory@LocalWorkflow@U2@@SAXXZ 10027c6c     SamtoolMpileupWorker.obj
 0002:000093a4       __unwindtable$?createWorker@CallVariantsWorkerFactory@LocalWorkflow@U2@@UAEPAVWorker@Workflow@3@PAVActor@53@@Z 100293a4     SamtoolMpileupWorker.obj
 0002:000093ac       __ehfuncinfo$?createWorker@CallVariantsWorkerFactory@LocalWorkflow@U2@@UAEPAVWorker@Workflow@3@PAVActor@53@@Z 100293ac     SamtoolMpileupWorker.obj
 0002:000093d0       __unwindtable$??0ScientificDoubleWidget@LocalWorkflow@U2@@QAE@PAVQWidget@@@Z 100293d0     SamtoolMpileupWorker.obj
 0002:000093e8       __ehfuncinfo$??0ScientificDoubleWidget@LocalWorkflow@U2@@QAE@PAVQWidget@@@Z 100293e8     SamtoolMpileupWorker.obj
 0002:0000940c       __unwindtable$?value@ScientificDoubleWidget@LocalWorkflow@U2@@UAE?AVQVariant@@XZ 1002940c     SamtoolMpileupWorker.obj
 0002:0000941c       __ehfuncinfo$?value@ScientificDoubleWidget@LocalWorkflow@U2@@UAE?AVQVariant@@XZ 1002941c     SamtoolMpileupWorker.obj
 0002:00009440       __unwindtable$?setValue@ScientificDoubleWidget@LocalWorkflow@U2@@UAEXABVQVariant@@@Z 10029440     SamtoolMpileupWorker.obj
 0002:00009448       __ehfuncinfo$?setValue@ScientificDoubleWidget@LocalWorkflow@U2@@UAEXABVQVariant@@@Z 10029448     SamtoolMpileupWorker.obj
 0002:0000946c       __unwindtable$?clone@ScientificDoubleDelegate@LocalWorkflow@U2@@UAEPAVPropertyDelegate@3@XZ 1002946c     SamtoolMpileupWorker.obj
 0002:00009474       __ehfuncinfo$?clone@ScientificDoubleDelegate@LocalWorkflow@U2@@UAEPAVPropertyDelegate@3@XZ 10029474     SamtoolMpileupWorker.obj
 0002:00009498       __unwindtable$?createWizardWidget@ScientificDoubleDelegate@LocalWorkflow@U2@@UBEPAVPropertyWidget@3@AAVU2OpStatus@3@PAVQWidget@@@Z 10029498     SamtoolMpileupWorker.obj
 0002:000094a0       __ehfuncinfo$?createWizardWidget@ScientificDoubleDelegate@LocalWorkflow@U2@@UBEPAVPropertyWidget@3@AAVU2OpStatus@3@PAVQWidget@@@Z 100294a0     SamtoolMpileupWorker.obj
 0002:000094c4       __unwindtable$?createEditor@ScientificDoubleDelegate@LocalWorkflow@U2@@UBEPAVQWidget@@PAV4@ABVQStyleOptionViewItem@@ABVQModelIndex@@@Z 100294c4     SamtoolMpileupWorker.obj
 0002:000094cc       __ehfuncinfo$?createEditor@ScientificDoubleDelegate@LocalWorkflow@U2@@UBEPAVQWidget@@PAV4@ABVQStyleOptionViewItem@@ABVQModelIndex@@@Z 100294cc     SamtoolMpileupWorker.obj
 0002:000094f0       __unwindtable$?setEditorData@ScientificDoubleDelegate@LocalWorkflow@U2@@UBEXPAVQWidget@@ABVQModelIndex@@@Z 100294f0     SamtoolMpileupWorker.obj
 0002:000094f8       __ehfuncinfo$?setEditorData@ScientificDoubleDelegate@LocalWorkflow@U2@@UBEXPAVQWidget@@ABVQModelIndex@@@Z 100294f8     SamtoolMpileupWorker.obj
 0002:0000951c       __unwindtable$?setModelData@ScientificDoubleDelegate@LocalWorkflow@U2@@UBEXPAVQWidget@@PAVQAbstractItemModel@@ABVQModelIndex@@@Z 1002951c     SamtoolMpileupWorker.obj
 0002:00009524       __ehfuncinfo$?setModelData@ScientificDoubleDelegate@LocalWorkflow@U2@@UBEXPAVQWidget@@PAVQAbstractItemModel@@ABVQModelIndex@@@Z 10029524     SamtoolMpileupWorker.obj
 0002:00009548       __unwindtable$??0EmptySlotValidator@LocalWorkflow@U2@@QAE@ABVQString@@@Z 10029548     SamtoolMpileupWorker.obj
 0002:00009550       __ehfuncinfo$??0EmptySlotValidator@LocalWorkflow@U2@@QAE@ABVQString@@@Z 10029550     SamtoolMpileupWorker.obj
 0002:00009574       __ehfuncinfo$?validate@EmptySlotValidator@LocalWorkflow@U2@@UBE_NPBVConfiguration@3@AAV?$QList@VWorkflowNotification@U2@@@@@Z 10029574     SamtoolMpileupWorker.obj
 0002:00009598       __unwindtable$?validate@EmptySlotValidator@LocalWorkflow@U2@@UBE_NPBVConfiguration@3@AAV?$QList@VWorkflowNotification@U2@@@@@Z 10029598     SamtoolMpileupWorker.obj
 0002:000095f0       __unwindtable$??1EmptySlotValidator@LocalWorkflow@U2@@UAE@XZ 100295f0     SamtoolMpileupWorker.obj
 0002:000095f8       __ehfuncinfo$??1EmptySlotValidator@LocalWorkflow@U2@@UAE@XZ 100295f8     SamtoolMpileupWorker.obj
 0002:0000961c       __unwindtable$??_GEmptySlotValidator@LocalWorkflow@U2@@UAEPAXI@Z 1002961c     SamtoolMpileupWorker.obj
 0002:00009624       __ehfuncinfo$??_GEmptySlotValidator@LocalWorkflow@U2@@UAEPAXI@Z 10029624     SamtoolMpileupWorker.obj
 0002:00009648       __catchsym$?createNode@?$QMapData@VQString@@VQScriptValue@@@@QAEPAU?$QMapNode@VQString@@VQScriptValue@@@@ABVQString@@ABVQScriptValue@@PAU2@_N@Z$7 10029648     SamtoolMpileupWorker.obj
 0002:00009658       __catchsym$?createNode@?$QMapData@VQString@@VQScriptValue@@@@QAEPAU?$QMapNode@VQString@@VQScriptValue@@@@ABVQString@@ABVQScriptValue@@PAU2@_N@Z$6 10029658     SamtoolMpileupWorker.obj
 0002:00009668       __ehfuncinfo$?createNode@?$QMapData@VQString@@VQScriptValue@@@@QAEPAU?$QMapNode@VQString@@VQScriptValue@@@@ABVQString@@ABVQScriptValue@@PAU2@_N@Z 10029668     SamtoolMpileupWorker.obj
 0002:0000968c       __tryblocktable$?createNode@?$QMapData@VQString@@VQScriptValue@@@@QAEPAU?$QMapNode@VQString@@VQScriptValue@@@@ABVQString@@ABVQScriptValue@@PAU2@_N@Z 1002968c     SamtoolMpileupWorker.obj
 0002:000096b4       __unwindtable$?createNode@?$QMapData@VQString@@VQScriptValue@@@@QAEPAU?$QMapNode@VQString@@VQScriptValue@@@@ABVQString@@ABVQScriptValue@@PAU2@_N@Z 100296b4     SamtoolMpileupWorker.obj
 0002:000096e4       __catchsym$?createNode@?$QMapData@VDescriptor@U2@@V?$QExplicitlySharedDataPointer@VDataType@U2@@@@@@QAEPAU?$QMapNode@VDescriptor@U2@@V?$QExplicitlySharedDataPointer@VDataType@U2@@@@@@ABVDescriptor@U2@@ABV?$QExplicitlySharedDataPointer@VDataType@U2@@@@PAU2@_N@Z$6 100296e4     SamtoolMpileupWorker.obj
 0002:000096f4       __tryblocktable$?createNode@?$QMapData@VDescriptor@U2@@V?$QExplicitlySharedDataPointer@VDataType@U2@@@@@@QAEPAU?$QMapNode@VDescriptor@U2@@V?$QExplicitlySharedDataPointer@VDataType@U2@@@@@@ABVDescriptor@U2@@ABV?$QExplicitlySharedDataPointer@VDataType@U2@@@@PAU2@_N@Z 100296f4     SamtoolMpileupWorker.obj
 0002:00009708       __ehfuncinfo$?createNode@?$QMapData@VDescriptor@U2@@V?$QExplicitlySharedDataPointer@VDataType@U2@@@@@@QAEPAU?$QMapNode@VDescriptor@U2@@V?$QExplicitlySharedDataPointer@VDataType@U2@@@@@@ABVDescriptor@U2@@ABV?$QExplicitlySharedDataPointer@VDataType@U2@@@@PAU2@_N@Z 10029708     SamtoolMpileupWorker.obj
 0002:0000972c       __unwindtable$?createNode@?$QMapData@VDescriptor@U2@@V?$QExplicitlySharedDataPointer@VDataType@U2@@@@@@QAEPAU?$QMapNode@VDescriptor@U2@@V?$QExplicitlySharedDataPointer@VDataType@U2@@@@@@ABVDescriptor@U2@@ABV?$QExplicitlySharedDataPointer@VDataType@U2@@@@PAU2@_N@Z 1002972c     SamtoolMpileupWorker.obj
 0002:00009754       __catchsym$?createNode@?$QMapData@VQString@@V1@@@QAEPAU?$QMapNode@VQString@@V1@@@ABVQString@@0PAU2@_N@Z$7 10029754     SamtoolMpileupWorker.obj
 0002:00009764       __catchsym$?createNode@?$QMapData@VQString@@V1@@@QAEPAU?$QMapNode@VQString@@V1@@@ABVQString@@0PAU2@_N@Z$6 10029764     SamtoolMpileupWorker.obj
 0002:00009774       __ehfuncinfo$?createNode@?$QMapData@VQString@@V1@@@QAEPAU?$QMapNode@VQString@@V1@@@ABVQString@@0PAU2@_N@Z 10029774     SamtoolMpileupWorker.obj
 0002:00009798       __tryblocktable$?createNode@?$QMapData@VQString@@V1@@@QAEPAU?$QMapNode@VQString@@V1@@@ABVQString@@0PAU2@_N@Z 10029798     SamtoolMpileupWorker.obj
 0002:000097c0       __unwindtable$?createNode@?$QMapData@VQString@@V1@@@QAEPAU?$QMapNode@VQString@@V1@@@ABVQString@@0PAU2@_N@Z 100297c0     SamtoolMpileupWorker.obj
 0002:000097f0       __catchsym$?createNode@?$QMapData@VQString@@PAVPropertyDelegate@U2@@@@QAEPAU?$QMapNode@VQString@@PAVPropertyDelegate@U2@@@@ABVQString@@ABQAVPropertyDelegate@U2@@PAU2@_N@Z$5 100297f0     SamtoolMpileupWorker.obj
 0002:00009800       __tryblocktable$?createNode@?$QMapData@VQString@@PAVPropertyDelegate@U2@@@@QAEPAU?$QMapNode@VQString@@PAVPropertyDelegate@U2@@@@ABVQString@@ABQAVPropertyDelegate@U2@@PAU2@_N@Z 10029800     SamtoolMpileupWorker.obj
 0002:00009814       __ehfuncinfo$?createNode@?$QMapData@VQString@@PAVPropertyDelegate@U2@@@@QAEPAU?$QMapNode@VQString@@PAVPropertyDelegate@U2@@@@ABVQString@@ABQAVPropertyDelegate@U2@@PAU2@_N@Z 10029814     SamtoolMpileupWorker.obj
 0002:00009838       __unwindtable$?createNode@?$QMapData@VQString@@PAVPropertyDelegate@U2@@@@QAEPAU?$QMapNode@VQString@@PAVPropertyDelegate@U2@@@@ABVQString@@ABQAVPropertyDelegate@U2@@PAU2@_N@Z 10029838     SamtoolMpileupWorker.obj
 0002:00009860       __catchsym$??0?$QList@PAVPort@Workflow@U2@@@@QAE@ABV0@@Z$2 10029860     SamtoolMpileupWorker.obj
 0002:00009870       __unwindtable$??0?$QList@PAVPort@Workflow@U2@@@@QAE@ABV0@@Z 10029870     SamtoolMpileupWorker.obj
 0002:00009880       __tryblocktable$??0?$QList@PAVPort@Workflow@U2@@@@QAE@ABV0@@Z 10029880     SamtoolMpileupWorker.obj
 0002:00009894       __ehfuncinfo$??0?$QList@PAVPort@Workflow@U2@@@@QAE@ABV0@@Z 10029894     SamtoolMpileupWorker.obj
 0002:000098b8       __unwindtable$?metaType@?$QVariantValueHelper@VQString@@@QtPrivate@@SA?AVQString@@ABVQVariant@@@Z 100298b8     SamtoolMpileupWorker.obj
 0002:000098c8       __ehfuncinfo$?metaType@?$QVariantValueHelper@VQString@@@QtPrivate@@SA?AVQString@@ABVQVariant@@@Z 100298c8     SamtoolMpileupWorker.obj
 0002:000098ec       __ehfuncinfo$??0SamtoolsPlugin@U2@@QAE@XZ 100298ec     SamtoolsPlugin.obj
 0002:00009910       __unwindtable$??0SamtoolsPlugin@U2@@QAE@XZ 10029910     SamtoolsPlugin.obj
 0002:00009938       __unwindtable$??__EalgoLog@U2@@YAXXZ 10029938     SamtoolsPlugin.obj
 0002:00009940       __ehfuncinfo$??__EalgoLog@U2@@YAXXZ 10029940     SamtoolsPlugin.obj
 0002:00009964       __unwindtable$??__EcmdLog@U2@@YAXXZ 10029964     SamtoolsPlugin.obj
 0002:0000996c       __ehfuncinfo$??__EcmdLog@U2@@YAXXZ 1002996c     SamtoolsPlugin.obj
 0002:00009990       __unwindtable$??__EcoreLog@U2@@YAXXZ 10029990     SamtoolsPlugin.obj
 0002:00009998       __ehfuncinfo$??__EcoreLog@U2@@YAXXZ 10029998     SamtoolsPlugin.obj
 0002:000099bc       __unwindtable$??__EioLog@U2@@YAXXZ 100299bc     SamtoolsPlugin.obj
 0002:000099c4       __ehfuncinfo$??__EioLog@U2@@YAXXZ 100299c4     SamtoolsPlugin.obj
 0002:000099e8       __unwindtable$??__EperfLog@U2@@YAXXZ 100299e8     SamtoolsPlugin.obj
 0002:000099f0       __ehfuncinfo$??__EperfLog@U2@@YAXXZ 100299f0     SamtoolsPlugin.obj
 0002:00009a14       __unwindtable$??__EscriptLog@U2@@YAXXZ 10029a14     SamtoolsPlugin.obj
 0002:00009a1c       __ehfuncinfo$??__EscriptLog@U2@@YAXXZ 10029a1c     SamtoolsPlugin.obj
 0002:00009a40       __unwindtable$??__EtaskLog@U2@@YAXXZ 10029a40     SamtoolsPlugin.obj
 0002:00009a48       __ehfuncinfo$??__EtaskLog@U2@@YAXXZ 10029a48     SamtoolsPlugin.obj
 0002:00009a6c       __unwindtable$??__EuiLog@U2@@YAXXZ 10029a6c     SamtoolsPlugin.obj
 0002:00009a74       __ehfuncinfo$??__EuiLog@U2@@YAXXZ 10029a74     SamtoolsPlugin.obj
 0002:00009a98       __unwindtable$??__EuserActLog@U2@@YAXXZ 10029a98     SamtoolsPlugin.obj
 0002:00009aa0       __ehfuncinfo$??__EuserActLog@U2@@YAXXZ 10029aa0     SamtoolsPlugin.obj
 0002:00009ac4       __unwindtable$??__EalgoLog@U2@@YAXXZ 10029ac4     moc_AssemblySamtoolsMpileup.obj
 0002:00009acc       __ehfuncinfo$??__EalgoLog@U2@@YAXXZ 10029acc     moc_AssemblySamtoolsMpileup.obj
 0002:00009af0       __unwindtable$??__EcmdLog@U2@@YAXXZ 10029af0     moc_AssemblySamtoolsMpileup.obj
 0002:00009af8       __ehfuncinfo$??__EcmdLog@U2@@YAXXZ 10029af8     moc_AssemblySamtoolsMpileup.obj
 0002:00009b1c       __unwindtable$??__EcoreLog@U2@@YAXXZ 10029b1c     moc_AssemblySamtoolsMpileup.obj
 0002:00009b24       __ehfuncinfo$??__EcoreLog@U2@@YAXXZ 10029b24     moc_AssemblySamtoolsMpileup.obj
 0002:00009b48       __unwindtable$??__EioLog@U2@@YAXXZ 10029b48     moc_AssemblySamtoolsMpileup.obj
 0002:00009b50       __ehfuncinfo$??__EioLog@U2@@YAXXZ 10029b50     moc_AssemblySamtoolsMpileup.obj
 0002:00009b74       __unwindtable$??__EperfLog@U2@@YAXXZ 10029b74     moc_AssemblySamtoolsMpileup.obj
 0002:00009b7c       __ehfuncinfo$??__EperfLog@U2@@YAXXZ 10029b7c     moc_AssemblySamtoolsMpileup.obj
 0002:00009ba0       __unwindtable$??__EscriptLog@U2@@YAXXZ 10029ba0     moc_AssemblySamtoolsMpileup.obj
 0002:00009ba8       __ehfuncinfo$??__EscriptLog@U2@@YAXXZ 10029ba8     moc_AssemblySamtoolsMpileup.obj
 0002:00009bcc       __unwindtable$??__EtaskLog@U2@@YAXXZ 10029bcc     moc_AssemblySamtoolsMpileup.obj
 0002:00009bd4       __ehfuncinfo$??__EtaskLog@U2@@YAXXZ 10029bd4     moc_AssemblySamtoolsMpileup.obj
 0002:00009bf8       __unwindtable$??__EuiLog@U2@@YAXXZ 10029bf8     moc_AssemblySamtoolsMpileup.obj
 0002:00009c00       __ehfuncinfo$??__EuiLog@U2@@YAXXZ 10029c00     moc_AssemblySamtoolsMpileup.obj
 0002:00009c24       __unwindtable$??__EuserActLog@U2@@YAXXZ 10029c24     moc_AssemblySamtoolsMpileup.obj
 0002:00009c2c       __ehfuncinfo$??__EuserActLog@U2@@YAXXZ 10029c2c     moc_AssemblySamtoolsMpileup.obj
 0002:00009c50       __unwindtable$??__EalgoLog@U2@@YAXXZ 10029c50     moc_SamtoolMpileupWorker.obj
 0002:00009c58       __ehfuncinfo$??__EalgoLog@U2@@YAXXZ 10029c58     moc_SamtoolMpileupWorker.obj
 0002:00009c7c       __unwindtable$??__EcmdLog@U2@@YAXXZ 10029c7c     moc_SamtoolMpileupWorker.obj
 0002:00009c84       __ehfuncinfo$??__EcmdLog@U2@@YAXXZ 10029c84     moc_SamtoolMpileupWorker.obj
 0002:00009ca8       __unwindtable$??__EcoreLog@U2@@YAXXZ 10029ca8     moc_SamtoolMpileupWorker.obj
 0002:00009cb0       __ehfuncinfo$??__EcoreLog@U2@@YAXXZ 10029cb0     moc_SamtoolMpileupWorker.obj
 0002:00009cd4       __unwindtable$??__EioLog@U2@@YAXXZ 10029cd4     moc_SamtoolMpileupWorker.obj
 0002:00009cdc       __ehfuncinfo$??__EioLog@U2@@YAXXZ 10029cdc     moc_SamtoolMpileupWorker.obj
 0002:00009d00       __unwindtable$??__EperfLog@U2@@YAXXZ 10029d00     moc_SamtoolMpileupWorker.obj
 0002:00009d08       __ehfuncinfo$??__EperfLog@U2@@YAXXZ 10029d08     moc_SamtoolMpileupWorker.obj
 0002:00009d2c       __unwindtable$??__EscriptLog@U2@@YAXXZ 10029d2c     moc_SamtoolMpileupWorker.obj
 0002:00009d34       __ehfuncinfo$??__EscriptLog@U2@@YAXXZ 10029d34     moc_SamtoolMpileupWorker.obj
 0002:00009d58       __unwindtable$??__EtaskLog@U2@@YAXXZ 10029d58     moc_SamtoolMpileupWorker.obj
 0002:00009d60       __ehfuncinfo$??__EtaskLog@U2@@YAXXZ 10029d60     moc_SamtoolMpileupWorker.obj
 0002:00009d84       __unwindtable$??__EuiLog@U2@@YAXXZ 10029d84     moc_SamtoolMpileupWorker.obj
 0002:00009d8c       __ehfuncinfo$??__EuiLog@U2@@YAXXZ 10029d8c     moc_SamtoolMpileupWorker.obj
 0002:00009db0       __unwindtable$??__EuserActLog@U2@@YAXXZ 10029db0     moc_SamtoolMpileupWorker.obj
 0002:00009db8       __ehfuncinfo$??__EuserActLog@U2@@YAXXZ 10029db8     moc_SamtoolMpileupWorker.obj
 0002:00009de0       __sehtable$__onexit        10029de0     MSVCRT:atonexit.obj
 0002:00009e00       __sehtable$___DllMainCRTStartup 10029e00     MSVCRT:crtdll.obj
 0002:00009e28       __sehtable$??_M@YGXPAXIHP6EX0@Z@Z 10029e28     MSVCRT:ehvecdtr.obj
 0002:00009e48       __sehtable$?__ArrayUnwind@@YGXPAXIHP6EX0@Z@Z 10029e48     MSVCRT:ehvecdtr.obj
 0002:00009e68       __sehtable$__IsNonwritableInCurrentImage 10029e68     MSVCRT:pesect.obj
 0002:00009e90       .edata                     10029e90     variants.exp
 0002:00009eb8       rgpv                       10029eb8     variants.exp
 0002:00009ebc       rgszName                   10029ebc     variants.exp
 0002:00009ec0       rgwOrd                     10029ec0     variants.exp
 0002:00009ec2       szName                     10029ec2     variants.exp
 0002:00009ecf       $N00001                    10029ecf     variants.exp
 0002:0000bc68       .idata$6                   1002bc68     U2Core:U2Core.dll
 0002:0000e4e4       .idata$6                   1002e4e4     U2Lang:U2Lang.dll
 0002:0000f4da       .idata$6                   1002f4da     U2Designer:U2Designer.dll
 0002:000105fc       .idata$6                   100305fc     Qt5Widgets:Qt5Widgets.dll
 0002:0001086c       .idata$6                   1003086c     Qt5Gui:Qt5Gui.dll
 0002:000109de       .idata$6                   100309de     Qt5Script:Qt5Script.dll
 0002:000117fa       .idata$6                   100317fa     Qt5Core:Qt5Core.dll
 0002:000118a0       .idata$6                   100318a0     msvcprt:MSVCP120.dll
 0002:00011936       .idata$6                   10031936     MSVCRT:MSVCR120.dll
 0002:00011b4a       .idata$6                   10031b4a     kernel32:KERNEL32.dll
 0003:00000a08       __Tuple_alloc              10032a08     AssemblySamtoolsMpileup.obj
 0003:00000a09       _ignore                    10032a09     AssemblySamtoolsMpileup.obj
 0003:00000a0a       _allocator_arg             10032a0a     AssemblySamtoolsMpileup.obj
 0003:00000a0b       _piecewise_construct       10032a0b     AssemblySamtoolsMpileup.obj
 0003:00000a10       _taskLog                   10032a10     AssemblySamtoolsMpileup.obj
 0003:00000a18       _algoLog                   10032a18     AssemblySamtoolsMpileup.obj
 0003:00000a20       _userActLog                10032a20     AssemblySamtoolsMpileup.obj
 0003:00000a28       _ioLog                     10032a28     AssemblySamtoolsMpileup.obj
 0003:00000a30       _coreLog                   10032a30     AssemblySamtoolsMpileup.obj
 0003:00000a3c       _uiLog                     10032a3c     AssemblySamtoolsMpileup.obj
 0003:00000a44       _scriptLog                 10032a44     AssemblySamtoolsMpileup.obj
 0003:00000a4c       _perfLog                   10032a4c     AssemblySamtoolsMpileup.obj
 0003:00000a54       _cmdLog                    10032a54     AssemblySamtoolsMpileup.obj
 0003:00000a70       ?cvar@?1???0CallVariantsTask@LocalWorkflow@U2@@QAE@ABVCallVariantsTaskSettings@23@PAVDbiDataStorage@Workflow@3@@Z@4VGReportableCounter@3@A 10032a70     AssemblySamtoolsMpileup.obj
 0003:00000a98       ?$S1@?1???0CallVariantsTask@LocalWorkflow@U2@@QAE@ABVCallVariantsTaskSettings@23@PAVDbiDataStorage@Workflow@3@@Z@4IA 10032a98     AssemblySamtoolsMpileup.obj
 0003:00000a9c       __Tuple_alloc              10032a9c     SamtoolMpileupWorker.obj
 0003:00000a9d       _ignore                    10032a9d     SamtoolMpileupWorker.obj
 0003:00000a9e       _allocator_arg             10032a9e     SamtoolMpileupWorker.obj
 0003:00000a9f       _piecewise_construct       10032a9f     SamtoolMpileupWorker.obj
 0003:00000aa0       _TANDEMQ                   10032aa0     SamtoolMpileupWorker.obj
 0003:00000aa4       _MAX_INDEL_DEPTH           10032aa4     SamtoolMpileupWorker.obj
 0003:00000aa8       _NO_INDEL                  10032aa8     SamtoolMpileupWorker.obj
 0003:00000aac       _MAX_DEPTH                 10032aac     SamtoolMpileupWorker.obj
 0003:00000ab0       _MIN_ALT                   10032ab0     SamtoolMpileupWorker.obj
 0003:00000ab4       _INDEL_FRAC                10032ab4     SamtoolMpileupWorker.obj
 0003:00000ab8       _FIX_PL                    10032ab8     SamtoolMpileupWorker.obj
 0003:00000abc       _MIN_PERM_P                10032abc     SamtoolMpileupWorker.obj
 0003:00000ac0       _N1                        10032ac0     SamtoolMpileupWorker.obj
 0003:00000ac4       _MIN_MQ                    10032ac4     SamtoolMpileupWorker.obj
 0003:00000ac8       _ACGT_ONLY                 10032ac8     SamtoolMpileupWorker.obj
 0003:00000ad0       _PVALUE4                   10032ad0     SamtoolMpileupWorker.obj
 0003:00000ad4       _taskLog                   10032ad4     SamtoolMpileupWorker.obj
 0003:00000adc       _algoLog                   10032adc     SamtoolMpileupWorker.obj
 0003:00000ae4       _userActLog                10032ae4     SamtoolMpileupWorker.obj
 0003:00000aec       _ioLog                     10032aec     SamtoolMpileupWorker.obj
 0003:00000af4       _coreLog                   10032af4     SamtoolMpileupWorker.obj
 0003:00000afc       _REF_SEQ_PORT_ID           10032afc     SamtoolMpileupWorker.obj
 0003:00000b00       _CALL_GT                   10032b00     SamtoolMpileupWorker.obj
 0003:00000b04       _PVALUE_HWE                10032b04     SamtoolMpileupWorker.obj
 0003:00000b08       _PRINT                     10032b08     SamtoolMpileupWorker.obj
 0003:00000b0c       _N_PERM                    10032b0c     SamtoolMpileupWorker.obj
 0003:00000b10       _REG                       10032b10     SamtoolMpileupWorker.obj
 0003:00000b14       _KEEPALT                   10032b14     SamtoolMpileupWorker.obj
 0003:00000b18       _REF_URL                   10032b18     SamtoolMpileupWorker.obj
 0003:00000b1c       _MIN_BASEQ                 10032b1c     SamtoolMpileupWorker.obj
 0003:00000b20       _uiLog                     10032b20     SamtoolMpileupWorker.obj
 0003:00000b28       _scriptLog                 10032b28     SamtoolMpileupWorker.obj
 0003:00000b30       _QCALL                     10032b30     SamtoolMpileupWorker.obj
 0003:00000b34       _WINDOW                    10032b34     SamtoolMpileupWorker.obj
 0003:00000b38       _MIN_DEP                   10032b38     SamtoolMpileupWorker.obj
 0003:00000b3c       _REF_SOURCE_PORT           10032b3c     SamtoolMpileupWorker.obj
 0003:00000b40       _MIN_SMPL_FRAC             10032b40     SamtoolMpileupWorker.obj
 0003:00000b44       _perfLog                   10032b44     SamtoolMpileupWorker.obj
 0003:00000b4c       _REF_SOURCE                10032b4c     SamtoolMpileupWorker.obj
 0003:00000b50       _BED                       10032b50     SamtoolMpileupWorker.obj
 0003:00000b54       _PVALUE2                   10032b54     SamtoolMpileupWorker.obj
 0003:00000b58       _PTYPE                     10032b58     SamtoolMpileupWorker.obj
 0003:00000b5c       _SAMPLES                   10032b5c     SamtoolMpileupWorker.obj
 0003:00000b60       _NO_GENO                   10032b60     SamtoolMpileupWorker.obj
 0003:00000b64       _PREF                      10032b64     SamtoolMpileupWorker.obj
 0003:00000b68       _cmdLog                    10032b68     SamtoolMpileupWorker.obj
 0003:00000b70       _ASSEMBLY_PORT_ID          10032b70     SamtoolMpileupWorker.obj
 0003:00000b74       _USE_ORPHAN                10032b74     SamtoolMpileupWorker.obj
 0003:00000b78       _CCALL                     10032b78     SamtoolMpileupWorker.obj
 0003:00000b7c       _REF_SOURCE_FILE           10032b7c     SamtoolMpileupWorker.obj
 0003:00000b80       _PVALUE1                   10032b80     SamtoolMpileupWorker.obj
 0003:00000b84       _CAPQ_THRES                10032b84     SamtoolMpileupWorker.obj
 0003:00000b88       _MIN_QUAL                  10032b88     SamtoolMpileupWorker.obj
 0003:00000b8c       _EXT_BAQ                   10032b8c     SamtoolMpileupWorker.obj
 0003:00000b90       _MAX_DEP                   10032b90     SamtoolMpileupWorker.obj
 0003:00000b94       _ILLUMINA13                10032b94     SamtoolMpileupWorker.obj
 0003:00000b98       _PVALUE3                   10032b98     SamtoolMpileupWorker.obj
 0003:00000b9c       _PL_LIST                   10032b9c     SamtoolMpileupWorker.obj
 0003:00000ba0       _THETA                     10032ba0     SamtoolMpileupWorker.obj
 0003:00000ba4       _EXTQ                      10032ba4     SamtoolMpileupWorker.obj
 0003:00000ba8       _BCF_BED                   10032ba8     SamtoolMpileupWorker.obj
 0003:00000bac       _OPENQ                     10032bac     SamtoolMpileupWorker.obj
 0003:00000bb0       _DISABLE_BAQ               10032bb0     SamtoolMpileupWorker.obj
 0003:00000bb4       _GAP_SIZE                  10032bb4     SamtoolMpileupWorker.obj
 0003:00000bb8       _OUT_URL                   10032bb8     SamtoolMpileupWorker.obj
 0003:00000bbc       __Tuple_alloc              10032bbc     SamtoolsPlugin.obj
 0003:00000bbd       _ignore                    10032bbd     SamtoolsPlugin.obj
 0003:00000bbe       _allocator_arg             10032bbe     SamtoolsPlugin.obj
 0003:00000bbf       _piecewise_construct       10032bbf     SamtoolsPlugin.obj
 0003:00000bc0       _taskLog                   10032bc0     SamtoolsPlugin.obj
 0003:00000bc8       _algoLog                   10032bc8     SamtoolsPlugin.obj
 0003:00000bd0       _userActLog                10032bd0     SamtoolsPlugin.obj
 0003:00000bd8       _ioLog                     10032bd8     SamtoolsPlugin.obj
 0003:00000be0       _coreLog                   10032be0     SamtoolsPlugin.obj
 0003:00000be8       _uiLog                     10032be8     SamtoolsPlugin.obj
 0003:00000bf0       _scriptLog                 10032bf0     SamtoolsPlugin.obj
 0003:00000bf8       _perfLog                   10032bf8     SamtoolsPlugin.obj
 0003:00000c00       _cmdLog                    10032c00     SamtoolsPlugin.obj
 0003:00000c08       __Tuple_alloc              10032c08     moc_AssemblySamtoolsMpileup.obj
 0003:00000c09       _ignore                    10032c09     moc_AssemblySamtoolsMpileup.obj
 0003:00000c0a       _allocator_arg             10032c0a     moc_AssemblySamtoolsMpileup.obj
 0003:00000c0b       _piecewise_construct       10032c0b     moc_AssemblySamtoolsMpileup.obj
 0003:00000c0c       _taskLog                   10032c0c     moc_AssemblySamtoolsMpileup.obj
 0003:00000c14       _algoLog                   10032c14     moc_AssemblySamtoolsMpileup.obj
 0003:00000c1c       _userActLog                10032c1c     moc_AssemblySamtoolsMpileup.obj
 0003:00000c24       _ioLog                     10032c24     moc_AssemblySamtoolsMpileup.obj
 0003:00000c2c       _coreLog                   10032c2c     moc_AssemblySamtoolsMpileup.obj
 0003:00000c34       _uiLog                     10032c34     moc_AssemblySamtoolsMpileup.obj
 0003:00000c3c       _scriptLog                 10032c3c     moc_AssemblySamtoolsMpileup.obj
 0003:00000c44       _perfLog                   10032c44     moc_AssemblySamtoolsMpileup.obj
 0003:00000c4c       _cmdLog                    10032c4c     moc_AssemblySamtoolsMpileup.obj
 0003:00000c54       __Tuple_alloc              10032c54     moc_SamtoolMpileupWorker.obj
 0003:00000c55       _ignore                    10032c55     moc_SamtoolMpileupWorker.obj
 0003:00000c56       _allocator_arg             10032c56     moc_SamtoolMpileupWorker.obj
 0003:00000c57       _piecewise_construct       10032c57     moc_SamtoolMpileupWorker.obj
 0003:00000c58       _taskLog                   10032c58     moc_SamtoolMpileupWorker.obj
 0003:00000c60       _algoLog                   10032c60     moc_SamtoolMpileupWorker.obj
 0003:00000c68       _userActLog                10032c68     moc_SamtoolMpileupWorker.obj
 0003:00000c70       _ioLog                     10032c70     moc_SamtoolMpileupWorker.obj
 0003:00000c78       _coreLog                   10032c78     moc_SamtoolMpileupWorker.obj
 0003:00000c80       _uiLog                     10032c80     moc_SamtoolMpileupWorker.obj
 0003:00000c88       _scriptLog                 10032c88     moc_SamtoolMpileupWorker.obj
 0003:00000c90       _perfLog                   10032c90     moc_SamtoolMpileupWorker.obj
 0003:00000c98       _cmdLog                    10032c98     moc_SamtoolMpileupWorker.obj
 0003:00000ca0       __Tuple_alloc              10032ca0     moc_SamtoolsPlugin.obj
 0003:00000ca1       _ignore                    10032ca1     moc_SamtoolsPlugin.obj
 0003:00000ca2       _allocator_arg             10032ca2     moc_SamtoolsPlugin.obj
 0003:00000ca3       _piecewise_construct       10032ca3     moc_SamtoolsPlugin.obj
 0003:00000ca4       ___proc_attached           10032ca4     MSVCRT:crtdll.obj
 0003:00000ca8       _GS_ExceptionRecord        10032ca8     MSVCRT:gs_report.obj
 0003:00000cf8       _GS_ContextRecord          10032cf8     MSVCRT:gs_report.obj
 0003:00000fc4       _DebuggerWasPresent        10032fc4     MSVCRT:gs_report.obj
 0004:00000060       $R000000                   10033060     * linker generated manifest res *

 Exports

  ordinal    name

        1    _ugene_plugin_init
               exported name: ugene_plugin_init
